 CryEntitySystem

 Timestamp is 5036d2a0 (Fri Aug 24 03:02:24 2012)

 Preferred load address is 32000000

 Start         Length     Name                   Class
 0001:00000000 000b20baH .text                   CODE
 0001:000b20c0 0000032cH .text$yc                CODE
 0001:000b23f0 000005bdH .text$yd                CODE
 0002:00000000 00000168H .idata$5                DATA
 0002:00000168 00000004H .CRT$XCA                DATA
 0002:0000016c 00000054H .CRT$XCU                DATA
 0002:000001c0 00000004H .CRT$XCZ                DATA
 0002:000001c4 00000004H .CRT$XIA                DATA
 0002:000001c8 00000004H .CRT$XIAA               DATA
 0002:000001cc 00000004H .CRT$XIC                DATA
 0002:000001d0 00000004H .CRT$XIZ                DATA
 0002:000001e0 0000b678H .rdata                  DATA
 0002:0000b858 0000005aH .rdata$debug            DATA
 0002:0000b8c0 00000004H .rdata$sxdata           DATA
 0002:0000b8c4 00000004H .rtc$IAA                DATA
 0002:0000b8c8 00000004H .rtc$IZZ                DATA
 0002:0000b8cc 00000004H .rtc$TAA                DATA
 0002:0000b8d0 00000004H .rtc$TZZ                DATA
 0002:0000b8d8 00000064H .xdata$x                DATA
 0002:0000b93c 0000003cH .idata$2                DATA
 0002:0000b978 00000014H .idata$3                DATA
 0002:0000b98c 00000168H .idata$4                DATA
 0002:0000baf4 000005a2H .idata$6                DATA
 0002:0000c0a0 00000079H .edata                  DATA
 0003:00000000 00000430H .data                   DATA
 0003:00000430 00012f84H .bss                    DATA
 0004:00000000 00000004H .tls$                   DATA
 0005:00000000 00000058H .rsrc$01                DATA
 0005:00000060 00000248H .rsrc$02                DATA

  Address         Publics by Value              Rva+Base       Lib:Object

 0000:00000000       __except_list              00000000     <absolute>
 0000:00000001       ___safe_se_handler_count   00000001     <absolute>
 0000:00009876       __ldused                   00009876     <absolute>
 0000:00009876       __fltused                  00009876     <absolute>
 0000:00000000       ___ImageBase               32000000     <linker-defined>
 0001:000000f0       ??0?$Vec3_tpl@M@@QAE@XZ    320010f0 f i AffineParts.obj
 0001:00002070       ?SpectralDecompose@AffineParts@@QAEXABU?$Matrix34_tpl@M@@@Z 32003070 f   AffineParts.obj
 0001:000021f0       ??_EIMemReplay@@UAEPAXI@Z  320031f0 f i AreaSolid.obj
 0001:000021f0       ??_ECDummyMemReplay@@UAEPAXI@Z 320031f0 f i AreaSolid.obj
 0001:000021f0       ??_GCDummyMemReplay@@UAEPAXI@Z 320031f0 f i AreaSolid.obj
 0001:000021f0       ??_GIMemReplay@@UAEPAXI@Z  320031f0 f i AreaSolid.obj
 0001:00002220       ?__stl_throw_length_error@stlpmtx_std@@YAXPBD@Z 32003220 f i AreaSolid.obj
 0001:00002240       ??_H@YGXPAXIHP6EPAX0@Z@Z   32003240 f i AreaSolid.obj
 0001:00002270       ?ComputeBasisTM@CPlane@AreaUtil@@AAEXXZ 32003270 f i AreaSolid.obj
 0001:00002380       ?ExitScope_Realloc@CDummyMemReplay@@UAEXIIII@Z 32003380 f i AreaSolid.obj
 0001:00002380       ?AddContextV@CDummyMemReplay@@UAEXHIPBDPAD@Z 32003380 f i AreaSolid.obj
 0001:00002380       ?MarkBucket@CDummyMemReplay@@UAEXHIPAXI@Z 32003380 f i AreaSolid.obj
 0001:00002390       ?AddTexturePoolContext@CDummyMemReplay@@UAEXPAXHHHPBDI@Z 32003390 f i AreaSolid.obj
 0001:00002390       ?SetLightmap@IRenderNode@@UAEXPAURenderLMData@@PAMIECH@Z 32003390 f i RenderProxy.obj
 0001:000023a0       ?Draw@CSegment@CAreaSolid@@QBEXABU?$Matrix34_tpl@M@@ABU?$Color_tpl@E@@1@Z 320033a0 f   AreaSolid.obj
 0001:00002780       ?IsInside@CAreaSolid@@QBE_NABU?$Vec3_tpl@M@@@Z 32003780 f   AreaSolid.obj
 0001:000027f0       ??0CPlane@AreaUtil@@QAE@ABU?$Vec3_tpl@M@@00@Z 320037f0 f i AreaSolid.obj
 0001:00002a20       ??0CSegment@CAreaSolid@@QAE@PBU?$Vec3_tpl@M@@HW4ESegmentType@1@@Z 32003a20 f   AreaSolid.obj
 0001:00002c20       ?CryGetIMemReplay@@YAPAUIMemReplay@@XZ 32003c20 f i AreaSolid.obj
 0001:00002c80       ?allocate@?$_STLP_alloc_proxy@PAHHV?$allocator@H@stlpmtx_std@@@priv@stlpmtx_std@@QAEPAHIAAI@Z 32003c80 f i AreaManager.obj
 0001:00002c80       ?allocate@?$_STLP_alloc_proxy@PAMMV?$allocator@M@stlpmtx_std@@@priv@stlpmtx_std@@QAEPAMIAAI@Z 32003c80 f i ScriptBind_Entity.obj
 0001:00002c80       ?allocate@?$_STLP_alloc_proxy@PAPAXPAXV?$allocator@PAX@stlpmtx_std@@@priv@stlpmtx_std@@QAEPAPAXIAAI@Z 32003c80 f i AreaSolid.obj
 0001:00002cd0       ??0?$_Vector_base@U?$Vec3_tpl@M@@V?$allocator@U?$Vec3_tpl@M@@@stlpmtx_std@@@priv@stlpmtx_std@@QAE@V?$__move_source@V?$_Vector_base@U?$Vec3_tpl@M@@V?$allocator@U?$Vec3_tpl@M@@@stlpmtx_std@@@priv@stlpmtx_std@@@2@@Z 32003cd0 f i AreaSolid.obj
 0001:00002d50       ?QueryNearest@CSegment@CAreaSolid@@QBE_NABU?$Vec2_tpl@M@@_NAAU3@@Z 32003d50 f   AreaSolid.obj
 0001:00003030       ?QueryNearest@CAreaSolid@@QBE_NABU?$Vec3_tpl@M@@HAAU2@AAMAAVCPlane@AreaUtil@@AAW4ESegmentType@1@@Z 32004030 f   AreaSolid.obj
 0001:00003330       ?Draw@CAreaSolid@@QBEXABU?$Matrix34_tpl@M@@ABU?$Color_tpl@E@@1@Z 32004330 f   AreaSolid.obj
 0001:000033a0       ?allocate@?$_STLP_alloc_proxy@PAUSEntityTimerEvent@@U1@V?$allocator@USEntityTimerEvent@@@stlpmtx_std@@@priv@stlpmtx_std@@QAEPAUSEntityTimerEvent@@IAAI@Z 320043a0 f i EntitySystem.obj
 0001:000033a0       ?allocate@?$_STLP_alloc_proxy@PAU?$Vec3_tpl@M@@U1@V?$allocator@U?$Vec3_tpl@M@@@stlpmtx_std@@@priv@stlpmtx_std@@QAEPAU?$Vec3_tpl@M@@IAAI@Z 320043a0 f i AreaSolid.obj
 0001:000033a0       ?allocate@?$_STLP_alloc_proxy@PAUSScriptState@@U1@V?$allocator@USScriptState@@@stlpmtx_std@@@priv@stlpmtx_std@@QAEPAUSScriptState@@IAAI@Z 320043a0 f i EntityScript.obj
 0001:00003400       ?_M_insert_overflow@?$_Impl_vector@HV?$allocator@H@stlpmtx_std@@@priv@stlpmtx_std@@AAEXPAHABHABU__true_type@3@I_N@Z 32004400 f i AreaManager.obj
 0001:00003400       ?_M_insert_overflow@?$_Impl_vector@PAXV?$allocator@PAX@stlpmtx_std@@@priv@stlpmtx_std@@AAEXPAPAXABQAXABU__true_type@3@I_N@Z 32004400 f i AreaSolid.obj
 0001:00003400       ?_M_insert_overflow@?$_Impl_vector@IV?$allocator@I@stlpmtx_std@@@priv@stlpmtx_std@@AAEXPAIABIABU__true_type@3@I_N@Z 32004400 f i EntitySystem.obj
 0001:00003550       ?_M_insert_overflow@?$_Impl_vector@USEntityTimerEvent@@V?$allocator@USEntityTimerEvent@@@stlpmtx_std@@@priv@stlpmtx_std@@AAEXPAUSEntityTimerEvent@@ABU4@ABU__true_type@3@I_N@Z 32004550 f i EntitySystem.obj
 0001:00003550       ?_M_insert_overflow@?$_Impl_vector@U?$Vec3_tpl@M@@V?$allocator@U?$Vec3_tpl@M@@@stlpmtx_std@@@priv@stlpmtx_std@@AAEXPAU?$Vec3_tpl@M@@ABU4@ABU__true_type@3@I_N@Z 32004550 f i AreaSolid.obj
 0001:00003550       ?_M_insert_overflow@?$_Impl_vector@USProximityEvent@@V?$allocator@USProximityEvent@@@stlpmtx_std@@@priv@stlpmtx_std@@AAEXPAUSProximityEvent@@ABU4@ABU__true_type@3@I_N@Z 32004550 f i ProximityTriggerSystem.obj
 0001:000036d0       ?QueryNearest@CAreaSolid@@QBE_NABU?$Vec3_tpl@M@@HAAU2@AAM@Z 320046d0 f   AreaSolid.obj
 0001:00003700       ?erase@?$_Impl_vector@PAXV?$allocator@PAX@stlpmtx_std@@@priv@stlpmtx_std@@QAEPAPAXPAPAX0@Z 32004700 f i AreaSolid.obj
 0001:00003750       ??0?$_Vector_base@USProximityEvent@@V?$allocator@USProximityEvent@@@stlpmtx_std@@@priv@stlpmtx_std@@QAE@IABV?$allocator@USProximityEvent@@@2@@Z 32004750 f i ProximityTriggerSystem.obj
 0001:00003750       ??0?$_Vector_base@U?$Vec3_tpl@M@@V?$allocator@U?$Vec3_tpl@M@@@stlpmtx_std@@@priv@stlpmtx_std@@QAE@IABV?$allocator@U?$Vec3_tpl@M@@@2@@Z 32004750 f i AreaSolid.obj
 0001:00003810       ?reserve@?$_Impl_vector@USEntityTimerEvent@@V?$allocator@USEntityTimerEvent@@@stlpmtx_std@@@priv@stlpmtx_std@@QAEXI@Z 32004810 f i EntitySystem.obj
 0001:00003810       ?reserve@?$_Impl_vector@U?$Vec3_tpl@M@@V?$allocator@U?$Vec3_tpl@M@@@stlpmtx_std@@@priv@stlpmtx_std@@QAEXI@Z 32004810 f i AreaSolid.obj
 0001:000038c0       ??0?$_Impl_vector@U?$Vec3_tpl@M@@V?$allocator@U?$Vec3_tpl@M@@@stlpmtx_std@@@priv@stlpmtx_std@@QAE@ABV012@@Z 320048c0 f i AreaSolid.obj
 0001:00003930       ??0CSegmentSet@CAreaSolid@@QAE@ABVCPlane@AreaUtil@@@Z 32004930 f i AreaSolid.obj
 0001:000039c0       ??0CAreaSolid@@QAE@XZ      320049c0 f   AreaSolid.obj
 0001:00003a60       ?AddSegment@CAreaSolid@@QAEXPBU?$Vec3_tpl@M@@_NH@Z 32004a60 f   AreaSolid.obj
 0001:00003d00       ??$__destroy_range_aux@V?$reverse_iterator@PAV?$vector@U?$Vec3_tpl@M@@V?$allocator@U?$Vec3_tpl@M@@@stlpmtx_std@@@stlpmtx_std@@@stlpmtx_std@@V?$vector@U?$Vec3_tpl@M@@V?$allocator@U?$Vec3_tpl@M@@@stlpmtx_std@@@2@@stlpmtx_std@@YAXV?$reverse_iterator@PAV?$vector@U?$Vec3_tpl@M@@V?$allocator@U?$Vec3_tpl@M@@@stlpmtx_std@@@stlpmtx_std@@@0@0PAV?$vector@U?$Vec3_tpl@M@@V?$allocator@U?$Vec3_tpl@M@@@stlpmtx_std@@@0@ABU__false_type@0@@Z 32004d00 f i AreaSolid.obj
 0001:00003da0       ??1CSegmentSet@CAreaSolid@@QAE@XZ 32004da0 f i AreaSolid.obj
 0001:00003f00       ?Clear@CAreaSolid@@AAEXXZ  32004f00 f   AreaSolid.obj
 0001:00004050       ??$__ufill@PAV?$vector@U?$Vec3_tpl@M@@V?$allocator@U?$Vec3_tpl@M@@@stlpmtx_std@@@stlpmtx_std@@V12@H@priv@stlpmtx_std@@YAXPAV?$vector@U?$Vec3_tpl@M@@V?$allocator@U?$Vec3_tpl@M@@@stlpmtx_std@@@1@0ABV21@ABUrandom_access_iterator_tag@1@PAH@Z 32005050 f i AreaSolid.obj
 0001:00004150       ?_M_insert_overflow_aux@?$_Impl_vector@V?$vector@U?$Vec3_tpl@M@@V?$allocator@U?$Vec3_tpl@M@@@stlpmtx_std@@@stlpmtx_std@@V?$allocator@V?$vector@U?$Vec3_tpl@M@@V?$allocator@U?$Vec3_tpl@M@@@stlpmtx_std@@@stlpmtx_std@@@2@@priv@stlpmtx_std@@AAEXPAV?$vector@U?$Vec3_tpl@M@@V?$allocator@U?$Vec3_tpl@M@@@stlpmtx_std@@@3@ABV43@ABU__false_type@3@I_N@Z 32005150 f i AreaSolid.obj
 0001:00004320       ?_M_insert_overflow_aux@?$_Impl_vector@V?$vector@U?$Vec3_tpl@M@@V?$allocator@U?$Vec3_tpl@M@@@stlpmtx_std@@@stlpmtx_std@@V?$allocator@V?$vector@U?$Vec3_tpl@M@@V?$allocator@U?$Vec3_tpl@M@@@stlpmtx_std@@@stlpmtx_std@@@2@@priv@stlpmtx_std@@AAEXPAV?$vector@U?$Vec3_tpl@M@@V?$allocator@U?$Vec3_tpl@M@@@stlpmtx_std@@@3@ABV43@ABU__true_type@3@I_N@Z 32005320 f i AreaSolid.obj
 0001:000043b0       ?BuildBSP@CAreaSolid@@QAEXXZ 320053b0 f   AreaSolid.obj
 0001:00004a50       ??_GISplineInterpolator@@UAEPAXI@Z 32005a50 f i BreakablePlane.obj
 0001:00004a50       ??_EISplineInterpolator@@UAEPAXI@Z 32005a50 f i BreakablePlane.obj
 0001:00004a80       ?UpdateBrokenMat@@YAHPAUIMaterial@@HPBD@Z 32005a80 f   BreakablePlane.obj
 0001:00004c60       ?CryLog@@YAXPBDZZ          32005c60 f i BreakablePlane.obj
 0001:00004c90       ?CryLogAlways@@YAXPBDZZ    32005c90 f i BreakablePlane.obj
 0001:00004cc0       ??_EIOwnedObject@@UAEPAXI@Z 32005cc0 f i BreakablePlane.obj
 0001:00004cc0       ??_GIOwnedObject@@UAEPAXI@Z 32005cc0 f i BreakablePlane.obj
 0001:00004cc0       ??_GISoundEventListener@@UAEPAXI@Z 32005cc0 f i SoundProxy.obj
 0001:00004cc0       ??_EISystemEventListener@@UAEPAXI@Z 32005cc0 f i CryEntityDLL.obj
 0001:00004cc0       ??_EISoundEventListener@@UAEPAXI@Z 32005cc0 f i SoundProxy.obj
 0001:00004cc0       ??_GISystemEventListener@@UAEPAXI@Z 32005cc0 f i CryEntityDLL.obj
 0001:00004cf0       ??0SEntityPhysicalizeParams@@QAE@XZ 32005cf0 f i BreakablePlane.obj
 0001:00004d40       ?alloc@StandardAlloc@NAlloc@@SAPAXAAI_NH@Z 32005d40 f i BreakablePlane.obj
 0001:00004dc0       ??1?$TVarEParam@U?$TRangedType@M$0A@$0HPPPPPPP@$0A@@@@@QAE@XZ 32005dc0 f i BreakablePlane.obj
 0001:00004dd0       ??1?$TVarEPParam@U?$TRangedType@M$0A@$0HPPPPPPP@$0A@@@@@QAE@XZ 32005dd0 f i BreakablePlane.obj
 0001:00004e00       ?Break@CBreakablePlane@@QAEPAHABU?$Vec3_tpl@M@@MAAPAU?$Vec2_tpl@M@@HMM@Z 32005e00 f   BreakablePlane.obj
 0001:00004ec0       ?circ_segment_area@@YAMMM@Z 32005ec0 f   BreakablePlane.obj
 0001:00004fa0       ??0?$Matrix34_tpl@M@@QAE@ABU?$Vec3_tpl@M@@ABU?$Quat_tpl@M@@0@Z 32005fa0 f i BreakablePlane.obj
 0001:00005110       ??0CFrameProfiler@@QAE@PAUISystem@@PBDW4EProfiledSubsystem@@@Z 32006110 f i BreakablePlane.obj
 0001:000051b0       ??$move_init@U?$SplineKey@M@spline@@@NArray@@YAXPAU?$SplineKey@M@spline@@0I@Z 320061b0 f i BreakablePlane.obj
 0001:00005200       ??$__unguarded_linear_insert@PAU?$SplineKey@M@spline@@U12@U?$less@U?$SplineKey@M@spline@@@stlpmtx_std@@@priv@stlpmtx_std@@YAXPAU?$SplineKey@M@spline@@U23@U?$less@U?$SplineKey@M@spline@@@1@@Z 32006200 f i BreakablePlane.obj
 0001:00005260       ??0pe_params_pos@@QAE@XZ   32006260 f i BreakablePlane.obj
 0001:000052c0       ??$__push_heap@PAU?$SplineKey@M@spline@@HU12@U?$less@U?$SplineKey@M@spline@@@stlpmtx_std@@@stlpmtx_std@@YAXPAU?$SplineKey@M@spline@@HHU12@U?$less@U?$SplineKey@M@spline@@@0@@Z 320062c0 f i BreakablePlane.obj
 0001:00005350       ??$__copy_backward_ptrs@PAU?$SplineKey@M@spline@@PAU12@@priv@stlpmtx_std@@YAPAU?$SplineKey@M@spline@@PAU23@00ABU__false_type@1@@Z 32006350 f i BreakablePlane.obj
 0001:000053b0       ??0pe_params_particle@@QAE@XZ 320063b0 f i BreakablePlane.obj
 0001:000054d0       ??0pe_action_impulse@@QAE@XZ 320064d0 f i BreakablePlane.obj
 0001:00005530       ?ToVec2@Vec2f16@@QBE?AU?$Vec2_tpl@M@@XZ 32006530 f i BreakablePlane.obj
 0001:00005610       ??0SEntitySpawnParams@@QAE@XZ 32006610 f i BreakablePlane.obj
 0001:000056a0       ?CryModuleCRTMalloc@@YAPAXI@Z 320066a0 f i BreakablePlane.obj
 0001:000056f0       ??0CBreakablePlane@@QAE@XZ 320066f0 f i BreakablePlane.obj
 0001:00005750       ?Release@CBreakablePlane@@UAEHXZ 32006750 f i BreakablePlane.obj
 0001:00005760       ??_ECBreakablePlane@@UAEPAXI@Z 32006760 f i BreakablePlane.obj
 0001:00005760       ??_GCBreakablePlane@@UAEPAXI@Z 32006760 f i BreakablePlane.obj
 0001:000057c0       ??1SLightSource@ParticleParams@@QAE@XZ 320067c0 f i BreakablePlane.obj
 0001:00005820       ?Spawn@IParticleEffect@@QAEPAUIParticleEmitter@@_NABU?$Matrix34_tpl@M@@@Z 32006820 f i BreakablePlane.obj
 0001:00005c40       ?_boxCircleIntersArea@@YAMABU?$Vec2_tpl@M@@0M@Z 32006c40 f   BreakablePlane.obj
 0001:00005f20       ?ExtractMeshIsland@CBreakablePlane@@SAXABUSExtractMeshIslandIn@@AAUSExtractMeshIslandOut@@@Z 32006f20 f   BreakablePlane.obj
 0001:00006d00       ??1ParticleParams@@QAE@XZ  32007d00 f i BreakablePlane.obj
 0001:00006fa0       ?init@?$DynArray@U?$SplineKey@M@spline@@HU?$SmallDynStorage@U?$SplineKey@M@spline@@HUStandardAlloc@NAlloc@@@NArray@@@@KAPAU?$SplineKey@M@spline@@U?$Array@U?$SplineKey@M@spline@@HU?$ArrayStorage@U?$SplineKey@M@spline@@H@NArray@@@@PBU23@@Z 32007fa0 f i BreakablePlane.obj
 0001:00006ff0       ?resize_raw@?$SmallDynStorage@U?$SplineKey@M@spline@@HUStandardAlloc@NAlloc@@@NArray@@QAEXHH_N@Z 32007ff0 f i BreakablePlane.obj
 0001:00007150       ??$__unguarded_insertion_sort_aux@PAU?$SplineKey@M@spline@@U12@U?$less@U?$SplineKey@M@spline@@@stlpmtx_std@@@priv@stlpmtx_std@@YAXPAU?$SplineKey@M@spline@@00U?$less@U?$SplineKey@M@spline@@@1@@Z 32008150 f i BreakablePlane.obj
 0001:000071e0       ??$__adjust_heap@PAU?$SplineKey@M@spline@@HU12@U?$less@U?$SplineKey@M@spline@@@stlpmtx_std@@@stlpmtx_std@@YAXPAU?$SplineKey@M@spline@@HHU12@U?$less@U?$SplineKey@M@spline@@@0@@Z 320081e0 f i BreakablePlane.obj
 0001:000072c0       ??0?$TVarParam@U?$Color3@U?$TFixed@E$00$0PP@@@@@@@QAE@XZ 320082c0 f i BreakablePlane.obj
 0001:00007330       ?set_size@?$SmallDynStorage@U?$SplineKey@M@spline@@HUStandardAlloc@NAlloc@@@NArray@@QAEXH@Z 32008330 f i BreakablePlane.obj
 0001:000073c0       ??$?0M@?$Color3@U?$TFixed@E$00$0PP@@@@@QAE@ABU?$Vec3_tpl@M@@@Z 320083c0 f i BreakablePlane.obj
 0001:00007480       ??$__unguarded_partition@PAU?$SplineKey@M@spline@@U12@U?$less@U?$SplineKey@M@spline@@@stlpmtx_std@@@priv@stlpmtx_std@@YAPAU?$SplineKey@M@spline@@PAU23@0U23@U?$less@U?$SplineKey@M@spline@@@1@@Z 32008480 f i BreakablePlane.obj
 0001:00007500       ??$__make_heap@PAU?$SplineKey@M@spline@@U?$less@U?$SplineKey@M@spline@@@stlpmtx_std@@U12@H@stlpmtx_std@@YAXPAU?$SplineKey@M@spline@@0U?$less@U?$SplineKey@M@spline@@@0@0PAH@Z 32008500 f i BreakablePlane.obj
 0001:00007640       ?SetGeometry@CBreakablePlane@@QAE_NPAUIStatObj@@PAUIMaterial@@HH@Z 32008640 f   BreakablePlane.obj
 0001:00008fa0       ?FillVertexData@CBreakablePlane@@QAEXPAVCMesh@@HABU?$Vec2_tpl@M@@H@Z 32009fa0 f   BreakablePlane.obj
 0001:00009c50       ?CreateFlatStatObj@CBreakablePlane@@QAEPAUIStatObj@@AAPAHPAU?$Vec2_tpl@M@@1ABU?$Matrix34_tpl@M@@PAUIParticleEffect@@_N4@Z 3200ac50 f   BreakablePlane.obj
 0001:0000c940       ?expand_raw@?$DynArray@U?$SplineKey@M@spline@@HU?$SmallDynStorage@U?$SplineKey@M@spline@@HUStandardAlloc@NAlloc@@@NArray@@@@IAEPAU?$SplineKey@M@spline@@PAU23@H@Z 3200d940 f i BreakablePlane.obj
 0001:0000c9d0       ??$__insertion_sort@PAU?$SplineKey@M@spline@@U12@U?$less@U?$SplineKey@M@spline@@@stlpmtx_std@@@priv@stlpmtx_std@@YAXPAU?$SplineKey@M@spline@@00U?$less@U?$SplineKey@M@spline@@@1@@Z 3200d9d0 f i BreakablePlane.obj
 0001:0000ca90       ??$sort_heap@PAU?$SplineKey@M@spline@@U?$less@U?$SplineKey@M@spline@@@stlpmtx_std@@@stlpmtx_std@@YAXPAU?$SplineKey@M@spline@@0U?$less@U?$SplineKey@M@spline@@@0@@Z 3200da90 f i BreakablePlane.obj
 0001:0000cb60       ??$AddContainer@U?$DynArray@U?$SplineKey@M@spline@@HU?$SmallDynStorage@U?$SplineKey@M@spline@@HUStandardAlloc@NAlloc@@@NArray@@@@@ICrySizer@@QAE_NABU?$DynArray@U?$SplineKey@M@spline@@HU?$SmallDynStorage@U?$SplineKey@M@spline@@HUStandardAlloc@NAlloc@@@NArray@@@@@Z 3200db60 f i BreakablePlane.obj
 0001:0000cbe0       ?GetMemoryUsage@?$TSpline@U?$SplineKey@M@spline@@U?$TCoeffBasis@M@2@@spline@@UBEXPAVICrySizer@@_N@Z 3200dbe0 f i BreakablePlane.obj
 0001:0000cc20       ??_E?$TSplineSlopes@MU?$SplineKey@M@spline@@$00@spline@@UAEPAXI@Z 3200dc20 f i BreakablePlane.obj
 0001:0000cc20       ??_G?$TSpline@U?$SplineKey@M@spline@@U?$TCoeffBasis@M@2@@spline@@UAEPAXI@Z 3200dc20 f i BreakablePlane.obj
 0001:0000cc20       ??_E?$TSpline@U?$SplineKey@M@spline@@U?$TCoeffBasis@M@2@@spline@@UAEPAXI@Z 3200dc20 f i BreakablePlane.obj
 0001:0000cc20       ??_G?$TSplineSlopes@MU?$SplineKey@M@spline@@$00@spline@@UAEPAXI@Z 3200dc20 f i BreakablePlane.obj
 0001:0000cc70       ??$__final_insertion_sort@PAU?$SplineKey@M@spline@@U?$less@U?$SplineKey@M@spline@@@stlpmtx_std@@@priv@stlpmtx_std@@YAXPAU?$SplineKey@M@spline@@0U?$less@U?$SplineKey@M@spline@@@1@@Z 3200dc70 f i BreakablePlane.obj
 0001:0000cce0       ??$__partial_sort@PAU?$SplineKey@M@spline@@U12@U?$less@U?$SplineKey@M@spline@@@stlpmtx_std@@@priv@stlpmtx_std@@YAXPAU?$SplineKey@M@spline@@000U?$less@U?$SplineKey@M@spline@@@1@@Z 3200dce0 f i BreakablePlane.obj
 0001:0000cdb0       ??0?$DynArray@U?$SplineKey@M@spline@@HU?$SmallDynStorage@U?$SplineKey@M@spline@@HUStandardAlloc@NAlloc@@@NArray@@@@QAE@ABU0@@Z 3200ddb0 f i BreakablePlane.obj
 0001:0000ce30       ?interp_keys@?$TSplineSlopes@MU?$SplineKey@M@spline@@$00@spline@@UAEXHHMAAM@Z 3200de30 f i BreakablePlane.obj
 0001:0000ced0       ?comp_deriv@?$TSplineSlopes@MU?$SplineKey@M@spline@@$00@spline@@UAEXXZ 3200ded0 f i BreakablePlane.obj
 0001:0000d450       ??$__introsort_loop@PAU?$SplineKey@M@spline@@U12@HU?$less@U?$SplineKey@M@spline@@@stlpmtx_std@@@priv@stlpmtx_std@@YAXPAU?$SplineKey@M@spline@@00HU?$less@U?$SplineKey@M@spline@@@1@@Z 3200e450 f i BreakablePlane.obj
 0001:0000d560       ??0?$TSplineSlopes@MU?$SplineKey@M@spline@@$00@spline@@QAE@ABV01@@Z 3200e560 f i BreakablePlane.obj
 0001:0000d5b0       ??$sort@PAU?$SplineKey@M@spline@@@stlpmtx_std@@YAXPAU?$SplineKey@M@spline@@0@Z 3200e5b0 f i BreakablePlane.obj
 0001:0000d610       ??0?$deep_ptr@V?$TSplineSlopes@MU?$SplineKey@M@spline@@$00@spline@@$00@@QAE@ABU0@@Z 3200e610 f i BreakablePlane.obj
 0001:0000d690       ??_EISplineBackup@@UAEPAXI@Z 3200e690 f i BreakablePlane.obj
 0001:0000d690       ??_GISplineBackup@@UAEPAXI@Z 3200e690 f i BreakablePlane.obj
 0001:0000d6c0       ?fast_interpolate@?$OptSpline@U?$TFixed@E$00$0PP@@@V?$TSplineSlopes@MU?$SplineKey@M@spline@@$00@spline@@@spline@@QBEXMAAM@Z 3200e6c0 f i BreakablePlane.obj
 0001:0000d7d0       ?find_keys_in_range@?$FinalizingSpline@V?$TSplineSlopes@MU?$SplineKey@M@spline@@$00@spline@@@spline@@QBEXMMAAH0@Z 3200e7d0 f i BreakablePlane.obj
 0001:0000d900       ?FindKeysInRange@?$CBaseSplineInterpolator@MV?$OptSpline@U?$TFixed@E$00$0PP@@@V?$TSplineSlopes@MU?$SplineKey@M@spline@@$00@spline@@@spline@@@spline@@UAEXMMAAH0@Z 3200e900 f i BreakablePlane.obj
 0001:0000d930       ?GetKeyCount@?$CBaseSplineInterpolator@MV?$OptSpline@U?$TFixed@E$00$0PP@@@V?$TSplineSlopes@MU?$SplineKey@M@spline@@$00@spline@@@spline@@@spline@@UAEHXZ 3200e930 f i BreakablePlane.obj
 0001:0000d940       ?erase@?$DynArray@U?$SplineKey@M@spline@@HU?$SmallDynStorage@U?$SplineKey@M@spline@@HUStandardAlloc@NAlloc@@@NArray@@@@QAEPAU?$SplineKey@M@spline@@PAU23@0@Z 3200e940 f i BreakablePlane.obj
 0001:0000d9c0       ?insert_raw@?$DynArray@U?$SplineKey@M@spline@@HU?$SmallDynStorage@U?$SplineKey@M@spline@@HUStandardAlloc@NAlloc@@@NArray@@@@QAE?AU?$Array@U?$SplineKey@M@spline@@HU?$ArrayStorage@U?$SplineKey@M@spline@@H@NArray@@@@PAU?$SplineKey@M@spline@@H@Z 3200e9c0 f i BreakablePlane.obj
 0001:0000da80       ?insert_key@?$FinalizingSpline@V?$TSplineSlopes@MU?$SplineKey@M@spline@@$00@spline@@@spline@@QAEHMABM@Z 3200ea80 f i BreakablePlane.obj
 0001:0000dbc0       ?remove_keys_in_range@?$FinalizingSpline@V?$TSplineSlopes@MU?$SplineKey@M@spline@@$00@spline@@@spline@@QAEXMM@Z 3200ebc0 f i BreakablePlane.obj
 0001:0000dcf0       ?InsertKey@?$CBaseSplineInterpolator@MV?$OptSpline@U?$TFixed@E$00$0PP@@@V?$TSplineSlopes@MU?$SplineKey@M@spline@@$00@spline@@@spline@@@spline@@UAEHMQAM@Z 3200ecf0 f i BreakablePlane.obj
 0001:0000dd20       ?RemoveKey@?$CBaseSplineInterpolator@MV?$OptSpline@U?$TFixed@E$00$0PP@@@V?$TSplineSlopes@MU?$SplineKey@M@spline@@$00@spline@@@spline@@@spline@@UAEXH@Z 3200ed20 f i BreakablePlane.obj
 0001:0000dd70       ?RemoveKeysInRange@?$CBaseSplineInterpolator@MV?$OptSpline@U?$TFixed@E$00$0PP@@@V?$TSplineSlopes@MU?$SplineKey@M@spline@@$00@spline@@@spline@@@spline@@UAEXMM@Z 3200ed70 f i BreakablePlane.obj
 0001:0000dd90       ?GetKeyTime@?$CBaseSplineInterpolator@MV?$OptSpline@U?$TFixed@E$00$0PP@@@V?$TSplineSlopes@MU?$SplineKey@M@spline@@$00@spline@@@spline@@@spline@@UAEMH@Z 3200ed90 f i BreakablePlane.obj
 0001:0000ddc0       ?GetKeyValue@?$CBaseSplineInterpolator@MV?$OptSpline@U?$TFixed@E$00$0PP@@@V?$TSplineSlopes@MU?$SplineKey@M@spline@@$00@spline@@@spline@@@spline@@UAE_NHAAY03M@Z 3200edc0 f i BreakablePlane.obj
 0001:0000de00       ?SetKeyValue@?$CBaseSplineInterpolator@MV?$OptSpline@U?$TFixed@E$00$0PP@@@V?$TSplineSlopes@MU?$SplineKey@M@spline@@$00@spline@@@spline@@@spline@@UAEXHQAM@Z 3200ee00 f i BreakablePlane.obj
 0001:0000de40       ?SetKeyTime@?$CBaseSplineInterpolator@MV?$OptSpline@U?$TFixed@E$00$0PP@@@V?$TSplineSlopes@MU?$SplineKey@M@spline@@$00@spline@@@spline@@@spline@@UAEXHM@Z 3200ee40 f i BreakablePlane.obj
 0001:0000de80       ?SetKeyInTangent@?$CBaseSplineInterpolator@MV?$OptSpline@U?$TFixed@E$00$0PP@@@V?$TSplineSlopes@MU?$SplineKey@M@spline@@$00@spline@@@spline@@@spline@@UAEXHQAM@Z 3200ee80 f i BreakablePlane.obj
 0001:0000dec0       ?SetKeyOutTangent@?$CBaseSplineInterpolator@MV?$OptSpline@U?$TFixed@E$00$0PP@@@V?$TSplineSlopes@MU?$SplineKey@M@spline@@$00@spline@@@spline@@@spline@@UAEXHQAM@Z 3200eec0 f i BreakablePlane.obj
 0001:0000df00       ?SetKeyTangents@?$CBaseSplineInterpolator@MV?$OptSpline@U?$TFixed@E$00$0PP@@@V?$TSplineSlopes@MU?$SplineKey@M@spline@@$00@spline@@@spline@@@spline@@UAEXHQAM0@Z 3200ef00 f i BreakablePlane.obj
 0001:0000df50       ?GetKeyTangents@?$CBaseSplineInterpolator@MV?$OptSpline@U?$TFixed@E$00$0PP@@@V?$TSplineSlopes@MU?$SplineKey@M@spline@@$00@spline@@@spline@@@spline@@UAE_NHAAY03M0@Z 3200ef50 f i BreakablePlane.obj
 0001:0000df90       ?SetKeyFlags@?$CBaseSplineInterpolator@MV?$OptSpline@U?$TFixed@E$00$0PP@@@V?$TSplineSlopes@MU?$SplineKey@M@spline@@$00@spline@@@spline@@@spline@@UAEXHH@Z 3200ef90 f i BreakablePlane.obj
 0001:0000dfd0       ?GetKeyFlags@?$CBaseSplineInterpolator@MV?$OptSpline@U?$TFixed@E$00$0PP@@@V?$TSplineSlopes@MU?$SplineKey@M@spline@@$00@spline@@@spline@@@spline@@UAEHH@Z 3200efd0 f i BreakablePlane.obj
 0001:0000e000       ??_G?$TCurve@U?$TFixed@E$00$0PP@@@@@UAEPAXI@Z 3200f000 f i BreakablePlane.obj
 0001:0000e000       ??_E?$TCurve@U?$TFixed@E$00$0PP@@@@@UAEPAXI@Z 3200f000 f i BreakablePlane.obj
 0001:0000e040       ?update@?$OptSpline@U?$TFixed@E$00$0PP@@@V?$TSplineSlopes@MU?$SplineKey@M@spline@@$00@spline@@@spline@@IAEXXZ 3200f040 f i BreakablePlane.obj
 0001:0000e270       ??4?$OptSpline@U?$TFixed@E$00$0PP@@@V?$TSplineSlopes@MU?$SplineKey@M@spline@@$00@spline@@@spline@@QAEAAV01@ABV01@@Z 3200f270 f i BreakablePlane.obj
 0001:0000e2f0       ?AddRef@?$SSplineBackup@V?$OptSpline@U?$TFixed@E$00$0PP@@@V?$TSplineSlopes@MU?$SplineKey@M@spline@@$00@spline@@@spline@@@spline@@UAEXXZ 3200f2f0 f i BreakablePlane.obj
 0001:0000e300       ?Release@?$SSplineBackup@V?$OptSpline@U?$TFixed@E$00$0PP@@@V?$TSplineSlopes@MU?$SplineKey@M@spline@@$00@spline@@@spline@@@spline@@UAEXXZ 3200f300 f i BreakablePlane.obj
 0001:0000e320       ??_G?$SSplineBackup@V?$OptSpline@U?$TFixed@E$00$0PP@@@V?$TSplineSlopes@MU?$SplineKey@M@spline@@$00@spline@@@spline@@@spline@@UAEPAXI@Z 3200f320 f i BreakablePlane.obj
 0001:0000e320       ??_E?$SSplineBackup@V?$OptSpline@U?$TFixed@E$00$0PP@@@V?$TSplineSlopes@MU?$SplineKey@M@spline@@$00@spline@@@spline@@@spline@@UAEPAXI@Z 3200f320 f i BreakablePlane.obj
 0001:0000e360       ??0?$TVarEParam@U?$TRangedType@M$0A@$0HPPPPPPP@$0A@@@@@QAE@ABM@Z 3200f360 f i BreakablePlane.obj
 0001:0000e3a0       ??0?$TVarEPParam@U?$TRangedType@M$0A@$0HPPPPPPP@$0A@@@@@QAE@ABM@Z 3200f3a0 f i BreakablePlane.obj
 0001:0000e3e0       ?Interpolate@?$CBaseSplineInterpolator@MV?$OptSpline@U?$TFixed@E$00$0PP@@@V?$TSplineSlopes@MU?$SplineKey@M@spline@@$00@spline@@@spline@@@spline@@UAEXMAAY03M@Z 3200f3e0 f i BreakablePlane.obj
 0001:0000e420       ?Backup@?$CBaseSplineInterpolator@MV?$OptSpline@U?$TFixed@E$00$0PP@@@V?$TSplineSlopes@MU?$SplineKey@M@spline@@$00@spline@@@spline@@@spline@@UAEPAUISplineBackup@@XZ 3200f420 f i BreakablePlane.obj
 0001:0000e4a0       ?Restore@?$CBaseSplineInterpolator@MV?$OptSpline@U?$TFixed@E$00$0PP@@@V?$TSplineSlopes@MU?$SplineKey@M@spline@@$00@spline@@@spline@@@spline@@UAEXPAUISplineBackup@@@Z 3200f4a0 f i BreakablePlane.obj
 0001:0000e4d0       ??0?$TCurve@U?$TFixed@E$00$0PP@@@@@QAE@ABV0@@Z 3200f4d0 f i BreakablePlane.obj
 0001:0000e540       ??0ParticleParams@@IAE@_N@Z 3200f540 f i BreakablePlane.obj
 0001:0000ea60       ??0ParticleParams@@QAE@XZ  3200fa60 f i BreakablePlane.obj
 0001:0000ef00       ??4?$TVarEParam@U?$TRangedType@M$0A@$0HPPPPPPP@$0A@@@@@QAEAAU0@ABU0@@Z 3200ff00 f i BreakablePlane.obj
 0001:0000ef60       ??4?$TVarEPParam@U?$TRangedType@M$0A@$0HPPPPPPP@$0A@@@@@QAEAAU0@ABU0@@Z 3200ff60 f i BreakablePlane.obj
 0001:0000f000       ?ProcessImpact@CBreakablePlane@@SAHABUSProcessImpactIn@@AAUSProcessImpactOut@@@Z 32010000 f   BreakablePlane.obj
 0001:00013e60       ??_GBSPTree@CBSPTree3D@@QAEPAXI@Z 32014e60 f i BSPTree3D.obj
 0001:00013ea0       ??1CBSPTree3D@@QAE@XZ      32014ea0 f   BSPTree3D.obj
 0001:00013ed0       ?IsPointIn@BSPTree@CBSPTree3D@@QBE?AW4EPointPosEnum@AreaUtil@@ABU?$Vec3_tpl@M@@@Z 32014ed0 f   BSPTree3D.obj
 0001:00013fb0       ?IsInside@CBSPTree3D@@QBE_NABU?$Vec3_tpl@M@@@Z 32014fb0 f   BSPTree3D.obj
 0001:00013fe0       ?_M_insert_overflow@?$_Impl_vector@DV?$allocator@D@stlpmtx_std@@@priv@stlpmtx_std@@AAEXPADABDABU__true_type@3@I_N@Z 32014fe0 f i BSPTree3D.obj
 0001:00014110       ?_M_fill_insert_aux@?$_Impl_vector@DV?$allocator@D@stlpmtx_std@@@priv@stlpmtx_std@@AAEXPADIABDABU__false_type@3@@Z 32015110 f i BSPTree3D.obj
 0001:00014230       ?resize@?$_Impl_vector@DV?$allocator@D@stlpmtx_std@@@priv@stlpmtx_std@@QAEXIABD@Z 32015230 f i BSPTree3D.obj
 0001:000142d0       ?SplitFaceByPlane@CBSPTree3D@@CA?AW4ESplitResult@AreaUtil@@ABVCPlane@3@ABV?$vector@U?$Vec3_tpl@M@@V?$allocator@U?$Vec3_tpl@M@@@stlpmtx_std@@@stlpmtx_std@@AAV56@2@Z 320152d0 f   BSPTree3D.obj
 0001:00014c90       ?BuildTree@CBSPTree3D@@AAEPAVBSPTree@1@ABV?$vector@V?$vector@U?$Vec3_tpl@M@@V?$allocator@U?$Vec3_tpl@M@@@stlpmtx_std@@@stlpmtx_std@@V?$allocator@V?$vector@U?$Vec3_tpl@M@@V?$allocator@U?$Vec3_tpl@M@@@stlpmtx_std@@@stlpmtx_std@@@2@@stlpmtx_std@@@Z 32015c90 f   BSPTree3D.obj
 0001:000152f0       ??0CBSPTree3D@@QAE@ABV?$vector@V?$vector@U?$Vec3_tpl@M@@V?$allocator@U?$Vec3_tpl@M@@@stlpmtx_std@@@stlpmtx_std@@V?$allocator@V?$vector@U?$Vec3_tpl@M@@V?$allocator@U?$Vec3_tpl@M@@@stlpmtx_std@@@stlpmtx_std@@@2@@stlpmtx_std@@@Z 320162f0 f   BSPTree3D.obj
 0001:00015310       ?NumToFromString@@YAMMH_NQADH@Z 32016310 f   CryEntityDLL.obj
 0001:000153a0       ?EndianDescSize@@YAIPBD@Z  320163a0 f   CryEntityDLL.obj
 0001:000153d0       ?IsType@CTypeInfo@@UBE_NABU1@@Z 320163d0 f i CryEntityDLL.obj
 0001:000153e0       ?EnterScope@CDummyMemReplay@@UAE_NW4Class@EMemReplayAllocClass@@GH@Z 320163e0 f i AreaSolid.obj
 0001:000153e0       ?FromValue@CTypeInfo@@UBE_NPAXPBXABU1@@Z 320163e0 f i CryEntityDLL.obj
 0001:000153e0       ?ToValue@CTypeInfo@@UBE_NPBXPAXABU1@@Z 320163e0 f i CryEntityDLL.obj
 0001:000153e0       ?FromString@CTypeInfo@@UBE_NPAXPBDUFFromString@@@Z 320163e0 f i CryEntityDLL.obj
 0001:000153f0       ?cry_frand@@YAMXZ          320163f0 f   CryEntityDLL.obj
 0001:00015450       ?Init@_CryMemoryManagerPoolHelper@@SAXXZ 32016450 f i CryEntityDLL.obj
 0001:000155d0       ?CryGetIMemoryManager@@YAPAUIMemoryManager@@XZ 320165d0 f   CryEntityDLL.obj
 0001:00015610       ?CryInterlockedIncrement@@YAJPCH@Z 32016610 f   CryEntityDLL.obj
 0001:00015620       ?CryInterlockedDecrement@@YAJPCH@Z 32016620 f   CryEntityDLL.obj
 0001:00015630       ?CryCreateCriticalSectionInplace@@YAXPAX@Z 32016630 f   CryEntityDLL.obj
 0001:00015640       ?CryGetCurrentThreadId@@YAIXZ 32016640 f   CryEntityDLL.obj
 0001:00015650       ?ToValue@?$TTypeInfo@M@@UBE_NPBXPAXABUCTypeInfo@@@Z 32016650 f i CryEntityDLL.obj
 0001:00015670       ?FromValue@?$TTypeInfo@M@@UBE_NPAXPBXABUCTypeInfo@@@Z 32016670 f i CryEntityDLL.obj
 0001:00015690       ?FromString@?$TTypeInfo@M@@UBE_NPAXPBDUFFromString@@@Z 32016690 f i CryEntityDLL.obj
 0001:000156d0       ?ValueEqual@?$TTypeInfo@M@@UBE_NPBX0@Z 320166d0 f i CryEntityDLL.obj
 0001:00015710       ?ValueEqual@?$TTypeInfo@H@@UBE_NPBX0@Z 32016710 f i CryEntityDLL.obj
 0001:00015710       ?ValueEqual@?$TTypeInfo@I@@UBE_NPBX0@Z 32016710 f i CryEntityDLL.obj
 0001:00015740       ?ValueEqual@?$TTypeInfo@_K@@UBE_NPBX0@Z 32016740 f i CryEntityDLL.obj
 0001:00015780       ??$ClampedIntFromString@_K@@YA_NAA_KPBD@Z 32016780 f i CryEntityDLL.obj
 0001:00015840       ??$ClampedIntFromString@H@@YA_NAAHPBD@Z 32016840 f i CryEntityDLL.obj
 0001:000158d0       ??$ClampedIntFromString@I@@YA_NAAIPBD@Z 320168d0 f i CryEntityDLL.obj
 0001:00015950       ??$ConvertInt@HF@@YA_NAAHFHH@Z 32016950 f i CryEntityDLL.obj
 0001:00015950       ??$ConvertInt@IF@@YA_NAAIFII@Z 32016950 f i CryEntityDLL.obj
 0001:00015990       ??$ConvertInt@H_J@@YA_NAAH_JHH@Z 32016990 f i CryEntityDLL.obj
 0001:000159e0       ??$ConvertInt@IG@@YA_NAAIGII@Z 320169e0 f i CryEntityDLL.obj
 0001:000159e0       ??$ConvertInt@HG@@YA_NAAHGHH@Z 320169e0 f i CryEntityDLL.obj
 0001:00015a20       ??$ConvertInt@H_K@@YA_NAAH_KHH@Z 32016a20 f i CryEntityDLL.obj
 0001:00015a70       ?CryFatalError@@YAXPBDZZ   32016a70 f i CryEntityDLL.obj
 0001:00015ae0       ?SwapEndian@CTypeInfo@@UBEXPAXI_N@Z 32016ae0 f   CryEntityDLL.obj
 0001:00015c30       ?WriteInt@@YA_NPAXIH@Z     32016c30 f i CryEntityDLL.obj
 0001:00015ce0       ?GetSize@CVarInfo@CTypeInfo@@QBEIXZ 32016ce0 f i CryEntityDLL.obj
 0001:00015d30       ?CryPureCallHandler@@YAXXZ 32016d30 f   CryEntityDLL.obj
 0001:00015d40       ?CryInvalidParameterHandler@@YAXPB_W00II@Z 32016d40 f   CryEntityDLL.obj
 0001:00015d50       _ModuleInitISystem         32016d50 f   CryEntityDLL.obj
 0001:00015e00       _CryGetMemoryInfoForModule 32016e00 f   CryEntityDLL.obj
 0001:00015e00       _CryModuleGetMemoryInfo    32016e00 f   CryEntityDLL.obj
 0001:00015e50       ?CryDeleteCriticalSectionInplace@@YAXPAX@Z 32016e50 f   CryEntityDLL.obj
 0001:00015e80       ?OnSystemEvent@CSystemEventListner_Entity@@UAEXW4ESystemEvent@@II@Z 32016e80 f i CryEntityDLL.obj
 0001:00015ef0       ?GetLimit@?$TIntTypeInfo@H@@UBE_NW4ENumericLimit@@AAM@Z 32016ef0 f i CryEntityDLL.obj
 0001:00015f50       ?FromString@?$TTypeInfo@H@@UBE_NPAXPBDUFFromString@@@Z 32016f50 f i CryEntityDLL.obj
 0001:00015f80       ?GetLimit@?$TIntTypeInfo@I@@UBE_NW4ENumericLimit@@AAM@Z 32016f80 f i CryEntityDLL.obj
 0001:00015fe0       ??$ConvertInt@HC@@YA_NAAHCHH@Z 32016fe0 f i CryEntityDLL.obj
 0001:00015fe0       ??$ConvertInt@IC@@YA_NAAICII@Z 32016fe0 f i CryEntityDLL.obj
 0001:00016020       ??$ConvertInt@HH@@YA_NAAHHHH@Z 32017020 f i CryEntityDLL.obj
 0001:00016020       ??$ConvertInt@IH@@YA_NAAIHII@Z 32017020 f i CryEntityDLL.obj
 0001:00016050       ??$ConvertInt@I_J@@YA_NAAI_JII@Z 32017050 f i CryEntityDLL.obj
 0001:000160a0       ??$ConvertInt@HE@@YA_NAAHEHH@Z 320170a0 f i CryEntityDLL.obj
 0001:000160a0       ??$ConvertInt@IE@@YA_NAAIEII@Z 320170a0 f i CryEntityDLL.obj
 0001:000160e0       ??$ConvertInt@II@@YA_NAAIIII@Z 320170e0 f i CryEntityDLL.obj
 0001:000160e0       ??$ConvertInt@HI@@YA_NAAHIHH@Z 320170e0 f i CryEntityDLL.obj
 0001:00016110       ??$ConvertInt@I_K@@YA_NAAI_KII@Z 32017110 f i CryEntityDLL.obj
 0001:00016160       ?FromString@?$TTypeInfo@I@@UBE_NPAXPBDUFFromString@@@Z 32017160 f i CryEntityDLL.obj
 0001:00016190       ?GetLimit@?$TIntTypeInfo@_K@@UBE_NW4ENumericLimit@@AAM@Z 32017190 f i CryEntityDLL.obj
 0001:00016230       ??$ConvertInt@_KC@@YA_NAA_KC_K1@Z 32017230 f i CryEntityDLL.obj
 0001:00016280       ??$ConvertInt@_KF@@YA_NAA_KF_K1@Z 32017280 f i CryEntityDLL.obj
 0001:000162d0       ??$ConvertInt@_KH@@YA_NAA_KH_K1@Z 320172d0 f i CryEntityDLL.obj
 0001:00016310       ??$ConvertInt@_K_J@@YA_NAA_K_J_K2@Z 32017310 f i CryEntityDLL.obj
 0001:00016360       ??$ConvertInt@_KE@@YA_NAA_KE_K1@Z 32017360 f i CryEntityDLL.obj
 0001:000163b0       ??$ConvertInt@_KG@@YA_NAA_KG_K1@Z 320173b0 f i CryEntityDLL.obj
 0001:00016400       ??$ConvertInt@_KI@@YA_NAA_KI_K1@Z 32017400 f i CryEntityDLL.obj
 0001:00016450       ??$ConvertInt@_K_K@@YA_NAA_K_K11@Z 32017450 f i CryEntityDLL.obj
 0001:000164a0       ?FromString@?$TTypeInfo@_K@@UBE_NPAXPBDUFFromString@@@Z 320174a0 f i CryEntityDLL.obj
 0001:000164e0       ?erase@?$CryStackStringT@D$0BA@@@QAEAAV1@II@Z 320174e0 f i CryEntityDLL.obj
 0001:00016530       ?FromValue@CStructInfo@@UBE_NPAXPBXABUCTypeInfo@@@Z 32017530 f   CryEntityDLL.obj
 0001:00016660       ?ToValue@CStructInfo@@UBE_NPBXPAXABUCTypeInfo@@@Z 32017660 f   CryEntityDLL.obj
 0001:00016790       ?ValueEqual@CStructInfo@@UBE_NPBX0@Z 32017790 f   CryEntityDLL.obj
 0001:00016800       ?GetMemoryUsage@CStructInfo@@UBEXPAVICrySizer@@PBX@Z 32017800 f   CryEntityDLL.obj
 0001:00016840       ?FindSubVar@CStructInfo@@UBEPBUCVarInfo@CTypeInfo@@PBD@Z 32017840 f   CryEntityDLL.obj
 0001:000168c0       ?IsType@CStructInfo@@UBE_NABUCTypeInfo@@@Z 320178c0 f   CryEntityDLL.obj
 0001:00016960       ??0CEnumInfo@@QAE@PBDIIPAUCEnumElem@0@@Z 32017960 f   CryEntityDLL.obj
 0001:00016ab0       ?FromString@CEnumInfo@@UBE_NPAXPBDUFFromString@@@Z 32017ab0 f   CryEntityDLL.obj
 0001:00016bb0       ?EnumElem@CEnumInfo@@UBEPBDI@Z 32017bb0 f i CryEntityDLL.obj
 0001:00016bd0       _CryModuleMalloc           32017bd0 f   CryEntityDLL.obj
 0001:00016c60       _CryModuleRealloc          32017c60 f   CryEntityDLL.obj
 0001:00016d00       _CryModuleFree             32017d00 f   CryEntityDLL.obj
 0001:00016d60       _CryModuleMemalign         32017d60 f   CryEntityDLL.obj
 0001:00016df0       ??2@YAPAXI@Z               32017df0 f   CryEntityDLL.obj
 0001:00016e40       ??_U@YAPAXI@Z              32017e40 f   CryEntityDLL.obj
 0001:00016e90       ??3@YAXPAX@Z               32017e90 f   CryEntityDLL.obj
 0001:00016f10       ??_V@YAXPAX@Z              32017f10 f   CryEntityDLL.obj
 0001:00016f90       ??_EICryFactory@@MAEPAXI@Z 32017f90 f i CryEntityDLL.obj
 0001:00016f90       ??_GICryFactory@@MAEPAXI@Z 32017f90 f i CryEntityDLL.obj
 0001:00016fc0       ??_ECSystemEventListner_Entity@@UAEPAXI@Z 32017fc0 f i CryEntityDLL.obj
 0001:00016fc0       ??_GCSystemEventListner_Entity@@UAEPAXI@Z 32017fc0 f i CryEntityDLL.obj
 0001:00016ff0       ?GetFactory@CEngineModule_EntitySystem@@UBEPAUICryFactory@@XZ 32017ff0 f i CryEntityDLL.obj
 0001:00017000       ?GetName@CEngineModule_EntitySystem@@MAEPBDXZ 32018000 f i CryEntityDLL.obj
 0001:00017010       ?GetCategory@CEngineModule_EntitySystem@@MAEPBDXZ 32018010 f i CryEntityDLL.obj
 0001:00017020       ?Initialize@CEngineModule_EntitySystem@@MAE_NAAUSSystemGlobalEnvironment@@ABUSSystemInitParams@@@Z 32018020 f i CryEntityDLL.obj
 0001:000170d0       ??_GCEngineModule_EntitySystem@@MAEPAXI@Z 320180d0 f i CryEntityDLL.obj
 0001:000170d0       ??_GICryUnknown@@MAEPAXI@Z 320180d0 f i CryEntityDLL.obj
 0001:000170d0       ??_EICryUnknown@@MAEPAXI@Z 320180d0 f i CryEntityDLL.obj
 0001:000170d0       ??_ECEngineModule_EntitySystem@@MAEPAXI@Z 320180d0 f i CryEntityDLL.obj
 0001:00017100       ??_E?$TIntTypeInfo@_K@@UAEPAXI@Z 32018100 f i CryEntityDLL.obj
 0001:00017100       ??_GCTypeInfo@@UAEPAXI@Z   32018100 f i CryEntityDLL.obj
 0001:00017100       ??_GCCustomInfo@?$TFixed@E$00$0PP@@@UAEPAXI@Z 32018100 f i ScriptBind_Entity.obj
 0001:00017100       ??_E?$TIntTypeInfo@H@@UAEPAXI@Z 32018100 f i CryEntityDLL.obj
 0001:00017100       ??_ECTypeInfo@@UAEPAXI@Z   32018100 f i CryEntityDLL.obj
 0001:00017100       ??_ECCustomInfo@?$TFixed@E$00$0PP@@@UAEPAXI@Z 32018100 f i ScriptBind_Entity.obj
 0001:00017100       ??_GCEnumInfo@@UAEPAXI@Z   32018100 f i CryEntityDLL.obj
 0001:00017100       ??_G?$TTypeInfo@M@@UAEPAXI@Z 32018100 f i CryEntityDLL.obj
 0001:00017100       ??_G?$TIntTypeInfo@H@@UAEPAXI@Z 32018100 f i CryEntityDLL.obj
 0001:00017100       ??_E?$TIntTypeInfo@I@@UAEPAXI@Z 32018100 f i CryEntityDLL.obj
 0001:00017100       ??_ECEnumInfo@@UAEPAXI@Z   32018100 f i CryEntityDLL.obj
 0001:00017100       ??_E?$TTypeInfo@M@@UAEPAXI@Z 32018100 f i CryEntityDLL.obj
 0001:00017100       ??_G?$TIntTypeInfo@_K@@UAEPAXI@Z 32018100 f i CryEntityDLL.obj
 0001:00017100       ??_G?$TIntTypeInfo@I@@UAEPAXI@Z 32018100 f i CryEntityDLL.obj
 0001:00017130       ?_AllocData@?$CryStackStringT@D$0BA@@@QAEXI@Z 32018130 f i CryEntityDLL.obj
 0001:000171a0       ?_Concatenate@?$CryStackStringT@D$0BA@@@QAEXPBDI0I@Z 320181a0 f i CryEntityDLL.obj
 0001:00017210       ?_AllocData@?$CryStackStringT@D$0BAA@@@QAEXI@Z 32018210 f i CryEntityDLL.obj
 0001:00017280       ?_AllocData@?$CryStringT@D@@IAEXI@Z 32018280 f i CryEntityDLL.obj
 0001:000172d0       ?_Free@?$CryStringT@D@@IAEXXZ 320182d0 f i CryEntityDLL.obj
 0001:00017310       ?_Assign@?$CryStringT@D@@IAEXPBDI@Z 32018310 f i CryEntityDLL.obj
 0001:000173c0       ?_MakeUnique@?$CryStringT@D@@IAEXXZ 320183c0 f i CryEntityDLL.obj
 0001:00017460       ?_Concatenate@?$CryStringT@D@@IAEXPBDI0I@Z 32018460 f i CryEntityDLL.obj
 0001:00017500       ??$TypeInfo@M@@YAABUCTypeInfo@@PBM@Z 32018500 f   CryEntityDLL.obj
 0001:00017550       ??0CFactory@CEngineModule_EntitySystem@@AAE@XZ 32018550 f i CryEntityDLL.obj
 0001:00017600       ?GetClassNameA@CFactory@CEngineModule_EntitySystem@@UBEPBDXZ 32018600 f i CryEntityDLL.obj
 0001:00017610       ?GetClassID@CFactory@CEngineModule_EntitySystem@@UBEABUCryGUID@@XZ 32018610 f i CryEntityDLL.obj
 0001:00017620       ?ClassSupports@CFactory@CEngineModule_EntitySystem@@UBE_NABUCryGUID@@@Z 32018620 f i CryEntityDLL.obj
 0001:00017670       ?ClassSupports@CFactory@CEngineModule_EntitySystem@@UBEXAAPBUCryGUID@@AAI@Z 32018670 f i CryEntityDLL.obj
 0001:00017690       ?dispose@?$sp_counted_impl_p@VCEngineModule_EntitySystem@@@detail@boost@@UAEXXZ 32018690 f i CryEntityDLL.obj
 0001:000176a0       ??$throw_exception@Vbad_alloc@std@@@boost@@YAXABVbad_alloc@std@@@Z 320186a0 f i CryEntityDLL.obj
 0001:000176d0       ??1?$shared_ptr@UICryUnknown@@@boost@@QAE@XZ 320186d0 f i CryEntityDLL.obj
 0001:000176d0       ??1?$shared_ptr@UIShaderParamCallback@@@boost@@QAE@XZ 320186d0 f i RenderProxy.obj
 0001:00017710       ??_ECFactory@CEngineModule_EntitySystem@@UAEPAXI@Z 32018710 f i CryEntityDLL.obj
 0001:00017710       ??_GCFactory@CEngineModule_EntitySystem@@UAEPAXI@Z 32018710 f i CryEntityDLL.obj
 0001:00017740       ??$?0VCEngineModule_EntitySystem@@@shared_count@detail@boost@@QAE@PAVCEngineModule_EntitySystem@@@Z 32018740 f i CryEntityDLL.obj
 0001:000177f0       ??_Gsp_counted_base@detail@boost@@UAEPAXI@Z 320187f0 f i CryEntityDLL.obj
 0001:000177f0       ??_Esp_counted_base@detail@boost@@UAEPAXI@Z 320187f0 f i CryEntityDLL.obj
 0001:000177f0       ??_G?$sp_counted_impl_p@VCEngineModule_EntitySystem@@@detail@boost@@UAEPAXI@Z 320187f0 f i CryEntityDLL.obj
 0001:000177f0       ??_E?$sp_counted_impl_p@VCEngineModule_EntitySystem@@@detail@boost@@UAEPAXI@Z 320187f0 f i CryEntityDLL.obj
 0001:00017820       ??_Gbad_alloc@std@@UAEPAXI@Z 32018820 f i CryEntityDLL.obj
 0001:00017820       ??_Ebad_alloc@std@@UAEPAXI@Z 32018820 f i CryEntityDLL.obj
 0001:00017850       ?QueryInterface@CEngineModule_EntitySystem@@MBEPAXABUCryGUID@@@Z 32018850 f i CryEntityDLL.obj
 0001:000178b0       ?append@?$CryStackStringT@D$0BA@@@QAEAAV1@ID@Z 320188b0 f i CryEntityDLL.obj
 0001:00017950       ?append@?$CryStringT@D@@QAEAAV1@ID@Z 32018950 f i CryEntityDLL.obj
 0001:00017a00       ?_Assign@?$CryStackStringT@D$0BAA@@@QAEXPBDI@Z 32018a00 f i CryEntityDLL.obj
 0001:00017a70       ??0?$CryStringT@D@@QAE@PBD@Z 32018a70 f i CryEntityDLL.obj
 0001:00017ae0       ??1?$CryStringT@D@@QAE@XZ  32018ae0 f i CryEntityDLL.obj
 0001:00017b10       ??4?$CryStringT@D@@QAEAAV0@PBD@Z 32018b10 f i CryEntityDLL.obj
 0001:00017b50       ??4?$CryStringT@D@@QAEAAV0@ABV0@@Z 32018b50 f i CryEntityDLL.obj
 0001:00017bb0       ??0?$CryStringT@D@@QAE@PBDI@Z 32018bb0 f i CryEntityDLL.obj
 0001:00017c10       ?_ConcatenateInPlace@?$CryStringT@D@@IAEXPBDI@Z 32018c10 f i CryEntityDLL.obj
 0001:00017ca0       ??$TypeInfo@H@@YAABUCTypeInfo@@PBH@Z 32018ca0 f   CryEntityDLL.obj
 0001:00017cf0       ??$TypeInfo@I@@YAABUCTypeInfo@@PBI@Z 32018cf0 f   CryEntityDLL.obj
 0001:00017d40       ?ToString@@YA?AV?$CryStringT@D@@ABM@Z 32018d40 f   CryEntityDLL.obj
 0001:00017e40       ??0CStructInfo@@QAE@PBDIIPAUCVarInfo@CTypeInfo@@0@Z 32018e40 f   CryEntityDLL.obj
 0001:000180f0       ?NextSubVar@CStructInfo@@UBEPBUCVarInfo@CTypeInfo@@PBU23@@Z 320190f0 f i CryEntityDLL.obj
 0001:00018120       ?ToString@CEnumInfo@@UBE?AV?$CryStringT@D@@PBXUFToString@@0@Z 32019120 f   CryEntityDLL.obj
 0001:00018280       ?ToString@CTypeInfo@@UBE?AV?$CryStringT@D@@PBXUFToString@@0@Z 32019280 f i CryEntityDLL.obj
 0001:000182a0       ?ValueEqual@CTypeInfo@@UBE_NPBX0@Z 320192a0 f i CryEntityDLL.obj
 0001:00018300       ?CreateClassInstance@CFactory@CEngineModule_EntitySystem@@UBE?AV?$shared_ptr@UICryUnknown@@@boost@@XZ 32019300 f i CryEntityDLL.obj
 0001:000183d0       ?IsType@?$TIntTypeInfo@H@@UBE_NABUCTypeInfo@@@Z 320193d0 f i CryEntityDLL.obj
 0001:00018400       ?ToString@?$TTypeInfo@H@@UBE?AV?$CryStringT@D@@PBXUFToString@@0@Z 32019400 f i CryEntityDLL.obj
 0001:00018460       ?ToString@?$TTypeInfo@I@@UBE?AV?$CryStringT@D@@PBXUFToString@@0@Z 32019460 f i CryEntityDLL.obj
 0001:000184c0       ?IsType@?$TIntTypeInfo@_K@@UBE_NABUCTypeInfo@@@Z 320194c0 f i CryEntityDLL.obj
 0001:000184c0       ?IsType@?$TIntTypeInfo@I@@UBE_NABUCTypeInfo@@@Z 320194c0 f i CryEntityDLL.obj
 0001:000184f0       ?ToString@?$TTypeInfo@_K@@UBE?AV?$CryStringT@D@@PBXUFToString@@0@Z 320194f0 f i CryEntityDLL.obj
 0001:00018560       ?ToString@?$TTypeInfo@M@@UBE?AV?$CryStringT@D@@PBXUFToString@@0@Z 32019560 f i CryEntityDLL.obj
 0001:000185b0       ??Y?$CryStackStringT@D$0BA@@@QAEAAV0@D@Z 320195b0 f i CryEntityDLL.obj
 0001:00018620       ??$ConvertInt@H@@YA_NAAHPBXABUCTypeInfo@@HH@Z 32019620 f i CryEntityDLL.obj
 0001:00018840       ??$ConvertInt@I@@YA_NAAIPBXABUCTypeInfo@@II@Z 32019840 f i CryEntityDLL.obj
 0001:00018a60       ??$ConvertInt@_K@@YA_NAA_KPBXABUCTypeInfo@@_K3@Z 32019a60 f i CryEntityDLL.obj
 0001:00018cc0       ??Y?$CryStringT@D@@QAEAAV0@PBD@Z 32019cc0 f i CryEntityDLL.obj
 0001:00018d00       ??_ECStructInfo@@UAEPAXI@Z 32019d00 f i CryEntityDLL.obj
 0001:00018d00       ??_GCStructInfo@@UAEPAXI@Z 32019d00 f i CryEntityDLL.obj
 0001:00018d50       ?AddEndianDesc@CStructInfo@@IAEIPBDII@Z 32019d50 f   CryEntityDLL.obj
 0001:00018f90       ?ToString@CStructInfo@@UBE?AV?$CryStringT@D@@PBXUFToString@@0@Z 32019f90 f   CryEntityDLL.obj
 0001:00019190       ?MakeEndianDesc@CStructInfo@@IAEXXZ 3201a190 f   CryEntityDLL.obj
 0001:000192f0       ?ToValue@CEnumInfo@@UBE_NPBXPAXABUCTypeInfo@@@Z 3201a2f0 f   CryEntityDLL.obj
 0001:000193e0       ?FromValue@CEnumInfo@@UBE_NPAXPBXABUCTypeInfo@@@Z 3201a3e0 f   CryEntityDLL.obj
 0001:00019430       ?FromValue@?$TIntTypeInfo@H@@UBE_NPAXPBXABUCTypeInfo@@@Z 3201a430 f i CryEntityDLL.obj
 0001:00019460       ?ToValue@?$TIntTypeInfo@H@@UBE_NPBXPAXABUCTypeInfo@@@Z 3201a460 f i CryEntityDLL.obj
 0001:000194c0       ?FromValue@?$TIntTypeInfo@I@@UBE_NPAXPBXABUCTypeInfo@@@Z 3201a4c0 f i CryEntityDLL.obj
 0001:000194e0       ?ToValue@?$TIntTypeInfo@I@@UBE_NPBXPAXABUCTypeInfo@@@Z 3201a4e0 f i CryEntityDLL.obj
 0001:00019540       ?FromValue@?$TIntTypeInfo@_K@@UBE_NPAXPBXABUCTypeInfo@@@Z 3201a540 f i CryEntityDLL.obj
 0001:00019570       ?ToValue@?$TIntTypeInfo@_K@@UBE_NPBXPAXABUCTypeInfo@@@Z 3201a570 f i CryEntityDLL.obj
 0001:000195d0       ?ParseElement@@YAPBDAAPBDAAV?$CryStackStringT@D$0BAA@@@@Z 3201a5d0 f   CryEntityDLL.obj
 0001:00019760       ?FromString@CStructInfo@@UBE_NPAXPBDUFFromString@@@Z 3201a760 f   CryEntityDLL.obj
 0001:00019870       ?SwapEndian@CStructInfo@@UBEXPAXI_N@Z 3201a870 f   CryEntityDLL.obj
 0001:00019ea0       ??1ScriptAnyValue@@QAE@XZ  3201aea0 f i Entity.obj
 0001:00019ef0       ?PhysicalizeAttachment@IAttachmentObject@@UAE_NPAUIAttachmentManager@@HHPAUIPhysicalEntity@@ABU?$Vec3_tpl@M@@@Z 3201aef0 f i Entity.obj
 0001:00019f00       ?UpdatePhysicalizedAttachment@IAttachmentObject@@UAE_NPAUIAttachmentManager@@HPAUIPhysicalEntity@@ABU?$QuatT_tpl@M@@@Z 3201af00 f i Entity.obj
 0001:00019f10       ?SetPoolControl@CEntity@@QAEX_N@Z 3201af10 f   Entity.obj
 0001:00019f50       ?SetFlags@CEntity@@UAEXI@Z 3201af50 f   Entity.obj
 0001:00019fb0       ?IsPrePhysicsActive@CEntity@@UAE_NXZ 3201afb0 f   Entity.obj
 0001:00019fc0       ?EnableInheritXForm@CEntity@@UAEX_N@Z 3201afc0 f   Entity.obj
 0001:00019fe0       ?GetWorldTM@CEntity@@UBEABU?$Matrix34_tpl@M@@XZ 3201afe0 f   Entity.obj
 0001:00019ff0       ?OnRellocate@CEntity@@IAEXH@Z 3201aff0 f   Entity.obj
 0001:0001a170       ?PrePhysicsActivate@CEntity@@UAEX_N@Z 3201b170 f   Entity.obj
 0001:0001a190       ?KillTimer@CEntity@@UAEXH@Z 3201b190 f   Entity.obj
 0001:0001a1b0       ?SetUpdatePolicy@CEntity@@UAEXW4EEntityUpdatePolicy@@@Z 3201b1b0 f   Entity.obj
 0001:0001a1d0       ?SerializeXML@CEntity@@UAEXAAVXmlNodeRef@@_N@Z 3201b1d0 f   Entity.obj
 0001:0001a240       ?AllocNewProxyIndex@CEntity@@QAEHXZ 3201b240 f   Entity.obj
 0001:0001a300       ?SetProxy@CEntity@@UAEXW4EEntityProxy@@PAUIEntityProxy@@@Z 3201b300 f   Entity.obj
 0001:0001a3a0       ?Physicalize@CEntity@@UAEXAAUSEntityPhysicalizeParams@@@Z 3201b3a0 f   Entity.obj
 0001:0001a410       ?EnablePhysics@CEntity@@UAEX_N@Z 3201b410 f   Entity.obj
 0001:0001a440       ?PhysicalizeSlot@CEntity@@UAEHHAAUSEntityPhysicalizeParams@@@Z 3201b440 f   Entity.obj
 0001:0001a490       ?UnphysicalizeSlot@CEntity@@UAEXH@Z 3201b490 f   Entity.obj
 0001:0001a4d0       ?UpdateSlotPhysics@CEntity@@UAEXH@Z 3201b4d0 f   Entity.obj
 0001:0001a530       ?FreeSlot@CEntity@@UAEXH@Z 3201b530 f   Entity.obj
 0001:0001a570       ?GetSlotCount@CEntity@@UBEHXZ 3201b570 f   Entity.obj
 0001:0001a5b0       ?GetSlotInfo@CEntity@@UBE_NHAAUSEntitySlotInfo@@@Z 3201b5b0 f   Entity.obj
 0001:0001a5f0       ?GetSlotWorldTM@CEntity@@UBEABU?$Matrix34_tpl@M@@H@Z 3201b5f0 f   Entity.obj
 0001:0001a630       ?GetSlotLocalTM@CEntity@@UBEABU?$Matrix34_tpl@M@@H_N@Z 3201b630 f   Entity.obj
 0001:0001a670       ?SetParentSlot@CEntity@@UAE_NHH@Z 3201b670 f   Entity.obj
 0001:0001a6b0       ?SetSlotMaterial@CEntity@@UAEXHPAUIMaterial@@@Z 3201b6b0 f   Entity.obj
 0001:0001a6f0       ?SetSlotFlags@CEntity@@UAEXHI@Z 3201b6f0 f   Entity.obj
 0001:0001a730       ?GetSlotFlags@CEntity@@UBEIH@Z 3201b730 f   Entity.obj
 0001:0001a770       ?GetCharacter@CEntity@@UAEPAUICharacterInstance@@H@Z 3201b770 f   Entity.obj
 0001:0001a7b0       ?SetCharacter@CEntity@@UAEHPAUICharacterInstance@@H@Z 3201b7b0 f   Entity.obj
 0001:0001a880       ?GetStatObj@CEntity@@UAEPAUIStatObj@@H@Z 3201b880 f   Entity.obj
 0001:0001a8c0       ?SetStatObj@CEntity@@UAEHPAUIStatObj@@H_NM@Z 3201b8c0 f   Entity.obj
 0001:0001a9b0       ?GetParticleEmitter@CEntity@@UAEPAUIParticleEmitter@@H@Z 3201b9b0 f   Entity.obj
 0001:0001a9f0       ?SetParticleEmitter@CEntity@@UAEHHPAUIParticleEmitter@@_N@Z 3201b9f0 f   Entity.obj
 0001:0001aa60       ?LoadParticleEmitter@CEntity@@UAEHHPAUIParticleEffect@@PBUSpawnParams@@_N2@Z 3201ba60 f   Entity.obj
 0001:0001aad0       ?LoadCloud@CEntity@@QAEHHPBD@Z 3201bad0 f   Entity.obj
 0001:0001ab40       ?SetCloudMovementProperties@CEntity@@QAEHHABUSCloudMovementProperties@@@Z 3201bb40 f   Entity.obj
 0001:0001abb0       ?LoadFogVolume@CEntity@@QAEHHABUSFogVolumeProperties@@@Z 3201bbb0 f   Entity.obj
 0001:0001ac20       ?LoadLightShape@CEntity@@UAEHHPBDI@Z 3201bc20 f   Entity.obj
 0001:0001ac90       ?FadeGlobalDensity@CEntity@@QAEHHMM@Z 3201bc90 f   Entity.obj
 0001:0001ad20       ?LoadVolumeObject@CEntity@@QAEHHPBD@Z 3201bd20 f   Entity.obj
 0001:0001ad90       ?SetVolumeObjectMovementProperties@CEntity@@QAEHHABUSVolumeObjectMovementProperties@@@Z 3201bd90 f   Entity.obj
 0001:0001ae00       ?LoadPrismObject@CEntity@@UAEHH@Z 3201be00 f   Entity.obj
 0001:0001ae70       ?GetEntityLinks@CEntity@@UAEPAUIEntityLink@@XZ 3201be70 f   Entity.obj
 0001:0001ae80       ?DebugDraw@CEntity@@UAEXABUSGeometryDebugDrawInfo@@@Z 3201be80 f   Entity.obj
 0001:0001aec0       ?CryWarning@@YAXW4EValidatorModule@@W4EValidatorSeverity@@PBDZZ 3201bec0 f i Entity.obj
 0001:0001af00       ??$GetValue@_N@IScriptTable@@QAE_NPBDAA_N@Z 3201bf00 f i Entity.obj
 0001:0001af80       ??$SetValue@H@IScriptTable@@QAEXPBDABH@Z 3201bf80 f i Entity.obj
 0001:0001aff0       ??$__find@PAPAUIAreaManagerEventListener@@PAU1@@priv@stlpmtx_std@@YAPAPAUIAreaManagerEventListener@@PAPAU2@0ABQAU2@ABUrandom_access_iterator_tag@1@@Z 3201bff0 f i AreaManager.obj
 0001:0001aff0       ??$__find@PBQAUIEntityClass@@PAU1@@priv@stlpmtx_std@@YAPBQAUIEntityClass@@PBQAU2@0ABQAU2@ABUrandom_access_iterator_tag@1@@Z 3201bff0 f i EntityPoolDefinition.obj
 0001:0001aff0       ??$__find@PAII@priv@stlpmtx_std@@YAPAIPAI0ABIABUrandom_access_iterator_tag@1@@Z 3201bff0 f i SoundProxy.obj
 0001:0001aff0       ??$__find@PAPAVCEntity@@PAV1@@priv@stlpmtx_std@@YAPAPAVCEntity@@PAPAV2@0ABQAV2@ABUrandom_access_iterator_tag@1@@Z 3201bff0 f i Entity.obj
 0001:0001aff0       ??$__find@PAPAUSProximityElement@@PAU1@@priv@stlpmtx_std@@YAPAPAUSProximityElement@@PAPAU2@0ABQAU2@ABUrandom_access_iterator_tag@1@@Z 3201bff0 f i ProximityTriggerSystem.obj
 0001:0001b060       ??_EIEntity@@UAEPAXI@Z     3201c060 f i Entity.obj
 0001:0001b060       ??_GIEntity@@UAEPAXI@Z     3201c060 f i Entity.obj
 0001:0001b090       ?GetScriptTable@IEntity@@QBEPAUIScriptTable@@XZ 3201c090 f i Entity.obj
 0001:0001b0b0       ?EntityWarning@@YAXPBDZZ   3201c0b0 f i Entity.obj
 0001:0001b0e0       ?HaveValue@IScriptTable@@QAE_NPBD@Z 3201c0e0 f i Entity.obj
 0001:0001b170       ?SetToNull@IScriptTable@@QAEXPBD@Z 3201c170 f i Entity.obj
 0001:0001b1e0       ?GetType@CEntityNodeProxy@@UAE?AW4EEntityProxy@@XZ 3201c1e0 f i Entity.obj
 0001:0001b1f0       ?Init@CEntityNodeProxy@@UAE_NPAUIEntity@@AAUSEntitySpawnParams@@@Z 3201c1f0 f i Entity.obj
 0001:0001b200       ?Reload@CEntityNodeProxy@@UAEXPAUIEntity@@AAUSEntitySpawnParams@@@Z 3201c200 f i Entity.obj
 0001:0001b210       ?NeedSerialize@CSoundProxy@@UAE_NXZ 3201c210 f i SoundProxy.obj
 0001:0001b210       ?NeedSerialize@CCameraProxy@@UAE_NXZ 3201c210 f i CameraProxy.obj
 0001:0001b210       ?NeedSerialize@CAreaProxy@@UAE_NXZ 3201c210 f i AreaProxy.obj
 0001:0001b210       ?NeedSerialize@CEntityNodeProxy@@UAE_NXZ 3201c210 f i Entity.obj
 0001:0001b210       ?HasChanged@CRenderProxy@@UAE_NXZ 3201c210 f i RenderProxy.obj
 0001:0001b210       ?GetSortPriority@IRenderNode@@UAEEXZ 3201c210 f i RenderProxy.obj
 0001:0001b220       ?GetAttachmentType@CEntityAttachment@@UAE?AW4EType@IAttachmentObject@@XZ 3201c220 f i Entity.obj
 0001:0001b230       ?Release@CEntityClass@@UAEXXZ 3201c230 f i EntityClass.obj
 0001:0001b230       ?Release@CEffectAttachment@@UAEXXZ 3201c230 f i ScriptBind_Entity.obj
 0001:0001b230       ?Release@CScriptProxy@@UAEXXZ 3201c230 f i ScriptProxy.obj
 0001:0001b230       ?Release@CTriggerProxy@@UAEXXZ 3201c230 f i TriggerProxy.obj
 0001:0001b230       ?Release@CEntityNodeProxy@@UAEXXZ 3201c230 f i Entity.obj
 0001:0001b230       ?destroy@sp_counted_base@detail@boost@@UAEXXZ 3201c230 f i CryEntityDLL.obj
 0001:0001b230       ?Release@CEntityAttachment@@UAEXXZ 3201c230 f i Entity.obj
 0001:0001b230       ?Release@CAreaProxy@@UAEXXZ 3201c230 f i AreaProxy.obj
 0001:0001b230       ?Release@CCGFAttachment@@UAEXXZ 3201c230 f i ScriptBind_Entity.obj
 0001:0001b230       ?Release@CEntityScript@@UAEXXZ 3201c230 f i EntityScript.obj
 0001:0001b230       ?Release@CCameraProxy@@UAEXXZ 3201c230 f i CameraProxy.obj
 0001:0001b230       ?Release@CArea@@QAEXXZ     3201c230 f i Area.obj
 0001:0001b230       ?Release@CLightAttachment@@UAEXXZ 3201c230 f i ScriptBind_Entity.obj
 0001:0001b230       ?Release@CFlowGraphProxy@@UAEXXZ 3201c230 f i FlowGraphProxy.obj
 0001:0001b230       ?Release@CEntitySystem@@UAEXXZ 3201c230 f i EntitySystem.obj
 0001:0001b230       ?ReleaseNode@IRenderNode@@UAEXXZ 3201c230 f i RenderProxy.obj
 0001:0001b230       ?Release@CSubstitutionProxy@@UAEXXZ 3201c230 f i Entity.obj
 0001:0001b240       ?GetAABB@CEntityAttachment@@UAE?AUAABB@@XZ 3201c240 f i Entity.obj
 0001:0001b2c0       ?GetRadiusSqr@CEntityAttachment@@UAEMXZ 3201c2c0 f i Entity.obj
 0001:0001b360       ??_ECEntityAttachment@@UAEPAXI@Z 3201c360 f i Entity.obj
 0001:0001b360       ??_GIAttachmentObject@@UAEPAXI@Z 3201c360 f i Entity.obj
 0001:0001b360       ??_EIAttachmentObject@@UAEPAXI@Z 3201c360 f i Entity.obj
 0001:0001b360       ??_GCEntityAttachment@@UAEPAXI@Z 3201c360 f i Entity.obj
 0001:0001b390       ?SetName@CEntity@@UAEXPBD@Z 3201c390 f   Entity.obj
 0001:0001b420       ?Init@CEntity@@QAE_NAAUSEntitySpawnParams@@@Z 3201c420 f   Entity.obj
 0001:0001b540       ?SetPos@CEntity@@UAEXABU?$Vec3_tpl@M@@H@Z 3201c540 f   Entity.obj
 0001:0001b5a0       ?SetRotation@CEntity@@UAEXABU?$Quat_tpl@M@@H@Z 3201c5a0 f   Entity.obj
 0001:0001b620       ?SetScale@CEntity@@UAEXABU?$Vec3_tpl@M@@H@Z 3201c620 f   Entity.obj
 0001:0001b680       ?GetWorldBounds@CEntity@@UBEXAAUAABB@@@Z 3201c680 f   Entity.obj
 0001:0001b8f0       ?GetLocalBounds@CEntity@@UBEXAAUAABB@@@Z 3201c8f0 f   Entity.obj
 0001:0001b9e0       ?SetUpdateStatus@CEntity@@QAEXXZ 3201c9e0 f   Entity.obj
 0001:0001ba80       ?Activate@CEntity@@UAEX_N@Z 3201ca80 f   Entity.obj
 0001:0001bab0       ?SetTimer@CEntity@@UAEXHH@Z 3201cab0 f   Entity.obj
 0001:0001bb10       ?GetProxy@CEntity@@UBEPAUIEntityProxy@@W4EEntityProxy@@@Z 3201cb10 f   Entity.obj
 0001:0001bc30       ?GetPhysics@CEntity@@UBEPAUIPhysicalEntity@@XZ 3201cc30 f   Entity.obj
 0001:0001bcf0       ?CheckMaterialFlags@CEntity@@QAEXXZ 3201ccf0 f   Entity.obj
 0001:0001bd90       ?GetMaterial@CEntity@@UAEPAUIMaterial@@XZ 3201cd90 f   Entity.obj
 0001:0001bda0       ?LoadLightImpl@CEntity@@QAEHHPAVCDLight@@_N@Z 3201cda0 f   Entity.obj
 0001:0001be60       ?UpdateAIObject@CEntity@@QAEXXZ 3201ce60 f   Entity.obj
 0001:0001bed0       ?ActivateForNumUpdates@CEntity@@QAEXH@Z 3201ced0 f   Entity.obj
 0001:0001bf60       ?RemoveBoneAttachLinkIfAny@CEntity@@AAEXXZ 3201cf60 f   Entity.obj
 0001:0001bfb0       ?LogEvent@CEntity@@IAEXAAUSEntityEvent@@VCTimeValue@@@Z 3201cfb0 f   Entity.obj
 0001:0001c080       ?OrthonormalizeFast@?$Matrix34_tpl@M@@QAEXXZ 3201d080 f i Entity.obj
 0001:0001c280       ?IsOrthonormal@?$Matrix34_tpl@M@@QBEHM@Z 3201d280 f i Entity.obj
 0001:0001c4a0       ??0pe_params_part@@QAE@XZ  3201d4a0 f i Entity.obj
 0001:0001c560       ??0pe_params_foreign_data@@QAE@XZ 3201d560 f i Entity.obj
 0001:0001c590       ??$?0M@?$Ang3_tpl@M@@QAE@ABU?$Matrix34_tpl@M@@@Z 3201d590 f i Entity.obj
 0001:0001c660       ??0CMemStatContextFormat@@QAA@W4Type@EMemStatContextTypes@@IPBDZZ 3201d660 f i Entity.obj
 0001:0001c690       ?CallMethod@Script@@SA_NPAUIScriptTable@@PBD@Z 3201d690 f i Entity.obj
 0001:0001c710       ?GetType@CSubstitutionProxy@@UAE?AW4EEntityProxy@@XZ 3201d710 f i Entity.obj
 0001:0001c720       ?GetMemoryUsage@CSubstitutionProxy@@UBEXPAVICrySizer@@@Z 3201d720 f i Entity.obj
 0001:0001c740       ??_GCSubstitutionProxy@@UAEPAXI@Z 3201d740 f i Entity.obj
 0001:0001c740       ??_ECSubstitutionProxy@@UAEPAXI@Z 3201d740 f i Entity.obj
 0001:0001c780       ?Update@CEntity@@QAEXAAUSEntityUpdateContext@@@Z 3201d780 f   Entity.obj
 0001:0001c910       ?PrePhysicsUpdate@CEntity@@QAEXM@Z 3201d910 f   Entity.obj
 0001:0001ca50       ?GetChildCount@CEntity@@UBEHXZ 3201da50 f   Entity.obj
 0001:0001ca70       ?SetWorldTM@CEntity@@UAEXABU?$Matrix34_tpl@M@@H@Z 3201da70 f   Entity.obj
 0001:0001d0b0       ?SetPosRotScale@CEntity@@UAEXABU?$Vec3_tpl@M@@ABU?$Quat_tpl@M@@0H@Z 3201e0b0 f   Entity.obj
 0001:0001d1d0       ?SetMaterial@CEntity@@UAEXPAUIMaterial@@@Z 3201e1d0 f   Entity.obj
 0001:0001d250       ?SetSlotLocalTM@CEntity@@UAEXHABU?$Matrix34_tpl@M@@H@Z 3201e250 f   Entity.obj
 0001:0001d290       ?LoadGeometry@CEntity@@UAEHHPBD0H@Z 3201e290 f   Entity.obj
 0001:0001d470       ?LoadCharacter@CEntity@@UAEHHPBDH@Z 3201e470 f   Entity.obj
 0001:0001d680       ?LoadLight@CEntity@@UAEHHPAVCDLight@@@Z 3201e680 f   Entity.obj
 0001:0001d6a0       ?GetMemoryUsage@CEntity@@UBEXPAVICrySizer@@@Z 3201e6a0 f   Entity.obj
 0001:0001d720       ??1AgentParameters@@QAE@XZ 3201e720 f i Entity.obj
 0001:0001d780       ??0AgentParameters@@QAE@ABU0@@Z 3201e780 f i Entity.obj
 0001:0001d9a0       ?ProcessAttachment@CEntityAttachment@@UAEXPAUIAttachment@@@Z 3201e9a0 f i Entity.obj
 0001:0001da30       ?GetGuid@CEntity@@UBE_KXZ  3201ea30 f i Entity.obj
 0001:0001da40       ?GetArchetype@CEntity@@UAEPAUIEntityArchetype@@XZ 3201ea40 f i Entity.obj
 0001:0001da40       ?GetEditorHelperObjectName@CEntityClass@@UBEPBDXZ 3201ea40 f i EntityClass.obj
 0001:0001da50       ?GetUserProxyData@CEntityClass@@UBEPAXXZ 3201ea50 f i EntityClass.obj
 0001:0001da50       ?GetFlags@CEntity@@UBEIXZ  3201ea50 f i Entity.obj
 0001:0001da60       ?AddFlags@CEntity@@UAEXI@Z 3201ea60 f i Entity.obj
 0001:0001da80       ?ClearFlags@CEntity@@UAEXI@Z 3201ea80 f i Entity.obj
 0001:0001daa0       ?CheckFlags@CEntity@@UBE_NI@Z 3201eaa0 f i Entity.obj
 0001:0001dac0       ?IsGarbage@CEntity@@UBE_NXZ 3201eac0 f i Entity.obj
 0001:0001dad0       ?GetParent@CEntity@@UBEPAUIEntity@@XZ 3201ead0 f i Entity.obj
 0001:0001daf0       ?GetAdam@CEntity@@UAEPAUIEntity@@XZ 3201eaf0 f i Entity.obj
 0001:0001db20       ?GetPos@CEntity@@UBEABU?$Vec3_tpl@M@@XZ 3201eb20 f i Entity.obj
 0001:0001db30       ?GetRotation@CEntity@@UBEABU?$Quat_tpl@M@@XZ 3201eb30 f i Entity.obj
 0001:0001db40       ?GetScale@CEntity@@UBEABU?$Vec3_tpl@M@@XZ 3201eb40 f i Entity.obj
 0001:0001db50       ?IsActive@CEntity@@UBE_NXZ 3201eb50 f i Entity.obj
 0001:0001db60       ?IsHidden@CEntity@@UBE_NXZ 3201eb60 f i Entity.obj
 0001:0001db70       ?IsInvisible@CEntity@@UBE_NXZ 3201eb70 f i Entity.obj
 0001:0001db80       ?HasAI@CEntity@@UBE_NXZ    3201eb80 f i Entity.obj
 0001:0001db90       ?GetAIObjectID@CEntity@@UBEIXZ 3201eb90 f i Entity.obj
 0001:0001dba0       ?SetAIObjectID@CEntity@@UAEXI@Z 3201eba0 f i Entity.obj
 0001:0001dbb0       ?GetUpdatePolicy@CEntity@@UBE?AW4EEntityUpdatePolicy@@XZ 3201ebb0 f i Entity.obj
 0001:0001dbc0       ?IsInitialized@CEntity@@UBE_NXZ 3201ebc0 f i Entity.obj
 0001:0001dbd0       ?IncKeepAliveCounter@CEntity@@UAEXXZ 3201ebd0 f i Entity.obj
 0001:0001dbe0       ?DecKeepAliveCounter@CEntity@@UAEXXZ 3201ebe0 f i Entity.obj
 0001:0001dbf0       ?ResetKeepAliveCounter@CEntity@@UAEXXZ 3201ebf0 f i Entity.obj
 0001:0001dc00       ?IsKeptAlive@CEntity@@UBE_NXZ 3201ec00 f i Entity.obj
 0001:0001dc10       ?GetName@CEntity@@UBEPBDXZ 3201ec10 f i Entity.obj
 0001:0001dc20       ?GetWorldPos@CEntity@@UBE?AU?$Vec3_tpl@M@@XZ 3201ec20 f i Entity.obj
 0001:0001dc50       ?IsFromPool@CEntity@@UBE_NXZ 3201ec50 f i Entity.obj
 0001:0001dc60       ?GetAI@CEntity@@UAEPAUIAIObject@@XZ 3201ec60 f i Entity.obj
 0001:0001dca0       ?GetForwardDir@CEntity@@UBEABU?$Vec3_tpl@M@@XZ 3201eca0 f i Entity.obj
 0001:0001ddd0       ?DetachAll@CEntity@@UAEXH@Z 3201edd0 f   Entity.obj
 0001:0001de20       ?GetChild@CEntity@@UBEPAUIEntity@@H@Z 3201ee20 f   Entity.obj
 0001:0001de50       ?SetLocalTM@CEntity@@UAEXABU?$Matrix34_tpl@M@@H@Z 3201ee50 f   Entity.obj
 0001:0001e120       ?CalcLocalTM@CEntity@@QBEXAAU?$Matrix34_tpl@M@@@Z 3201f120 f   Entity.obj
 0001:0001e440       ?GetLocalTM@CEntity@@UBE?AU?$Matrix34_tpl@M@@XZ 3201f440 f   Entity.obj
 0001:0001e460       ?InvalidateTM@CEntity@@UAEXH@Z 3201f460 f   Entity.obj
 0001:0001e780       ?GetWorldAngles@CEntity@@UBE?AU?$Ang3_tpl@M@@XZ 3201f780 f   Entity.obj
 0001:0001e870       ?GetWorldRotation@CEntity@@UBE?AU?$Quat_tpl@M@@XZ 3201f870 f   Entity.obj
 0001:0001ed20       ?Hide@CEntity@@UAEX_N@Z    3201fd20 f   Entity.obj
 0001:0001ee20       ?Invisible@CEntity@@UAEX_N@Z 3201fe20 f   Entity.obj
 0001:0001ef00       ?IsSlotValid@CEntity@@UBE_NH@Z 3201ff00 f   Entity.obj
 0001:0001ef60       ?GetSlot@CEntity@@QBEPAVCEntityObject@@H@Z 3201ff60 f   Entity.obj
 0001:0001efc0       ?MoveSlot@CEntity@@UAEXPAUIEntity@@H@Z 3201ffc0 f   Entity.obj
 0001:0001f210       ??0AIObjectParams@@QAE@ABU0@@Z 32020210 f i Entity.obj
 0001:0001f280       ?SetPhysicsState@CEntity@@UAEXAAVXmlNodeRef@@@Z 32020280 f   Entity.obj
 0001:0001f470       ??0CEntity@@AAE@AAUSEntitySpawnParams@@@Z 32020470 f   Entity.obj
 0001:0001f720       ??_GCEntity@@UAEPAXI@Z     32020720 f i Entity.obj
 0001:0001f720       ??_ECEntity@@UAEPAXI@Z     32020720 f i Entity.obj
 0001:0001f790       ?Serialize@CEntity@@UAEXV?$CSerializeWrapper@UISerialize@@@@H@Z 32020790 f   Entity.obj
 0001:000203a0       ?UpdateLightClipBounds@CEntity@@UAE_NAAVCDLight@@@Z 320213a0 f   Entity.obj
 0001:00020a00       ?RegisterInAISystem@CEntity@@UAE_NABUAIObjectParams@@@Z 32021a00 f   Entity.obj
 0001:00020b10       ??2CRenderProxy@@SAPAXI@Z  32021b10 f i Entity.obj
 0001:00020b50       ?CreateProxy@CEntity@@UAEPAUIEntityProxy@@W4EEntityProxy@@@Z 32021b50 f   Entity.obj
 0001:00020e60       ?AttachToBone@CEntity@@AAEXPBDPAUIEntity@@ABU?$Quat_tpl@M@@ABU?$Vec3_tpl@M@@@Z 32021e60 f   Entity.obj
 0001:00020fc0       ?DetachFromBone@CEntity@@AAEXPBDPAUIEntity@@@Z 32021fc0 f   Entity.obj
 0001:00021040       ?RemoveAllEntityLinks@CEntity@@UAEXXZ 32022040 f   Entity.obj
 0001:000210e0       ??$?HD@@YA?AV?$CryStringT@D@@ABV0@PBD@Z 320220e0 f i Entity.obj
 0001:00021140       ?DetachThis@CEntity@@UAEXHH@Z 32022140 f   Entity.obj
 0001:000212e0       ?DeallocBindings@CEntity@@IAEXXZ 320222e0 f   Entity.obj
 0001:00021350       ?GetEntityTextDescription@CEntity@@UBEPBDXZ 32022350 f   Entity.obj
 0001:000214b0       ?AddEntityLink@CEntity@@UAEPAUIEntityLink@@PBDIABU?$Quat_tpl@M@@ABU?$Vec3_tpl@M@@@Z 320224b0 f   Entity.obj
 0001:000215d0       ?RemoveEntityLink@CEntity@@UAEXPAUIEntityLink@@@Z 320225d0 f   Entity.obj
 0001:000216c0       ?ReapplyBoneAttachLinkIfAny@CEntity@@AAEXXZ 320226c0 f   Entity.obj
 0001:00021730       ?SendEvent@CEntity@@UAE_NAAUSEntityEvent@@@Z 32022730 f   Entity.obj
 0001:00021c60       ?ShutDown@CEntity@@QAEX_N0@Z 32022c60 f   Entity.obj
 0001:00022010       ?AllocBindings@CEntity@@IAEXXZ 32023010 f   Entity.obj
 0001:00022080       ?ReloadEntity@CEntity@@QAE_NAAUSEntityLoadParams@@@Z 32023080 f   Entity.obj
 0001:00022450       ?AttachChild@CEntity@@UAEXPAUIEntity@@H@Z 32023450 f   Entity.obj
 0001:00022730       ??$GetValue@PBD@IScriptTable@@QAE_NPBDAAPBD@Z 32023730 f i EntityArchetype.obj
 0001:000227b0       ??$SetValue@PBD@IScriptTable@@QAEXPBDABQBD@Z 320237b0 f i EntityArchetype.obj
 0001:00022820       ?_Rotate_left@?$_Rb_global@_N@priv@stlpmtx_std@@SAXPAU_Rb_tree_node_base@23@AAPAU423@@Z 32023820 f i EntityArchetype.obj
 0001:00022870       ?_Rotate_right@?$_Rb_global@_N@priv@stlpmtx_std@@SAXPAU_Rb_tree_node_base@23@AAPAU423@@Z 32023870 f i EntityArchetype.obj
 0001:000228c0       ?AddRef@?$_i_reference_target@H@@UAEXXZ 320238c0 f i EntityArchetype.obj
 0001:000228d0       ?Release@?$_i_reference_target@H@@UAEXXZ 320238d0 f i EntityArchetype.obj
 0001:00022900       ??_E?$_i_reference_target@H@@UAEPAXI@Z 32023900 f i EntityArchetype.obj
 0001:00022900       ??_G?$_i_reference_target@H@@UAEPAXI@Z 32023900 f i EntityArchetype.obj
 0001:00022930       ?LoadFromXML@CEntityArchetype@@UAEXAAVXmlNodeRef@@@Z 32023930 f   EntityArchetype.obj
 0001:00022a10       ??R?$less_stricmp@PBD@stl@@QBE_NABQBD0@Z 32023a10 f i EntityArchetype.obj
 0001:00022a40       ?_Rebalance@?$_Rb_global@_N@priv@stlpmtx_std@@SAXPAU_Rb_tree_node_base@23@AAPAU423@@Z 32023a40 f i EntityArchetype.obj
 0001:00022c00       ??$_M_find@PBD@?$_Rb_tree@PBDU?$less_stricmp@PBD@stl@@U?$pair@QBDV?$_smart_ptr@VCEntityArchetype@@@@@stlpmtx_std@@U?$_Select1st@U?$pair@QBDV?$_smart_ptr@VCEntityArchetype@@@@@stlpmtx_std@@@priv@4@U?$_MapTraitsT@U?$pair@QBDV?$_smart_ptr@VCEntityArchetype@@@@@stlpmtx_std@@@64@V?$allocator@U?$pair@QBDV?$_smart_ptr@VCEntityArchetype@@@@@stlpmtx_std@@@4@@priv@stlpmtx_std@@ABEPAU_Rb_tree_node_base@12@ABQBD@Z 32023c00 f i EntityArchetype.obj
 0001:00022c80       ?init@?$DynArray@V?$CryStringT@D@@HU?$SmallDynStorage@V?$CryStringT@D@@HUStandardAlloc@NAlloc@@@NArray@@@@KAPAV?$CryStringT@D@@U?$Array@V?$CryStringT@D@@HU?$ArrayStorage@V?$CryStringT@D@@H@NArray@@@@ABV2@@Z 32023c80 f i EntityArchetype.obj
 0001:00022cc0       ?set_size@?$SmallDynStorage@PAUIPhysicalEntity@@HUStandardAlloc@NAlloc@@@NArray@@QAEXH@Z 32023cc0 f i PhysicsProxy.obj
 0001:00022cc0       ?set_size@?$SmallDynStorage@V?$CryStringT@D@@HUStandardAlloc@NAlloc@@@NArray@@QAEXH@Z 32023cc0 f i EntityArchetype.obj
 0001:00022d40       ??$__find@PAV?$CryStringT@D@@V1@@priv@stlpmtx_std@@YAPAV?$CryStringT@D@@PAV2@0ABV2@ABUrandom_access_iterator_tag@1@@Z 32023d40 f i EntityArchetype.obj
 0001:00022f10       ??0CEntityArchetype@@QAE@PAUIEntityClass@@@Z 32023f10 f   EntityArchetype.obj
 0001:00022fb0       ??_ECEntityArchetype@@W3AEPAXI@Z 32023fb0 f i EntityArchetype.obj
 0001:00022fc0       ?destroy@?$DynArray@V?$CryStringT@D@@HU?$SmallDynStorage@V?$CryStringT@D@@HUStandardAlloc@NAlloc@@@NArray@@@@KAXU?$Array@V?$CryStringT@D@@HU?$ArrayStorage@V?$CryStringT@D@@H@NArray@@@@@Z 32023fc0 f i EntityArchetype.obj
 0001:00023010       ?_M_erase@?$_Rb_tree@PBDU?$less_stricmp@PBD@stl@@U?$pair@QBDV?$_smart_ptr@VCEntityArchetype@@@@@stlpmtx_std@@U?$_Select1st@U?$pair@QBDV?$_smart_ptr@VCEntityArchetype@@@@@stlpmtx_std@@@priv@4@U?$_MapTraitsT@U?$pair@QBDV?$_smart_ptr@VCEntityArchetype@@@@@stlpmtx_std@@@64@V?$allocator@U?$pair@QBDV?$_smart_ptr@VCEntityArchetype@@@@@stlpmtx_std@@@4@@priv@stlpmtx_std@@AAEXPAU_Rb_tree_node_base@23@@Z 32024010 f i EntityArchetype.obj
 0001:00023060       ?_M_create_node@?$_Rb_tree@PBDU?$less_stricmp@PBD@stl@@U?$pair@QBDV?$_smart_ptr@VCEntityArchetype@@@@@stlpmtx_std@@U?$_Select1st@U?$pair@QBDV?$_smart_ptr@VCEntityArchetype@@@@@stlpmtx_std@@@priv@4@U?$_MapTraitsT@U?$pair@QBDV?$_smart_ptr@VCEntityArchetype@@@@@stlpmtx_std@@@64@V?$allocator@U?$pair@QBDV?$_smart_ptr@VCEntityArchetype@@@@@stlpmtx_std@@@4@@priv@stlpmtx_std@@IAEPAU_Rb_tree_node_base@23@ABU?$pair@QBDV?$_smart_ptr@VCEntityArchetype@@@@@3@@Z 32024060 f i EntityArchetype.obj
 0001:000230c0       ??_GCEntityArchetype@@UAEPAXI@Z 320240c0 f i EntityArchetype.obj
 0001:000230c0       ??_ECEntityArchetype@@UAEPAXI@Z 320240c0 f i EntityArchetype.obj
 0001:00023130       ??$move_init@V?$CryStringT@D@@@NArray@@YAXPAV?$CryStringT@D@@0I@Z 32024130 f i EntityArchetype.obj
 0001:000231b0       ?_M_insert@?$_Rb_tree@PBDU?$less_stricmp@PBD@stl@@U?$pair@QBDV?$_smart_ptr@VCEntityArchetype@@@@@stlpmtx_std@@U?$_Select1st@U?$pair@QBDV?$_smart_ptr@VCEntityArchetype@@@@@stlpmtx_std@@@priv@4@U?$_MapTraitsT@U?$pair@QBDV?$_smart_ptr@VCEntityArchetype@@@@@stlpmtx_std@@@64@V?$allocator@U?$pair@QBDV?$_smart_ptr@VCEntityArchetype@@@@@stlpmtx_std@@@4@@priv@stlpmtx_std@@AAE?AU?$_Rb_tree_iterator@U?$pair@QBDV?$_smart_ptr@VCEntityArchetype@@@@@stlpmtx_std@@U?$_MapTraitsT@U?$pair@QBDV?$_smart_ptr@VCEntityArchetype@@@@@stlpmtx_std@@@priv@2@@23@PAU_Rb_tree_node_base@23@ABU?$pair@QBDV?$_smart_ptr@VCEntityArchetype@@@@@3@00@Z 320241b0 f i EntityArchetype.obj
 0001:00023250       ?insert_unique@?$_Rb_tree@PBDU?$less_stricmp@PBD@stl@@U?$pair@QBDV?$_smart_ptr@VCEntityArchetype@@@@@stlpmtx_std@@U?$_Select1st@U?$pair@QBDV?$_smart_ptr@VCEntityArchetype@@@@@stlpmtx_std@@@priv@4@U?$_MapTraitsT@U?$pair@QBDV?$_smart_ptr@VCEntityArchetype@@@@@stlpmtx_std@@@64@V?$allocator@U?$pair@QBDV?$_smart_ptr@VCEntityArchetype@@@@@stlpmtx_std@@@4@@priv@stlpmtx_std@@QAE?AU?$pair@U?$_Rb_tree_iterator@U?$pair@QBDV?$_smart_ptr@VCEntityArchetype@@@@@stlpmtx_std@@U?$_MapTraitsT@U?$pair@QBDV?$_smart_ptr@VCEntityArchetype@@@@@stlpmtx_std@@@priv@2@@priv@stlpmtx_std@@_N@3@ABU?$pair@QBDV?$_smart_ptr@VCEntityArchetype@@@@@3@@Z 32024250 f i EntityArchetype.obj
 0001:00023390       ?substr@?$CryStringT@D@@QBE?AV1@II@Z 32024390 f i EntityArchetype.obj
 0001:000233e0       ?FindArchetype@CEntityArchetypeManager@@QAEPAUIEntityArchetype@@PBD@Z 320243e0 f   EntityArchetype.obj
 0001:00023420       ?resize_raw@?$SmallDynStorage@V?$CryStringT@D@@HUStandardAlloc@NAlloc@@@NArray@@QAEXHH_N@Z 32024420 f i EntityArchetype.obj
 0001:00023570       ?insert_unique@?$_Rb_tree@PBDU?$less_stricmp@PBD@stl@@U?$pair@QBDV?$_smart_ptr@VCEntityArchetype@@@@@stlpmtx_std@@U?$_Select1st@U?$pair@QBDV?$_smart_ptr@VCEntityArchetype@@@@@stlpmtx_std@@@priv@4@U?$_MapTraitsT@U?$pair@QBDV?$_smart_ptr@VCEntityArchetype@@@@@stlpmtx_std@@@64@V?$allocator@U?$pair@QBDV?$_smart_ptr@VCEntityArchetype@@@@@stlpmtx_std@@@4@@priv@stlpmtx_std@@QAE?AU?$_Rb_tree_iterator@U?$pair@QBDV?$_smart_ptr@VCEntityArchetype@@@@@stlpmtx_std@@U?$_MapTraitsT@U?$pair@QBDV?$_smart_ptr@VCEntityArchetype@@@@@stlpmtx_std@@@priv@2@@23@U423@ABU?$pair@QBDV?$_smart_ptr@VCEntityArchetype@@@@@3@@Z 32024570 f i EntityArchetype.obj
 0001:00023800       ?RemoveExtension@PathUtil@@YAXAAV?$CryStringT@D@@@Z 32024800 f i EntityArchetype.obj
 0001:00023940       ??$?HD@@YA?AV?$CryStringT@D@@ABV0@0@Z 32024940 f i EntityArchetype.obj
 0001:00023980       ?expand_raw@?$DynArray@V?$CryStringT@D@@HU?$SmallDynStorage@V?$CryStringT@D@@HUStandardAlloc@NAlloc@@@NArray@@@@IAEPAV?$CryStringT@D@@PAV2@H@Z 32024980 f i EntityArchetype.obj
 0001:00023a00       ?AddSlash@PathUtil@@YA?AV?$CryStringT@D@@ABV2@@Z 32024a00 f i EntityArchetype.obj
 0001:00023aa0       ?Make@PathUtil@@YA?AV?$CryStringT@D@@ABV2@00@Z 32024aa0 f i EntityArchetype.obj
 0001:00023bd0       ?Reset@CEntityArchetypeManager@@QAEXXZ 32024bd0 f   EntityArchetype.obj
 0001:00023ce0       ?CreateArchetype@CEntityArchetypeManager@@QAEPAUIEntityArchetype@@PAUIEntityClass@@PBD@Z 32024ce0 f   EntityArchetype.obj
 0001:00023e60       ?LoadLibrary@CEntityArchetypeManager@@AAE_NABV?$CryStringT@D@@@Z 32024e60 f   EntityArchetype.obj
 0001:00024250       ?LoadArchetype@CEntityArchetypeManager@@QAEPAUIEntityArchetype@@PBD@Z 32025250 f   EntityArchetype.obj
 0001:00024410       ?DumpEntities@CVar@@SAXPAUIConsoleCmdArgs@@@Z 32025410 f   EntityCVars.obj
 0001:00024420       ?CompileAreaGrid@CVar@@SAXPAUIConsoleCmdArgs@@@Z 32025420 f   EntityCVars.obj
 0001:00024450       ?DumpEntityBookmarks@CVar@@SAXPAUIConsoleCmdArgs@@@Z 32025450 f   EntityCVars.obj
 0001:000244f0       ?EnableDebugAnimText@CVar@@SAXPAUIConsoleCmdArgs@@@Z 320254f0 f   EntityCVars.obj
 0001:00024660       ??R?$less@V?$CryStringT@D@@@stlpmtx_std@@QBE_NABV?$CryStringT@D@@0@Z 32025660 f i EntityCVars.obj
 0001:000246b0       ??$_M_lower_bound@PBD@?$_Rb_tree@V?$CryStringT@D@@U?$less@V?$CryStringT@D@@@stlpmtx_std@@U?$pair@$$CBV?$CryStringT@D@@PAVCEntityLayer@@@3@U?$_Select1st@U?$pair@$$CBV?$CryStringT@D@@PAVCEntityLayer@@@stlpmtx_std@@@priv@3@U?$_MapTraitsT@U?$pair@$$CBV?$CryStringT@D@@PAVCEntityLayer@@@stlpmtx_std@@@63@V?$allocator@U?$pair@$$CBV?$CryStringT@D@@PAVCEntityLayer@@@stlpmtx_std@@@3@@priv@stlpmtx_std@@ABEPAU_Rb_tree_node_base@12@ABQBD@Z 320256b0 f i EntitySystem.obj
 0001:000246b0       ??$_M_lower_bound@PBD@?$_Rb_tree@V?$CryStringT@D@@U?$less@V?$CryStringT@D@@@stlpmtx_std@@U?$pair@$$CBV?$CryStringT@D@@H@3@U?$_Select1st@U?$pair@$$CBV?$CryStringT@D@@H@stlpmtx_std@@@priv@3@U?$_MapTraitsT@U?$pair@$$CBV?$CryStringT@D@@H@stlpmtx_std@@@63@V?$allocator@U?$pair@$$CBV?$CryStringT@D@@H@stlpmtx_std@@@3@@priv@stlpmtx_std@@ABEPAU_Rb_tree_node_base@12@ABQBD@Z 320256b0 f i EntityCVars.obj
 0001:000246b0       ??$_M_lower_bound@PBD@?$_Rb_tree@V?$CryStringT@D@@U?$less@V?$CryStringT@D@@@stlpmtx_std@@U?$pair@$$CBV?$CryStringT@D@@PAUIEntityClass@@@3@U?$_Select1st@U?$pair@$$CBV?$CryStringT@D@@PAUIEntityClass@@@stlpmtx_std@@@priv@3@U?$_MapTraitsT@U?$pair@$$CBV?$CryStringT@D@@PAUIEntityClass@@@stlpmtx_std@@@63@V?$allocator@U?$pair@$$CBV?$CryStringT@D@@PAUIEntityClass@@@stlpmtx_std@@@3@@priv@stlpmtx_std@@ABEPAU_Rb_tree_node_base@12@ABQBD@Z 320256b0 f i EntityClassRegistry.obj
 0001:000247b0       ?insert_unique@?$_Rb_tree@V?$CryStringT@D@@U?$less@V?$CryStringT@D@@@stlpmtx_std@@U?$pair@$$CBV?$CryStringT@D@@PAVCEntityLayer@@@3@U?$_Select1st@U?$pair@$$CBV?$CryStringT@D@@PAVCEntityLayer@@@stlpmtx_std@@@priv@3@U?$_MapTraitsT@U?$pair@$$CBV?$CryStringT@D@@PAVCEntityLayer@@@stlpmtx_std@@@63@V?$allocator@U?$pair@$$CBV?$CryStringT@D@@PAVCEntityLayer@@@stlpmtx_std@@@3@@priv@stlpmtx_std@@QAE?AU?$_Rb_tree_iterator@U?$pair@$$CBV?$CryStringT@D@@PAVCEntityLayer@@@stlpmtx_std@@U?$_MapTraitsT@U?$pair@$$CBV?$CryStringT@D@@PAVCEntityLayer@@@stlpmtx_std@@@priv@2@@23@U423@ABU?$pair@$$CBV?$CryStringT@D@@PAVCEntityLayer@@@3@@Z 320257b0 f i EntitySystem.obj
 0001:000247b0       ?insert_unique@?$_Rb_tree@V?$CryStringT@D@@U?$less@V?$CryStringT@D@@@stlpmtx_std@@U?$pair@$$CBV?$CryStringT@D@@PAUIEntityClass@@@3@U?$_Select1st@U?$pair@$$CBV?$CryStringT@D@@PAUIEntityClass@@@stlpmtx_std@@@priv@3@U?$_MapTraitsT@U?$pair@$$CBV?$CryStringT@D@@PAUIEntityClass@@@stlpmtx_std@@@63@V?$allocator@U?$pair@$$CBV?$CryStringT@D@@PAUIEntityClass@@@stlpmtx_std@@@3@@priv@stlpmtx_std@@QAE?AU?$_Rb_tree_iterator@U?$pair@$$CBV?$CryStringT@D@@PAUIEntityClass@@@stlpmtx_std@@U?$_MapTraitsT@U?$pair@$$CBV?$CryStringT@D@@PAUIEntityClass@@@stlpmtx_std@@@priv@2@@23@U423@ABU?$pair@$$CBV?$CryStringT@D@@PAUIEntityClass@@@3@@Z 320257b0 f i EntityClassRegistry.obj
 0001:000247b0       ?insert_unique@?$_Rb_tree@V?$CryStringT@D@@U?$less@V?$CryStringT@D@@@stlpmtx_std@@U?$pair@$$CBV?$CryStringT@D@@H@3@U?$_Select1st@U?$pair@$$CBV?$CryStringT@D@@H@stlpmtx_std@@@priv@3@U?$_MapTraitsT@U?$pair@$$CBV?$CryStringT@D@@H@stlpmtx_std@@@63@V?$allocator@U?$pair@$$CBV?$CryStringT@D@@H@stlpmtx_std@@@3@@priv@stlpmtx_std@@QAE?AU?$_Rb_tree_iterator@U?$pair@$$CBV?$CryStringT@D@@H@stlpmtx_std@@U?$_MapTraitsT@U?$pair@$$CBV?$CryStringT@D@@H@stlpmtx_std@@@priv@2@@23@U423@ABU?$pair@$$CBV?$CryStringT@D@@H@3@@Z 320257b0 f i EntityCVars.obj
 0001:00024a80       ??$?APBD@?$map@V?$CryStringT@D@@PAUIEntityClass@@U?$less@V?$CryStringT@D@@@stlpmtx_std@@V?$allocator@U?$pair@$$CBV?$CryStringT@D@@PAUIEntityClass@@@stlpmtx_std@@@4@@stlpmtx_std@@QAEAAPAUIEntityClass@@ABQBD@Z 32025a80 f i EntityClassRegistry.obj
 0001:00024a80       ??$?APBD@?$map@V?$CryStringT@D@@HU?$less@V?$CryStringT@D@@@stlpmtx_std@@V?$allocator@U?$pair@$$CBV?$CryStringT@D@@H@stlpmtx_std@@@3@@stlpmtx_std@@QAEAAHABQBD@Z 32025a80 f i EntityCVars.obj
 0001:00024a80       ??$?APBD@?$map@V?$CryStringT@D@@PAVCEntityLayer@@U?$less@V?$CryStringT@D@@@stlpmtx_std@@V?$allocator@U?$pair@$$CBV?$CryStringT@D@@PAVCEntityLayer@@@stlpmtx_std@@@4@@stlpmtx_std@@QAEAAPAVCEntityLayer@@ABQBD@Z 32025a80 f i EntitySystem.obj
 0001:00024be0       ?DumpEntityClassesInUse@CVar@@SAXPAUIConsoleCmdArgs@@@Z 32025be0 f   EntityCVars.obj
 0001:00024da0       ?Init@CVar@@SAXPAUIConsole@@@Z 32025da0 f   EntityCVars.obj
 0001:00025950       ??_GIEntityEventDistributer@@UAEPAXI@Z 32026950 f i EntityEventDistributer.obj
 0001:00025950       ??_EIEntityEventDistributer@@UAEPAXI@Z 32026950 f i EntityEventDistributer.obj
 0001:00025980       ??RFEntityEventSort@?A0xcc9d3949@@QBE_NABUSEventPtr@CEntityEventDistributer@@0@Z 32026980 f i EntityEventDistributer.obj
 0001:000259f0       ??$__median@USEventPtr@CEntityEventDistributer@@UFEntityEventSort@?A0xcc9d3949@@@priv@stlpmtx_std@@YAABUSEventPtr@CEntityEventDistributer@@ABU23@00UFEntityEventSort@?A0xcc9d3949@@@Z 320269f0 f i EntityEventDistributer.obj
 0001:00025aa0       ??$__find@PAUSEventPtr@CEntityEventDistributer@@U12@@priv@stlpmtx_std@@YAPAUSEventPtr@CEntityEventDistributer@@PAU23@0ABU23@ABUrandom_access_iterator_tag@1@@Z 32026aa0 f i EntityEventDistributer.obj
 0001:00025b50       ??$__unguarded_linear_insert@PAUSEventPtr@CEntityEventDistributer@@U12@UFEntityEventSortByEntityFirst@?A0xcc9d3949@@@priv@stlpmtx_std@@YAXPAUSEventPtr@CEntityEventDistributer@@U23@UFEntityEventSortByEntityFirst@?A0xcc9d3949@@@Z 32026b50 f i EntityEventDistributer.obj
 0001:00025bd0       ??$__unguarded_linear_insert@PAUSEventPtr@CEntityEventDistributer@@U12@UFEntityEventSort@?A0xcc9d3949@@@priv@stlpmtx_std@@YAXPAUSEventPtr@CEntityEventDistributer@@U23@UFEntityEventSort@?A0xcc9d3949@@@Z 32026bd0 f i EntityEventDistributer.obj
 0001:00025c50       ??$__push_heap@PAUSEventPtr@CEntityEventDistributer@@HU12@UFEntityEventSortByEntityFirst@?A0xcc9d3949@@@stlpmtx_std@@YAXPAUSEventPtr@CEntityEventDistributer@@HHU12@UFEntityEventSortByEntityFirst@?A0xcc9d3949@@@Z 32026c50 f i EntityEventDistributer.obj
 0001:00025d10       ??$__push_heap@PAUSEventPtr@CEntityEventDistributer@@HU12@UFEntityEventSort@?A0xcc9d3949@@@stlpmtx_std@@YAXPAUSEventPtr@CEntityEventDistributer@@HHU12@UFEntityEventSort@?A0xcc9d3949@@@Z 32026d10 f i EntityEventDistributer.obj
 0001:00025dd0       ??$__unguarded_insertion_sort_aux@PAUSEventPtr@CEntityEventDistributer@@U12@UFEntityEventSortByEntityFirst@?A0xcc9d3949@@@priv@stlpmtx_std@@YAXPAUSEventPtr@CEntityEventDistributer@@00UFEntityEventSortByEntityFirst@?A0xcc9d3949@@@Z 32026dd0 f i EntityEventDistributer.obj
 0001:00025e70       ??$__unguarded_insertion_sort_aux@PAUSEventPtr@CEntityEventDistributer@@U12@UFEntityEventSort@?A0xcc9d3949@@@priv@stlpmtx_std@@YAXPAUSEventPtr@CEntityEventDistributer@@00UFEntityEventSort@?A0xcc9d3949@@@Z 32026e70 f i EntityEventDistributer.obj
 0001:00025f10       ??$__adjust_heap@PAUSEventPtr@CEntityEventDistributer@@HU12@UFEntityEventSortByEntityFirst@?A0xcc9d3949@@@stlpmtx_std@@YAXPAUSEventPtr@CEntityEventDistributer@@HHU12@UFEntityEventSortByEntityFirst@?A0xcc9d3949@@@Z 32026f10 f i EntityEventDistributer.obj
 0001:00025fe0       ??$__adjust_heap@PAUSEventPtr@CEntityEventDistributer@@HU12@UFEntityEventSort@?A0xcc9d3949@@@stlpmtx_std@@YAXPAUSEventPtr@CEntityEventDistributer@@HHU12@UFEntityEventSort@?A0xcc9d3949@@@Z 32026fe0 f i EntityEventDistributer.obj
 0001:000260b0       ??$__make_heap@PAUSEventPtr@CEntityEventDistributer@@UFEntityEventSortByEntityFirst@?A0xcc9d3949@@U12@H@stlpmtx_std@@YAXPAUSEventPtr@CEntityEventDistributer@@0UFEntityEventSortByEntityFirst@?A0xcc9d3949@@0PAH@Z 320270b0 f i EntityEventDistributer.obj
 0001:000261d0       ??$__make_heap@PAUSEventPtr@CEntityEventDistributer@@UFEntityEventSort@?A0xcc9d3949@@U12@H@stlpmtx_std@@YAXPAUSEventPtr@CEntityEventDistributer@@0UFEntityEventSort@?A0xcc9d3949@@0PAH@Z 320271d0 f i EntityEventDistributer.obj
 0001:000262f0       ??$_M_allocate_and_copy@PAM@?$_Impl_vector@MV?$allocator@M@stlpmtx_std@@@priv@stlpmtx_std@@AAEPAMAAIPAM1@Z 320272f0 f i ScriptBind_Entity.obj
 0001:000262f0       ??$_M_allocate_and_copy@PBQAX@?$_Impl_vector@PAXV?$allocator@PAX@stlpmtx_std@@@priv@stlpmtx_std@@AAEPAPAXAAIPBQAX1@Z 320272f0 f i EntitySystem.obj
 0001:000262f0       ??$_M_allocate_and_copy@PAH@?$_Impl_vector@HV?$allocator@H@stlpmtx_std@@@priv@stlpmtx_std@@AAEPAHAAIPAH1@Z 320272f0 f i AreaManager.obj
 0001:000262f0       ??$_M_allocate_and_copy@PAPAX@?$_Impl_vector@PAXV?$allocator@PAX@stlpmtx_std@@@priv@stlpmtx_std@@AAEPAPAXAAIPAPAX1@Z 320272f0 f i EntityEventDistributer.obj
 0001:00026360       ??$_M_find@W4EEntityEvent@@@?$hashtable@U?$pair@$$CBHUSEventPtrs@CEntityEventDistributer@@@stlpmtx_std@@HU?$hash@H@2@U?$_HashMapTraitsT@U?$pair@$$CBHUSEventPtrs@CEntityEventDistributer@@@stlpmtx_std@@@priv@2@U?$_Select1st@U?$pair@$$CBHUSEventPtrs@CEntityEventDistributer@@@stlpmtx_std@@@52@U?$equal_to@H@2@V?$allocator@U?$pair@$$CBHUSEventPtrs@CEntityEventDistributer@@@stlpmtx_std@@@2@@stlpmtx_std@@ABE?AV?$_Slist_iterator@U?$pair@$$CBHUSEventPtrs@CEntityEventDistributer@@@stlpmtx_std@@U?$_Nonconst_traits@U?$pair@$$CBHUSEventPtrs@CEntityEventDistributer@@@stlpmtx_std@@@2@@priv@1@ABW4EEntityEvent@@@Z 32027360 f i EntityEventDistributer.obj
 0001:00026360       ??$_M_find@H@?$hashtable@U?$pair@$$CBHUSEventPtrs@CEntityEventDistributer@@@stlpmtx_std@@HU?$hash@H@2@U?$_HashMapTraitsT@U?$pair@$$CBHUSEventPtrs@CEntityEventDistributer@@@stlpmtx_std@@@priv@2@U?$_Select1st@U?$pair@$$CBHUSEventPtrs@CEntityEventDistributer@@@stlpmtx_std@@@52@U?$equal_to@H@2@V?$allocator@U?$pair@$$CBHUSEventPtrs@CEntityEventDistributer@@@stlpmtx_std@@@2@@stlpmtx_std@@ABE?AV?$_Slist_iterator@U?$pair@$$CBHUSEventPtrs@CEntityEventDistributer@@@stlpmtx_std@@U?$_Nonconst_traits@U?$pair@$$CBHUSEventPtrs@CEntityEventDistributer@@@stlpmtx_std@@@2@@priv@1@ABH@Z 32027360 f i EntityEventDistributer.obj
 0001:00026360       ??$_M_find@I@?$hashtable@U?$pair@$$CBIUEntityProp@CEntityLayer@@@stlpmtx_std@@IU?$hash@I@2@U?$_UnorderedMapTraitsT@U?$pair@$$CBIUEntityProp@CEntityLayer@@@stlpmtx_std@@@priv@2@U?$_Select1st@U?$pair@$$CBIUEntityProp@CEntityLayer@@@stlpmtx_std@@@52@U?$equal_to@I@2@V?$allocator@U?$pair@$$CBIUEntityProp@CEntityLayer@@@stlpmtx_std@@@2@@stlpmtx_std@@ABE?AV?$_Slist_iterator@U?$pair@$$CBIUEntityProp@CEntityLayer@@@stlpmtx_std@@U?$_Nonconst_traits@U?$pair@$$CBIUEntityProp@CEntityLayer@@@stlpmtx_std@@@2@@priv@1@ABI@Z 32027360 f i EntityLayer.obj
 0001:000263c0       ??$__unguarded_partition@PAUSEventPtr@CEntityEventDistributer@@U12@UFEntityEventSortByEntityFirst@?A0xcc9d3949@@@priv@stlpmtx_std@@YAPAUSEventPtr@CEntityEventDistributer@@PAU23@0U23@UFEntityEventSortByEntityFirst@?A0xcc9d3949@@@Z 320273c0 f i EntityEventDistributer.obj
 0001:00026490       ??$__unguarded_partition@PAUSEventPtr@CEntityEventDistributer@@U12@UFEntityEventSort@?A0xcc9d3949@@@priv@stlpmtx_std@@YAPAUSEventPtr@CEntityEventDistributer@@PAU23@0U23@UFEntityEventSort@?A0xcc9d3949@@@Z 32027490 f i EntityEventDistributer.obj
 0001:00026550       ??0?$_Vector_base@UListenerRecord@?$CListenerSet@PAUIEntityPoolListener@@@@V?$allocator@UListenerRecord@?$CListenerSet@PAUIEntityPoolListener@@@@@stlpmtx_std@@@priv@stlpmtx_std@@QAE@IABV?$allocator@UListenerRecord@?$CListenerSet@PAUIEntityPoolListener@@@@@2@@Z 32027550 f i EntityPoolManager.obj
 0001:00026550       ??0?$_Vector_base@U?$pair@II@stlpmtx_std@@V?$allocator@U?$pair@II@stlpmtx_std@@@2@@priv@stlpmtx_std@@QAE@IABV?$allocator@U?$pair@II@stlpmtx_std@@@2@@Z 32027550 f i EntitySystem.obj
 0001:00026550       ??0?$_Vector_base@USAreaCacheEntry@CAreaManager@@V?$allocator@USAreaCacheEntry@CAreaManager@@@stlpmtx_std@@@priv@stlpmtx_std@@QAE@IABV?$allocator@USAreaCacheEntry@CAreaManager@@@2@@Z 32027550 f i AreaManager.obj
 0001:00026550       ??0?$_Vector_base@USEventPtr@CEntityEventDistributer@@V?$allocator@USEventPtr@CEntityEventDistributer@@@stlpmtx_std@@@priv@stlpmtx_std@@QAE@IABV?$allocator@USEventPtr@CEntityEventDistributer@@@2@@Z 32027550 f i EntityEventDistributer.obj
 0001:00026600       ??$__insertion_sort@PAUSEventPtr@CEntityEventDistributer@@U12@UFEntityEventSortByEntityFirst@?A0xcc9d3949@@@priv@stlpmtx_std@@YAXPAUSEventPtr@CEntityEventDistributer@@00UFEntityEventSortByEntityFirst@?A0xcc9d3949@@@Z 32027600 f i EntityEventDistributer.obj
 0001:000266c0       ??$__insertion_sort@PAUSEventPtr@CEntityEventDistributer@@U12@UFEntityEventSort@?A0xcc9d3949@@@priv@stlpmtx_std@@YAXPAUSEventPtr@CEntityEventDistributer@@00UFEntityEventSort@?A0xcc9d3949@@@Z 320276c0 f i EntityEventDistributer.obj
 0001:00026780       ??$sort_heap@PAUSEventPtr@CEntityEventDistributer@@UFEntityEventSortByEntityFirst@?A0xcc9d3949@@@stlpmtx_std@@YAXPAUSEventPtr@CEntityEventDistributer@@0UFEntityEventSortByEntityFirst@?A0xcc9d3949@@@Z 32027780 f i EntityEventDistributer.obj
 0001:000267e0       ??$sort_heap@PAUSEventPtr@CEntityEventDistributer@@UFEntityEventSort@?A0xcc9d3949@@@stlpmtx_std@@YAXPAUSEventPtr@CEntityEventDistributer@@0UFEntityEventSort@?A0xcc9d3949@@@Z 320277e0 f i EntityEventDistributer.obj
 0001:00026840       ?ErasePtr@CEntityEventDistributer@@AAEXAAV?$vector@USEventPtr@CEntityEventDistributer@@V?$allocator@USEventPtr@CEntityEventDistributer@@@stlpmtx_std@@@stlpmtx_std@@PAUIEntityEvent@@@Z 32027840 f   EntityEventDistributer.obj
 0001:00026900       ?_M_fill_assign@?$_Impl_vector@PAXV?$allocator@PAX@stlpmtx_std@@@priv@stlpmtx_std@@QAEXIABQAX@Z 32027900 f i EntityEventDistributer.obj
 0001:00026a70       ??$__partial_sort@PAUSEventPtr@CEntityEventDistributer@@U12@UFEntityEventSortByEntityFirst@?A0xcc9d3949@@@priv@stlpmtx_std@@YAXPAUSEventPtr@CEntityEventDistributer@@000UFEntityEventSortByEntityFirst@?A0xcc9d3949@@@Z 32027a70 f i EntityEventDistributer.obj
 0001:00026b30       ??$__partial_sort@PAUSEventPtr@CEntityEventDistributer@@U12@UFEntityEventSort@?A0xcc9d3949@@@priv@stlpmtx_std@@YAXPAUSEventPtr@CEntityEventDistributer@@000UFEntityEventSort@?A0xcc9d3949@@@Z 32027b30 f i EntityEventDistributer.obj
 0001:00026bf0       ?SetFlags@CEntityEventDistributer@@QAEXH@Z 32027bf0 f   EntityEventDistributer.obj
 0001:00026c20       ??0SEventPtrs@CEntityEventDistributer@@QAE@ABU01@@Z 32027c20 f i EntityEventDistributer.obj
 0001:00026c90       ?_M_erase_after@?$_Slist_base@U?$pair@$$CBHUSEventPtrs@CEntityEventDistributer@@@stlpmtx_std@@V?$allocator@U?$pair@$$CBHUSEventPtrs@CEntityEventDistributer@@@stlpmtx_std@@@2@@priv@stlpmtx_std@@IAEPAU_Slist_node_base@23@PAU423@0@Z 32027c90 f i EntityEventDistributer.obj
 0001:00026d50       ??$__introsort_loop@PAUSEventPtr@CEntityEventDistributer@@U12@HUFEntityEventSortByEntityFirst@?A0xcc9d3949@@@priv@stlpmtx_std@@YAXPAUSEventPtr@CEntityEventDistributer@@00HUFEntityEventSortByEntityFirst@?A0xcc9d3949@@@Z 32027d50 f i EntityEventDistributer.obj
 0001:00026f90       ??$__introsort_loop@PAUSEventPtr@CEntityEventDistributer@@U12@HUFEntityEventSort@?A0xcc9d3949@@@priv@stlpmtx_std@@YAXPAUSEventPtr@CEntityEventDistributer@@00HUFEntityEventSort@?A0xcc9d3949@@@Z 32027f90 f i EntityEventDistributer.obj
 0001:00027030       ??$sort@PAUSEventPtr@CEntityEventDistributer@@UFEntityEventSortByEntityFirst@?A0xcc9d3949@@@stlpmtx_std@@YAXPAUSEventPtr@CEntityEventDistributer@@0UFEntityEventSortByEntityFirst@?A0xcc9d3949@@@Z 32028030 f i EntityEventDistributer.obj
 0001:000270b0       ??$sort@PAUSEventPtr@CEntityEventDistributer@@UFEntityEventSort@?A0xcc9d3949@@@stlpmtx_std@@YAXPAUSEventPtr@CEntityEventDistributer@@0UFEntityEventSort@?A0xcc9d3949@@@Z 320280b0 f i EntityEventDistributer.obj
 0001:00027130       ?SendEvent@CEntityEventDistributer@@EAEXABUSEntityEvent@@@Z 32028130 f   EntityEventDistributer.obj
 0001:000271e0       ??0?$hashtable@U?$pair@$$CBHUSEventPtrs@CEntityEventDistributer@@@stlpmtx_std@@HU?$hash@H@2@U?$_HashMapTraitsT@U?$pair@$$CBHUSEventPtrs@CEntityEventDistributer@@@stlpmtx_std@@@priv@2@U?$_Select1st@U?$pair@$$CBHUSEventPtrs@CEntityEventDistributer@@@stlpmtx_std@@@52@U?$equal_to@H@2@V?$allocator@U?$pair@$$CBHUSEventPtrs@CEntityEventDistributer@@@stlpmtx_std@@@2@@stlpmtx_std@@QAE@IABU?$hash@H@1@ABU?$equal_to@H@1@ABV?$allocator@U?$pair@$$CBHUSEventPtrs@CEntityEventDistributer@@@stlpmtx_std@@@1@@Z 320281e0 f i EntityEventDistributer.obj
 0001:000271e0       ??0?$hashtable@U?$pair@$$CBIUEntityProp@CEntityLayer@@@stlpmtx_std@@IU?$hash@I@2@U?$_UnorderedMapTraitsT@U?$pair@$$CBIUEntityProp@CEntityLayer@@@stlpmtx_std@@@priv@2@U?$_Select1st@U?$pair@$$CBIUEntityProp@CEntityLayer@@@stlpmtx_std@@@52@U?$equal_to@I@2@V?$allocator@U?$pair@$$CBIUEntityProp@CEntityLayer@@@stlpmtx_std@@@2@@stlpmtx_std@@QAE@IABU?$hash@I@1@ABU?$equal_to@I@1@ABV?$allocator@U?$pair@$$CBIUEntityProp@CEntityLayer@@@stlpmtx_std@@@1@@Z 320281e0 f i EntityLayer.obj
 0001:00027280       ??1?$hashtable@U?$pair@$$CBHUSEventPtrs@CEntityEventDistributer@@@stlpmtx_std@@HU?$hash@H@2@U?$_HashMapTraitsT@U?$pair@$$CBHUSEventPtrs@CEntityEventDistributer@@@stlpmtx_std@@@priv@2@U?$_Select1st@U?$pair@$$CBHUSEventPtrs@CEntityEventDistributer@@@stlpmtx_std@@@52@U?$equal_to@H@2@V?$allocator@U?$pair@$$CBHUSEventPtrs@CEntityEventDistributer@@@stlpmtx_std@@@2@@stlpmtx_std@@QAE@XZ 32028280 f i EntityEventDistributer.obj
 0001:000272f0       ??0CEntityEventDistributer@@QAE@H@Z 320282f0 f   EntityEventDistributer.obj
 0001:00027370       ??_GCEntityEventDistributer@@UAEPAXI@Z 32028370 f i EntityEventDistributer.obj
 0001:00027370       ??_ECEntityEventDistributer@@UAEPAXI@Z 32028370 f i EntityEventDistributer.obj
 0001:000273d0       ?_M_insert_noresize@?$hashtable@U?$pair@$$CBHUSEventPtrs@CEntityEventDistributer@@@stlpmtx_std@@HU?$hash@H@2@U?$_HashMapTraitsT@U?$pair@$$CBHUSEventPtrs@CEntityEventDistributer@@@stlpmtx_std@@@priv@2@U?$_Select1st@U?$pair@$$CBHUSEventPtrs@CEntityEventDistributer@@@stlpmtx_std@@@52@U?$equal_to@H@2@V?$allocator@U?$pair@$$CBHUSEventPtrs@CEntityEventDistributer@@@stlpmtx_std@@@2@@stlpmtx_std@@IAE?AU?$_Ht_iterator@V?$_Slist_iterator@U?$pair@$$CBHUSEventPtrs@CEntityEventDistributer@@@stlpmtx_std@@U?$_Nonconst_traits@U?$pair@$$CBHUSEventPtrs@CEntityEventDistributer@@@stlpmtx_std@@@2@@priv@stlpmtx_std@@U?$_NonLocalHashMapTraitsT@U?$pair@$$CBHUSEventPtrs@CEntityEventDistributer@@@stlpmtx_std@@@23@@priv@2@IABU?$pair@$$CBHUSEventPtrs@CEntityEventDistributer@@@2@@Z 320283d0 f i EntityEventDistributer.obj
 0001:000274a0       ?insert_unique_noresize@?$hashtable@U?$pair@$$CBHUSEventPtrs@CEntityEventDistributer@@@stlpmtx_std@@HU?$hash@H@2@U?$_HashMapTraitsT@U?$pair@$$CBHUSEventPtrs@CEntityEventDistributer@@@stlpmtx_std@@@priv@2@U?$_Select1st@U?$pair@$$CBHUSEventPtrs@CEntityEventDistributer@@@stlpmtx_std@@@52@U?$equal_to@H@2@V?$allocator@U?$pair@$$CBHUSEventPtrs@CEntityEventDistributer@@@stlpmtx_std@@@2@@stlpmtx_std@@QAE?AU?$pair@U?$_Ht_iterator@V?$_Slist_iterator@U?$pair@$$CBHUSEventPtrs@CEntityEventDistributer@@@stlpmtx_std@@U?$_Nonconst_traits@U?$pair@$$CBHUSEventPtrs@CEntityEventDistributer@@@stlpmtx_std@@@2@@priv@stlpmtx_std@@U?$_NonLocalHashMapTraitsT@U?$pair@$$CBHUSEventPtrs@CEntityEventDistributer@@@stlpmtx_std@@@23@@priv@stlpmtx_std@@_N@2@ABU?$pair@$$CBHUSEventPtrs@CEntityEventDistributer@@@2@@Z 320284a0 f i EntityEventDistributer.obj
 0001:00027570       ?_M_rehash@?$hashtable@U?$pair@$$CBHUSEventPtrs@CEntityEventDistributer@@@stlpmtx_std@@HU?$hash@H@2@U?$_HashMapTraitsT@U?$pair@$$CBHUSEventPtrs@CEntityEventDistributer@@@stlpmtx_std@@@priv@2@U?$_Select1st@U?$pair@$$CBHUSEventPtrs@CEntityEventDistributer@@@stlpmtx_std@@@52@U?$equal_to@H@2@V?$allocator@U?$pair@$$CBHUSEventPtrs@CEntityEventDistributer@@@stlpmtx_std@@@2@@stlpmtx_std@@AAEXI@Z 32028570 f i EntityEventDistributer.obj
 0001:000277e0       ?_M_enlarge@?$hashtable@U?$pair@$$CBHUSEventPtrs@CEntityEventDistributer@@@stlpmtx_std@@HU?$hash@H@2@U?$_HashMapTraitsT@U?$pair@$$CBHUSEventPtrs@CEntityEventDistributer@@@stlpmtx_std@@@priv@2@U?$_Select1st@U?$pair@$$CBHUSEventPtrs@CEntityEventDistributer@@@stlpmtx_std@@@52@U?$equal_to@H@2@V?$allocator@U?$pair@$$CBHUSEventPtrs@CEntityEventDistributer@@@stlpmtx_std@@@2@@stlpmtx_std@@AAEXI@Z 320287e0 f i EntityEventDistributer.obj
 0001:00027880       ?_M_reduce@?$hashtable@U?$pair@$$CBHUSEventPtrs@CEntityEventDistributer@@@stlpmtx_std@@HU?$hash@H@2@U?$_HashMapTraitsT@U?$pair@$$CBHUSEventPtrs@CEntityEventDistributer@@@stlpmtx_std@@@priv@2@U?$_Select1st@U?$pair@$$CBHUSEventPtrs@CEntityEventDistributer@@@stlpmtx_std@@@52@U?$equal_to@H@2@V?$allocator@U?$pair@$$CBHUSEventPtrs@CEntityEventDistributer@@@stlpmtx_std@@@2@@stlpmtx_std@@AAEXXZ 32028880 f i EntityEventDistributer.obj
 0001:00027990       ?erase@?$hashtable@U?$pair@$$CBHUSEventPtrs@CEntityEventDistributer@@@stlpmtx_std@@HU?$hash@H@2@U?$_HashMapTraitsT@U?$pair@$$CBHUSEventPtrs@CEntityEventDistributer@@@stlpmtx_std@@@priv@2@U?$_Select1st@U?$pair@$$CBHUSEventPtrs@CEntityEventDistributer@@@stlpmtx_std@@@52@U?$equal_to@H@2@V?$allocator@U?$pair@$$CBHUSEventPtrs@CEntityEventDistributer@@@stlpmtx_std@@@2@@stlpmtx_std@@QAEXU?$_Ht_iterator@V?$_Slist_iterator@U?$pair@$$CBHUSEventPtrs@CEntityEventDistributer@@@stlpmtx_std@@U?$_Nonconst_traits@U?$pair@$$CBHUSEventPtrs@CEntityEventDistributer@@@stlpmtx_std@@@2@@priv@stlpmtx_std@@U?$_ConstNonLocalHashMapTraitsT@U?$pair@$$CBHUSEventPtrs@CEntityEventDistributer@@@stlpmtx_std@@@23@@priv@2@@Z 32028990 f i EntityEventDistributer.obj
 0001:00027af0       ?RegisterEvent@CEntityEventDistributer@@EAEXIPAUIEntityEvent@@H@Z 32028af0 f   EntityEventDistributer.obj
 0001:00027c20       ?UnRegisterEvent@CEntityEventDistributer@@EAEXPAUIEntityEvent@@H@Z 32028c20 f   EntityEventDistributer.obj
 0001:00027c80       ?RegisterEvents@CEntityEventDistributer@@EAEXIPAUIEntityEvent@@PBHH@Z 32028c80 f   EntityEventDistributer.obj
 0001:00027ed0       ?UnRegisterEvents@CEntityEventDistributer@@EAEXPAUIEntityEvent@@PBHH@Z 32028ed0 f   EntityEventDistributer.obj
 0001:00028000       ?UnRegisterAllEvents@CEntityEventDistributer@@EAEXPAUIEntityEvent@@@Z 32029000 f   EntityEventDistributer.obj
 0001:00028050       ?RegisterToEvents@CEntityEventDistributer@@EAEXIPAUIEntityEvent@@PBHH@Z 32029050 f   EntityEventDistributer.obj
 0001:00028090       ?IsSkippedBySpec@CEntityLayer@@QBE_NXZ 32029090 f   EntityLayer.obj
 0001:000280e0       ??$fill@PAUSLayerProfile@CEntitySystem@@U12@@stlpmtx_std@@YAXPAUSLayerProfile@CEntitySystem@@0ABU12@@Z 320290e0 f i EntityLayer.obj
 0001:00028120       ??$__uninitialized_fill_n@PAUSLayerProfile@CEntitySystem@@IU12@@priv@stlpmtx_std@@YAPAUSLayerProfile@CEntitySystem@@PAU23@IABU23@@Z 32029120 f i EntityLayer.obj
 0001:00028180       ?SetSharedSerializeString@?$CSerializeWrapper@UISerialize@@@@QAEAAUSSerializeString@@ABV?$CryStringT@D@@@Z 32029180 f i EntityLayer.obj
 0001:000281e0       ?_M_insert_overflow@?$_Impl_vector@USLayerProfile@CEntitySystem@@V?$allocator@USLayerProfile@CEntitySystem@@@stlpmtx_std@@@priv@stlpmtx_std@@AAEXPAUSLayerProfile@CEntitySystem@@ABU45@ABU__true_type@3@I_N@Z 320291e0 f i EntityLayer.obj
 0001:00028350       ?_M_fill_insert_aux@?$_Impl_vector@USLayerProfile@CEntitySystem@@V?$allocator@USLayerProfile@CEntitySystem@@@stlpmtx_std@@@priv@stlpmtx_std@@AAEXPAUSLayerProfile@CEntitySystem@@IABU45@ABU__false_type@3@@Z 32029350 f i EntityLayer.obj
 0001:00028460       ?EnableEntities@CEntityLayer@@AAEX_N@Z 32029460 f   EntityLayer.obj
 0001:000287b0       ?GetMemoryUsage@CEntityLayer@@QAEXPAVICrySizer@@PAH@Z 320297b0 f   EntityLayer.obj
 0001:00028810       ?Value@?$CSerializeWrapper@UISerialize@@@@QAEXPBDAAV?$CryStringT@D@@H@Z 32029810 f i EntityLayer.obj
 0001:000288c0       ?_M_insert_noresize@?$hashtable@U?$pair@$$CBIUEntityProp@CEntityLayer@@@stlpmtx_std@@IU?$hash@I@2@U?$_UnorderedMapTraitsT@U?$pair@$$CBIUEntityProp@CEntityLayer@@@stlpmtx_std@@@priv@2@U?$_Select1st@U?$pair@$$CBIUEntityProp@CEntityLayer@@@stlpmtx_std@@@52@U?$equal_to@I@2@V?$allocator@U?$pair@$$CBIUEntityProp@CEntityLayer@@@stlpmtx_std@@@2@@stlpmtx_std@@IAE?AU?$_Ht_iterator@V?$_Slist_iterator@U?$pair@$$CBIUEntityProp@CEntityLayer@@@stlpmtx_std@@U?$_Nonconst_traits@U?$pair@$$CBIUEntityProp@CEntityLayer@@@stlpmtx_std@@@2@@priv@stlpmtx_std@@U?$_NonLocalUnorderedMapTraitsT@U?$pair@$$CBIUEntityProp@CEntityLayer@@@stlpmtx_std@@@23@@priv@2@IABU?$pair@$$CBIUEntityProp@CEntityLayer@@@2@@Z 320298c0 f i EntityLayer.obj
 0001:00028990       ?clear@?$hashtable@U?$pair@$$CBIUEntityProp@CEntityLayer@@@stlpmtx_std@@IU?$hash@I@2@U?$_UnorderedMapTraitsT@U?$pair@$$CBIUEntityProp@CEntityLayer@@@stlpmtx_std@@@priv@2@U?$_Select1st@U?$pair@$$CBIUEntityProp@CEntityLayer@@@stlpmtx_std@@@52@U?$equal_to@I@2@V?$allocator@U?$pair@$$CBIUEntityProp@CEntityLayer@@@stlpmtx_std@@@2@@stlpmtx_std@@QAEXXZ 32029990 f i EntityLayer.obj
 0001:000289e0       ?insert_unique_noresize@?$hashtable@U?$pair@$$CBIUEntityProp@CEntityLayer@@@stlpmtx_std@@IU?$hash@I@2@U?$_UnorderedMapTraitsT@U?$pair@$$CBIUEntityProp@CEntityLayer@@@stlpmtx_std@@@priv@2@U?$_Select1st@U?$pair@$$CBIUEntityProp@CEntityLayer@@@stlpmtx_std@@@52@U?$equal_to@I@2@V?$allocator@U?$pair@$$CBIUEntityProp@CEntityLayer@@@stlpmtx_std@@@2@@stlpmtx_std@@QAE?AU?$pair@U?$_Ht_iterator@V?$_Slist_iterator@U?$pair@$$CBIUEntityProp@CEntityLayer@@@stlpmtx_std@@U?$_Nonconst_traits@U?$pair@$$CBIUEntityProp@CEntityLayer@@@stlpmtx_std@@@2@@priv@stlpmtx_std@@U?$_NonLocalUnorderedMapTraitsT@U?$pair@$$CBIUEntityProp@CEntityLayer@@@stlpmtx_std@@@23@@priv@stlpmtx_std@@_N@2@ABU?$pair@$$CBIUEntityProp@CEntityLayer@@@2@@Z 320299e0 f i EntityLayer.obj
 0001:00028ab0       ?Enable@CEntityLayer@@QAEX_N0@Z 32029ab0 f   EntityLayer.obj
 0001:00028ce0       ??1CEntityLayer@@UAE@XZ    32029ce0 f   EntityLayer.obj
 0001:00028f70       ??_ECEntityLayer@@UAEPAXI@Z 32029f70 f i EntityLayer.obj
 0001:00028f70       ??_GCEntityLayer@@UAEPAXI@Z 32029f70 f i EntityLayer.obj
 0001:00028fa0       ??0CEntityLayer@@QAE@PBDG_NH1@Z 32029fa0 f   EntityLayer.obj
 0001:00029030       ?_M_rehash@?$hashtable@U?$pair@$$CBIUEntityProp@CEntityLayer@@@stlpmtx_std@@IU?$hash@I@2@U?$_UnorderedMapTraitsT@U?$pair@$$CBIUEntityProp@CEntityLayer@@@stlpmtx_std@@@priv@2@U?$_Select1st@U?$pair@$$CBIUEntityProp@CEntityLayer@@@stlpmtx_std@@@52@U?$equal_to@I@2@V?$allocator@U?$pair@$$CBIUEntityProp@CEntityLayer@@@stlpmtx_std@@@2@@stlpmtx_std@@AAEXI@Z 3202a030 f i EntityLayer.obj
 0001:000292b0       ?_M_reduce@?$hashtable@U?$pair@$$CBIUEntityProp@CEntityLayer@@@stlpmtx_std@@IU?$hash@I@2@U?$_UnorderedMapTraitsT@U?$pair@$$CBIUEntityProp@CEntityLayer@@@stlpmtx_std@@@priv@2@U?$_Select1st@U?$pair@$$CBIUEntityProp@CEntityLayer@@@stlpmtx_std@@@52@U?$equal_to@I@2@V?$allocator@U?$pair@$$CBIUEntityProp@CEntityLayer@@@stlpmtx_std@@@2@@stlpmtx_std@@AAEXXZ 3202a2b0 f i EntityLayer.obj
 0001:000293c0       ?_M_enlarge@?$hashtable@U?$pair@$$CBIUEntityProp@CEntityLayer@@@stlpmtx_std@@IU?$hash@I@2@U?$_UnorderedMapTraitsT@U?$pair@$$CBIUEntityProp@CEntityLayer@@@stlpmtx_std@@@priv@2@U?$_Select1st@U?$pair@$$CBIUEntityProp@CEntityLayer@@@stlpmtx_std@@@52@U?$equal_to@I@2@V?$allocator@U?$pair@$$CBIUEntityProp@CEntityLayer@@@stlpmtx_std@@@2@@stlpmtx_std@@AAEXI@Z 3202a3c0 f i EntityLayer.obj
 0001:00029460       ?erase@?$hashtable@U?$pair@$$CBIUEntityProp@CEntityLayer@@@stlpmtx_std@@IU?$hash@I@2@U?$_UnorderedMapTraitsT@U?$pair@$$CBIUEntityProp@CEntityLayer@@@stlpmtx_std@@@priv@2@U?$_Select1st@U?$pair@$$CBIUEntityProp@CEntityLayer@@@stlpmtx_std@@@52@U?$equal_to@I@2@V?$allocator@U?$pair@$$CBIUEntityProp@CEntityLayer@@@stlpmtx_std@@@2@@stlpmtx_std@@QAEXU?$_Ht_iterator@V?$_Slist_iterator@U?$pair@$$CBIUEntityProp@CEntityLayer@@@stlpmtx_std@@U?$_Nonconst_traits@U?$pair@$$CBIUEntityProp@CEntityLayer@@@stlpmtx_std@@@2@@priv@stlpmtx_std@@U?$_ConstNonLocalUnorderedMapTraitsT@U?$pair@$$CBIUEntityProp@CEntityLayer@@@stlpmtx_std@@@23@@priv@2@@Z 3202a460 f i EntityLayer.obj
 0001:00029560       ?AddObject@CEntityLayer@@QAEXI@Z 3202a560 f   EntityLayer.obj
 0001:00029620       ?RemoveObject@CEntityLayer@@QAEXI@Z 3202a620 f   EntityLayer.obj
 0001:00029660       ?Serialize@CEntityLayer@@QAEXV?$CSerializeWrapper@UISerialize@@@@@Z 3202a660 f   EntityLayer.obj
 0001:00029980       ?MoveFirst@CEntityItMap@@UAEXXZ 3202a980 f i EntitySystem.obj
 0001:00029990       ?OnRemoveEntityCVarChange@@YAXPAUICVar@@@Z 3202a990 f   EntitySystem.obj
 0001:000299f0       ?OnActivateEntityCVarChange@@YAXPAUICVar@@@Z 3202a9f0 f   EntitySystem.obj
 0001:00029a30       ?OnDeactivateEntityCVarChange@@YAXPAUICVar@@@Z 3202aa30 f   EntitySystem.obj
 0001:00029a70       ?GetClassRegistry@CEntitySystem@@UAEPAUIEntityClassRegistry@@XZ 3202aa70 f   EntitySystem.obj
 0001:00029a80       ?RegisterPhysicCallbacks@CEntitySystem@@UAEXXZ 3202aa80 f   EntitySystem.obj
 0001:00029aa0       ?UnregisterPhysicCallbacks@CEntitySystem@@UAEXXZ 3202aaa0 f   EntitySystem.obj
 0001:00029ac0       ??4XmlNodeRef@@QAEAAV0@ABV0@@Z 3202aac0 f i EntitySystem.obj
 0001:00029af0       ?GetEntityFromPhysics@CEntitySystem@@UBEPAUIEntity@@PAUIPhysicalEntity@@@Z 3202aaf0 f   EntitySystem.obj
 0001:00029b10       ?OnLoadLevel@CEntitySystem@@UAE_NPBD@Z 3202ab10 f   EntitySystem.obj
 0001:00029b60       ?OnLevelLoadStart@CEntitySystem@@QAEXXZ 3202ab60 f   EntitySystem.obj
 0001:00029b70       ?LoadEntityArchetype@CEntitySystem@@UAEPAUIEntityArchetype@@PBD@Z 3202ab70 f   EntitySystem.obj
 0001:00029b80       ?CreateEntityArchetype@CEntitySystem@@UAEPAUIEntityArchetype@@PAUIEntityClass@@PBD@Z 3202ab80 f   EntitySystem.obj
 0001:00029b90       ?ResizeProximityGrid@CEntitySystem@@UAEXHH@Z 3202ab90 f   EntitySystem.obj
 0001:00029bd0       ?SetNextSpawnId@CEntitySystem@@UAEXI@Z 3202abd0 f   EntitySystem.obj
 0001:00029c00       ?ResetAreas@CEntitySystem@@UAEXXZ 3202ac00 f   EntitySystem.obj
 0001:00029c10       ?UnloadAreas@CEntitySystem@@UAEXXZ 3202ac10 f   EntitySystem.obj
 0001:00029c30       ?UpdateEngineCVars@CEntitySystem@@AAEXXZ 3202ac30 f   EntitySystem.obj
 0001:00029d30       ?RegisterForEvents@CEntitySystem@@UAEXIPAUIEntityEvent@@PBHH@Z 3202ad30 f   EntitySystem.obj
 0001:00029d50       ?UnRegisterForEvents@CEntitySystem@@UAEXPAUIEntityEvent@@PBHH@Z 3202ad50 f   EntitySystem.obj
 0001:00029d70       ?Reset@?$CSaltBufferArray@GG$0PPPN@@@QAEXXZ 3202ad70 f i EntitySystem.obj
 0001:00029dc0       ?RemoveFromFreeList@?$CSaltBufferArray@GG$0PPPN@@@AAEXG@Z 3202adc0 f i EntitySystem.obj
 0001:00029e40       ?DrawLabelEx@IRenderer@@QAAXU?$Vec3_tpl@M@@MPBM_N2PBDZZ 3202ae40 f i EntitySystem.obj
 0001:00029ef0       ??_EIEntitySystem@@UAEPAXI@Z 3202aef0 f i EntitySystem.obj
 0001:00029ef0       ??_GIEntitySystem@@UAEPAXI@Z 3202aef0 f i EntitySystem.obj
 0001:00029f20       ??F?$_Rb_tree_iterator@U?$pair@$$CBV?$CryStringT@D@@PAVCEntityLayer@@@stlpmtx_std@@U?$_MapTraitsT@U?$pair@$$CBV?$CryStringT@D@@PAVCEntityLayer@@@stlpmtx_std@@@priv@2@@priv@stlpmtx_std@@QAEAAU012@XZ 3202af20 f i EntitySystem.obj
 0001:00029f20       ??F?$_Rb_tree_iterator@U?$pair@$$CB_KI@stlpmtx_std@@U?$_MapTraitsT@U?$pair@$$CB_KI@stlpmtx_std@@@priv@2@@priv@stlpmtx_std@@QAEAAU012@XZ 3202af20 f i EntitySystem.obj
 0001:00029f20       ??F?$_Rb_tree_iterator@U?$pair@$$CBV?$CryStringT@D@@V?$vector@PAVCEntityLayer@@V?$allocator@PAVCEntityLayer@@@stlpmtx_std@@@stlpmtx_std@@@stlpmtx_std@@U?$_MapTraitsT@U?$pair@$$CBV?$CryStringT@D@@V?$vector@PAVCEntityLayer@@V?$allocator@PAVCEntityLayer@@@stlpmtx_std@@@stlpmtx_std@@@stlpmtx_std@@@priv@2@@priv@stlpmtx_std@@QAEAAU012@XZ 3202af20 f i EntitySystem.obj
 0001:00029f20       ??F?$_Rb_tree_iterator@IU?$_SetTraitsT@I@priv@stlpmtx_std@@@priv@stlpmtx_std@@QAEAAU012@XZ 3202af20 f i EntitySystem.obj
 0001:00029f20       ??F?$_Rb_tree_iterator@U?$pair@$$CBIUSEntityBookmark@CEntityPoolManager@@@stlpmtx_std@@U?$_MapTraitsT@U?$pair@$$CBIUSEntityBookmark@CEntityPoolManager@@@stlpmtx_std@@@priv@2@@priv@stlpmtx_std@@QAEAAU012@XZ 3202af20 f i EntityPoolManager.obj
 0001:00029f20       ??F?$_Rb_tree_iterator@U?$pair@$$CBIPAVCEntity@@@stlpmtx_std@@U?$_MapTraitsT@U?$pair@$$CBIPAVCEntity@@@stlpmtx_std@@@priv@2@@priv@stlpmtx_std@@QAEAAU012@XZ 3202af20 f i EntitySystem.obj
 0001:00029f20       ??F?$_Rb_tree_iterator@V?$CryStringT@D@@U?$_SetTraitsT@V?$CryStringT@D@@@priv@stlpmtx_std@@@priv@stlpmtx_std@@QAEAAU012@XZ 3202af20 f i EntitySystem.obj
 0001:00029f20       ??F?$_Rb_tree_iterator@U?$pair@$$CBIPAVCEntityPool@@@stlpmtx_std@@U?$_MapTraitsT@U?$pair@$$CBIPAVCEntityPool@@@stlpmtx_std@@@priv@2@@priv@stlpmtx_std@@QAEAAU012@XZ 3202af20 f i EntityPoolManager.obj
 0001:00029f20       ??F?$_Rb_tree_iterator@U?$pair@$$CBIPAVCEntityPoolDefinition@@@stlpmtx_std@@U?$_MapTraitsT@U?$pair@$$CBIPAVCEntityPoolDefinition@@@stlpmtx_std@@@priv@2@@priv@stlpmtx_std@@QAEAAU012@XZ 3202af20 f i EntityPoolManager.obj
 0001:00029f20       ??F?$_Rb_tree_iterator@U?$pair@QBDV?$_smart_ptr@VCEntityArchetype@@@@@stlpmtx_std@@U?$_MapTraitsT@U?$pair@QBDV?$_smart_ptr@VCEntityArchetype@@@@@stlpmtx_std@@@priv@2@@priv@stlpmtx_std@@QAEAAU012@XZ 3202af20 f i EntityArchetype.obj
 0001:00029f20       ??F?$_Rb_tree_iterator@U?$pair@QAUIEntityClass@@V?$vector@U?$pair@II@stlpmtx_std@@V?$allocator@U?$pair@II@stlpmtx_std@@@2@@stlpmtx_std@@@stlpmtx_std@@U?$_MapTraitsT@U?$pair@QAUIEntityClass@@V?$vector@U?$pair@II@stlpmtx_std@@V?$allocator@U?$pair@II@stlpmtx_std@@@2@@stlpmtx_std@@@stlpmtx_std@@@priv@2@@priv@stlpmtx_std@@QAEAAU012@XZ 3202af20 f i EntitySystem.obj
 0001:00029f20       ??F?$_Rb_tree_iterator@U?$pair@$$CBV?$CryStringT@D@@PAUIEntityClass@@@stlpmtx_std@@U?$_MapTraitsT@U?$pair@$$CBV?$CryStringT@D@@PAUIEntityClass@@@stlpmtx_std@@@priv@2@@priv@stlpmtx_std@@QAEAAU012@XZ 3202af20 f i EntityClassRegistry.obj
 0001:00029f20       ??F?$_Rb_tree_iterator@U?$pair@$$CBHUSAreasCache@CAreaManager@@@stlpmtx_std@@U?$_MapTraitsT@U?$pair@$$CBHUSAreasCache@CAreaManager@@@stlpmtx_std@@@priv@2@@priv@stlpmtx_std@@QAEAAU012@XZ 3202af20 f i AreaManager.obj
 0001:00029f20       ??F?$_Rb_tree_iterator@U?$pair@QAUIEntityClass@@_N@stlpmtx_std@@U?$_MapTraitsT@U?$pair@QAUIEntityClass@@_N@stlpmtx_std@@@priv@2@@priv@stlpmtx_std@@QAEAAU012@XZ 3202af20 f i EntityPoolDefinition.obj
 0001:00029f20       ??F?$_Rb_tree_iterator@U?$pair@$$CBV?$CryStringT@D@@H@stlpmtx_std@@U?$_MapTraitsT@U?$pair@$$CBV?$CryStringT@D@@H@stlpmtx_std@@@priv@2@@priv@stlpmtx_std@@QAEAAU012@XZ 3202af20 f i EntityCVars.obj
 0001:00029f70       ??E?$_Rb_tree_iterator@U?$pair@$$CBIPAVCEntityPoolDefinition@@@stlpmtx_std@@U?$_MapTraitsT@U?$pair@$$CBIPAVCEntityPoolDefinition@@@stlpmtx_std@@@priv@2@@priv@stlpmtx_std@@QAEAAU012@XZ 3202af70 f i EntityPoolManager.obj
 0001:00029f70       ??E?$_Rb_tree_iterator@U?$pair@QAUIEntityClass@@_N@stlpmtx_std@@U?$_MapTraitsT@U?$pair@QAUIEntityClass@@_N@stlpmtx_std@@@priv@2@@priv@stlpmtx_std@@QAEAAU012@XZ 3202af70 f i EntityPoolDefinition.obj
 0001:00029f70       ??E?$_Rb_tree_iterator@U?$pair@$$CBV?$CryStringT@D@@PAUIEntityClass@@@stlpmtx_std@@U?$_MapTraitsT@U?$pair@$$CBV?$CryStringT@D@@PAUIEntityClass@@@stlpmtx_std@@@priv@2@@priv@stlpmtx_std@@QAEAAU012@XZ 3202af70 f i EntityClassRegistry.obj
 0001:00029f70       ??E?$_Rb_tree_iterator@U?$pair@$$CBIPAVCEntityPool@@@stlpmtx_std@@U?$_MapTraitsT@U?$pair@$$CBIPAVCEntityPool@@@stlpmtx_std@@@priv@2@@priv@stlpmtx_std@@QAEAAU012@XZ 3202af70 f i EntityPoolManager.obj
 0001:00029f70       ??E?$_Rb_tree_iterator@U?$pair@$$CBV?$CryStringT@D@@H@stlpmtx_std@@U?$_MapTraitsT@U?$pair@$$CBV?$CryStringT@D@@H@stlpmtx_std@@@priv@2@@priv@stlpmtx_std@@QAEAAU012@XZ 3202af70 f i EntityCVars.obj
 0001:00029f70       ??E?$_Rb_tree_iterator@U?$pair@$$CBHUSAreasCache@CAreaManager@@@stlpmtx_std@@U?$_MapTraitsT@U?$pair@$$CBHUSAreasCache@CAreaManager@@@stlpmtx_std@@@priv@2@@priv@stlpmtx_std@@QAEAAU012@XZ 3202af70 f i AreaManager.obj
 0001:00029f70       ??E?$_Rb_tree_iterator@U?$pair@QBDV?$_smart_ptr@VCEntityArchetype@@@@@stlpmtx_std@@U?$_MapTraitsT@U?$pair@QBDV?$_smart_ptr@VCEntityArchetype@@@@@stlpmtx_std@@@priv@2@@priv@stlpmtx_std@@QAEAAU012@XZ 3202af70 f i EntityArchetype.obj
 0001:00029f70       ??E?$_Rb_tree_iterator@U?$pair@$$CBV?$CryStringT@D@@V?$vector@PAVCEntityLayer@@V?$allocator@PAVCEntityLayer@@@stlpmtx_std@@@stlpmtx_std@@@stlpmtx_std@@U?$_MapTraitsT@U?$pair@$$CBV?$CryStringT@D@@V?$vector@PAVCEntityLayer@@V?$allocator@PAVCEntityLayer@@@stlpmtx_std@@@stlpmtx_std@@@stlpmtx_std@@@priv@2@@priv@stlpmtx_std@@QAEAAU012@XZ 3202af70 f i EntitySystem.obj
 0001:00029f70       ??E?$_Rb_tree_iterator@U?$pair@$$CBIPAVCEntity@@@stlpmtx_std@@U?$_MapTraitsT@U?$pair@$$CBIPAVCEntity@@@stlpmtx_std@@@priv@2@@priv@stlpmtx_std@@QAEAAU012@XZ 3202af70 f i EntitySystem.obj
 0001:00029f70       ??E?$_Rb_tree_iterator@U?$pair@$$CBV?$CryStringT@D@@PAVCEntityLayer@@@stlpmtx_std@@U?$_MapTraitsT@U?$pair@$$CBV?$CryStringT@D@@PAVCEntityLayer@@@stlpmtx_std@@@priv@2@@priv@stlpmtx_std@@QAEAAU012@XZ 3202af70 f i EntitySystem.obj
 0001:00029f70       ??E?$_Rb_tree_iterator@U?$pair@QAUIEntityClass@@V?$vector@U?$pair@II@stlpmtx_std@@V?$allocator@U?$pair@II@stlpmtx_std@@@2@@stlpmtx_std@@@stlpmtx_std@@U?$_MapTraitsT@U?$pair@QAUIEntityClass@@V?$vector@U?$pair@II@stlpmtx_std@@V?$allocator@U?$pair@II@stlpmtx_std@@@2@@stlpmtx_std@@@stlpmtx_std@@@priv@2@@priv@stlpmtx_std@@QAEAAU012@XZ 3202af70 f i EntitySystem.obj
 0001:00029fb0       ??$__median@IVCCompareEntityIdsByClass@CEntitySystem@@@priv@stlpmtx_std@@YAABIABI00VCCompareEntityIdsByClass@CEntitySystem@@@Z 3202afb0 f i EntitySystem.obj
 0001:0002a070       ??$__unguarded_linear_insert@PAIIVCCompareEntityIdsByClass@CEntitySystem@@@priv@stlpmtx_std@@YAXPAIIVCCompareEntityIdsByClass@CEntitySystem@@@Z 3202b070 f i EntitySystem.obj
 0001:0002a0e0       ??$__push_heap@PAIHIVCCompareEntityIdsByClass@CEntitySystem@@@stlpmtx_std@@YAXPAIHHIVCCompareEntityIdsByClass@CEntitySystem@@@Z 3202b0e0 f i EntitySystem.obj
 0001:0002a170       ?AddRef@CEntityItMap@@UAEXXZ 3202b170 f i EntitySystem.obj
 0001:0002a180       ?Release@CEntityItMap@@UAEXXZ 3202b180 f i EntitySystem.obj
 0001:0002a1a0       ??1SEntityLoadParams@@QAE@XZ 3202b1a0 f   EntitySystem.obj
 0001:0002a1e0       ??4SEntitySpawnParams@@QAEAAU0@ABU0@@Z 3202b1e0 f i EntitySystem.obj
 0001:0002a290       ?CloneXmlNode@SEntityLoadParams@@CA_NVXmlNodeRef@@V2@@Z 3202b290 f   EntitySystem.obj
 0001:0002a410       ?Release@CMultiThreadRefCount@@QAEHXZ 3202b410 f i EntitySystem.obj
 0001:0002a450       ?GetPhysicalEntitiesInBox@CEntitySystem@@UBEHABU?$Vec3_tpl@M@@MAAPAPAUIPhysicalEntity@@H@Z 3202b450 f   EntitySystem.obj
 0001:0002a510       ?DrawText@?A0x21648d16@@YAXMMU?$Color_tpl@M@@PBDZZ 3202b510 f   EntitySystem.obj
 0001:0002a5c0       ??0CCamera@@QAE@ABV0@@Z    3202b5c0 f i EntitySystem.obj
 0001:0002aba0       ?GetEntityIterator@CEntitySystem@@UAEPAUIEntityIt@@XZ 3202bba0 f   EntitySystem.obj
 0001:0002abd0       ?IsIDUsed@CEntitySystem@@UBE_NI@Z 3202bbd0 f   EntitySystem.obj
 0001:0002abf0       ?DebugDrawProximityTriggers@CEntitySystem@@AAEXXZ 3202bbf0 f   EntitySystem.obj
 0001:0002adc0       ?DoPrePhysicsUpdateFast@CEntitySystem@@AAEXXZ 3202bdc0 f   EntitySystem.obj
 0001:0002aef0       ?InsertKnownHandle@?$CSaltBufferArray@GG$0PPPN@@@QAEXV?$CSaltHandle@GG@@@Z 3202bef0 f i EntitySystem.obj
 0001:0002af50       ??0pe_status_pos@@QAE@XZ   3202bf50 f i EntitySystem.obj
 0001:0002af80       ?Draw2dLabel@IRenderer@@QAAXMMMPBM_NPBDZZ 3202bf80 f i EntitySystem.obj
 0001:0002b050       ?_Rebalance_for_erase@?$_Rb_global@_N@priv@stlpmtx_std@@SAPAU_Rb_tree_node_base@23@PAU423@AAPAU423@11@Z 3202c050 f i EntitySystem.obj
 0001:0002b340       ??$_M_find@_K@?$_Rb_tree@_KU?$less@_K@stlpmtx_std@@U?$pair@$$CB_KI@2@U?$_Select1st@U?$pair@$$CB_KI@stlpmtx_std@@@priv@2@U?$_MapTraitsT@U?$pair@$$CB_KI@stlpmtx_std@@@52@V?$allocator@U?$pair@$$CB_KI@stlpmtx_std@@@2@@priv@stlpmtx_std@@ABEPAU_Rb_tree_node_base@12@AB_K@Z 3202c340 f i EntitySystem.obj
 0001:0002b390       ??$fill@PAU?$Vec3_tpl@M@@U1@@stlpmtx_std@@YAXPAU?$Vec3_tpl@M@@0ABU1@@Z 3202c390 f i ScriptBind_Entity.obj
 0001:0002b390       ??$fill@PAUSEntityTimerEvent@@U1@@stlpmtx_std@@YAXPAUSEntityTimerEvent@@0ABU1@@Z 3202c390 f i EntitySystem.obj
 0001:0002b390       ??$fill@PAUSProximityEvent@@U1@@stlpmtx_std@@YAXPAUSProximityEvent@@0ABU1@@Z 3202c390 f i ProximityTriggerSystem.obj
 0001:0002b3d0       ??$_M_lower_bound@PBD@?$_Rb_tree@PBDU?$less_stricmp@PBD@stl@@U?$pair@QBDI@stlpmtx_std@@U?$_Select1st@U?$pair@QBDI@stlpmtx_std@@@priv@4@U?$_MultimapTraitsT@U?$pair@QBDI@stlpmtx_std@@@64@V?$allocator@U?$pair@QBDI@stlpmtx_std@@@4@@priv@stlpmtx_std@@ABEPAU_Rb_tree_node_base@12@ABQBD@Z 3202c3d0 f i EntitySystem.obj
 0001:0002b3d0       ??$_M_lower_bound@PBD@?$_Rb_tree@PBDU?$less_stricmp@PBD@stl@@U?$pair@QBDV?$_smart_ptr@VCEntityArchetype@@@@@stlpmtx_std@@U?$_Select1st@U?$pair@QBDV?$_smart_ptr@VCEntityArchetype@@@@@stlpmtx_std@@@priv@4@U?$_MapTraitsT@U?$pair@QBDV?$_smart_ptr@VCEntityArchetype@@@@@stlpmtx_std@@@64@V?$allocator@U?$pair@QBDV?$_smart_ptr@VCEntityArchetype@@@@@stlpmtx_std@@@4@@priv@stlpmtx_std@@ABEPAU_Rb_tree_node_base@12@ABQBD@Z 3202c3d0 f i EntityArchetype.obj
 0001:0002b420       ??$__unguarded_insertion_sort_aux@PAIIVCCompareEntityIdsByClass@CEntitySystem@@@priv@stlpmtx_std@@YAXPAI00VCCompareEntityIdsByClass@CEntitySystem@@@Z 3202c420 f i EntitySystem.obj
 0001:0002b4a0       ??$__adjust_heap@PAIHIVCCompareEntityIdsByClass@CEntitySystem@@@stlpmtx_std@@YAXPAIHHIVCCompareEntityIdsByClass@CEntitySystem@@@Z 3202c4a0 f i EntitySystem.obj
 0001:0002b530       ??_EIEntityIt@@UAEPAXI@Z   3202c530 f i EntitySystem.obj
 0001:0002b530       ??_GIEntityIt@@UAEPAXI@Z   3202c530 f i EntitySystem.obj
 0001:0002b530       ??_ECEntityItMap@@UAEPAXI@Z 3202c530 f i EntitySystem.obj
 0001:0002b530       ??_GCEntityItMap@@UAEPAXI@Z 3202c530 f i EntitySystem.obj
 0001:0002b560       ??0SEntityLoadParams@@QAE@XZ 3202c560 f   EntitySystem.obj
 0001:0002b5a0       ??4SEntityLoadParams@@QAEAAU0@ABU0@@Z 3202c5a0 f   EntitySystem.obj
 0001:0002b610       ?UseClonedEntityNode@SEntityLoadParams@@QAEXVXmlNodeRef@@V2@@Z 3202c610 f   EntitySystem.obj
 0001:0002b780       ?PostPumpLoggedEvents@CEntitySystem@@UAEXXZ 3202c780 f   EntitySystem.obj
 0001:0002b8c0       ?ReserveEntityId@CEntitySystem@@UAEXI@Z 3202c8c0 f   EntitySystem.obj
 0001:0002b940       ?LoadEntities@CEntitySystem@@UAEXAAVXmlNodeRef@@@Z 3202c940 f   EntitySystem.obj
 0001:0002ba40       ?DebugDraw@CEntitySystem@@AAEXPAVCEntity@@M@Z 3202ca40 f   EntitySystem.obj
 0001:0002bf40       ?DebugDraw@CEntitySystem@@UAEXXZ 3202cf40 f   EntitySystem.obj
 0001:0002bf50       ?InsertDynamic@?$CSaltBufferArray@GG$0PPPN@@@QAE?AV?$CSaltHandle@GG@@XZ 3202cf50 f i EntitySystem.obj
 0001:0002bfc0       ?InsertStatic@?$CSaltBufferArray@GG$0PPPN@@@QAE?AV?$CSaltHandle@GG@@XZ 3202cfc0 f i EntitySystem.obj
 0001:0002c060       ?_M_erase@?$_Rb_tree@IU?$less@I@stlpmtx_std@@U?$pair@$$CBIPAUIEntityEventListener@@@2@U?$_Select1st@U?$pair@$$CBIPAUIEntityEventListener@@@stlpmtx_std@@@priv@2@U?$_MultimapTraitsT@U?$pair@$$CBIPAUIEntityEventListener@@@stlpmtx_std@@@52@V?$allocator@U?$pair@$$CBIPAUIEntityEventListener@@@stlpmtx_std@@@2@@priv@stlpmtx_std@@AAEXPAU_Rb_tree_node_base@23@@Z 3202d060 f i EntitySystem.obj
 0001:0002c060       ?_M_erase@?$_Rb_tree@PBDU?$less_stricmp@PBD@stl@@U?$pair@QBDI@stlpmtx_std@@U?$_Select1st@U?$pair@QBDI@stlpmtx_std@@@priv@4@U?$_MultimapTraitsT@U?$pair@QBDI@stlpmtx_std@@@64@V?$allocator@U?$pair@QBDI@stlpmtx_std@@@4@@priv@stlpmtx_std@@AAEXPAU_Rb_tree_node_base@23@@Z 3202d060 f i EntitySystem.obj
 0001:0002c060       ?_M_erase@?$_Rb_tree@_KU?$less@_K@stlpmtx_std@@U?$pair@$$CB_KI@2@U?$_Select1st@U?$pair@$$CB_KI@stlpmtx_std@@@priv@2@U?$_MapTraitsT@U?$pair@$$CB_KI@stlpmtx_std@@@52@V?$allocator@U?$pair@$$CB_KI@stlpmtx_std@@@2@@priv@stlpmtx_std@@AAEXPAU_Rb_tree_node_base@23@@Z 3202d060 f i EntitySystem.obj
 0001:0002c060       ?_M_erase@?$_Rb_tree@IU?$less@I@stlpmtx_std@@U?$pair@$$CBIPAVCEntityPoolDefinition@@@2@U?$_Select1st@U?$pair@$$CBIPAVCEntityPoolDefinition@@@stlpmtx_std@@@priv@2@U?$_MapTraitsT@U?$pair@$$CBIPAVCEntityPoolDefinition@@@stlpmtx_std@@@52@V?$allocator@U?$pair@$$CBIPAVCEntityPoolDefinition@@@stlpmtx_std@@@2@@priv@stlpmtx_std@@AAEXPAU_Rb_tree_node_base@23@@Z 3202d060 f i EntityPoolManager.obj
 0001:0002c060       ?_M_erase@?$_Rb_tree@IU?$less@I@stlpmtx_std@@IU?$_Identity@I@priv@2@U?$_SetTraitsT@I@42@V?$allocator@I@2@@priv@stlpmtx_std@@AAEXPAU_Rb_tree_node_base@23@@Z 3202d060 f i EntitySystem.obj
 0001:0002c060       ?_M_erase@?$_Rb_tree@PAUIEntityClass@@U?$less@PAUIEntityClass@@@stlpmtx_std@@U?$pair@QAUIEntityClass@@_N@3@U?$_Select1st@U?$pair@QAUIEntityClass@@_N@stlpmtx_std@@@priv@3@U?$_MapTraitsT@U?$pair@QAUIEntityClass@@_N@stlpmtx_std@@@63@V?$allocator@U?$pair@QAUIEntityClass@@_N@stlpmtx_std@@@3@@priv@stlpmtx_std@@AAEXPAU_Rb_tree_node_base@23@@Z 3202d060 f i EntityPoolDefinition.obj
 0001:0002c060       ?_M_erase@?$_Rb_tree@IU?$less@I@stlpmtx_std@@U?$pair@$$CBIPAVCEntity@@@2@U?$_Select1st@U?$pair@$$CBIPAVCEntity@@@stlpmtx_std@@@priv@2@U?$_MapTraitsT@U?$pair@$$CBIPAVCEntity@@@stlpmtx_std@@@52@V?$allocator@U?$pair@$$CBIPAVCEntity@@@stlpmtx_std@@@2@@priv@stlpmtx_std@@AAEXPAU_Rb_tree_node_base@23@@Z 3202d060 f i EntitySystem.obj
 0001:0002c060       ?_M_erase@?$_Rb_tree@IU?$less@I@stlpmtx_std@@U?$pair@$$CBIPAVCEntityPool@@@2@U?$_Select1st@U?$pair@$$CBIPAVCEntityPool@@@stlpmtx_std@@@priv@2@U?$_MapTraitsT@U?$pair@$$CBIPAVCEntityPool@@@stlpmtx_std@@@52@V?$allocator@U?$pair@$$CBIPAVCEntityPool@@@stlpmtx_std@@@2@@priv@stlpmtx_std@@AAEXPAU_Rb_tree_node_base@23@@Z 3202d060 f i EntityPoolManager.obj
 0001:0002c0a0       ??$find@I@?$_Rb_tree@IU?$less@I@stlpmtx_std@@IU?$_Identity@I@priv@2@U?$_SetTraitsT@I@42@V?$allocator@I@2@@priv@stlpmtx_std@@QAE?AU?$_Rb_tree_iterator@IU?$_SetTraitsT@I@priv@stlpmtx_std@@@12@ABI@Z 3202d0a0 f i EntitySystem.obj
 0001:0002c0a0       ??$find@I@?$_Rb_tree@IU?$less@I@stlpmtx_std@@U?$pair@$$CBIUSEntityBookmark@CEntityPoolManager@@@2@U?$_Select1st@U?$pair@$$CBIUSEntityBookmark@CEntityPoolManager@@@stlpmtx_std@@@priv@2@U?$_MapTraitsT@U?$pair@$$CBIUSEntityBookmark@CEntityPoolManager@@@stlpmtx_std@@@52@V?$allocator@U?$pair@$$CBIUSEntityBookmark@CEntityPoolManager@@@stlpmtx_std@@@2@@priv@stlpmtx_std@@QAE?AU?$_Rb_tree_iterator@U?$pair@$$CBIUSEntityBookmark@CEntityPoolManager@@@stlpmtx_std@@U?$_MapTraitsT@U?$pair@$$CBIUSEntityBookmark@CEntityPoolManager@@@stlpmtx_std@@@priv@2@@12@ABI@Z 3202d0a0 f i EntityPoolManager.obj
 0001:0002c0f0       ??$_M_find@V?$CryStringT@D@@@?$_Rb_tree@V?$CryStringT@D@@U?$less@V?$CryStringT@D@@@stlpmtx_std@@U?$pair@$$CBV?$CryStringT@D@@PAUIEntityClass@@@3@U?$_Select1st@U?$pair@$$CBV?$CryStringT@D@@PAUIEntityClass@@@stlpmtx_std@@@priv@3@U?$_MapTraitsT@U?$pair@$$CBV?$CryStringT@D@@PAUIEntityClass@@@stlpmtx_std@@@63@V?$allocator@U?$pair@$$CBV?$CryStringT@D@@PAUIEntityClass@@@stlpmtx_std@@@3@@priv@stlpmtx_std@@ABEPAU_Rb_tree_node_base@12@ABV?$CryStringT@D@@@Z 3202d0f0 f i EntityClassRegistry.obj
 0001:0002c0f0       ??$_M_find@V?$CryStringT@D@@@?$_Rb_tree@V?$CryStringT@D@@U?$less@V?$CryStringT@D@@@stlpmtx_std@@U?$pair@$$CBV?$CryStringT@D@@PAVCEntityLayer@@@3@U?$_Select1st@U?$pair@$$CBV?$CryStringT@D@@PAVCEntityLayer@@@stlpmtx_std@@@priv@3@U?$_MapTraitsT@U?$pair@$$CBV?$CryStringT@D@@PAVCEntityLayer@@@stlpmtx_std@@@63@V?$allocator@U?$pair@$$CBV?$CryStringT@D@@PAVCEntityLayer@@@stlpmtx_std@@@3@@priv@stlpmtx_std@@ABEPAU_Rb_tree_node_base@12@ABV?$CryStringT@D@@@Z 3202d0f0 f i EntitySystem.obj
 0001:0002c0f0       ??$_M_find@V?$CryStringT@D@@@?$_Rb_tree@V?$CryStringT@D@@U?$less@V?$CryStringT@D@@@stlpmtx_std@@U?$pair@$$CBV?$CryStringT@D@@V?$vector@PAVCEntityLayer@@V?$allocator@PAVCEntityLayer@@@stlpmtx_std@@@stlpmtx_std@@@3@U?$_Select1st@U?$pair@$$CBV?$CryStringT@D@@V?$vector@PAVCEntityLayer@@V?$allocator@PAVCEntityLayer@@@stlpmtx_std@@@stlpmtx_std@@@stlpmtx_std@@@priv@3@U?$_MapTraitsT@U?$pair@$$CBV?$CryStringT@D@@V?$vector@PAVCEntityLayer@@V?$allocator@PAVCEntityLayer@@@stlpmtx_std@@@stlpmtx_std@@@stlpmtx_std@@@63@V?$allocator@U?$pair@$$CBV?$CryStringT@D@@V?$vector@PAVCEntityLayer@@V?$allocator@PAVCEntityLayer@@@stlpmtx_std@@@stlpmtx_std@@@stlpmtx_std@@@3@@priv@stlpmtx_std@@ABEPAU_Rb_tree_node_base@12@ABV?$CryStringT@D@@@Z 3202d0f0 f i EntitySystem.obj
 0001:0002c190       ??$_M_lower_bound@V?$CryStringT@D@@@?$_Rb_tree@V?$CryStringT@D@@U?$less@V?$CryStringT@D@@@stlpmtx_std@@U?$pair@$$CBV?$CryStringT@D@@V?$vector@PAVCEntityLayer@@V?$allocator@PAVCEntityLayer@@@stlpmtx_std@@@stlpmtx_std@@@3@U?$_Select1st@U?$pair@$$CBV?$CryStringT@D@@V?$vector@PAVCEntityLayer@@V?$allocator@PAVCEntityLayer@@@stlpmtx_std@@@stlpmtx_std@@@stlpmtx_std@@@priv@3@U?$_MapTraitsT@U?$pair@$$CBV?$CryStringT@D@@V?$vector@PAVCEntityLayer@@V?$allocator@PAVCEntityLayer@@@stlpmtx_std@@@stlpmtx_std@@@stlpmtx_std@@@63@V?$allocator@U?$pair@$$CBV?$CryStringT@D@@V?$vector@PAVCEntityLayer@@V?$allocator@PAVCEntityLayer@@@stlpmtx_std@@@stlpmtx_std@@@stlpmtx_std@@@3@@priv@stlpmtx_std@@ABEPAU_Rb_tree_node_base@12@ABV?$CryStringT@D@@@Z 3202d190 f i EntitySystem.obj
 0001:0002c1f0       ??$__make_heap@PAIVCCompareEntityIdsByClass@CEntitySystem@@IH@stlpmtx_std@@YAXPAI0VCCompareEntityIdsByClass@CEntitySystem@@0PAH@Z 3202d1f0 f i EntitySystem.obj
 0001:0002c2c0       ?IsEnd@CEntityItMap@@UAE_NXZ 3202d2c0 f i EntitySystem.obj
 0001:0002c300       ?This@CEntityItMap@@UAEPAUIEntity@@XZ 3202d300 f i EntitySystem.obj
 0001:0002c320       ?Next@CEntityItMap@@UAEPAUIEntity@@XZ 3202d320 f i EntitySystem.obj
 0001:0002c350       ?OnBeforeSpawn@CEntitySystem@@QAE_NAAUSEntitySpawnParams@@@Z 3202d350 f   EntitySystem.obj
 0001:0002c390       ?OnEntityReused@CEntitySystem@@QAEXPAUIEntity@@AAUSEntitySpawnParams@@@Z 3202d390 f   EntitySystem.obj
 0001:0002c3f0       ?GenerateEntityId@CEntitySystem@@QAEI_N@Z 3202d3f0 f   EntitySystem.obj
 0001:0002c440       ?GetEntityFromID@CEntitySystem@@QBEPAVCEntity@@I@Z 3202d440 f   EntitySystem.obj
 0001:0002c440       ?GetEntity@CEntitySystem@@UBEPAUIEntity@@I@Z 3202d440 f   EntitySystem.obj
 0001:0002c480       ?GetNumEntities@CEntitySystem@@UBEIXZ 3202d480 f   EntitySystem.obj
 0001:0002c4a0       ?QueryProximity@CEntitySystem@@UAEHAAUSEntityProximityQuery@@@Z 3202d4a0 f   EntitySystem.obj
 0001:0002c520       ?UpdateNotSeenTimeouts@CEntitySystem@@AAEXXZ 3202d520 f   EntitySystem.obj
 0001:0002c670       ?SendEventToAll@CEntitySystem@@UAEXAAUSEntityEvent@@@Z 3202d670 f   EntitySystem.obj
 0001:0002c7d0       ?RemoveEntityFromLayers@CEntitySystem@@UAEXI@Z 3202d7d0 f   EntitySystem.obj
 0001:0002c850       ?EnableDefaultLayers@CEntitySystem@@UAEX_N@Z 3202d850 f   EntitySystem.obj
 0001:0002c8e0       ?DoPrePhysicsUpdate@CEntitySystem@@AAEXXZ 3202d8e0 f   EntitySystem.obj
 0001:0002ca60       ?clear@?$_Rb_tree@PBDU?$less_stricmp@PBD@stl@@U?$pair@QBDI@stlpmtx_std@@U?$_Select1st@U?$pair@QBDI@stlpmtx_std@@@priv@4@U?$_MultimapTraitsT@U?$pair@QBDI@stlpmtx_std@@@64@V?$allocator@U?$pair@QBDI@stlpmtx_std@@@4@@priv@stlpmtx_std@@QAEXXZ 3202da60 f i EntitySystem.obj
 0001:0002ca60       ?clear@?$_Rb_tree@_KU?$less@_K@stlpmtx_std@@U?$pair@$$CB_KI@2@U?$_Select1st@U?$pair@$$CB_KI@stlpmtx_std@@@priv@2@U?$_MapTraitsT@U?$pair@$$CB_KI@stlpmtx_std@@@52@V?$allocator@U?$pair@$$CB_KI@stlpmtx_std@@@2@@priv@stlpmtx_std@@QAEXXZ 3202da60 f i EntitySystem.obj
 0001:0002ca60       ?clear@?$_Rb_tree@IU?$less@I@stlpmtx_std@@U?$pair@$$CBIPAVCEntityPool@@@2@U?$_Select1st@U?$pair@$$CBIPAVCEntityPool@@@stlpmtx_std@@@priv@2@U?$_MapTraitsT@U?$pair@$$CBIPAVCEntityPool@@@stlpmtx_std@@@52@V?$allocator@U?$pair@$$CBIPAVCEntityPool@@@stlpmtx_std@@@2@@priv@stlpmtx_std@@QAEXXZ 3202da60 f i EntityPoolManager.obj
 0001:0002ca60       ?clear@?$_Rb_tree@IU?$less@I@stlpmtx_std@@U?$pair@$$CBIPAVCEntity@@@2@U?$_Select1st@U?$pair@$$CBIPAVCEntity@@@stlpmtx_std@@@priv@2@U?$_MapTraitsT@U?$pair@$$CBIPAVCEntity@@@stlpmtx_std@@@52@V?$allocator@U?$pair@$$CBIPAVCEntity@@@stlpmtx_std@@@2@@priv@stlpmtx_std@@QAEXXZ 3202da60 f i EntitySystem.obj
 0001:0002ca60       ?clear@?$_Rb_tree@IU?$less@I@stlpmtx_std@@IU?$_Identity@I@priv@2@U?$_SetTraitsT@I@42@V?$allocator@I@2@@priv@stlpmtx_std@@QAEXXZ 3202da60 f i EntitySystem.obj
 0001:0002ca60       ?clear@?$_Rb_tree@IU?$less@I@stlpmtx_std@@U?$pair@$$CBIPAVCEntityPoolDefinition@@@2@U?$_Select1st@U?$pair@$$CBIPAVCEntityPoolDefinition@@@stlpmtx_std@@@priv@2@U?$_MapTraitsT@U?$pair@$$CBIPAVCEntityPoolDefinition@@@stlpmtx_std@@@52@V?$allocator@U?$pair@$$CBIPAVCEntityPoolDefinition@@@stlpmtx_std@@@2@@priv@stlpmtx_std@@QAEXXZ 3202da60 f i EntityPoolManager.obj
 0001:0002ca60       ?clear@?$_Rb_tree@PAUIEntityClass@@U?$less@PAUIEntityClass@@@stlpmtx_std@@U?$pair@QAUIEntityClass@@_N@3@U?$_Select1st@U?$pair@QAUIEntityClass@@_N@stlpmtx_std@@@priv@3@U?$_MapTraitsT@U?$pair@QAUIEntityClass@@_N@stlpmtx_std@@@63@V?$allocator@U?$pair@QAUIEntityClass@@_N@stlpmtx_std@@@3@@priv@stlpmtx_std@@QAEXXZ 3202da60 f i EntityPoolDefinition.obj
 0001:0002cab0       ?FreeMemory@?$HeapAllocator@UPSyncNone@stl@@$00VHeapSysAllocator@2@@stl@@QAEXPAUPageNodeHandle@12@@Z 3202dab0 f i EntitySystem.obj
 0001:0002cab0       ?FreeMemory@?$HeapAllocator@UPSyncNone@stl@@$00VGlobalHeapSysAllocator@2@@stl@@QAEXPAUPageNodeHandle@12@@Z 3202dab0 f i EntitySystem.obj
 0001:0002cbb0       ??$AddObject@PAVCEntity@@V?$allocator@PAVCEntity@@@stlpmtx_std@@@ICrySizer@@QAEXABV?$vector@PAVCEntity@@V?$allocator@PAVCEntity@@@stlpmtx_std@@@stlpmtx_std@@@Z 3202dbb0 f i EntitySystem.obj
 0001:0002cc30       ??$_M_allocate_and_copy@PAU?$Vec3_tpl@M@@@?$_Impl_vector@U?$Vec3_tpl@M@@V?$allocator@U?$Vec3_tpl@M@@@stlpmtx_std@@@priv@stlpmtx_std@@AAEPAU?$Vec3_tpl@M@@AAIPAU3@1@Z 3202dc30 f i AreaSolid.obj
 0001:0002cc30       ??$_M_allocate_and_copy@PAUSEntityTimerEvent@@@?$_Impl_vector@USEntityTimerEvent@@V?$allocator@USEntityTimerEvent@@@stlpmtx_std@@@priv@stlpmtx_std@@AAEPAUSEntityTimerEvent@@AAIPAU3@1@Z 3202dc30 f i EntitySystem.obj
 0001:0002cca0       ?MakeLower@?$CryStringT@D@@QAEAAV1@XZ 3202dca0 f i EntitySystem.obj
 0001:0002cce0       ?_M_create_node@?$_Rb_tree@_KU?$less@_K@stlpmtx_std@@U?$pair@$$CB_KI@2@U?$_Select1st@U?$pair@$$CB_KI@stlpmtx_std@@@priv@2@U?$_MapTraitsT@U?$pair@$$CB_KI@stlpmtx_std@@@52@V?$allocator@U?$pair@$$CB_KI@stlpmtx_std@@@2@@priv@stlpmtx_std@@IAEPAU_Rb_tree_node_base@23@ABU?$pair@$$CB_KI@3@@Z 3202dce0 f i EntitySystem.obj
 0001:0002cd40       ?_M_create_node@?$_Rb_tree@V?$CryStringT@D@@U?$less@V?$CryStringT@D@@@stlpmtx_std@@V1@U?$_Identity@V?$CryStringT@D@@@priv@3@U?$_SetTraitsT@V?$CryStringT@D@@@53@V?$allocator@V?$CryStringT@D@@@3@@priv@stlpmtx_std@@IAEPAU_Rb_tree_node_base@23@ABV?$CryStringT@D@@@Z 3202dd40 f i EntitySystem.obj
 0001:0002cda0       ?Allocate@?$HeapAllocator@UPSyncNone@stl@@$00VHeapSysAllocator@2@@stl@@QAEPAXII@Z 3202dda0 f i Entity.obj
 0001:0002cda0       ?Allocate@?$HeapAllocator@UPSyncNone@stl@@$00VGlobalHeapSysAllocator@2@@stl@@QAEPAXII@Z 3202dda0 f i EntitySystem.obj
 0001:0002d050       ??$__uninitialized_fill_n@PAUSEntityTimerEvent@@IU1@@priv@stlpmtx_std@@YAPAUSEntityTimerEvent@@PAU2@IABU2@@Z 3202e050 f i EntitySystem.obj
 0001:0002d050       ??$__uninitialized_fill_n@PAUSProximityEvent@@IU1@@priv@stlpmtx_std@@YAPAUSProximityEvent@@PAU2@IABU2@@Z 3202e050 f i ProximityTriggerSystem.obj
 0001:0002d0b0       ??$__unguarded_partition@PAIIVCCompareEntityIdsByClass@CEntitySystem@@@priv@stlpmtx_std@@YAPAIPAI0IVCCompareEntityIdsByClass@CEntitySystem@@@Z 3202e0b0 f i EntitySystem.obj
 0001:0002d140       ?Enable@CLogIndenter@@QAAX_NPBDZZ 3202e140 f i EntitySystem.obj
 0001:0002d1e0       ?FindEntityByName@CEntitySystem@@UBEPAUIEntity@@PBD@Z 3202e1e0 f   EntitySystem.obj
 0001:0002d290       ?PrePhysicsUpdate@CEntitySystem@@UAEXXZ 3202e290 f   EntitySystem.obj
 0001:0002d2b0       ?IsPrePhysicsActive@CEntitySystem@@QAE_NPAVCEntity@@@Z 3202e2b0 f   EntitySystem.obj
 0001:0002d300       ?OnEntityEvent@CEntitySystem@@QAEXPAVCEntity@@AAUSEntityEvent@@@Z 3202e300 f   EntitySystem.obj
 0001:0002d400       ?RemoveEntityEventListener@CEntitySystem@@UAEXIW4EEntityEvent@@PAUIEntityEventListener@@@Z 3202e400 f   EntitySystem.obj
 0001:0002d4c0       ?RemoveEntityEventListeners@CEntitySystem@@QAEXPAVCEntity@@@Z 3202e4c0 f   EntitySystem.obj
 0001:0002d5b0       ?FindEntityByGuid@CEntitySystem@@UBEIAB_K@Z 3202e5b0 f   EntitySystem.obj
 0001:0002d600       ?erase@?$set@IU?$less@I@stlpmtx_std@@V?$allocator@I@2@@stlpmtx_std@@QAEIABI@Z 3202e600 f i EntitySystem.obj
 0001:0002d660       ?_M_insert_overflow@?$_Impl_vector@PAXV?$STLGlobalAllocator@PAX@stl@@@priv@stlpmtx_std@@AAEXPAPAXABQAXABU__true_type@3@I_N@Z 3202e660 f i EntitySystem.obj
 0001:0002d780       ?_M_insert_overflow@?$_Impl_vector@UOnEventSink@CEntitySystem@@V?$STLGlobalAllocator@UOnEventSink@CEntitySystem@@@stl@@@priv@stlpmtx_std@@AAEXPAUOnEventSink@CEntitySystem@@ABU45@ABU__true_type@3@I_N@Z 3202e780 f i EntitySystem.obj
 0001:0002d8b0       ?Format@?$CryStringT@D@@QAAAAV1@PBDZZ 3202e8b0 f i EntitySystem.obj
 0001:0002d920       ??4?$_Impl_vector@PAXV?$allocator@PAX@stlpmtx_std@@@priv@stlpmtx_std@@QAEAAV012@ABV012@@Z 3202e920 f i EntitySystem.obj
 0001:0002da30       ??1?$pair@$$CBV?$CryStringT@D@@V?$vector@PAVCEntityLayer@@V?$allocator@PAVCEntityLayer@@@stlpmtx_std@@@stlpmtx_std@@@stlpmtx_std@@QAE@XZ 3202ea30 f i EntitySystem.obj
 0001:0002da90       ?_M_insert@?$_Rb_tree@IU?$less@I@stlpmtx_std@@IU?$_Identity@I@priv@2@U?$_SetTraitsT@I@42@V?$allocator@I@2@@priv@stlpmtx_std@@AAE?AU?$_Rb_tree_iterator@IU?$_SetTraitsT@I@priv@stlpmtx_std@@@23@PAU_Rb_tree_node_base@23@ABI00@Z 3202ea90 f i EntitySystem.obj
 0001:0002db90       ?_M_insert@?$_Rb_tree@PBDU?$less_stricmp@PBD@stl@@U?$pair@QBDI@stlpmtx_std@@U?$_Select1st@U?$pair@QBDI@stlpmtx_std@@@priv@4@U?$_MultimapTraitsT@U?$pair@QBDI@stlpmtx_std@@@64@V?$allocator@U?$pair@QBDI@stlpmtx_std@@@4@@priv@stlpmtx_std@@AAE?AU?$_Rb_tree_iterator@U?$pair@QBDI@stlpmtx_std@@U?$_MultimapTraitsT@U?$pair@QBDI@stlpmtx_std@@@priv@2@@23@PAU_Rb_tree_node_base@23@ABU?$pair@QBDI@3@00@Z 3202eb90 f i EntitySystem.obj
 0001:0002dc60       ?_M_insert@?$_Rb_tree@_KU?$less@_K@stlpmtx_std@@U?$pair@$$CB_KI@2@U?$_Select1st@U?$pair@$$CB_KI@stlpmtx_std@@@priv@2@U?$_MapTraitsT@U?$pair@$$CB_KI@stlpmtx_std@@@52@V?$allocator@U?$pair@$$CB_KI@stlpmtx_std@@@2@@priv@stlpmtx_std@@AAE?AU?$_Rb_tree_iterator@U?$pair@$$CB_KI@stlpmtx_std@@U?$_MapTraitsT@U?$pair@$$CB_KI@stlpmtx_std@@@priv@2@@23@PAU_Rb_tree_node_base@23@ABU?$pair@$$CB_KI@3@00@Z 3202ec60 f i EntitySystem.obj
 0001:0002dd30       ?_M_fill_insert_aux@?$_Impl_vector@IV?$allocator@I@stlpmtx_std@@@priv@stlpmtx_std@@AAEXPAIIABIABU__false_type@3@@Z 3202ed30 f i EntitySystem.obj
 0001:0002dd30       ?_M_fill_insert_aux@?$_Impl_vector@PAXV?$allocator@PAX@stlpmtx_std@@@priv@stlpmtx_std@@AAEXPAPAXIABQAXABU__false_type@3@@Z 3202ed30 f i EntitySystem.obj
 0001:0002de70       ?_M_insert@?$_Rb_tree@V?$CryStringT@D@@U?$less@V?$CryStringT@D@@@stlpmtx_std@@V1@U?$_Identity@V?$CryStringT@D@@@priv@3@U?$_SetTraitsT@V?$CryStringT@D@@@53@V?$allocator@V?$CryStringT@D@@@3@@priv@stlpmtx_std@@AAE?AU?$_Rb_tree_iterator@V?$CryStringT@D@@U?$_SetTraitsT@V?$CryStringT@D@@@priv@stlpmtx_std@@@23@PAU_Rb_tree_node_base@23@ABV?$CryStringT@D@@00@Z 3202ee70 f i EntitySystem.obj
 0001:0002df10       ??$__insertion_sort@PAIIVCCompareEntityIdsByClass@CEntitySystem@@@priv@stlpmtx_std@@YAXPAI00VCCompareEntityIdsByClass@CEntitySystem@@@Z 3202ef10 f i EntitySystem.obj
 0001:0002dfa0       ??$sort_heap@PAIVCCompareEntityIdsByClass@CEntitySystem@@@stlpmtx_std@@YAXPAI0VCCompareEntityIdsByClass@CEntitySystem@@@Z 3202efa0 f i EntitySystem.obj
 0001:0002e000       ??0?$pair@$$CBV?$CryStringT@D@@V?$vector@PAVCEntityLayer@@V?$allocator@PAVCEntityLayer@@@stlpmtx_std@@@stlpmtx_std@@@stlpmtx_std@@QAE@ABU01@@Z 3202f000 f i EntitySystem.obj
 0001:0002e090       ?UnregisterEntityGuid@CEntitySystem@@QAEXAB_K@Z 3202f090 f   EntitySystem.obj
 0001:0002e0e0       ?LoadEntityArchetype@CEntitySystem@@UAEPAUIEntityArchetype@@VXmlNodeRef@@@Z 3202f0e0 f   EntitySystem.obj
 0001:0002e220       ?FindLayer@CEntitySystem@@QAEPAVCEntityLayer@@PBD@Z 3202f220 f   EntitySystem.obj
 0001:0002e290       ?AddEntityToLayer@CEntitySystem@@UAEXPBDI@Z 3202f290 f   EntitySystem.obj
 0001:0002e2b0       ?EnableLayer@CEntitySystem@@UAEXPBD_N1@Z 3202f2b0 f   EntitySystem.obj
 0001:0002e360       ??0?$set@IU?$less@I@stlpmtx_std@@V?$allocator@I@2@@stlpmtx_std@@QAE@XZ 3202f360 f i EntitySystem.obj
 0001:0002e3a0       ?insert_unique@?$_Rb_tree@IU?$less@I@stlpmtx_std@@IU?$_Identity@I@priv@2@U?$_SetTraitsT@I@42@V?$allocator@I@2@@priv@stlpmtx_std@@QAE?AU?$pair@U?$_Rb_tree_iterator@IU?$_SetTraitsT@I@priv@stlpmtx_std@@@priv@stlpmtx_std@@_N@3@ABI@Z 3202f3a0 f i EntitySystem.obj
 0001:0002e460       ?_M_erase@?$_Rb_tree@VCTimeValue@@U?$less@VCTimeValue@@@stlpmtx_std@@U?$pair@$$CBVCTimeValue@@USEntityTimerEvent@@@3@U?$_Select1st@U?$pair@$$CBVCTimeValue@@USEntityTimerEvent@@@stlpmtx_std@@@priv@3@U?$_MultimapTraitsT@U?$pair@$$CBVCTimeValue@@USEntityTimerEvent@@@stlpmtx_std@@@63@V?$STLPoolAllocator@U?$pair@VCTimeValue@@USEntityTimerEvent@@@stlpmtx_std@@UPSyncNone@stl@@$0A@$0A@@stl@@@priv@stlpmtx_std@@AAEXPAU_Rb_tree_node_base@23@@Z 3202f460 f i EntitySystem.obj
 0001:0002e4d0       ?insert_unique@?$_Rb_tree@_KU?$less@_K@stlpmtx_std@@U?$pair@$$CB_KI@2@U?$_Select1st@U?$pair@$$CB_KI@stlpmtx_std@@@priv@2@U?$_MapTraitsT@U?$pair@$$CB_KI@stlpmtx_std@@@52@V?$allocator@U?$pair@$$CB_KI@stlpmtx_std@@@2@@priv@stlpmtx_std@@QAE?AU?$pair@U?$_Rb_tree_iterator@U?$pair@$$CB_KI@stlpmtx_std@@U?$_MapTraitsT@U?$pair@$$CB_KI@stlpmtx_std@@@priv@2@@priv@stlpmtx_std@@_N@3@ABU?$pair@$$CB_KI@3@@Z 3202f4d0 f i EntitySystem.obj
 0001:0002e5a0       ??$push_back_unique@V?$vector@PAUIAreaManagerEventListener@@V?$allocator@PAUIAreaManagerEventListener@@@stlpmtx_std@@@stlpmtx_std@@PAUIAreaManagerEventListener@@@stl@@YA_NAAV?$vector@PAUIAreaManagerEventListener@@V?$allocator@PAUIAreaManagerEventListener@@@stlpmtx_std@@@stlpmtx_std@@ABQAUIAreaManagerEventListener@@@Z 3202f5a0 f i AreaManager.obj
 0001:0002e5a0       ??$push_back_unique@V?$vector@PAVCEntity@@V?$allocator@PAVCEntity@@@stlpmtx_std@@@stlpmtx_std@@PAVCEntity@@@stl@@YA_NAAV?$vector@PAVCEntity@@V?$allocator@PAVCEntity@@@stlpmtx_std@@@stlpmtx_std@@ABQAVCEntity@@@Z 3202f5a0 f i EntitySystem.obj
 0001:0002e5a0       ??$push_back_unique@V?$vector@IV?$allocator@I@stlpmtx_std@@@stlpmtx_std@@I@stl@@YA_NAAV?$vector@IV?$allocator@I@stlpmtx_std@@@stlpmtx_std@@ABI@Z 3202f5a0 f i SoundProxy.obj
 0001:0002e610       ?insert_unique@?$_Rb_tree@V?$CryStringT@D@@U?$less@V?$CryStringT@D@@@stlpmtx_std@@V1@U?$_Identity@V?$CryStringT@D@@@priv@3@U?$_SetTraitsT@V?$CryStringT@D@@@53@V?$allocator@V?$CryStringT@D@@@3@@priv@stlpmtx_std@@QAE?AU?$pair@U?$_Rb_tree_iterator@V?$CryStringT@D@@U?$_SetTraitsT@V?$CryStringT@D@@@priv@stlpmtx_std@@@priv@stlpmtx_std@@_N@3@ABV?$CryStringT@D@@@Z 3202f610 f i EntitySystem.obj
 0001:0002e790       ??0?$pair@$$CBV?$CryStringT@D@@V?$vector@PAVCEntityLayer@@V?$allocator@PAVCEntityLayer@@@stlpmtx_std@@@stlpmtx_std@@@stlpmtx_std@@QAE@ABV?$CryStringT@D@@ABV?$vector@PAVCEntityLayer@@V?$allocator@PAVCEntityLayer@@@stlpmtx_std@@@1@@Z 3202f790 f i EntitySystem.obj
 0001:0002e820       ??$__destroy_range_aux@V?$reverse_iterator@PAUSEntry@SLayerPakStats@@@stlpmtx_std@@USEntry@SLayerPakStats@@@stlpmtx_std@@YAXV?$reverse_iterator@PAUSEntry@SLayerPakStats@@@0@0PAUSEntry@SLayerPakStats@@ABU__false_type@0@@Z 3202f820 f i EntitySystem.obj
 0001:0002e8a0       ?_M_create_node@?$_Rb_tree@V?$CryStringT@D@@U?$less@V?$CryStringT@D@@@stlpmtx_std@@U?$pair@$$CBV?$CryStringT@D@@PAUIEntityClass@@@3@U?$_Select1st@U?$pair@$$CBV?$CryStringT@D@@PAUIEntityClass@@@stlpmtx_std@@@priv@3@U?$_MapTraitsT@U?$pair@$$CBV?$CryStringT@D@@PAUIEntityClass@@@stlpmtx_std@@@63@V?$allocator@U?$pair@$$CBV?$CryStringT@D@@PAUIEntityClass@@@stlpmtx_std@@@3@@priv@stlpmtx_std@@IAEPAU_Rb_tree_node_base@23@ABU?$pair@$$CBV?$CryStringT@D@@PAUIEntityClass@@@3@@Z 3202f8a0 f i EntityClassRegistry.obj
 0001:0002e8a0       ?_M_create_node@?$_Rb_tree@V?$CryStringT@D@@U?$less@V?$CryStringT@D@@@stlpmtx_std@@U?$pair@$$CBV?$CryStringT@D@@H@3@U?$_Select1st@U?$pair@$$CBV?$CryStringT@D@@H@stlpmtx_std@@@priv@3@U?$_MapTraitsT@U?$pair@$$CBV?$CryStringT@D@@H@stlpmtx_std@@@63@V?$allocator@U?$pair@$$CBV?$CryStringT@D@@H@stlpmtx_std@@@3@@priv@stlpmtx_std@@IAEPAU_Rb_tree_node_base@23@ABU?$pair@$$CBV?$CryStringT@D@@H@3@@Z 3202f8a0 f i EntityCVars.obj
 0001:0002e8a0       ?_M_create_node@?$_Rb_tree@V?$CryStringT@D@@U?$less@V?$CryStringT@D@@@stlpmtx_std@@U?$pair@$$CBV?$CryStringT@D@@PAVCEntityLayer@@@3@U?$_Select1st@U?$pair@$$CBV?$CryStringT@D@@PAVCEntityLayer@@@stlpmtx_std@@@priv@3@U?$_MapTraitsT@U?$pair@$$CBV?$CryStringT@D@@PAVCEntityLayer@@@stlpmtx_std@@@63@V?$allocator@U?$pair@$$CBV?$CryStringT@D@@PAVCEntityLayer@@@stlpmtx_std@@@3@@priv@stlpmtx_std@@IAEPAU_Rb_tree_node_base@23@ABU?$pair@$$CBV?$CryStringT@D@@PAVCEntityLayer@@@3@@Z 3202f8a0 f i EntitySystem.obj
 0001:0002e910       ??$__partial_sort@PAIIVCCompareEntityIdsByClass@CEntitySystem@@@priv@stlpmtx_std@@YAXPAI000VCCompareEntityIdsByClass@CEntitySystem@@@Z 3202f910 f i EntitySystem.obj
 0001:0002e9c0       ?RemoveSink@CEntitySystem@@UAEXPAUIEntitySystemSink@@@Z 3202f9c0 f   EntitySystem.obj
 0001:0002eb90       ?GetMemoryStatistics@CEntitySystem@@UBEXPAVICrySizer@@@Z 3202fb90 f   EntitySystem.obj
 0001:0002ee00       ?LoadLayers@CEntitySystem@@UAEXPBD@Z 3202fe00 f   EntitySystem.obj
 0001:0002f1a0       ?GetLayerForEntity@CEntitySystem@@QAEPAVCEntityLayer@@I@Z 320301a0 f   EntitySystem.obj
 0001:0002f270       ?ShouldSerializedEntity@CEntitySystem@@UAE_NPAUIEntity@@@Z 32030270 f   EntitySystem.obj
 0001:0002f370       ?PurgeDeferredCollisionEvents@CEntitySystem@@UAEX_N@Z 32030370 f   EntitySystem.obj
 0001:0002f510       ?erase@?$_Rb_tree@VCTimeValue@@U?$less@VCTimeValue@@@stlpmtx_std@@U?$pair@$$CBVCTimeValue@@USEntityTimerEvent@@@3@U?$_Select1st@U?$pair@$$CBVCTimeValue@@USEntityTimerEvent@@@stlpmtx_std@@@priv@3@U?$_MultimapTraitsT@U?$pair@$$CBVCTimeValue@@USEntityTimerEvent@@@stlpmtx_std@@@63@V?$STLPoolAllocator@U?$pair@VCTimeValue@@USEntityTimerEvent@@@stlpmtx_std@@UPSyncNone@stl@@$0A@$0A@@stl@@@priv@stlpmtx_std@@QAEXU?$_Rb_tree_iterator@U?$pair@$$CBVCTimeValue@@USEntityTimerEvent@@@stlpmtx_std@@U?$_MultimapTraitsT@U?$pair@$$CBVCTimeValue@@USEntityTimerEvent@@@stlpmtx_std@@@priv@2@@23@@Z 32030510 f i EntitySystem.obj
 0001:0002f580       ?_M_erase@?$_Rb_tree@V?$CryStringT@D@@U?$less@V?$CryStringT@D@@@stlpmtx_std@@V1@U?$_Identity@V?$CryStringT@D@@@priv@3@U?$_SetTraitsT@V?$CryStringT@D@@@53@V?$allocator@V?$CryStringT@D@@@3@@priv@stlpmtx_std@@AAEXPAU_Rb_tree_node_base@23@@Z 32030580 f i EntitySystem.obj
 0001:0002f580       ?_M_erase@?$_Rb_tree@V?$CryStringT@D@@U?$less@V?$CryStringT@D@@@stlpmtx_std@@U?$pair@$$CBV?$CryStringT@D@@PAVCEntityLayer@@@3@U?$_Select1st@U?$pair@$$CBV?$CryStringT@D@@PAVCEntityLayer@@@stlpmtx_std@@@priv@3@U?$_MapTraitsT@U?$pair@$$CBV?$CryStringT@D@@PAVCEntityLayer@@@stlpmtx_std@@@63@V?$allocator@U?$pair@$$CBV?$CryStringT@D@@PAVCEntityLayer@@@stlpmtx_std@@@3@@priv@stlpmtx_std@@AAEXPAU_Rb_tree_node_base@23@@Z 32030580 f i EntitySystem.obj
 0001:0002f580       ?_M_erase@?$_Rb_tree@V?$CryStringT@D@@U?$less@V?$CryStringT@D@@@stlpmtx_std@@U?$pair@$$CBV?$CryStringT@D@@H@3@U?$_Select1st@U?$pair@$$CBV?$CryStringT@D@@H@stlpmtx_std@@@priv@3@U?$_MapTraitsT@U?$pair@$$CBV?$CryStringT@D@@H@stlpmtx_std@@@63@V?$allocator@U?$pair@$$CBV?$CryStringT@D@@H@stlpmtx_std@@@3@@priv@stlpmtx_std@@AAEXPAU_Rb_tree_node_base@23@@Z 32030580 f i EntityCVars.obj
 0001:0002f580       ?_M_erase@?$_Rb_tree@V?$CryStringT@D@@U?$less@V?$CryStringT@D@@@stlpmtx_std@@U?$pair@$$CBV?$CryStringT@D@@PAUIEntityClass@@@3@U?$_Select1st@U?$pair@$$CBV?$CryStringT@D@@PAUIEntityClass@@@stlpmtx_std@@@priv@3@U?$_MapTraitsT@U?$pair@$$CBV?$CryStringT@D@@PAUIEntityClass@@@stlpmtx_std@@@63@V?$allocator@U?$pair@$$CBV?$CryStringT@D@@PAUIEntityClass@@@stlpmtx_std@@@3@@priv@stlpmtx_std@@AAEXPAU_Rb_tree_node_base@23@@Z 32030580 f i EntityClassRegistry.obj
 0001:0002f5e0       ?GetOrCreateAllocator@?$STLPoolAllocatorStatic@$0CI@UPSyncNone@stl@@$0A@$0A@U?$_Rb_tree_node@U?$pair@$$CBVCTimeValue@@USEntityTimerEvent@@@stlpmtx_std@@@priv@stlpmtx_std@@@stl@@SAPAV?$SizePoolAllocator@V?$HeapAllocator@UPSyncNone@stl@@$00VGlobalHeapSysAllocator@2@@stl@@@2@XZ 320305e0 f i EntitySystem.obj
 0001:0002f640       ?_M_insert@?$_Rb_tree@V?$CryStringT@D@@U?$less@V?$CryStringT@D@@@stlpmtx_std@@U?$pair@$$CBV?$CryStringT@D@@PAUIEntityClass@@@3@U?$_Select1st@U?$pair@$$CBV?$CryStringT@D@@PAUIEntityClass@@@stlpmtx_std@@@priv@3@U?$_MapTraitsT@U?$pair@$$CBV?$CryStringT@D@@PAUIEntityClass@@@stlpmtx_std@@@63@V?$allocator@U?$pair@$$CBV?$CryStringT@D@@PAUIEntityClass@@@stlpmtx_std@@@3@@priv@stlpmtx_std@@AAE?AU?$_Rb_tree_iterator@U?$pair@$$CBV?$CryStringT@D@@PAUIEntityClass@@@stlpmtx_std@@U?$_MapTraitsT@U?$pair@$$CBV?$CryStringT@D@@PAUIEntityClass@@@stlpmtx_std@@@priv@2@@23@PAU_Rb_tree_node_base@23@ABU?$pair@$$CBV?$CryStringT@D@@PAUIEntityClass@@@3@00@Z 32030640 f i EntityClassRegistry.obj
 0001:0002f640       ?_M_insert@?$_Rb_tree@V?$CryStringT@D@@U?$less@V?$CryStringT@D@@@stlpmtx_std@@U?$pair@$$CBV?$CryStringT@D@@PAVCEntityLayer@@@3@U?$_Select1st@U?$pair@$$CBV?$CryStringT@D@@PAVCEntityLayer@@@stlpmtx_std@@@priv@3@U?$_MapTraitsT@U?$pair@$$CBV?$CryStringT@D@@PAVCEntityLayer@@@stlpmtx_std@@@63@V?$allocator@U?$pair@$$CBV?$CryStringT@D@@PAVCEntityLayer@@@stlpmtx_std@@@3@@priv@stlpmtx_std@@AAE?AU?$_Rb_tree_iterator@U?$pair@$$CBV?$CryStringT@D@@PAVCEntityLayer@@@stlpmtx_std@@U?$_MapTraitsT@U?$pair@$$CBV?$CryStringT@D@@PAVCEntityLayer@@@stlpmtx_std@@@priv@2@@23@PAU_Rb_tree_node_base@23@ABU?$pair@$$CBV?$CryStringT@D@@PAVCEntityLayer@@@3@00@Z 32030640 f i EntitySystem.obj
 0001:0002f640       ?_M_insert@?$_Rb_tree@V?$CryStringT@D@@U?$less@V?$CryStringT@D@@@stlpmtx_std@@U?$pair@$$CBV?$CryStringT@D@@H@3@U?$_Select1st@U?$pair@$$CBV?$CryStringT@D@@H@stlpmtx_std@@@priv@3@U?$_MapTraitsT@U?$pair@$$CBV?$CryStringT@D@@H@stlpmtx_std@@@63@V?$allocator@U?$pair@$$CBV?$CryStringT@D@@H@stlpmtx_std@@@3@@priv@stlpmtx_std@@AAE?AU?$_Rb_tree_iterator@U?$pair@$$CBV?$CryStringT@D@@H@stlpmtx_std@@U?$_MapTraitsT@U?$pair@$$CBV?$CryStringT@D@@H@stlpmtx_std@@@priv@2@@23@PAU_Rb_tree_node_base@23@ABU?$pair@$$CBV?$CryStringT@D@@H@3@00@Z 32030640 f i EntityCVars.obj
 0001:0002f6e0       ?insert_unique@?$_Rb_tree@V?$CryStringT@D@@U?$less@V?$CryStringT@D@@@stlpmtx_std@@U?$pair@$$CBV?$CryStringT@D@@H@3@U?$_Select1st@U?$pair@$$CBV?$CryStringT@D@@H@stlpmtx_std@@@priv@3@U?$_MapTraitsT@U?$pair@$$CBV?$CryStringT@D@@H@stlpmtx_std@@@63@V?$allocator@U?$pair@$$CBV?$CryStringT@D@@H@stlpmtx_std@@@3@@priv@stlpmtx_std@@QAE?AU?$pair@U?$_Rb_tree_iterator@U?$pair@$$CBV?$CryStringT@D@@H@stlpmtx_std@@U?$_MapTraitsT@U?$pair@$$CBV?$CryStringT@D@@H@stlpmtx_std@@@priv@2@@priv@stlpmtx_std@@_N@3@ABU?$pair@$$CBV?$CryStringT@D@@H@3@@Z 320306e0 f i EntityCVars.obj
 0001:0002f6e0       ?insert_unique@?$_Rb_tree@V?$CryStringT@D@@U?$less@V?$CryStringT@D@@@stlpmtx_std@@U?$pair@$$CBV?$CryStringT@D@@PAVCEntityLayer@@@3@U?$_Select1st@U?$pair@$$CBV?$CryStringT@D@@PAVCEntityLayer@@@stlpmtx_std@@@priv@3@U?$_MapTraitsT@U?$pair@$$CBV?$CryStringT@D@@PAVCEntityLayer@@@stlpmtx_std@@@63@V?$allocator@U?$pair@$$CBV?$CryStringT@D@@PAVCEntityLayer@@@stlpmtx_std@@@3@@priv@stlpmtx_std@@QAE?AU?$pair@U?$_Rb_tree_iterator@U?$pair@$$CBV?$CryStringT@D@@PAVCEntityLayer@@@stlpmtx_std@@U?$_MapTraitsT@U?$pair@$$CBV?$CryStringT@D@@PAVCEntityLayer@@@stlpmtx_std@@@priv@2@@priv@stlpmtx_std@@_N@3@ABU?$pair@$$CBV?$CryStringT@D@@PAVCEntityLayer@@@3@@Z 320306e0 f i EntitySystem.obj
 0001:0002f6e0       ?insert_unique@?$_Rb_tree@V?$CryStringT@D@@U?$less@V?$CryStringT@D@@@stlpmtx_std@@U?$pair@$$CBV?$CryStringT@D@@PAUIEntityClass@@@3@U?$_Select1st@U?$pair@$$CBV?$CryStringT@D@@PAUIEntityClass@@@stlpmtx_std@@@priv@3@U?$_MapTraitsT@U?$pair@$$CBV?$CryStringT@D@@PAUIEntityClass@@@stlpmtx_std@@@63@V?$allocator@U?$pair@$$CBV?$CryStringT@D@@PAUIEntityClass@@@stlpmtx_std@@@3@@priv@stlpmtx_std@@QAE?AU?$pair@U?$_Rb_tree_iterator@U?$pair@$$CBV?$CryStringT@D@@PAUIEntityClass@@@stlpmtx_std@@U?$_MapTraitsT@U?$pair@$$CBV?$CryStringT@D@@PAUIEntityClass@@@stlpmtx_std@@@priv@2@@priv@stlpmtx_std@@_N@3@ABU?$pair@$$CBV?$CryStringT@D@@PAUIEntityClass@@@3@@Z 320306e0 f i EntityClassRegistry.obj
 0001:0002f860       ??$_Copy_Construct_aux@U?$pair@QAUIEntityClass@@V?$vector@U?$pair@II@stlpmtx_std@@V?$allocator@U?$pair@II@stlpmtx_std@@@2@@stlpmtx_std@@@stlpmtx_std@@@stlpmtx_std@@YAXPAU?$pair@QAUIEntityClass@@V?$vector@U?$pair@II@stlpmtx_std@@V?$allocator@U?$pair@II@stlpmtx_std@@@2@@stlpmtx_std@@@0@ABU10@ABU__false_type@0@@Z 32030860 f i EntitySystem.obj
 0001:0002f8d0       ?Unload@CEntitySystem@@UAEXXZ 320308d0 f   EntitySystem.obj
 0001:0002f980       ?AddSink@CEntitySystem@@UAEXPAUIEntitySystemSink@@I_K@Z 32030980 f   EntitySystem.obj
 0001:0002fa80       ?ActivatePrePhysicsUpdateForEntity@CEntitySystem@@QAEXPAVCEntity@@_N@Z 32030a80 f   EntitySystem.obj
 0001:0002fbe0       ?AddEntityEventListener@CEntitySystem@@UAEXIW4EEntityEvent@@PAUIEntityEventListener@@@Z 32030be0 f   EntitySystem.obj
 0001:0002fc50       ?RegisterEntityGuid@CEntitySystem@@QAEXAB_KI@Z 32030c50 f   EntitySystem.obj
 0001:0002fcb0       ?ChangeEntityName@CEntitySystem@@QAEXPAVCEntity@@PBD@Z 32030cb0 f   EntitySystem.obj
 0001:0002fe40       ?resize@?$_Impl_vector@PAXV?$allocator@PAX@stlpmtx_std@@@priv@stlpmtx_std@@QAEXIABQAX@Z 32030e40 f i EntitySystem.obj
 0001:0002fe40       ?resize@?$_Impl_vector@IV?$allocator@I@stlpmtx_std@@@priv@stlpmtx_std@@QAEXIABI@Z 32030e40 f i EntitySystem.obj
 0001:0002fee0       ?erase@?$_Rb_tree@VCTimeValue@@U?$less@VCTimeValue@@@stlpmtx_std@@U?$pair@$$CBVCTimeValue@@USEntityTimerEvent@@@3@U?$_Select1st@U?$pair@$$CBVCTimeValue@@USEntityTimerEvent@@@stlpmtx_std@@@priv@3@U?$_MultimapTraitsT@U?$pair@$$CBVCTimeValue@@USEntityTimerEvent@@@stlpmtx_std@@@63@V?$STLPoolAllocator@U?$pair@VCTimeValue@@USEntityTimerEvent@@@stlpmtx_std@@UPSyncNone@stl@@$0A@$0A@@stl@@@priv@stlpmtx_std@@QAEXU?$_Rb_tree_iterator@U?$pair@$$CBVCTimeValue@@USEntityTimerEvent@@@stlpmtx_std@@U?$_MultimapTraitsT@U?$pair@$$CBVCTimeValue@@USEntityTimerEvent@@@stlpmtx_std@@@priv@2@@23@0@Z 32030ee0 f i EntitySystem.obj
 0001:0002ffe0       ?_M_erase@?$_Rb_tree@V?$CryStringT@D@@U?$less@V?$CryStringT@D@@@stlpmtx_std@@U?$pair@$$CBV?$CryStringT@D@@V?$vector@PAVCEntityLayer@@V?$allocator@PAVCEntityLayer@@@stlpmtx_std@@@stlpmtx_std@@@3@U?$_Select1st@U?$pair@$$CBV?$CryStringT@D@@V?$vector@PAVCEntityLayer@@V?$allocator@PAVCEntityLayer@@@stlpmtx_std@@@stlpmtx_std@@@stlpmtx_std@@@priv@3@U?$_MapTraitsT@U?$pair@$$CBV?$CryStringT@D@@V?$vector@PAVCEntityLayer@@V?$allocator@PAVCEntityLayer@@@stlpmtx_std@@@stlpmtx_std@@@stlpmtx_std@@@63@V?$allocator@U?$pair@$$CBV?$CryStringT@D@@V?$vector@PAVCEntityLayer@@V?$allocator@PAVCEntityLayer@@@stlpmtx_std@@@stlpmtx_std@@@stlpmtx_std@@@3@@priv@stlpmtx_std@@AAEXPAU_Rb_tree_node_base@23@@Z 32030fe0 f i EntitySystem.obj
 0001:000300d0       ??$__introsort_loop@PAIIHVCCompareEntityIdsByClass@CEntitySystem@@@priv@stlpmtx_std@@YAXPAI00HVCCompareEntityIdsByClass@CEntitySystem@@@Z 320310d0 f i EntitySystem.obj
 0001:00030160       ?_M_create_node@?$_Rb_tree@V?$CryStringT@D@@U?$less@V?$CryStringT@D@@@stlpmtx_std@@U?$pair@$$CBV?$CryStringT@D@@V?$vector@PAVCEntityLayer@@V?$allocator@PAVCEntityLayer@@@stlpmtx_std@@@stlpmtx_std@@@3@U?$_Select1st@U?$pair@$$CBV?$CryStringT@D@@V?$vector@PAVCEntityLayer@@V?$allocator@PAVCEntityLayer@@@stlpmtx_std@@@stlpmtx_std@@@stlpmtx_std@@@priv@3@U?$_MapTraitsT@U?$pair@$$CBV?$CryStringT@D@@V?$vector@PAVCEntityLayer@@V?$allocator@PAVCEntityLayer@@@stlpmtx_std@@@stlpmtx_std@@@stlpmtx_std@@@63@V?$allocator@U?$pair@$$CBV?$CryStringT@D@@V?$vector@PAVCEntityLayer@@V?$allocator@PAVCEntityLayer@@@stlpmtx_std@@@stlpmtx_std@@@stlpmtx_std@@@3@@priv@stlpmtx_std@@IAEPAU_Rb_tree_node_base@23@ABU?$pair@$$CBV?$CryStringT@D@@V?$vector@PAVCEntityLayer@@V?$allocator@PAVCEntityLayer@@@stlpmtx_std@@@stlpmtx_std@@@3@@Z 32031160 f i EntitySystem.obj
 0001:000301b0       ??1CEntityArchetypeManager@@QAE@XZ 320311b0 f i EntitySystem.obj
 0001:00030230       ?SpawnEntity@CEntitySystem@@UAEPAUIEntity@@AAUSEntitySpawnParams@@_N@Z 32031230 f   EntitySystem.obj
 0001:00030620       ?RemoveEntityFromActiveList@CEntitySystem@@AAEXPAVCEntity@@@Z 32031620 f   EntitySystem.obj
 0001:00030700       ?RemoveTimerEvent@CEntitySystem@@QAEXIH@Z 32031700 f   EntitySystem.obj
 0001:00030810       ?ActivateEntity@CEntitySystem@@QAEXPAVCEntity@@_N@Z 32031810 f   EntitySystem.obj
 0001:00030940       ??$sort@PAIVCCompareEntityIdsByClass@CEntitySystem@@@stlpmtx_std@@YAXPAI0VCCompareEntityIdsByClass@CEntitySystem@@@Z 32031940 f i EntitySystem.obj
 0001:000309c0       ?_M_insert@?$_Rb_tree@V?$CryStringT@D@@U?$less@V?$CryStringT@D@@@stlpmtx_std@@U?$pair@$$CBV?$CryStringT@D@@V?$vector@PAVCEntityLayer@@V?$allocator@PAVCEntityLayer@@@stlpmtx_std@@@stlpmtx_std@@@3@U?$_Select1st@U?$pair@$$CBV?$CryStringT@D@@V?$vector@PAVCEntityLayer@@V?$allocator@PAVCEntityLayer@@@stlpmtx_std@@@stlpmtx_std@@@stlpmtx_std@@@priv@3@U?$_MapTraitsT@U?$pair@$$CBV?$CryStringT@D@@V?$vector@PAVCEntityLayer@@V?$allocator@PAVCEntityLayer@@@stlpmtx_std@@@stlpmtx_std@@@stlpmtx_std@@@63@V?$allocator@U?$pair@$$CBV?$CryStringT@D@@V?$vector@PAVCEntityLayer@@V?$allocator@PAVCEntityLayer@@@stlpmtx_std@@@stlpmtx_std@@@stlpmtx_std@@@3@@priv@stlpmtx_std@@AAE?AU?$_Rb_tree_iterator@U?$pair@$$CBV?$CryStringT@D@@V?$vector@PAVCEntityLayer@@V?$allocator@PAVCEntityLayer@@@stlpmtx_std@@@stlpmtx_std@@@stlpmtx_std@@U?$_MapTraitsT@U?$pair@$$CBV?$CryStringT@D@@V?$vector@PAVCEntityLayer@@V?$allocator@PAVCEntityLayer@@@stlpmtx_std@@@stlpmtx_std@@@stlpmtx_std@@@priv@2@@23@PAU_Rb_tree_node_base@23@ABU?$pair@$$CBV?$CryStringT@D@@V?$vector@PAVCEntityLayer@@V?$allocator@PAVCEntityLayer@@@stlpmtx_std@@@stlpmtx_std@@@3@00@Z 320319c0 f i EntitySystem.obj
 0001:00030a90       ?insert_unique@?$_Rb_tree@V?$CryStringT@D@@U?$less@V?$CryStringT@D@@@stlpmtx_std@@U?$pair@$$CBV?$CryStringT@D@@V?$vector@PAVCEntityLayer@@V?$allocator@PAVCEntityLayer@@@stlpmtx_std@@@stlpmtx_std@@@3@U?$_Select1st@U?$pair@$$CBV?$CryStringT@D@@V?$vector@PAVCEntityLayer@@V?$allocator@PAVCEntityLayer@@@stlpmtx_std@@@stlpmtx_std@@@stlpmtx_std@@@priv@3@U?$_MapTraitsT@U?$pair@$$CBV?$CryStringT@D@@V?$vector@PAVCEntityLayer@@V?$allocator@PAVCEntityLayer@@@stlpmtx_std@@@stlpmtx_std@@@stlpmtx_std@@@63@V?$allocator@U?$pair@$$CBV?$CryStringT@D@@V?$vector@PAVCEntityLayer@@V?$allocator@PAVCEntityLayer@@@stlpmtx_std@@@stlpmtx_std@@@stlpmtx_std@@@3@@priv@stlpmtx_std@@QAE?AU?$pair@U?$_Rb_tree_iterator@U?$pair@$$CBV?$CryStringT@D@@V?$vector@PAVCEntityLayer@@V?$allocator@PAVCEntityLayer@@@stlpmtx_std@@@stlpmtx_std@@@stlpmtx_std@@U?$_MapTraitsT@U?$pair@$$CBV?$CryStringT@D@@V?$vector@PAVCEntityLayer@@V?$allocator@PAVCEntityLayer@@@stlpmtx_std@@@stlpmtx_std@@@stlpmtx_std@@@priv@2@@priv@stlpmtx_std@@_N@3@ABU?$pair@$$CBV?$CryStringT@D@@V?$vector@PAVCEntityLayer@@V?$allocator@PAVCEntityLayer@@@stlpmtx_std@@@stlpmtx_std@@@3@@Z 32031a90 f i EntitySystem.obj
 0001:00030bb0       ?Init@CEntitySystem@@QAE_NPAUISystem@@@Z 32031bb0 f   EntitySystem.obj
 0001:00030ce0       ?ResetEntityId@CEntitySystem@@QAE_NPAVCEntity@@I@Z 32031ce0 f   EntitySystem.obj
 0001:00030d90       ?DeleteEntity@CEntitySystem@@AAEXPAVCEntity@@@Z 32031d90 f   EntitySystem.obj
 0001:00030f90       ?RemoveEntity@CEntitySystem@@UAEXI_N@Z 32031f90 f   EntitySystem.obj
 0001:00031270       ?UpdateDeletedEntities@CEntitySystem@@AAEXXZ 32032270 f   EntitySystem.obj
 0001:00031320       ?UpdateTempActiveEntities@CEntitySystem@@AAEXXZ 32032320 f   EntitySystem.obj
 0001:000313f0       ?DoUpdateLoop@CEntitySystem@@AAEXM@Z 320323f0 f   EntitySystem.obj
 0001:00031b90       ?UpdateTimers@CEntitySystem@@AAEXXZ 32032b90 f   EntitySystem.obj
 0001:00031e10       ?DumpEntity@CEntitySystem@@AAEXPAUIEntity@@@Z 32032e10 f   EntitySystem.obj
 0001:00032340       ?DeletePendingEntities@CEntitySystem@@UAEXXZ 32033340 f   EntitySystem.obj
 0001:00032350       ?ClearLayers@CEntitySystem@@UAEXXZ 32033350 f   EntitySystem.obj
 0001:00032440       ?insert_unique@?$_Rb_tree@V?$CryStringT@D@@U?$less@V?$CryStringT@D@@@stlpmtx_std@@U?$pair@$$CBV?$CryStringT@D@@V?$vector@PAVCEntityLayer@@V?$allocator@PAVCEntityLayer@@@stlpmtx_std@@@stlpmtx_std@@@3@U?$_Select1st@U?$pair@$$CBV?$CryStringT@D@@V?$vector@PAVCEntityLayer@@V?$allocator@PAVCEntityLayer@@@stlpmtx_std@@@stlpmtx_std@@@stlpmtx_std@@@priv@3@U?$_MapTraitsT@U?$pair@$$CBV?$CryStringT@D@@V?$vector@PAVCEntityLayer@@V?$allocator@PAVCEntityLayer@@@stlpmtx_std@@@stlpmtx_std@@@stlpmtx_std@@@63@V?$allocator@U?$pair@$$CBV?$CryStringT@D@@V?$vector@PAVCEntityLayer@@V?$allocator@PAVCEntityLayer@@@stlpmtx_std@@@stlpmtx_std@@@stlpmtx_std@@@3@@priv@stlpmtx_std@@QAE?AU?$_Rb_tree_iterator@U?$pair@$$CBV?$CryStringT@D@@V?$vector@PAVCEntityLayer@@V?$allocator@PAVCEntityLayer@@@stlpmtx_std@@@stlpmtx_std@@@stlpmtx_std@@U?$_MapTraitsT@U?$pair@$$CBV?$CryStringT@D@@V?$vector@PAVCEntityLayer@@V?$allocator@PAVCEntityLayer@@@stlpmtx_std@@@stlpmtx_std@@@stlpmtx_std@@@priv@2@@23@U423@ABU?$pair@$$CBV?$CryStringT@D@@V?$vector@PAVCEntityLayer@@V?$allocator@PAVCEntityLayer@@@stlpmtx_std@@@stlpmtx_std@@@3@@Z 32033440 f i EntitySystem.obj
 0001:00032710       ?_M_create_node@?$_Rb_tree@VCTimeValue@@U?$less@VCTimeValue@@@stlpmtx_std@@U?$pair@$$CBVCTimeValue@@USEntityTimerEvent@@@3@U?$_Select1st@U?$pair@$$CBVCTimeValue@@USEntityTimerEvent@@@stlpmtx_std@@@priv@3@U?$_MultimapTraitsT@U?$pair@$$CBVCTimeValue@@USEntityTimerEvent@@@stlpmtx_std@@@63@V?$STLPoolAllocator@U?$pair@VCTimeValue@@USEntityTimerEvent@@@stlpmtx_std@@UPSyncNone@stl@@$0A@$0A@@stl@@@priv@stlpmtx_std@@IAEPAU_Rb_tree_node_base@23@ABU?$pair@$$CBVCTimeValue@@USEntityTimerEvent@@@3@@Z 32033710 f i EntitySystem.obj
 0001:000327a0       ?_M_insert@?$_Rb_tree@PAUIEntityClass@@U?$less@PAUIEntityClass@@@stlpmtx_std@@U?$pair@QAUIEntityClass@@V?$vector@U?$pair@II@stlpmtx_std@@V?$allocator@U?$pair@II@stlpmtx_std@@@2@@stlpmtx_std@@@3@U?$_Select1st@U?$pair@QAUIEntityClass@@V?$vector@U?$pair@II@stlpmtx_std@@V?$allocator@U?$pair@II@stlpmtx_std@@@2@@stlpmtx_std@@@stlpmtx_std@@@priv@3@U?$_MapTraitsT@U?$pair@QAUIEntityClass@@V?$vector@U?$pair@II@stlpmtx_std@@V?$allocator@U?$pair@II@stlpmtx_std@@@2@@stlpmtx_std@@@stlpmtx_std@@@63@V?$allocator@U?$pair@QAUIEntityClass@@V?$vector@U?$pair@II@stlpmtx_std@@V?$allocator@U?$pair@II@stlpmtx_std@@@2@@stlpmtx_std@@@stlpmtx_std@@@3@@priv@stlpmtx_std@@AAE?AU?$_Rb_tree_iterator@U?$pair@QAUIEntityClass@@V?$vector@U?$pair@II@stlpmtx_std@@V?$allocator@U?$pair@II@stlpmtx_std@@@2@@stlpmtx_std@@@stlpmtx_std@@U?$_MapTraitsT@U?$pair@QAUIEntityClass@@V?$vector@U?$pair@II@stlpmtx_std@@V?$allocator@U?$pair@II@stlpmtx_std@@@2@@stlpmtx_std@@@stlpmtx_std@@@priv@2@@23@PAU_Rb_tree_node_base@23@ABU?$pair@QAUIEntityClass@@V?$vector@U?$pair@II@stlpmtx_std@@V?$allocator@U?$pair@II@stlpmtx_std@@@2@@stlpmtx_std@@@3@00@Z 320337a0 f i EntitySystem.obj
 0001:000328c0       ?insert_unique@?$_Rb_tree@PAUIEntityClass@@U?$less@PAUIEntityClass@@@stlpmtx_std@@U?$pair@QAUIEntityClass@@V?$vector@U?$pair@II@stlpmtx_std@@V?$allocator@U?$pair@II@stlpmtx_std@@@2@@stlpmtx_std@@@3@U?$_Select1st@U?$pair@QAUIEntityClass@@V?$vector@U?$pair@II@stlpmtx_std@@V?$allocator@U?$pair@II@stlpmtx_std@@@2@@stlpmtx_std@@@stlpmtx_std@@@priv@3@U?$_MapTraitsT@U?$pair@QAUIEntityClass@@V?$vector@U?$pair@II@stlpmtx_std@@V?$allocator@U?$pair@II@stlpmtx_std@@@2@@stlpmtx_std@@@stlpmtx_std@@@63@V?$allocator@U?$pair@QAUIEntityClass@@V?$vector@U?$pair@II@stlpmtx_std@@V?$allocator@U?$pair@II@stlpmtx_std@@@2@@stlpmtx_std@@@stlpmtx_std@@@3@@priv@stlpmtx_std@@QAE?AU?$pair@U?$_Rb_tree_iterator@U?$pair@QAUIEntityClass@@V?$vector@U?$pair@II@stlpmtx_std@@V?$allocator@U?$pair@II@stlpmtx_std@@@2@@stlpmtx_std@@@stlpmtx_std@@U?$_MapTraitsT@U?$pair@QAUIEntityClass@@V?$vector@U?$pair@II@stlpmtx_std@@V?$allocator@U?$pair@II@stlpmtx_std@@@2@@stlpmtx_std@@@stlpmtx_std@@@priv@2@@priv@stlpmtx_std@@_N@3@ABU?$pair@QAUIEntityClass@@V?$vector@U?$pair@II@stlpmtx_std@@V?$allocator@U?$pair@II@stlpmtx_std@@@2@@stlpmtx_std@@@3@@Z 320338c0 f i EntitySystem.obj
 0001:00032980       ??0CEntitySystem@@QAE@PAUISystem@@@Z 32033980 f   EntitySystem.obj
 0001:00033210       ?GetSystem@CEntitySystem@@UBEPAUISystem@@XZ 32034210 f i EntitySystem.obj
 0001:00033220       ?LockSpawning@CEntitySystem@@UAEX_N@Z 32034220 f i EntitySystem.obj
 0001:00033230       ?GetAreaManager@CEntitySystem@@UBEPAUIAreaManager@@XZ 32034230 f i EntitySystem.obj
 0001:00033240       ?GetBreakableManager@CEntitySystem@@UBEPAUIBreakableManager@@XZ 32034240 f i EntitySystem.obj
 0001:00033250       ?GetIEntityPoolManager@CEntitySystem@@UBEPAUIEntityPoolManager@@XZ 32034250 f i EntitySystem.obj
 0001:00033260       ??1CEntitySystem@@UAE@XZ   32034260 f   EntitySystem.obj
 0001:000337d0       ?Reset@CEntitySystem@@UAEXXZ 320347d0 f   EntitySystem.obj
 0001:00033b90       ?InitEntity@CEntitySystem@@UAE_NPAUIEntity@@AAUSEntitySpawnParams@@@Z 32034b90 f   EntitySystem.obj
 0001:00033d10       ?DumpEntities@CEntitySystem@@UAEXXZ 32034d10 f   EntitySystem.obj
 0001:00033dd0       ?AddLayer@CEntitySystem@@UAEPAVCEntityLayer@@PBD0G_NH1@Z 32034dd0 f   EntitySystem.obj
 0001:00033e50       ?insert_unique@?$_Rb_tree@PAUIEntityClass@@U?$less@PAUIEntityClass@@@stlpmtx_std@@U?$pair@QAUIEntityClass@@V?$vector@U?$pair@II@stlpmtx_std@@V?$allocator@U?$pair@II@stlpmtx_std@@@2@@stlpmtx_std@@@3@U?$_Select1st@U?$pair@QAUIEntityClass@@V?$vector@U?$pair@II@stlpmtx_std@@V?$allocator@U?$pair@II@stlpmtx_std@@@2@@stlpmtx_std@@@stlpmtx_std@@@priv@3@U?$_MapTraitsT@U?$pair@QAUIEntityClass@@V?$vector@U?$pair@II@stlpmtx_std@@V?$allocator@U?$pair@II@stlpmtx_std@@@2@@stlpmtx_std@@@stlpmtx_std@@@63@V?$allocator@U?$pair@QAUIEntityClass@@V?$vector@U?$pair@II@stlpmtx_std@@V?$allocator@U?$pair@II@stlpmtx_std@@@2@@stlpmtx_std@@@stlpmtx_std@@@3@@priv@stlpmtx_std@@QAE?AU?$_Rb_tree_iterator@U?$pair@QAUIEntityClass@@V?$vector@U?$pair@II@stlpmtx_std@@V?$allocator@U?$pair@II@stlpmtx_std@@@2@@stlpmtx_std@@@stlpmtx_std@@U?$_MapTraitsT@U?$pair@QAUIEntityClass@@V?$vector@U?$pair@II@stlpmtx_std@@V?$allocator@U?$pair@II@stlpmtx_std@@@2@@stlpmtx_std@@@stlpmtx_std@@@priv@2@@23@U423@ABU?$pair@QAUIEntityClass@@V?$vector@U?$pair@II@stlpmtx_std@@V?$allocator@U?$pair@II@stlpmtx_std@@@2@@stlpmtx_std@@@3@@Z 32034e50 f i EntitySystem.obj
 0001:00034040       ??_ECEntitySystem@@UAEPAXI@Z 32035040 f i EntitySystem.obj
 0001:00034040       ??_GCEntitySystem@@UAEPAXI@Z 32035040 f i EntitySystem.obj
 0001:00034070       ?insert_equal@?$_Rb_tree@VCTimeValue@@U?$less@VCTimeValue@@@stlpmtx_std@@U?$pair@$$CBVCTimeValue@@USEntityTimerEvent@@@3@U?$_Select1st@U?$pair@$$CBVCTimeValue@@USEntityTimerEvent@@@stlpmtx_std@@@priv@3@U?$_MultimapTraitsT@U?$pair@$$CBVCTimeValue@@USEntityTimerEvent@@@stlpmtx_std@@@63@V?$STLPoolAllocator@U?$pair@VCTimeValue@@USEntityTimerEvent@@@stlpmtx_std@@UPSyncNone@stl@@$0A@$0A@@stl@@@priv@stlpmtx_std@@QAE?AU?$_Rb_tree_iterator@U?$pair@$$CBVCTimeValue@@USEntityTimerEvent@@@stlpmtx_std@@U?$_MultimapTraitsT@U?$pair@$$CBVCTimeValue@@USEntityTimerEvent@@@stlpmtx_std@@@priv@2@@23@ABU?$pair@$$CBVCTimeValue@@USEntityTimerEvent@@@3@@Z 32035070 f i EntitySystem.obj
 0001:00034120       ??$?AV?$CryStringT@D@@@?$map@V?$CryStringT@D@@V?$vector@PAVCEntityLayer@@V?$allocator@PAVCEntityLayer@@@stlpmtx_std@@@stlpmtx_std@@U?$less@V?$CryStringT@D@@@3@V?$allocator@U?$pair@$$CBV?$CryStringT@D@@V?$vector@PAVCEntityLayer@@V?$allocator@PAVCEntityLayer@@@stlpmtx_std@@@stlpmtx_std@@@stlpmtx_std@@@3@@stlpmtx_std@@QAEAAV?$vector@PAVCEntityLayer@@V?$allocator@PAVCEntityLayer@@@stlpmtx_std@@@1@ABV?$CryStringT@D@@@Z 32035120 f i EntitySystem.obj
 0001:000341f0       ?DebugDrawLayerInfo@CEntitySystem@@AAEXXZ 320351f0 f   EntitySystem.obj
 0001:00034f20       ??$?APAUIEntityClass@@@?$map@PAUIEntityClass@@V?$vector@U?$pair@II@stlpmtx_std@@V?$allocator@U?$pair@II@stlpmtx_std@@@2@@stlpmtx_std@@U?$less@PAUIEntityClass@@@3@V?$allocator@U?$pair@QAUIEntityClass@@V?$vector@U?$pair@II@stlpmtx_std@@V?$allocator@U?$pair@II@stlpmtx_std@@@2@@stlpmtx_std@@@stlpmtx_std@@@3@@stlpmtx_std@@QAEAAV?$vector@U?$pair@II@stlpmtx_std@@V?$allocator@U?$pair@II@stlpmtx_std@@@2@@1@ABQAUIEntityClass@@@Z 32035f20 f i EntitySystem.obj
 0001:00035060       ?DebugDrawEntityUsage@CEntitySystem@@AAEXXZ 32036060 f   EntitySystem.obj
 0001:00035840       ?AddTimerEvent@CEntitySystem@@QAEXAAUSEntityTimerEvent@@VCTimeValue@@@Z 32036840 f   EntitySystem.obj
 0001:000358f0       ?PauseTimers@CEntitySystem@@UAEX_N0@Z 320368f0 f   EntitySystem.obj
 0001:00035bb0       ?Serialize@CEntitySystem@@UAEXV?$CSerializeWrapper@UISerialize@@@@@Z 32036bb0 f   EntitySystem.obj
 0001:00035ec0       ?Update@CEntitySystem@@UAEXXZ 32036ec0 f   EntitySystem.obj
 0001:000360f0       ??$move_init@VCEntry@CEntityTimeoutList@@@NArray@@YAXPAVCEntry@CEntityTimeoutList@@0I@Z 320370f0 f i EntityTimeoutList.obj
 0001:00036140       ?PopTimeoutEntity@CEntityTimeoutList@@QAEIM@Z 32037140 f   EntityTimeoutList.obj
 0001:000361e0       ?set_size@?$SmallDynStorage@VCEntry@CEntityTimeoutList@@HUStandardAlloc@NAlloc@@@NArray@@QAEXH@Z 320371e0 f i EntityTimeoutList.obj
 0001:00036270       ?resize_raw@?$SmallDynStorage@VCEntry@CEntityTimeoutList@@HUStandardAlloc@NAlloc@@@NArray@@QAEXHH_N@Z 32037270 f i EntityTimeoutList.obj
 0001:000363c0       ?expand_raw@?$DynArray@VCEntry@CEntityTimeoutList@@HU?$SmallDynStorage@VCEntry@CEntityTimeoutList@@HUStandardAlloc@NAlloc@@@NArray@@@@IAEPAVCEntry@CEntityTimeoutList@@PAV23@H@Z 320373c0 f i EntityTimeoutList.obj
 0001:00036440       ?grow@?$DynArray@VCEntry@CEntityTimeoutList@@HU?$SmallDynStorage@VCEntry@CEntityTimeoutList@@HUStandardAlloc@NAlloc@@@NArray@@@@QAEPAVCEntry@CEntityTimeoutList@@H@Z 32037440 f i EntityTimeoutList.obj
 0001:000364a0       ??$reconstruct@U?$DynArray@VCEntry@CEntityTimeoutList@@HU?$SmallDynStorage@VCEntry@CEntityTimeoutList@@HUStandardAlloc@NAlloc@@@NArray@@@@@stl@@YAXAAU?$DynArray@VCEntry@CEntityTimeoutList@@HU?$SmallDynStorage@VCEntry@CEntityTimeoutList@@HUStandardAlloc@NAlloc@@@NArray@@@@@Z 320374a0 f i EntityTimeoutList.obj
 0001:00036510       ?ResetTimeout@CEntityTimeoutList@@QAEXI@Z 32037510 f   EntityTimeoutList.obj
 0001:00036650       ?Clear@CEntityTimeoutList@@QAEXXZ 32037650 f   EntityTimeoutList.obj
 0001:00036660       ??0CEntityTimeoutList@@QAE@PAUITimer@@@Z 32037660 f   EntityTimeoutList.obj
 0001:000366d0       ?DeInitialize@?$Node_Alloc_Lock@$00$00@@SAXXZ 320376d0 f i stdafx.obj
 0001:00036720       ??0ScriptAnyValue@@QAE@ABU0@@Z 32037720 f i EntityScript.obj
 0001:00036800       ??_GIEntityScript@@UAEPAXI@Z 32037800 f i EntityScript.obj
 0001:00036800       ??_EIEntityScript@@UAEPAXI@Z 32037800 f i EntityScript.obj
 0001:00036830       ??1Iterator@IScriptTable@@QAE@XZ 32037830 f i EntityScript.obj
 0001:000368c0       ?CountInOutEvents@CEntityScript@@AAEIPAUIScriptTable@@AAV?$vector@USEntityScriptEvent@@V?$allocator@USEntityScriptEvent@@@stlpmtx_std@@@stlpmtx_std@@_N@Z 320378c0 f   EntityScript.obj
 0001:00036940       ??$GetGlobalValue@PAUIScriptTable@@@IScriptSystem@@QAE_NPBDAAPAUIScriptTable@@@Z 32037940 f i EntityScript.obj
 0001:000369d0       ??$GetValue@PAUIScriptTable@@@IScriptTable@@QAE_NPBDAAPAU0@@Z 320379d0 f i EntityScript.obj
 0001:00036a70       ??$GetValue@PAUSScriptFuncHandle@@@IScriptTable@@QAE_NPBDAAPAUSScriptFuncHandle@@@Z 32037a70 f i EntityScript.obj
 0001:00036b10       ??$GetAt@PAUSScriptFuncHandle@@@IScriptTable@@QAE_NHAAPAUSScriptFuncHandle@@@Z 32037b10 f i EntityScript.obj
 0001:00036bb0       ??$GetAt@PBD@IScriptTable@@QAE_NHAAPBD@Z 32037bb0 f i EntityScript.obj
 0001:00036c30       ??$PushFuncParam@_N@IScriptSystem@@QAEXAB_N@Z 32037c30 f i EntityScript.obj
 0001:00036c90       ??4ScriptAnyValue@@QAEAAU0@ABU0@@Z 32037c90 f i EntityScript.obj
 0001:00036d10       ?InitializeStateTable@CEntityScript@@AAEXPAUIScriptTable@@PAUSScriptStateFunctions@@@Z 32037d10 f   EntityScript.obj
 0001:00036dd0       ??$PushParams@PAUIScriptTable@@_N@Script@@CAXPAUIScriptSystem@@ABQAUIScriptTable@@AB_N@Z 32037dd0 f i EntityScript.obj
 0001:00036e40       ??$PushParams@PAUIScriptTable@@UScriptAnyValue@@M@Script@@CAXPAUIScriptSystem@@ABQAUIScriptTable@@ABUScriptAnyValue@@ABM@Z 32037e40 f i EntityScript.obj
 0001:00036ec0       ??$PushParams@PAUIScriptTable@@UScriptAnyValue@@_N@Script@@CAXPAUIScriptSystem@@ABQAUIScriptTable@@ABUScriptAnyValue@@AB_N@Z 32037ec0 f i EntityScript.obj
 0001:00036f40       ??$PushParams@PAUIScriptTable@@UScriptAnyValue@@PBD@Script@@CAXPAUIScriptSystem@@ABQAUIScriptTable@@ABUScriptAnyValue@@ABQBD@Z 32037f40 f i EntityScript.obj
 0001:00036fc0       ??$PushParams@PAUIScriptTable@@UScriptAnyValue@@U?$Vec3_tpl@M@@@Script@@CAXPAUIScriptSystem@@ABQAUIScriptTable@@ABUScriptAnyValue@@ABU?$Vec3_tpl@M@@@Z 32037fc0 f i EntityScript.obj
 0001:00037060       ?Call_OnShutDown@CEntityScript@@QAEXPAUIScriptTable@@@Z 32038060 f   EntityScript.obj
 0001:00037110       ?EntityEventLess@@YA_NABUSEntityScriptEvent@@0@Z 32038110 f i EntityScript.obj
 0001:00037160       ??$Call@PAUIScriptTable@@_N@Script@@SA_NPAUIScriptSystem@@PAUSScriptFuncHandle@@ABQAUIScriptTable@@AB_N@Z 32038160 f i EntityScript.obj
 0001:000371a0       ?allocate@?$_STLP_alloc_proxy@PAUSEntityScriptEvent@@U1@V?$allocator@USEntityScriptEvent@@@stlpmtx_std@@@priv@stlpmtx_std@@QAEPAUSEntityScriptEvent@@IAAI@Z 320381a0 f i EntityScript.obj
 0001:000371f0       ??1SScriptState@@QAE@XZ    320381f0 f   EntityScript.obj
 0001:00037240       ?InitializeNamedStates@CEntityScript@@AAEXPAUIScriptTable@@H@Z 32038240 f   EntityScript.obj
 0001:000372f0       ?GetState@CEntityScript@@QAEPAUSScriptState@@H@Z 320382f0 f   EntityScript.obj
 0001:00037330       ?GetStateId@CEntityScript@@QBEHPBD@Z 32038330 f   EntityScript.obj
 0001:000373b0       ?GetStateName@CEntityScript@@QBEPBDH@Z 320383b0 f   EntityScript.obj
 0001:000373f0       ?Call_OnInit@CEntityScript@@QAEXPAUIScriptTable@@_N@Z 320383f0 f   EntityScript.obj
 0001:000374e0       ?Call_OnReset@CEntityScript@@QAEXPAUIScriptTable@@_N@Z 320384e0 f   EntityScript.obj
 0001:00037520       ?CallEvent@CEntityScript@@QAEXPAUIScriptTable@@PBDM@Z 32038520 f   EntityScript.obj
 0001:00037630       ?CallEvent@CEntityScript@@QAEXPAUIScriptTable@@PBD_N@Z 32038630 f   EntityScript.obj
 0001:00037750       ?CallEvent@CEntityScript@@QAEXPAUIScriptTable@@PBD1@Z 32038750 f   EntityScript.obj
 0001:000378c0       ?CallEvent@CEntityScript@@QAEXPAUIScriptTable@@PBD0@Z 320388c0 f   EntityScript.obj
 0001:00037a40       ?CallEvent@CEntityScript@@QAEXPAUIScriptTable@@PBDABU?$Vec3_tpl@M@@@Z 32038a40 f   EntityScript.obj
 0001:00037b50       ?FindEvent@CEntityScript@@QBEPBUSEntityScriptEvent@@PBD@Z 32038b50 f   EntityScript.obj
 0001:00037bd0       ??4SEntityScriptEvent@@QAEAAU0@ABU0@@Z 32038bd0 f i EntityScript.obj
 0001:00037c40       ??$__unguarded_linear_insert@PAUSEntityScriptEvent@@U1@P6A_NABU1@0@Z@priv@stlpmtx_std@@YAXPAUSEntityScriptEvent@@U2@P6A_NABU2@2@Z@Z 32038c40 f i EntityScript.obj
 0001:00037d60       ??$__push_heap@PAUSEntityScriptEvent@@HU1@P6A_NABU1@0@Z@stlpmtx_std@@YAXPAUSEntityScriptEvent@@HHU1@P6A_NABU1@2@Z@Z 32038d60 f i EntityScript.obj
 0001:00037eb0       ??$__copy_backward@PAUSEntityScriptEvent@@PAU1@H@priv@stlpmtx_std@@YAPAUSEntityScriptEvent@@PAU2@00ABUrandom_access_iterator_tag@1@PAH@Z 32038eb0 f i EntityScript.obj
 0001:00037fb0       ?Init@CEntityScript@@UAE_NPBD0@Z 32038fb0 f   EntityScript.obj
 0001:00038020       ??$__copy@PAUSScriptState@@PAU1@H@priv@stlpmtx_std@@YAPAUSScriptState@@PAU2@00ABUrandom_access_iterator_tag@1@PAH@Z 32039020 f i EntityScript.obj
 0001:00038100       ??$__copy@PAUSEntityScriptEvent@@PAU1@H@priv@stlpmtx_std@@YAPAUSEntityScriptEvent@@PAU2@00ABUrandom_access_iterator_tag@1@PAH@Z 32039100 f i EntityScript.obj
 0001:000381f0       ??$__unguarded_insertion_sort_aux@PAUSEntityScriptEvent@@U1@P6A_NABU1@0@Z@priv@stlpmtx_std@@YAXPAUSEntityScriptEvent@@00P6A_NABU2@1@Z@Z 320391f0 f i EntityScript.obj
 0001:00038260       ??$__adjust_heap@PAUSEntityScriptEvent@@HU1@P6A_NABU1@0@Z@stlpmtx_std@@YAXPAUSEntityScriptEvent@@HHU1@P6A_NABU1@2@Z@Z 32039260 f i EntityScript.obj
 0001:00038410       ??$__ufill@PAUSScriptState@@U1@H@priv@stlpmtx_std@@YAXPAUSScriptState@@0ABU2@ABUrandom_access_iterator_tag@1@PAH@Z 32039410 f i EntityScript.obj
 0001:00038470       ??$__ufill@PAUSEntityScriptEvent@@U1@H@priv@stlpmtx_std@@YAXPAUSEntityScriptEvent@@0ABU2@ABUrandom_access_iterator_tag@1@PAH@Z 32039470 f i EntityScript.obj
 0001:000384e0       ??$__destroy_range_aux@V?$reverse_iterator@PAUSScriptState@@@stlpmtx_std@@USScriptState@@@stlpmtx_std@@YAXV?$reverse_iterator@PAUSScriptState@@@0@0PAUSScriptState@@ABU__false_type@0@@Z 320394e0 f i EntityScript.obj
 0001:00038550       ??$__destroy_range_aux@V?$reverse_iterator@PAUSEntityScriptEvent@@@stlpmtx_std@@USEntityScriptEvent@@@stlpmtx_std@@YAXV?$reverse_iterator@PAUSEntityScriptEvent@@@0@0PAUSEntityScriptEvent@@ABU__false_type@0@@Z 32039550 f i EntityScript.obj
 0001:000385a0       ??$__destroy_range_aux@PAUSScriptState@@U1@@stlpmtx_std@@YAXPAUSScriptState@@00ABU__false_type@0@@Z 320395a0 f i EntityScript.obj
 0001:00038600       ??$__destroy_range_aux@PAUSEntityScriptEvent@@U1@@stlpmtx_std@@YAXPAUSEntityScriptEvent@@00ABU__false_type@0@@Z 32039600 f i EntityScript.obj
 0001:00038650       ??$__ucopy@PAUSScriptState@@PAU1@H@priv@stlpmtx_std@@YAPAUSScriptState@@PAU2@00ABUrandom_access_iterator_tag@1@PAH@Z 32039650 f i EntityScript.obj
 0001:000386b0       ??$__ucopy@PAUSEntityScriptEvent@@PAU1@H@priv@stlpmtx_std@@YAPAUSEntityScriptEvent@@PAU2@00ABUrandom_access_iterator_tag@1@PAH@Z 320396b0 f i EntityScript.obj
 0001:00038730       ??$__pop_heap@PAUSEntityScriptEvent@@U1@P6A_NABU1@0@ZH@stlpmtx_std@@YAXPAUSEntityScriptEvent@@00U1@P6A_NABU1@2@ZPAH@Z 32039730 f i EntityScript.obj
 0001:000387d0       ??$__make_heap@PAUSEntityScriptEvent@@P6A_NABU1@0@ZU1@H@stlpmtx_std@@YAXPAUSEntityScriptEvent@@0P6A_NABU1@1@Z0PAH@Z 320397d0 f i EntityScript.obj
 0001:00038860       ??$__unguarded_partition@PAUSEntityScriptEvent@@U1@P6A_NABU1@0@Z@priv@stlpmtx_std@@YAPAUSEntityScriptEvent@@PAU2@0U2@P6A_NABU2@2@Z@Z 32039860 f i EntityScript.obj
 0001:00038a80       ??$__linear_insert@PAUSEntityScriptEvent@@U1@P6A_NABU1@0@Z@priv@stlpmtx_std@@YAXPAUSEntityScriptEvent@@0U2@P6A_NABU2@2@Z@Z 32039a80 f i EntityScript.obj
 0001:00038b40       ??$sort_heap@PAUSEntityScriptEvent@@P6A_NABU1@0@Z@stlpmtx_std@@YAXPAUSEntityScriptEvent@@0P6A_NABU1@1@Z@Z 32039b40 f i EntityScript.obj
 0001:00038bd0       ?_M_insert_overflow_aux@?$_Impl_vector@USScriptState@@V?$allocator@USScriptState@@@stlpmtx_std@@@priv@stlpmtx_std@@AAEXPAUSScriptState@@ABU4@ABU__false_type@3@I_N@Z 32039bd0 f i EntityScript.obj
 0001:00038da0       ?_M_insert_overflow_aux@?$_Impl_vector@USEntityScriptEvent@@V?$allocator@USEntityScriptEvent@@@stlpmtx_std@@@priv@stlpmtx_std@@AAEXPAUSEntityScriptEvent@@ABU4@ABU__false_type@3@I_N@Z 32039da0 f i EntityScript.obj
 0001:00038f60       ??$_M_allocate_and_copy@PAUSScriptState@@@?$_Impl_vector@USScriptState@@V?$allocator@USScriptState@@@stlpmtx_std@@@priv@stlpmtx_std@@AAEPAUSScriptState@@AAIPAU3@1@Z 32039f60 f i EntityScript.obj
 0001:00038fd0       ??$_M_allocate_and_copy@PAUSEntityScriptEvent@@@?$_Impl_vector@USEntityScriptEvent@@V?$allocator@USEntityScriptEvent@@@stlpmtx_std@@@priv@stlpmtx_std@@AAEPAUSEntityScriptEvent@@AAIPAU3@1@Z 32039fd0 f i EntityScript.obj
 0001:00039040       ??$__insertion_sort@PAUSEntityScriptEvent@@U1@P6A_NABU1@0@Z@priv@stlpmtx_std@@YAXPAUSEntityScriptEvent@@00P6A_NABU2@1@Z@Z 3203a040 f i EntityScript.obj
 0001:000390c0       ??$__partial_sort@PAUSEntityScriptEvent@@U1@P6A_NABU1@0@Z@priv@stlpmtx_std@@YAXPAUSEntityScriptEvent@@000P6A_NABU2@1@Z@Z 3203a0c0 f i EntityScript.obj
 0001:00039170       ?reserve@?$_Impl_vector@USScriptState@@V?$allocator@USScriptState@@@stlpmtx_std@@@priv@stlpmtx_std@@QAEXI@Z 3203a170 f i EntityScript.obj
 0001:00039240       ?reserve@?$_Impl_vector@USEntityScriptEvent@@V?$allocator@USEntityScriptEvent@@@stlpmtx_std@@@priv@stlpmtx_std@@QAEXI@Z 3203a240 f i EntityScript.obj
 0001:000392e0       ??0CEntityScript@@QAE@XZ   3203a2e0 f   EntityScript.obj
 0001:00039370       ?push_back@?$_Impl_vector@USEntityScriptEvent@@V?$allocator@USEntityScriptEvent@@@stlpmtx_std@@@priv@stlpmtx_std@@QAEXABUSEntityScriptEvent@@@Z 3203a370 f i EntityScript.obj
 0001:00039400       ??$__introsort_loop@PAUSEntityScriptEvent@@U1@HP6A_NABU1@0@Z@priv@stlpmtx_std@@YAXPAUSEntityScriptEvent@@00HP6A_NABU2@1@Z@Z 3203a400 f i EntityScript.obj
 0001:00039530       ??$sort@PAUSEntityScriptEvent@@P6A_NABU1@0@Z@stlpmtx_std@@YAXPAUSEntityScriptEvent@@0P6A_NABU1@1@Z@Z 3203a530 f i EntityScript.obj
 0001:000395b0       ?Clear@CEntityScript@@AAEXXZ 3203a5b0 f   EntityScript.obj
 0001:00039820       ?EnumStates@CEntityScript@@AAEXXZ 3203a820 f   EntityScript.obj
 0001:00039b70       ?ParseInOutEvents@CEntityScript@@AAEXPAUIScriptTable@@AAV?$vector@USEntityScriptEvent@@V?$allocator@USEntityScriptEvent@@@stlpmtx_std@@@stlpmtx_std@@_N@Z 3203ab70 f   EntityScript.obj
 0001:00039d40       ?LoadEvents@CEntityScript@@AAEXXZ 3203ad40 f   EntityScript.obj
 0001:0003a030       ??1CEntityScript@@UAE@XZ   3203b030 f   EntityScript.obj
 0001:0003a140       ?LoadScript@CEntityScript@@UAE_N_N@Z 3203b140 f   EntityScript.obj
 0001:0003a270       ??_GCEntityScript@@UAEPAXI@Z 3203b270 f i EntityScript.obj
 0001:0003a270       ??_ECEntityScript@@UAEPAXI@Z 3203b270 f i EntityScript.obj
 0001:0003a2a0       ?Init@CScriptableBase@@UAEXPAUIScriptSystem@@PAUISystem@@H@Z 3203b2a0 f i ScriptBind_Entity.obj
 0001:0003a2d0       ?Done@CScriptableBase@@UAEXXZ 3203b2d0 f i ScriptBind_Entity.obj
 0001:0003a310       ?GetAttachmentType@CLightAttachment@@UAE?AW4EType@IAttachmentObject@@XZ 3203b310 f i ScriptBind_Entity.obj
 0001:0003a310       ?GetType@CAreaProxy@@UAE?AW4EEntityProxy@@XZ 3203b310 f i AreaProxy.obj
 0001:0003a320       ?LoadLight@CLightAttachment@@QAEXABVCDLight@@@Z 3203b320 f i ScriptBind_Entity.obj
 0001:0003a360       ?Dephysicalize@IRenderNode@@UAEX_N@Z 3203b360 f i RenderProxy.obj
 0001:0003a360       ?AddSizerTree@CDummyMemReplay@@UAEXPBD@Z 3203b360 f i AreaSolid.obj
 0001:0003a360       ?SetReplacementMaterial@CEntityAttachment@@UAEXPAUIMaterial@@@Z 3203b360 f i Entity.obj
 0001:0003a360       ?Physicalize@IRenderNode@@UAEX_N@Z 3203b360 f i RenderProxy.obj
 0001:0003a360       ?Update@CSoundProxy@@UAEXAAUSEntityUpdateContext@@@Z 3203b360 f i SoundProxy.obj
 0001:0003a360       ?Serialize@CSoundProxy@@UAEXV?$CSerializeWrapper@UISerialize@@@@@Z 3203b360 f i SoundProxy.obj
 0001:0003a360       ?Update@CAreaProxy@@UAEXAAUSEntityUpdateContext@@@Z 3203b360 f i AreaProxy.obj
 0001:0003a360       ?GetInfo@CDummyMemReplay@@UAEXAAUCryReplayInfo@@@Z 3203b360 f i AreaSolid.obj
 0001:0003a360       ?Serialize@CCameraProxy@@UAEXV?$CSerializeWrapper@UISerialize@@@@@Z 3203b360 f i CameraProxy.obj
 0001:0003a360       ?Update@CTriggerProxy@@UAEXAAUSEntityUpdateContext@@@Z 3203b360 f i TriggerProxy.obj
 0001:0003a360       ?SetReplacementMaterial@CLightAttachment@@UAEXPAUIMaterial@@@Z 3203b360 f i ScriptBind_Entity.obj
 0001:0003a360       ?GetMemoryStatistics@CScriptableBase@@UAEXPAVICrySizer@@@Z 3203b360 f i ScriptBind_Entity.obj
 0001:0003a360       ?GetMemoryUsage@CEntityNodeProxy@@UBEXPAVICrySizer@@@Z 3203b360 f i Entity.obj
 0001:0003a360       ?Update@CCameraProxy@@UAEXAAUSEntityUpdateContext@@@Z 3203b360 f i CameraProxy.obj
 0001:0003a360       ?ProcessAttachment@CCGFAttachment@@UAEXPAUIAttachment@@@Z 3203b360 f i ScriptBind_Entity.obj
 0001:0003a360       ?RemoveAllocReference@CDummyMemReplay@@UAEXPAX@Z 3203b360 f i AreaSolid.obj
 0001:0003a360       ?SetLayerId@IRenderNode@@UAEXG@Z 3203b360 f i RenderProxy.obj
 0001:0003a360       ?SetPhysics@CRenderProxy@@UAEXPAUIPhysicalEntity@@@Z 3203b360 f i RenderProxy.obj
 0001:0003a360       ?GetMemoryUsage@IEntityScript@@UBEXPAVICrySizer@@@Z 3203b360 f i EntityScript.obj
 0001:0003a360       ?Update@CFlowGraphProxy@@UAEXAAUSEntityUpdateContext@@@Z 3203b360 f i FlowGraphProxy.obj
 0001:0003a360       ?SetEditorObjectId@IRenderNode@@UAEXH@Z 3203b360 f i RenderProxy.obj
 0001:0003a360       ?Update@CEntityNodeProxy@@UAEXAAUSEntityUpdateContext@@@Z 3203b360 f i Entity.obj
 0001:0003a360       ?ProcessEvent@CSubstitutionProxy@@UAEXAAUSEntityEvent@@@Z 3203b360 f i Entity.obj
 0001:0003a360       ?AddLabel@CDummyMemReplay@@UAEXPBD@Z 3203b360 f i AreaSolid.obj
 0001:0003a360       ?Serialize@CEntityNodeProxy@@UAEXV?$CSerializeWrapper@UISerialize@@@@@Z 3203b360 f i Entity.obj
 0001:0003a360       ?Update@CSubstitutionProxy@@UAEXAAUSEntityUpdateContext@@@Z 3203b360 f i Entity.obj
 0001:0003a360       ?SetMatrix@IRenderNode@@UAEXABU?$Matrix34_tpl@M@@@Z 3203b360 f i RenderProxy.obj
 0001:0003a360       ?SetStatObjGroupId@IRenderNode@@UAEXH@Z 3203b360 f i RenderProxy.obj
 0001:0003a360       ?Serialize@CAreaProxy@@UAEXV?$CSerializeWrapper@UISerialize@@@@@Z 3203b360 f i AreaProxy.obj
 0001:0003a360       ?StartOnCommandLine@CDummyMemReplay@@UAEXPBD@Z 3203b360 f i AreaSolid.obj
 0001:0003a360       ?SetMergeGroupId@IRenderNode@@UAEXH@Z 3203b360 f i RenderProxy.obj
 0001:0003a360       ?Update@CRopeProxy@@UAEXAAUSEntityUpdateContext@@@Z 3203b360 f i RopeProxy.obj
 0001:0003a360       ?OnRenderNodeBecomeVisible@IRenderNode@@UAEXABUSRenderingPassInfo@@@Z 3203b360 f i RenderProxy.obj
 0001:0003a360       ?UnregisterContainer@CDummyMemReplay@@UAEXPBX@Z 3203b360 f i AreaSolid.obj
 0001:0003a360       ?GetMemoryUsage@IEntityProxy@@UBEXPAVICrySizer@@@Z 3203b360 f i Entity.obj
 0001:0003a360       ?SetReplacementMaterial@CEffectAttachment@@UAEXPAUIMaterial@@@Z 3203b360 f i ScriptBind_Entity.obj
 0001:0003a360       ?ExitScope_Free@CDummyMemReplay@@UAEXI@Z 3203b360 f i AreaSolid.obj
 0001:0003a370       ??_ECLightAttachment@@UAEPAXI@Z 3203b370 f i ScriptBind_Entity.obj
 0001:0003a370       ??_GCLightAttachment@@UAEPAXI@Z 3203b370 f i ScriptBind_Entity.obj
 0001:0003a3c0       ?CastToIPuppetSafe@@YAPAUIPuppet@@PAUIAIObject@@@Z 3203b3c0 f i ScriptBind_Entity.obj
 0001:0003a3e0       ?GetExt@PathUtil@@YAPBDPBD@Z 3203b3e0 f i ScriptBind_Entity.obj
 0001:0003a470       ?DelegateCalls@CScriptBind_Entity@@QAEXPAUIScriptTable@@@Z 3203b470 f   ScriptBind_Entity.obj
 0001:0003a490       ?SetLensOpticsElement@SRenderLight@@QAEXPAVIOpticsElementBase@@@Z 3203b490 f i ScriptBind_Entity.obj
 0001:0003a500       ?DropResources@SRenderLight@@QAEXXZ 3203b500 f i ScriptBind_Entity.obj
 0001:0003a5c0       ?ReleaseCubemaps@CDLight@@QAEXXZ 3203b5c0 f i ScriptBind_Entity.obj
 0001:0003a5f0       ?ReleaseDeferredRenderMesh@CDLight@@QAEXXZ 3203b5f0 f i ScriptBind_Entity.obj
 0001:0003a610       ?DisableAnimationEvent@CScriptBind_Entity@@IAEHPAUIFunctionHandler@@HPBD@Z 3203b610 f   ScriptBind_Entity.obj
 0001:0003a610       ?SetAnimationEvent@CScriptBind_Entity@@IAEHPAUIFunctionHandler@@HPBD@Z 3203b610 f   ScriptBind_Entity.obj
 0001:0003a620       ?Damage@CScriptBind_Entity@@IAEHPAUIFunctionHandler@@@Z 3203b620 f   ScriptBind_Entity.obj
 0001:0003a640       ?GetLink@@YAPAUIEntityLink@@PAU1@PBDH@Z 3203b640 f   ScriptBind_Entity.obj
 0001:0003a680       ?cmpIntersectionResult@CScriptBind_Entity@@CAHPBX0@Z 3203b680 f   ScriptBind_Entity.obj
 0001:0003a6a0       ??4?$_smart_ptr@UIStatObj@@@@QAEAAV0@PAUIStatObj@@@Z 3203b6a0 f i ScriptBind_Entity.obj
 0001:0003a6d0       ??4?$_smart_ptr@UICharacterInstance@@@@QAEAAV0@PAUICharacterInstance@@@Z 3203b6d0 f i ScriptBind_Entity.obj
 0001:0003a700       ??$SetGlobalValue@PAUIScriptTable@@@IScriptSystem@@QAEXPBDABQAUIScriptTable@@@Z 3203b700 f i ScriptBind_Entity.obj
 0001:0003a780       ??$GetAt@M@IScriptTable@@QAE_NHAAM@Z 3203b780 f i ScriptBind_Entity.obj
 0001:0003a810       ??$GetParam@VSmartScriptTable@@@IFunctionHandler@@QAE_NHAAVSmartScriptTable@@@Z 3203b810 f i ScriptBind_Entity.obj
 0001:0003a8d0       ??$SetGlobalValue@TScriptHandle@@@IScriptSystem@@QAEXPBDABTScriptHandle@@@Z 3203b8d0 f i ScriptBind_Entity.obj
 0001:0003a940       ??$SetGlobalValue@W4geom_flags@@@IScriptSystem@@QAEXPBDABW4geom_flags@@@Z 3203b940 f i ScriptBind_Entity.obj
 0001:0003a940       ??$SetGlobalValue@W4EAreaType@AreaDefinition@SEntityPhysicalizeParams@@@IScriptSystem@@QAEXPBDABW4EAreaType@AreaDefinition@SEntityPhysicalizeParams@@@Z 3203b940 f i ScriptBind_Entity.obj
 0001:0003a940       ??$SetGlobalValue@W4phentity_flags@@@IScriptSystem@@QAEXPBDABW4phentity_flags@@@Z 3203b940 f i ScriptBind_Entity.obj
 0001:0003a940       ??$SetGlobalValue@W4EMaterialLayerFlags@@@IScriptSystem@@QAEXPBDABW4EMaterialLayerFlags@@@Z 3203b940 f i ScriptBind_Entity.obj
 0001:0003a940       ??$SetGlobalValue@W4EPhysForeignFlags@@@IScriptSystem@@QAEXPBDABW4EPhysForeignFlags@@@Z 3203b940 f i ScriptBind_Entity.obj
 0001:0003a940       ??$SetGlobalValue@W4EAttachmentFlags@IEntity@@@IScriptSystem@@QAEXPBDABW4EAttachmentFlags@IEntity@@@Z 3203b940 f i ScriptBind_Entity.obj
 0001:0003a940       ??$SetGlobalValue@W4entity_query_flags@@@IScriptSystem@@QAEXPBDABW4entity_query_flags@@@Z 3203b940 f i ScriptBind_Entity.obj
 0001:0003a940       ??$SetGlobalValue@H@IScriptSystem@@QAEXPBDABH@Z 3203b940 f i ScriptBind_Entity.obj
 0001:0003a9b0       ??$GetSelf@VSmartScriptTable@@@IFunctionHandler@@QAE_NAAVSmartScriptTable@@@Z 3203b9b0 f i ScriptBind_Entity.obj
 0001:0003aa70       ??$GetValue@TScriptHandle@@@IScriptTable@@QAE_NPBDAATScriptHandle@@@Z 3203ba70 f i ScriptBind_Entity.obj
 0001:0003aaf0       ??$GetSelf@TScriptHandle@@@IFunctionHandler@@QAE_NAATScriptHandle@@@Z 3203baf0 f i ScriptBind_Entity.obj
 0001:0003ab70       ??$EndFunction@VSmartScriptTable@@@IFunctionHandler@@QAEHABVSmartScriptTable@@@Z 3203bb70 f i ScriptBind_Entity.obj
 0001:0003ab70       ??$EndFunction@PAUIScriptTable@@@IFunctionHandler@@QAEHABQAUIScriptTable@@@Z 3203bb70 f i ScriptBind_Entity.obj
 0001:0003abf0       ??$EndFunction@M@IFunctionHandler@@QAEHABM@Z 3203bbf0 f i ScriptBind_Entity.obj
 0001:0003ac60       ??$EndFunction@U?$Vec3_tpl@M@@@IFunctionHandler@@QAEHABU?$Vec3_tpl@M@@@Z 3203bc60 f i ScriptBind_Entity.obj
 0001:0003ace0       ??$?0M@?$Ang3_tpl@M@@QAE@ABU?$Matrix33_tpl@M@@@Z 3203bce0 f i ScriptBind_Entity.obj
 0001:0003adb0       ??$EndFunction@_N@IFunctionHandler@@QAEHAB_N@Z 3203bdb0 f i ScriptBind_Entity.obj
 0001:0003ae20       ??$GetParam@PAD@IFunctionHandler@@QAE_NHAAPAD@Z 3203be20 f i ScriptBind_Entity.obj
 0001:0003ae20       ??$GetParam@PBD@IFunctionHandler@@QAE_NHAAPBD@Z 3203be20 f i ScriptBind_Entity.obj
 0001:0003aea0       ??$EndFunction@PBD@IFunctionHandler@@QAEHABQBD@Z 3203bea0 f i ScriptBind_Entity.obj
 0001:0003af10       ??$EndFunction@H@IFunctionHandler@@QAEHABH@Z 3203bf10 f i ScriptBind_Entity.obj
 0001:0003af80       ??$EndFunction@I@IFunctionHandler@@QAEHABI@Z 3203bf80 f i ScriptBind_Entity.obj
 0001:0003b000       ??$EndFunction@$$BY0CA@D@IFunctionHandler@@QAEHAAY0CA@$$CBD@Z 3203c000 f i ScriptBind_Entity.obj
 0001:0003b000       ??$EndFunction@$$BY00$$CBD@IFunctionHandler@@QAEHAAY00$$CBD@Z 3203c000 f i ScriptBind_Entity.obj
 0001:0003b070       ??$EndFunction@TScriptHandle@@@IFunctionHandler@@QAEHABTScriptHandle@@@Z 3203c070 f i ScriptBind_Entity.obj
 0001:0003b0e0       ??$GetValue@H@IScriptTable@@QAE_NPBDAAH@Z 3203c0e0 f i ScriptBind_Entity.obj
 0001:0003b170       ??$GetParam@H@IFunctionHandler@@QAE_NHAAH@Z 3203c170 f i ScriptBind_Entity.obj
 0001:0003b1f0       ??$GetParam@U?$Ang3_tpl@M@@@IFunctionHandler@@QAE_NHAAU?$Ang3_tpl@M@@@Z 3203c1f0 f i ScriptBind_Entity.obj
 0001:0003b1f0       ??$GetParam@U?$Vec3_tpl@M@@@IFunctionHandler@@QAE_NHAAU?$Vec3_tpl@M@@@Z 3203c1f0 f i ScriptBind_Entity.obj
 0001:0003b290       ??$GetParam@_N@IFunctionHandler@@QAE_NHAA_N@Z 3203c290 f i ScriptBind_Entity.obj
 0001:0003b310       ??$GetParam@M@IFunctionHandler@@QAE_NHAAM@Z 3203c310 f i ScriptBind_Entity.obj
 0001:0003b3a0       ??$EndFunction@_NM@IFunctionHandler@@QAEHAB_NABM@Z 3203c3a0 f i ScriptBind_Entity.obj
 0001:0003b470       ??$GetValue@M@IScriptTable@@QAE_NPBDAAM@Z 3203c470 f i ScriptBind_Entity.obj
 0001:0003b500       ??$GetValue@U?$Vec3_tpl@M@@@IScriptTable@@QAE_NPBDAAU?$Vec3_tpl@M@@@Z 3203c500 f i ScriptBind_Entity.obj
 0001:0003b5a0       ??$GetParam@TScriptHandle@@@IFunctionHandler@@QAE_NHAATScriptHandle@@@Z 3203c5a0 f i ScriptBind_Entity.obj
 0001:0003b620       ??$EndFunction@VSmartScriptTable@@V1@@IFunctionHandler@@QAEHABVSmartScriptTable@@0@Z 3203c620 f i ScriptBind_Entity.obj
 0001:0003b700       ??$EndFunction@U?$Vec3_tpl@M@@U1@@IFunctionHandler@@QAEHABU?$Vec3_tpl@M@@0@Z 3203c700 f i ScriptBind_Entity.obj
 0001:0003b7f0       ??$EndFunction@MM@IFunctionHandler@@QAEHABM0@Z 3203c7f0 f i ScriptBind_Entity.obj
 0001:0003b8c0       ??$GetAt@VSmartScriptTable@@@IScriptTable@@QAE_NHAAVSmartScriptTable@@@Z 3203c8c0 f i ScriptBind_Entity.obj
 0001:0003b980       ??$SetAt@PAUIScriptTable@@@IScriptTable@@QAEXHABQAU0@@Z 3203c980 f i ScriptBind_Entity.obj
 0001:0003ba00       ??$SetValueChain@PAUIScriptTable@@@IScriptTable@@QAEXPBDABQAU0@@Z 3203ca00 f i ScriptBind_Entity.obj
 0001:0003ba80       ??$SetValue@M@IScriptTable@@QAEXPBDABM@Z 3203ca80 f i ScriptBind_Entity.obj
 0001:0003baf0       ?thunk@?$CBMemberTranslator1wRet@PAUIFunctionHandler@@HVCScriptBind_Entity@@P82@AEHPAU1@@Z@@SAHABVFunctorBase@@PAUIFunctionHandler@@@Z 3203caf0 f i ScriptBind_Entity.obj
 0001:0003bb10       ??$GetValueChain@M@IScriptTable@@QAE_NPBDAAM@Z 3203cb10 f i ScriptBind_Entity.obj
 0001:0003bba0       ??$GetValueChain@VSmartScriptTable@@@IScriptTable@@QAE_NPBDAAVSmartScriptTable@@@Z 3203cba0 f i ScriptBind_Entity.obj
 0001:0003bc60       ??$GetValueChain@_N@IScriptTable@@QAE_NPBDAA_N@Z 3203cc60 f i ScriptBind_Entity.obj
 0001:0003bce0       ??$GetValueChain@PBD@IScriptTable@@QAE_NPBDAAPBD@Z 3203cce0 f i ScriptBind_Entity.obj
 0001:0003bd60       ??$?0M@?$Ang3_tpl@M@@QAE@ABU?$Quat_tpl@M@@@Z 3203cd60 f i ScriptBind_Entity.obj
 0001:0003beb0       ??$GetValueChain@H@IScriptTable@@QAE_NPBDAAH@Z 3203ceb0 f i ScriptBind_Entity.obj
 0001:0003bf40       ??$GetValueChain@U?$Vec3_tpl@M@@@IScriptTable@@QAE_NPBDAAU?$Vec3_tpl@M@@@Z 3203cf40 f i ScriptBind_Entity.obj
 0001:0003bfe0       ??$GetValueChain@TScriptHandle@@@IScriptTable@@QAE_NPBDAATScriptHandle@@@Z 3203cfe0 f i ScriptBind_Entity.obj
 0001:0003c060       ??$GetValueChain@I@IScriptTable@@QAE_NPBDAAI@Z 3203d060 f i ScriptBind_Entity.obj
 0001:0003c100       ??$Call@VCScriptBind_Entity@@HVSmartScriptTable@@@ScriptTemplateCallHelper@@SAHPAVCScriptBind_Entity@@P81@AEHPAUIFunctionHandler@@HVSmartScriptTable@@@Z1@Z 3203d100 f i ScriptBind_Entity.obj
 0001:0003c180       ??$GetParams@HPBDPBDU?$Vec3_tpl@M@@U1@MH@IFunctionHandler@@QAE_NAAHAAPBD1AAU?$Vec3_tpl@M@@2AAM0@Z 3203d180 f i ScriptBind_Entity.obj
 0001:0003c210       ??$GetParams@HHMU?$Vec3_tpl@M@@U1@M_N@IFunctionHandler@@QAE_NAAH0AAMAAU?$Vec3_tpl@M@@21AA_N@Z 3203d210 f i ScriptBind_Entity.obj
 0001:0003c2a0       ??$GetParams@HPBD_NPBDPBDMM@IFunctionHandler@@QAE_NAAHAAPBDAA_N11AAM3@Z 3203d2a0 f i ScriptBind_Entity.obj
 0001:0003c330       ??$__fill@PAMMH@priv@stlpmtx_std@@YAXPAM0ABMABUrandom_access_iterator_tag@1@PAH@Z 3203d330 f i ScriptBind_Entity.obj
 0001:0003c390       ??$GetParam@I@IFunctionHandler@@QAE_NHAAI@Z 3203d390 f i ScriptBind_Entity.obj
 0001:0003c430       ?RegisterGlobal@CScriptableBase@@IAEXPBDH@Z 3203d430 f i ScriptBind_Entity.obj
 0001:0003c4a0       ?RegisterFunction@CScriptableBase@@IAEXPBDV?$Functor1wRet@PAUIFunctionHandler@@H@@@Z 3203d4a0 f i ScriptBind_Entity.obj
 0001:0003c500       ??_GCScriptableBase@@UAEPAXI@Z 3203d500 f i ScriptBind_Entity.obj
 0001:0003c500       ??_ECScriptableBase@@UAEPAXI@Z 3203d500 f i ScriptBind_Entity.obj
 0001:0003c550       ?GetCachedTable@Script@@SA?AVSmartScriptTable@@PAUIFunctionHandler@@H@Z 3203d550 f i ScriptBind_Entity.obj
 0001:0003c5e0       ?GetType@CScriptProxy@@UAE?AW4EEntityProxy@@XZ 3203d5e0 f i ScriptProxy.obj
 0001:0003c5e0       ?GetAttachmentType@CSKELAttachment@@UAE?AW4EType@IAttachmentObject@@XZ 3203d5e0 f i ScriptBind_Entity.obj
 0001:0003c5f0       ?ProcessAttachment@CSKELAttachment@@UAEXPAUIAttachment@@@Z 3203d5f0 f i ScriptBind_Entity.obj
 0001:0003c610       ?GetRadiusSqr@CSKELAttachment@@UAEMXZ 3203d610 f i ScriptBind_Entity.obj
 0001:0003c640       ?Release@CSKELAttachment@@UAEXXZ 3203d640 f i ScriptBind_Entity.obj
 0001:0003c660       ?GetBaseMaterial@CSKELAttachment@@UBEPAUIMaterial@@XZ 3203d660 f i ScriptBind_Entity.obj
 0001:0003c680       ?GetAABB@CLightAttachment@@UAE?AUAABB@@XZ 3203d680 f i ScriptBind_Entity.obj
 0001:0003c6f0       ?GetRadiusSqr@CLightAttachment@@UAEMXZ 3203d6f0 f i ScriptBind_Entity.obj
 0001:0003c710       ??0pe_simulation_params@@QAE@XZ 3203d710 f i ScriptBind_Entity.obj
 0001:0003c7c0       ??0pe_params_joint@@QAE@XZ 3203d7c0 f i ScriptBind_Entity.obj
 0001:0003c8d0       ??0pe_params_articulated_body@@QAE@XZ 3203d8d0 f i ScriptBind_Entity.obj
 0001:0003c9d0       ??0pe_player_dynamics@@QAE@XZ 3203d9d0 f i ScriptBind_Entity.obj
 0001:0003cac0       ??0pe_params_car@@QAE@XZ   3203dac0 f i ScriptBind_Entity.obj
 0001:0003cc20       ??0pe_params_rope@@QAE@XZ  3203dc20 f i ScriptBind_Entity.obj
 0001:0003ce00       ??0pe_params_softbody@@QAE@XZ 3203de00 f i ScriptBind_Entity.obj
 0001:0003cf30       ??0pe_action_add_constraint@@QAE@XZ 3203df30 f i ScriptBind_Entity.obj
 0001:0003cff0       ??0pe_status_dynamics@@QAE@XZ 3203dff0 f i ScriptBind_Entity.obj
 0001:0003d070       ??0intersection_params@@QAE@XZ 3203e070 f i ScriptBind_Entity.obj
 0001:0003d140       ??$TypeInfo@W4EGeomType@@@@YAABUCTypeInfo@@PBW4EGeomType@@@Z 3203e140 f   ScriptBind_Entity.obj
 0001:0003d180       ??$TypeInfo@W4EGeomForm@@@@YAABUCTypeInfo@@PBW4EGeomForm@@@Z 3203e180 f   ScriptBind_Entity.obj
 0001:0003d1c0       ?GetEntity@CScriptBind_Entity@@AAEPAUIEntity@@PAUIFunctionHandler@@@Z 3203e1c0 f   ScriptBind_Entity.obj
 0001:0003d250       ?DeleteThis@CScriptBind_Entity@@IAEHPAUIFunctionHandler@@@Z 3203e250 f   ScriptBind_Entity.obj
 0001:0003d2a0       ?SetWorldPos@CScriptBind_Entity@@IAEHPAUIFunctionHandler@@U?$Vec3_tpl@M@@@Z 3203e2a0 f   ScriptBind_Entity.obj
 0001:0003d2a0       ?SetPos@CScriptBind_Entity@@IAEHPAUIFunctionHandler@@U?$Vec3_tpl@M@@@Z 3203e2a0 f   ScriptBind_Entity.obj
 0001:0003d370       ?SetScale@CScriptBind_Entity@@IAEHPAUIFunctionHandler@@M@Z 3203e370 f   ScriptBind_Entity.obj
 0001:0003d3d0       ?GetScale@CScriptBind_Entity@@IAEHPAUIFunctionHandler@@@Z 3203e3d0 f   ScriptBind_Entity.obj
 0001:0003d3d0       ?GetLocalScale@CScriptBind_Entity@@IAEHPAUIFunctionHandler@@@Z 3203e3d0 f   ScriptBind_Entity.obj
 0001:0003d3d0       ?GetWorldScale@CScriptBind_Entity@@IAEHPAUIFunctionHandler@@@Z 3203e3d0 f   ScriptBind_Entity.obj
 0001:0003d470       ?CalcWorldAnglesFromRelativeDir@CScriptBind_Entity@@IAEHPAUIFunctionHandler@@U?$Vec3_tpl@M@@@Z 3203e470 f   ScriptBind_Entity.obj
 0001:0003d7a0       ?SetLocalPos@CScriptBind_Entity@@IAEHPAUIFunctionHandler@@U?$Vec3_tpl@M@@@Z 3203e7a0 f   ScriptBind_Entity.obj
 0001:0003d7d0       ?SetName@CScriptBind_Entity@@IAEHPAUIFunctionHandler@@@Z 3203e7d0 f   ScriptBind_Entity.obj
 0001:0003d850       ?GetAIName@CScriptBind_Entity@@IAEHPAUIFunctionHandler@@@Z 3203e850 f   ScriptBind_Entity.obj
 0001:0003d8e0       ?SetFlags@CScriptBind_Entity@@IAEHPAUIFunctionHandler@@HH@Z 3203e8e0 f   ScriptBind_Entity.obj
 0001:0003d950       ?GetFlags@CScriptBind_Entity@@IAEHPAUIFunctionHandler@@@Z 3203e950 f   ScriptBind_Entity.obj
 0001:0003d9f0       ?HasFlags@CScriptBind_Entity@@IAEHPAUIFunctionHandler@@H@Z 3203e9f0 f   ScriptBind_Entity.obj
 0001:0003da40       ?GetName@CScriptBind_Entity@@IAEHPAUIFunctionHandler@@@Z 3203ea40 f   ScriptBind_Entity.obj
 0001:0003dab0       ?GetRawId@CScriptBind_Entity@@IAEHPAUIFunctionHandler@@@Z 3203eab0 f   ScriptBind_Entity.obj
 0001:0003db20       ?GetArchetype@CScriptBind_Entity@@IAEHPAUIFunctionHandler@@@Z 3203eb20 f   ScriptBind_Entity.obj
 0001:0003dbb0       ?CreateRenderProxy@CScriptBind_Entity@@IAEHPAUIFunctionHandler@@@Z 3203ebb0 f   ScriptBind_Entity.obj
 0001:0003dc10       ?CheckShaderParamCallbacks@CScriptBind_Entity@@IAEHPAUIFunctionHandler@@@Z 3203ec10 f   ScriptBind_Entity.obj
 0001:0003dc70       ?LoadCharacter@CScriptBind_Entity@@IAEHPAUIFunctionHandler@@HPBD@Z 3203ec70 f   ScriptBind_Entity.obj
 0001:0003dcd0       ?LoadObject@CScriptBind_Entity@@IAEHPAUIFunctionHandler@@HPBD@Z 3203ecd0 f   ScriptBind_Entity.obj
 0001:0003dda0       ?LoadObjectWithFlags@CScriptBind_Entity@@IAEHPAUIFunctionHandler@@HPBDH@Z 3203eda0 f   ScriptBind_Entity.obj
 0001:0003de70       ?LoadObjectLattice@CScriptBind_Entity@@IAEHPAUIFunctionHandler@@H@Z 3203ee70 f   ScriptBind_Entity.obj
 0001:0003df70       ?LoadSubObject@CScriptBind_Entity@@IAEHPAUIFunctionHandler@@HPBD1@Z 3203ef70 f   ScriptBind_Entity.obj
 0001:0003dfd0       ?UpdateLightClipBounds@CScriptBind_Entity@@IAEHPAUIFunctionHandler@@H@Z 3203efd0 f   ScriptBind_Entity.obj
 0001:0003e060       ?SetSelfAsLightCasterException@CScriptBind_Entity@@IAEHPAUIFunctionHandler@@H@Z 3203f060 f   ScriptBind_Entity.obj
 0001:0003e100       ?LoadCloud@CScriptBind_Entity@@IAEHPAUIFunctionHandler@@HPBD@Z 3203f100 f   ScriptBind_Entity.obj
 0001:0003e1a0       ?LoadLightShape@CScriptBind_Entity@@IAEHPAUIFunctionHandler@@HPBDI@Z 3203f1a0 f   ScriptBind_Entity.obj
 0001:0003e250       ?FadeGlobalDensity@CScriptBind_Entity@@IAEHPAUIFunctionHandler@@HMM@Z 3203f250 f   ScriptBind_Entity.obj
 0001:0003e300       ?LoadVolumeObject@CScriptBind_Entity@@IAEHPAUIFunctionHandler@@HPBD@Z 3203f300 f   ScriptBind_Entity.obj
 0001:0003e3a0       ?LoadPrismObject@CScriptBind_Entity@@IAEHPAUIFunctionHandler@@H@Z 3203f3a0 f   ScriptBind_Entity.obj
 0001:0003e440       ?PreLoadParticleEffect@CScriptBind_Entity@@IAEHPAUIFunctionHandler@@PBD@Z 3203f440 f   ScriptBind_Entity.obj
 0001:0003e4f0       ?IsSlotParticleEmitter@CScriptBind_Entity@@IAEHPAUIFunctionHandler@@H@Z 3203f4f0 f   ScriptBind_Entity.obj
 0001:0003e560       ?IsSlotLight@CScriptBind_Entity@@IAEHPAUIFunctionHandler@@H@Z 3203f560 f   ScriptBind_Entity.obj
 0001:0003e5d0       ?IsSlotGeometry@CScriptBind_Entity@@IAEHPAUIFunctionHandler@@H@Z 3203f5d0 f   ScriptBind_Entity.obj
 0001:0003e640       ?IsSlotCharacter@CScriptBind_Entity@@IAEHPAUIFunctionHandler@@H@Z 3203f640 f   ScriptBind_Entity.obj
 0001:0003e6b0       ?SetParentSlot@CScriptBind_Entity@@IAEHPAUIFunctionHandler@@HH@Z 3203f6b0 f   ScriptBind_Entity.obj
 0001:0003e6f0       ?GetParentSlot@CScriptBind_Entity@@IAEHPAUIFunctionHandler@@H@Z 3203f6f0 f   ScriptBind_Entity.obj
 0001:0003e770       ?GetSlotCount@CScriptBind_Entity@@IAEHPAUIFunctionHandler@@@Z 3203f770 f   ScriptBind_Entity.obj
 0001:0003e810       ?SetSlotPos@CScriptBind_Entity@@IAEHPAUIFunctionHandler@@HU?$Vec3_tpl@M@@@Z 3203f810 f   ScriptBind_Entity.obj
 0001:0003e900       ?SetSlotPosAndDir@CScriptBind_Entity@@IAEHPAUIFunctionHandler@@HU?$Vec3_tpl@M@@1@Z 3203f900 f   ScriptBind_Entity.obj
 0001:0003ead0       ?GetSlotScale@CScriptBind_Entity@@IAEHPAUIFunctionHandler@@H@Z 3203fad0 f   ScriptBind_Entity.obj
 0001:0003eba0       ?CopySlotTM@CScriptBind_Entity@@IAEHPAUIFunctionHandler@@HH_N@Z 3203fba0 f   ScriptBind_Entity.obj
 0001:0003ecc0       ?MultiplyWithSlotTM@CScriptBind_Entity@@IAEHPAUIFunctionHandler@@HU?$Vec3_tpl@M@@@Z 3203fcc0 f   ScriptBind_Entity.obj
 0001:0003edf0       ?GetCharacter@CScriptBind_Entity@@IAEHPAUIFunctionHandler@@H@Z 3203fdf0 f   ScriptBind_Entity.obj
 0001:0003ee50       ?IsSlotValid@CScriptBind_Entity@@IAEHPAUIFunctionHandler@@H@Z 3203fe50 f   ScriptBind_Entity.obj
 0001:0003eea0       ?DrawSlot@CScriptBind_Entity@@IAEHPAUIFunctionHandler@@HH@Z 3203fea0 f   ScriptBind_Entity.obj
 0001:0003ef40       ?IgnorePhysicsUpdatesOnSlot@CScriptBind_Entity@@IAEHPAUIFunctionHandler@@H@Z 3203ff40 f   ScriptBind_Entity.obj
 0001:0003efa0       ?FreeSlot@CScriptBind_Entity@@IAEHPAUIFunctionHandler@@H@Z 3203ffa0 f   ScriptBind_Entity.obj
 0001:0003efd0       ?FreeAllSlots@CScriptBind_Entity@@IAEHPAUIFunctionHandler@@@Z 3203ffd0 f   ScriptBind_Entity.obj
 0001:0003f070       ?DestroyPhysics@CScriptBind_Entity@@IAEHPAUIFunctionHandler@@@Z 32040070 f   ScriptBind_Entity.obj
 0001:0003f110       ?EnablePhysics@CScriptBind_Entity@@IAEHPAUIFunctionHandler@@_N@Z 32040110 f   ScriptBind_Entity.obj
 0001:0003f180       ?ReattachSoftEntityVtx@CScriptBind_Entity@@IAEHPAUIFunctionHandler@@TScriptHandle@@H@Z 32040180 f   ScriptBind_Entity.obj
 0001:0003f210       ?UpdateSlotPhysics@CScriptBind_Entity@@IAEHPAUIFunctionHandler@@H@Z 32040210 f   ScriptBind_Entity.obj
 0001:0003f240       ?CreateBoneAttachment@CScriptBind_Entity@@IAEHPAUIFunctionHandler@@HPBD1@Z 32040240 f   ScriptBind_Entity.obj
 0001:0003f2e0       ?CreateSkinAttachment@CScriptBind_Entity@@IAEHPAUIFunctionHandler@@HPBD@Z 320402e0 f   ScriptBind_Entity.obj
 0001:0003f350       ?DestroyAttachment@CScriptBind_Entity@@IAEHPAUIFunctionHandler@@HPBD@Z 32040350 f   ScriptBind_Entity.obj
 0001:0003f3d0       ?GetAttachmentBone@CScriptBind_Entity@@IAEHPAUIFunctionHandler@@HPBD@Z 320403d0 f   ScriptBind_Entity.obj
 0001:0003f480       ?GetAttachmentCGF@CScriptBind_Entity@@IAEHPAUIFunctionHandler@@HPBD@Z 32040480 f   ScriptBind_Entity.obj
 0001:0003f520       ?ResetAttachment@CScriptBind_Entity@@IAEHPAUIFunctionHandler@@HPBD@Z 32040520 f   ScriptBind_Entity.obj
 0001:0003f590       ?GetSplineType@?$CBaseSplineInterpolator@MV?$OptSpline@U?$TFixed@E$00$0PP@@@V?$TSplineSlopes@MU?$SplineKey@M@spline@@$00@spline@@@spline@@@spline@@UAE?AW4ESplineType@@XZ 32040590 f i BreakablePlane.obj
 0001:0003f590       ?GetType@CPhysicalProxy@@UAE?AW4EEntityProxy@@XZ 32040590 f i PhysicsProxy.obj
 0001:0003f590       ?GetAttachmentType@CCGFAttachment@@UAE?AW4EType@IAttachmentObject@@XZ 32040590 f i ScriptBind_Entity.obj
 0001:0003f590       ?GetNumDimensions@?$CBaseSplineInterpolator@MV?$OptSpline@U?$TFixed@E$00$0PP@@@V?$TSplineSlopes@MU?$SplineKey@M@spline@@$00@spline@@@spline@@@spline@@UAEHXZ 32040590 f i BreakablePlane.obj
 0001:0003f5a0       ?RenderAttachment@CCGFAttachment@@UAEXAAUSRendParams@@ABUSRenderingPassInfo@@@Z 320405a0 f i ScriptBind_Entity.obj
 0001:0003f5f0       ?GetAABB@CCGFAttachment@@UAE?AUAABB@@XZ 320405f0 f i ScriptBind_Entity.obj
 0001:0003f610       ?GetRadiusSqr@CCGFAttachment@@UAEMXZ 32040610 f i ScriptBind_Entity.obj
 0001:0003f620       ?GetBaseMaterial@CCGFAttachment@@UBEPAUIMaterial@@XZ 32040620 f i ScriptBind_Entity.obj
 0001:0003f640       ?SetReplacementMaterial@CSKELAttachment@@UAEXPAUIMaterial@@@Z 32040640 f i ScriptBind_Entity.obj
 0001:0003f640       ?SetReplacementMaterial@CCGFAttachment@@UAEXPAUIMaterial@@@Z 32040640 f i ScriptBind_Entity.obj
 0001:0003f670       ?SetAttachmentCGF@CScriptBind_Entity@@IAEHPAUIFunctionHandler@@HPBD1@Z 32040670 f   ScriptBind_Entity.obj
 0001:0003f740       ??0?$QuatT_tpl@M@@QAE@ABU0@@Z 32040740 f i ScriptBind_Entity.obj
 0001:0003f780       ?HideAttachment@CScriptBind_Entity@@IAEHPAUIFunctionHandler@@HPBD_N2@Z 32040780 f   ScriptBind_Entity.obj
 0001:0003f800       ?HideAllAttachments@CScriptBind_Entity@@IAEHPAUIFunctionHandler@@H_N1@Z 32040800 f   ScriptBind_Entity.obj
 0001:0003f8c0       ?HideAttachmentMaster@CScriptBind_Entity@@IAEHPAUIFunctionHandler@@H_N@Z 320408c0 f   ScriptBind_Entity.obj
 0001:0003f910       ?PhysicalizeAttachment@CScriptBind_Entity@@IAEHPAUIFunctionHandler@@HPBD_N@Z 32040910 f   ScriptBind_Entity.obj
 0001:0003f9a0       ?AttachChild@CScriptBind_Entity@@IAEHPAUIFunctionHandler@@TScriptHandle@@H@Z 320409a0 f   ScriptBind_Entity.obj
 0001:0003fa30       ?DetachThis@CScriptBind_Entity@@IAEHPAUIFunctionHandler@@@Z 32040a30 f   ScriptBind_Entity.obj
 0001:0003fa90       ?DetachAll@CScriptBind_Entity@@IAEHPAUIFunctionHandler@@@Z 32040a90 f   ScriptBind_Entity.obj
 0001:0003fae0       ?GetParent@CScriptBind_Entity@@IAEHPAUIFunctionHandler@@@Z 32040ae0 f   ScriptBind_Entity.obj
 0001:0003fb50       ?GetChildCount@CScriptBind_Entity@@IAEHPAUIFunctionHandler@@@Z 32040b50 f   ScriptBind_Entity.obj
 0001:0003fbf0       ?GetChild@CScriptBind_Entity@@IAEHPAUIFunctionHandler@@H@Z 32040bf0 f   ScriptBind_Entity.obj
 0001:0003fc90       ?EnableInheritXForm@CScriptBind_Entity@@IAEHPAUIFunctionHandler@@_N@Z 32040c90 f   ScriptBind_Entity.obj
 0001:0003fcc0       ?NetPresent@CScriptBind_Entity@@IAEHPAUIFunctionHandler@@@Z 32040cc0 f   ScriptBind_Entity.obj
 0001:0003fd30       ?SetStateClientside@CScriptBind_Entity@@IAEHPAUIFunctionHandler@@@Z 32040d30 f   ScriptBind_Entity.obj
 0001:0003fda0       ?StartAnimation@CScriptBind_Entity@@IAEHPAUIFunctionHandler@@@Z 32040da0 f   ScriptBind_Entity.obj
 0001:000400b0       ?StopAnimation@CScriptBind_Entity@@IAEHPAUIFunctionHandler@@HH@Z 320410b0 f   ScriptBind_Entity.obj
 0001:00040140       ?ResetAnimation@CScriptBind_Entity@@IAEHPAUIFunctionHandler@@HH@Z 32041140 f   ScriptBind_Entity.obj
 0001:00040150       ?RedirectAnimationToLayer0@CScriptBind_Entity@@IAEHPAUIFunctionHandler@@H_N@Z 32041150 f   ScriptBind_Entity.obj
 0001:00040180       ?SetAnimationBlendOut@CScriptBind_Entity@@IAEHPAUIFunctionHandler@@HHM@Z 32041180 f   ScriptBind_Entity.obj
 0001:00040180       ?EnableBoneAnimationAll@CScriptBind_Entity@@IAEHPAUIFunctionHandler@@HH_N@Z 32041180 f   ScriptBind_Entity.obj
 0001:000401b0       ?EnableBoneAnimation@CScriptBind_Entity@@IAEHPAUIFunctionHandler@@HHPBD_N@Z 320411b0 f   ScriptBind_Entity.obj
 0001:000401b0       ?SetAnimationFlip@CScriptBind_Entity@@IAEHPAUIFunctionHandler@@HU?$Vec3_tpl@M@@@Z 320411b0 f   ScriptBind_Entity.obj
 0001:000401e0       ?EnableProceduralFacialAnimation@CScriptBind_Entity@@IAEHPAUIFunctionHandler@@_N@Z 320411e0 f   ScriptBind_Entity.obj
 0001:00040220       ?PlayFacialAnimation@CScriptBind_Entity@@IAEHPAUIFunctionHandler@@PAD_N@Z 32041220 f   ScriptBind_Entity.obj
 0001:000402a0       ?GetHelperDir@CScriptBind_Entity@@IAEHPAUIFunctionHandler@@@Z 320412a0 f   ScriptBind_Entity.obj
 0001:000406e0       ?RenderShadow@CScriptBind_Entity@@IAEHPAUIFunctionHandler@@@Z 320416e0 f   ScriptBind_Entity.obj
 0001:000407a0       ?SetRegisterInSectors@CScriptBind_Entity@@IAEHPAUIFunctionHandler@@@Z 320417a0 f   ScriptBind_Entity.obj
 0001:00040810       ?AwakePhysics@CScriptBind_Entity@@IAEHPAUIFunctionHandler@@H@Z 32041810 f   ScriptBind_Entity.obj
 0001:00040870       ?ResetPhysics@CScriptBind_Entity@@IAEHPAUIFunctionHandler@@@Z 32041870 f   ScriptBind_Entity.obj
 0001:000408d0       ?AwakeCharacterPhysics@CScriptBind_Entity@@IAEHPAUIFunctionHandler@@HPBDH@Z 320418d0 f   ScriptBind_Entity.obj
 0001:00040970       ??0SRenderLight@@QAE@XZ    32041970 f i ScriptBind_Entity.obj
 0001:00040c00       ?IsColliding@CScriptBind_Entity@@IAEHPAUIFunctionHandler@@@Z 32041c00 f   ScriptBind_Entity.obj
 0001:00040ca0       ?IsAnimationRunning@CScriptBind_Entity@@IAEHPAUIFunctionHandler@@HH@Z 32041ca0 f   ScriptBind_Entity.obj
 0001:00040d20       ?AddImpulse@CScriptBind_Entity@@IAEHPAUIFunctionHandler@@@Z 32041d20 f   ScriptBind_Entity.obj
 0001:000411b0       ?PlaySoundEvent@CScriptBind_Entity@@IAEHPAUIFunctionHandler@@PBDU?$Vec3_tpl@M@@2III@Z 320421b0 f   ScriptBind_Entity.obj
 0001:000412a0       ?PlaySoundEventEx@CScriptBind_Entity@@IAEHPAUIFunctionHandler@@PBDIIMU?$Vec3_tpl@M@@MMI@Z 320422a0 f   ScriptBind_Entity.obj
 0001:000413c0       ?SetSoundSphereSpec@CScriptBind_Entity@@IAEHPAUIFunctionHandler@@TScriptHandle@@M@Z 320423c0 f   ScriptBind_Entity.obj
 0001:00041430       ?SetStaticSound@CScriptBind_Entity@@IAEHPAUIFunctionHandler@@TScriptHandle@@_N@Z 32042430 f   ScriptBind_Entity.obj
 0001:00041480       ?StopAllSounds@CScriptBind_Entity@@IAEHPAUIFunctionHandler@@@Z 32042480 f   ScriptBind_Entity.obj
 0001:000414d0       ?PauseSound@CScriptBind_Entity@@IAEHPAUIFunctionHandler@@TScriptHandle@@_N@Z 320424d0 f   ScriptBind_Entity.obj
 0001:00041520       ?SetSoundEffectRadius@CScriptBind_Entity@@IAEHPAUIFunctionHandler@@M@Z 32042520 f   ScriptBind_Entity.obj
 0001:000415c0       ?TriggerEvent@CScriptBind_Entity@@IAEHPAUIFunctionHandler@@@Z 320425c0 f   ScriptBind_Entity.obj
 0001:00041700       ?SetLocalBBox@CScriptBind_Entity@@IAEHPAUIFunctionHandler@@U?$Vec3_tpl@M@@1@Z 32042700 f   ScriptBind_Entity.obj
 0001:00041770       ?SetTriggerBBox@CScriptBind_Entity@@IAEHPAUIFunctionHandler@@U?$Vec3_tpl@M@@1@Z 32042770 f   ScriptBind_Entity.obj
 0001:00041800       ?GetTriggerBBox@CScriptBind_Entity@@IAEHPAUIFunctionHandler@@@Z 32042800 f   ScriptBind_Entity.obj
 0001:000418a0       ?InvalidateTrigger@CScriptBind_Entity@@IAEHPAUIFunctionHandler@@@Z 320428a0 f   ScriptBind_Entity.obj
 0001:000418f0       ?ForwardTriggerEventsTo@CScriptBind_Entity@@IAEHPAUIFunctionHandler@@TScriptHandle@@@Z 320428f0 f   ScriptBind_Entity.obj
 0001:00041930       ?SetUpdateRadius@CScriptBind_Entity@@IAEHPAUIFunctionHandler@@@Z 32042930 f   ScriptBind_Entity.obj
 0001:00041990       ?GetUpdateRadius@CScriptBind_Entity@@IAEHPAUIFunctionHandler@@@Z 32042990 f   ScriptBind_Entity.obj
 0001:000419d0       ?Activate@CScriptBind_Entity@@IAEHPAUIFunctionHandler@@H@Z 320429d0 f   ScriptBind_Entity.obj
 0001:00041a10       ?IsActive@CScriptBind_Entity@@IAEHPAUIFunctionHandler@@@Z 32042a10 f   ScriptBind_Entity.obj
 0001:00041a50       ?IsFromPool@CScriptBind_Entity@@IAEHPAUIFunctionHandler@@@Z 32042a50 f   ScriptBind_Entity.obj
 0001:00041a90       ?SetUpdatePolicy@CScriptBind_Entity@@IAEHPAUIFunctionHandler@@H@Z 32042a90 f   ScriptBind_Entity.obj
 0001:00041ac0       ?SetAnimationSpeed@CScriptBind_Entity@@IAEHPAUIFunctionHandler@@HHM@Z 32042ac0 f   ScriptBind_Entity.obj
 0001:00041b40       ?SetAnimationTime@CScriptBind_Entity@@IAEHPAUIFunctionHandler@@HHM@Z 32042b40 f   ScriptBind_Entity.obj
 0001:00041b90       ?GetAnimationTime@CScriptBind_Entity@@IAEHPAUIFunctionHandler@@HH@Z 32042b90 f   ScriptBind_Entity.obj
 0001:00041c50       ?CancelSubpipe@CScriptBind_Entity@@IAEHPAUIFunctionHandler@@@Z 32042c50 f   ScriptBind_Entity.obj
 0001:00041d20       ?IsUsingPipe@CScriptBind_Entity@@IAEHPAUIFunctionHandler@@@Z 32042d20 f   ScriptBind_Entity.obj
 0001:00041df0       ?GotoState@CScriptBind_Entity@@IAEHPAUIFunctionHandler@@PBD@Z 32042df0 f   ScriptBind_Entity.obj
 0001:00041e50       ?IsInState@CScriptBind_Entity@@IAEHPAUIFunctionHandler@@PBD@Z 32042e50 f   ScriptBind_Entity.obj
 0001:00041eb0       ?GetState@CScriptBind_Entity@@IAEHPAUIFunctionHandler@@@Z 32042eb0 f   ScriptBind_Entity.obj
 0001:00041f10       ?GetCurAnimation@CScriptBind_Entity@@IAEHPAUIFunctionHandler@@@Z 32042f10 f   ScriptBind_Entity.obj
 0001:00041f90       ?SetTimer@CScriptBind_Entity@@IAEHPAUIFunctionHandler@@@Z 32042f90 f   ScriptBind_Entity.obj
 0001:00041ff0       ?KillTimer@CScriptBind_Entity@@IAEHPAUIFunctionHandler@@@Z 32042ff0 f   ScriptBind_Entity.obj
 0001:00042040       ?SetScriptUpdateRate@CScriptBind_Entity@@IAEHPAUIFunctionHandler@@H@Z 32043040 f   ScriptBind_Entity.obj
 0001:000420a0       ?IsHidden@CScriptBind_Entity@@IAEHPAUIFunctionHandler@@@Z 320430a0 f   ScriptBind_Entity.obj
 0001:000420e0       ?GetBoneNameFromTable@CScriptBind_Entity@@IAEHPAUIFunctionHandler@@@Z 320430e0 f   ScriptBind_Entity.obj
 0001:00042190       ?GetExplosionObstruction@CScriptBind_Entity@@IAEHPAUIFunctionHandler@@@Z 32043190 f   ScriptBind_Entity.obj
 0001:00042220       ?GetExplosionImpulse@CScriptBind_Entity@@IAEHPAUIFunctionHandler@@@Z 32043220 f   ScriptBind_Entity.obj
 0001:00042330       ?ActivatePlayerPhysics@CScriptBind_Entity@@IAEHPAUIFunctionHandler@@_N@Z 32043330 f   ScriptBind_Entity.obj
 0001:000423a0       ?SetDefaultIdleAnimations@CScriptBind_Entity@@IAEHPAUIFunctionHandler@@@Z 320433a0 f   ScriptBind_Entity.obj
 0001:00042400       ?GetAnimationLength@CScriptBind_Entity@@IAEHPAUIFunctionHandler@@HPBD@Z 32043400 f   ScriptBind_Entity.obj
 0001:00042510       ?SetMaterial@CScriptBind_Entity@@IAEHPAUIFunctionHandler@@@Z 32043510 f   ScriptBind_Entity.obj
 0001:000425c0       ?GetEntityMaterial@CScriptBind_Entity@@IAEHPAUIFunctionHandler@@@Z 320435c0 f   ScriptBind_Entity.obj
 0001:00042630       ?ReplaceMaterial@CScriptBind_Entity@@IAEHPAUIFunctionHandler@@HPBD1@Z 32043630 f   ScriptBind_Entity.obj
 0001:00042850       ?ResetMaterial@CScriptBind_Entity@@IAEHPAUIFunctionHandler@@H@Z 32043850 f   ScriptBind_Entity.obj
 0001:00042940       ?CloneMaterial@CScriptBind_Entity@@IAEHPAUIFunctionHandler@@H@Z 32043940 f   ScriptBind_Entity.obj
 0001:000429e0       ?SetMaterialFloat@CScriptBind_Entity@@IAEHPAUIFunctionHandler@@HHPBDM@Z 320439e0 f   ScriptBind_Entity.obj
 0001:00042a70       ?GetMaterialFloat@CScriptBind_Entity@@IAEHPAUIFunctionHandler@@HHPBD@Z 32043a70 f   ScriptBind_Entity.obj
 0001:00042b70       ?SetMaterialVec3@CScriptBind_Entity@@IAEHPAUIFunctionHandler@@HHPBDU?$Vec3_tpl@M@@@Z 32043b70 f   ScriptBind_Entity.obj
 0001:00042c00       ?GetMaterialVec3@CScriptBind_Entity@@IAEHPAUIFunctionHandler@@HHPBD@Z 32043c00 f   ScriptBind_Entity.obj
 0001:00042d20       ?MaterialFlashInvoke@CScriptBind_Entity@@IAEHPAUIFunctionHandler@@@Z 32043d20 f   ScriptBind_Entity.obj
 0001:000430f0       ?EnableMaterialLayer@CScriptBind_Entity@@IAEHPAUIFunctionHandler@@_NH@Z 320440f0 f   ScriptBind_Entity.obj
 0001:00043170       ?SetVelocity@CScriptBind_Entity@@IAEHPAUIFunctionHandler@@U?$Vec3_tpl@M@@@Z 32044170 f   ScriptBind_Entity.obj
 0001:000431f0       ?SetVelocityEx@CScriptBind_Entity@@IAEHPAUIFunctionHandler@@U?$Vec3_tpl@M@@1@Z 320441f0 f   ScriptBind_Entity.obj
 0001:00043270       ?GetSpeed@CScriptBind_Entity@@IAEHPAUIFunctionHandler@@@Z 32044270 f   ScriptBind_Entity.obj
 0001:000433e0       ?GetMass@CScriptBind_Entity@@IAEHPAUIFunctionHandler@@@Z 320443e0 f   ScriptBind_Entity.obj
 0001:00043500       ?GetVolume@CScriptBind_Entity@@IAEHPAUIFunctionHandler@@H@Z 32044500 f   ScriptBind_Entity.obj
 0001:000435e0       ?GetSubmergedVolume@CScriptBind_Entity@@IAEHPAUIFunctionHandler@@HU?$Vec3_tpl@M@@1@Z 320445e0 f   ScriptBind_Entity.obj
 0001:000438b0       ?CreateLink@CScriptBind_Entity@@IAEHPAUIFunctionHandler@@PBD@Z 320448b0 f   ScriptBind_Entity.obj
 0001:00043970       ?GetLinkName@CScriptBind_Entity@@IAEHPAUIFunctionHandler@@TScriptHandle@@@Z 32044970 f   ScriptBind_Entity.obj
 0001:00043a20       ?SetLinkTarget@CScriptBind_Entity@@IAEHPAUIFunctionHandler@@PBDTScriptHandle@@@Z 32044a20 f   ScriptBind_Entity.obj
 0001:00043ab0       ?GetLinkTarget@CScriptBind_Entity@@IAEHPAUIFunctionHandler@@PBD@Z 32044ab0 f   ScriptBind_Entity.obj
 0001:00043b90       ?RemoveLink@CScriptBind_Entity@@IAEHPAUIFunctionHandler@@PBD@Z 32044b90 f   ScriptBind_Entity.obj
 0001:00043c20       ?RemoveAllLinks@CScriptBind_Entity@@IAEHPAUIFunctionHandler@@@Z 32044c20 f   ScriptBind_Entity.obj
 0001:00043c60       ?GetLink@CScriptBind_Entity@@IAEHPAUIFunctionHandler@@H@Z 32044c60 f   ScriptBind_Entity.obj
 0001:00043d40       ?CountLinks@CScriptBind_Entity@@IAEHPAUIFunctionHandler@@@Z 32044d40 f   ScriptBind_Entity.obj
 0001:00043df0       ?GetTimeSinceLastSeen@CScriptBind_Entity@@IAEHPAUIFunctionHandler@@@Z 32044df0 f   ScriptBind_Entity.obj
 0001:00043ec0       ?GetViewDistRatio@CScriptBind_Entity@@IAEHPAUIFunctionHandler@@@Z 32044ec0 f   ScriptBind_Entity.obj
 0001:00043f80       ?SetViewDistRatio@CScriptBind_Entity@@IAEHPAUIFunctionHandler@@@Z 32044f80 f   ScriptBind_Entity.obj
 0001:00044020       ?SetViewDistUnlimited@CScriptBind_Entity@@IAEHPAUIFunctionHandler@@@Z 32045020 f   ScriptBind_Entity.obj
 0001:00044080       ?SetLodRatio@CScriptBind_Entity@@IAEHPAUIFunctionHandler@@@Z 32045080 f   ScriptBind_Entity.obj
 0001:00044120       ?GetLodRatio@CScriptBind_Entity@@IAEHPAUIFunctionHandler@@@Z 32045120 f   ScriptBind_Entity.obj
 0001:000441e0       ?RemoveDecals@CScriptBind_Entity@@IAEHPAUIFunctionHandler@@@Z 320451e0 f   ScriptBind_Entity.obj
 0001:00044240       ?EnableDecals@CScriptBind_Entity@@IAEHPAUIFunctionHandler@@H_N@Z 32045240 f   ScriptBind_Entity.obj
 0001:00044290       ?ForceCharacterUpdate@CScriptBind_Entity@@IAEHPAUIFunctionHandler@@H_N@Z 32045290 f   ScriptBind_Entity.obj
 0001:00044330       ?CharacterUpdateAlways@CScriptBind_Entity@@IAEHPAUIFunctionHandler@@H_N@Z 32045330 f   ScriptBind_Entity.obj
 0001:00044390       ?CharacterUpdateOnRender@CScriptBind_Entity@@IAEHPAUIFunctionHandler@@H_N@Z 32045390 f   ScriptBind_Entity.obj
 0001:00044410       ?Hide@CScriptBind_Entity@@IAEHPAUIFunctionHandler@@@Z 32045410 f   ScriptBind_Entity.obj
 0001:000444a0       ?AwakeEnvironment@CScriptBind_Entity@@IAEHPAUIFunctionHandler@@@Z 320454a0 f   ScriptBind_Entity.obj
 0001:00044630       ?NoExplosionCollision@CScriptBind_Entity@@IAEHPAUIFunctionHandler@@@Z 32045630 f   ScriptBind_Entity.obj
 0001:000446e0       ?NoBulletForce@CScriptBind_Entity@@IAEHPAUIFunctionHandler@@_N@Z 320456e0 f   ScriptBind_Entity.obj
 0001:00044790       ?GetPhysicalStats@CScriptBind_Entity@@IAEHPAUIFunctionHandler@@@Z 32045790 f   ScriptBind_Entity.obj
 0001:00044930       ?UpdateAreas@CScriptBind_Entity@@IAEHPAUIFunctionHandler@@@Z 32045930 f   ScriptBind_Entity.obj
 0001:000449c0       ??4pe_params_particle@@QAEAAU0@ABU0@@Z 320459c0 f i ScriptBind_Entity.obj
 0001:00044ae0       ?GetDistance@CScriptBind_Entity@@IAEHPAUIFunctionHandler@@@Z 32045ae0 f   ScriptBind_Entity.obj
 0001:00044be0       ?IStatObjRayIntersect@CScriptBind_Entity@@AAEHPAUIStatObj@@ABU?$Vec3_tpl@M@@1MPAUSIntersectionResult@1@I@Z 32045be0 f   ScriptBind_Entity.obj
 0001:00045080       ?GetSoundPtr@CScriptBind_Entity@@AAEPAUISound@@PAUIFunctionHandler@@H@Z 32046080 f   ScriptBind_Entity.obj
 0001:00045110       ?CreateCameraProxy@CScriptBind_Entity@@IAEHPAUIFunctionHandler@@@Z 32046110 f   ScriptBind_Entity.obj
 0001:00045190       ?BreakToPieces@CScriptBind_Entity@@IAEHPAUIFunctionHandler@@HHMU?$Vec3_tpl@M@@1M_N@Z 32046190 f   ScriptBind_Entity.obj
 0001:00045230       ?AttachSurfaceEffect@CScriptBind_Entity@@IAEHPAUIFunctionHandler@@HPBD_N11MM@Z 32046230 f   ScriptBind_Entity.obj
 0001:000453c0       ?SetColliderMode@CScriptBind_Entity@@IAEHPAUIFunctionHandler@@H@Z 320463c0 f   ScriptBind_Entity.obj
 0001:00045420       ?UnSeenFrames@CScriptBind_Entity@@IAEHPAUIFunctionHandler@@@Z 32046420 f   ScriptBind_Entity.obj
 0001:00045510       ?DeleteParticleEmitter@CScriptBind_Entity@@IAEHPAUIFunctionHandler@@H@Z 32046510 f   ScriptBind_Entity.obj
 0001:000455b0       ?RegisterForAreaEvents@CScriptBind_Entity@@IAEHPAUIFunctionHandler@@H@Z 320465b0 f   ScriptBind_Entity.obj
 0001:00045610       ?RenderAlways@CScriptBind_Entity@@IAEHPAUIFunctionHandler@@H@Z 32046610 f   ScriptBind_Entity.obj
 0001:000456a0       ?IsValid@?$Vec3_tpl@M@@QBE_NXZ 320466a0 f i ScriptBind_Entity.obj
 0001:000456e0       ?init@?$DynArray@UGoalParams@@HU?$SmallDynStorage@UGoalParams@@HUStandardAlloc@NAlloc@@@NArray@@@@KAPAUGoalParams@@U?$Array@UGoalParams@@HU?$ArrayStorage@UGoalParams@@H@NArray@@@@PBU2@@Z 320466e0 f i ScriptBind_Entity.obj
 0001:00045740       ??$Construct@Upe_player_dimensions@@@@YAXAAUpe_player_dimensions@@@Z 32046740 f i ScriptBind_Entity.obj
 0001:000457e0       ??$Construct@Upe_params_area@@@@YAXAAUpe_params_area@@@Z 320467e0 f i ScriptBind_Entity.obj
 0001:00045840       ??$Construct@UAreaDefinition@SEntityPhysicalizeParams@@@@YAXAAUAreaDefinition@SEntityPhysicalizeParams@@@Z 32046840 f i ScriptBind_Entity.obj
 0001:000458b0       ??$move_init@UGoalParams@@@NArray@@YAXPAUGoalParams@@0I@Z 320468b0 f i ScriptBind_Entity.obj
 0001:000458f0       ?Dispatch@?$CallDispatcher@VCScriptBind_Entity@@P81@AEHPAUIFunctionHandler@@H@Z@ScriptTemplateCallHelper@@SAHPAUIFunctionHandler@@PAXH@Z 320468f0 f i ScriptBind_Entity.obj
 0001:00045930       ?Dispatch@?$CallDispatcher@VCScriptBind_Entity@@P81@AEHPAUIFunctionHandler@@HVSmartScriptTable@@@Z@ScriptTemplateCallHelper@@SAHPAUIFunctionHandler@@PAXH@Z 32046930 f i ScriptBind_Entity.obj
 0001:00045950       ?Dispatch@?$CallDispatcher@VCScriptBind_Entity@@P81@AEHPAUIFunctionHandler@@HH@Z@ScriptTemplateCallHelper@@SAHPAUIFunctionHandler@@PAXH@Z 32046950 f i ScriptBind_Entity.obj
 0001:000459b0       ?Dispatch@?$CallDispatcher@VCScriptBind_Entity@@P81@AEHPAUIFunctionHandler@@@Z@ScriptTemplateCallHelper@@SAHPAUIFunctionHandler@@PAXH@Z 320469b0 f i ScriptBind_Entity.obj
 0001:000459d0       ?Dispatch@?$CallDispatcher@VCScriptBind_Entity@@P81@AEHPAUIFunctionHandler@@_N@Z@ScriptTemplateCallHelper@@SAHPAUIFunctionHandler@@PAXH@Z 320469d0 f i ScriptBind_Entity.obj
 0001:00045a10       ?GetLimit@CCustomInfo@?$TFixed@E$00$0PP@@@UBE_NW4ENumericLimit@@AAM@Z 32046a10 f i ScriptBind_Entity.obj
 0001:00045a70       ?IsType@?$TProxyTypeInfo@MU?$TFixed@E$00$0PP@@@@@UBE_NABUCTypeInfo@@@Z 32046a70 f i ScriptBind_Entity.obj
 0001:00045ab0       ?ToValue@?$TProxyTypeInfo@MU?$TFixed@E$00$0PP@@@@@UBE_NPBXPAXABUCTypeInfo@@@Z 32046ab0 f i ScriptBind_Entity.obj
 0001:00045b10       ?EnumElem@?$TProxyTypeInfo@MU?$TFixed@E$00$0PP@@@@@UBEPBDI@Z 32046b10 f i ScriptBind_Entity.obj
 0001:00045b30       ??$Call@VCScriptBind_Entity@@HPBDH@ScriptTemplateCallHelper@@SAHPAVCScriptBind_Entity@@P81@AEHPAUIFunctionHandler@@HPBDH@Z1@Z 32046b30 f i ScriptBind_Entity.obj
 0001:00045ba0       ??$Call@VCScriptBind_Entity@@HPBDPBD@ScriptTemplateCallHelper@@SAHPAVCScriptBind_Entity@@P81@AEHPAUIFunctionHandler@@HPBD2@Z1@Z 32046ba0 f i ScriptBind_Entity.obj
 0001:00045c10       ??$Call@VCScriptBind_Entity@@HMM@ScriptTemplateCallHelper@@SAHPAVCScriptBind_Entity@@P81@AEHPAUIFunctionHandler@@HMM@Z1@Z 32046c10 f i ScriptBind_Entity.obj
 0001:00045c80       ??$Call@VCScriptBind_Entity@@HPBDVSmartScriptTable@@@ScriptTemplateCallHelper@@SAHPAVCScriptBind_Entity@@P81@AEHPAUIFunctionHandler@@HPBDVSmartScriptTable@@@Z1@Z 32046c80 f i ScriptBind_Entity.obj
 0001:00045d20       ??$Call@VCScriptBind_Entity@@HU?$Vec3_tpl@M@@U2@@ScriptTemplateCallHelper@@SAHPAVCScriptBind_Entity@@P81@AEHPAUIFunctionHandler@@HU?$Vec3_tpl@M@@2@Z1@Z 32046d20 f i ScriptBind_Entity.obj
 0001:00045db0       ??$Call@VCScriptBind_Entity@@HH_N@ScriptTemplateCallHelper@@SAHPAVCScriptBind_Entity@@P81@AEHPAUIFunctionHandler@@HH_N@Z1@Z 32046db0 f i ScriptBind_Entity.obj
 0001:00045e20       ??$Call@VCScriptBind_Entity@@HHVSmartScriptTable@@@ScriptTemplateCallHelper@@SAHPAVCScriptBind_Entity@@P81@AEHPAUIFunctionHandler@@HHVSmartScriptTable@@@Z1@Z 32046e20 f i ScriptBind_Entity.obj
 0001:00045ec0       ??$Call@VCScriptBind_Entity@@HU?$Vec3_tpl@M@@U2@M@ScriptTemplateCallHelper@@SAHPAVCScriptBind_Entity@@P81@AEHPAUIFunctionHandler@@HU?$Vec3_tpl@M@@2M@Z1@Z 32046ec0 f i ScriptBind_Entity.obj
 0001:00045f60       ??$Call@VCScriptBind_Entity@@HHM@ScriptTemplateCallHelper@@SAHPAVCScriptBind_Entity@@P81@AEHPAUIFunctionHandler@@HHM@Z1@Z 32046f60 f i ScriptBind_Entity.obj
 0001:00045fd0       ??$Call@VCScriptBind_Entity@@HHPBD_N@ScriptTemplateCallHelper@@SAHPAVCScriptBind_Entity@@P81@AEHPAUIFunctionHandler@@HHPBD_N@Z1@Z 32046fd0 f i ScriptBind_Entity.obj
 0001:00046050       ??$Call@VCScriptBind_Entity@@HPBD_N@ScriptTemplateCallHelper@@SAHPAVCScriptBind_Entity@@P81@AEHPAUIFunctionHandler@@HPBD_N@Z1@Z 32047050 f i ScriptBind_Entity.obj
 0001:000460c0       ??$Call@VCScriptBind_Entity@@U?$Vec3_tpl@M@@U2@@ScriptTemplateCallHelper@@SAHPAVCScriptBind_Entity@@P81@AEHPAUIFunctionHandler@@U?$Vec3_tpl@M@@2@Z1@Z 320470c0 f i ScriptBind_Entity.obj
 0001:00046140       ??$Call@VCScriptBind_Entity@@HPBDPBDU?$Vec3_tpl@M@@U2@MH@ScriptTemplateCallHelper@@SAHPAVCScriptBind_Entity@@P81@AEHPAUIFunctionHandler@@HPBD2U?$Vec3_tpl@M@@3MH@Z1@Z 32047140 f i ScriptBind_Entity.obj
 0001:000461d0       ??$Call@VCScriptBind_Entity@@HPBDTScriptHandle@@HH@ScriptTemplateCallHelper@@SAHPAVCScriptBind_Entity@@P81@AEHPAUIFunctionHandler@@HPBDTScriptHandle@@HH@Z1@Z 320471d0 f i ScriptBind_Entity.obj
 0001:00046270       ??$Call@VCScriptBind_Entity@@HPBDVSmartScriptTable@@H@ScriptTemplateCallHelper@@SAHPAVCScriptBind_Entity@@P81@AEHPAUIFunctionHandler@@HPBDVSmartScriptTable@@H@Z1@Z 32047270 f i ScriptBind_Entity.obj
 0001:00046330       ??$Call@VCScriptBind_Entity@@HPBDU?$Vec3_tpl@M@@@ScriptTemplateCallHelper@@SAHPAVCScriptBind_Entity@@P81@AEHPAUIFunctionHandler@@HPBDU?$Vec3_tpl@M@@@Z1@Z 32047330 f i ScriptBind_Entity.obj
 0001:000463b0       ??$Call@VCScriptBind_Entity@@HPBDU?$Vec3_tpl@M@@_N@ScriptTemplateCallHelper@@SAHPAVCScriptBind_Entity@@P81@AEHPAUIFunctionHandler@@HPBDU?$Vec3_tpl@M@@_N@Z1@Z 320473b0 f i ScriptBind_Entity.obj
 0001:00046440       ??$Call@VCScriptBind_Entity@@HPBD_N_N@ScriptTemplateCallHelper@@SAHPAVCScriptBind_Entity@@P81@AEHPAUIFunctionHandler@@HPBD_N3@Z1@Z 32047440 f i ScriptBind_Entity.obj
 0001:000464c0       ??$Call@VCScriptBind_Entity@@H_N_N@ScriptTemplateCallHelper@@SAHPAVCScriptBind_Entity@@P81@AEHPAUIFunctionHandler@@H_N2@Z1@Z 320474c0 f i ScriptBind_Entity.obj
 0001:00046530       ??$Call@VCScriptBind_Entity@@HHPBDM@ScriptTemplateCallHelper@@SAHPAVCScriptBind_Entity@@P81@AEHPAUIFunctionHandler@@HHPBDM@Z1@Z 32047530 f i ScriptBind_Entity.obj
 0001:000465b0       ??$Call@VCScriptBind_Entity@@HHPBD@ScriptTemplateCallHelper@@SAHPAVCScriptBind_Entity@@P81@AEHPAUIFunctionHandler@@HHPBD@Z1@Z 320475b0 f i ScriptBind_Entity.obj
 0001:00046620       ??$Call@VCScriptBind_Entity@@HHPBDU?$Vec3_tpl@M@@@ScriptTemplateCallHelper@@SAHPAVCScriptBind_Entity@@P81@AEHPAUIFunctionHandler@@HHPBDU?$Vec3_tpl@M@@@Z1@Z 32047620 f i ScriptBind_Entity.obj
 0001:000466b0       ??$Call@VCScriptBind_Entity@@HHMU?$Vec3_tpl@M@@U2@M_N@ScriptTemplateCallHelper@@SAHPAVCScriptBind_Entity@@P81@AEHPAUIFunctionHandler@@HHMU?$Vec3_tpl@M@@2M_N@Z1@Z 320476b0 f i ScriptBind_Entity.obj
 0001:00046750       ??$Call@VCScriptBind_Entity@@HPBD_NPBDPBDMM@ScriptTemplateCallHelper@@SAHPAVCScriptBind_Entity@@P81@AEHPAUIFunctionHandler@@HPBD_N22MM@Z1@Z 32047750 f i ScriptBind_Entity.obj
 0001:000467c0       ??$GetParams@PBDIIMU?$Vec3_tpl@M@@MMI@IFunctionHandler@@QAE_NAAPBDAAI1AAMAAU?$Vec3_tpl@M@@221@Z 320477c0 f i ScriptBind_Entity.obj
 0001:00046860       ?Set@CScriptVector@@QAEXABU?$Vec3_tpl@M@@@Z 32047860 f i ScriptBind_Entity.obj
 0001:000469b0       ?SetCachedVector@Script@@SA?AVSmartScriptTable@@ABU?$Vec3_tpl@M@@PAUIFunctionHandler@@H@Z 320479b0 f i ScriptBind_Entity.obj
 0001:00046b10       ?RenderAttachment@CSKELAttachment@@UAEXAAUSRendParams@@ABUSRenderingPassInfo@@@Z 32047b10 f i ScriptBind_Entity.obj
 0001:00046bb0       ?GetAABB@CSKELAttachment@@UAE?AUAABB@@XZ 32047bb0 f i ScriptBind_Entity.obj
 0001:00046c90       ??_ECSKELAttachment@@UAEPAXI@Z 32047c90 f i ScriptBind_Entity.obj
 0001:00046c90       ??_GCSKELAttachment@@UAEPAXI@Z 32047c90 f i ScriptBind_Entity.obj
 0001:00046cd0       ??0CEffectAttachment@@QAE@PBDABU?$Vec3_tpl@M@@1M@Z 32047cd0 f i ScriptBind_Entity.obj
 0001:00046d60       ?GetAttachmentType@CEffectAttachment@@UAE?AW4EType@IAttachmentObject@@XZ 32047d60 f i ScriptBind_Entity.obj
 0001:00046d70       ?GetAABB@CEffectAttachment@@UAE?AUAABB@@XZ 32047d70 f i ScriptBind_Entity.obj
 0001:00046e30       ?GetRadiusSqr@CEffectAttachment@@UAEMXZ 32047e30 f i ScriptBind_Entity.obj
 0001:00046ec0       ??4?$_smart_ptr@UIParticleEmitter@@@@QAEAAV0@PAUIParticleEmitter@@@Z 32047ec0 f i ScriptBind_Entity.obj
 0001:00046f30       ??1CEffectAttachment@@UAE@XZ 32047f30 f i ScriptBind_Entity.obj
 0001:00047000       ?CreateEffect@CEffectAttachment@@QAEXABU?$Matrix34_tpl@M@@@Z 32048000 f i ScriptBind_Entity.obj
 0001:00047470       ?ProcessAttachment@CEffectAttachment@@UAEXPAUIAttachment@@@Z 32048470 f i ScriptBind_Entity.obj
 0001:000479e0       ??_GCEffectAttachment@@UAEPAXI@Z 320489e0 f i ScriptBind_Entity.obj
 0001:000479e0       ??_ECEffectAttachment@@UAEPAXI@Z 320489e0 f i ScriptBind_Entity.obj
 0001:00047a10       ?OBB_OBB@Overlap@@YA_NABU?$Vec3_tpl@M@@ABU?$OBB_tpl@M@@01@Z 32048a10 f i ScriptBind_Entity.obj
 0001:00048180       ??0pe_params_buoyancy@@QAE@XZ 32049180 f i ScriptBind_Entity.obj
 0001:00048220       ?GetWorldPos@CScriptBind_Entity@@IAEHPAUIFunctionHandler@@@Z 32049220 f   ScriptBind_Entity.obj
 0001:00048220       ?GetPos@CScriptBind_Entity@@IAEHPAUIFunctionHandler@@@Z 32049220 f   ScriptBind_Entity.obj
 0001:00048290       ?GetCenterOfMassPos@CScriptBind_Entity@@IAEHPAUIFunctionHandler@@@Z 32049290 f   ScriptBind_Entity.obj
 0001:000483b0       ?GetWorldBoundsCenter@CScriptBind_Entity@@IAEHPAUIFunctionHandler@@@Z 320493b0 f   ScriptBind_Entity.obj
 0001:000484b0       ?SetAngles@CScriptBind_Entity@@IAEHPAUIFunctionHandler@@U?$Ang3_tpl@M@@@Z 320494b0 f   ScriptBind_Entity.obj
 0001:00048610       ?SetWorldAngles@CScriptBind_Entity@@IAEHPAUIFunctionHandler@@U?$Ang3_tpl@M@@@Z 32049610 f   ScriptBind_Entity.obj
 0001:000488a0       ?GetAngles@CScriptBind_Entity@@IAEHPAUIFunctionHandler@@@Z 320498a0 f   ScriptBind_Entity.obj
 0001:00048a40       ?GetWorldAngles@CScriptBind_Entity@@IAEHPAUIFunctionHandler@@@Z 32049a40 f   ScriptBind_Entity.obj
 0001:00048ad0       ?GetBoneLocal@CScriptBind_Entity@@IAEHPAUIFunctionHandler@@PBDU?$Vec3_tpl@M@@@Z 32049ad0 f   ScriptBind_Entity.obj
 0001:00048f90       ?IsEntityInside@CScriptBind_Entity@@IAEHPAUIFunctionHandler@@TScriptHandle@@@Z 32049f90 f   ScriptBind_Entity.obj
 0001:000492a0       ?GetLocalPos@CScriptBind_Entity@@IAEHPAUIFunctionHandler@@@Z 3204a2a0 f   ScriptBind_Entity.obj
 0001:00049300       ?SetLocalAngles@CScriptBind_Entity@@IAEHPAUIFunctionHandler@@U?$Ang3_tpl@M@@@Z 3204a300 f   ScriptBind_Entity.obj
 0001:00049460       ?GetLocalAngles@CScriptBind_Entity@@IAEHPAUIFunctionHandler@@@Z 3204a460 f   ScriptBind_Entity.obj
 0001:00049600       ?SetAIName@CScriptBind_Entity@@IAEHPAUIFunctionHandler@@@Z 3204a600 f   ScriptBind_Entity.obj
 0001:00049670       ?LoadParticleEffect@CScriptBind_Entity@@IAEHPAUIFunctionHandler@@HPBDVSmartScriptTable@@@Z 3204a670 f   ScriptBind_Entity.obj
 0001:000498f0       ?GetSlotPos@CScriptBind_Entity@@IAEHPAUIFunctionHandler@@H@Z 3204a8f0 f   ScriptBind_Entity.obj
 0001:00049980       ?GetSlotAngles@CScriptBind_Entity@@IAEHPAUIFunctionHandler@@H@Z 3204a980 f   ScriptBind_Entity.obj
 0001:00049bd0       ?SetSlotWorldTM@CScriptBind_Entity@@IAEHPAUIFunctionHandler@@HU?$Vec3_tpl@M@@1@Z 3204abd0 f   ScriptBind_Entity.obj
 0001:0004a270       ?GetSlotWorldPos@CScriptBind_Entity@@IAEHPAUIFunctionHandler@@H@Z 3204b270 f   ScriptBind_Entity.obj
 0001:0004a270       ?GetSlotWorldDir@CScriptBind_Entity@@IAEHPAUIFunctionHandler@@H@Z 3204b270 f   ScriptBind_Entity.obj
 0001:0004a300       ?GetDirectionVector@CScriptBind_Entity@@IAEHPAUIFunctionHandler@@@Z 3204b300 f   ScriptBind_Entity.obj
 0001:0004a4a0       ?SetDirectionVector@CScriptBind_Entity@@IAEHPAUIFunctionHandler@@U?$Vec3_tpl@M@@@Z 3204b4a0 f   ScriptBind_Entity.obj
 0001:0004a780       ?SetAttachmentEffect@CScriptBind_Entity@@IAEHPAUIFunctionHandler@@HPBD1U?$Vec3_tpl@M@@2MH@Z 3204b780 f   ScriptBind_Entity.obj
 0001:0004a830       ?SetAttachmentObject@CScriptBind_Entity@@IAEHPAUIFunctionHandler@@HPBDTScriptHandle@@HH@Z 3204b830 f   ScriptBind_Entity.obj
 0001:0004a9c0       ??_GCCGFAttachment@@UAEPAXI@Z 3204b9c0 f i ScriptBind_Entity.obj
 0001:0004a9c0       ??_ECCGFAttachment@@UAEPAXI@Z 3204b9c0 f i ScriptBind_Entity.obj
 0001:0004aa00       ?SetAttachmentPos@CScriptBind_Entity@@IAEHPAUIFunctionHandler@@HPBDU?$Vec3_tpl@M@@@Z 3204ba00 f   ScriptBind_Entity.obj
 0001:0004aac0       ?SetAttachmentAngles@CScriptBind_Entity@@IAEHPAUIFunctionHandler@@HPBDU?$Vec3_tpl@M@@@Z 3204bac0 f   ScriptBind_Entity.obj
 0001:0004ac90       ?GetHelperPos@CScriptBind_Entity@@IAEHPAUIFunctionHandler@@@Z 3204bc90 f   ScriptBind_Entity.obj
 0001:0004b2d0       ?GetHelperAngles@CScriptBind_Entity@@IAEHPAUIFunctionHandler@@@Z 3204c2d0 f   ScriptBind_Entity.obj
 0001:0004b870       ?GetSlotHelperPos@CScriptBind_Entity@@IAEHPAUIFunctionHandler@@HPBD_N@Z 3204c870 f   ScriptBind_Entity.obj
 0001:0004bba0       ?SetEntityPhysicParams@CScriptBind_Entity@@AAEHPAUIFunctionHandler@@PAUIPhysicalEntity@@HPAUIScriptTable@@PAUICharacterInstance@@@Z 3204cba0 f   ScriptBind_Entity.obj
 0001:0004e2d0       ?AddConstraint@CScriptBind_Entity@@IAEHPAUIFunctionHandler@@@Z 3204f2d0 f   ScriptBind_Entity.obj
 0001:0004e910       ?PlaySound@CScriptBind_Entity@@IAEHPAUIFunctionHandler@@@Z 3204f910 f   ScriptBind_Entity.obj
 0001:0004ea00       ?SetMatrix@CDLight@@QAEXABU?$Matrix34_tpl@M@@_N@Z 3204fa00 f i ScriptBind_Entity.obj
 0001:0004f010       ?StopSound@CScriptBind_Entity@@IAEHPAUIFunctionHandler@@@Z 32050010 f   ScriptBind_Entity.obj
 0001:0004f090       ?GetLocalBBox@CScriptBind_Entity@@IAEHPAUIFunctionHandler@@@Z 32050090 f   ScriptBind_Entity.obj
 0001:0004f390       ?GetWorldBBox@CScriptBind_Entity@@IAEHPAUIFunctionHandler@@@Z 32050390 f   ScriptBind_Entity.obj
 0001:0004f470       ?GetProjectedWorldBBox@CScriptBind_Entity@@IAEHPAUIFunctionHandler@@@Z 32050470 f   ScriptBind_Entity.obj
 0001:0004fb80       ?GetBonePos@CScriptBind_Entity@@IAEHPAUIFunctionHandler@@@Z 32050b80 f   ScriptBind_Entity.obj
 0001:0004fd30       ?GetBoneDir@CScriptBind_Entity@@IAEHPAUIFunctionHandler@@@Z 32050d30 f   ScriptBind_Entity.obj
 0001:0004ff60       ?GetBoneVelocity@CScriptBind_Entity@@IAEHPAUIFunctionHandler@@HPBD@Z 32050f60 f   ScriptBind_Entity.obj
 0001:00050050       ?GetBoneAngularVelocity@CScriptBind_Entity@@IAEHPAUIFunctionHandler@@HPBD@Z 32051050 f   ScriptBind_Entity.obj
 0001:00050130       ?GetTouchedSurfaceID@CScriptBind_Entity@@IAEHPAUIFunctionHandler@@@Z 32051130 f   ScriptBind_Entity.obj
 0001:000501d0       ?GetTouchedPoint@CScriptBind_Entity@@IAEHPAUIFunctionHandler@@@Z 320511d0 f   ScriptBind_Entity.obj
 0001:000502c0       ?ToLocal@CScriptBind_Entity@@IAEHPAUIFunctionHandler@@HU?$Vec3_tpl@M@@@Z 320512c0 f   ScriptBind_Entity.obj
 0001:000504a0       ?ToGlobal@CScriptBind_Entity@@IAEHPAUIFunctionHandler@@HU?$Vec3_tpl@M@@@Z 320514a0 f   ScriptBind_Entity.obj
 0001:000505f0       ?VectorToLocal@CScriptBind_Entity@@IAEHPAUIFunctionHandler@@HU?$Vec3_tpl@M@@@Z 320515f0 f   ScriptBind_Entity.obj
 0001:00050720       ?VectorToGlobal@CScriptBind_Entity@@IAEHPAUIFunctionHandler@@HU?$Vec3_tpl@M@@@Z 32051720 f   ScriptBind_Entity.obj
 0001:00050850       ?GetVelocity@CScriptBind_Entity@@IAEHPAUIFunctionHandler@@@Z 32051850 f   ScriptBind_Entity.obj
 0001:00050970       ?GetVelocityEx@CScriptBind_Entity@@IAEHPAUIFunctionHandler@@@Z 32051970 f   ScriptBind_Entity.obj
 0001:00050ad0       ?GetGravity@CScriptBind_Entity@@IAEHPAUIFunctionHandler@@@Z 32051ad0 f   ScriptBind_Entity.obj
 0001:00050c00       ?CheckCollisions@CScriptBind_Entity@@IAEHPAUIFunctionHandler@@@Z 32051c00 f   ScriptBind_Entity.obj
 0001:00052070       ?ParseFogVolumesParams@CScriptBind_Entity@@AAE_NPAUIScriptTable@@PAUIEntity@@AAUSFogVolumeProperties@@@Z 32053070 f   ScriptBind_Entity.obj
 0001:00052350       ?ParseCloudMovementProperties@CScriptBind_Entity@@AAE_NPAUIScriptTable@@PAUIEntity@@AAUSCloudMovementProperties@@@Z 32053350 f   ScriptBind_Entity.obj
 0001:00052350       ?ParseVolumeObjectMovementProperties@CScriptBind_Entity@@AAE_NPAUIScriptTable@@PAUIEntity@@AAUSVolumeObjectMovementProperties@@@Z 32053350 f   ScriptBind_Entity.obj
 0001:00052460       ?IntersectRay@CScriptBind_Entity@@IAEHPAUIFunctionHandler@@HU?$Vec3_tpl@M@@1M@Z 32053460 f   ScriptBind_Entity.obj
 0001:00053110       ?ProcessBroadcastEvent@CScriptBind_Entity@@IAEHPAUIFunctionHandler@@@Z 32054110 f   ScriptBind_Entity.obj
 0001:000531a0       ?ActivateOutput@CScriptBind_Entity@@IAEHPAUIFunctionHandler@@@Z 320541a0 f   ScriptBind_Entity.obj
 0001:00053410       ?RagDollize@CScriptBind_Entity@@IAEHPAUIFunctionHandler@@H@Z 32054410 f   ScriptBind_Entity.obj
 0001:00053800       ?set_size@?$SmallDynStorage@UGoalParams@@HUStandardAlloc@NAlloc@@@NArray@@QAEXH@Z 32054800 f i ScriptBind_Entity.obj
 0001:00053890       ?resize_raw@?$SmallDynStorage@UGoalParams@@HUStandardAlloc@NAlloc@@@NArray@@QAEXHH_N@Z 32054890 f i ScriptBind_Entity.obj
 0001:000539f0       ??$RegisterTemplateFunction@VCScriptBind_Entity@@P81@AEHPAUIFunctionHandler@@H@Z@CScriptableBase@@IAEXPBD0AAVCScriptBind_Entity@@ABQ81@AEHPAUIFunctionHandler@@H@Z@Z 320549f0 f i ScriptBind_Entity.obj
 0001:00053a60       ??$RegisterTemplateFunction@VCScriptBind_Entity@@P81@AEHPAUIFunctionHandler@@HVSmartScriptTable@@@Z@CScriptableBase@@IAEXPBD0AAVCScriptBind_Entity@@ABQ81@AEHPAUIFunctionHandler@@HVSmartScriptTable@@@Z@Z 32054a60 f i ScriptBind_Entity.obj
 0001:00053ad0       ??$RegisterTemplateFunction@VCScriptBind_Entity@@P81@AEHPAUIFunctionHandler@@HH@Z@CScriptableBase@@IAEXPBD0AAVCScriptBind_Entity@@ABQ81@AEHPAUIFunctionHandler@@HH@Z@Z 32054ad0 f i ScriptBind_Entity.obj
 0001:00053b40       ??$RegisterTemplateFunction@VCScriptBind_Entity@@P81@AEHPAUIFunctionHandler@@@Z@CScriptableBase@@IAEXPBD0AAVCScriptBind_Entity@@ABQ81@AEHPAUIFunctionHandler@@@Z@Z 32054b40 f i ScriptBind_Entity.obj
 0001:00053bb0       ??$RegisterTemplateFunction@VCScriptBind_Entity@@P81@AEHPAUIFunctionHandler@@_N@Z@CScriptableBase@@IAEXPBD0AAVCScriptBind_Entity@@ABQ81@AEHPAUIFunctionHandler@@_N@Z@Z 32054bb0 f i ScriptBind_Entity.obj
 0001:00053c20       ?Dispatch@?$CallDispatcher@VCScriptBind_Entity@@P81@AEHPAUIFunctionHandler@@HPBD@Z@ScriptTemplateCallHelper@@SAHPAUIFunctionHandler@@PAXH@Z 32054c20 f i ScriptBind_Entity.obj
 0001:00053c80       ?Dispatch@?$CallDispatcher@VCScriptBind_Entity@@P81@AEHPAUIFunctionHandler@@HPBDH@Z@ScriptTemplateCallHelper@@SAHPAUIFunctionHandler@@PAXH@Z 32054c80 f i ScriptBind_Entity.obj
 0001:00053ca0       ?Dispatch@?$CallDispatcher@VCScriptBind_Entity@@P81@AEHPAUIFunctionHandler@@HPBD1@Z@ScriptTemplateCallHelper@@SAHPAUIFunctionHandler@@PAXH@Z 32054ca0 f i ScriptBind_Entity.obj
 0001:00053cc0       ?Dispatch@?$CallDispatcher@VCScriptBind_Entity@@P81@AEHPAUIFunctionHandler@@HMM@Z@ScriptTemplateCallHelper@@SAHPAUIFunctionHandler@@PAXH@Z 32054cc0 f i ScriptBind_Entity.obj
 0001:00053ce0       ?Dispatch@?$CallDispatcher@VCScriptBind_Entity@@P81@AEHPAUIFunctionHandler@@HPBDVSmartScriptTable@@@Z@ScriptTemplateCallHelper@@SAHPAUIFunctionHandler@@PAXH@Z 32054ce0 f i ScriptBind_Entity.obj
 0001:00053d00       ?Dispatch@?$CallDispatcher@VCScriptBind_Entity@@P81@AEHPAUIFunctionHandler@@PBD@Z@ScriptTemplateCallHelper@@SAHPAUIFunctionHandler@@PAXH@Z 32054d00 f i ScriptBind_Entity.obj
 0001:00053d40       ?Dispatch@?$CallDispatcher@VCScriptBind_Entity@@P81@AEHPAUIFunctionHandler@@HU?$Ang3_tpl@M@@@Z@ScriptTemplateCallHelper@@SAHPAUIFunctionHandler@@PAXH@Z 32054d40 f i ScriptBind_Entity.obj
 0001:00053d40       ?Dispatch@?$CallDispatcher@VCScriptBind_Entity@@P81@AEHPAUIFunctionHandler@@HU?$Vec3_tpl@M@@@Z@ScriptTemplateCallHelper@@SAHPAUIFunctionHandler@@PAXH@Z 32054d40 f i ScriptBind_Entity.obj
 0001:00053db0       ?Dispatch@?$CallDispatcher@VCScriptBind_Entity@@P81@AEHPAUIFunctionHandler@@HU?$Vec3_tpl@M@@1@Z@ScriptTemplateCallHelper@@SAHPAUIFunctionHandler@@PAXH@Z 32054db0 f i ScriptBind_Entity.obj
 0001:00053dd0       ?Dispatch@?$CallDispatcher@VCScriptBind_Entity@@P81@AEHPAUIFunctionHandler@@HH_N@Z@ScriptTemplateCallHelper@@SAHPAUIFunctionHandler@@PAXH@Z 32054dd0 f i ScriptBind_Entity.obj
 0001:00053df0       ?Dispatch@?$CallDispatcher@VCScriptBind_Entity@@P81@AEHPAUIFunctionHandler@@U?$Vec3_tpl@M@@@Z@ScriptTemplateCallHelper@@SAHPAUIFunctionHandler@@PAXH@Z 32054df0 f i ScriptBind_Entity.obj
 0001:00053df0       ?Dispatch@?$CallDispatcher@VCScriptBind_Entity@@P81@AEHPAUIFunctionHandler@@U?$Ang3_tpl@M@@@Z@ScriptTemplateCallHelper@@SAHPAUIFunctionHandler@@PAXH@Z 32054df0 f i ScriptBind_Entity.obj
 0001:00053e50       ?Dispatch@?$CallDispatcher@VCScriptBind_Entity@@P81@AEHPAUIFunctionHandler@@M@Z@ScriptTemplateCallHelper@@SAHPAUIFunctionHandler@@PAXH@Z 32054e50 f i ScriptBind_Entity.obj
 0001:00053e90       ?Dispatch@?$CallDispatcher@VCScriptBind_Entity@@P81@AEHPAUIFunctionHandler@@PBDU?$Vec3_tpl@M@@@Z@ScriptTemplateCallHelper@@SAHPAUIFunctionHandler@@PAXH@Z 32054e90 f i ScriptBind_Entity.obj
 0001:00053f00       ?Dispatch@?$CallDispatcher@VCScriptBind_Entity@@P81@AEHPAUIFunctionHandler@@TScriptHandle@@@Z@ScriptTemplateCallHelper@@SAHPAUIFunctionHandler@@PAXH@Z 32054f00 f i ScriptBind_Entity.obj
 0001:00053f50       ?Dispatch@?$CallDispatcher@VCScriptBind_Entity@@P81@AEHPAUIFunctionHandler@@HHVSmartScriptTable@@@Z@ScriptTemplateCallHelper@@SAHPAUIFunctionHandler@@PAXH@Z 32054f50 f i ScriptBind_Entity.obj
 0001:00053f70       ?Dispatch@?$CallDispatcher@VCScriptBind_Entity@@P81@AEHPAUIFunctionHandler@@TScriptHandle@@H@Z@ScriptTemplateCallHelper@@SAHPAUIFunctionHandler@@PAXH@Z 32054f70 f i ScriptBind_Entity.obj
 0001:00053fd0       ?Dispatch@?$CallDispatcher@VCScriptBind_Entity@@P81@AEHPAUIFunctionHandler@@HU?$Vec3_tpl@M@@1M@Z@ScriptTemplateCallHelper@@SAHPAUIFunctionHandler@@PAXH@Z 32054fd0 f i ScriptBind_Entity.obj
 0001:00053ff0       ?Dispatch@?$CallDispatcher@VCScriptBind_Entity@@P81@AEHPAUIFunctionHandler@@H_N@Z@ScriptTemplateCallHelper@@SAHPAUIFunctionHandler@@PAXH@Z 32054ff0 f i ScriptBind_Entity.obj
 0001:00054050       ?Dispatch@?$CallDispatcher@VCScriptBind_Entity@@P81@AEHPAUIFunctionHandler@@HHM@Z@ScriptTemplateCallHelper@@SAHPAUIFunctionHandler@@PAXH@Z 32055050 f i ScriptBind_Entity.obj
 0001:00054070       ?Dispatch@?$CallDispatcher@VCScriptBind_Entity@@P81@AEHPAUIFunctionHandler@@HHPBD_N@Z@ScriptTemplateCallHelper@@SAHPAUIFunctionHandler@@PAXH@Z 32055070 f i ScriptBind_Entity.obj
 0001:00054090       ?Dispatch@?$CallDispatcher@VCScriptBind_Entity@@P81@AEHPAUIFunctionHandler@@HPBD_N@Z@ScriptTemplateCallHelper@@SAHPAUIFunctionHandler@@PAXH@Z 32055090 f i ScriptBind_Entity.obj
 0001:000540b0       ?Dispatch@?$CallDispatcher@VCScriptBind_Entity@@P81@AEHPAUIFunctionHandler@@U?$Vec3_tpl@M@@1@Z@ScriptTemplateCallHelper@@SAHPAUIFunctionHandler@@PAXH@Z 320550b0 f i ScriptBind_Entity.obj
 0001:000540d0       ?Dispatch@?$CallDispatcher@VCScriptBind_Entity@@P81@AEHPAUIFunctionHandler@@TScriptHandle@@M@Z@ScriptTemplateCallHelper@@SAHPAUIFunctionHandler@@PAXH@Z 320550d0 f i ScriptBind_Entity.obj
 0001:00054140       ?Dispatch@?$CallDispatcher@VCScriptBind_Entity@@P81@AEHPAUIFunctionHandler@@TScriptHandle@@_N@Z@ScriptTemplateCallHelper@@SAHPAUIFunctionHandler@@PAXH@Z 32055140 f i ScriptBind_Entity.obj
 0001:000541a0       ?Dispatch@?$CallDispatcher@VCScriptBind_Entity@@P81@AEHPAUIFunctionHandler@@HPBD1U?$Vec3_tpl@M@@2MH@Z@ScriptTemplateCallHelper@@SAHPAUIFunctionHandler@@PAXH@Z 320551a0 f i ScriptBind_Entity.obj
 0001:000541c0       ?Dispatch@?$CallDispatcher@VCScriptBind_Entity@@P81@AEHPAUIFunctionHandler@@HPBDTScriptHandle@@HH@Z@ScriptTemplateCallHelper@@SAHPAUIFunctionHandler@@PAXH@Z 320551c0 f i ScriptBind_Entity.obj
 0001:000541e0       ?Dispatch@?$CallDispatcher@VCScriptBind_Entity@@P81@AEHPAUIFunctionHandler@@HPBDVSmartScriptTable@@H@Z@ScriptTemplateCallHelper@@SAHPAUIFunctionHandler@@PAXH@Z 320551e0 f i ScriptBind_Entity.obj
 0001:00054200       ?Dispatch@?$CallDispatcher@VCScriptBind_Entity@@P81@AEHPAUIFunctionHandler@@HPBDU?$Vec3_tpl@M@@@Z@ScriptTemplateCallHelper@@SAHPAUIFunctionHandler@@PAXH@Z 32055200 f i ScriptBind_Entity.obj
 0001:00054220       ?Dispatch@?$CallDispatcher@VCScriptBind_Entity@@P81@AEHPAUIFunctionHandler@@HPBDU?$Vec3_tpl@M@@_N@Z@ScriptTemplateCallHelper@@SAHPAUIFunctionHandler@@PAXH@Z 32055220 f i ScriptBind_Entity.obj
 0001:00054240       ?Dispatch@?$CallDispatcher@VCScriptBind_Entity@@P81@AEHPAUIFunctionHandler@@HPBD_N2@Z@ScriptTemplateCallHelper@@SAHPAUIFunctionHandler@@PAXH@Z 32055240 f i ScriptBind_Entity.obj
 0001:00054260       ?Dispatch@?$CallDispatcher@VCScriptBind_Entity@@P81@AEHPAUIFunctionHandler@@H_N1@Z@ScriptTemplateCallHelper@@SAHPAUIFunctionHandler@@PAXH@Z 32055260 f i ScriptBind_Entity.obj
 0001:00054280       ?Dispatch@?$CallDispatcher@VCScriptBind_Entity@@P81@AEHPAUIFunctionHandler@@HHPBDM@Z@ScriptTemplateCallHelper@@SAHPAUIFunctionHandler@@PAXH@Z 32055280 f i ScriptBind_Entity.obj
 0001:000542a0       ?Dispatch@?$CallDispatcher@VCScriptBind_Entity@@P81@AEHPAUIFunctionHandler@@HHPBD@Z@ScriptTemplateCallHelper@@SAHPAUIFunctionHandler@@PAXH@Z 320552a0 f i ScriptBind_Entity.obj
 0001:000542c0       ?Dispatch@?$CallDispatcher@VCScriptBind_Entity@@P81@AEHPAUIFunctionHandler@@HHPBDU?$Vec3_tpl@M@@@Z@ScriptTemplateCallHelper@@SAHPAUIFunctionHandler@@PAXH@Z 320552c0 f i ScriptBind_Entity.obj
 0001:000542e0       ?Dispatch@?$CallDispatcher@VCScriptBind_Entity@@P81@AEHPAUIFunctionHandler@@_NH@Z@ScriptTemplateCallHelper@@SAHPAUIFunctionHandler@@PAXH@Z 320552e0 f i ScriptBind_Entity.obj
 0001:00054340       ?Dispatch@?$CallDispatcher@VCScriptBind_Entity@@P81@AEHPAUIFunctionHandler@@PBDTScriptHandle@@@Z@ScriptTemplateCallHelper@@SAHPAUIFunctionHandler@@PAXH@Z 32055340 f i ScriptBind_Entity.obj
 0001:000543a0       ?Dispatch@?$CallDispatcher@VCScriptBind_Entity@@P81@AEHPAUIFunctionHandler@@HTScriptHandle@@@Z@ScriptTemplateCallHelper@@SAHPAUIFunctionHandler@@PAXH@Z 320553a0 f i ScriptBind_Entity.obj
 0001:00054400       ?Dispatch@?$CallDispatcher@VCScriptBind_Entity@@P81@AEHPAUIFunctionHandler@@HHMU?$Vec3_tpl@M@@1M_N@Z@ScriptTemplateCallHelper@@SAHPAUIFunctionHandler@@PAXH@Z 32055400 f i ScriptBind_Entity.obj
 0001:00054420       ?Dispatch@?$CallDispatcher@VCScriptBind_Entity@@P81@AEHPAUIFunctionHandler@@HPBD_N11MM@Z@ScriptTemplateCallHelper@@SAHPAUIFunctionHandler@@PAXH@Z 32055420 f i ScriptBind_Entity.obj
 0001:00054440       ?FromValue@?$TProxyTypeInfo@MU?$TFixed@E$00$0PP@@@@@UBE_NPAXPBXABUCTypeInfo@@@Z 32055440 f i ScriptBind_Entity.obj
 0001:000544d0       ?FromString@?$TProxyTypeInfo@MU?$TFixed@E$00$0PP@@@@@UBE_NPAXPBDUFFromString@@@Z 320554d0 f i ScriptBind_Entity.obj
 0001:00054560       ??$Call@VCScriptBind_Entity@@HPBDI@ScriptTemplateCallHelper@@SAHPAVCScriptBind_Entity@@P81@AEHPAUIFunctionHandler@@HPBDI@Z1@Z 32055560 f i ScriptBind_Entity.obj
 0001:000545d0       ??$Call@VCScriptBind_Entity@@PBDU?$Vec3_tpl@M@@U2@III@ScriptTemplateCallHelper@@SAHPAVCScriptBind_Entity@@P81@AEHPAUIFunctionHandler@@PBDU?$Vec3_tpl@M@@3III@Z1@Z 320555d0 f i ScriptBind_Entity.obj
 0001:000546a0       ??$Call@VCScriptBind_Entity@@PBDIIMU?$Vec3_tpl@M@@MMI@ScriptTemplateCallHelper@@SAHPAVCScriptBind_Entity@@P81@AEHPAUIFunctionHandler@@PBDIIMU?$Vec3_tpl@M@@MMI@Z1@Z 320556a0 f i ScriptBind_Entity.obj
 0001:00054730       ?ProcessAttachment@CLightAttachment@@UAEXPAUIAttachment@@@Z 32055730 f i ScriptBind_Entity.obj
 0001:000549b0       ?SetCloudMovementProperties@CScriptBind_Entity@@IAEHPAUIFunctionHandler@@HVSmartScriptTable@@@Z 320559b0 f   ScriptBind_Entity.obj
 0001:00054a50       ?LoadFogVolume@CScriptBind_Entity@@IAEHPAUIFunctionHandler@@HVSmartScriptTable@@@Z 32055a50 f   ScriptBind_Entity.obj
 0001:00054af0       ?SetVolumeObjectMovementProperties@CScriptBind_Entity@@IAEHPAUIFunctionHandler@@HVSmartScriptTable@@@Z 32055af0 f   ScriptBind_Entity.obj
 0001:00054b90       ?SetAttachmentDir@CScriptBind_Entity@@IAEHPAUIFunctionHandler@@HPBDU?$Vec3_tpl@M@@_N@Z 32055b90 f   ScriptBind_Entity.obj
 0001:000551d0       ?SetCharacterPhysicParams@CScriptBind_Entity@@IAEHPAUIFunctionHandler@@@Z 320561d0 f   ScriptBind_Entity.obj
 0001:00055390       ?SetPhysicParams@CScriptBind_Entity@@IAEHPAUIFunctionHandler@@@Z 32056390 f   ScriptBind_Entity.obj
 0001:00055460       ?SetPublicParam@CScriptBind_Entity@@IAEHPAUIFunctionHandler@@@Z 32056460 f   ScriptBind_Entity.obj
 0001:00055710       ?GetMaterial@CScriptBind_Entity@@IAEHPAUIFunctionHandler@@@Z 32056710 f   ScriptBind_Entity.obj
 0001:00055840       ?destroy@?$DynArray@UGoalParams@@HU?$SmallDynStorage@UGoalParams@@HUStandardAlloc@NAlloc@@@NArray@@@@IAEXXZ 32056840 f i ScriptBind_Entity.obj
 0001:00055890       ?expand_raw@?$DynArray@UGoalParams@@HU?$SmallDynStorage@UGoalParams@@HUStandardAlloc@NAlloc@@@NArray@@@@IAEPAUGoalParams@@PAU2@H@Z 32056890 f i ScriptBind_Entity.obj
 0001:00055920       ??$RegisterTemplateFunction@VCScriptBind_Entity@@P81@AEHPAUIFunctionHandler@@HPBD@Z@CScriptableBase@@IAEXPBD0AAVCScriptBind_Entity@@ABQ81@AEHPAUIFunctionHandler@@H0@Z@Z 32056920 f i ScriptBind_Entity.obj
 0001:00055990       ??$RegisterTemplateFunction@VCScriptBind_Entity@@P81@AEHPAUIFunctionHandler@@HPBDH@Z@CScriptableBase@@IAEXPBD0AAVCScriptBind_Entity@@ABQ81@AEHPAUIFunctionHandler@@H0H@Z@Z 32056990 f i ScriptBind_Entity.obj
 0001:00055a00       ??$RegisterTemplateFunction@VCScriptBind_Entity@@P81@AEHPAUIFunctionHandler@@HPBD1@Z@CScriptableBase@@IAEXPBD0AAVCScriptBind_Entity@@ABQ81@AEHPAUIFunctionHandler@@H00@Z@Z 32056a00 f i ScriptBind_Entity.obj
 0001:00055a70       ??$RegisterTemplateFunction@VCScriptBind_Entity@@P81@AEHPAUIFunctionHandler@@PBD@Z@CScriptableBase@@IAEXPBD0AAVCScriptBind_Entity@@ABQ81@AEHPAUIFunctionHandler@@0@Z@Z 32056a70 f i ScriptBind_Entity.obj
 0001:00055ae0       ??$RegisterTemplateFunction@VCScriptBind_Entity@@P81@AEHPAUIFunctionHandler@@HU?$Vec3_tpl@M@@@Z@CScriptableBase@@IAEXPBD0AAVCScriptBind_Entity@@ABQ81@AEHPAUIFunctionHandler@@HU?$Vec3_tpl@M@@@Z@Z 32056ae0 f i ScriptBind_Entity.obj
 0001:00055b50       ??$RegisterTemplateFunction@VCScriptBind_Entity@@P81@AEHPAUIFunctionHandler@@HU?$Vec3_tpl@M@@1@Z@CScriptableBase@@IAEXPBD0AAVCScriptBind_Entity@@ABQ81@AEHPAUIFunctionHandler@@HU?$Vec3_tpl@M@@3@Z@Z 32056b50 f i ScriptBind_Entity.obj
 0001:00055bc0       ??$RegisterTemplateFunction@VCScriptBind_Entity@@P81@AEHPAUIFunctionHandler@@HH_N@Z@CScriptableBase@@IAEXPBD0AAVCScriptBind_Entity@@ABQ81@AEHPAUIFunctionHandler@@HH_N@Z@Z 32056bc0 f i ScriptBind_Entity.obj
 0001:00055c30       ??$RegisterTemplateFunction@VCScriptBind_Entity@@P81@AEHPAUIFunctionHandler@@M@Z@CScriptableBase@@IAEXPBD0AAVCScriptBind_Entity@@ABQ81@AEHPAUIFunctionHandler@@M@Z@Z 32056c30 f i ScriptBind_Entity.obj
 0001:00055ca0       ??$RegisterTemplateFunction@VCScriptBind_Entity@@P81@AEHPAUIFunctionHandler@@PBDU?$Vec3_tpl@M@@@Z@CScriptableBase@@IAEXPBD0AAVCScriptBind_Entity@@ABQ81@AEHPAUIFunctionHandler@@0U?$Vec3_tpl@M@@@Z@Z 32056ca0 f i ScriptBind_Entity.obj
 0001:00055d10       ??$RegisterTemplateFunction@VCScriptBind_Entity@@P81@AEHPAUIFunctionHandler@@TScriptHandle@@@Z@CScriptableBase@@IAEXPBD0AAVCScriptBind_Entity@@ABQ81@AEHPAUIFunctionHandler@@TScriptHandle@@@Z@Z 32056d10 f i ScriptBind_Entity.obj
 0001:00055d80       ??$RegisterTemplateFunction@VCScriptBind_Entity@@P81@AEHPAUIFunctionHandler@@HHVSmartScriptTable@@@Z@CScriptableBase@@IAEXPBD0AAVCScriptBind_Entity@@ABQ81@AEHPAUIFunctionHandler@@HHVSmartScriptTable@@@Z@Z 32056d80 f i ScriptBind_Entity.obj
 0001:00055df0       ??$RegisterTemplateFunction@VCScriptBind_Entity@@P81@AEHPAUIFunctionHandler@@TScriptHandle@@H@Z@CScriptableBase@@IAEXPBD0AAVCScriptBind_Entity@@ABQ81@AEHPAUIFunctionHandler@@TScriptHandle@@H@Z@Z 32056df0 f i ScriptBind_Entity.obj
 0001:00055e60       ??$RegisterTemplateFunction@VCScriptBind_Entity@@P81@AEHPAUIFunctionHandler@@HU?$Vec3_tpl@M@@1M@Z@CScriptableBase@@IAEXPBD0AAVCScriptBind_Entity@@ABQ81@AEHPAUIFunctionHandler@@HU?$Vec3_tpl@M@@3M@Z@Z 32056e60 f i ScriptBind_Entity.obj
 0001:00055ed0       ??$RegisterTemplateFunction@VCScriptBind_Entity@@P81@AEHPAUIFunctionHandler@@H_N@Z@CScriptableBase@@IAEXPBD0AAVCScriptBind_Entity@@ABQ81@AEHPAUIFunctionHandler@@H_N@Z@Z 32056ed0 f i ScriptBind_Entity.obj
 0001:00055f40       ??$RegisterTemplateFunction@VCScriptBind_Entity@@P81@AEHPAUIFunctionHandler@@HHM@Z@CScriptableBase@@IAEXPBD0AAVCScriptBind_Entity@@ABQ81@AEHPAUIFunctionHandler@@HHM@Z@Z 32056f40 f i ScriptBind_Entity.obj
 0001:00055fb0       ??$RegisterTemplateFunction@VCScriptBind_Entity@@P81@AEHPAUIFunctionHandler@@HHPBD_N@Z@CScriptableBase@@IAEXPBD0AAVCScriptBind_Entity@@ABQ81@AEHPAUIFunctionHandler@@HH0_N@Z@Z 32056fb0 f i ScriptBind_Entity.obj
 0001:00056020       ??$RegisterTemplateFunction@VCScriptBind_Entity@@P81@AEHPAUIFunctionHandler@@HPBD_N@Z@CScriptableBase@@IAEXPBD0AAVCScriptBind_Entity@@ABQ81@AEHPAUIFunctionHandler@@H0_N@Z@Z 32057020 f i ScriptBind_Entity.obj
 0001:00056090       ??$RegisterTemplateFunction@VCScriptBind_Entity@@P81@AEHPAUIFunctionHandler@@U?$Vec3_tpl@M@@1@Z@CScriptableBase@@IAEXPBD0AAVCScriptBind_Entity@@ABQ81@AEHPAUIFunctionHandler@@U?$Vec3_tpl@M@@3@Z@Z 32057090 f i ScriptBind_Entity.obj
 0001:00056100       ??$RegisterTemplateFunction@VCScriptBind_Entity@@P81@AEHPAUIFunctionHandler@@TScriptHandle@@M@Z@CScriptableBase@@IAEXPBD0AAVCScriptBind_Entity@@ABQ81@AEHPAUIFunctionHandler@@TScriptHandle@@M@Z@Z 32057100 f i ScriptBind_Entity.obj
 0001:00056170       ??$RegisterTemplateFunction@VCScriptBind_Entity@@P81@AEHPAUIFunctionHandler@@TScriptHandle@@_N@Z@CScriptableBase@@IAEXPBD0AAVCScriptBind_Entity@@ABQ81@AEHPAUIFunctionHandler@@TScriptHandle@@_N@Z@Z 32057170 f i ScriptBind_Entity.obj
 0001:000561e0       ??$RegisterTemplateFunction@VCScriptBind_Entity@@P81@AEHPAUIFunctionHandler@@HPBD1U?$Vec3_tpl@M@@2MH@Z@CScriptableBase@@IAEXPBD0AAVCScriptBind_Entity@@ABQ81@AEHPAUIFunctionHandler@@H00U?$Vec3_tpl@M@@3MH@Z@Z 320571e0 f i ScriptBind_Entity.obj
 0001:00056250       ??$RegisterTemplateFunction@VCScriptBind_Entity@@P81@AEHPAUIFunctionHandler@@HPBDTScriptHandle@@HH@Z@CScriptableBase@@IAEXPBD0AAVCScriptBind_Entity@@ABQ81@AEHPAUIFunctionHandler@@H0TScriptHandle@@HH@Z@Z 32057250 f i ScriptBind_Entity.obj
 0001:000562c0       ??$RegisterTemplateFunction@VCScriptBind_Entity@@P81@AEHPAUIFunctionHandler@@HPBDVSmartScriptTable@@H@Z@CScriptableBase@@IAEXPBD0AAVCScriptBind_Entity@@ABQ81@AEHPAUIFunctionHandler@@H0VSmartScriptTable@@H@Z@Z 320572c0 f i ScriptBind_Entity.obj
 0001:00056330       ??$RegisterTemplateFunction@VCScriptBind_Entity@@P81@AEHPAUIFunctionHandler@@HPBDU?$Vec3_tpl@M@@@Z@CScriptableBase@@IAEXPBD0AAVCScriptBind_Entity@@ABQ81@AEHPAUIFunctionHandler@@H0U?$Vec3_tpl@M@@@Z@Z 32057330 f i ScriptBind_Entity.obj
 0001:000563a0       ??$RegisterTemplateFunction@VCScriptBind_Entity@@P81@AEHPAUIFunctionHandler@@HPBDU?$Vec3_tpl@M@@_N@Z@CScriptableBase@@IAEXPBD0AAVCScriptBind_Entity@@ABQ81@AEHPAUIFunctionHandler@@H0U?$Vec3_tpl@M@@_N@Z@Z 320573a0 f i ScriptBind_Entity.obj
 0001:00056410       ??$RegisterTemplateFunction@VCScriptBind_Entity@@P81@AEHPAUIFunctionHandler@@HPBD_N2@Z@CScriptableBase@@IAEXPBD0AAVCScriptBind_Entity@@ABQ81@AEHPAUIFunctionHandler@@H0_N3@Z@Z 32057410 f i ScriptBind_Entity.obj
 0001:00056480       ??$RegisterTemplateFunction@VCScriptBind_Entity@@P81@AEHPAUIFunctionHandler@@H_N1@Z@CScriptableBase@@IAEXPBD0AAVCScriptBind_Entity@@ABQ81@AEHPAUIFunctionHandler@@H_N3@Z@Z 32057480 f i ScriptBind_Entity.obj
 0001:000564f0       ??$RegisterTemplateFunction@VCScriptBind_Entity@@P81@AEHPAUIFunctionHandler@@HHPBDM@Z@CScriptableBase@@IAEXPBD0AAVCScriptBind_Entity@@ABQ81@AEHPAUIFunctionHandler@@HH0M@Z@Z 320574f0 f i ScriptBind_Entity.obj
 0001:00056560       ??$RegisterTemplateFunction@VCScriptBind_Entity@@P81@AEHPAUIFunctionHandler@@HHPBD@Z@CScriptableBase@@IAEXPBD0AAVCScriptBind_Entity@@ABQ81@AEHPAUIFunctionHandler@@HH0@Z@Z 32057560 f i ScriptBind_Entity.obj
 0001:000565d0       ??$RegisterTemplateFunction@VCScriptBind_Entity@@P81@AEHPAUIFunctionHandler@@HHPBDU?$Vec3_tpl@M@@@Z@CScriptableBase@@IAEXPBD0AAVCScriptBind_Entity@@ABQ81@AEHPAUIFunctionHandler@@HH0U?$Vec3_tpl@M@@@Z@Z 320575d0 f i ScriptBind_Entity.obj
 0001:00056640       ??$RegisterTemplateFunction@VCScriptBind_Entity@@P81@AEHPAUIFunctionHandler@@_NH@Z@CScriptableBase@@IAEXPBD0AAVCScriptBind_Entity@@ABQ81@AEHPAUIFunctionHandler@@_NH@Z@Z 32057640 f i ScriptBind_Entity.obj
 0001:000566b0       ??$RegisterTemplateFunction@VCScriptBind_Entity@@P81@AEHPAUIFunctionHandler@@PBDTScriptHandle@@@Z@CScriptableBase@@IAEXPBD0AAVCScriptBind_Entity@@ABQ81@AEHPAUIFunctionHandler@@0TScriptHandle@@@Z@Z 320576b0 f i ScriptBind_Entity.obj
 0001:00056720       ??$RegisterTemplateFunction@VCScriptBind_Entity@@P81@AEHPAUIFunctionHandler@@HTScriptHandle@@@Z@CScriptableBase@@IAEXPBD0AAVCScriptBind_Entity@@ABQ81@AEHPAUIFunctionHandler@@HTScriptHandle@@@Z@Z 32057720 f i ScriptBind_Entity.obj
 0001:00056790       ??$RegisterTemplateFunction@VCScriptBind_Entity@@P81@AEHPAUIFunctionHandler@@HHMU?$Vec3_tpl@M@@1M_N@Z@CScriptableBase@@IAEXPBD0AAVCScriptBind_Entity@@ABQ81@AEHPAUIFunctionHandler@@HHMU?$Vec3_tpl@M@@3M_N@Z@Z 32057790 f i ScriptBind_Entity.obj
 0001:00056800       ??$RegisterTemplateFunction@VCScriptBind_Entity@@P81@AEHPAUIFunctionHandler@@HPBD_N11MM@Z@CScriptableBase@@IAEXPBD0AAVCScriptBind_Entity@@ABQ81@AEHPAUIFunctionHandler@@H0_N00MM@Z@Z 32057800 f i ScriptBind_Entity.obj
 0001:00056870       ?_M_insert_overflow@?$_Impl_vector@MV?$allocator@M@stlpmtx_std@@@priv@stlpmtx_std@@AAEXPAMABMABU__true_type@3@I_N@Z 32057870 f i ScriptBind_Entity.obj
 0001:000569c0       ?Dispatch@?$CallDispatcher@VCScriptBind_Entity@@P81@AEHPAUIFunctionHandler@@HPBDI@Z@ScriptTemplateCallHelper@@SAHPAUIFunctionHandler@@PAXH@Z 320579c0 f i ScriptBind_Entity.obj
 0001:000569e0       ?Dispatch@?$CallDispatcher@VCScriptBind_Entity@@P81@AEHPAUIFunctionHandler@@PAD_N@Z@ScriptTemplateCallHelper@@SAHPAUIFunctionHandler@@PAXH@Z 320579e0 f i ScriptBind_Entity.obj
 0001:00056a40       ?Dispatch@?$CallDispatcher@VCScriptBind_Entity@@P81@AEHPAUIFunctionHandler@@PBDU?$Vec3_tpl@M@@2III@Z@ScriptTemplateCallHelper@@SAHPAUIFunctionHandler@@PAXH@Z 32057a40 f i ScriptBind_Entity.obj
 0001:00056a60       ?Dispatch@?$CallDispatcher@VCScriptBind_Entity@@P81@AEHPAUIFunctionHandler@@PBDIIMU?$Vec3_tpl@M@@MMI@Z@ScriptTemplateCallHelper@@SAHPAUIFunctionHandler@@PAXH@Z 32057a60 f i ScriptBind_Entity.obj
 0001:00056a80       ??$NumToString@U?$TFixed@E$00$0PP@@@@@YA?AV?$CryStringT@D@@U?$TFixed@E$00$0PP@@@HH_N@Z 32057a80 f i ScriptBind_Entity.obj
 0001:00056b60       ??$__uninitialized_fill_n@PAU?$Vec3_tpl@M@@IU1@@priv@stlpmtx_std@@YAPAU?$Vec3_tpl@M@@PAU2@IABU2@@Z 32057b60 f i ScriptBind_Entity.obj
 0001:00056bc0       ?ToUnixPath@PathUtil@@YA?AV?$CryStringT@D@@ABV2@@Z 32057bc0 f i ScriptBind_Entity.obj
 0001:00056c90       ??1CScriptBind_Entity@@UAE@XZ 32057c90 f   ScriptBind_Entity.obj
 0001:00056d10       ?GetMemoryUsage@CScriptBind_Entity@@UBEXPAVICrySizer@@@Z 32057d10 f i ScriptBind_Entity.obj
 0001:00056d70       ?SetSlotAngles@CScriptBind_Entity@@IAEHPAUIFunctionHandler@@HU?$Ang3_tpl@M@@@Z 32057d70 f   ScriptBind_Entity.obj
 0001:00057010       ??1?$DynArrayRef@UGoalParams@@HU?$SmallDynStorage@UGoalParams@@HUStandardAlloc@NAlloc@@@NArray@@@@QAE@XZ 32058010 f i ScriptBind_Entity.obj
 0001:00057040       ??$RegisterTemplateFunction@VCScriptBind_Entity@@P81@AEHPAUIFunctionHandler@@U?$Vec3_tpl@M@@@Z@CScriptableBase@@IAEXPBD0AAVCScriptBind_Entity@@ABQ81@AEHPAUIFunctionHandler@@U?$Vec3_tpl@M@@@Z@Z 32058040 f i ScriptBind_Entity.obj
 0001:00057040       ??$RegisterTemplateFunction@VCScriptBind_Entity@@P81@AEHPAUIFunctionHandler@@U?$Ang3_tpl@M@@@Z@CScriptableBase@@IAEXPBD0AAVCScriptBind_Entity@@ABQ81@AEHPAUIFunctionHandler@@U?$Ang3_tpl@M@@@Z@Z 32058040 f i ScriptBind_Entity.obj
 0001:000570b0       ??$RegisterTemplateFunction@VCScriptBind_Entity@@P81@AEHPAUIFunctionHandler@@PAD_N@Z@CScriptableBase@@IAEXPBD0AAVCScriptBind_Entity@@ABQ81@AEHPAUIFunctionHandler@@PAD_N@Z@Z 320580b0 f i ScriptBind_Entity.obj
 0001:00057120       ??$RegisterTemplateFunction@VCScriptBind_Entity@@P81@AEHPAUIFunctionHandler@@PBDU?$Vec3_tpl@M@@2III@Z@CScriptableBase@@IAEXPBD0AAVCScriptBind_Entity@@ABQ81@AEHPAUIFunctionHandler@@0U?$Vec3_tpl@M@@3III@Z@Z 32058120 f i ScriptBind_Entity.obj
 0001:00057190       ??$RegisterTemplateFunction@VCScriptBind_Entity@@P81@AEHPAUIFunctionHandler@@PBDIIMU?$Vec3_tpl@M@@MMI@Z@CScriptableBase@@IAEXPBD0AAVCScriptBind_Entity@@ABQ81@AEHPAUIFunctionHandler@@0IIMU?$Vec3_tpl@M@@MMI@Z@Z 32058190 f i ScriptBind_Entity.obj
 0001:00057200       ?reserve@?$_Impl_vector@MV?$allocator@M@stlpmtx_std@@@priv@stlpmtx_std@@QAEXI@Z 32058200 f i ScriptBind_Entity.obj
 0001:00057200       ?reserve@?$_Impl_vector@PAXV?$allocator@PAX@stlpmtx_std@@@priv@stlpmtx_std@@QAEXI@Z 32058200 f i EntityEventDistributer.obj
 0001:00057290       ?ToString@CCustomInfo@?$TFixed@E$00$0PP@@@UBE?AV?$CryStringT@D@@PBXUFToString@@0@Z 32058290 f i ScriptBind_Entity.obj
 0001:00057320       ?_M_fill_insert_aux@?$_Impl_vector@U?$Vec3_tpl@M@@V?$allocator@U?$Vec3_tpl@M@@@stlpmtx_std@@@priv@stlpmtx_std@@AAEXPAU?$Vec3_tpl@M@@IABU4@ABU__false_type@3@@Z 32058320 f i ScriptBind_Entity.obj
 0001:00057440       ?_M_fill_insert_aux@?$_Impl_vector@MV?$allocator@M@stlpmtx_std@@@priv@stlpmtx_std@@AAEXPAMIABMABU__false_type@3@@Z 32058440 f i ScriptBind_Entity.obj
 0001:00057570       ?grow@?$DynArray@U?$SplineKey@M@spline@@HU?$SmallDynStorage@U?$SplineKey@M@spline@@HUStandardAlloc@NAlloc@@@NArray@@@@QAEPAU?$SplineKey@M@spline@@H@Z 32058570 f i ScriptBind_Entity.obj
 0001:000575c0       ?TypeInfo@?$SplineElem@U?$TFixed@E$00$0PP@@@@@QBEABUCTypeInfo@@XZ 320585c0 f i ScriptBind_Entity.obj
 0001:000576f0       ?TypeInfo@?$SplineElem@M@@QBEABUCTypeInfo@@XZ 320586f0 f i ScriptBind_Entity.obj
 0001:000577f0       ?GetPath@PathUtil@@YA?AV?$CryStringT@D@@ABV2@@Z 320587f0 f i ScriptBind_Entity.obj
 0001:000578a0       ?GetPath@PathUtil@@YA?AV?$CryStringT@D@@PBD@Z 320588a0 f i ScriptBind_Entity.obj
 0001:000578f0       ?GetFile@PathUtil@@YA?AV?$CryStringT@D@@ABV2@@Z 320588f0 f i ScriptBind_Entity.obj
 0001:000579a0       ?GetFileName@PathUtil@@YA?AV?$CryStringT@D@@ABV2@@Z 320589a0 f i ScriptBind_Entity.obj
 0001:00057a10       ??_GCScriptBind_Entity@@UAEPAXI@Z 32058a10 f i ScriptBind_Entity.obj
 0001:00057a10       ??_ECScriptBind_Entity@@UAEPAXI@Z 32058a10 f i ScriptBind_Entity.obj
 0001:00057a40       ??0?$vector@MV?$allocator@M@stlpmtx_std@@@stlpmtx_std@@QAE@ABV?$allocator@M@1@@Z 32058a40 f i ScriptBind_Entity.obj
 0001:00057a80       ?push_back@?$vector@MV?$allocator@M@stlpmtx_std@@@stlpmtx_std@@QAEXABM@Z 32058a80 f i ScriptBind_Entity.obj
 0001:00057ad0       ??0?$DynArray@UGoalParams@@HU?$SmallDynStorage@UGoalParams@@HUStandardAlloc@NAlloc@@@NArray@@@@QAE@ABU0@@Z 32058ad0 f i ScriptBind_Entity.obj
 0001:00057b50       ?ParseLightParams@CScriptBind_Entity@@AAE_NPAUIScriptTable@@AAVCDLight@@PA_N@Z 32058b50 f   ScriptBind_Entity.obj
 0001:00058dc0       ?ToString@?$TCurve@U?$TFixed@E$00$0PP@@@@@QBE?AV?$CryStringT@D@@UFToString@@@Z 32059dc0 f i ScriptBind_Entity.obj
 0001:00058ee0       ??$move_init@UGoalParams@@@@YAXAAUGoalParams@@0@Z 32059ee0 f i ScriptBind_Entity.obj
 0001:00058f50       ??0GoalParams@@QAE@XZ      32059f50 f i ScriptBind_Entity.obj
 0001:00058fb0       ?LoadLight@CScriptBind_Entity@@IAEHPAUIFunctionHandler@@HVSmartScriptTable@@@Z 32059fb0 f   ScriptBind_Entity.obj
 0001:000590a0       ?SetAttachmentLight@CScriptBind_Entity@@IAEHPAUIFunctionHandler@@HPBDVSmartScriptTable@@H@Z 3205a0a0 f   ScriptBind_Entity.obj
 0001:000591c0       ?resize@?$_Impl_vector@U?$Vec3_tpl@M@@V?$allocator@U?$Vec3_tpl@M@@@stlpmtx_std@@@priv@stlpmtx_std@@QAEXIABU?$Vec3_tpl@M@@@Z 3205a1c0 f i ScriptBind_Entity.obj
 0001:00059270       ?resize@?$_Impl_vector@MV?$allocator@M@stlpmtx_std@@@priv@stlpmtx_std@@QAEXIABM@Z 3205a270 f i ScriptBind_Entity.obj
 0001:00059310       ?init@?$DynArray@UGoalParams@@HU?$SmallDynStorage@UGoalParams@@HUStandardAlloc@NAlloc@@@NArray@@@@KAPAUGoalParams@@U?$Array@UGoalParams@@HU?$ArrayStorage@UGoalParams@@H@NArray@@@@ABU2@@Z 3205a310 f i ScriptBind_Entity.obj
 0001:00059370       ?IsPointInsideArea@CScriptBind_Entity@@IAEHPAUIFunctionHandler@@HU?$Vec3_tpl@M@@@Z 3205a370 f   ScriptBind_Entity.obj
 0001:000594e0       ?IsEntityInsideArea@CScriptBind_Entity@@IAEHPAUIFunctionHandler@@HTScriptHandle@@@Z 3205a4e0 f   ScriptBind_Entity.obj
 0001:00059c20       ?ParsePhysicsParams@CScriptBind_Entity@@AAE_NPAUIScriptTable@@AAUSEntityPhysicalizeParams@@@Z 3205ac20 f   ScriptBind_Entity.obj
 0001:0005aae0       ?Physicalize@CScriptBind_Entity@@IAEHPAUIFunctionHandler@@HHVSmartScriptTable@@@Z 3205bae0 f   ScriptBind_Entity.obj
 0001:0005ac50       ?PhysicalizeSlot@CScriptBind_Entity@@IAEHPAUIFunctionHandler@@HVSmartScriptTable@@@Z 3205bc50 f   ScriptBind_Entity.obj
 0001:0005add0       ?GoalParamsHelper@CScriptBind_Entity@@QAEXPAUIFunctionHandler@@IAAUGoalParams@@@Z 3205bdd0 f   ScriptBind_Entity.obj
 0001:0005b0f0       ?InsertSubpipe@CScriptBind_Entity@@IAEHPAUIFunctionHandler@@@Z 3205c0f0 f   ScriptBind_Entity.obj
 0001:0005b390       ?PassParamsToPipe@CScriptBind_Entity@@IAEHPAUIFunctionHandler@@@Z 3205c390 f   ScriptBind_Entity.obj
 0001:0005b460       ?SelectPipe@CScriptBind_Entity@@IAEHPAUIFunctionHandler@@@Z 3205c460 f   ScriptBind_Entity.obj
 0001:0005b730       ??0CScriptBind_Entity@@QAE@PAUIScriptSystem@@PAUISystem@@PAUIEntitySystem@@@Z 3205c730 f   ScriptBind_Entity.obj
 0001:0005f0a0       ?FromString@?$TCurve@U?$TFixed@E$00$0PP@@@@@QAE_NPBDUFFromString@@@Z 320600a0 f i ScriptBind_Entity.obj
 0001:0005f3a0       ?SerializeSpline@?$TCurve@U?$TFixed@E$00$0PP@@@@@UAEXAAVXmlNodeRef@@_N@Z 320603a0 f i ScriptBind_Entity.obj
 0001:0005f430       ??$GetValue@VCScriptVector@@@IScriptTable@@QAE_NPBDAAVCScriptVector@@@Z 32060430 f i ScriptProperties.obj
 0001:0005f430       ??$GetValue@VSmartScriptTable@@@IScriptTable@@QAE_NPBDAAVSmartScriptTable@@@Z 32060430 f i EntitySystem.obj
 0001:0005f4f0       ?Assign@CScriptProperties@@QAEXAAVXmlNodeRef@@PAUIScriptTable@@@Z 320604f0 f   ScriptProperties.obj
 0001:0005f6b0       ?SetProperties@CScriptProperties@@QAE_NAAVXmlNodeRef@@PAUIScriptTable@@@Z 320606b0 f   ScriptProperties.obj
 0001:0005f7b0       ?IsStateFunctionImplemented@SScriptState@@QBE_NW4EScriptStateFunctions@@@Z 320607b0 f i ScriptProxy.obj
 0001:0005f7e0       ?CurrentState@CScriptProxy@@AAEPAUSScriptState@@XZ 320607e0 f i ScriptProxy.obj
 0001:0005f800       ?Done@CScriptProxy@@UAEXXZ 32060800 f   ScriptProxy.obj
 0001:0005f810       ?IsInState@CScriptProxy@@UAE_NPBD@Z 32060810 f   ScriptProxy.obj
 0001:0005f840       ?GetState@CScriptProxy@@UAEPBDXZ 32060840 f   ScriptProxy.obj
 0001:0005f860       ?GetStateId@CScriptProxy@@UAEHXZ 32060860 f   ScriptProxy.obj
 0001:0005f870       ?CallEvent@CScriptProxy@@UAEXPBD@Z 32060870 f   ScriptProxy.obj
 0001:0005f890       ?CallEvent@CScriptProxy@@UAEXPBDM@Z 32060890 f   ScriptProxy.obj
 0001:0005f8b0       ?CallEvent@CScriptProxy@@UAEXPBD_N@Z 320608b0 f   ScriptProxy.obj
 0001:0005f8d0       ?CallEvent@CScriptProxy@@UAEXPBD0@Z 320608d0 f   ScriptProxy.obj
 0001:0005f8f0       ?CallEvent@CScriptProxy@@UAEXPBDABU?$Vec3_tpl@M@@@Z 320608f0 f   ScriptProxy.obj
 0001:0005f910       ?CallInitEvent@CScriptProxy@@QAEX_N@Z 32060910 f   ScriptProxy.obj
 0001:0005f930       ?RegisterForAreaEvents@CScriptProxy@@QAEX_N@Z 32060930 f   ScriptProxy.obj
 0001:0005f950       ?GetMemoryUsage@CScriptProxy@@UBEXPAVICrySizer@@@Z 32060950 f   ScriptProxy.obj
 0001:0005f970       ??$SetValue@VSmartScriptTable@@@IScriptTable@@QAEXPBDABVSmartScriptTable@@@Z 32060970 f i ScriptBind_Entity.obj
 0001:0005f970       ??$SetValue@PAUIScriptTable@@@IScriptTable@@QAEXPBDABQAU0@@Z 32060970 f i ScriptProxy.obj
 0001:0005f9f0       ??$EndCall@_N@IScriptSystem@@QAE_NAA_N@Z 320609f0 f i ScriptProxy.obj
 0001:0005fa70       ??$PushFuncParam@PAUIScriptTable@@@IScriptSystem@@QAEXABQAUIScriptTable@@@Z 32060a70 f i Entity.obj
 0001:0005fa70       ??$PushFuncParam@VSmartScriptTable@@@IScriptSystem@@QAEXABVSmartScriptTable@@@Z 32060a70 f i ScriptProxy.obj
 0001:0005fae0       ?SetScriptUpdateRate@CScriptProxy@@UAEXM@Z 32060ae0 f i ScriptProxy.obj
 0001:0005fb00       ?CreateScriptTable@CScriptProxy@@AAEXPAUSEntitySpawnParams@@@Z 32060b00 f   ScriptProxy.obj
 0001:0005fd80       ?NeedSerialize@CScriptProxy@@UAE_NXZ 32060d80 f   ScriptProxy.obj
 0001:0005fde0       ?CallEvent@CScriptProxy@@UAEXPBDI@Z 32060de0 f   ScriptProxy.obj
 0001:0005fe40       ??$PushParams@PAUIScriptTable@@HPAU1@@Script@@CAXPAUIScriptSystem@@ABQAUIScriptTable@@ABH1@Z 32060e40 f i ScriptProxy.obj
 0001:0005fed0       ??$PushParams@PAUIScriptTable@@HPBD@Script@@CAXPAUIScriptSystem@@ABQAUIScriptTable@@ABHABQBD@Z 32060ed0 f i ScriptProxy.obj
 0001:0005ffa0       ??$PushParams@PAUIScriptTable@@HH@Script@@CAXPAUIScriptSystem@@ABQAUIScriptTable@@ABH2@Z 32060fa0 f i ScriptProxy.obj
 0001:00060070       ??$PushParams@PAUIScriptTable@@M@Script@@CAXPAUIScriptSystem@@ABQAUIScriptTable@@ABM@Z 32061070 f i ScriptProxy.obj
 0001:000600f0       ??$PushParams@PAUIScriptTable@@PAU1@HMPAU1@@Script@@CAXPAUIScriptSystem@@ABQAUIScriptTable@@1ABHABM1@Z 320610f0 f i ScriptProxy.obj
 0001:000601e0       ??$PushParams@PAUIScriptTable@@PAU1@HM@Script@@CAXPAUIScriptSystem@@ABQAUIScriptTable@@1ABHABM@Z 320611e0 f i ScriptProxy.obj
 0001:000602c0       ??$PushParams@PAUIScriptTable@@PAU1@HMM@Script@@CAXPAUIScriptSystem@@ABQAUIScriptTable@@1ABHABM3@Z 320612c0 f i ScriptProxy.obj
 0001:000603f0       ??$PushParams@PAUIScriptTable@@U?$Vec3_tpl@M@@HH@Script@@CAXPAUIScriptSystem@@ABQAUIScriptTable@@ABU?$Vec3_tpl@M@@ABH3@Z 320613f0 f i ScriptProxy.obj
 0001:00060530       ??$PushParams@PAUIScriptTable@@PBD@Script@@CAXPAUIScriptSystem@@ABQAUIScriptTable@@ABQBD@Z 32061530 f i ScriptProxy.obj
 0001:000605a0       ?CallStateFunction@CEntityScript@@QAEXPAUSScriptState@@PAUIScriptTable@@W4EScriptStateFunctions@@@Z 320615a0 f i ScriptProxy.obj
 0001:00060630       ??0CScriptProxy@@QAE@PAVCEntity@@PAVCEntityScript@@PAUSEntitySpawnParams@@@Z 32061630 f   ScriptProxy.obj
 0001:000606c0       ??_ECScriptProxy@@UAEPAXI@Z 320616c0 f i ScriptProxy.obj
 0001:000606c0       ??_GCScriptProxy@@UAEPAXI@Z 320616c0 f i ScriptProxy.obj
 0001:00060710       ?Init@CScriptProxy@@UAE_NPAUIEntity@@AAUSEntitySpawnParams@@@Z 32061710 f   ScriptProxy.obj
 0001:000607b0       ?Reload@CScriptProxy@@UAEXPAUIEntity@@AAUSEntitySpawnParams@@@Z 320617b0 f   ScriptProxy.obj
 0001:00060900       ?ChangeScript@CScriptProxy@@UAEXPAUIEntityScript@@PAUSEntitySpawnParams@@@Z 32061900 f   ScriptProxy.obj
 0001:00060990       ?GotoState@CScriptProxy@@QAE_NH@Z 32061990 f   ScriptProxy.obj
 0001:00060ac0       ?OnPreparedFromPool@CScriptProxy@@UAEXXZ 32061ac0 f   ScriptProxy.obj
 0001:00060af0       ?Value@?$CSerializeWrapper@UISerialize@@@@QAEXPBDPAUIScriptTable@@@Z 32061af0 f i ScriptProxy.obj
 0001:00060b70       ?Value@?$CSerializeWrapper@UISerialize@@@@QAEXPBDAAVSmartScriptTable@@@Z 32061b70 f i ScriptProxy.obj
 0001:00060c40       ??$CallMethod@VSmartScriptTable@@@Script@@SA_NPAUIScriptTable@@PBDABVSmartScriptTable@@@Z 32061c40 f i ScriptProxy.obj
 0001:00060cd0       ??$CallStateFunction@PAUIScriptTable@@@CEntityScript@@QAEXPAUSScriptState@@PAUIScriptTable@@W4EScriptStateFunctions@@ABQAU2@@Z 32061cd0 f i ScriptProxy.obj
 0001:00060cd0       ??$CallStateFunction@VSmartScriptTable@@@CEntityScript@@QAEXPAUSScriptState@@PAUIScriptTable@@W4EScriptStateFunctions@@ABVSmartScriptTable@@@Z 32061cd0 f i ScriptProxy.obj
 0001:00060d70       ?GotoStateId@CScriptProxy@@UAE_NH@Z 32061d70 f i ScriptProxy.obj
 0001:00060d80       ?CreateScriptProxy@@YAPAUIEntityProxy@@PAVCEntity@@PAUIEntityScript@@PAUSEntitySpawnParams@@@Z 32061d80 f   ScriptProxy.obj
 0001:00060dc0       ?GotoState@CScriptProxy@@UAE_NPBD@Z 32061dc0 f   ScriptProxy.obj
 0001:00060e10       ?GetSignature@CScriptProxy@@UAE_NV?$CSerializeWrapper@UISerialize@@@@@Z 32061e10 f   ScriptProxy.obj
 0001:00060ea0       ?Serialize@CScriptProxy@@UAEXV?$CSerializeWrapper@UISerialize@@@@@Z 32061ea0 f   ScriptProxy.obj
 0001:00061120       ?SerializeTable@CScriptProxy@@AAEXV?$CSerializeWrapper@UISerialize@@@@PBD@Z 32062120 f   ScriptProxy.obj
 0001:00061220       ??1SEntityEventTarget@@QAE@XZ 32062220 f i ScriptProxy.obj
 0001:00061280       ?OnCollision@CScriptProxy@@UAEXPAVCEntity@@HABU?$Vec3_tpl@M@@111HM@Z 32062280 f   ScriptProxy.obj
 0001:00061990       ?SendScriptEvent@CScriptProxy@@UAEXHPAUIScriptTable@@PA_N@Z 32062990 f   ScriptProxy.obj
 0001:00061a90       ?SendScriptEvent@CScriptProxy@@UAEXHPBDPA_N@Z 32062a90 f   ScriptProxy.obj
 0001:00061b70       ?SendScriptEvent@CScriptProxy@@UAEXHHPA_N@Z 32062b70 f   ScriptProxy.obj
 0001:00061c50       ??$CallStateFunction@M@CEntityScript@@QAEXPAUSScriptState@@PAUIScriptTable@@W4EScriptStateFunctions@@ABM@Z 32062c50 f i ScriptProxy.obj
 0001:00061ce0       ??$CallStateFunction@HH@CEntityScript@@QAEXPAUSScriptState@@PAUIScriptTable@@W4EScriptStateFunctions@@ABH3@Z 32062ce0 f i ScriptProxy.obj
 0001:00061d80       ??$CallStateFunction@PAUIScriptTable@@HMPAU1@@CEntityScript@@QAEXPAUSScriptState@@PAUIScriptTable@@W4EScriptStateFunctions@@ABQAU2@ABHABM3@Z 32062d80 f i ScriptProxy.obj
 0001:00061e20       ??$CallStateFunction@PAUIScriptTable@@HM@CEntityScript@@QAEXPAUSScriptState@@PAUIScriptTable@@W4EScriptStateFunctions@@ABQAU2@ABHABM@Z 32062e20 f i ScriptProxy.obj
 0001:00061ec0       ??$CallStateFunction@PAUIScriptTable@@HMM@CEntityScript@@QAEXPAUSScriptState@@PAUIScriptTable@@W4EScriptStateFunctions@@ABQAU2@ABHABM5@Z 32062ec0 f i ScriptProxy.obj
 0001:00061f60       ??$CallStateFunction@U?$Vec3_tpl@M@@HH@CEntityScript@@QAEXPAUSScriptState@@PAUIScriptTable@@W4EScriptStateFunctions@@ABU?$Vec3_tpl@M@@ABH4@Z 32062f60 f i ScriptProxy.obj
 0001:00062000       ??$CallStateFunction@PBD@CEntityScript@@QAEXPAUSScriptState@@PAUIScriptTable@@W4EScriptStateFunctions@@ABQBD@Z 32063000 f i ScriptProxy.obj
 0001:00062090       ?Update@CScriptProxy@@UAEXAAUSEntityUpdateContext@@@Z 32063090 f   ScriptProxy.obj
 0001:00062190       ?ProcessEvent@CScriptProxy@@UAEXAAUSEntityEvent@@@Z 32063190 f   ScriptProxy.obj
 0001:000628e0       ?SerializeProperties@CScriptProxy@@QAEXV?$CSerializeWrapper@UISerialize@@@@@Z 320638e0 f   ScriptProxy.obj
 0001:00062920       ?OnStartAnimation@CScriptProxy@@UAEXPBD@Z 32063920 f   ScriptProxy.obj
 0001:00062950       ?OnEndAnimation@CScriptProxy@@UAEXPBD@Z 32063950 f   ScriptProxy.obj
 0001:00062980       ??$__ufill@PAUSEntityEventTarget@@U1@H@priv@stlpmtx_std@@YAXPAUSEntityEventTarget@@0ABU2@ABUrandom_access_iterator_tag@1@PAH@Z 32063980 f i ScriptProxy.obj
 0001:00062a00       ??$__destroy_range_aux@V?$reverse_iterator@PAUSEntityEventTarget@@@stlpmtx_std@@USEntityEventTarget@@@stlpmtx_std@@YAXV?$reverse_iterator@PAUSEntityEventTarget@@@0@0PAUSEntityEventTarget@@ABU__false_type@0@@Z 32063a00 f i ScriptProxy.obj
 0001:00062a80       ??$__ucopy@PAUSEntityEventTarget@@PAU1@H@priv@stlpmtx_std@@YAPAUSEntityEventTarget@@PAU2@00ABUrandom_access_iterator_tag@1@PAH@Z 32063a80 f i ScriptProxy.obj
 0001:00062b00       ?_M_insert_overflow_aux@?$_Impl_vector@USEntityEventTarget@@V?$allocator@USEntityEventTarget@@@stlpmtx_std@@@priv@stlpmtx_std@@AAEXPAUSEntityEventTarget@@ABU4@ABU__false_type@3@I_N@Z 32063b00 f i ScriptProxy.obj
 0001:00062cd0       ?push_back@?$_Impl_vector@USEntityEventTarget@@V?$allocator@USEntityEventTarget@@@stlpmtx_std@@@priv@stlpmtx_std@@QAEXABUSEntityEventTarget@@@Z 32063cd0 f i ScriptProxy.obj
 0001:00062d60       ?SetEventTargets@CScriptProxy@@AAEXAAVXmlNodeRef@@@Z 32063d60 f   ScriptProxy.obj
 0001:000633e0       ?SerializeXML@CScriptProxy@@UAEXAAVXmlNodeRef@@_N@Z 320643e0 f   ScriptProxy.obj
 0001:00063440       ?OnBBoxOverlap@CPhysicsEventListener@@SAHPBUEventPhys@@@Z 32064440 f   PhysicsEventListener.obj
 0001:000634d0       ??_EIThreadTask@@UAEPAXI@Z 320644d0 f i PhysicsEventListener.obj
 0001:000634d0       ??_GIThreadTask@@UAEPAXI@Z 320644d0 f i PhysicsEventListener.obj
 0001:00063500       ?MatchPartId@@YAPAVCEntity@@PAV1@H@Z 32064500 f   PhysicsEventListener.obj
 0001:000635a0       ?UnmapAttachedChild@CEntity@@UAEPAUIEntity@@AAH@Z 320645a0 f   PhysicsEventListener.obj
 0001:00063630       ??_ECMultiThreadRefCount@@UAEPAXI@Z 32064630 f i PhysicsEventListener.obj
 0001:00063630       ??_ESThreadTaskInfo@@UAEPAXI@Z 32064630 f i PhysicsEventListener.obj
 0001:00063630       ??_GCMultiThreadRefCount@@UAEPAXI@Z 32064630 f i PhysicsEventListener.obj
 0001:00063630       ??_GSThreadTaskInfo@@UAEPAXI@Z 32064630 f i PhysicsEventListener.obj
 0001:00063660       ??0SCreateParams@IBreakableManager@@QAE@XZ 32064660 f i PhysicsEventListener.obj
 0001:00063710       ?Result@CDeferredMeshUpdatePrep@@UAEHPAUEventPhys@@@Z 32064710 f i PhysicsEventListener.obj
 0001:00063710       ?EnumElem@CTypeInfo@@UBEPBDI@Z 32064710 f i CryEntityDLL.obj
 0001:00063710       ?get_deleter@?$sp_counted_impl_p@VCEngineModule_EntitySystem@@@detail@boost@@UAEPAXABVsp_typeinfo@23@@Z 32064710 f i CryEntityDLL.obj
 0001:00063710       ?GetLightmap@IRenderNode@@UAEHH@Z 32064710 f i RenderProxy.obj
 0001:00063710       ?GetLightmapTexCoord@IRenderNode@@UAEHH@Z 32064710 f i RenderProxy.obj
 0001:00063710       ?SetAnimationKeyEvent@CScriptBind_Entity@@IAEHPAUIFunctionHandler@@@Z 32064710 f i ScriptBind_Entity.obj
 0001:00063710       ?GetRenderMesh@IRenderNode@@UAEPAUIRenderMesh@@H@Z 32064710 f i RenderProxy.obj
 0001:00063710       ?FindSubVar@CTypeInfo@@UBEPBUCVarInfo@1@PBD@Z 32064710 f i CryEntityDLL.obj
 0001:00063710       ?NextSubVar@CTypeInfo@@UBEPBUCVarInfo@1@PBU21@@Z 32064710 f i CryEntityDLL.obj
 0001:00063710       ?QueryComposite@CEngineModule_EntitySystem@@MBEPAXPBD@Z 32064710 f i CryEntityDLL.obj
 0001:00063720       ?HasFinished@CDeferredMeshUpdatePrep@@UAE_NXZ 32064720 f i PhysicsEventListener.obj
 0001:00063730       ?GetTaskInfo@CDeferredMeshUpdatePrep@@UAEPAUSThreadTaskInfo@@XZ 32064730 f i PhysicsEventListener.obj
 0001:00063740       ?OnUpdate@CDeferredMeshUpdatePrep@@UAEXXZ 32064740 f i PhysicsEventListener.obj
 0001:000637d0       ?OnUpdateMesh@CPhysicsEventListener@@SAHPBUEventPhys@@@Z 320647d0 f   PhysicsEventListener.obj
 0001:00063800       ?OnCreatePhysEntityPart@CPhysicsEventListener@@SAHPBUEventPhys@@@Z 32064800 f   PhysicsEventListener.obj
 0001:00063830       ?OnRemovePhysEntityParts@CPhysicsEventListener@@SAHPBUEventPhys@@@Z 32064830 f   PhysicsEventListener.obj
 0001:00063860       ?OnRevealPhysEntityPart@CPhysicsEventListener@@SAHPBUEventPhys@@@Z 32064860 f   PhysicsEventListener.obj
 0001:00063890       ?OnCollision@CPhysicsEventListener@@SAHPBUEventPhys@@@Z 32064890 f   PhysicsEventListener.obj
 0001:00063ab0       ?OnPostStep@CPhysicsEventListener@@SAHPBUEventPhys@@@Z 32064ab0 f   PhysicsEventListener.obj
 0001:00063df0       ?OnStateChange@CPhysicsEventListener@@SAHPBUEventPhys@@@Z 32064df0 f   PhysicsEventListener.obj
 0001:00064000       ??_GCDeferredMeshUpdatePrep@@UAEPAXI@Z 32065000 f i PhysicsEventListener.obj
 0001:00064000       ??_ECDeferredMeshUpdatePrep@@UAEPAXI@Z 32065000 f i PhysicsEventListener.obj
 0001:00064030       ?SetTailName@CSoundProxy@@QAEXQBD@Z 32065030 f i PhysicsEventListener.obj
 0001:00064070       ?OnJointBreak@CPhysicsEventListener@@SAHPBUEventPhys@@@Z 32065070 f   PhysicsEventListener.obj
 0001:00065200       ?OnTailObstructionTest@CPhysicsEventListener@@SAHPBUEventPhys@@@Z 32066200 f   PhysicsEventListener.obj
 0001:00065270       ?RegisterPhysicCallbacks@CPhysicsEventListener@@QAEXXZ 32066270 f   PhysicsEventListener.obj
 0001:000653e0       ?UnregisterPhysicCallbacks@CPhysicsEventListener@@QAEXXZ 320663e0 f   PhysicsEventListener.obj
 0001:00065500       ??0CPhysicsEventListener@@QAE@PAVCEntitySystem@@PAUIPhysicalWorld@@@Z 32066500 f   PhysicsEventListener.obj
 0001:00065520       ??1CPhysicsEventListener@@QAE@XZ 32066520 f   PhysicsEventListener.obj
 0001:00065540       ?ReleasePhysicalEntity@CPhysicalProxy@@IAEXXZ 32066540 f   PhysicsProxy.obj
 0001:00065580       ?Done@CPhysicalProxy@@UAEXXZ 32066580 f   PhysicsProxy.obj
 0001:00065590       ?OffsetPartId0@@YAXPAVCEntity@@H@Z 32066590 f   PhysicsProxy.obj
 0001:00065630       ?HasPartId@@YA_NPAVCEntity@@H@Z 32066630 f   PhysicsProxy.obj
 0001:00065700       ?ReclaimPhysParts@@YAXPAVCEntity@@PAUIPhysicalEntity@@AAUpe_action_move_parts@@@Z 32066700 f   PhysicsProxy.obj
 0001:000657a0       ?NeedSerialize@CPhysicalProxy@@UAE_NXZ 320667a0 f   PhysicsProxy.obj
 0001:000657b0       ?IsPhysicsEnabled@CPhysicalProxy@@UBE_NXZ 320667b0 f   PhysicsProxy.obj
 0001:000657c0       ?RemoveSlotGeometry@CPhysicalProxy@@QAEXH@Z 320667c0 f   PhysicsProxy.obj
 0001:00065880       ?GetSlotGeometry@CPhysicalProxy@@IAEPAUphys_geometry@@H@Z 32066880 f   PhysicsProxy.obj
 0001:000658c0       ?PhysicalizeFoliage@CPhysicalProxy@@UAE_NH@Z 320668c0 f   PhysicsProxy.obj
 0001:00065990       ?DephysicalizeFoliage@CPhysicalProxy@@UAEXH@Z 32066990 f   PhysicsProxy.obj
 0001:000659c0       ?GetFoliage@CPhysicalProxy@@UAEPAUIFoliage@@H@Z 320669c0 f   PhysicsProxy.obj
 0001:000659e0       ?OnContactWithEntity@CPhysicalProxy@@QAEXPAVCEntity@@@Z 320669e0 f   PhysicsProxy.obj
 0001:00065a00       ?GetMemoryUsage@CPhysicalProxy@@UBEXPAVICrySizer@@@Z 32066a00 f   PhysicsProxy.obj
 0001:00065a20       ?EnableNetworkSerialization@CPhysicalProxy@@UAEX_N@Z 32066a20 f   PhysicsProxy.obj
 0001:00065a70       ?GetMaxPartId0@@YAHPAVCEntity@@@Z 32066a70 f   PhysicsProxy.obj
 0001:00065b10       ?GetSignature@CPhysicalProxy@@UAE_NV?$CSerializeWrapper@UISerialize@@@@@Z 32066b10 f   PhysicsProxy.obj
 0001:00065b40       ?Serialize@CPhysicalProxy@@UAEXV?$CSerializeWrapper@UISerialize@@@@@Z 32066b40 f   PhysicsProxy.obj
 0001:00065d30       ?SerializeTyped@CPhysicalProxy@@UAEXV?$CSerializeWrapper@UISerialize@@@@HH@Z 32066d30 f   PhysicsProxy.obj
 0001:00065e60       ?SerializeXML@CPhysicalProxy@@UAEXAAVXmlNodeRef@@_N@Z 32066e60 f   PhysicsProxy.obj
 0001:00065eb0       ??$move_init@PAUIPhysicalEntity@@@NArray@@YAXPAPAUIPhysicalEntity@@0I@Z 32066eb0 f i PhysicsProxy.obj
 0001:00066010       ?EnableValidation@CPhysicalProxy@@SAXXZ 32067010 f   PhysicsProxy.obj
 0001:00066040       ?DisableValidation@CPhysicalProxy@@SAXXZ 32067040 f   PhysicsProxy.obj
 0001:00066060       ??0CPhysicalProxy@@QAE@PAVCEntity@@@Z 32067060 f   PhysicsProxy.obj
 0001:00066090       ?GetScriptTable@CScriptProxy@@UAEPAUIScriptTable@@XZ 32067090 f i ScriptProxy.obj
 0001:00066090       ?GetPhysicalEntity@CPhysicalProxy@@UBEPAUIPhysicalEntity@@XZ 32067090 f i PhysicsProxy.obj
 0001:00066090       ?GetName@CEntityArchetype@@UBEPBDXZ 32067090 f i EntityArchetype.obj
 0001:00066090       ?GetScriptFile@CEntityClass@@UBEPBDXZ 32067090 f i EntityClass.obj
 0001:00066090       ?GetId@CEntity@@UBEIXZ     32067090 f i Entity.obj
 0001:000660a0       ?OnEntityXForm@CPhysicalProxy@@IAEXAAUSEntityEvent@@@Z 320670a0 f   PhysicsProxy.obj
 0001:00066210       ?GetLocalBounds@CPhysicalProxy@@UAEXAAUAABB@@@Z 32067210 f   PhysicsProxy.obj
 0001:00066330       ?GetWorldBounds@CPhysicalProxy@@UAEXAAUAABB@@@Z 32067330 f   PhysicsProxy.obj
 0001:000663b0       ?EnablePhysics@CPhysicalProxy@@UAEX_N@Z 320673b0 f   PhysicsProxy.obj
 0001:000665a0       ?CreatePhysicalEntity@CPhysicalProxy@@IAEXAAUSEntityPhysicalizeParams@@@Z 320675a0 f   PhysicsProxy.obj
 0001:00066700       ?MovePhysics@CPhysicalProxy@@QAEXPAV1@@Z 32067700 f   PhysicsProxy.obj
 0001:00066790       ?DestroyPhysicalEntity@CPhysicalProxy@@IAEX_NH@Z 32067790 f   PhysicsProxy.obj
 0001:000669f0       ?AttachSoftVtx@CPhysicalProxy@@IAEXPAUIRenderMesh@@PAUIPhysicalEntity@@H@Z 320679f0 f   PhysicsProxy.obj
 0001:00066b40       ?PhysicalizeSoft@CPhysicalProxy@@IAEXAAUSEntityPhysicalizeParams@@@Z 32067b40 f   PhysicsProxy.obj
 0001:00066e30       ?PhysicalizeArea@CPhysicalProxy@@IAEXAAUSEntityPhysicalizeParams@@@Z 32067e30 f   PhysicsProxy.obj
 0001:00067860       ?PhysicalizeCharacter@CPhysicalProxy@@IAE_NAAUSEntityPhysicalizeParams@@@Z 32068860 f   PhysicsProxy.obj
 0001:00067f10       ?ConvertCharacterToRagdoll@CPhysicalProxy@@IAE_NAAUSEntityPhysicalizeParams@@ABU?$Vec3_tpl@M@@@Z 32068f10 f   PhysicsProxy.obj
 0001:00068280       ?AddImpulse@CPhysicalProxy@@UAEXHABU?$Vec3_tpl@M@@0_NMM@Z 32069280 f   PhysicsProxy.obj
 0001:00068710       ?GetTriggerBounds@CPhysicalProxy@@UAEXAAUAABB@@@Z 32069710 f   PhysicsProxy.obj
 0001:00068880       ?OnPhysicsPostStep@CPhysicalProxy@@QAEXPAUEventPhysPostStep@@@Z 32069880 f   PhysicsProxy.obj
 0001:00068d90       ?AttachToPhysicalEntity@CPhysicalProxy@@QAEXPAUIPhysicalEntity@@@Z 32069d90 f   PhysicsProxy.obj
 0001:00068e50       ?resize_raw@?$SmallDynStorage@PAUIPhysicalEntity@@HUStandardAlloc@NAlloc@@@NArray@@QAEXHH_N@Z 32069e50 f i PhysicsProxy.obj
 0001:00068fa0       ?AssignPhysicalEntity@CPhysicalProxy@@UAEXPAUIPhysicalEntity@@H@Z 32069fa0 f   PhysicsProxy.obj
 0001:00069310       ?AddSlotGeometry@CPhysicalProxy@@QAEHHAAUSEntityPhysicalizeParams@@H@Z 3206a310 f   PhysicsProxy.obj
 0001:00069a90       ?UpdateSlotGeometry@CPhysicalProxy@@QAEXHPAUIStatObj@@MH@Z 3206aa90 f   PhysicsProxy.obj
 0001:0006a500       ?ReattachSoftEntityVtx@CPhysicalProxy@@UAEXPAUIPhysicalEntity@@H@Z 3206b500 f   PhysicsProxy.obj
 0001:0006a590       ?expand_raw@?$DynArray@PAUIPhysicalEntity@@HU?$SmallDynStorage@PAUIPhysicalEntity@@HUStandardAlloc@NAlloc@@@NArray@@@@IAEPAPAUIPhysicalEntity@@PAPAU2@H@Z 3206b590 f i PhysicsProxy.obj
 0001:0006a610       ?ProcessEvent@CPhysicalProxy@@UAEXAAUSEntityEvent@@@Z 3206b610 f   PhysicsProxy.obj
 0001:0006d290       ?PhysicalizeSimple@CPhysicalProxy@@IAEXAAUSEntityPhysicalizeParams@@@Z 3206e290 f   PhysicsProxy.obj
 0001:0006e250       ?OnCollision@CPhysicalProxy@@QAEXPAVCEntity@@HABU?$Vec3_tpl@M@@111HM@Z 3206f250 f   PhysicsProxy.obj
 0001:0006e390       ?_M_copy@?$_Rb_tree@IU?$less@I@stlpmtx_std@@IU?$_Identity@I@priv@2@U?$_SetTraitsT@I@42@V?$allocator@I@2@@priv@stlpmtx_std@@AAEPAU_Rb_tree_node_base@23@PAU423@0@Z 3206f390 f i PhysicsProxy.obj
 0001:0006e4c0       ?Physicalize@CPhysicalProxy@@UAEXAAUSEntityPhysicalizeParams@@@Z 3206f4c0 f   PhysicsProxy.obj
 0001:0006eb50       ?RemoveCollider@CPhysicalProxy@@IAEXI@Z 3206fb50 f   PhysicsProxy.obj
 0001:0006ec10       ??4?$_Rb_tree@IU?$less@I@stlpmtx_std@@IU?$_Identity@I@priv@2@U?$_SetTraitsT@I@42@V?$allocator@I@2@@priv@stlpmtx_std@@QAEAAV012@ABV012@@Z 3206fc10 f i PhysicsProxy.obj
 0001:0006ec90       ??0Colliders@CPhysicalProxy@@QAE@XZ 3206fc90 f i PhysicsProxy.obj
 0001:0006ecd0       ??0?$DynArray@PAUIPhysicalEntity@@HU?$SmallDynStorage@PAUIPhysicalEntity@@HUStandardAlloc@NAlloc@@@NArray@@@@QAE@XZ 3206fcd0 f i PhysicsProxy.obj
 0001:0006ed20       ?resize@?$DynArray@PAUIPhysicalEntity@@HU?$SmallDynStorage@PAUIPhysicalEntity@@HUStandardAlloc@NAlloc@@@NArray@@@@QAEXH@Z 3206fd20 f i PhysicsProxy.obj
 0001:0006ed60       ?SetTriggerBounds@CPhysicalProxy@@UAEXABUAABB@@@Z 3206fd60 f   PhysicsProxy.obj
 0001:0006f0d0       ?AddCollider@CPhysicalProxy@@IAEXI@Z 320700d0 f   PhysicsProxy.obj
 0001:0006f140       ?CheckColliders@CPhysicalProxy@@IAEXXZ 32070140 f   PhysicsProxy.obj
 0001:0006f450       ?Release@CPhysicalProxy@@UAEXXZ 32070450 f   PhysicsProxy.obj
 0001:0006f4e0       ?Update@CPhysicalProxy@@UAEXAAUSEntityUpdateContext@@@Z 320704e0 f   PhysicsProxy.obj
 0001:0006f4f0       ?Reload@CPhysicalProxy@@UAEXPAUIEntity@@AAUSEntitySpawnParams@@@Z 320704f0 f   PhysicsProxy.obj
 0001:0006f580       ?Release@CRopeProxy@@UAEXXZ 32070580 f   RopeProxy.obj
 0001:0006f5c0       ?Reload@CRopeProxy@@UAEXPAUIEntity@@AAUSEntitySpawnParams@@@Z 320705c0 f   RopeProxy.obj
 0001:0006f640       ?ProcessEvent@CRopeProxy@@UAEXAAUSEntityEvent@@@Z 32070640 f   RopeProxy.obj
 0001:0006f730       ?GetSignature@CRopeProxy@@UAE_NV?$CSerializeWrapper@UISerialize@@@@@Z 32070730 f   RopeProxy.obj
 0001:0006f760       ?Serialize@CRopeProxy@@UAEXV?$CSerializeWrapper@UISerialize@@@@@Z 32070760 f   RopeProxy.obj
 0001:0006f7e0       ?RopeParamsToXml@@YAXAAUSRopeParams@IRopeRenderNode@@AAVXmlNodeRef@@_N@Z 320707e0 f i RopeProxy.obj
 0001:0006fb30       ??$move_init@U?$Vec3_tpl@M@@@NArray@@YAXPAU?$Vec3_tpl@M@@0I@Z 32070b30 f i RopeProxy.obj
 0001:0006fb80       ??0CRopeProxy@@QAE@PAVCEntity@@@Z 32070b80 f   RopeProxy.obj
 0001:0006fbd0       ?GetType@CRopeProxy@@UAE?AW4EEntityProxy@@XZ 32070bd0 f i RopeProxy.obj
 0001:0006fbe0       ?GetName@CEntityClass@@UBEPBDXZ 32070be0 f i EntityClass.obj
 0001:0006fbe0       ?GetReplacementMaterial@CCGFAttachment@@UBEPAUIMaterial@@XZ 32070be0 f i ScriptBind_Entity.obj
 0001:0006fbe0       ?GetFlowGraph@CFlowGraphProxy@@UAEPAUIFlowGraph@@XZ 32070be0 f i FlowGraphProxy.obj
 0001:0006fbe0       ?GetFlags@CAreaProxy@@UAEHXZ 32070be0 f i AreaProxy.obj
 0001:0006fbe0       ?GetRopeRenderNode@CRopeProxy@@UAEPAUIRopeRenderNode@@XZ 32070be0 f i RopeProxy.obj
 0001:0006fbe0       ?GetEntity@CSoundProxy@@UBEPAUIEntity@@XZ 32070be0 f i SoundProxy.obj
 0001:0006fbe0       ?GetReplacementMaterial@CSKELAttachment@@UBEPAUIMaterial@@XZ 32070be0 f i ScriptBind_Entity.obj
 0001:0006fbf0       ?GetMemoryUsage@CRopeProxy@@UBEXPAVICrySizer@@@Z 32070bf0 f i RopeProxy.obj
 0001:0006fc10       ?resize_raw@?$SmallDynStorage@U?$Vec3_tpl@M@@HUStandardAlloc@NAlloc@@@NArray@@QAEXHH_N@Z 32070c10 f i RopeProxy.obj
 0001:0006fd70       ?set_size@?$SmallDynStorage@U?$Vec3_tpl@M@@HUStandardAlloc@NAlloc@@@NArray@@QAEXH@Z 32070d70 f i RopeProxy.obj
 0001:0006fe00       ?expand_raw@?$DynArray@U?$Vec3_tpl@M@@HU?$SmallDynStorage@U?$Vec3_tpl@M@@HUStandardAlloc@NAlloc@@@NArray@@@@IAEPAU?$Vec3_tpl@M@@PAU2@H@Z 32070e00 f i RopeProxy.obj
 0001:0006fe90       ??0?$DynArray@U?$Vec3_tpl@M@@HU?$SmallDynStorage@U?$Vec3_tpl@M@@HUStandardAlloc@NAlloc@@@NArray@@@@QAE@XZ 32070e90 f i RopeProxy.obj
 0001:0006fee0       ?SerializeXML@CRopeProxy@@UAEXAAVXmlNodeRef@@_N@Z 32070ee0 f   RopeProxy.obj
 0001:00070160       ?GetParticleEmitter@CEntityObject@@QBEPAUIParticleEmitter@@XZ 32071160 f   EntityObject.obj
 0001:00070190       ?GetLocalTM@CEntityObject@@QBEABU?$Matrix34_tpl@M@@XZ 32071190 f   EntityObject.obj
 0001:000701a0       ?GetWorldTM@CEntityObject@@QAEABU?$Matrix34_tpl@M@@PAVCEntity@@@Z 320711a0 f   EntityObject.obj
 0001:000701c0       ?OnEntityEvent@CEntityObject@@QAEXPAVCEntity@@ABUSEntityEvent@@@Z 320711c0 f   EntityObject.obj
 0001:000701e0       ?IsEquivalent@?$Matrix34_tpl@M@@SA_NABU1@0M@Z 320711e0 f i EntityObject.obj
 0001:000702d0       ?SetParent@CEntityObject@@QAEXPAV1@@Z 320712d0 f   EntityObject.obj
 0001:00070360       ?SetLocalTM@CEntityObject@@QAEXABU?$Matrix34_tpl@M@@@Z 32071360 f   EntityObject.obj
 0001:00070430       ?IsValid@?$Matrix34_tpl@M@@QBE_NXZ 32071430 f i EntityObject.obj
 0001:00070500       ?ReleaseObjects@CEntityObject@@QAEXXZ 32071500 f   EntityObject.obj
 0001:00070600       ?UpdateWorldTM@CEntityObject@@QAEXPAVCEntity@@@Z 32071600 f   EntityObject.obj
 0001:00070bc0       ??1CEntityObject@@QAE@XZ   32071bc0 f   EntityObject.obj
 0001:00070bf0       ?GetLocalBounds@CEntityObject@@QAE_NAAUAABB@@@Z 32071bf0 f   EntityObject.obj
 0001:00070dd0       ?Render@CEntityObject@@QAE_NPAVCEntity@@AAUSRendParams@@HPAVCRenderProxy@@ABUSRenderingPassInfo@@@Z 32071dd0 f   EntityObject.obj
 0001:000724d0       ?OnXForm@CEntityObject@@QAEXPAVCEntity@@@Z 320734d0 f   EntityObject.obj
 0001:000725e0       ?Update@CEntityObject@@QAEXPAVCEntity@@_NAA_N@Z 320735e0 f   EntityObject.obj
 0001:00072b00       ?Release@CRenderProxy@@UAEXXZ 32073b00 f   RenderProxy.obj
 0001:00072b10       ?UpdateEntityFlags@CRenderProxy@@QAEXXZ 32073b10 f   RenderProxy.obj
 0001:00072c30       ?NeedSerialize@CRenderProxy@@UAE_NXZ 32073c30 f   RenderProxy.obj
 0001:00072c60       ?SetMaterial@CRenderProxy@@UAEXPAUIMaterial@@@Z 32073c60 f   RenderProxy.obj
 0001:00072c80       ?GetEntityClassName@CRenderProxy@@UBEPBDXZ 32073c80 f   RenderProxy.obj
 0001:00072ca0       ?GetPos@CRenderProxy@@UBE?AU?$Vec3_tpl@M@@_N@Z 32073ca0 f   RenderProxy.obj
 0001:00072cf0       ?GetAngles@CRenderProxy@@UBEABU?$Ang3_tpl@M@@H@Z 32073cf0 f   RenderProxy.obj
 0001:00072d20       ?GetScale@CRenderProxy@@UBEMXZ 32073d20 f   RenderProxy.obj
 0001:00072d30       ?GetName@CRenderProxy@@UBEPBDXZ 32073d30 f   RenderProxy.obj
 0001:00072d40       ?GetBBox@CRenderProxy@@UAEXAAU?$Vec3_tpl@M@@0@Z 32073d40 f   RenderProxy.obj
 0001:00072d40       ?GetRenderBBox@CRenderProxy@@UAEXAAU?$Vec3_tpl@M@@0@Z 32073d40 f   RenderProxy.obj
 0001:00072d90       ?SetCustomPostEffect@CRenderProxy@@UAEXPBD@Z 32073d90 f   RenderProxy.obj
 0001:00072dd0       ?SetAsPost3dRenderObject@CRenderProxy@@UAEX_NEQAM@Z 32073dd0 f   RenderProxy.obj
 0001:00072e10       ?IsMovableByGame@CRenderProxy@@EBE_NXZ 32073e10 f   RenderProxy.obj
 0001:00072e50       ?GetRenderNodeType@CRenderProxy@@UAE?AW4EERType@@XZ 32073e50 f   RenderProxy.obj
 0001:00072e60       ?NeedSerialize@CTriggerProxy@@UAE_NXZ 32073e60 f i TriggerProxy.obj
 0001:00072e60       ?IsRenderNode@IShadowCaster@@UAE_NXZ 32073e60 f i RenderProxy.obj
 0001:00072e60       ?NeedSerialize@CRopeProxy@@UAE_NXZ 32073e60 f i RopeProxy.obj
 0001:00072e70       ??_EIShadowCaster@@UAEPAXI@Z 32073e70 f i RenderProxy.obj
 0001:00072e70       ??_GIShadowCaster@@UAEPAXI@Z 32073e70 f i RenderProxy.obj
 0001:00072ea0       ?SetCloakBlendTimeScale@CRenderProxy@@UAEXM@Z 32073ea0 f i RenderProxy.obj
 0001:00072ef0       ??_GCCameraProxy@@UAEPAXI@Z 32073ef0 f i CameraProxy.obj
 0001:00072ef0       ??_ECRopeProxy@@UAEPAXI@Z  32073ef0 f i RopeProxy.obj
 0001:00072ef0       ??_GCPhysicalProxy@@UAEPAXI@Z 32073ef0 f i PhysicsProxy.obj
 0001:00072ef0       ??_ECPhysicalProxy@@UAEPAXI@Z 32073ef0 f i PhysicsProxy.obj
 0001:00072ef0       ??_GCRopeProxy@@UAEPAXI@Z  32073ef0 f i RopeProxy.obj
 0001:00072ef0       ??_GIEntityRenderProxy@@UAEPAXI@Z 32073ef0 f i RenderProxy.obj
 0001:00072ef0       ??_ECEntityNodeProxy@@UAEPAXI@Z 32073ef0 f i Entity.obj
 0001:00072ef0       ??_GIEntityProxy@@UAEPAXI@Z 32073ef0 f i Entity.obj
 0001:00072ef0       ??_ECCameraProxy@@UAEPAXI@Z 32073ef0 f i CameraProxy.obj
 0001:00072ef0       ??_GCEntityNodeProxy@@UAEPAXI@Z 32073ef0 f i Entity.obj
 0001:00072ef0       ??_EIEntityProxy@@UAEPAXI@Z 32073ef0 f i Entity.obj
 0001:00072ef0       ??_EIEntityRenderProxy@@UAEPAXI@Z 32073ef0 f i RenderProxy.obj
 0001:00072f20       ?UpdateMaterialLayersRendParams@CRenderProxy@@AAEXAAUSRendParams@@ABUSRenderingPassInfo@@@Z 32073f20 f   RenderProxy.obj
 0001:00073220       ??0SRendParams@@QAE@ABU0@@Z 32074220 f i RenderProxy.obj
 0001:000733a0       ?SerializeXML@CRenderProxy@@UAEXAAVXmlNodeRef@@_N@Z 320743a0 f   RenderProxy.obj
 0001:00073430       ?GetSignature@CRenderProxy@@UAE_NV?$CSerializeWrapper@UISerialize@@@@@Z 32074430 f   RenderProxy.obj
 0001:00073460       ?GetShaderPublicParams@CRenderProxy@@UAEPAUIShaderPublicParams@@_N@Z 32074460 f   RenderProxy.obj
 0001:000734c0       ?SetMaterialLayersMask@CRenderProxy@@UAEXE@Z 320744c0 f   RenderProxy.obj
 0001:00073520       ?GetMaterial@CRenderProxy@@UAEPAUIMaterial@@PAU?$Vec3_tpl@M@@@Z 32074520 f   RenderProxy.obj
 0001:00073530       ?GetMaxViewDist@CRenderProxy@@UAEMXZ 32074530 f   RenderProxy.obj
 0001:00073720       ?IsRenderProxyVisAreaVisible@CRenderProxy@@UBE_NXZ 32074720 f   RenderProxy.obj
 0001:00073770       ??0SGeometryDebugDrawInfo@@QAE@ABU0@@Z 32074770 f i RenderProxy.obj
 0001:00073800       ?GetImportance@IRenderNode@@UBEMXZ 32074800 f i RenderProxy.obj
 0001:00073810       ?GetType@CRenderProxy@@UAE?AW4EEntityProxy@@XZ 32074810 f i RenderProxy.obj
 0001:00073810       ?GetICharacterInstance@IAttachmentObject@@UBEPAUICharacterInstance@@XZ 32074810 f i Entity.obj
 0001:00073810       ?GetType@CDeferredMeshUpdatePrep@@UBE?AW4DeferredEventType@IDeferredPhysicsEvent@@XZ 32074810 f i PhysicsEventListener.obj
 0001:00073810       ?GetBaseMaterial@CEffectAttachment@@UBEPAUIMaterial@@XZ 32074810 f i ScriptBind_Entity.obj
 0001:00073810       ?GetEditorObjectId@IRenderNode@@UAEHXZ 32074810 f i RenderProxy.obj
 0001:00073810       ?GetReplacementMaterial@CLightAttachment@@UBEPAUIMaterial@@XZ 32074810 f i ScriptBind_Entity.obj
 0001:00073810       ?GetLayerId@IRenderNode@@UAEGXZ 32074810 f i RenderProxy.obj
 0001:00073810       ?PhysicsEvent@CDeferredMeshUpdatePrep@@UAEPAUEventPhys@@XZ 32074810 f i PhysicsEventListener.obj
 0001:00073810       ?GetBaseMaterial@CEntityAttachment@@UBEPAUIMaterial@@XZ 32074810 f i Entity.obj
 0001:00073810       ?GetReplacementMaterial@CEntityAttachment@@UBEPAUIMaterial@@XZ 32074810 f i Entity.obj
 0001:00073810       ?GetPhysics@CRenderProxy@@UBEPAUIPhysicalEntity@@XZ 32074810 f i RenderProxy.obj
 0001:00073810       ?GetIStatObj@IAttachmentObject@@UBEPAUIStatObj@@XZ 32074810 f i Entity.obj
 0001:00073810       ?GetBaseMaterial@CLightAttachment@@UBEPAUIMaterial@@XZ 32074810 f i ScriptBind_Entity.obj
 0001:00073810       ?GetIAttachmentSkin@IAttachmentObject@@UBEPAUIAttachmentSkin@@XZ 32074810 f i Entity.obj
 0001:00073810       ?GetReplacementMaterial@CEffectAttachment@@UBEPAUIMaterial@@XZ 32074810 f i ScriptBind_Entity.obj
 0001:00073810       ?Clone@IRenderNode@@UBEPAU1@XZ 32074810 f i RenderProxy.obj
 0001:00073820       ?HasLightmap@IRenderNode@@UAE_NH@Z 32074820 f i RenderProxy.obj
 0001:00073820       ?ShouldUpdateCharacter@CEntity@@UBE_NH@Z 32074820 f i Entity.obj
 0001:00073820       ?PostRender@IRenderNode@@UAE_NABUSRenderingPassInfo@@@Z 32074820 f i RenderProxy.obj
 0001:00073830       ?GetLimit@CTypeInfo@@UBE_NW4ENumericLimit@@AAM@Z 32074830 f i CryEntityDLL.obj
 0001:00073830       ?HasOcclusionmap@IShadowCaster@@UAE_NHPAUIRenderNode@@@Z 32074830 f i RenderProxy.obj
 0001:00073830       ?HasOcclusionmap@IRenderNode@@UAE_NHPAU1@@Z 32074830 f i RenderProxy.obj
 0001:00073840       ?GetLightmapData@IRenderNode@@UAEPAUSLMData@@HH@Z 32074840 f i RenderProxy.obj
 0001:00073850       ?GetMaterialLayers@IRenderNode@@UBEEXZ 32074850 f i RenderProxy.obj
 0001:00073860       ?Stop@CDummyMemReplay@@UAEXXZ 32074860 f i AreaSolid.obj
 0001:00073860       ?Precache@IRenderNode@@UAEXXZ 32074860 f i RenderProxy.obj
 0001:00073860       ?Done@CTriggerProxy@@UAEXXZ 32074860 f i TriggerProxy.obj
 0001:00073860       ?Reset@CEntityLoadManager@@QAEXXZ 32074860 f i EntityLoadManager.obj
 0001:00073860       ?Done@CRopeProxy@@UAEXXZ   32074860 f i RopeProxy.obj
 0001:00073860       ?Done@CAreaProxy@@UAEXXZ   32074860 f i AreaProxy.obj
 0001:00073860       ?Done@CEntityNodeProxy@@UAEXXZ 32074860 f i Entity.obj
 0001:00073860       ?AddFrameStart@CDummyMemReplay@@UAEXXZ 32074860 f i AreaSolid.obj
 0001:00073860       ?Done@CSoundProxy@@UAEXXZ  32074860 f i SoundProxy.obj
 0001:00073860       ?AddLabelFmt@CDummyMemReplay@@UAAXPBDZZ 32074860 f i AreaSolid.obj
 0001:00073860       ?OnPhysAreaChange@IRenderNode@@UAEXXZ 32074860 f i RenderProxy.obj
 0001:00073860       ?UpdateIndirLightForChildren@IEntityRenderProxy@@UAEXXZ 32074860 f i RenderProxy.obj
 0001:00073860       ?CheckPhysicalized@IRenderNode@@UAEXXZ 32074860 f i RenderProxy.obj
 0001:00073860       ?OnNotSeenTimeout@CEntityObject@@QAEXXZ 32074860 f i EntityObject.obj
 0001:00073860       ?Done@Test@CryUnitTest@@UAEXXZ 32074860 f i PartitionGrid.obj
 0001:00073860       ?DumpStats@CDummyMemReplay@@UAEXXZ 32074860 f i AreaSolid.obj
 0001:00073860       ?DumpSymbols@CDummyMemReplay@@UAEXXZ 32074860 f i AreaSolid.obj
 0001:00073860       ?sp_enable_shared_from_this@detail@boost@@YAXZZ 32074860 f i CryEntityDLL.obj
 0001:00073860       ?Done@CCameraProxy@@UAEXXZ 32074860 f i CameraProxy.obj
 0001:00073860       ?Stop@CDeferredMeshUpdatePrep@@UAEXXZ 32074860 f i PhysicsEventListener.obj
 0001:00073860       ?ExitScope@CDummyMemReplay@@UAEXXZ 32074860 f i AreaSolid.obj
 0001:00073860       ?Sync@CDeferredMeshUpdatePrep@@UAEXXZ 32074860 f i PhysicsEventListener.obj
 0001:00073860       ?AddScreenshot@CDummyMemReplay@@UAEXXZ 32074860 f i AreaSolid.obj
 0001:00073860       ?Done@CRenderProxy@@UAEXXZ 32074860 f i RenderProxy.obj
 0001:00073860       ?Init@Test@CryUnitTest@@UAEXXZ 32074860 f i PartitionGrid.obj
 0001:00073860       ?Dematerialize@IRenderNode@@UAEXXZ 32074860 f i RenderProxy.obj
 0001:00073860       ?RemoveContext@CDummyMemReplay@@UAEXXZ 32074860 f i AreaSolid.obj
 0001:00073860       ?Start@CDeferredMeshUpdatePrep@@UAEXXZ 32074860 f i PhysicsEventListener.obj
 0001:00073860       ?Flush@CDummyMemReplay@@UAEXXZ 32074860 f i AreaSolid.obj
 0001:00073870       ?GetStatObjGroupId@IRenderNode@@UBEHXZ 32074870 f i RenderProxy.obj
 0001:00073880       ?IsAllocatedOutsideOf3DEngineDLL@IRenderNode@@UAE_NXZ 32074880 f i RenderProxy.obj
 0001:00073890       ?GetBBoxVirtual@IRenderNode@@UAE?BUAABB@@XZ 32074890 f i RenderProxy.obj
 0001:000738b0       ?SetIntegrationType@IRenderNode@@UAEXW4EMeshIntegrationType@@@Z 320748b0 f i RenderProxy.obj
 0001:00073900       ?Hide@IRenderNode@@UAEX_N@Z 32074900 f i RenderProxy.obj
 0001:00073920       ?GetBBox@CRenderProxy@@UBE?BUAABB@@XZ 32074920 f i RenderProxy.obj
 0001:00073960       ?AnimEventCallback@CRenderProxy@@SAHPAUICharacterInstance@@PAX@Z 32074960 f   RenderProxy.obj
 0001:000739d0       ??0?$shared_ptr@UIShaderParamCallback@@@boost@@QAE@ABV01@@Z 320749d0 f i RenderProxy.obj
 0001:00073a00       ?FillBBox@CRenderProxy@@UAEXAAUAABB@@@Z 32074a00 f   RenderProxy.obj
 0001:00073a80       ??4?$shared_ptr@UIShaderParamCallback@@@boost@@QAEAAV01@ABV01@@Z 32074a80 f i RenderProxy.obj
 0001:00073ae0       ??$__copy@PAV?$shared_ptr@UIShaderParamCallback@@@boost@@PAV12@H@priv@stlpmtx_std@@YAPAV?$shared_ptr@UIShaderParamCallback@@@boost@@PAV23@00ABUrandom_access_iterator_tag@1@PAH@Z 32074ae0 f i RenderProxy.obj
 0001:00073b70       ?Op@?$cryinterface_cast_boost_helper@UIShaderParamCallback@@UICryUnknown@@@Internal@InterfaceCastSemantics@@SA?AV?$shared_ptr@UIShaderParamCallback@@@boost@@ABV?$shared_ptr@UICryUnknown@@@5@@Z 32074b70 f i RenderProxy.obj
 0001:00073c70       ?SetParentSlot@CRenderProxy@@QAE_NHH@Z 32074c70 f   RenderProxy.obj
 0001:00073cb0       ?GetCompoundObj@CRenderProxy@@QBEPAUIStatObj@@XZ 32074cb0 f   RenderProxy.obj
 0001:00073cf0       ?GetSlotWorldTM@CRenderProxy@@QBEABU?$Matrix34_tpl@M@@H@Z 32074cf0 f   RenderProxy.obj
 0001:000744b0       ?GetSlotLocalTM@CRenderProxy@@QBEABU?$Matrix34_tpl@M@@H_N@Z 320754b0 f   RenderProxy.obj
 0001:00075000       ?CalcLocalBounds@CRenderProxy@@AAEXXZ 32076000 f   RenderProxy.obj
 0001:00075840       ?GetLocalBounds@CRenderProxy@@UAEXAAUAABB@@@Z 32076840 f   RenderProxy.obj
 0001:00075880       ?GetWorldBounds@CRenderProxy@@UAEXAAUAABB@@@Z 32076880 f   RenderProxy.obj
 0001:00075b50       ?Render@CRenderProxy@@UAEXABUSRendParams@@ABUSRenderingPassInfo@@@Z 32076b50 f   RenderProxy.obj
 0001:00075e30       ?GetEntityStatObj@CRenderProxy@@UAEPAUIStatObj@@IIPAU?$Matrix34_tpl@M@@_N@Z 32076e30 f   RenderProxy.obj
 0001:00075ee0       ?GetEntityCharacter@CRenderProxy@@UAEPAUICharacterInstance@@IPAU?$Matrix34_tpl@M@@_N@Z 32076ee0 f   RenderProxy.obj
 0001:00075f90       ?GetEntitySlotMaterial@CRenderProxy@@UAEPAUIMaterial@@I_NPA_N@Z 32076f90 f   RenderProxy.obj
 0001:00076000       ?SetCustomMaterial@CRenderProxy@@QAEXPAUIMaterial@@@Z 32077000 f   RenderProxy.obj
 0001:000760f0       ?RegisterForRendering@CRenderProxy@@QAEX_N@Z 320770f0 f   RenderProxy.obj
 0001:000764e0       ?GetSlotInfo@CRenderProxy@@QBE_NHAAUSEntitySlotInfo@@@Z 320774e0 f   RenderProxy.obj
 0001:000765d0       ?GetSlotFlags@CRenderProxy@@QAEIH@Z 320775d0 f   RenderProxy.obj
 0001:00076610       ?SetSlotMaterial@CRenderProxy@@UAEXHPAUIMaterial@@@Z 32077610 f   RenderProxy.obj
 0001:00076670       ?GetSlotMaterial@CRenderProxy@@UAEPAUIMaterial@@H@Z 32077670 f   RenderProxy.obj
 0001:000766a0       ?GetCharacter@CRenderProxy@@QAEPAUICharacterInstance@@H@Z 320776a0 f   RenderProxy.obj
 0001:000766e0       ?GetStatObj@CRenderProxy@@QAEPAUIStatObj@@H@Z 320776e0 f   RenderProxy.obj
 0001:00076800       ?GetParticleEmitter@CRenderProxy@@QAEPAUIParticleEmitter@@H@Z 32077800 f   RenderProxy.obj
 0001:00076840       ?GetRenderMaterial@CRenderProxy@@UAEPAUIMaterial@@H@Z 32077840 f   RenderProxy.obj
 0001:00076900       ?SetViewDistRatio@CRenderProxy@@UAEXH@Z 32077900 f   RenderProxy.obj
 0001:000769d0       ?SetMinSpec@CRenderProxy@@UAEXH@Z 320779d0 f   RenderProxy.obj
 0001:00076a60       ?SetLodRatio@CRenderProxy@@UAEXH@Z 32077a60 f   RenderProxy.obj
 0001:00076af0       ?DebugDraw@CRenderProxy@@QAEXABUSGeometryDebugDrawInfo@@@Z 32077af0 f   RenderProxy.obj
 0001:00076c00       ?PhysicalizeFoliage@CRenderProxy@@UAE_N_NHH@Z 32077c00 f   RenderProxy.obj
 0001:00076fd0       ?GetFoliage@CRenderProxy@@UAEPAUIFoliage@@H@Z 32077fd0 f   RenderProxy.obj
 0001:00077050       ?SetSubObjHideMask@CRenderProxy@@UAEXH_K@Z 32078050 f   RenderProxy.obj
 0001:00077090       ?GetSubObjHideMask@CRenderProxy@@UBE_KH@Z 32078090 f   RenderProxy.obj
 0001:000770d0       ??$__destroy_range_aux@V?$reverse_iterator@PAV?$shared_ptr@UIShaderParamCallback@@@boost@@@stlpmtx_std@@V?$shared_ptr@UIShaderParamCallback@@@boost@@@stlpmtx_std@@YAXV?$reverse_iterator@PAV?$shared_ptr@UIShaderParamCallback@@@boost@@@0@0PAV?$shared_ptr@UIShaderParamCallback@@@boost@@ABU__false_type@0@@Z 320780d0 f i RenderProxy.obj
 0001:00077130       ??$__destroy_range_aux@PAV?$shared_ptr@UIShaderParamCallback@@@boost@@V12@@stlpmtx_std@@YAXPAV?$shared_ptr@UIShaderParamCallback@@@boost@@00ABU__false_type@0@@Z 32078130 f i RenderProxy.obj
 0001:00077190       ?InvalidateBounds@CRenderProxy@@QAEX_N0@Z 32078190 f   RenderProxy.obj
 0001:000771c0       ?SetSlotFlags@CRenderProxy@@QAEXHI@Z 320781c0 f   RenderProxy.obj
 0001:00077270       ?GetMemoryUsage@CRenderProxy@@UBEXPAVICrySizer@@@Z 32078270 f   RenderProxy.obj
 0001:000772e0       ??$CryCreateClassInstance@UIShaderParamCallback@@@@YA_NPBDAAV?$shared_ptr@UIShaderParamCallback@@@boost@@@Z 320782e0 f i RenderProxy.obj
 0001:000773b0       ??$__ufill@PAV?$shared_ptr@UIShaderParamCallback@@@boost@@V12@H@priv@stlpmtx_std@@YAXPAV?$shared_ptr@UIShaderParamCallback@@@boost@@0ABV23@ABUrandom_access_iterator_tag@1@PAH@Z 320783b0 f i RenderProxy.obj
 0001:00077400       ??$__ucopy@PAV?$shared_ptr@UIShaderParamCallback@@@boost@@PAV12@H@priv@stlpmtx_std@@YAPAV?$shared_ptr@UIShaderParamCallback@@@boost@@PAV23@00ABUrandom_access_iterator_tag@1@PAH@Z 32078400 f i RenderProxy.obj
 0001:00077450       ?GetDebugString@IRenderNode@@UBE?AV?$CryStringT@D@@D@Z 32078450 f i RenderProxy.obj
 0001:00077470       ??2CEntityObject@@SAPAXI@Z 32078470 f i RenderProxy.obj
 0001:000774d0       ??3CEntityObject@@SAXPAX@Z 320784d0 f i RenderProxy.obj
 0001:00077530       ?FreeSlot@CRenderProxy@@QAEXH@Z 32078530 f   RenderProxy.obj
 0001:00077600       ?SetSlotLocalTM@CRenderProxy@@QAEXHABU?$Matrix34_tpl@M@@H@Z 32078600 f   RenderProxy.obj
 0001:000776f0       ?SetLocalBounds@CRenderProxy@@UAEXABUAABB@@_N@Z 320786f0 f   RenderProxy.obj
 0001:00077750       ?InvalidateLocalBounds@CRenderProxy@@UAEXXZ 32078750 f   RenderProxy.obj
 0001:00077770       ?OnEntityXForm@CRenderProxy@@AAEXH@Z 32078770 f   RenderProxy.obj
 0001:000777d0       ?OnHide@CRenderProxy@@AAEX_N@Z 320787d0 f   RenderProxy.obj
 0001:00077910       ?Update@CRenderProxy@@UAEXAAUSEntityUpdateContext@@@Z 32078910 f   RenderProxy.obj
 0001:00077a20       ?CheckShaderParamCallbacks@CRenderProxy@@UAEXXZ 32078a20 f   RenderProxy.obj
 0001:00077bb0       ?_M_erase@?$_Impl_vector@V?$shared_ptr@UIShaderParamCallback@@@boost@@V?$allocator@V?$shared_ptr@UIShaderParamCallback@@@boost@@@stlpmtx_std@@@priv@stlpmtx_std@@AAEPAV?$shared_ptr@UIShaderParamCallback@@@boost@@PAV45@ABU__false_type@3@@Z 32078bb0 f i RenderProxy.obj
 0001:00077c30       ?PostInit@CRenderProxy@@QAEXXZ 32078c30 f   RenderProxy.obj
 0001:00077c60       ?ProcessEvent@CRenderProxy@@UAEXAAUSEntityEvent@@@Z 32078c60 f   RenderProxy.obj
 0001:00077ed0       ?FreeAllSlots@CRenderProxy@@QAEXXZ 32078ed0 f   RenderProxy.obj
 0001:00077fb0       ?_M_insert_overflow_aux@?$_Impl_vector@V?$shared_ptr@UIShaderParamCallback@@@boost@@V?$allocator@V?$shared_ptr@UIShaderParamCallback@@@boost@@@stlpmtx_std@@@priv@stlpmtx_std@@AAEXPAV?$shared_ptr@UIShaderParamCallback@@@boost@@ABV45@ABU__false_type@3@I_N@Z 32078fb0 f i RenderProxy.obj
 0001:00078150       ??0CRenderProxy@@QAE@PAVCEntity@@@Z 32079150 f   RenderProxy.obj
 0001:00078320       ?Init@CSubstitutionProxy@@UAE_NPAUIEntity@@AAUSEntitySpawnParams@@@Z 32079320 f i Entity.obj
 0001:00078320       ?Init@CTriggerProxy@@UAE_NPAUIEntity@@AAUSEntitySpawnParams@@@Z 32079320 f i TriggerProxy.obj
 0001:00078320       ?Init@CFlowGraphProxy@@UAE_NPAUIEntity@@AAUSEntitySpawnParams@@@Z 32079320 f i FlowGraphProxy.obj
 0001:00078320       ?Init@CRenderProxy@@UAE_NPAUIEntity@@AAUSEntitySpawnParams@@@Z 32079320 f i RenderProxy.obj
 0001:00078320       ?Init@CSoundProxy@@UAE_NPAUIEntity@@AAUSEntitySpawnParams@@@Z 32079320 f i SoundProxy.obj
 0001:00078320       ?Init@CRopeProxy@@UAE_NPAUIEntity@@AAUSEntitySpawnParams@@@Z 32079320 f i RopeProxy.obj
 0001:00078320       ?Init@CAreaProxy@@UAE_NPAUIEntity@@AAUSEntitySpawnParams@@@Z 32079320 f i AreaProxy.obj
 0001:00078320       ?Init@CPhysicalProxy@@UAE_NPAUIEntity@@AAUSEntitySpawnParams@@@Z 32079320 f i PhysicsProxy.obj
 0001:00078330       ?GetBranchPhys@CRenderProxy@@UAEPAUIPhysicalEntity@@HH@Z 32079330 f i RenderProxy.obj
 0001:00078360       ?GetRenderNode@CRenderProxy@@UAEPAUIRenderNode@@XZ 32079360 f i RenderProxy.obj
 0001:00078370       ?AllocUsage@CDummyMemReplay@@UAEXW4Class@EMemReplayAllocClass@@II@Z 32079370 f i AreaSolid.obj
 0001:00078370       ?ExitScope_Alloc@CDummyMemReplay@@UAEXIII@Z 32079370 f i AreaSolid.obj
 0001:00078370       ?AddContext@CDummyMemReplay@@UAEXHIPBD@Z 32079370 f i AreaSolid.obj
 0001:00078370       ?RegisterFixedAddressRange@CDummyMemReplay@@UAEXPAXIPBD@Z 32079370 f i AreaSolid.obj
 0001:00078370       ?SetEntityStatObj@CRenderProxy@@UAEXIPAUIStatObj@@PBU?$Matrix34_tpl@M@@@Z 32079370 f i RenderProxy.obj
 0001:00078380       ?SetLightmap@IRenderNode@@UAEXPAURenderLMData@@PAMIHH@Z 32079380 f i RenderProxy.obj
 0001:00078380       ?MarkPool@CDummyMemReplay@@UAEXHIPAXIPBD@Z 32079380 f i AreaSolid.obj
 0001:00078380       ?PreloadInstanceResources@CRenderProxy@@UAEXU?$Vec3_tpl@M@@MM@Z 32079380 f i RenderProxy.obj
 0001:00078390       ?GetMaterialLayersMask@CRenderProxy@@UBEEXZ 32079390 f i RenderProxy.obj
 0001:000783a0       ?SetMaterialLayersBlend@CRenderProxy@@UAEXI@Z 320793a0 f i RenderProxy.obj
 0001:000783b0       ?GetMaterialLayersBlend@CRenderProxy@@UBEIXZ 320793b0 f i RenderProxy.obj
 0001:000783c0       ?GetCloakInterferenceState@CRenderProxy@@UBE_NXZ 320793c0 f i RenderProxy.obj
 0001:000783d0       ?SetCloakColorChannel@CRenderProxy@@UAEXE@Z 320793d0 f i RenderProxy.obj
 0001:000783e0       ?GetCloakColorChannel@CRenderProxy@@UBEEXZ 320793e0 f i RenderProxy.obj
 0001:000783f0       ?DoesCloakFadeByDistance@CRenderProxy@@UBE_NXZ 320793f0 f i RenderProxy.obj
 0001:00078400       ?GetCloakBlendTimeScale@CRenderProxy@@UBEMXZ 32079400 f i RenderProxy.obj
 0001:00078420       ?DoesIgnoreCloakRefractionColor@CRenderProxy@@UBE_NXZ 32079420 f i RenderProxy.obj
 0001:00078430       ?GetMaterialOverride@CRenderProxy@@UAEPAUIMaterial@@XZ 32079430 f i RenderProxy.obj
 0001:00078430       ?GetVisionParams@CRenderProxy@@UBEIXZ 32079430 f i RenderProxy.obj
 0001:00078440       ?GetHUDSilhouettesParams@CRenderProxy@@UBEIXZ 32079440 f i RenderProxy.obj
 0001:00078450       ?SetEffectLayerParams@CRenderProxy@@UAEXI@Z 32079450 f i RenderProxy.obj
 0001:00078460       ?GetEffectLayerParams@CRenderProxy@@UBE?BIXZ 32079460 f i RenderProxy.obj
 0001:00078470       ?GetOpacity@CRenderProxy@@UBEMXZ 32079470 f i RenderProxy.obj
 0001:00078490       ?SetBBox@CRenderProxy@@UAEXABUAABB@@@Z 32079490 f i RenderProxy.obj
 0001:000784d0       ?GetLastSeenTime@CRenderProxy@@UBEMXZ 320794d0 f i RenderProxy.obj
 0001:000784e0       ??_ECRenderProxy@@WCE@AEPAXI@Z 320794e0 f i RenderProxy.obj
 0001:000784f0       ?SetCloakHighlightStrength@CRenderProxy@@UAEXM@Z 320794f0 f i RenderProxy.obj
 0001:00078540       ?SetCloakInterferenceState@CRenderProxy@@UAEX_N@Z 32079540 f i RenderProxy.obj
 0001:00078560       ?SetCloakFadeByDistance@CRenderProxy@@UAEX_N@Z 32079560 f i RenderProxy.obj
 0001:00078580       ?SetIgnoreCloakRefractionColor@CRenderProxy@@UAEX_N@Z 32079580 f i RenderProxy.obj
 0001:000785a0       ?SetIgnoreHudInterferenceFilter@CRenderProxy@@UAEX_N@Z 320795a0 f i RenderProxy.obj
 0001:000785c0       ?SetHUDRequireDepthTest@CRenderProxy@@UAEX_N@Z 320795c0 f i RenderProxy.obj
 0001:000785e0       ?SetHUDDisableBloom@CRenderProxy@@UAEX_N@Z 320795e0 f i RenderProxy.obj
 0001:00078600       ?SetIgnoreHeatAmount@CRenderProxy@@UAEX_N@Z 32079600 f i RenderProxy.obj
 0001:00078620       ?SetVisionParams@CRenderProxy@@UAEXMMMM@Z 32079620 f i RenderProxy.obj
 0001:000786a0       ?SetHUDSilhouettesParams@CRenderProxy@@UAEXMMMM@Z 320796a0 f i RenderProxy.obj
 0001:00078720       ?SetShadowDissolve@CRenderProxy@@UAEX_N@Z 32079720 f i RenderProxy.obj
 0001:00078740       ?GetShadowDissolve@CRenderProxy@@UBE_NXZ 32079740 f i RenderProxy.obj
 0001:00078760       ?SetEffectLayerParams@CRenderProxy@@UAEXABU?$Vec4_tpl@M@@@Z 32079760 f i RenderProxy.obj
 0001:000787f0       ?SetOpacity@CRenderProxy@@UAEXM@Z 320797f0 f i RenderProxy.obj
 0001:00078830       ?UpdateCharactersBeforePhysics@CRenderProxy@@UAEX_N@Z 32079830 f i RenderProxy.obj
 0001:00078850       ?IsCharactersUpdatedBeforePhysics@CRenderProxy@@UAE_NXZ 32079850 f i RenderProxy.obj
 0001:00078870       ?GetSlotCount@CRenderProxy@@UBEHXZ 32079870 f i RenderProxy.obj
 0001:00078880       ?GetLocalBounds@CRenderProxy@@WCE@AEXAAUAABB@@@Z 32079880 f i RenderProxy.obj
 0001:00078890       ?GetMemoryUsage@CRenderProxy@@WCE@BEXPAVICrySizer@@@Z 32079890 f i RenderProxy.obj
 0001:000788a0       ??3CRenderProxy@@SAXPAX@Z  320798a0 f i RenderProxy.obj
 0001:00078900       ?ClearSlots@CRenderProxy@@UAEXXZ 32079900 f i RenderProxy.obj
 0001:00078910       ?AllocSlot@CRenderProxy@@QAEPAVCEntityObject@@H@Z 32079910 f   RenderProxy.obj
 0001:00078a00       ?SetSlotGeometry@CRenderProxy@@QAEHHPAUIStatObj@@@Z 32079a00 f   RenderProxy.obj
 0001:00078cd0       ?SetSlotCharacter@CRenderProxy@@QAEHHPAUICharacterInstance@@@Z 32079cd0 f   RenderProxy.obj
 0001:00078e20       ?LoadGeometry@CRenderProxy@@QAEHHPBD0H@Z 32079e20 f   RenderProxy.obj
 0001:00078f80       ?LoadCharacter@CRenderProxy@@QAEHHPBDH@Z 32079f80 f   RenderProxy.obj
 0001:00079150       ?SetParticleEmitter@CRenderProxy@@QAEHHPAUIParticleEmitter@@_N@Z 3207a150 f   RenderProxy.obj
 0001:00079220       ?LoadParticleEmitter@CRenderProxy@@QAEHHPAUIParticleEffect@@PBUSpawnParams@@_N2@Z 3207a220 f   RenderProxy.obj
 0001:000796d0       ?LoadLight@CRenderProxy@@QAEHHPAVCDLight@@_N@Z 3207a6d0 f   RenderProxy.obj
 0001:00079800       ?LoadCloud@CRenderProxy@@QAEHHPBD@Z 3207a800 f   RenderProxy.obj
 0001:000798a0       ?SetCloudMovementProperties@CRenderProxy@@QAEHHABUSCloudMovementProperties@@@Z 3207a8a0 f   RenderProxy.obj
 0001:000798f0       ?LoadFogVolume@CRenderProxy@@QAEHHABUSFogVolumeProperties@@@Z 3207a8f0 f   RenderProxy.obj
 0001:00079a20       ?LoadLightShape@CRenderProxy@@QAEHHPBDI@Z 3207aa20 f   RenderProxy.obj
 0001:00079ab0       ?FadeGlobalDensity@CRenderProxy@@QAEHHMM@Z 3207aab0 f   RenderProxy.obj
 0001:00079b10       ?LoadVolumeObject@CRenderProxy@@QAEHHPBD@Z 3207ab10 f   RenderProxy.obj
 0001:00079bc0       ?SetVolumeObjectMovementProperties@CRenderProxy@@QAEHHABUSVolumeObjectMovementProperties@@@Z 3207abc0 f   RenderProxy.obj
 0001:00079c10       ?LoadPrismObject@CRenderProxy@@QAEHH@Z 3207ac10 f   RenderProxy.obj
 0001:00079ca0       ?Serialize@CRenderProxy@@UAEXV?$CSerializeWrapper@UISerialize@@@@@Z 3207aca0 f   RenderProxy.obj
 0001:00079f70       ?RemoveShaderParamCallback@CRenderProxy@@UAE_NV?$shared_ptr@UIShaderParamCallback@@@boost@@@Z 3207af70 f   RenderProxy.obj
 0001:0007a010       ?Reload@CRenderProxy@@UAEXPAUIEntity@@AAUSEntitySpawnParams@@@Z 3207b010 f   RenderProxy.obj
 0001:0007a1a0       ?ClearShaderParamCallbacks@CRenderProxy@@UAEXXZ 3207b1a0 f   RenderProxy.obj
 0001:0007a290       ??1CRenderProxy@@UAE@XZ    3207b290 f   RenderProxy.obj
 0001:0007a4e0       ?AddShaderParamCallback@CRenderProxy@@UAEXV?$shared_ptr@UIShaderParamCallback@@@boost@@@Z 3207b4e0 f   RenderProxy.obj
 0001:0007a5f0       ??_GCRenderProxy@@UAEPAXI@Z 3207b5f0 f i RenderProxy.obj
 0001:0007a5f0       ??_ECRenderProxy@@UAEPAXI@Z 3207b5f0 f i RenderProxy.obj
 0001:0007a620       ?GetBox@CArea@@QAEXAAU?$Vec3_tpl@M@@0@Z 3207b620 f i AreaProxy.obj
 0001:0007a670       ?BeginSettingSolid@CAreaProxy@@UAEXABU?$Matrix34_tpl@M@@@Z 3207b670 f   AreaProxy.obj
 0001:0007a6a0       ?AddConvexHullToSolid@CAreaProxy@@UAEXPBU?$Vec3_tpl@M@@_NH@Z 3207b6a0 f   AreaProxy.obj
 0001:0007a6b0       ?EndSettingSolid@CAreaProxy@@UAEXXZ 3207b6b0 f   AreaProxy.obj
 0001:0007a6c0       ??$__fill@U?$_Bit_iter@U_Bit_reference@priv@stlpmtx_std@@PAU123@@priv@stlpmtx_std@@_NH@priv@stlpmtx_std@@YAXU?$_Bit_iter@U_Bit_reference@priv@stlpmtx_std@@PAU123@@01@0AB_NABUrandom_access_iterator_tag@1@PAH@Z 3207b6c0 f i AreaProxy.obj
 0001:0007a720       ??$__fill_n@U?$_Bit_iter@U_Bit_reference@priv@stlpmtx_std@@PAU123@@priv@stlpmtx_std@@I_N@priv@stlpmtx_std@@YA?AU?$_Bit_iter@U_Bit_reference@priv@stlpmtx_std@@PAU123@@01@U201@IAB_N@Z 3207b720 f i AreaProxy.obj
 0001:0007a780       ??$__copy@U?$_Bit_iter@U_Bit_reference@priv@stlpmtx_std@@PAU123@@priv@stlpmtx_std@@U123@H@priv@stlpmtx_std@@YA?AU?$_Bit_iter@U_Bit_reference@priv@stlpmtx_std@@PAU123@@01@U201@00ABUrandom_access_iterator_tag@1@PAH@Z 3207b780 f i AreaProxy.obj
 0001:0007a810       ??0CCryFile@@QAE@XZ        3207b810 f i AreaProxy.obj
 0001:0007a840       ?ReadRaw@CCryFile@@QAEIPAXI@Z 3207b840 f i AreaProxy.obj
 0001:0007a8a0       ?ReadPolygonsForAreaSolid@CAreaProxy@@AAEXAAVCCryFile@@H_N@Z 3207b8a0 f   AreaProxy.obj
 0001:0007a9c0       ?GetSignature@CAreaProxy@@UAE_NV?$CSerializeWrapper@UISerialize@@@@@Z 3207b9c0 f   AreaProxy.obj
 0001:0007a9f0       ??H?$_Bit_iter@U_Bit_reference@priv@stlpmtx_std@@PAU123@@priv@stlpmtx_std@@QBE?AU012@H@Z 3207b9f0 f i AreaProxy.obj
 0001:0007aa40       ??$__copy_backward@U?$_Bit_iter@U_Bit_reference@priv@stlpmtx_std@@PAU123@@priv@stlpmtx_std@@U123@H@priv@stlpmtx_std@@YA?AU?$_Bit_iter@U_Bit_reference@priv@stlpmtx_std@@PAU123@@01@U201@00ABUrandom_access_iterator_tag@1@PAH@Z 3207ba40 f i AreaProxy.obj
 0001:0007aad0       ?_AllocData@?$CryStackStringT@D$0CAA@@@QAEXI@Z 3207bad0 f i AreaProxy.obj
 0001:0007ab40       ?Reload@CAreaProxy@@UAEXPAUIEntity@@AAUSEntitySpawnParams@@@Z 3207bb40 f   AreaProxy.obj
 0001:0007abc0       ??1CCryFile@@QAE@XZ        3207bbc0 f i AreaProxy.obj
 0001:0007abc0       ?Close@CCryFile@@QAEXXZ    3207bbc0 f i AreaProxy.obj
 0001:0007ac10       ?_Assign@?$CryStackStringT@D$0CAA@@@QAEXPBDI@Z 3207bc10 f i AreaProxy.obj
 0001:0007ac80       ?GetPoints@CAreaProxy@@UAEPBU?$Vec3_tpl@M@@XZ 3207bc80 f   AreaProxy.obj
 0001:0007ac90       ?_M_bit_alloc@?$_Bvector_base@V?$allocator@_N@stlpmtx_std@@@priv@stlpmtx_std@@IAEPAII@Z 3207bc90 f i AreaProxy.obj
 0001:0007ace0       ??1CAreaProxy@@UAE@XZ      3207bce0 f   AreaProxy.obj
 0001:0007ada0       ?AddBreakEventListener@CBreakableManager@@UAEXPAUIBreakEventListener@@@Z 3207bda0 f i BreakableManager.obj
 0001:0007ada0       ?SetFlags@CAreaProxy@@UAEXH@Z 3207bda0 f i AreaProxy.obj
 0001:0007adb0       ?GetAreaType@CAreaProxy@@UBE?AW4EEntityAreaType@@XZ 3207bdb0 f i AreaProxy.obj
 0001:0007adc0       ?GetHeight@CAreaProxy@@UAEMXZ 3207bdc0 f i AreaProxy.obj
 0001:0007add0       ?GetBox@CAreaProxy@@UAEXAAU?$Vec3_tpl@M@@0@Z 3207bdd0 f i AreaProxy.obj
 0001:0007ae20       ?GetSphere@CAreaProxy@@UAEXAAU?$Vec3_tpl@M@@AAM@Z 3207be20 f i AreaProxy.obj
 0001:0007ae60       ?SetID@CAreaProxy@@UAEXH@Z 3207be60 f i AreaProxy.obj
 0001:0007ae70       ?GetID@CAreaProxy@@UBEHXZ  3207be70 f i AreaProxy.obj
 0001:0007ae80       ?SetGroup@CAreaProxy@@UAEXH@Z 3207be80 f i AreaProxy.obj
 0001:0007ae90       ?GetGroup@CAreaProxy@@UBEHXZ 3207be90 f i AreaProxy.obj
 0001:0007aea0       ?SetPriority@CAreaProxy@@UAEXH@Z 3207bea0 f i AreaProxy.obj
 0001:0007aeb0       ?GetPriority@CAreaProxy@@UBEHXZ 3207beb0 f i AreaProxy.obj
 0001:0007aec0       ?SetSoundObstructionOnAreaFace@CAreaProxy@@UAEXI_N@Z 3207bec0 f i AreaProxy.obj
 0001:0007aed0       ?AddEntity@CAreaProxy@@UAEXI@Z 3207bed0 f i AreaProxy.obj
 0001:0007aee0       ?ClearEntities@CAreaProxy@@UAEXXZ 3207bee0 f i AreaProxy.obj
 0001:0007aef0       ?SetProximity@CAreaProxy@@UAEXM@Z 3207bef0 f i AreaProxy.obj
 0001:0007af10       ?GetProximity@CAreaProxy@@UAEMXZ 3207bf10 f i AreaProxy.obj
 0001:0007af20       ?ClosestPointOnHullDistSq@CAreaProxy@@UAEMABU?$Vec3_tpl@M@@AAU2@@Z 3207bf20 f i AreaProxy.obj
 0001:0007af40       ?CalcPointNearDistSq@CAreaProxy@@UAEMABU?$Vec3_tpl@M@@AAU2@@Z 3207bf40 f i AreaProxy.obj
 0001:0007af60       ?CalcPointWithin@CAreaProxy@@UBE_NABU?$Vec3_tpl@M@@_N@Z 3207bf60 f i AreaProxy.obj
 0001:0007af80       ?GetPointsCount@CAreaProxy@@UAEHXZ 3207bf80 f i AreaProxy.obj
 0001:0007afa0       ?GetMemoryUsage@CAreaProxy@@UBEXPAVICrySizer@@@Z 3207bfa0 f i AreaProxy.obj
 0001:0007b060       ?_M_insert_aux@?$vector@_NV?$allocator@_N@stlpmtx_std@@@stlpmtx_std@@IAEXU?$_Bit_iter@U_Bit_reference@priv@stlpmtx_std@@PAU123@@priv@2@_N@Z 3207c060 f i AreaProxy.obj
 0001:0007b290       ?_M_fill_insert@?$vector@_NV?$allocator@_N@stlpmtx_std@@@stlpmtx_std@@QAEXU?$_Bit_iter@U_Bit_reference@priv@stlpmtx_std@@PAU123@@priv@2@I_N@Z 3207c290 f i AreaProxy.obj
 0001:0007b4f0       ?Format@?$CryStackStringT@D$0CAA@@@QAAAAV1@PBDZZ 3207c4f0 f i AreaProxy.obj
 0001:0007b560       ?ToLower@PathUtil@@YA?AV?$CryStringT@D@@ABV2@@Z 3207c560 f i AreaProxy.obj
 0001:0007b5c0       ?Open@CCryFile@@QAE_NPBD0H@Z 3207c5c0 f i AreaProxy.obj
 0001:0007b6e0       ??_GCAreaProxy@@UAEPAXI@Z  3207c6e0 f i AreaProxy.obj
 0001:0007b6e0       ??_ECAreaProxy@@UAEPAXI@Z  3207c6e0 f i AreaProxy.obj
 0001:0007b710       ?push_back@?$vector@_NV?$allocator@_N@stlpmtx_std@@@stlpmtx_std@@QAEX_N@Z 3207c710 f i AreaProxy.obj
 0001:0007b780       ??0CAreaProxy@@QAE@PAVCEntity@@@Z 3207c780 f   AreaProxy.obj
 0001:0007b970       ?resize@?$vector@_NV?$allocator@_N@stlpmtx_std@@@stlpmtx_std@@QAEXI_N@Z 3207c970 f i AreaProxy.obj
 0001:0007ba60       ?ResetTempState@CAreaProxy@@SAXXZ 3207ca60 f   AreaProxy.obj
 0001:0007bac0       ?SetSphere@CAreaProxy@@UAEXABU?$Vec3_tpl@M@@M@Z 3207cac0 f   AreaProxy.obj
 0001:0007bbf0       ?OnMove@CAreaProxy@@AAEXXZ 3207cbf0 f   AreaProxy.obj
 0001:0007bf30       ?OnEnable@CAreaProxy@@AAEX_N0@Z 3207cf30 f   AreaProxy.obj
 0001:0007c150       ?ProcessEvent@CAreaProxy@@UAEXAAUSEntityEvent@@@Z 3207d150 f   AreaProxy.obj
 0001:0007c310       ?SerializeXML@CAreaProxy@@UAEXAAVXmlNodeRef@@_N@Z 3207d310 f   AreaProxy.obj
 0001:0007d810       ?SetPoints@CAreaProxy@@UAEXQBU?$Vec3_tpl@M@@QB_NHM@Z 3207e810 f   AreaProxy.obj
 0001:0007d8e0       ?SetBox@CAreaProxy@@UAEXABU?$Vec3_tpl@M@@0QB_NI@Z 3207e8e0 f   AreaProxy.obj
 0001:0007da20       ?SetGravityVolume@CAreaProxy@@UAEXPBU?$Vec3_tpl@M@@HMM_NMM@Z 3207ea20 f   AreaProxy.obj
 0001:0007dad0       ?Release@CSoundProxy@@UAEXXZ 3207ead0 f   SoundProxy.obj
 0001:0007daf0       ?PrecacheHeadBone@CSoundProxy@@AAEXXZ 3207eaf0 f   SoundProxy.obj
 0001:0007db80       ?GetSignature@CEntityNodeProxy@@UAE_NV?$CSerializeWrapper@UISerialize@@@@@Z 3207eb80 f   Entity.obj
 0001:0007db80       ?GetSignature@CSoundProxy@@UAE_NV?$CSerializeWrapper@UISerialize@@@@@Z 3207eb80 f   SoundProxy.obj
 0001:0007db90       ?PlaySound@CSoundProxy@@UAEIPBDABU?$Vec3_tpl@M@@1IIW4ESoundSemantic@@@Z 3207eb90 f   SoundProxy.obj
 0001:0007dbe0       ?PlaySoundEx@CSoundProxy@@UAEIPBDABU?$Vec3_tpl@M@@1IIMMMW4ESoundSemantic@@@Z 3207ebe0 f   SoundProxy.obj
 0001:0007dc40       ?PlaySound@CSoundProxy@@UAEIPBDABU?$Vec3_tpl@M@@1IIW4ESoundSemantic@@PAIH@Z 3207ec40 f   SoundProxy.obj
 0001:0007dd90       ?PlaySoundEx@CSoundProxy@@UAEIPBDABU?$Vec3_tpl@M@@1IIMMMW4ESoundSemantic@@PAIH@Z 3207ed90 f   SoundProxy.obj
 0001:0007df40       ??$__copy@PAUSAttachedSound@CSoundProxy@@PAU12@H@priv@stlpmtx_std@@YAPAUSAttachedSound@CSoundProxy@@PAU23@00ABUrandom_access_iterator_tag@1@PAH@Z 3207ef40 f i SoundProxy.obj
 0001:0007dfe0       ?RayWorldIntersection@IPhysicalWorld@@QAEHABU?$Vec3_tpl@M@@0HIPAUray_hit@@HPAPAUIPhysicalEntity@@HPAXHPBDPAUray_hit_cached@@H@Z 3207efe0 f i SoundProxy.obj
 0001:0007e080       ?OnMoveInside@CSoundProxy@@AAEXPAUIEntity@@0@Z 3207f080 f   SoundProxy.obj
 0001:0007e190       ?OnExclusiveMoveInside@CSoundProxy@@AAEXPAUIEntity@@00@Z 3207f190 f   SoundProxy.obj
 0001:0007e400       ?OnEnter@CSoundProxy@@AAEXQBUIEntity@@QBUIListener@@@Z 3207f400 f   SoundProxy.obj
 0001:0007e600       ?OnLeave@CSoundProxy@@AAEXQBUIEntity@@QBUIListener@@@Z 3207f600 f   SoundProxy.obj
 0001:0007e770       ?OnAreaCrossing@CSoundProxy@@AAEXQBUIEntity@@QBUIListener@@@Z 3207f770 f   SoundProxy.obj
 0001:0007e8e0       ?OnMoveNear@CSoundProxy@@AAEXPAUIEntity@@0MM@Z 3207f8e0 f   SoundProxy.obj
 0001:0007eaf0       ?FindAttachedSound@CSoundProxy@@AAEQAUSAttachedSound@1@I@Z 3207faf0 f   SoundProxy.obj
 0001:0007eb20       ?SetStaticSound@CSoundProxy@@UAE_NI_N@Z 3207fb20 f   SoundProxy.obj
 0001:0007eb50       ?GetStaticSound@CSoundProxy@@UAE_NI@Z 3207fb50 f   SoundProxy.obj
 0001:0007eb80       ?PauseSound@CSoundProxy@@UAEXI_N@Z 3207fb80 f   SoundProxy.obj
 0001:0007ebc0       ?SetSoundPos@CSoundProxy@@UAEXIABU?$Vec3_tpl@M@@@Z 3207fbc0 f   SoundProxy.obj
 0001:0007ec70       ?GetSoundPos@CSoundProxy@@UAE?AU?$Vec3_tpl@M@@I@Z 3207fc70 f   SoundProxy.obj
 0001:0007ecc0       ?SetSoundDirection@CSoundProxy@@UAEXIABU?$Vec3_tpl@M@@@Z 3207fcc0 f   SoundProxy.obj
 0001:0007ed70       ?GetSoundDirection@CSoundProxy@@UAE?AU?$Vec3_tpl@M@@I@Z 3207fd70 f   SoundProxy.obj
 0001:0007edd0       ?CheckVisibilityForTailName@CSoundProxy@@UAEXMM@Z 3207fdd0 f   SoundProxy.obj
 0001:0007f0f0       ?SetSoundPosition@CSoundProxy@@AAEXQAUISound@@QIBU?$Vec3_tpl@M@@1ABU?$Matrix34_tpl@M@@@Z 320800f0 f   SoundProxy.obj
 0001:00080460       ?OnMove@CSoundProxy@@AAEXXZ 32081460 f   SoundProxy.obj
 0001:000804f0       ?OnHide@CSoundProxy@@AAEX_N@Z 320814f0 f   SoundProxy.obj
 0001:000805b0       ?ProcessEvent@CSoundProxy@@UAEXAAUSEntityEvent@@@Z 320815b0 f   SoundProxy.obj
 0001:00080af0       ?GetSound@CSoundProxy@@UAEQAUISound@@I@Z 32081af0 f   SoundProxy.obj
 0001:00080b80       ??$_Copy_Construct@USAttachedSound@CSoundProxy@@@stlpmtx_std@@YAXPAUSAttachedSound@CSoundProxy@@ABU12@@Z 32081b80 f i SoundProxy.obj
 0001:00080be0       ??$__ufill@PAUSAttachedSound@CSoundProxy@@U12@H@priv@stlpmtx_std@@YAXPAUSAttachedSound@CSoundProxy@@0ABU23@ABUrandom_access_iterator_tag@1@PAH@Z 32081be0 f i SoundProxy.obj
 0001:00080c70       ??$__ucopy@PAUSAttachedSound@CSoundProxy@@PAU12@H@priv@stlpmtx_std@@YAPAUSAttachedSound@CSoundProxy@@PAU23@00ABUrandom_access_iterator_tag@1@PAH@Z 32081c70 f i SoundProxy.obj
 0001:00080d10       ?UpdateSounds@CSoundProxy@@UAEXXZ 32081d10 f   SoundProxy.obj
 0001:00080d20       ?erase@?$vector@IV?$allocator@I@stlpmtx_std@@@stlpmtx_std@@QAEPAIPAI@Z 32081d20 f i SoundProxy.obj
 0001:00080d70       ??1?$_Impl_vector@USAttachedSound@CSoundProxy@@V?$allocator@USAttachedSound@CSoundProxy@@@stlpmtx_std@@@priv@stlpmtx_std@@QAE@XZ 32081d70 f i SoundProxy.obj
 0001:00080dc0       ?_M_insert_overflow_aux@?$_Impl_vector@USAttachedSound@CSoundProxy@@V?$allocator@USAttachedSound@CSoundProxy@@@stlpmtx_std@@@priv@stlpmtx_std@@AAEXPAUSAttachedSound@CSoundProxy@@ABU45@ABU__false_type@3@I_N@Z 32081dc0 f i SoundProxy.obj
 0001:00080f70       ?RemoveAttachedSound@CSoundProxy@@AAE_NI@Z 32081f70 f   SoundProxy.obj
 0001:00081080       ?OnSoundEvent@CSoundProxy@@UAEXW4ESoundCallbackEvent@@PAUISound@@@Z 32082080 f   SoundProxy.obj
 0001:00081260       ?StopSound@CSoundProxy@@UAEXIW4ESoundStopMode@@_N@Z 32082260 f   SoundProxy.obj
 0001:00081340       ?Reset@CSoundProxy@@AAEXXZ 32082340 f   SoundProxy.obj
 0001:000813d0       ?StopAllSounds@CSoundProxy@@UAEXXZ 320823d0 f   SoundProxy.obj
 0001:00081540       ??0CSoundProxy@@QAE@PAVCEntity@@@Z 32082540 f   SoundProxy.obj
 0001:000815c0       ?GetType@CSoundProxy@@UAE?AW4EEntityProxy@@XZ 320825c0 f i SoundProxy.obj
 0001:000815d0       ?RegisterContainer@CDummyMemReplay@@UAEXPBXH@Z 320825d0 f i AreaSolid.obj
 0001:000815d0       ?BindToContainer@CDummyMemReplay@@UAEXPBX0@Z 320825d0 f i AreaSolid.obj
 0001:000815d0       ?Start@CDummyMemReplay@@UAEX_NPBD@Z 320825d0 f i AreaSolid.obj
 0001:000815d0       ?UnMapPage@CDummyMemReplay@@UAEXPAXI@Z 320825d0 f i AreaSolid.obj
 0001:000815d0       ?AddAllocReference@CDummyMemReplay@@UAEXPAX0@Z 320825d0 f i AreaSolid.obj
 0001:000815d0       ?MapPage@CDummyMemReplay@@UAEXPAXI@Z 320825d0 f i AreaSolid.obj
 0001:000815d0       ?SerializeXML@CSoundProxy@@UAEXAAVXmlNodeRef@@_N@Z 320825d0 f i SoundProxy.obj
 0001:000815d0       ?UnMarkBucket@CDummyMemReplay@@UAEXHPAX@Z 320825d0 f i AreaSolid.obj
 0001:000815d0       ?RenderAttachment@IAttachmentObject@@UAEXAAUSRendParams@@ABUSRenderingPassInfo@@@Z 320825d0 f i Entity.obj
 0001:000815d0       ?OnRemoveAttachment@IAttachmentObject@@UAEXPAUIAttachmentManager@@H@Z 320825d0 f i Entity.obj
 0001:000815d0       ?UnbindFromContainer@CDummyMemReplay@@UAEXPBX0@Z 320825d0 f i AreaSolid.obj
 0001:000815d0       ?SerializeXML@CEntityNodeProxy@@UAEXAAVXmlNodeRef@@_N@Z 320825d0 f i Entity.obj
 0001:000815d0       ?SwapContainers@CDummyMemReplay@@UAEXPBX0@Z 320825d0 f i AreaSolid.obj
 0001:000815d0       ?GetMemoryUsage@CTypeInfo@@UBEXPAVICrySizer@@PBX@Z 320825d0 f i CryEntityDLL.obj
 0001:000815d0       ?BucketEnableCleanups@CDummyMemReplay@@UAEXPAX_N@Z 320825d0 f i AreaSolid.obj
 0001:000815d0       ?GetMemoryUsage@?$TTypeInfo@I@@UBEXPAVICrySizer@@PBX@Z 320825d0 f i CryEntityDLL.obj
 0001:000815d0       ?OnEntityEvent@IRenderNode@@UAEXPAUIEntity@@ABUSEntityEvent@@@Z 320825d0 f i RenderProxy.obj
 0001:000815d0       ?SerializeXML@CCameraProxy@@UAEXAAVXmlNodeRef@@_N@Z 320825d0 f i CameraProxy.obj
 0001:000815d0       ?GetMemoryUsage@?$TTypeInfo@H@@UBEXPAVICrySizer@@PBX@Z 320825d0 f i CryEntityDLL.obj
 0001:000815d0       ?UnMarkPool@CDummyMemReplay@@UAEXHPAX@Z 320825d0 f i AreaSolid.obj
 0001:000815d0       ?GetMemoryUsage@?$TTypeInfo@_K@@UBEXPAVICrySizer@@PBX@Z 320825d0 f i CryEntityDLL.obj
 0001:000815d0       ?GetMemoryUsage@?$TTypeInfo@M@@UBEXPAVICrySizer@@PBX@Z 320825d0 f i CryEntityDLL.obj
 0001:000815d0       ?SerializeXML@CTriggerProxy@@UAEXAAVXmlNodeRef@@_N@Z 320825d0 f i TriggerProxy.obj
 0001:000815d0       ?SerializeXML@CSubstitutionProxy@@UAEXAAVXmlNodeRef@@_N@Z 320825d0 f i Entity.obj
 0001:000815e0       ?SetFlags@CSoundProxy@@UAEXH@Z 320825e0 f i SoundProxy.obj
 0001:000815f0       ?GetFlags@CSoundProxy@@UBEHXZ 320825f0 f i SoundProxy.obj
 0001:00081600       ?SetEffectRadius@CSoundProxy@@UAEXM@Z 32082600 f i SoundProxy.obj
 0001:00081620       ?GetEffectRadius@CSoundProxy@@UAEMXZ 32082620 f i SoundProxy.obj
 0001:00081630       ??_ECSoundProxy@@W3AEPAXI@Z 32082630 f i SoundProxy.obj
 0001:00081640       ?GetMemoryUsage@CSoundProxy@@UBEXPAVICrySizer@@@Z 32082640 f i SoundProxy.obj
 0001:000816a0       ??1CSoundProxy@@UAE@XZ     320826a0 f i SoundProxy.obj
 0001:00081710       ??_GCSoundProxy@@UAEPAXI@Z 32082710 f i SoundProxy.obj
 0001:00081710       ??_ECSoundProxy@@UAEPAXI@Z 32082710 f i SoundProxy.obj
 0001:00081740       ?Reload@CSoundProxy@@UAEXPAUIEntity@@AAUSEntitySpawnParams@@@Z 32082740 f   SoundProxy.obj
 0001:00081770       ?AddAttachedSound@CSoundProxy@@AAE_NPAUISound@@_NABU?$Vec3_tpl@M@@2@Z 32082770 f   SoundProxy.obj
 0001:00081880       ?PlaySound@CSoundProxy@@UAE_NPAUISound@@ABU?$Vec3_tpl@M@@1M_N@Z 32082880 f   SoundProxy.obj
 0001:00081aa0       ?Done@CFlowGraphProxy@@UAEXXZ 32082aa0 f   FlowGraphProxy.obj
 0001:00081ac0       ?SetFlowGraph@CFlowGraphProxy@@UAEXPAUIFlowGraph@@@Z 32082ac0 f   FlowGraphProxy.obj
 0001:00081af0       ?NeedSerialize@CFlowGraphProxy@@UAE_NXZ 32082af0 f   FlowGraphProxy.obj
 0001:00081b00       ?SerializeXML@CFlowGraphProxy@@UAEXAAVXmlNodeRef@@_N@Z 32082b00 f   FlowGraphProxy.obj
 0001:00081d60       ?GetSignature@CFlowGraphProxy@@UAE_NV?$CSerializeWrapper@UISerialize@@@@@Z 32082d60 f   FlowGraphProxy.obj
 0001:00081d90       ?Serialize@CFlowGraphProxy@@UAEXV?$CSerializeWrapper@UISerialize@@@@@Z 32082d90 f   FlowGraphProxy.obj
 0001:00081e10       ?ProcessEvent@CFlowGraphProxy@@UAEXAAUSEntityEvent@@@Z 32082e10 f   FlowGraphProxy.obj
 0001:00081eb0       ?Reload@CFlowGraphProxy@@UAEXPAUIEntity@@AAUSEntitySpawnParams@@@Z 32082eb0 f   FlowGraphProxy.obj
 0001:00081f00       ?RemoveEventListener@CFlowGraphProxy@@UAEXPAUIEntityEventListener@@@Z 32082f00 f   FlowGraphProxy.obj
 0001:00081f50       ??0CFlowGraphProxy@@QAE@PAVCEntity@@@Z 32082f50 f   FlowGraphProxy.obj
 0001:00081f80       ?GetType@CFlowGraphProxy@@UAE?AW4EEntityProxy@@XZ 32082f80 f i FlowGraphProxy.obj
 0001:00081f90       ?GetMemoryUsage@CFlowGraphProxy@@UBEXPAVICrySizer@@@Z 32082f90 f i FlowGraphProxy.obj
 0001:00081fb0       ??_GCFlowGraphProxy@@UAEPAXI@Z 32082fb0 f i FlowGraphProxy.obj
 0001:00081fb0       ??_ECFlowGraphProxy@@UAEPAXI@Z 32082fb0 f i FlowGraphProxy.obj
 0001:00082000       ?AddEventListener@CFlowGraphProxy@@UAEXPAUIEntityEventListener@@@Z 32083000 f   FlowGraphProxy.obj
 0001:00082030       ?SetFlags@CEntityClass@@UAEXI@Z 32083030 f   EntityClass.obj
 0001:00082030       ?SetSubstitute@CSubstitutionProxy@@UAEXPAUIRenderNode@@@Z 32083030 f   SubstitutionProxy.obj
 0001:00082040       ?Reload@CSubstitutionProxy@@UAEXPAUIEntity@@AAUSEntitySpawnParams@@@Z 32083040 f   SubstitutionProxy.obj
 0001:00082050       ?NeedSerialize@CSubstitutionProxy@@UAE_NXZ 32083050 f   SubstitutionProxy.obj
 0001:00082060       ?Done@CSubstitutionProxy@@UAEXXZ 32083060 f   SubstitutionProxy.obj
 0001:000821c0       ?GetSignature@CSubstitutionProxy@@UAE_NV?$CSerializeWrapper@UISerialize@@@@@Z 320831c0 f   SubstitutionProxy.obj
 0001:000821f0       ?Serialize@CSubstitutionProxy@@UAEXV?$CSerializeWrapper@UISerialize@@@@@Z 320831f0 f   SubstitutionProxy.obj
 0001:000824e0       ?GetType@CTriggerProxy@@UAE?AW4EEntityProxy@@XZ 320834e0 f i TriggerProxy.obj
 0001:000824f0       ?GetTriggerBounds@CTriggerProxy@@UAEXAAUAABB@@@Z 320834f0 f i TriggerProxy.obj
 0001:00082520       ?ForwardEventsTo@CTriggerProxy@@UAEXI@Z 32083520 f i TriggerProxy.obj
 0001:00082530       ?GetMemoryUsage@CTriggerProxy@@UBEXPAVICrySizer@@@Z 32083530 f i TriggerProxy.obj
 0001:00082550       ?Reload@CTriggerProxy@@UAEXPAUIEntity@@AAUSEntitySpawnParams@@@Z 32083550 f   TriggerProxy.obj
 0001:000825c0       ?GetSignature@CTriggerProxy@@UAE_NV?$CSerializeWrapper@UISerialize@@@@@Z 320835c0 f   TriggerProxy.obj
 0001:000825f0       ??0CTriggerProxy@@QAE@PAVCEntity@@@Z 320835f0 f   TriggerProxy.obj
 0001:00082680       ??_GCTriggerProxy@@UAEPAXI@Z 32083680 f i TriggerProxy.obj
 0001:00082680       ??_ECTriggerProxy@@UAEPAXI@Z 32083680 f i TriggerProxy.obj
 0001:000826c0       ?OnMove@CTriggerProxy@@AAEX_N@Z 320836c0 f   TriggerProxy.obj
 0001:00082780       ?InvalidateTrigger@CTriggerProxy@@UAEXXZ 32083780 f   TriggerProxy.obj
 0001:00082790       ?SetTriggerBounds@CTriggerProxy@@UAEXABUAABB@@@Z 32083790 f i TriggerProxy.obj
 0001:000827d0       ?ProcessEvent@CTriggerProxy@@UAEXAAUSEntityEvent@@@Z 320837d0 f   TriggerProxy.obj
 0001:00082830       ?Serialize@CTriggerProxy@@UAEXV?$CSerializeWrapper@UISerialize@@@@@Z 32083830 f   TriggerProxy.obj
 0001:000828b0       ??4CCamera@@QAEAAV0@ABV0@@Z 320838b0 f i CameraProxy.obj
 0001:00082e90       ?GetSignature@CCameraProxy@@UAE_NV?$CSerializeWrapper@UISerialize@@@@@Z 32083e90 f   CameraProxy.obj
 0001:00082ec0       ?IsOrthonormalRH@?$Matrix34_tpl@M@@QBEHM@Z 32083ec0 f i CameraProxy.obj
 0001:00083100       ?UpdateFrustum@CCamera@@QAEXXZ 32084100 f i CameraProxy.obj
 0001:00084a00       ?UpdateMaterialCamera@CCameraProxy@@QAEXXZ 32085a00 f   CameraProxy.obj
 0001:00084c40       ?SetCamera@CCameraProxy@@UAEXAAVCCamera@@@Z 32085c40 f   CameraProxy.obj
 0001:00084c60       ??0CCamera@@QAE@XZ         32085c60 f i CameraProxy.obj
 0001:00084de0       ??0CCameraProxy@@QAE@PAVCEntity@@@Z 32085de0 f   CameraProxy.obj
 0001:00084e10       ?GetType@CCameraProxy@@UAE?AW4EEntityProxy@@XZ 32085e10 f i CameraProxy.obj
 0001:00084e20       ?GetCamera@CCameraProxy@@UAEAAVCCamera@@XZ 32085e20 f i CameraProxy.obj
 0001:00084e30       ?GetMemoryUsage@CCameraProxy@@UBEXPAVICrySizer@@@Z 32085e30 f i CameraProxy.obj
 0001:00084e50       ?Init@CCameraProxy@@UAE_NPAUIEntity@@AAUSEntitySpawnParams@@@Z 32085e50 f   CameraProxy.obj
 0001:00084e60       ?Reload@CCameraProxy@@UAEXPAUIEntity@@AAUSEntitySpawnParams@@@Z 32085e60 f   CameraProxy.obj
 0001:00084e70       ?ProcessEvent@CCameraProxy@@UAEXAAUSEntityEvent@@@Z 32085e70 f   CameraProxy.obj
 0001:00084e90       ??0SMFXRunTimeEffectParams@@QAE@XZ 32085e90 f i EntityNodeProxy.obj
 0001:00084fd0       ?ProcessEvent@CEntityNodeProxy@@UAEXAAUSEntityEvent@@@Z 32085fd0 f   EntityNodeProxy.obj
 0001:00085460       ?GetScriptTable@CEntityClass@@UBEPAUIScriptTable@@XZ 32086460 f   EntityClass.obj
 0001:00085470       ?LoadScript@CEntityClass@@UAE_N_N@Z 32086470 f   EntityClass.obj
 0001:000854a0       ?SetEntityScript@CEntityClass@@QAEXPAUIEntityScript@@@Z 320864a0 f   EntityClass.obj
 0001:000854b0       ?SetUserProxyCreateFunc@CEntityClass@@QAEXP6APAUIEntityProxy@@PAUIEntity@@AAUSEntitySpawnParams@@PAX@Z2@Z 320864b0 f   EntityClass.obj
 0001:000854d0       ??_GIEntityClass@@UAEPAXI@Z 320864d0 f i EntityClass.obj
 0001:000854d0       ??_EIEntityClass@@UAEPAXI@Z 320864d0 f i EntityClass.obj
 0001:00085500       ?FindEventInfo@CEntityClass@@UAE_NPBDAAUSEventInfo@IEntityClass@@@Z 32086500 f   EntityClass.obj
 0001:00085550       ?GetEditorIconName@CEntityClass@@UBEPBDXZ 32086550 f   EntityClass.obj
 0001:00085560       ?GetEventCount@CEntityClass@@UAEHXZ 32086560 f   EntityClass.obj
 0001:00085590       ??0CEntityClass@@QAE@XZ    32086590 f   EntityClass.obj
 0001:000855c0       ?GetIStatObj@CCGFAttachment@@UBEPAUIStatObj@@XZ 320865c0 f i ScriptBind_Entity.obj
 0001:000855c0       ?GetICharacterInstance@CSKELAttachment@@UBEPAUICharacterInstance@@XZ 320865c0 f i ScriptBind_Entity.obj
 0001:000855c0       ?GetFlags@CEntityClass@@UBEIXZ 320865c0 f i EntityClass.obj
 0001:000855c0       ?GetSubstitute@CSubstitutionProxy@@UAEPAUIRenderNode@@XZ 320865c0 f i Entity.obj
 0001:000855d0       ?GetIEntityScript@CEntityClass@@UBEPAUIEntityScript@@XZ 320865d0 f i EntityClass.obj
 0001:000855d0       ?GetProperties@CEntityArchetype@@UAEPAUIScriptTable@@XZ 320865d0 f i EntityArchetype.obj
 0001:000855e0       ?GetMemoryUsage@CEntityClass@@UBEXPAVICrySizer@@@Z 320865e0 f i EntityClass.obj
 0001:00085650       ??1CEntityClass@@UAE@XZ    32086650 f   EntityClass.obj
 0001:00085730       ?GetEventInfo@CEntityClass@@UAE?AUSEventInfo@IEntityClass@@H@Z 32086730 f   EntityClass.obj
 0001:00085780       ??_GCEntityClass@@UAEPAXI@Z 32086780 f i EntityClass.obj
 0001:00085780       ??_ECEntityClass@@UAEPAXI@Z 32086780 f i EntityClass.obj
 0001:000857b0       ?SetName@CEntityClass@@QAEXPBD@Z 320867b0 f   EntityClass.obj
 0001:000857f0       ?SetScriptFile@CEntityClass@@QAEXPBD@Z 320867f0 f   EntityClass.obj
 0001:00085830       ?GetClass@CEntity@@UBEPAUIEntityClass@@XZ 32086830 f   Entity.obj
 0001:00085830       ?GetDefaultClass@CEntityClassRegistry@@UBEPAUIEntityClass@@XZ 32086830 f   EntityClassRegistry.obj
 0001:00085840       ??_GIEntityClassRegistry@@UAEPAXI@Z 32086840 f i EntityClassRegistry.obj
 0001:00085840       ??_EIEntityClassRegistry@@UAEPAXI@Z 32086840 f i EntityClassRegistry.obj
 0001:00085840       ??_EIAreaManager@@UAEPAXI@Z 32086840 f i AreaManager.obj
 0001:00085840       ??_GIAreaManager@@UAEPAXI@Z 32086840 f i AreaManager.obj
 0001:00085870       ?RegisterStdClass@CEntityClassRegistry@@UAEPAUIEntityClass@@ABUSEntityClassDesc@IEntityClassRegistry@@@Z 32086870 f   EntityClassRegistry.obj
 0001:00085960       ?InitializeDefaultClasses@CEntityClassRegistry@@QAEXXZ 32086960 f   EntityClassRegistry.obj
 0001:00085a10       ?LoadClassDescription@CEntityClassRegistry@@AAEXAAVXmlNodeRef@@_N@Z 32086a10 f   EntityClassRegistry.obj
 0001:00085ae0       ?TrimRight@?$CryStringT@D@@QAEAAV1@PBD@Z 32086ae0 f i EntityClassRegistry.obj
 0001:00085b50       ?IteratorMoveFirst@CEntityClassRegistry@@UAEXXZ 32086b50 f   EntityClassRegistry.obj
 0001:00085b60       ?IteratorNext@CEntityClassRegistry@@UAEPAUIEntityClass@@XZ 32086b60 f   EntityClassRegistry.obj
 0001:00085bb0       ?FindClass@CEntityClassRegistry@@UBEPAUIEntityClass@@PBD@Z 32086bb0 f   EntityClassRegistry.obj
 0001:00085c20       ?LoadClasses@CEntityClassRegistry@@UAEXPBD_N@Z 32086c20 f   EntityClassRegistry.obj
 0001:00085df0       ?erase@?$_Rb_tree@V?$CryStringT@D@@U?$less@V?$CryStringT@D@@@stlpmtx_std@@U?$pair@$$CBV?$CryStringT@D@@PAUIEntityClass@@@3@U?$_Select1st@U?$pair@$$CBV?$CryStringT@D@@PAUIEntityClass@@@stlpmtx_std@@@priv@3@U?$_MapTraitsT@U?$pair@$$CBV?$CryStringT@D@@PAUIEntityClass@@@stlpmtx_std@@@63@V?$allocator@U?$pair@$$CBV?$CryStringT@D@@PAUIEntityClass@@@stlpmtx_std@@@3@@priv@stlpmtx_std@@QAEXU?$_Rb_tree_iterator@U?$pair@$$CBV?$CryStringT@D@@PAUIEntityClass@@@stlpmtx_std@@U?$_MapTraitsT@U?$pair@$$CBV?$CryStringT@D@@PAUIEntityClass@@@stlpmtx_std@@@priv@2@@23@@Z 32086df0 f i EntityClassRegistry.obj
 0001:00085e60       ?GetClass@CEntityArchetype@@UBEPAUIEntityClass@@XZ 32086e60 f i EntityArchetype.obj
 0001:00085e60       ?GetUserProxyCreateFunc@CEntityClass@@UBEP6APAUIEntityProxy@@PAUIEntity@@AAUSEntitySpawnParams@@PAX@ZXZ 32086e60 f i EntityClass.obj
 0001:00085e60       ?GetPartId0@CPhysicalProxy@@UAEHXZ 32086e60 f i PhysicsProxy.obj
 0001:00085e60       ?GetClassCount@CEntityClassRegistry@@UBEHXZ 32086e60 f i EntityClassRegistry.obj
 0001:00085e60       ?GetTailName@CSoundProxy@@UAEPBDXZ 32086e60 f i SoundProxy.obj
 0001:00085e70       ?UnregisterClass@CEntityClassRegistry@@UAE_NPAUIEntityClass@@@Z 32086e70 f   EntityClassRegistry.obj
 0001:00085f10       ??0CEntityClassRegistry@@QAE@XZ 32086f10 f   EntityClassRegistry.obj
 0001:00085f70       ??_GCEntityClassRegistry@@UAEPAXI@Z 32086f70 f i EntityClassRegistry.obj
 0001:00085f70       ??_ECEntityClassRegistry@@UAEPAXI@Z 32086f70 f i EntityClassRegistry.obj
 0001:00085fe0       ?RegisterClass@CEntityClassRegistry@@UAE_NPAUIEntityClass@@@Z 32086fe0 f   EntityClassRegistry.obj
 0001:00086050       ?ReserveEntityIds@CEntityLoadManager@@AAE_NAAVXmlNodeRef@@@Z 32087050 f   EntityLoadManager.obj
 0001:00086100       ?CanParseEntity@CEntityLoadManager@@AAE_NAAVXmlNodeRef@@@Z 32087100 f   EntityLoadManager.obj
 0001:000861d0       ??0SEntityAttachment@@QAE@XZ 320871d0 f i EntityLoadManager.obj
 0001:00086300       ?allocate@?$_STLP_alloc_proxy@PAUSEntityAttachment@@U1@V?$allocator@USEntityAttachment@@@stlpmtx_std@@@priv@stlpmtx_std@@QAEPAUSEntityAttachment@@IAAI@Z 32087300 f i EntityLoadManager.obj
 0001:00086360       ?allocate@?$_STLP_alloc_proxy@PAUListenerRecord@?$CListenerSet@PAUIEntityPoolListener@@@@U12@V?$allocator@UListenerRecord@?$CListenerSet@PAUIEntityPoolListener@@@@@stlpmtx_std@@@priv@stlpmtx_std@@QAEPAUListenerRecord@?$CListenerSet@PAUIEntityPoolListener@@@@IAAI@Z 32087360 f i EntityPoolManager.obj
 0001:00086360       ?allocate@?$_STLP_alloc_proxy@PAUSQueuedFlowGraph@CEntityLoadManager@@U12@V?$allocator@USQueuedFlowGraph@CEntityLoadManager@@@stlpmtx_std@@@priv@stlpmtx_std@@QAEPAUSQueuedFlowGraph@CEntityLoadManager@@IAAI@Z 32087360 f i EntityLoadManager.obj
 0001:00086360       ?allocate@?$_STLP_alloc_proxy@PAUSEntityIds@CEntityPool@@U12@V?$allocator@USEntityIds@CEntityPool@@@stlpmtx_std@@@priv@stlpmtx_std@@QAEPAUSEntityIds@CEntityPool@@IAAI@Z 32087360 f i EntityPool.obj
 0001:00086360       ?allocate@?$_STLP_alloc_proxy@PAUSReturnToPoolWeight@CEntityPool@@U12@V?$allocator@USReturnToPoolWeight@CEntityPool@@@stlpmtx_std@@@priv@stlpmtx_std@@QAEPAUSReturnToPoolWeight@CEntityPool@@IAAI@Z 32087360 f i EntityPool.obj
 0001:000863b0       ?ExtractEntityLoadParams@CEntityLoadManager@@ABE_NAAVXmlNodeRef@@AAUSEntityLoadParams@@@Z 320873b0 f   EntityLoadManager.obj
 0001:000866d0       ??$__ucopy@PAUSQueuedFlowGraph@CEntityLoadManager@@PAU12@H@priv@stlpmtx_std@@YAPAUSQueuedFlowGraph@CEntityLoadManager@@PAU23@00ABUrandom_access_iterator_tag@1@PAH@Z 320876d0 f i EntityLoadManager.obj
 0001:00086720       ??$_Copy_Construct@USEntityAttachment@@@stlpmtx_std@@YAXPAUSEntityAttachment@@ABU1@@Z 32087720 f i EntityLoadManager.obj
 0001:00086780       ??$__uninitialized_fill_n@PAUSQueuedFlowGraph@CEntityLoadManager@@IU12@@priv@stlpmtx_std@@YAPAUSQueuedFlowGraph@CEntityLoadManager@@PAU23@IABU23@@Z 32087780 f i EntityLoadManager.obj
 0001:000867d0       ??$__ufill@PAUSEntityAttachment@@U1@H@priv@stlpmtx_std@@YAXPAUSEntityAttachment@@0ABU2@ABUrandom_access_iterator_tag@1@PAH@Z 320877d0 f i EntityLoadManager.obj
 0001:00086860       ??$__ucopy@PBUSEntityAttachment@@PAU1@H@priv@stlpmtx_std@@YAPAUSEntityAttachment@@PBU2@0PAU2@ABUrandom_access_iterator_tag@1@PAH@Z 32087860 f i EntityPoolManager.obj
 0001:00086860       ??$__ucopy@PAUSEntityAttachment@@PAU1@H@priv@stlpmtx_std@@YAPAUSEntityAttachment@@PAU2@00ABUrandom_access_iterator_tag@1@PAH@Z 32087860 f i EntityLoadManager.obj
 0001:000868f0       ?_M_clear@?$_Impl_vector@USQueuedFlowGraph@CEntityLoadManager@@V?$allocator@USQueuedFlowGraph@CEntityLoadManager@@@stlpmtx_std@@@priv@stlpmtx_std@@AAEXXZ 320878f0 f i EntityLoadManager.obj
 0001:00086930       ??1?$_Impl_vector@USQueuedFlowGraph@CEntityLoadManager@@V?$allocator@USQueuedFlowGraph@CEntityLoadManager@@@stlpmtx_std@@@priv@stlpmtx_std@@QAE@XZ 32087930 f i EntityLoadManager.obj
 0001:00086980       ?_M_insert_overflow_aux@?$_Impl_vector@USQueuedFlowGraph@CEntityLoadManager@@V?$allocator@USQueuedFlowGraph@CEntityLoadManager@@@stlpmtx_std@@@priv@stlpmtx_std@@AAEXPAUSQueuedFlowGraph@CEntityLoadManager@@ABU45@ABU__false_type@3@I_N@Z 32087980 f i EntityLoadManager.obj
 0001:00086b20       ??$_M_allocate_and_copy@PAUSQueuedFlowGraph@CEntityLoadManager@@@?$_Impl_vector@USQueuedFlowGraph@CEntityLoadManager@@V?$allocator@USQueuedFlowGraph@CEntityLoadManager@@@stlpmtx_std@@@priv@stlpmtx_std@@AAEPAUSQueuedFlowGraph@CEntityLoadManager@@AAIPAU34@1@Z 32087b20 f i EntityLoadManager.obj
 0001:00086b90       ??1CEntityLoadManager@@QAE@XZ 32087b90 f   EntityLoadManager.obj
 0001:00086bc0       ?_M_insert_overflow_aux@?$_Impl_vector@USEntityAttachment@@V?$allocator@USEntityAttachment@@@stlpmtx_std@@@priv@stlpmtx_std@@AAEXPAUSEntityAttachment@@ABU4@ABU__false_type@3@I_N@Z 32087bc0 f i EntityLoadManager.obj
 0001:00086d50       ?reserve@?$_Impl_vector@USQueuedFlowGraph@CEntityLoadManager@@V?$allocator@USQueuedFlowGraph@CEntityLoadManager@@@stlpmtx_std@@@priv@stlpmtx_std@@QAEXI@Z 32087d50 f i EntityLoadManager.obj
 0001:00086dd0       ??$_M_allocate_and_copy@PAUSEntityAttachment@@@?$_Impl_vector@USEntityAttachment@@V?$allocator@USEntityAttachment@@@stlpmtx_std@@@priv@stlpmtx_std@@AAEPAUSEntityAttachment@@AAIPAU3@1@Z 32087dd0 f i EntityLoadManager.obj
 0001:00086e40       ??0CEntityLoadManager@@QAE@PAVCEntitySystem@@@Z 32087e40 f   EntityLoadManager.obj
 0001:00086ea0       ?push_back@?$_Impl_vector@USQueuedFlowGraph@CEntityLoadManager@@V?$allocator@USQueuedFlowGraph@CEntityLoadManager@@@stlpmtx_std@@@priv@stlpmtx_std@@QAEXABUSQueuedFlowGraph@CEntityLoadManager@@@Z 32087ea0 f i EntityLoadManager.obj
 0001:00086f10       ?reserve@?$_Impl_vector@USEntityAttachment@@V?$allocator@USEntityAttachment@@@stlpmtx_std@@@priv@stlpmtx_std@@QAEXI@Z 32087f10 f i EntityLoadManager.obj
 0001:00086fc0       ?PrepareBatchCreation@CEntityLoadManager@@QAEXH@Z 32087fc0 f   EntityLoadManager.obj
 0001:00086fe0       ?OnBatchCreationCompleted@CEntityLoadManager@@QAEXXZ 32087fe0 f   EntityLoadManager.obj
 0001:00087430       ?push_back@?$vector@USEntityAttachment@@V?$allocator@USEntityAttachment@@@stlpmtx_std@@@stlpmtx_std@@QAEXABUSEntityAttachment@@@Z 32088430 f i EntityLoadManager.obj
 0001:00087490       ?AddQueuedAttachment@CEntityLoadManager@@AAEXIIABU?$Vec3_tpl@M@@ABU?$Quat_tpl@M@@0@Z 32088490 f   EntityLoadManager.obj
 0001:00087560       ?CreateEntity@CEntityLoadManager@@QAE_NAAUSEntityLoadParams@@AAI@Z 32088560 f   EntityLoadManager.obj
 0001:00087bb0       ?ParseEntities@CEntityLoadManager@@AAE_NAAVXmlNodeRef@@@Z 32088bb0 f   EntityLoadManager.obj
 0001:00087ef0       ?LoadEntities@CEntityLoadManager@@QAE_NAAVXmlNodeRef@@@Z 32088ef0 f   EntityLoadManager.obj
 0001:00087f50       ?PointOutBBox2D@a2DBBox@CArea@@QBE_NABUa2DPoint@2@@Z 32088f50 f i Area.obj
 0001:00087f90       ?PointOutBBox2DVertical@a2DBBox@CArea@@QBE_NABUa2DPoint@2@@Z 32088f90 f i Area.obj
 0001:00087fd0       ?IntersectsXPosVertical@a2DSegment@CArea@@QBE_NABUa2DPoint@2@@Z 32088fd0 f i Area.obj
 0001:00088010       ?SetAreaType@CArea@@QAEXW4EEntityAreaType@@@Z 32089010 f   Area.obj
 0001:00088030       ?AddConvexHullToSolid@CArea@@QAEXPBU?$Vec3_tpl@M@@_NH@Z 32089030 f   Area.obj
 0001:00088060       ?EndSettingSolid@CArea@@QAEXXZ 32089060 f   Area.obj
 0001:00088090       ?GetSolidBoundBox@CArea@@QBEXAAUAABB@@@Z 32089090 f   Area.obj
 0001:000880d0       ?_M_allocate@?$allocator@USEntityEvent@@@stlpmtx_std@@QAEPAUSEntityEvent@@IAAI@Z 320890d0 f i Area.obj
 0001:00088140       ??_EIArea@@UAEPAXI@Z       32089140 f i Area.obj
 0001:00088140       ??_GIEntityArchetype@@UAEPAXI@Z 32089140 f i EntityArchetype.obj
 0001:00088140       ??_EIEntityArchetype@@UAEPAXI@Z 32089140 f i EntityArchetype.obj
 0001:00088140       ??_GIArea@@UAEPAXI@Z       32089140 f i Area.obj
 0001:00088170       ?GetStart@a2DSegment@CArea@@QBE?BUa2DPoint@2@XZ 32089170 f i Area.obj
 0001:000881b0       ?GetEnd@a2DSegment@CArea@@QBE?BUa2DPoint@2@XZ 320891b0 f i Area.obj
 0001:000881f0       ?CalcClosestPointToObstructedBox@CArea@@ABEXAAU?$Vec3_tpl@M@@AAMABU2@@Z 320891f0 f   Area.obj
 0001:00089000       ?CalcClosestPointToSolid@CArea@@ABEXABU?$Vec3_tpl@M@@_NAAMPAU2@@Z 3208a000 f   Area.obj
 0001:000891c0       ?InvalidateCachedAreaData@CArea@@QAEXXZ 3208a1c0 f   Area.obj
 0001:00089210       ?GetMatrix@CArea@@QBEXAAU?$Matrix34_tpl@M@@@Z 3208a210 f   Area.obj
 0001:00089270       ?GetBBox@CArea@@QBEXAAU?$Vec2_tpl@M@@0@Z 3208a270 f   Area.obj
 0001:000892b0       ?SetMatrix@CArea@@QAEXABU?$Matrix34_tpl@M@@@Z 3208a2b0 f   Area.obj
 0001:000896d0       ?OnAreaCrossing@CArea@@QAEXQIBUIEntity@@@Z 3208a6d0 f   Area.obj
 0001:00089770       ?SetSoundObstructionOnAreaFace@CArea@@QAEXI_N@Z 3208a770 f   Area.obj
 0001:00089890       ?CalcPointWithin@CArea@@QAE_NABU?$Vec3_tpl@M@@_N_N@Z 3208a890 f   Area.obj
 0001:00089d20       ?CalcCachedPointPosType@CArea@@QAE?BW4EAreaPosType@@ABU?$Vec3_tpl@M@@_N@Z 3208ad20 f   Area.obj
 0001:00089fc0       ?CalcBBox@CArea@@AAEXXZ    3208afc0 f   Area.obj
 0001:0008a0b0       ?GetMaximumEffectRadius@CArea@@QAEMXZ 3208b0b0 f   Area.obj
 0001:0008a150       ?ExclusiveUpdateAreaInside@CArea@@QAEXQIBUIEntity@@IM@Z 3208b150 f   Area.obj
 0001:0008a240       ?ExclusiveUpdateAreaNear@CArea@@QAEXQIBUIEntity@@IM@Z 3208b240 f   Area.obj
 0001:0008a330       ?Draw@CArea@@QAEXH@Z       3208b330 f   Area.obj
 0001:0008ad90       ?_M_insert_overflow@?$_Impl_vector@USEntityEvent@@V?$allocator@USEntityEvent@@@stlpmtx_std@@@priv@stlpmtx_std@@AAEXPAUSEntityEvent@@ABU4@ABU__true_type@3@I_N@Z 3208bd90 f i Area.obj
 0001:0008aee0       ?ClosestPointOnHullDistSq@CArea@@QAE?BMABU?$Vec3_tpl@M@@AAU2@_N2@Z 3208bee0 f   Area.obj
 0001:0008cba0       ?CalcPointNearDistSq@CArea@@QAEMABU?$Vec3_tpl@M@@AAU2@_N2@Z 3208dba0 f   Area.obj
 0001:0008e900       ?CalcPointNearDistSq@CArea@@QAEMABU?$Vec3_tpl@M@@_N_N2@Z 3208f900 f   Area.obj
 0001:0008fe90       ?CalcPointWithinDist@CArea@@QAEMABU?$Vec3_tpl@M@@_N1@Z 32090e90 f   Area.obj
 0001:00090c00       ?ClearCachedEventsFor@CArea@@QAEXI@Z 32091c00 f   Area.obj
 0001:00090ce0       ?SendCachedEventsFor@CArea@@QAEXI@Z 32091ce0 f   Area.obj
 0001:00090ee0       ?EnterArea@CArea@@QAEXQIBUIEntity@@@Z 32091ee0 f   Area.obj
 0001:00090ff0       ?LeaveArea@CArea@@QAEXQIBUIEntity@@@Z 32091ff0 f   Area.obj
 0001:000910f0       ?EnterNearArea@CArea@@QAEXQIBUIEntity@@M@Z 320920f0 f   Area.obj
 0001:000911d0       ?LeaveNearArea@CArea@@QAEXQIBUIEntity@@@Z 320921d0 f   Area.obj
 0001:000912b0       ??0CArea@@QAE@PAVCAreaManager@@@Z 320922b0 f   Area.obj
 0001:00091510       ?GetMinMax@CArea@@UBEXPAPAU?$Vec3_tpl@M@@0@Z 32092510 f i Area.obj
 0001:00091570       ?GetPriority@CArea@@UBEHXZ 32092570 f i Area.obj
 0001:00091580       ?GetEntityAmount@CArea@@UBEHXZ 32092580 f i Area.obj
 0001:00091590       ?GetEntityByIdx@CArea@@UBE?BIH@Z 32092590 f i Area.obj
 0001:000915a0       ?AddSegment@CArea@@AAEXABUa2DPoint@1@0_N@Z 320925a0 f   Area.obj
 0001:00091710       ?AddCachedEvent@CArea@@QAEXABUSEntityEvent@@@Z 32092710 f   Area.obj
 0001:00091770       ?ClearPoints@CArea@@AAEXXZ 32092770 f   Area.obj
 0001:00091860       ?AddEntity@CArea@@QAEXI@Z  32092860 f   Area.obj
 0001:000918d0       ?ClearEntities@CArea@@QAEXXZ 320928d0 f   Area.obj
 0001:00091a20       ?ClearCachedEvents@CArea@@QAEXXZ 32092a20 f   Area.obj
 0001:00091a70       ?ReleaseAreaData@CArea@@AAEXXZ 32092a70 f   Area.obj
 0001:00091ad0       ??1CArea@@EAE@XZ           32092ad0 f   Area.obj
 0001:00091b70       ?SetPoints@CArea@@QAEXQBU?$Vec3_tpl@M@@QB_NH@Z 32092b70 f   Area.obj
 0001:00091ca0       ?SetBox@CArea@@QAEXABU?$Vec3_tpl@M@@0ABU?$Matrix34_tpl@M@@@Z 32092ca0 f   Area.obj
 0001:000920e0       ?BeginSettingSolid@CArea@@QAEXABU?$Matrix34_tpl@M@@@Z 320930e0 f   Area.obj
 0001:00092540       ?SetSphere@CArea@@QAEXABU?$Vec3_tpl@M@@M@Z 32093540 f   Area.obj
 0001:000925b0       ??_ECArea@@EAEPAXI@Z       320935b0 f i Area.obj
 0001:000925b0       ??_GCArea@@EAEPAXI@Z       320935b0 f i Area.obj
 0001:000925e0       ?GetAreas@CAreaBitField@@SAPAIAAV1@0AAI@Z 320935e0 f   AreaGrid.obj
 0001:00092690       ?AllocateMem@CAreaBitField@@SAXXZ 32093690 f   AreaGrid.obj
 0001:00092710       ??0CAreaGrid@@QAE@XZ       32093710 f   AreaGrid.obj
 0001:00092730       ?GetAreas@CAreaGrid@@QAEPAIABU?$Vec3_tpl@M@@AAI@Z 32093730 f   AreaGrid.obj
 0001:000927c0       ?Reset@CAreaGrid@@QAEXXZ   320937c0 f   AreaGrid.obj
 0001:00092850       ?Draw@CAreaGrid@@QAEXXZ    32093850 f   AreaGrid.obj
 0001:000928f0       ?GetMaximumEffectRadius@CAreaGrid@@IAEMPAVCArea@@@Z 320938f0 f   AreaGrid.obj
 0001:00092980       ?Compile@CAreaGrid@@QAEXPAVCEntitySystem@@AAV?$vector@PAVCArea@@V?$allocator@PAVCArea@@@stlpmtx_std@@@stlpmtx_std@@@Z 32093980 f   AreaGrid.obj
 0001:000931a0       ?DrawGrid@CAreaManager@@QAEXXZ 320941a0 f   AreaManager.obj
 0001:000931b0       ?SetAreasDirty@CAreaManager@@UAEXXZ 320941b0 f   AreaManager.obj
 0001:000931c0       ?GetArea@CAreaManager@@UBEPBUIArea@@H@Z 320941c0 f   AreaManager.obj
 0001:000931d0       ?GetLinkedAreas@CAreaManager@@UBE_NIPAIAAH@Z 320941d0 f   AreaManager.obj
 0001:00093280       ?QueryAreas@CAreaManager@@UAE_NABU?$Vec3_tpl@M@@PAUSAreaManagerResult@@H_N@Z 32094280 f   AreaManager.obj
 0001:00093430       ?NotifyAreas@CAreaManager@@QAEXQBUSAreasCache@1@IQBUIEntity@@@Z 32094430 f   AreaManager.obj
 0001:000934a0       ?OnEvent@CAreaManager@@QAEXW4EEntityEvent@@IPAUIArea@@@Z 320944a0 f   AreaManager.obj
 0001:000934e0       ?GetNumberOfPlayersInArea@CAreaManager@@QBEHPBVCArea@@@Z 320944e0 f   AreaManager.obj
 0001:000935b0       ??$find_and_erase@V?$vector@PAUIAreaManagerEventListener@@V?$allocator@PAUIAreaManagerEventListener@@@stlpmtx_std@@@stlpmtx_std@@PAUIAreaManagerEventListener@@@stl@@YA_NAAV?$vector@PAUIAreaManagerEventListener@@V?$allocator@PAUIAreaManagerEventListener@@@stlpmtx_std@@@stlpmtx_std@@ABQAUIAreaManagerEventListener@@@Z 320945b0 f i AreaManager.obj
 0001:000935b0       ??$find_and_erase@V?$vector@PAUSProximityElement@@V?$allocator@PAUSProximityElement@@@stlpmtx_std@@@stlpmtx_std@@PAUSProximityElement@@@stl@@YA_NAAV?$vector@PAUSProximityElement@@V?$allocator@PAUSProximityElement@@@stlpmtx_std@@@stlpmtx_std@@ABQAUSProximityElement@@@Z 320945b0 f i ProximityTriggerSystem.obj
 0001:000935b0       ??$find_and_erase@V?$vector@PAVCEntity@@V?$allocator@PAVCEntity@@@stlpmtx_std@@@stlpmtx_std@@PAVCEntity@@@stl@@YA_NAAV?$vector@PAVCEntity@@V?$allocator@PAVCEntity@@@stlpmtx_std@@@stlpmtx_std@@ABQAVCEntity@@@Z 320945b0 f i Entity.obj
 0001:00093620       ?RemoveEventListener@CAreaManager@@UAEXPAUIAreaManagerEventListener@@@Z 32094620 f   AreaManager.obj
 0001:00093640       ?CreateArea@CAreaManager@@QAEPAVCArea@@XZ 32094640 f   AreaManager.obj
 0001:000936c0       ?GetLinkedAreas@CAreaManager@@QBEHIHAAV?$vector@PAVCArea@@V?$allocator@PAVCArea@@@stlpmtx_std@@@stlpmtx_std@@@Z 320946c0 f   AreaManager.obj
 0001:000937b0       ?MarkPlayerForUpdate@CAreaManager@@QAEXI@Z 320947b0 f   AreaManager.obj
 0001:000938a0       ?AddEventListener@CAreaManager@@UAEXPAUIAreaManagerEventListener@@@Z 320948a0 f   AreaManager.obj
 0001:000938c0       ?DrawLinkedAreas@CAreaManager@@UBEXI@Z 320948c0 f   AreaManager.obj
 0001:000939a0       ?ProceedExclusiveUpdateByHigherArea@CAreaManager@@QAE_NQBUSAreasCache@1@QBUIEntity@@IQAVCArea@@ABU?$Vec3_tpl@M@@@Z 320949a0 f   AreaManager.obj
 0001:00093dd0       ??0SAreasCache@CAreaManager@@QAE@ABU01@@Z 32094dd0 f i AreaManager.obj
 0001:00093e50       ?ProcessArea@CAreaManager@@AAEXQIAVCArea@@IHQAUSAreasCache@1@ABU?$Vec3_tpl@M@@QBUIEntity@@@Z 32094e50 f   AreaManager.obj
 0001:00094150       ?DrawAreas@CAreaManager@@QAEXQBUISystem@@@Z 32095150 f   AreaManager.obj
 0001:000946e0       ?_M_erase@?$_Rb_tree@PAUIEntityClass@@U?$less@PAUIEntityClass@@@stlpmtx_std@@U?$pair@QAUIEntityClass@@V?$vector@U?$pair@II@stlpmtx_std@@V?$allocator@U?$pair@II@stlpmtx_std@@@2@@stlpmtx_std@@@3@U?$_Select1st@U?$pair@QAUIEntityClass@@V?$vector@U?$pair@II@stlpmtx_std@@V?$allocator@U?$pair@II@stlpmtx_std@@@2@@stlpmtx_std@@@stlpmtx_std@@@priv@3@U?$_MapTraitsT@U?$pair@QAUIEntityClass@@V?$vector@U?$pair@II@stlpmtx_std@@V?$allocator@U?$pair@II@stlpmtx_std@@@2@@stlpmtx_std@@@stlpmtx_std@@@63@V?$allocator@U?$pair@QAUIEntityClass@@V?$vector@U?$pair@II@stlpmtx_std@@V?$allocator@U?$pair@II@stlpmtx_std@@@2@@stlpmtx_std@@@stlpmtx_std@@@3@@priv@stlpmtx_std@@AAEXPAU_Rb_tree_node_base@23@@Z 320956e0 f i EntitySystem.obj
 0001:000946e0       ?_M_erase@?$_Rb_tree@HU?$less@H@stlpmtx_std@@U?$pair@$$CBHUSAreasCache@CAreaManager@@@2@U?$_Select1st@U?$pair@$$CBHUSAreasCache@CAreaManager@@@stlpmtx_std@@@priv@2@U?$_MapTraitsT@U?$pair@$$CBHUSAreasCache@CAreaManager@@@stlpmtx_std@@@52@V?$allocator@U?$pair@$$CBHUSAreasCache@CAreaManager@@@stlpmtx_std@@@2@@priv@stlpmtx_std@@AAEXPAU_Rb_tree_node_base@23@@Z 320956e0 f i AreaManager.obj
 0001:000947a0       ?_M_create_node@?$_Rb_tree@HU?$less@H@stlpmtx_std@@U?$pair@$$CBHUSAreasCache@CAreaManager@@@2@U?$_Select1st@U?$pair@$$CBHUSAreasCache@CAreaManager@@@stlpmtx_std@@@priv@2@U?$_MapTraitsT@U?$pair@$$CBHUSAreasCache@CAreaManager@@@stlpmtx_std@@@52@V?$allocator@U?$pair@$$CBHUSAreasCache@CAreaManager@@@stlpmtx_std@@@2@@priv@stlpmtx_std@@IAEPAU_Rb_tree_node_base@23@ABU?$pair@$$CBHUSAreasCache@CAreaManager@@@3@@Z 320957a0 f i AreaManager.obj
 0001:00094800       ??1CAreaManager@@UAE@XZ    32095800 f   AreaManager.obj
 0001:000948f0       ?GetAreaAmount@CAreaManager@@UBEHXZ 320958f0 f i AreaManager.obj
 0001:00094900       ?Unregister@CAreaManager@@IAEXPAVCArea@@@Z 32095900 f   AreaManager.obj
 0001:00094af0       ?ExitAllAreas@CAreaManager@@UAEXQBUIEntity@@@Z 32095af0 f   AreaManager.obj
 0001:00094cb0       ?ResetAreas@CAreaManager@@QAEXXZ 32095cb0 f   AreaManager.obj
 0001:00094f50       ?UnloadAreas@CAreaManager@@QAEXXZ 32095f50 f   AreaManager.obj
 0001:00094f70       ?_M_insert@?$_Rb_tree@HU?$less@H@stlpmtx_std@@U?$pair@$$CBHUSAreasCache@CAreaManager@@@2@U?$_Select1st@U?$pair@$$CBHUSAreasCache@CAreaManager@@@stlpmtx_std@@@priv@2@U?$_MapTraitsT@U?$pair@$$CBHUSAreasCache@CAreaManager@@@stlpmtx_std@@@52@V?$allocator@U?$pair@$$CBHUSAreasCache@CAreaManager@@@stlpmtx_std@@@2@@priv@stlpmtx_std@@AAE?AU?$_Rb_tree_iterator@U?$pair@$$CBHUSAreasCache@CAreaManager@@@stlpmtx_std@@U?$_MapTraitsT@U?$pair@$$CBHUSAreasCache@CAreaManager@@@stlpmtx_std@@@priv@2@@23@PAU_Rb_tree_node_base@23@ABU?$pair@$$CBHUSAreasCache@CAreaManager@@@3@00@Z 32095f70 f i AreaManager.obj
 0001:00095040       ?insert_unique@?$_Rb_tree@HU?$less@H@stlpmtx_std@@U?$pair@$$CBHUSAreasCache@CAreaManager@@@2@U?$_Select1st@U?$pair@$$CBHUSAreasCache@CAreaManager@@@stlpmtx_std@@@priv@2@U?$_MapTraitsT@U?$pair@$$CBHUSAreasCache@CAreaManager@@@stlpmtx_std@@@52@V?$allocator@U?$pair@$$CBHUSAreasCache@CAreaManager@@@stlpmtx_std@@@2@@priv@stlpmtx_std@@QAE?AU?$pair@U?$_Rb_tree_iterator@U?$pair@$$CBHUSAreasCache@CAreaManager@@@stlpmtx_std@@U?$_MapTraitsT@U?$pair@$$CBHUSAreasCache@CAreaManager@@@stlpmtx_std@@@priv@2@@priv@stlpmtx_std@@_N@3@ABU?$pair@$$CBHUSAreasCache@CAreaManager@@@3@@Z 32096040 f i AreaManager.obj
 0001:00095100       ??0CAreaManager@@QAE@PAVCEntitySystem@@@Z 32096100 f   AreaManager.obj
 0001:00095260       ??_GCAreaManager@@UAEPAXI@Z 32096260 f i AreaManager.obj
 0001:00095260       ??_ECAreaManager@@UAEPAXI@Z 32096260 f i AreaManager.obj
 0001:00095290       ?insert_unique@?$_Rb_tree@HU?$less@H@stlpmtx_std@@U?$pair@$$CBHUSAreasCache@CAreaManager@@@2@U?$_Select1st@U?$pair@$$CBHUSAreasCache@CAreaManager@@@stlpmtx_std@@@priv@2@U?$_MapTraitsT@U?$pair@$$CBHUSAreasCache@CAreaManager@@@stlpmtx_std@@@52@V?$allocator@U?$pair@$$CBHUSAreasCache@CAreaManager@@@stlpmtx_std@@@2@@priv@stlpmtx_std@@QAE?AU?$_Rb_tree_iterator@U?$pair@$$CBHUSAreasCache@CAreaManager@@@stlpmtx_std@@U?$_MapTraitsT@U?$pair@$$CBHUSAreasCache@CAreaManager@@@stlpmtx_std@@@priv@2@@23@U423@ABU?$pair@$$CBHUSAreasCache@CAreaManager@@@3@@Z 32096290 f i AreaManager.obj
 0001:00095480       ??$?AH@?$map@HUSAreasCache@CAreaManager@@U?$less@H@stlpmtx_std@@V?$allocator@U?$pair@$$CBHUSAreasCache@CAreaManager@@@stlpmtx_std@@@4@@stlpmtx_std@@QAEAAUSAreasCache@CAreaManager@@ABH@Z 32096480 f i AreaManager.obj
 0001:00095570       ?UpdatePlayer@CAreaManager@@QAEXABU?$Vec3_tpl@M@@PAUIEntity@@@Z 32096570 f   AreaManager.obj
 0001:00095be0       ?Update@CAreaManager@@QAEXXZ 32096be0 f   AreaManager.obj
 0001:00095df0       ??_GIBreakableManager@@UAEPAXI@Z 32096df0 f i BreakableManager.obj
 0001:00095df0       ??_EIBreakableManager@@UAEPAXI@Z 32096df0 f i BreakableManager.obj
 0001:00095e20       ?RemoveBreakEventListener@CBreakableManager@@UAEXPAUIBreakEventListener@@@Z 32096e20 f   BreakableManager.obj
 0001:00095e30       ?EntityDrawSlot@CBreakableManager@@UAEXPAVCEntity@@HH@Z 32096e30 f   BreakableManager.obj
 0001:00095e50       ?GetBrokenObjectIndicesForCloning@CBreakableManager@@UAEXPAHAAH01PBUEventPhysRemoveEntityParts@@@Z 32096e50 f   BreakableManager.obj
 0001:00095fb0       ?UnhidePartRemovedObjectsByIndex@CBreakableManager@@UAEXPBHHPBUEventPhysRemoveEntityParts@@@Z 32096fb0 f   BreakableManager.obj
 0001:00096080       ?ProcessPlaneImpact@CBreakableManager@@UAE?AW4EProcessImpactResult@@ABUSProcessImpactIn@@AAUSProcessImpactOut@@@Z 32097080 f   BreakableManager.obj
 0001:000960a0       ?ExtractPlaneMeshIsland@CBreakableManager@@UAEXABUSExtractMeshIslandIn@@AAUSExtractMeshIslandOut@@@Z 320970a0 f   BreakableManager.obj
 0001:000960c0       ?GetPlaneMemoryStatistics@CBreakableManager@@UAEXPAXPAVICrySizer@@@Z 320970c0 f   BreakableManager.obj
 0001:000960e0       ?SetMatrix@SMFXBreakageParams@@QAEXABU?$Matrix34_tpl@M@@@Z 320970e0 f i BreakableManager.obj
 0001:00096140       ?GetSurfaceType@@YAPAUISurfaceType@@PAUIRenderMesh@@PAUIMaterial@@@Z 32097140 f   BreakableManager.obj
 0001:000961e0       ?GetSurfaceType@@YAPAUISurfaceType@@PAUIStatObj@@@Z 320971e0 f   BreakableManager.obj
 0001:000962c0       ?GetFirstSurfaceType@CBreakableManager@@UAEPAUISurfaceType@@PAUIStatObj@@@Z 320972c0 f   BreakableManager.obj
 0001:000962e0       ?CanShatterRenderMesh@CBreakableManager@@QAE_NPAUIRenderMesh@@PAUIMaterial@@@Z 320972e0 f   BreakableManager.obj
 0001:00096390       ?CanShatter@CBreakableManager@@UAE_NPAUIStatObj@@@Z 32097390 f   BreakableManager.obj
 0001:00096460       ?CanShatterEntity@CBreakableManager@@UAE_NPAUIEntity@@H@Z 32097460 f   BreakableManager.obj
 0001:00096520       ?ClonePartRemovedEntitiesByIndex@CBreakableManager@@UAEXPAHHPAIAAHPBIHAAUSRenderNodeCloneLookup@@@Z 32097520 f   BreakableManager.obj
 0001:00096860       ??0pe_params_structural_joint@@QAE@XZ 32097860 f i BreakableManager.obj
 0001:00096940       ??0SMFXBreakageParams@@QAE@XZ 32097940 f i BreakableManager.obj
 0001:000969d0       ?AssociateStatObjWithPhysics@@YAXPAUIStatObj@@PAUIPhysicalEntity@@H@Z 320979d0 f   BreakableManager.obj
 0001:00096a60       ?GetSurfaceType@@YAPAUISurfaceType@@PAUICharacterInstance@@@Z 32097a60 f   BreakableManager.obj
 0001:00096b70       ?GetFirstSurfaceType@CBreakableManager@@UAEPAUISurfaceType@@PAUICharacterInstance@@@Z 32097b70 f   BreakableManager.obj
 0001:00096b90       ?GetPhysicsStatus@?A0x46d751d7@@YAXPAUIPhysicalEntity@@AAM11AAU?$Vec3_tpl@M@@22@Z 32097b90 f   BreakableManager.obj
 0001:00096e40       ?CreateObjectCommon@CBreakableManager@@AAEXPAUIStatObj@@PAUIPhysicalEntity@@AAUSCreateParams@IBreakableManager@@@Z 32097e40 f   BreakableManager.obj
 0001:00096f20       ?CheckSubObjBreak@CBreakableManager@@QAEPAUSSubObject@IStatObj@@PAU3@PAU23@PBUEventPhysCreateEntityPart@@@Z 32097f20 f   BreakableManager.obj
 0001:00097030       ?HandlePhysicsRevealSubPartEvent@CBreakableManager@@QAEXPBUEventPhysRevealEntityPart@@@Z 32098030 f   BreakableManager.obj
 0001:000973a0       ?IsGeometryBreakable@CBreakableManager@@UAE_NPAUIPhysicalEntity@@PAUIStatObj@@PAUIMaterial@@@Z 320983a0 f   BreakableManager.obj
 0001:00097610       ?HideBrokenObjectsByIndex@CBreakableManager@@UAEXPBHH@Z 32098610 f   BreakableManager.obj
 0001:000976a0       ?ApplyPartBreakToClonedObjectFromEvent@CBreakableManager@@AAEXABUSRenderNodeCloneLookup@@ABUEventPhysRemoveEntityParts@@@Z 320986a0 f   BreakableManager.obj
 0001:000977d0       ??$__ufill@PAUSBrokenObjRec@IBreakableManager@@U12@H@priv@stlpmtx_std@@YAXPAUSBrokenObjRec@IBreakableManager@@0ABU23@ABUrandom_access_iterator_tag@1@PAH@Z 320987d0 f i BreakableManager.obj
 0001:00097830       ?ExtractStringKeyFromString@@YA?AV?$CryStringT@D@@PBDABV1@@Z 32098830 f   BreakableManager.obj
 0001:00097910       ?ApplySinglePartRemovalFromEventIndex@CBreakableManager@@UAEXHABUSRenderNodeCloneLookup@@PBUEventPhysRemoveEntityParts@@@Z 32098910 f   BreakableManager.obj
 0001:00097930       ?ApplyPartRemovalsUntilIndexToObjectList@CBreakableManager@@UAEXHABUSRenderNodeCloneLookup@@PBUEventPhysRemoveEntityParts@@@Z 32098930 f   BreakableManager.obj
 0001:00097a80       ??$__ucopy_ptrs@PAUSBrokenObjRec@IBreakableManager@@PAU12@@priv@stlpmtx_std@@YAPAUSBrokenObjRec@IBreakableManager@@PAU23@00ABU__false_type@1@@Z 32098a80 f i BreakableManager.obj
 0001:00097af0       ??1?$DynArray@UGeomQuery@@HU?$SmallDynStorage@UGeomQuery@@HUStandardAlloc@NAlloc@@@NArray@@@@QAE@XZ 32098af0 f i BreakableManager.obj
 0001:00097b50       ?GetSurfaceEffect@@YAPAUIParticleEffect@@PAUISurfaceType@@PBDAAUSpawnParams@@@Z 32098b50 f   BreakableManager.obj
 0001:00097e60       ?CreateSurfaceEffect@CBreakableManager@@UAEXPAUIStatObj@@ABU?$Matrix34_tpl@M@@PBD@Z 32098e60 f   BreakableManager.obj
 0001:00097ff0       ?AttachSurfaceEffect@CBreakableManager@@UAEXPAUIEntity@@HPBDABUSpawnParams@@I@Z 32098ff0 f   BreakableManager.obj
 0001:000980d0       ??1?$_Impl_vector@USBrokenObjRec@IBreakableManager@@V?$allocator@USBrokenObjRec@IBreakableManager@@@stlpmtx_std@@@priv@stlpmtx_std@@QAE@XZ 320990d0 f i BreakableManager.obj
 0001:00098120       ??_GGeomQuery@@QAEPAXI@Z   32099120 f i BreakableManager.obj
 0001:00098170       ?_M_insert_overflow_aux@?$_Impl_vector@USBrokenObjRec@IBreakableManager@@V?$allocator@USBrokenObjRec@IBreakableManager@@@stlpmtx_std@@@priv@stlpmtx_std@@AAEXPAUSBrokenObjRec@IBreakableManager@@ABU45@ABU__false_type@3@I_N@Z 32099170 f i BreakableManager.obj
 0001:00098340       ??0GeomQuery@@QAE@XZ       32099340 f i BreakableManager.obj
 0001:000983e0       ??0CBreakableManager@@QAE@PAVCEntitySystem@@@Z 320993e0 f   BreakableManager.obj
 0001:00098440       ?GetPartBrokenObjects@CBreakableManager@@UAEPBUSBrokenObjRec@IBreakableManager@@AAH@Z 32099440 f i BreakableManager.obj
 0001:00098470       ??_ECBreakableManager@@UAEPAXI@Z 32099470 f i BreakableManager.obj
 0001:00098470       ??_GCBreakableManager@@UAEPAXI@Z 32099470 f i BreakableManager.obj
 0001:000984d0       ?push_back@?$_Impl_vector@USBrokenObjRec@IBreakableManager@@V?$allocator@USBrokenObjRec@IBreakableManager@@@stlpmtx_std@@@priv@stlpmtx_std@@QAEXABUSBrokenObjRec@IBreakableManager@@@Z 320994d0 f i BreakableManager.obj
 0001:00098540       ?CreateObjectAsEntity@CBreakableManager@@UAEPAUIEntity@@PAUIStatObj@@PAUIPhysicalEntity@@1AAUSCreateParams@IBreakableManager@@_N@Z 32099540 f   BreakableManager.obj
 0001:00098930       ?HandlePhysicsRemoveSubPartsEvent@CBreakableManager@@QAEXPBUEventPhysRemoveEntityParts@@@Z 32099930 f   BreakableManager.obj
 0001:00099060       ?HandlePhysics_UpdateMeshEvent@CBreakableManager@@QAEHPBUEventPhysUpdateMesh@@@Z 3209a060 f   BreakableManager.obj
 0001:00099e30       ?ResetBrokenObjects@CBreakableManager@@UAEXXZ 3209ae30 f   BreakableManager.obj
 0001:0009a000       ?ReplayRemoveSubPartsEvent@CBreakableManager@@UAEXPBUEventPhysRemoveEntityParts@@@Z 3209b000 f   BreakableManager.obj
 0001:0009a010       ?BreakIntoPieces@CBreakableManager@@QAEXAAUGeomRef@@ABU?$Matrix34_tpl@M@@PAUIStatObj@@1ABUBreakageParams@IBreakableManager@@H@Z 3209b010 f   BreakableManager.obj
 0001:0009d290       ?BreakIntoPieces@CBreakableManager@@UAEXPAUIEntity@@HHABUBreakageParams@IBreakableManager@@@Z 3209e290 f   BreakableManager.obj
 0001:0009d4a0       ?CreateObjectAsParticles@CBreakableManager@@QAEXPAUIStatObj@@PAUIPhysicalEntity@@AAUSCreateParams@IBreakableManager@@@Z 3209e4a0 f   BreakableManager.obj
 0001:0009d8d0       ?CheckForPieces@CBreakableManager@@QAE_NPAUIStatObj@@PAUSSubObject@2@ABU?$Matrix34_tpl@M@@HPAUIPhysicalEntity@@@Z 3209e8d0 f   BreakableManager.obj
 0001:0009df10       ?HandlePhysicsCreateEntityPartEvent@CBreakableManager@@QAEXPBUEventPhysCreateEntityPart@@@Z 3209ef10 f   BreakableManager.obj
 0001:0009f920       ?FakePhysicsEvent@CBreakableManager@@UAEXPAUEventPhys@@@Z 320a0920 f   BreakableManager.obj
 0001:0009f960       ?AllocateGrid@CPartitionGrid@@QAEXMM@Z 320a0960 f   PartitionGrid.obj
 0001:0009fa00       ?SectorLink@CPartitionGrid@@AAEXPAUSGridLocation@@AAULocationInfo@1@@Z 320a0a00 f   PartitionGrid.obj
 0001:0009fa50       ?SectorUnlink@CPartitionGrid@@AAEXPAUSGridLocation@@AAULocationInfo@1@@Z 320a0a50 f   PartitionGrid.obj
 0001:0009fac0       ?BeginReset@CPartitionGrid@@QAEXXZ 320a0ac0 f   PartitionGrid.obj
 0001:0009fad0       ?GetMemoryUsage@CPartitionGrid@@QBEXPAVICrySizer@@@Z 320a0ad0 f   PartitionGrid.obj
 0001:0009fb50       ??_GCUT_PartitionGrid@@UAEPAXI@Z 320a0b50 f i PartitionGrid.obj
 0001:0009fb50       ??_GTest@CryUnitTest@@UAEPAXI@Z 320a0b50 f i PartitionGrid.obj
 0001:0009fb50       ??_ETest@CryUnitTest@@UAEPAXI@Z 320a0b50 f i PartitionGrid.obj
 0001:0009fb50       ??_ECUT_PartitionGrid@@UAEPAXI@Z 320a0b50 f i PartitionGrid.obj
 0001:0009fba0       ??3SectorGroup@CPartitionGrid@@SAXPAX@Z 320a0ba0 f i PartitionGrid.obj
 0001:0009fc00       ??3SGridLocation@@SAXPAX@Z 320a0c00 f i PartitionGrid.obj
 0001:0009fc60       ?DeallocateGrid@CPartitionGrid@@QAEXXZ 320a0c60 f   PartitionGrid.obj
 0001:0009fcd0       ?AllocateGroup@CPartitionGrid@@AAEPAUSectorGroup@1@XZ 320a0cd0 f   PartitionGrid.obj
 0001:0009fd40       ?AllocateLocation@CPartitionGrid@@AAEPAUSGridLocation@@XZ 320a0d40 f   PartitionGrid.obj
 0001:0009fdb0       ?FreeGroup@CPartitionGrid@@AAEXAAULocationInfo@1@@Z 320a0db0 f   PartitionGrid.obj
 0001:0009fe00       ?GetSectorGroup@CPartitionGrid@@AAEPAUSectorGroup@1@HH@Z 320a0e00 f i PartitionGrid.obj
 0001:0009fe50       ?GetSector@CPartitionGrid@@AAEXHAAULocationInfo@1@@Z 320a0e50 f i PartitionGrid.obj
 0001:0009feb0       ?GetSector@CPartitionGrid@@AAEXABU?$Vec3_tpl@M@@AAULocationInfo@1@@Z 320a0eb0 f i PartitionGrid.obj
 0001:0009ff70       ?FreeLocation@CPartitionGrid@@QAEXPAUSGridLocation@@@Z 320a0f70 f   PartitionGrid.obj
 0001:0009ffe0       ?Rellocate@CPartitionGrid@@QAEPAUSGridLocation@@PAU2@ABU?$Vec3_tpl@M@@PAVCEntity@@@Z 320a0fe0 f   PartitionGrid.obj
 0001:000a01b0       ?AddSectorsToQuery@CPartitionGrid@@AAEXHHHHHHABUSPartitionGridQuery@@AAV?$vector@PAUIEntity@@V?$allocator@PAUIEntity@@@stlpmtx_std@@@stlpmtx_std@@@Z 320a11b0 f   PartitionGrid.obj
 0001:000a0310       ??0CPartitionGrid@@QAE@XZ  320a1310 f   PartitionGrid.obj
 0001:000a0470       ?Reset@CPartitionGrid@@QAEXXZ 320a1470 f   PartitionGrid.obj
 0001:000a0490       ??1CPartitionGrid@@QAE@XZ  320a1490 f   PartitionGrid.obj
 0001:000a0560       ?GetEntitiesInBox@CPartitionGrid@@QAEXAAUSPartitionGridQuery@@@Z 320a1560 f   PartitionGrid.obj
 0001:000a07a0       ?Run@CUT_PartitionGrid@@EAEXXZ 320a17a0 f   PartitionGrid.obj
 0001:000a0c50       ?BeginReset@CProximityTriggerSystem@@QAEXXZ 320a1c50 f   ProximityTriggerSystem.obj
 0001:000a0c60       ??$__fill_n@PAUAABB@@IU1@@priv@stlpmtx_std@@YAPAUAABB@@PAU2@IABU2@@Z 320a1c60 f i ProximityTriggerSystem.obj
 0001:000a0ca0       ??$fill@PAUAABB@@U1@@stlpmtx_std@@YAXPAUAABB@@0ABU1@@Z 320a1ca0 f i ProximityTriggerSystem.obj
 0001:000a0d00       ??$__unguarded_linear_insert@PAUInOut@?A0xeda18add@@U12@U?$less@UInOut@?A0xeda18add@@@stlpmtx_std@@@priv@stlpmtx_std@@YAXPAUInOut@?A0xeda18add@@U23@U?$less@UInOut@?A0xeda18add@@@1@@Z 320a1d00 f i ProximityTriggerSystem.obj
 0001:000a0d50       ??$__push_heap@PAUInOut@?A0xeda18add@@HU12@U?$less@UInOut@?A0xeda18add@@@stlpmtx_std@@@stlpmtx_std@@YAXPAUInOut@?A0xeda18add@@HHU12@U?$less@UInOut@?A0xeda18add@@@0@@Z 320a1d50 f i ProximityTriggerSystem.obj
 0001:000a0dd0       ??$__lower_bound@PBIIU?$less@I@stlpmtx_std@@U12@H@priv@stlpmtx_std@@YAPBIPBI0ABIU?$less@I@1@2PAH@Z 320a1dd0 f i EntityEventDistributer.obj
 0001:000a0dd0       ??$__lower_bound@PAPAUSProximityElement@@PAU1@U?$__less_2@PAUSProximityElement@@PAU1@@priv@stlpmtx_std@@U234@H@priv@stlpmtx_std@@YAPAPAUSProximityElement@@PAPAU2@0ABQAU2@U?$__less_2@PAUSProximityElement@@PAU1@@01@2PAH@Z 320a1dd0 f i ProximityTriggerSystem.obj
 0001:000a0e10       ??$__ucopy@PAUAABB@@PAU1@H@priv@stlpmtx_std@@YAPAUAABB@@PAU2@00ABUrandom_access_iterator_tag@1@PAH@Z 320a1e10 f i ProximityTriggerSystem.obj
 0001:000a0e70       ??$__ufill@PAUAABB@@U1@H@priv@stlpmtx_std@@YAXPAUAABB@@0ABU2@ABUrandom_access_iterator_tag@1@PAH@Z 320a1e70 f i ProximityTriggerSystem.obj
 0001:000a0ed0       ??$__unguarded_insertion_sort_aux@PAUInOut@?A0xeda18add@@U12@U?$less@UInOut@?A0xeda18add@@@stlpmtx_std@@@priv@stlpmtx_std@@YAXPAUInOut@?A0xeda18add@@00U?$less@UInOut@?A0xeda18add@@@1@@Z 320a1ed0 f i ProximityTriggerSystem.obj
 0001:000a0f50       ??$__adjust_heap@PAUInOut@?A0xeda18add@@HU12@U?$less@UInOut@?A0xeda18add@@@stlpmtx_std@@@stlpmtx_std@@YAXPAUInOut@?A0xeda18add@@HHU12@U?$less@UInOut@?A0xeda18add@@@0@@Z 320a1f50 f i ProximityTriggerSystem.obj
 0001:000a1010       ?_M_insert_overflow@?$_Impl_vector@UAABB@@V?$allocator@UAABB@@@stlpmtx_std@@@priv@stlpmtx_std@@AAEXPAUAABB@@ABU4@ABU__true_type@3@I_N@Z 320a2010 f i ProximityTriggerSystem.obj
 0001:000a1180       ??$__unguarded_partition@PAUInOut@?A0xeda18add@@U12@U?$less@UInOut@?A0xeda18add@@@stlpmtx_std@@@priv@stlpmtx_std@@YAPAUInOut@?A0xeda18add@@PAU23@0U23@U?$less@UInOut@?A0xeda18add@@@1@@Z 320a2180 f i ProximityTriggerSystem.obj
 0001:000a11f0       ??$__make_heap@PAUInOut@?A0xeda18add@@U?$less@UInOut@?A0xeda18add@@@stlpmtx_std@@U12@H@stlpmtx_std@@YAXPAUInOut@?A0xeda18add@@0U?$less@UInOut@?A0xeda18add@@@0@0PAH@Z 320a21f0 f i ProximityTriggerSystem.obj
 0001:000a1310       ?GetMemoryUsage@CProximityTriggerSystem@@QBEXPAVICrySizer@@@Z 320a2310 f   ProximityTriggerSystem.obj
 0001:000a1480       ??0?$_Vector_base@UAABB@@V?$allocator@UAABB@@@stlpmtx_std@@@priv@stlpmtx_std@@QAE@IABV?$allocator@UAABB@@@2@@Z 320a2480 f i ProximityTriggerSystem.obj
 0001:000a1540       ??0?$_Vector_base@MV?$allocator@M@stlpmtx_std@@@priv@stlpmtx_std@@QAE@IABV?$allocator@M@2@@Z 320a2540 f i ProximityTriggerSystem.obj
 0001:000a1540       ??0?$_Vector_base@V?$CryStringT@D@@V?$allocator@V?$CryStringT@D@@@stlpmtx_std@@@priv@stlpmtx_std@@QAE@IABV?$allocator@V?$CryStringT@D@@@2@@Z 320a2540 f i EntityPoolManager.obj
 0001:000a1540       ??0?$_Vector_base@PAXV?$allocator@PAX@stlpmtx_std@@@priv@stlpmtx_std@@QAE@IABV?$allocator@PAX@2@@Z 320a2540 f i EntityEventDistributer.obj
 0001:000a15f0       ??$binary_erase@V?$vector@PAUSProximityElement@@V?$allocator@PAUSProximityElement@@@stlpmtx_std@@@stlpmtx_std@@PAUSProximityElement@@@stl@@YA_NAAV?$vector@PAUSProximityElement@@V?$allocator@PAUSProximityElement@@@stlpmtx_std@@@stlpmtx_std@@ABQAUSProximityElement@@@Z 320a25f0 f i ProximityTriggerSystem.obj
 0001:000a1680       ?_M_fill_insert_aux@?$_Impl_vector@UAABB@@V?$allocator@UAABB@@@stlpmtx_std@@@priv@stlpmtx_std@@AAEXPAUAABB@@IABU4@ABU__false_type@3@@Z 320a2680 f i ProximityTriggerSystem.obj
 0001:000a17e0       ?_M_fill_insert_aux@?$_Impl_vector@USEntityTimerEvent@@V?$allocator@USEntityTimerEvent@@@stlpmtx_std@@@priv@stlpmtx_std@@AAEXPAUSEntityTimerEvent@@IABU4@ABU__false_type@3@@Z 320a27e0 f i EntitySystem.obj
 0001:000a17e0       ?_M_fill_insert_aux@?$_Impl_vector@USProximityEvent@@V?$allocator@USProximityEvent@@@stlpmtx_std@@@priv@stlpmtx_std@@AAEXPAUSProximityEvent@@IABU4@ABU__false_type@3@@Z 320a27e0 f i ProximityTriggerSystem.obj
 0001:000a1900       ??$__insertion_sort@PAUInOut@?A0xeda18add@@U12@U?$less@UInOut@?A0xeda18add@@@stlpmtx_std@@@priv@stlpmtx_std@@YAXPAUInOut@?A0xeda18add@@00U?$less@UInOut@?A0xeda18add@@@1@@Z 320a2900 f i ProximityTriggerSystem.obj
 0001:000a19b0       ??_GSProximityElement@@QAEPAXI@Z 320a29b0 f i ProximityTriggerSystem.obj
 0001:000a1a40       ?push_back@?$vector@PAUIEntityClass@@V?$allocator@PAUIEntityClass@@@stlpmtx_std@@@stlpmtx_std@@QAEXABQAUIEntityClass@@@Z 320a2a40 f i EntityPoolDefinition.obj
 0001:000a1a40       ?push_back@?$vector@PAUSProximityElement@@V?$allocator@PAUSProximityElement@@@stlpmtx_std@@@stlpmtx_std@@QAEXABQAUSProximityElement@@@Z 320a2a40 f i ProximityTriggerSystem.obj
 0001:000a1a40       ?push_back@?$vector@HV?$allocator@H@stlpmtx_std@@@stlpmtx_std@@QAEXABH@Z 320a2a40 f i AreaManager.obj
 0001:000a1a40       ?push_back@?$vector@PAVCEntity@@V?$allocator@PAVCEntity@@@stlpmtx_std@@@stlpmtx_std@@QAEXABQAVCEntity@@@Z 320a2a40 f i Entity.obj
 0001:000a1a90       ?push_back@?$vector@USProximityEvent@@V?$allocator@USProximityEvent@@@stlpmtx_std@@@stlpmtx_std@@QAEXABUSProximityEvent@@@Z 320a2a90 f i ProximityTriggerSystem.obj
 0001:000a1af0       ??$sort_heap@PAUInOut@?A0xeda18add@@U?$less@UInOut@?A0xeda18add@@@stlpmtx_std@@@stlpmtx_std@@YAXPAUInOut@?A0xeda18add@@0U?$less@UInOut@?A0xeda18add@@@0@@Z 320a2af0 f i ProximityTriggerSystem.obj
 0001:000a1b80       ?CreateTrigger@CProximityTriggerSystem@@QAEPAUSProximityElement@@XZ 320a2b80 f   ProximityTriggerSystem.obj
 0001:000a1c60       ?RemoveTrigger@CProximityTriggerSystem@@QAEXPAUSProximityElement@@@Z 320a2c60 f   ProximityTriggerSystem.obj
 0001:000a1cb0       ?CreateEntity@CProximityTriggerSystem@@QAEPAUSProximityElement@@I@Z 320a2cb0 f   ProximityTriggerSystem.obj
 0001:000a1d60       ?MoveEntity@CProximityTriggerSystem@@QAEXPAUSProximityElement@@ABU?$Vec3_tpl@M@@@Z 320a2d60 f   ProximityTriggerSystem.obj
 0001:000a1e20       ?RemoveFromTriggers@CProximityTriggerSystem@@AAEXPAUSProximityElement@@_N@Z 320a2e20 f   ProximityTriggerSystem.obj
 0001:000a1ef0       ?CheckIfLeavingTrigger@CProximityTriggerSystem@@AAEXPAUSProximityElement@@@Z 320a2ef0 f   ProximityTriggerSystem.obj
 0001:000a20f0       ?insert@?$vector@PAUSProximityElement@@V?$allocator@PAUSProximityElement@@@stlpmtx_std@@@stlpmtx_std@@QAEPAPAUSProximityElement@@PAPAU3@ABQAU3@@Z 320a30f0 f i ProximityTriggerSystem.obj
 0001:000a2150       ??$__partial_sort@PAUInOut@?A0xeda18add@@U12@U?$less@UInOut@?A0xeda18add@@@stlpmtx_std@@@priv@stlpmtx_std@@YAXPAUInOut@?A0xeda18add@@000U?$less@UInOut@?A0xeda18add@@@1@@Z 320a3150 f i ProximityTriggerSystem.obj
 0001:000a2200       ??0CProximityTriggerSystem@@QAE@XZ 320a3200 f   ProximityTriggerSystem.obj
 0001:000a2390       ?MoveTrigger@CProximityTriggerSystem@@QAEXPAUSProximityElement@@ABUAABB@@_N@Z 320a3390 f   ProximityTriggerSystem.obj
 0001:000a26f0       ?RemoveEntity@CProximityTriggerSystem@@QAEXPAUSProximityElement@@_N@Z 320a36f0 f   ProximityTriggerSystem.obj
 0001:000a2780       ?Reset@CProximityTriggerSystem@@QAEXXZ 320a3780 f   ProximityTriggerSystem.obj
 0001:000a39e0       ?resize@?$_Impl_vector@UAABB@@V?$allocator@UAABB@@@stlpmtx_std@@@priv@stlpmtx_std@@QAEXIABUAABB@@@Z 320a49e0 f i ProximityTriggerSystem.obj
 0001:000a3aa0       ?resize@?$_Impl_vector@USProximityEvent@@V?$allocator@USProximityEvent@@@stlpmtx_std@@@priv@stlpmtx_std@@QAEXIABUSProximityEvent@@@Z 320a4aa0 f i ProximityTriggerSystem.obj
 0001:000a3aa0       ?resize@?$_Impl_vector@USEntityTimerEvent@@V?$allocator@USEntityTimerEvent@@@stlpmtx_std@@@priv@stlpmtx_std@@QAEXIABUSEntityTimerEvent@@@Z 320a4aa0 f i EntitySystem.obj
 0001:000a3b50       ??$binary_insert_unique@V?$vector@PAUSProximityElement@@V?$allocator@PAUSProximityElement@@@stlpmtx_std@@@stlpmtx_std@@PAUSProximityElement@@@stl@@YA_NAAV?$vector@PAUSProximityElement@@V?$allocator@PAUSProximityElement@@@stlpmtx_std@@@stlpmtx_std@@ABQAUSProximityElement@@@Z 320a4b50 f i ProximityTriggerSystem.obj
 0001:000a3bf0       ??1CProximityTriggerSystem@@QAE@XZ 320a4bf0 f   ProximityTriggerSystem.obj
 0001:000a3da0       ??$__introsort_loop@PAUInOut@?A0xeda18add@@U12@HU?$less@UInOut@?A0xeda18add@@@stlpmtx_std@@@priv@stlpmtx_std@@YAXPAUInOut@?A0xeda18add@@00HU?$less@UInOut@?A0xeda18add@@@1@@Z 320a4da0 f i ProximityTriggerSystem.obj
 0001:000a3e80       ?SendEvents@CProximityTriggerSystem@@AAEXXZ 320a4e80 f   ProximityTriggerSystem.obj
 0001:000a3fd0       ?PurgeRemovedTriggers@CProximityTriggerSystem@@AAEXXZ 320a4fd0 f   ProximityTriggerSystem.obj
 0001:000a42f0       ??$sort@PAUInOut@?A0xeda18add@@@stlpmtx_std@@YAXPAUInOut@?A0xeda18add@@0@Z 320a52f0 f i ProximityTriggerSystem.obj
 0001:000a4990       ?SortTriggers@CProximityTriggerSystem@@AAEXXZ 320a5990 f   ProximityTriggerSystem.obj
 0001:000a4eb0       ?Update@CProximityTriggerSystem@@QAEXXZ 320a5eb0 f   ProximityTriggerSystem.obj
 0001:000a54a0       ??0RadixSort@@QAE@XZ       320a64a0 f   RadixSort.obj
 0001:000a54c0       ??1RadixSort@@QAE@XZ       320a64c0 f   RadixSort.obj
 0001:000a54e0       ?Resize@RadixSort@@AAE_NI@Z 320a64e0 f   RadixSort.obj
 0001:000a5580       ?Sort@RadixSort@@QAEAAV1@PBMI@Z 320a6580 f   RadixSort.obj
 0001:000a5a90       ??$__find@PAUSEntityIds@CEntityPool@@I@priv@stlpmtx_std@@YAPAUSEntityIds@CEntityPool@@PAU23@0ABIABUrandom_access_iterator_tag@1@@Z 320a6a90 f i EntityPool.obj
 0001:000a5b10       ??$__find@PAUSEntityIds@CEntityPool@@U12@@priv@stlpmtx_std@@YAPAUSEntityIds@CEntityPool@@PAU23@0ABU23@ABUrandom_access_iterator_tag@1@@Z 320a6b10 f i EntityPool.obj
 0001:000a5b90       ??$__find_if@PBUSEntityIds@CEntityPool@@V?$binder2nd@VCompareUsingIds@SEntityIds@CEntityPool@@@stlpmtx_std@@@priv@stlpmtx_std@@YAPBUSEntityIds@CEntityPool@@PBU23@0V?$binder2nd@VCompareUsingIds@SEntityIds@CEntityPool@@@1@ABUrandom_access_iterator_tag@1@@Z 320a6b90 f i EntityPool.obj
 0001:000a5c00       ??$__unique_copy@PAUSEntityIds@CEntityPool@@PAU12@U?$equal_to@USEntityIds@CEntityPool@@@stlpmtx_std@@@priv@stlpmtx_std@@YAPAUSEntityIds@CEntityPool@@PAU23@00U?$equal_to@USEntityIds@CEntityPool@@@1@ABUforward_iterator_tag@1@@Z 320a6c00 f i EntityPool.obj
 0001:000a5c50       ?ContainsEntityClass@CEntityPool@@QBE_NPAUIEntityClass@@@Z 320a6c50 f   EntityPool.obj
 0001:000a5d80       ?GetPoolEntityWithPoolId@CEntityPool@@AAEPAVCEntity@@AA_NI@Z 320a6d80 f   EntityPool.obj
 0001:000a5eb0       ?GetPoolEntityFromInactiveSet@CEntityPool@@AAEPAVCEntity@@XZ 320a6eb0 f   EntityPool.obj
 0001:000a5f80       ?UpdateActiveEntityBookmarks@CEntityPool@@QAEXXZ 320a6f80 f   EntityPool.obj
 0001:000a5fb0       ??$__unguarded_insertion_sort_aux@PAUSEntityIds@CEntityPool@@U12@U?$less@USEntityIds@CEntityPool@@@stlpmtx_std@@@priv@stlpmtx_std@@YAXPAUSEntityIds@CEntityPool@@00U?$less@USEntityIds@CEntityPool@@@1@@Z 320a6fb0 f i EntityPool.obj
 0001:000a6000       ??$__unguarded_insertion_sort_aux@PAIIU?$less@I@stlpmtx_std@@@priv@stlpmtx_std@@YAXPAI00U?$less@I@1@@Z 320a7000 f i EntityPool.obj
 0001:000a6040       ??$__unguarded_insertion_sort_aux@PAUSReturnToPoolWeight@CEntityPool@@U12@U?$less@USReturnToPoolWeight@CEntityPool@@@stlpmtx_std@@@priv@stlpmtx_std@@YAXPAUSReturnToPoolWeight@CEntityPool@@00U?$less@USReturnToPoolWeight@CEntityPool@@@1@@Z 320a7040 f i EntityPool.obj
 0001:000a60a0       ??$_M_range_insert_aux@PAUSEntityIds@CEntityPool@@@?$_Impl_vector@USEntityIds@CEntityPool@@V?$allocator@USEntityIds@CEntityPool@@@stlpmtx_std@@@priv@stlpmtx_std@@AAEXPAUSEntityIds@CEntityPool@@00IABU__false_type@2@@Z 320a70a0 f i EntityPool.obj
 0001:000a61b0       ??$__adjust_heap@PAUSEntityIds@CEntityPool@@HU12@U?$less@USEntityIds@CEntityPool@@@stlpmtx_std@@@stlpmtx_std@@YAXPAUSEntityIds@CEntityPool@@HHU12@U?$less@USEntityIds@CEntityPool@@@0@@Z 320a71b0 f i EntityPool.obj
 0001:000a6250       ??$__adjust_heap@PAUSReturnToPoolWeight@CEntityPool@@HU12@U?$less@USReturnToPoolWeight@CEntityPool@@@stlpmtx_std@@@stlpmtx_std@@YAXPAUSReturnToPoolWeight@CEntityPool@@HHU12@U?$less@USReturnToPoolWeight@CEntityPool@@@0@@Z 320a7250 f i EntityPool.obj
 0001:000a6300       ?GetMemoryStatistics@CEntityPool@@QBEXPAVICrySizer@@@Z 320a7300 f   EntityPool.obj
 0001:000a63a0       ?GetPoolId@CEntityPool@@QBEII@Z 320a73a0 f   EntityPool.obj
 0001:000a6400       ?IsInActiveList@CEntityPool@@QBE_NI@Z 320a7400 f   EntityPool.obj
 0001:000a6430       ?_M_insert_overflow@?$_Impl_vector@USEventPtr@CEntityEventDistributer@@V?$allocator@USEventPtr@CEntityEventDistributer@@@stlpmtx_std@@@priv@stlpmtx_std@@AAEXPAUSEventPtr@CEntityEventDistributer@@ABU45@ABU__true_type@3@I_N@Z 320a7430 f i EntityEventDistributer.obj
 0001:000a6430       ?_M_insert_overflow@?$_Impl_vector@USAreaCacheEntry@CAreaManager@@V?$allocator@USAreaCacheEntry@CAreaManager@@@stlpmtx_std@@@priv@stlpmtx_std@@AAEXPAUSAreaCacheEntry@CAreaManager@@ABU45@ABU__true_type@3@I_N@Z 320a7430 f i AreaManager.obj
 0001:000a6430       ?_M_insert_overflow@?$_Impl_vector@USReturnToPoolWeight@CEntityPool@@V?$allocator@USReturnToPoolWeight@CEntityPool@@@stlpmtx_std@@@priv@stlpmtx_std@@AAEXPAUSReturnToPoolWeight@CEntityPool@@ABU45@ABU__true_type@3@I_N@Z 320a7430 f i EntityPool.obj
 0001:000a6430       ?_M_insert_overflow@?$_Impl_vector@USEntityIds@CEntityPool@@V?$allocator@USEntityIds@CEntityPool@@@stlpmtx_std@@@priv@stlpmtx_std@@AAEXPAUSEntityIds@CEntityPool@@ABU45@ABU__true_type@3@I_N@Z 320a7430 f i EntityPool.obj
 0001:000a6430       ?_M_insert_overflow@?$_Impl_vector@UListenerRecord@?$CListenerSet@PAUIEntityPoolListener@@@@V?$allocator@UListenerRecord@?$CListenerSet@PAUIEntityPoolListener@@@@@stlpmtx_std@@@priv@stlpmtx_std@@AAEXPAUListenerRecord@?$CListenerSet@PAUIEntityPoolListener@@@@ABU45@ABU__true_type@3@I_N@Z 320a7430 f i EntityPoolManager.obj
 0001:000a6430       ?_M_insert_overflow@?$_Impl_vector@U?$pair@II@stlpmtx_std@@V?$allocator@U?$pair@II@stlpmtx_std@@@2@@priv@stlpmtx_std@@AAEXPAU?$pair@II@3@ABU43@ABU__true_type@3@I_N@Z 320a7430 f i EntitySystem.obj
 0001:000a6590       ??$unique@PAUSEntityIds@CEntityPool@@@stlpmtx_std@@YAPAUSEntityIds@CEntityPool@@PAU12@0@Z 320a7590 f i EntityPool.obj
 0001:000a65f0       ??$unique@PAI@stlpmtx_std@@YAPAIPAI0@Z 320a75f0 f i EntityPool.obj
 0001:000a6650       ??$_M_allocate_and_copy@PBUSEventPtr@CEntityEventDistributer@@@?$_Impl_vector@USEventPtr@CEntityEventDistributer@@V?$allocator@USEventPtr@CEntityEventDistributer@@@stlpmtx_std@@@priv@stlpmtx_std@@AAEPAUSEventPtr@CEntityEventDistributer@@AAIPBU34@1@Z 320a7650 f i EntityEventDistributer.obj
 0001:000a6650       ??$_M_allocate_and_copy@PBUListenerRecord@?$CListenerSet@PAUIEntityPoolListener@@@@@?$_Impl_vector@UListenerRecord@?$CListenerSet@PAUIEntityPoolListener@@@@V?$allocator@UListenerRecord@?$CListenerSet@PAUIEntityPoolListener@@@@@stlpmtx_std@@@priv@stlpmtx_std@@AAEPAUListenerRecord@?$CListenerSet@PAUIEntityPoolListener@@@@AAIPBU34@1@Z 320a7650 f i EntityPoolManager.obj
 0001:000a6650       ??$_M_allocate_and_copy@PAUSReturnToPoolWeight@CEntityPool@@@?$_Impl_vector@USReturnToPoolWeight@CEntityPool@@V?$allocator@USReturnToPoolWeight@CEntityPool@@@stlpmtx_std@@@priv@stlpmtx_std@@AAEPAUSReturnToPoolWeight@CEntityPool@@AAIPAU34@1@Z 320a7650 f i EntityPool.obj
 0001:000a6650       ??$_M_allocate_and_copy@PAUSEntityIds@CEntityPool@@@?$_Impl_vector@USEntityIds@CEntityPool@@V?$allocator@USEntityIds@CEntityPool@@@stlpmtx_std@@@priv@stlpmtx_std@@AAEPAUSEntityIds@CEntityPool@@AAIPAU34@1@Z 320a7650 f i EntityPool.obj
 0001:000a6650       ??$_M_allocate_and_copy@PAUListenerRecord@?$CListenerSet@PAUIEntityPoolListener@@@@@?$_Impl_vector@UListenerRecord@?$CListenerSet@PAUIEntityPoolListener@@@@V?$allocator@UListenerRecord@?$CListenerSet@PAUIEntityPoolListener@@@@@stlpmtx_std@@@priv@stlpmtx_std@@AAEPAUListenerRecord@?$CListenerSet@PAUIEntityPoolListener@@@@AAIPAU34@1@Z 320a7650 f i EntityPoolManager.obj
 0001:000a66c0       ??$__uninitialized_fill_n@PAUSEntityIds@CEntityPool@@IU12@@priv@stlpmtx_std@@YAPAUSEntityIds@CEntityPool@@PAU23@IABU23@@Z 320a76c0 f i EntityPool.obj
 0001:000a6700       ??$__unguarded_partition@PAUSEntityIds@CEntityPool@@U12@U?$less@USEntityIds@CEntityPool@@@stlpmtx_std@@@priv@stlpmtx_std@@YAPAUSEntityIds@CEntityPool@@PAU23@0U23@U?$less@USEntityIds@CEntityPool@@@1@@Z 320a7700 f i EntityPool.obj
 0001:000a6750       ??$__insertion_sort@PAUSEntityIds@CEntityPool@@U12@U?$less@USEntityIds@CEntityPool@@@stlpmtx_std@@@priv@stlpmtx_std@@YAXPAUSEntityIds@CEntityPool@@00U?$less@USEntityIds@CEntityPool@@@1@@Z 320a7750 f i EntityPool.obj
 0001:000a67e0       ??$_M_range_insert_realloc@PAUSEntityIds@CEntityPool@@@?$_Impl_vector@USEntityIds@CEntityPool@@V?$allocator@USEntityIds@CEntityPool@@@stlpmtx_std@@@priv@stlpmtx_std@@AAEXPAUSEntityIds@CEntityPool@@00I@Z 320a77e0 f i EntityPool.obj
 0001:000a6940       ??$_M_range_insert_aux@PAI@?$_Impl_vector@IV?$allocator@I@stlpmtx_std@@@priv@stlpmtx_std@@AAEXPAI00IABU__false_type@2@@Z 320a7940 f i EntityPool.obj
 0001:000a6a40       ??$__make_heap@PAUSEntityIds@CEntityPool@@U?$less@USEntityIds@CEntityPool@@@stlpmtx_std@@U12@H@stlpmtx_std@@YAXPAUSEntityIds@CEntityPool@@0U?$less@USEntityIds@CEntityPool@@@0@0PAH@Z 320a7a40 f i EntityPool.obj
 0001:000a6b20       ??$__make_heap@PAIU?$less@I@stlpmtx_std@@IH@stlpmtx_std@@YAXPAI0U?$less@I@0@0PAH@Z 320a7b20 f i EntityPool.obj
 0001:000a6bd0       ??$__make_heap@PAUSReturnToPoolWeight@CEntityPool@@U?$less@USReturnToPoolWeight@CEntityPool@@@stlpmtx_std@@U12@H@stlpmtx_std@@YAXPAUSReturnToPoolWeight@CEntityPool@@0U?$less@USReturnToPoolWeight@CEntityPool@@@0@0PAH@Z 320a7bd0 f i EntityPool.obj
 0001:000a6cc0       ?CreateSpawnParams@CEntityPool@@QBEXAAUSEntitySpawnParams@@I_N@Z 320a7cc0 f   EntityPool.obj
 0001:000a6d30       ?reserve@?$_Impl_vector@USEntityIds@CEntityPool@@V?$allocator@USEntityIds@CEntityPool@@@stlpmtx_std@@@priv@stlpmtx_std@@QAEXI@Z 320a7d30 f i EntityPool.obj
 0001:000a6d30       ?reserve@?$_Impl_vector@USReturnToPoolWeight@CEntityPool@@V?$allocator@USReturnToPoolWeight@CEntityPool@@@stlpmtx_std@@@priv@stlpmtx_std@@QAEXI@Z 320a7d30 f i EntityPool.obj
 0001:000a6dc0       ??$find_and_erase@V?$vector@USEntityIds@CEntityPool@@V?$allocator@USEntityIds@CEntityPool@@@stlpmtx_std@@@stlpmtx_std@@I@stl@@YA_NAAV?$vector@USEntityIds@CEntityPool@@V?$allocator@USEntityIds@CEntityPool@@@stlpmtx_std@@@stlpmtx_std@@ABI@Z 320a7dc0 f i EntityPool.obj
 0001:000a6e30       ?push_back@?$vector@USEntityIds@CEntityPool@@V?$allocator@USEntityIds@CEntityPool@@@stlpmtx_std@@@stlpmtx_std@@QAEXABUSEntityIds@CEntityPool@@@Z 320a7e30 f i EntityPool.obj
 0001:000a6e30       ?push_back@?$vector@USEventPtr@CEntityEventDistributer@@V?$allocator@USEventPtr@CEntityEventDistributer@@@stlpmtx_std@@@stlpmtx_std@@QAEXABUSEventPtr@CEntityEventDistributer@@@Z 320a7e30 f i EntityEventDistributer.obj
 0001:000a6e90       ?_M_fill_insert_aux@?$_Impl_vector@USEntityIds@CEntityPool@@V?$allocator@USEntityIds@CEntityPool@@@stlpmtx_std@@@priv@stlpmtx_std@@AAEXPAUSEntityIds@CEntityPool@@IABU45@ABU__false_type@3@@Z 320a7e90 f i EntityPool.obj
 0001:000a6fd0       ??$__insertion_sort@PAIIU?$less@I@stlpmtx_std@@@priv@stlpmtx_std@@YAXPAI00U?$less@I@1@@Z 320a7fd0 f i EntityPool.obj
 0001:000a7050       ??$__insertion_sort@PAUSReturnToPoolWeight@CEntityPool@@U12@U?$less@USReturnToPoolWeight@CEntityPool@@@stlpmtx_std@@@priv@stlpmtx_std@@YAXPAUSReturnToPoolWeight@CEntityPool@@00U?$less@USReturnToPoolWeight@CEntityPool@@@1@@Z 320a8050 f i EntityPool.obj
 0001:000a7100       ??$_M_range_insert_realloc@PAI@?$_Impl_vector@IV?$allocator@I@stlpmtx_std@@@priv@stlpmtx_std@@AAEXPAI00I@Z 320a8100 f i EntityPool.obj
 0001:000a7260       ?DestroyPoolEntity@CEntityPool@@ABE_NI@Z 320a8260 f   EntityPool.obj
 0001:000a7380       ??$push_back_unique@V?$vector@USEntityIds@CEntityPool@@V?$allocator@USEntityIds@CEntityPool@@@stlpmtx_std@@@stlpmtx_std@@I@stl@@YA_NAAV?$vector@USEntityIds@CEntityPool@@V?$allocator@USEntityIds@CEntityPool@@@stlpmtx_std@@@stlpmtx_std@@ABI@Z 320a8380 f i EntityPool.obj
 0001:000a73d0       ??$sort_heap@PAUSEntityIds@CEntityPool@@U?$less@USEntityIds@CEntityPool@@@stlpmtx_std@@@stlpmtx_std@@YAXPAUSEntityIds@CEntityPool@@0U?$less@USEntityIds@CEntityPool@@@0@@Z 320a83d0 f i EntityPool.obj
 0001:000a7430       ??$sort_heap@PAIU?$less@I@stlpmtx_std@@@stlpmtx_std@@YAXPAI0U?$less@I@0@@Z 320a8430 f i EntityPool.obj
 0001:000a74d0       ??$sort_heap@PAUSReturnToPoolWeight@CEntityPool@@U?$less@USReturnToPoolWeight@CEntityPool@@@stlpmtx_std@@@stlpmtx_std@@YAXPAUSReturnToPoolWeight@CEntityPool@@0U?$less@USReturnToPoolWeight@CEntityPool@@@0@@Z 320a84d0 f i EntityPool.obj
 0001:000a7530       ??0CEntityPool@@QAE@PAVCEntityPoolManager@@I@Z 320a8530 f   EntityPool.obj
 0001:000a75f0       ?CreatePoolEntity@CEntityPool@@AAE_NAAPAVCEntity@@_N@Z 320a85f0 f   EntityPool.obj
 0001:000a77b0       ?OnPoolEntityInUse@CEntityPool@@QAEXPAVCEntity@@I@Z 320a87b0 f   EntityPool.obj
 0001:000a7920       ?OnPoolEntityReturned@CEntityPool@@QAEXPAVCEntity@@I@Z 320a8920 f   EntityPool.obj
 0001:000a7a20       ??$__partial_sort@PAUSEntityIds@CEntityPool@@U12@U?$less@USEntityIds@CEntityPool@@@stlpmtx_std@@@priv@stlpmtx_std@@YAXPAUSEntityIds@CEntityPool@@000U?$less@USEntityIds@CEntityPool@@@1@@Z 320a8a20 f i EntityPool.obj
 0001:000a7a90       ??$__partial_sort@PAIIU?$less@I@stlpmtx_std@@@priv@stlpmtx_std@@YAXPAI000U?$less@I@1@@Z 320a8a90 f i EntityPool.obj
 0001:000a7b60       ??$__partial_sort@PAUSReturnToPoolWeight@CEntityPool@@U12@U?$less@USReturnToPoolWeight@CEntityPool@@@stlpmtx_std@@@priv@stlpmtx_std@@YAXPAUSReturnToPoolWeight@CEntityPool@@000U?$less@USReturnToPoolWeight@CEntityPool@@@1@@Z 320a8b60 f i EntityPool.obj
 0001:000a7be0       ?CreatePool@CEntityPool@@QAE_NABVCEntityPoolDefinition@@@Z 320a8be0 f   EntityPool.obj
 0001:000a7e70       ?DestroyPool@CEntityPool@@QAEXXZ 320a8e70 f   EntityPool.obj
 0001:000a7fe0       ?resize@?$_Impl_vector@USEntityIds@CEntityPool@@V?$allocator@USEntityIds@CEntityPool@@@stlpmtx_std@@@priv@stlpmtx_std@@QAEXIABUSEntityIds@CEntityPool@@@Z 320a8fe0 f i EntityPool.obj
 0001:000a8080       ??1CEntityPool@@QAE@XZ     320a9080 f   EntityPool.obj
 0001:000a81a0       ??$__introsort_loop@PAUSEntityIds@CEntityPool@@U12@HU?$less@USEntityIds@CEntityPool@@@stlpmtx_std@@@priv@stlpmtx_std@@YAXPAUSEntityIds@CEntityPool@@00HU?$less@USEntityIds@CEntityPool@@@1@@Z 320a91a0 f i EntityPool.obj
 0001:000a8260       ??$__introsort_loop@PAIIHU?$less@I@stlpmtx_std@@@priv@stlpmtx_std@@YAXPAI00HU?$less@I@1@@Z 320a9260 f i EntityPool.obj
 0001:000a8340       ??$__introsort_loop@PAUSReturnToPoolWeight@CEntityPool@@U12@HU?$less@USReturnToPoolWeight@CEntityPool@@@stlpmtx_std@@@priv@stlpmtx_std@@YAXPAUSReturnToPoolWeight@CEntityPool@@00HU?$less@USReturnToPoolWeight@CEntityPool@@@1@@Z 320a9340 f i EntityPool.obj
 0001:000a8450       ?ReturnAllActive@CEntityPool@@AAEX_N@Z 320a9450 f   EntityPool.obj
 0001:000a8560       ??$sort@PAUSEntityIds@CEntityPool@@@stlpmtx_std@@YAXPAUSEntityIds@CEntityPool@@0@Z 320a9560 f i EntityPool.obj
 0001:000a85e0       ??$sort@PAI@stlpmtx_std@@YAXPAI0@Z 320a95e0 f i EntityPool.obj
 0001:000a8660       ??$sort@PAUSReturnToPoolWeight@CEntityPool@@@stlpmtx_std@@YAXPAUSReturnToPoolWeight@CEntityPool@@0@Z 320a9660 f i EntityPool.obj
 0001:000a86e0       ?ResetPool@CEntityPool@@QAEX_N@Z 320a96e0 f   EntityPool.obj
 0001:000a8700       ?ConsumePool@CEntityPool@@QAE_NAAV1@@Z 320a9700 f   EntityPool.obj
 0001:000a89f0       ?GetPoolEntityFromActiveSet@CEntityPool@@AAEPAVCEntity@@XZ 320a99f0 f   EntityPool.obj
 0001:000a8be0       ?DebugDraw@CEntityPool@@QBEXPAUIRenderer@@AAM1_N@Z 320a9be0 f   EntityPool.obj
 0001:000a92e0       ?GetEntityFromPool@CEntityPool@@QAEPAVCEntity@@AA_NI@Z 320aa2e0 f   EntityPool.obj
 0001:000a9400       ?OnLevelLoadStart@CEntityPoolDefinition@@QAEXXZ 320aa400 f   EntityPoolDefinition.obj
 0001:000a9410       ?ParseLevelXml@CEntityPoolDefinition@@QAE_NVXmlNodeRef@@@Z 320aa410 f   EntityPoolDefinition.obj
 0001:000a9460       ?ContainsEntityClass@CEntityPoolDefinition@@QBE_NPAUIEntityClass@@@Z 320aa460 f   EntityPoolDefinition.obj
 0001:000a9490       ?_M_create_node@?$_Rb_tree@PAUIEntityClass@@U?$less@PAUIEntityClass@@@stlpmtx_std@@U?$pair@QAUIEntityClass@@_N@3@U?$_Select1st@U?$pair@QAUIEntityClass@@_N@stlpmtx_std@@@priv@3@U?$_MapTraitsT@U?$pair@QAUIEntityClass@@_N@stlpmtx_std@@@63@V?$allocator@U?$pair@QAUIEntityClass@@_N@stlpmtx_std@@@3@@priv@stlpmtx_std@@IAEPAU_Rb_tree_node_base@23@ABU?$pair@QAUIEntityClass@@_N@3@@Z 320aa490 f i EntityPoolDefinition.obj
 0001:000a94e0       ?GetMemoryStatistics@CEntityPoolDefinition@@QBEXPAVICrySizer@@@Z 320aa4e0 f   EntityPoolDefinition.obj
 0001:000a9550       ?_M_insert@?$_Rb_tree@PAUIEntityClass@@U?$less@PAUIEntityClass@@@stlpmtx_std@@U?$pair@QAUIEntityClass@@_N@3@U?$_Select1st@U?$pair@QAUIEntityClass@@_N@stlpmtx_std@@@priv@3@U?$_MapTraitsT@U?$pair@QAUIEntityClass@@_N@stlpmtx_std@@@63@V?$allocator@U?$pair@QAUIEntityClass@@_N@stlpmtx_std@@@3@@priv@stlpmtx_std@@AAE?AU?$_Rb_tree_iterator@U?$pair@QAUIEntityClass@@_N@stlpmtx_std@@U?$_MapTraitsT@U?$pair@QAUIEntityClass@@_N@stlpmtx_std@@@priv@2@@23@PAU_Rb_tree_node_base@23@ABU?$pair@QAUIEntityClass@@_N@3@00@Z 320aa550 f i EntityPoolDefinition.obj
 0001:000a9610       ?insert_unique@?$_Rb_tree@PAUIEntityClass@@U?$less@PAUIEntityClass@@@stlpmtx_std@@U?$pair@QAUIEntityClass@@_N@3@U?$_Select1st@U?$pair@QAUIEntityClass@@_N@stlpmtx_std@@@priv@3@U?$_MapTraitsT@U?$pair@QAUIEntityClass@@_N@stlpmtx_std@@@63@V?$allocator@U?$pair@QAUIEntityClass@@_N@stlpmtx_std@@@3@@priv@stlpmtx_std@@QAE?AU?$pair@U?$_Rb_tree_iterator@U?$pair@QAUIEntityClass@@_N@stlpmtx_std@@U?$_MapTraitsT@U?$pair@QAUIEntityClass@@_N@stlpmtx_std@@@priv@2@@priv@stlpmtx_std@@_N@3@ABU?$pair@QAUIEntityClass@@_N@3@@Z 320aa610 f i EntityPoolDefinition.obj
 0001:000a96d0       ?DebugDraw@CEntityPoolDefinition@@QBEXPAUIRenderer@@AAM1@Z 320aa6d0 f   EntityPoolDefinition.obj
 0001:000a98b0       ?insert_unique@?$_Rb_tree@PAUIEntityClass@@U?$less@PAUIEntityClass@@@stlpmtx_std@@U?$pair@QAUIEntityClass@@_N@3@U?$_Select1st@U?$pair@QAUIEntityClass@@_N@stlpmtx_std@@@priv@3@U?$_MapTraitsT@U?$pair@QAUIEntityClass@@_N@stlpmtx_std@@@63@V?$allocator@U?$pair@QAUIEntityClass@@_N@stlpmtx_std@@@3@@priv@stlpmtx_std@@QAE?AU?$_Rb_tree_iterator@U?$pair@QAUIEntityClass@@_N@stlpmtx_std@@U?$_MapTraitsT@U?$pair@QAUIEntityClass@@_N@stlpmtx_std@@@priv@2@@23@U423@ABU?$pair@QAUIEntityClass@@_N@3@@Z 320aa8b0 f i EntityPoolDefinition.obj
 0001:000a9aa0       ??0CEntityPoolDefinition@@QAE@I@Z 320aaaa0 f   EntityPoolDefinition.obj
 0001:000a9b20       ?LoadFromXml@CEntityPoolDefinition@@QAE_NPAVCEntitySystem@@VXmlNodeRef@@@Z 320aab20 f   EntityPoolDefinition.obj
 0001:000a9dc0       ??$?APAUIEntityClass@@@?$map@PAUIEntityClass@@_NU?$less@PAUIEntityClass@@@stlpmtx_std@@V?$allocator@U?$pair@QAUIEntityClass@@_N@stlpmtx_std@@@3@@stlpmtx_std@@QAEAA_NABQAUIEntityClass@@@Z 320aadc0 f i EntityPoolDefinition.obj
 0001:000a9e40       ?TestEntityClassSignature@CEntityPoolDefinition@@QBE_NPAVCEntitySystem@@PAUIEntityClass@@ABVCEntityPoolSignature@@@Z 320aae40 f   EntityPoolDefinition.obj
 0001:000aa010       ??_EIEntityPoolManager@@UAEPAXI@Z 320ab010 f i EntityPoolManager.obj
 0001:000aa010       ??_GIEntityPoolManager@@UAEPAXI@Z 320ab010 f i EntityPoolManager.obj
 0001:000aa040       ?IsUsingPools@CEntityPoolManager@@QBE_NXZ 320ab040 f   EntityPoolManager.obj
 0001:000aa080       ?IsPreparingEntity@CEntityPoolManager@@UBE_NAAUSPreparingParams@IEntityPoolManager@@@Z 320ab080 f   EntityPoolManager.obj
 0001:000aa0b0       ??$PushFuncParam@TScriptHandle@@@IScriptSystem@@QAEXABTScriptHandle@@@Z 320ab0b0 f i EntityPoolManager.obj
 0001:000aa110       ??$EndCall@M@IScriptSystem@@QAE_NAAM@Z 320ab110 f i EntityPoolManager.obj
 0001:000aa190       ??$__find@PAUListenerRecord@?$CListenerSet@PAUIEntityPoolListener@@@@U12@@priv@stlpmtx_std@@YAPAUListenerRecord@?$CListenerSet@PAUIEntityPoolListener@@@@PAU23@0ABU23@ABUrandom_access_iterator_tag@1@@Z 320ab190 f i EntityPoolManager.obj
 0001:000aa190       ??$__find@PBUListenerRecord@?$CListenerSet@PAUIEntityPoolListener@@@@PAUIEntityPoolListener@@@priv@stlpmtx_std@@YAPBUListenerRecord@?$CListenerSet@PAUIEntityPoolListener@@@@PBU23@0ABQAUIEntityPoolListener@@ABUrandom_access_iterator_tag@1@@Z 320ab190 f i EntityPoolManager.obj
 0001:000aa200       ?RecursiveParseTableFromXml@?A0xf71e8af1@@YA_NVXmlNodeRef@@AAVSmartScriptTable@@@Z 320ab200 f   EntityPoolManager.obj
 0001:000aa3f0       ?CreateTableFromXml@CEntityPoolManager@@CA_NVXmlNodeRef@@AAVSmartScriptTable@@@Z 320ab3f0 f   EntityPoolManager.obj
 0001:000aa480       ??1?$_Deque_base@USEntityPrepareRequest@CEntityPoolManager@@V?$allocator@USEntityPrepareRequest@CEntityPoolManager@@@stlpmtx_std@@@priv@stlpmtx_std@@QAE@XZ 320ab480 f i EntityPoolManager.obj
 0001:000aa4d0       ?GetReturnToPoolWeight@CEntityPoolManager@@QBEMPAVCEntity@@_N@Z 320ab4d0 f   EntityPoolManager.obj
 0001:000aa5d0       ??$__ucopy@U?$_Deque_iterator@USEntityPrepareRequest@CEntityPoolManager@@U?$_Const_traits@USEntityPrepareRequest@CEntityPoolManager@@@stlpmtx_std@@@priv@stlpmtx_std@@U?$_Deque_iterator@USEntityPrepareRequest@CEntityPoolManager@@U?$_Nonconst_traits@USEntityPrepareRequest@CEntityPoolManager@@@stlpmtx_std@@@23@H@priv@stlpmtx_std@@YA?AU?$_Deque_iterator@USEntityPrepareRequest@CEntityPoolManager@@U?$_Nonconst_traits@USEntityPrepareRequest@CEntityPoolManager@@@stlpmtx_std@@@01@U?$_Deque_iterator@USEntityPrepareRequest@CEntityPoolManager@@U?$_Const_traits@USEntityPrepareRequest@CEntityPoolManager@@@stlpmtx_std@@@01@0U201@ABUrandom_access_iterator_tag@1@PAH@Z 320ab5d0 f i EntityPoolManager.obj
 0001:000aa6b0       ?_M_set@?$_Impl_vector@UListenerRecord@?$CListenerSet@PAUIEntityPoolListener@@@@V?$allocator@UListenerRecord@?$CListenerSet@PAUIEntityPoolListener@@@@@stlpmtx_std@@@priv@stlpmtx_std@@AAEXPAUListenerRecord@?$CListenerSet@PAUIEntityPoolListener@@@@00@Z 320ab6b0 f i EntityPoolManager.obj
 0001:000aa6b0       ?_M_set@?$_Impl_vector@USEntityAttachment@@V?$allocator@USEntityAttachment@@@stlpmtx_std@@@priv@stlpmtx_std@@AAEXPAUSEntityAttachment@@00@Z 320ab6b0 f i EntityLoadManager.obj
 0001:000aa6b0       ?_M_set@?$_Impl_vector@USReturnToPoolWeight@CEntityPool@@V?$allocator@USReturnToPoolWeight@CEntityPool@@@stlpmtx_std@@@priv@stlpmtx_std@@AAEXPAUSReturnToPoolWeight@CEntityPool@@00@Z 320ab6b0 f i EntityPool.obj
 0001:000aa6b0       ?_M_set@?$_Impl_vector@PAXV?$allocator@PAX@stlpmtx_std@@@priv@stlpmtx_std@@AAEXPAPAX00@Z 320ab6b0 f i AreaSolid.obj
 0001:000aa6b0       ?_M_set@?$_Impl_vector@HV?$allocator@H@stlpmtx_std@@@priv@stlpmtx_std@@AAEXPAH00@Z 320ab6b0 f i AreaManager.obj
 0001:000aa6b0       ?_M_set@?$_Impl_vector@MV?$allocator@M@stlpmtx_std@@@priv@stlpmtx_std@@AAEXPAM00@Z 320ab6b0 f i ScriptBind_Entity.obj
 0001:000aa6b0       ?_M_set@?$_Impl_vector@USEntityScriptEvent@@V?$allocator@USEntityScriptEvent@@@stlpmtx_std@@@priv@stlpmtx_std@@AAEXPAUSEntityScriptEvent@@00@Z 320ab6b0 f i EntityScript.obj
 0001:000aa6b0       ?_M_set@?$_Impl_vector@UOnEventSink@CEntitySystem@@V?$STLGlobalAllocator@UOnEventSink@CEntitySystem@@@stl@@@priv@stlpmtx_std@@AAEXPAUOnEventSink@CEntitySystem@@00@Z 320ab6b0 f i EntitySystem.obj
 0001:000aa6b0       ?_M_set@?$_Impl_vector@USScriptState@@V?$allocator@USScriptState@@@stlpmtx_std@@@priv@stlpmtx_std@@AAEXPAUSScriptState@@00@Z 320ab6b0 f i EntityScript.obj
 0001:000aa6b0       ?_M_set@?$_Impl_vector@USEntityTimerEvent@@V?$allocator@USEntityTimerEvent@@@stlpmtx_std@@@priv@stlpmtx_std@@AAEXPAUSEntityTimerEvent@@00@Z 320ab6b0 f i EntitySystem.obj
 0001:000aa6b0       ?_M_set@?$_Impl_vector@U?$Vec3_tpl@M@@V?$allocator@U?$Vec3_tpl@M@@@stlpmtx_std@@@priv@stlpmtx_std@@AAEXPAU?$Vec3_tpl@M@@00@Z 320ab6b0 f i AreaSolid.obj
 0001:000aa6b0       ?_M_set@?$_Impl_vector@USQueuedFlowGraph@CEntityLoadManager@@V?$allocator@USQueuedFlowGraph@CEntityLoadManager@@@stlpmtx_std@@@priv@stlpmtx_std@@AAEXPAUSQueuedFlowGraph@CEntityLoadManager@@00@Z 320ab6b0 f i EntityLoadManager.obj
 0001:000aa6b0       ?_M_set@?$_Impl_vector@USEntityIds@CEntityPool@@V?$allocator@USEntityIds@CEntityPool@@@stlpmtx_std@@@priv@stlpmtx_std@@AAEXPAUSEntityIds@CEntityPool@@00@Z 320ab6b0 f i EntityPool.obj
 0001:000aa710       ??1SDynamicSerializeHelper@CEntityPoolManager@@QAE@XZ 320ab710 f i EntityPoolManager.obj
 0001:000aa7c0       ?OnLevelLoadStart@CEntityPoolManager@@QAEXXZ 320ab7c0 f   EntityPoolManager.obj
 0001:000aa860       ?IsClassDefaultBookmarked@CEntityPoolManager@@UBE_NPBD@Z 320ab860 f   EntityPoolManager.obj
 0001:000aa900       ?IsClassUsingPools@CEntityPoolManager@@QBE_NPAUIEntityClass@@@Z 320ab900 f   EntityPoolManager.obj
 0001:000aa970       ?IsClassForcedBookmarked@CEntityPoolManager@@QBE_NPAUIEntityClass@@@Z 320ab970 f   EntityPoolManager.obj
 0001:000aa9f0       ?ResetPools@CEntityPoolManager@@UAEX_N@Z 320ab9f0 f   EntityPoolManager.obj
 0001:000aaa70       ?GetPoolSizeByClass@CEntityPoolManager@@QBEIPBD@Z 320aba70 f   EntityPoolManager.obj
 0001:000aab00       ?GetPoolEntity@CEntityPoolManager@@AAEPAVCEntity@@PAUIEntityClass@@IAAIAA_N2@Z 320abb00 f   EntityPoolManager.obj
 0001:000aac40       ?_M_initialize_map@?$_Deque_base@USEntityPrepareRequest@CEntityPoolManager@@V?$allocator@USEntityPrepareRequest@CEntityPoolManager@@@stlpmtx_std@@@priv@stlpmtx_std@@IAEXI@Z 320abc40 f i EntityPoolManager.obj
 0001:000aad30       ??$__ucopy@U?$_Deque_iterator@USEntityPrepareRequest@CEntityPoolManager@@U?$_Const_traits@USEntityPrepareRequest@CEntityPoolManager@@@stlpmtx_std@@@priv@stlpmtx_std@@U?$_Deque_iterator@USEntityPrepareRequest@CEntityPoolManager@@U?$_Nonconst_traits@USEntityPrepareRequest@CEntityPoolManager@@@stlpmtx_std@@@23@@priv@stlpmtx_std@@YA?AU?$_Deque_iterator@USEntityPrepareRequest@CEntityPoolManager@@U?$_Nonconst_traits@USEntityPrepareRequest@CEntityPoolManager@@@stlpmtx_std@@@01@U?$_Deque_iterator@USEntityPrepareRequest@CEntityPoolManager@@U?$_Const_traits@USEntityPrepareRequest@CEntityPoolManager@@@stlpmtx_std@@@01@0U201@@Z 320abd30 f i EntityPoolManager.obj
 0001:000aada0       ?_M_reallocate_map@?$_Impl_deque@USEntityPrepareRequest@CEntityPoolManager@@V?$allocator@USEntityPrepareRequest@CEntityPoolManager@@@stlpmtx_std@@@priv@stlpmtx_std@@IAEXI_N@Z 320abda0 f i EntityPoolManager.obj
 0001:000aaf00       ??$__ucopy@PBV?$CryStringT@D@@PAV1@H@priv@stlpmtx_std@@YAPAV?$CryStringT@D@@PBV2@0PAV2@ABUrandom_access_iterator_tag@1@PAH@Z 320abf00 f i EntityPoolManager.obj
 0001:000aaf50       ?_M_create_node@?$_Rb_tree@IU?$less@I@stlpmtx_std@@U?$pair@$$CBIPAVCEntityPool@@@2@U?$_Select1st@U?$pair@$$CBIPAVCEntityPool@@@stlpmtx_std@@@priv@2@U?$_MapTraitsT@U?$pair@$$CBIPAVCEntityPool@@@stlpmtx_std@@@52@V?$allocator@U?$pair@$$CBIPAVCEntityPool@@@stlpmtx_std@@@2@@priv@stlpmtx_std@@IAEPAU_Rb_tree_node_base@23@ABU?$pair@$$CBIPAVCEntityPool@@@3@@Z 320abf50 f i EntityPoolManager.obj
 0001:000aaf50       ?_M_create_node@?$_Rb_tree@IU?$less@I@stlpmtx_std@@U?$pair@$$CBIPAUIEntityEventListener@@@2@U?$_Select1st@U?$pair@$$CBIPAUIEntityEventListener@@@stlpmtx_std@@@priv@2@U?$_MultimapTraitsT@U?$pair@$$CBIPAUIEntityEventListener@@@stlpmtx_std@@@52@V?$allocator@U?$pair@$$CBIPAUIEntityEventListener@@@stlpmtx_std@@@2@@priv@stlpmtx_std@@IAEPAU_Rb_tree_node_base@23@ABU?$pair@$$CBIPAUIEntityEventListener@@@3@@Z 320abf50 f i EntitySystem.obj
 0001:000aaf50       ?_M_create_node@?$_Rb_tree@IU?$less@I@stlpmtx_std@@U?$pair@$$CBIPAVCEntity@@@2@U?$_Select1st@U?$pair@$$CBIPAVCEntity@@@stlpmtx_std@@@priv@2@U?$_MapTraitsT@U?$pair@$$CBIPAVCEntity@@@stlpmtx_std@@@52@V?$allocator@U?$pair@$$CBIPAVCEntity@@@stlpmtx_std@@@2@@priv@stlpmtx_std@@IAEPAU_Rb_tree_node_base@23@ABU?$pair@$$CBIPAVCEntity@@@3@@Z 320abf50 f i EntitySystem.obj
 0001:000aaf50       ?_M_create_node@?$_Rb_tree@IU?$less@I@stlpmtx_std@@U?$pair@$$CBIPAVCEntityPoolDefinition@@@2@U?$_Select1st@U?$pair@$$CBIPAVCEntityPoolDefinition@@@stlpmtx_std@@@priv@2@U?$_MapTraitsT@U?$pair@$$CBIPAVCEntityPoolDefinition@@@stlpmtx_std@@@52@V?$allocator@U?$pair@$$CBIPAVCEntityPoolDefinition@@@stlpmtx_std@@@2@@priv@stlpmtx_std@@IAEPAU_Rb_tree_node_base@23@ABU?$pair@$$CBIPAVCEntityPoolDefinition@@@3@@Z 320abf50 f i EntityPoolManager.obj
 0001:000aaf50       ?_M_create_node@?$_Rb_tree@PBDU?$less_stricmp@PBD@stl@@U?$pair@QBDI@stlpmtx_std@@U?$_Select1st@U?$pair@QBDI@stlpmtx_std@@@priv@4@U?$_MultimapTraitsT@U?$pair@QBDI@stlpmtx_std@@@64@V?$allocator@U?$pair@QBDI@stlpmtx_std@@@4@@priv@stlpmtx_std@@IAEPAU_Rb_tree_node_base@23@ABU?$pair@QBDI@3@@Z 320abf50 f i EntitySystem.obj
 0001:000aafa0       ??$__copy@PBV?$CryStringT@D@@PAV1@H@priv@stlpmtx_std@@YAPAV?$CryStringT@D@@PBV2@0PAV2@ABUrandom_access_iterator_tag@1@PAH@Z 320abfa0 f i EntityPoolManager.obj
 0001:000aafa0       ??$__copy@PAV?$CryStringT@D@@PAV1@H@priv@stlpmtx_std@@YAPAV?$CryStringT@D@@PAV2@00ABUrandom_access_iterator_tag@1@PAH@Z 320abfa0 f i EntityPoolManager.obj
 0001:000ab070       ??0SDynamicSerializeHelper@CEntityPoolManager@@QAE@ABUSEntityBookmark@1@@Z 320ac070 f   EntityPoolManager.obj
 0001:000ab130       ?GetMemoryStatistics@CEntityPoolManager@@QBEXPAVICrySizer@@@Z 320ac130 f   EntityPoolManager.obj
 0001:000ab2d0       ?GetEntityPoolDefinition@CEntityPoolManager@@QBEPBVCEntityPoolDefinition@@I@Z 320ac2d0 f   EntityPoolManager.obj
 0001:000ab320       ?OnPoolEntityInUse@CEntityPoolManager@@QAEXPAVCEntity@@I@Z 320ac320 f   EntityPoolManager.obj
 0001:000ab430       ?ResetBookmark@CEntityPoolManager@@UAEXI@Z 320ac430 f   EntityPoolManager.obj
 0001:000ab480       ?IsEntityBookmarked@CEntityPoolManager@@UBE_NI@Z 320ac480 f   EntityPoolManager.obj
 0001:000ab4c0       ?GetBookmarkedEntityName@CEntityPoolManager@@UBEPBDI@Z 320ac4c0 f   EntityPoolManager.obj
 0001:000ab510       ??1SEntityBookmark@CEntityPoolManager@@QAE@XZ 320ac510 f i EntityPoolManager.obj
 0001:000ab5b0       ?DebugDraw@CEntityPoolManager@@QBEXXZ 320ac5b0 f   EntityPoolManager.obj
 0001:000ab810       ?pop@?$queue@USEntityPrepareRequest@CEntityPoolManager@@V?$deque@USEntityPrepareRequest@CEntityPoolManager@@V?$allocator@USEntityPrepareRequest@CEntityPoolManager@@@stlpmtx_std@@@stlpmtx_std@@@stlpmtx_std@@QAEXXZ 320ac810 f i EntityPoolManager.obj
 0001:000ab860       ??0?$_Vector_base@USEntityAttachment@@V?$allocator@USEntityAttachment@@@stlpmtx_std@@@priv@stlpmtx_std@@QAE@IABV?$allocator@USEntityAttachment@@@2@@Z 320ac860 f i EntityPoolManager.obj
 0001:000ab920       ?_M_insert@?$_Rb_tree@IU?$less@I@stlpmtx_std@@U?$pair@$$CBIPAUIEntityEventListener@@@2@U?$_Select1st@U?$pair@$$CBIPAUIEntityEventListener@@@stlpmtx_std@@@priv@2@U?$_MultimapTraitsT@U?$pair@$$CBIPAUIEntityEventListener@@@stlpmtx_std@@@52@V?$allocator@U?$pair@$$CBIPAUIEntityEventListener@@@stlpmtx_std@@@2@@priv@stlpmtx_std@@AAE?AU?$_Rb_tree_iterator@U?$pair@$$CBIPAUIEntityEventListener@@@stlpmtx_std@@U?$_MultimapTraitsT@U?$pair@$$CBIPAUIEntityEventListener@@@stlpmtx_std@@@priv@2@@23@PAU_Rb_tree_node_base@23@ABU?$pair@$$CBIPAUIEntityEventListener@@@3@00@Z 320ac920 f i EntitySystem.obj
 0001:000ab920       ?_M_insert@?$_Rb_tree@IU?$less@I@stlpmtx_std@@U?$pair@$$CBIPAVCEntityPool@@@2@U?$_Select1st@U?$pair@$$CBIPAVCEntityPool@@@stlpmtx_std@@@priv@2@U?$_MapTraitsT@U?$pair@$$CBIPAVCEntityPool@@@stlpmtx_std@@@52@V?$allocator@U?$pair@$$CBIPAVCEntityPool@@@stlpmtx_std@@@2@@priv@stlpmtx_std@@AAE?AU?$_Rb_tree_iterator@U?$pair@$$CBIPAVCEntityPool@@@stlpmtx_std@@U?$_MapTraitsT@U?$pair@$$CBIPAVCEntityPool@@@stlpmtx_std@@@priv@2@@23@PAU_Rb_tree_node_base@23@ABU?$pair@$$CBIPAVCEntityPool@@@3@00@Z 320ac920 f i EntityPoolManager.obj
 0001:000ab920       ?_M_insert@?$_Rb_tree@IU?$less@I@stlpmtx_std@@U?$pair@$$CBIPAVCEntity@@@2@U?$_Select1st@U?$pair@$$CBIPAVCEntity@@@stlpmtx_std@@@priv@2@U?$_MapTraitsT@U?$pair@$$CBIPAVCEntity@@@stlpmtx_std@@@52@V?$allocator@U?$pair@$$CBIPAVCEntity@@@stlpmtx_std@@@2@@priv@stlpmtx_std@@AAE?AU?$_Rb_tree_iterator@U?$pair@$$CBIPAVCEntity@@@stlpmtx_std@@U?$_MapTraitsT@U?$pair@$$CBIPAVCEntity@@@stlpmtx_std@@@priv@2@@23@PAU_Rb_tree_node_base@23@ABU?$pair@$$CBIPAVCEntity@@@3@00@Z 320ac920 f i EntitySystem.obj
 0001:000ab920       ?_M_insert@?$_Rb_tree@IU?$less@I@stlpmtx_std@@U?$pair@$$CBIPAVCEntityPoolDefinition@@@2@U?$_Select1st@U?$pair@$$CBIPAVCEntityPoolDefinition@@@stlpmtx_std@@@priv@2@U?$_MapTraitsT@U?$pair@$$CBIPAVCEntityPoolDefinition@@@stlpmtx_std@@@52@V?$allocator@U?$pair@$$CBIPAVCEntityPoolDefinition@@@stlpmtx_std@@@2@@priv@stlpmtx_std@@AAE?AU?$_Rb_tree_iterator@U?$pair@$$CBIPAVCEntityPoolDefinition@@@stlpmtx_std@@U?$_MapTraitsT@U?$pair@$$CBIPAVCEntityPoolDefinition@@@stlpmtx_std@@@priv@2@@23@PAU_Rb_tree_node_base@23@ABU?$pair@$$CBIPAVCEntityPoolDefinition@@@3@00@Z 320ac920 f i EntityPoolManager.obj
 0001:000ab9e0       ?insert_unique@?$_Rb_tree@IU?$less@I@stlpmtx_std@@U?$pair@$$CBIPAVCEntityPool@@@2@U?$_Select1st@U?$pair@$$CBIPAVCEntityPool@@@stlpmtx_std@@@priv@2@U?$_MapTraitsT@U?$pair@$$CBIPAVCEntityPool@@@stlpmtx_std@@@52@V?$allocator@U?$pair@$$CBIPAVCEntityPool@@@stlpmtx_std@@@2@@priv@stlpmtx_std@@QAE?AU?$pair@U?$_Rb_tree_iterator@U?$pair@$$CBIPAVCEntityPool@@@stlpmtx_std@@U?$_MapTraitsT@U?$pair@$$CBIPAVCEntityPool@@@stlpmtx_std@@@priv@2@@priv@stlpmtx_std@@_N@3@ABU?$pair@$$CBIPAVCEntityPool@@@3@@Z 320ac9e0 f i EntityPoolManager.obj
 0001:000ab9e0       ?insert_unique@?$_Rb_tree@IU?$less@I@stlpmtx_std@@U?$pair@$$CBIPAVCEntityPoolDefinition@@@2@U?$_Select1st@U?$pair@$$CBIPAVCEntityPoolDefinition@@@stlpmtx_std@@@priv@2@U?$_MapTraitsT@U?$pair@$$CBIPAVCEntityPoolDefinition@@@stlpmtx_std@@@52@V?$allocator@U?$pair@$$CBIPAVCEntityPoolDefinition@@@stlpmtx_std@@@2@@priv@stlpmtx_std@@QAE?AU?$pair@U?$_Rb_tree_iterator@U?$pair@$$CBIPAVCEntityPoolDefinition@@@stlpmtx_std@@U?$_MapTraitsT@U?$pair@$$CBIPAVCEntityPoolDefinition@@@stlpmtx_std@@@priv@2@@priv@stlpmtx_std@@_N@3@ABU?$pair@$$CBIPAVCEntityPoolDefinition@@@3@@Z 320ac9e0 f i EntityPoolManager.obj
 0001:000ab9e0       ?insert_unique@?$_Rb_tree@IU?$less@I@stlpmtx_std@@U?$pair@$$CBIPAVCEntity@@@2@U?$_Select1st@U?$pair@$$CBIPAVCEntity@@@stlpmtx_std@@@priv@2@U?$_MapTraitsT@U?$pair@$$CBIPAVCEntity@@@stlpmtx_std@@@52@V?$allocator@U?$pair@$$CBIPAVCEntity@@@stlpmtx_std@@@2@@priv@stlpmtx_std@@QAE?AU?$pair@U?$_Rb_tree_iterator@U?$pair@$$CBIPAVCEntity@@@stlpmtx_std@@U?$_MapTraitsT@U?$pair@$$CBIPAVCEntity@@@stlpmtx_std@@@priv@2@@priv@stlpmtx_std@@_N@3@ABU?$pair@$$CBIPAVCEntity@@@3@@Z 320ac9e0 f i EntitySystem.obj
 0001:000abaa0       ??4?$_Impl_vector@USEventPtr@CEntityEventDistributer@@V?$allocator@USEventPtr@CEntityEventDistributer@@@stlpmtx_std@@@priv@stlpmtx_std@@QAEAAV012@ABV012@@Z 320acaa0 f i EntityEventDistributer.obj
 0001:000abaa0       ??4?$_Impl_vector@UListenerRecord@?$CListenerSet@PAUIEntityPoolListener@@@@V?$allocator@UListenerRecord@?$CListenerSet@PAUIEntityPoolListener@@@@@stlpmtx_std@@@priv@stlpmtx_std@@QAEAAV012@ABV012@@Z 320acaa0 f i EntityPoolManager.obj
 0001:000abbb0       ??$__destroy_range_aux@PAV?$CryStringT@D@@V1@@stlpmtx_std@@YAXPAV?$CryStringT@D@@00ABU__false_type@0@@Z 320acbb0 f i EntityPoolManager.obj
 0001:000abc00       ??$__destroy_range_aux@V?$reverse_iterator@PAV?$CryStringT@D@@@stlpmtx_std@@V?$CryStringT@D@@@stlpmtx_std@@YAXV?$reverse_iterator@PAV?$CryStringT@D@@@0@0PAV?$CryStringT@D@@ABU__false_type@0@@Z 320acc00 f i EntityPoolManager.obj
 0001:000abc50       ?ReleasePools@CEntityPoolManager@@AAEXXZ 320acc50 f   EntityPoolManager.obj
 0001:000abd00       ?DumpEntityBookmarks@CEntityPoolManager@@QBEXPBD_N@Z 320acd00 f   EntityPoolManager.obj
 0001:000ac210       ??0?$_Impl_deque@USEntityPrepareRequest@CEntityPoolManager@@V?$allocator@USEntityPrepareRequest@CEntityPoolManager@@@stlpmtx_std@@@priv@stlpmtx_std@@QAE@ABV012@@Z 320ad210 f i EntityPoolManager.obj
 0001:000ac300       ??0?$_Impl_vector@USEntityAttachment@@V?$allocator@USEntityAttachment@@@stlpmtx_std@@@priv@stlpmtx_std@@QAE@ABV012@@Z 320ad300 f i EntityPoolManager.obj
 0001:000ac370       ?_M_push_back_aux_v@?$_Impl_deque@USEntityPrepareRequest@CEntityPoolManager@@V?$allocator@USEntityPrepareRequest@CEntityPoolManager@@@stlpmtx_std@@@priv@stlpmtx_std@@IAEXABUSEntityPrepareRequest@CEntityPoolManager@@@Z 320ad370 f i EntityPoolManager.obj
 0001:000ac3e0       ?insert_unique@?$_Rb_tree@IU?$less@I@stlpmtx_std@@U?$pair@$$CBIPAVCEntity@@@2@U?$_Select1st@U?$pair@$$CBIPAVCEntity@@@stlpmtx_std@@@priv@2@U?$_MapTraitsT@U?$pair@$$CBIPAVCEntity@@@stlpmtx_std@@@52@V?$allocator@U?$pair@$$CBIPAVCEntity@@@stlpmtx_std@@@2@@priv@stlpmtx_std@@QAE?AU?$_Rb_tree_iterator@U?$pair@$$CBIPAVCEntity@@@stlpmtx_std@@U?$_MapTraitsT@U?$pair@$$CBIPAVCEntity@@@stlpmtx_std@@@priv@2@@23@U423@ABU?$pair@$$CBIPAVCEntity@@@3@@Z 320ad3e0 f i EntitySystem.obj
 0001:000ac3e0       ?insert_unique@?$_Rb_tree@IU?$less@I@stlpmtx_std@@U?$pair@$$CBIPAVCEntityPool@@@2@U?$_Select1st@U?$pair@$$CBIPAVCEntityPool@@@stlpmtx_std@@@priv@2@U?$_MapTraitsT@U?$pair@$$CBIPAVCEntityPool@@@stlpmtx_std@@@52@V?$allocator@U?$pair@$$CBIPAVCEntityPool@@@stlpmtx_std@@@2@@priv@stlpmtx_std@@QAE?AU?$_Rb_tree_iterator@U?$pair@$$CBIPAVCEntityPool@@@stlpmtx_std@@U?$_MapTraitsT@U?$pair@$$CBIPAVCEntityPool@@@stlpmtx_std@@@priv@2@@23@U423@ABU?$pair@$$CBIPAVCEntityPool@@@3@@Z 320ad3e0 f i EntityPoolManager.obj
 0001:000ac3e0       ?insert_unique@?$_Rb_tree@IU?$less@I@stlpmtx_std@@U?$pair@$$CBIPAVCEntityPoolDefinition@@@2@U?$_Select1st@U?$pair@$$CBIPAVCEntityPoolDefinition@@@stlpmtx_std@@@priv@2@U?$_MapTraitsT@U?$pair@$$CBIPAVCEntityPoolDefinition@@@stlpmtx_std@@@52@V?$allocator@U?$pair@$$CBIPAVCEntityPoolDefinition@@@stlpmtx_std@@@2@@priv@stlpmtx_std@@QAE?AU?$_Rb_tree_iterator@U?$pair@$$CBIPAVCEntityPoolDefinition@@@stlpmtx_std@@U?$_MapTraitsT@U?$pair@$$CBIPAVCEntityPoolDefinition@@@stlpmtx_std@@@priv@2@@23@U423@ABU?$pair@$$CBIPAVCEntityPoolDefinition@@@3@@Z 320ad3e0 f i EntityPoolManager.obj
 0001:000ac5d0       ?_M_erase@?$_Impl_vector@V?$CryStringT@D@@V?$allocator@V?$CryStringT@D@@@stlpmtx_std@@@priv@stlpmtx_std@@AAEPAV?$CryStringT@D@@PAV4@ABU__false_type@3@@Z 320ad5d0 f i EntityPoolManager.obj
 0001:000ac650       ??$find_and_erase_all@V?$vector@UListenerRecord@?$CListenerSet@PAUIEntityPoolListener@@@@V?$allocator@UListenerRecord@?$CListenerSet@PAUIEntityPoolListener@@@@@stlpmtx_std@@@stlpmtx_std@@@stl@@YAXAAV?$vector@UListenerRecord@?$CListenerSet@PAUIEntityPoolListener@@@@V?$allocator@UListenerRecord@?$CListenerSet@PAUIEntityPoolListener@@@@@stlpmtx_std@@@stlpmtx_std@@ABUListenerRecord@?$CListenerSet@PAUIEntityPoolListener@@@@@Z 320ad650 f i EntityPoolManager.obj
 0001:000ac6e0       ??$reconstruct@V?$vector@UListenerRecord@?$CListenerSet@PAUIEntityPoolListener@@@@V?$allocator@UListenerRecord@?$CListenerSet@PAUIEntityPoolListener@@@@@stlpmtx_std@@@stlpmtx_std@@@stl@@YAXAAV?$vector@UListenerRecord@?$CListenerSet@PAUIEntityPoolListener@@@@V?$allocator@UListenerRecord@?$CListenerSet@PAUIEntityPoolListener@@@@@stlpmtx_std@@@stlpmtx_std@@@Z 320ad6e0 f i EntityPoolManager.obj
 0001:000ac6e0       ??$reconstruct@V?$vector@HV?$allocator@H@stlpmtx_std@@@stlpmtx_std@@@stl@@YAXAAV?$vector@HV?$allocator@H@stlpmtx_std@@@stlpmtx_std@@@Z 320ad6e0 f i AreaManager.obj
 0001:000ac6e0       ??$reconstruct@V?$vector@IV?$allocator@I@stlpmtx_std@@@stlpmtx_std@@@stl@@YAXAAV?$vector@IV?$allocator@I@stlpmtx_std@@@stlpmtx_std@@@Z 320ad6e0 f i EntitySystem.obj
 0001:000ac6e0       ??$reconstruct@V?$vector@PAVCEntity@@V?$allocator@PAVCEntity@@@stlpmtx_std@@@stlpmtx_std@@@stl@@YAXAAV?$vector@PAVCEntity@@V?$allocator@PAVCEntity@@@stlpmtx_std@@@stlpmtx_std@@@Z 320ad6e0 f i EntitySystem.obj
 0001:000ac6e0       ??$reconstruct@V?$vector@USEntityTimerEvent@@V?$allocator@USEntityTimerEvent@@@stlpmtx_std@@@stlpmtx_std@@@stl@@YAXAAV?$vector@USEntityTimerEvent@@V?$allocator@USEntityTimerEvent@@@stlpmtx_std@@@stlpmtx_std@@@Z 320ad6e0 f i EntitySystem.obj
 0001:000ac6e0       ??$reconstruct@V?$vector@PAUIEntity@@V?$allocator@PAUIEntity@@@stlpmtx_std@@@stlpmtx_std@@@stl@@YAXAAV?$vector@PAUIEntity@@V?$allocator@PAUIEntity@@@stlpmtx_std@@@stlpmtx_std@@@Z 320ad6e0 f i PartitionGrid.obj
 0001:000ac740       ??0SEntityBookmark@CEntityPoolManager@@QAE@ABUSEntityLoadParams@@_NPAUISerializeHelper@@@Z 320ad740 f   EntityPoolManager.obj
 0001:000ac820       ??1CEntityPoolDefinition@@QAE@XZ 320ad820 f i EntityPoolManager.obj
 0001:000ac8c0       ?Make@PathUtil@@YA?AV?$CryStringT@D@@ABV2@0@Z 320ad8c0 f i EntityPoolManager.obj
 0001:000ac930       ?Make@PathUtil@@YA?AV?$CryStringT@D@@QBD0@Z 320ad930 f i EntityPoolManager.obj
 0001:000ac9c0       ??$_M_allocate_and_copy@PBV?$CryStringT@D@@@?$_Impl_vector@V?$CryStringT@D@@V?$allocator@V?$CryStringT@D@@@stlpmtx_std@@@priv@stlpmtx_std@@AAEPAV?$CryStringT@D@@AAIPBV3@1@Z 320ad9c0 f i EntityPoolManager.obj
 0001:000aca30       ?Serialize@SDynamicSerializeHelper@CEntityPoolManager@@QAEXV?$CSerializeWrapper@UISerialize@@@@@Z 320ada30 f   EntityPoolManager.obj
 0001:000acad0       ?OnLoadLevel@CEntityPoolManager@@QAE_NPBD@Z 320adad0 f   EntityPoolManager.obj
 0001:000acc70       ??0SEntityBookmark@CEntityPoolManager@@QAE@ABU01@@Z 320adc70 f i EntityPoolManager.obj
 0001:000acd30       ?_M_erase@?$_Rb_tree@IU?$less@I@stlpmtx_std@@U?$pair@$$CBIUSEntityBookmark@CEntityPoolManager@@@2@U?$_Select1st@U?$pair@$$CBIUSEntityBookmark@CEntityPoolManager@@@stlpmtx_std@@@priv@2@U?$_MapTraitsT@U?$pair@$$CBIUSEntityBookmark@CEntityPoolManager@@@stlpmtx_std@@@52@V?$allocator@U?$pair@$$CBIUSEntityBookmark@CEntityPoolManager@@@stlpmtx_std@@@2@@priv@stlpmtx_std@@AAEXPAU_Rb_tree_node_base@23@@Z 320add30 f i EntityPoolManager.obj
 0001:000acd70       ??$?AI@?$map@IPAVCEntity@@U?$less@I@stlpmtx_std@@V?$allocator@U?$pair@$$CBIPAVCEntity@@@stlpmtx_std@@@3@@stlpmtx_std@@QAEAAPAVCEntity@@ABI@Z 320add70 f i EntitySystem.obj
 0001:000acd70       ??$?AI@?$map@IPAVCEntityPoolDefinition@@U?$less@I@stlpmtx_std@@V?$allocator@U?$pair@$$CBIPAVCEntityPoolDefinition@@@stlpmtx_std@@@3@@stlpmtx_std@@QAEAAPAVCEntityPoolDefinition@@ABI@Z 320add70 f i EntityPoolManager.obj
 0001:000acdf0       ?ReleaseDefinitions@CEntityPoolManager@@AAEXXZ 320addf0 f   EntityPoolManager.obj
 0001:000acea0       ?PreparePools@CEntityPoolManager@@AAE_NXZ 320adea0 f   EntityPoolManager.obj
 0001:000ad2c0       ??4?$_Impl_vector@V?$CryStringT@D@@V?$allocator@V?$CryStringT@D@@@stlpmtx_std@@@priv@stlpmtx_std@@QAEAAV012@ABV012@@Z 320ae2c0 f i EntityPoolManager.obj
 0001:000ad3f0       ?CreatePools@CEntityPoolManager@@QAE_NXZ 320ae3f0 f   EntityPoolManager.obj
 0001:000ad440       ??0?$CListenerSet@PAUIEntityPoolListener@@@@QAE@ABV0@@Z 320ae440 f i EntityPoolManager.obj
 0001:000ad500       ?RemovePoolBookmark@CEntityPoolManager@@QAE_NI@Z 320ae500 f   EntityPoolManager.obj
 0001:000ad590       ?AddAttachmentToBookmark@CEntityPoolManager@@QAE_NIABUSEntityAttachment@@@Z 320ae590 f   EntityPoolManager.obj
 0001:000ad5e0       ??1?$CListenerSet@PAUIEntityPoolListener@@@@QAE@XZ 320ae5e0 f i EntityPoolManager.obj
 0001:000ad660       ?Reset@CEntityPoolManager@@QAEXXZ 320ae660 f   EntityPoolManager.obj
 0001:000ad6e0       ?NotifyEntityPreparedFromPool@CEntityPoolManager@@AAEXI@Z 320ae6e0 f   EntityPoolManager.obj
 0001:000ad800       ?OnBookmarkEntitySerialize@CEntityPoolManager@@CA_NV?$CSerializeWrapper@UISerialize@@@@PAX@Z 320ae800 f   EntityPoolManager.obj
 0001:000adb10       ?RemoveListener@CEntityPoolManager@@UAEXPAUIEntityPoolListener@@@Z 320aeb10 f   EntityPoolManager.obj
 0001:000adc40       ?LoadDefinitions@CEntityPoolManager@@AAE_NXZ 320aec40 f   EntityPoolManager.obj
 0001:000adee0       ?_M_create_node@?$_Rb_tree@IU?$less@I@stlpmtx_std@@U?$pair@$$CBIUSEntityBookmark@CEntityPoolManager@@@2@U?$_Select1st@U?$pair@$$CBIUSEntityBookmark@CEntityPoolManager@@@stlpmtx_std@@@priv@2@U?$_MapTraitsT@U?$pair@$$CBIUSEntityBookmark@CEntityPoolManager@@@stlpmtx_std@@@52@V?$allocator@U?$pair@$$CBIUSEntityBookmark@CEntityPoolManager@@@stlpmtx_std@@@2@@priv@stlpmtx_std@@IAEPAU_Rb_tree_node_base@23@ABU?$pair@$$CBIUSEntityBookmark@CEntityPoolManager@@@3@@Z 320aeee0 f i EntityPoolManager.obj
 0001:000adf40       ??$__copy_backward@PAV?$CListenerSet@PAUIEntityPoolListener@@@@PAV1@H@priv@stlpmtx_std@@YAPAV?$CListenerSet@PAUIEntityPoolListener@@@@PAV2@00ABUrandom_access_iterator_tag@1@PAH@Z 320aef40 f i EntityPoolManager.obj
 0001:000adfa0       ??$__fill@PAV?$CListenerSet@PAUIEntityPoolListener@@@@V1@H@priv@stlpmtx_std@@YAXPAV?$CListenerSet@PAUIEntityPoolListener@@@@0ABV2@ABUrandom_access_iterator_tag@1@PAH@Z 320aefa0 f i EntityPoolManager.obj
 0001:000ae000       ?SerializeBookmarkEntity@CEntityPoolManager@@ABEXAAUSEntityBookmark@1@PAVCEntity@@_N@Z 320af000 f   EntityPoolManager.obj
 0001:000ae120       ?Enable@CEntityPoolManager@@UAEX_N@Z 320af120 f   EntityPoolManager.obj
 0001:000ae190       ?UpdatePoolBookmark@CEntityPoolManager@@QAE_NII@Z 320af190 f   EntityPoolManager.obj
 0001:000ae220       ?_M_insert@?$_Rb_tree@IU?$less@I@stlpmtx_std@@U?$pair@$$CBIUSEntityBookmark@CEntityPoolManager@@@2@U?$_Select1st@U?$pair@$$CBIUSEntityBookmark@CEntityPoolManager@@@stlpmtx_std@@@priv@2@U?$_MapTraitsT@U?$pair@$$CBIUSEntityBookmark@CEntityPoolManager@@@stlpmtx_std@@@52@V?$allocator@U?$pair@$$CBIUSEntityBookmark@CEntityPoolManager@@@stlpmtx_std@@@2@@priv@stlpmtx_std@@AAE?AU?$_Rb_tree_iterator@U?$pair@$$CBIUSEntityBookmark@CEntityPoolManager@@@stlpmtx_std@@U?$_MapTraitsT@U?$pair@$$CBIUSEntityBookmark@CEntityPoolManager@@@stlpmtx_std@@@priv@2@@23@PAU_Rb_tree_node_base@23@ABU?$pair@$$CBIUSEntityBookmark@CEntityPoolManager@@@3@00@Z 320af220 f i EntityPoolManager.obj
 0001:000ae2f0       ??$__copy@PAV?$CListenerSet@PAUIEntityPoolListener@@@@PAV1@H@priv@stlpmtx_std@@YAPAV?$CListenerSet@PAUIEntityPoolListener@@@@PAV2@00ABUrandom_access_iterator_tag@1@PAH@Z 320af2f0 f i EntityPoolManager.obj
 0001:000ae350       ??$__destroy_range_aux@V?$reverse_iterator@PAV?$CListenerSet@PAUIEntityPoolListener@@@@@stlpmtx_std@@V?$CListenerSet@PAUIEntityPoolListener@@@@@stlpmtx_std@@YAXV?$reverse_iterator@PAV?$CListenerSet@PAUIEntityPoolListener@@@@@0@0PAV?$CListenerSet@PAUIEntityPoolListener@@@@ABU__false_type@0@@Z 320af350 f i EntityPoolManager.obj
 0001:000ae480       ??$__destroy_range_aux@PAV?$CListenerSet@PAUIEntityPoolListener@@@@V1@@stlpmtx_std@@YAXPAV?$CListenerSet@PAUIEntityPoolListener@@@@00ABU__false_type@0@@Z 320af480 f i EntityPoolManager.obj
 0001:000ae5c0       ?LoadBookmarkedFromPool@CEntityPoolManager@@AAE_NII_N@Z 320af5c0 f   EntityPoolManager.obj
 0001:000aec70       ?LoadDynamicFromPool@CEntityPoolManager@@AAEPAVCEntity@@AAUSEntityBookmark@1@I_N@Z 320afc70 f   EntityPoolManager.obj
 0001:000aeec0       ?PrepareDynamicFromPool@CEntityPoolManager@@AAEPAVCEntity@@AAUSEntityBookmark@1@I_N@Z 320afec0 f   EntityPoolManager.obj
 0001:000aef80       ?ProcessPrepareRequest@CEntityPoolManager@@AAE_NABUSEntityPrepareRequest@1@@Z 320aff80 f   EntityPoolManager.obj
 0001:000aefd0       ?ReturnToPool@CEntityPoolManager@@QAE_NI_N0@Z 320affd0 f   EntityPoolManager.obj
 0001:000af520       ?AddListener@CEntityPoolManager@@UAEXPAUIEntityPoolListener@@PBDI@Z 320b0520 f   EntityPoolManager.obj
 0001:000af5f0       ?insert_unique@?$_Rb_tree@IU?$less@I@stlpmtx_std@@U?$pair@$$CBIUSEntityBookmark@CEntityPoolManager@@@2@U?$_Select1st@U?$pair@$$CBIUSEntityBookmark@CEntityPoolManager@@@stlpmtx_std@@@priv@2@U?$_MapTraitsT@U?$pair@$$CBIUSEntityBookmark@CEntityPoolManager@@@stlpmtx_std@@@52@V?$allocator@U?$pair@$$CBIUSEntityBookmark@CEntityPoolManager@@@stlpmtx_std@@@2@@priv@stlpmtx_std@@QAE?AU?$pair@U?$_Rb_tree_iterator@U?$pair@$$CBIUSEntityBookmark@CEntityPoolManager@@@stlpmtx_std@@U?$_MapTraitsT@U?$pair@$$CBIUSEntityBookmark@CEntityPoolManager@@@stlpmtx_std@@@priv@2@@priv@stlpmtx_std@@_N@3@ABU?$pair@$$CBIUSEntityBookmark@CEntityPoolManager@@@3@@Z 320b05f0 f i EntityPoolManager.obj
 0001:000af6b0       ??$__uninitialized_fill_n@PAV?$CListenerSet@PAUIEntityPoolListener@@@@IV1@@priv@stlpmtx_std@@YAPAV?$CListenerSet@PAUIEntityPoolListener@@@@PAV2@IABV2@@Z 320b06b0 f i EntityPoolManager.obj
 0001:000af6f0       ??$__ucopy_ptrs@PAV?$CListenerSet@PAUIEntityPoolListener@@@@PAV1@@priv@stlpmtx_std@@YAPAV?$CListenerSet@PAUIEntityPoolListener@@@@PAV2@00ABU__false_type@1@@Z 320b06f0 f i EntityPoolManager.obj
 0001:000af730       ?Update@CEntityPoolManager@@QAEXXZ 320b0730 f   EntityPoolManager.obj
 0001:000af790       ?PrepareFromPool@CEntityPoolManager@@QAE_NII_N0@Z 320b0790 f   EntityPoolManager.obj
 0001:000af910       ?ReturnToPool@CEntityPoolManager@@UAE_NI_N@Z 320b0910 f   EntityPoolManager.obj
 0001:000af930       ?_M_fill_insert_aux@?$_Impl_vector@V?$CListenerSet@PAUIEntityPoolListener@@@@V?$allocator@V?$CListenerSet@PAUIEntityPoolListener@@@@@stlpmtx_std@@@priv@stlpmtx_std@@AAEXPAV?$CListenerSet@PAUIEntityPoolListener@@@@IABV4@ABU__false_type@3@@Z 320b0930 f i EntityPoolManager.obj
 0001:000afa30       ?PrepareFromPool@CEntityPoolManager@@UAE_NI_N@Z 320b0a30 f   EntityPoolManager.obj
 0001:000afad0       ?AddPoolBookmark@CEntityPoolManager@@QAE_NAAUSEntityLoadParams@@_N@Z 320b0ad0 f   EntityPoolManager.obj
 0001:000aff30       ?_M_insert_overflow_aux@?$_Impl_vector@V?$CListenerSet@PAUIEntityPoolListener@@@@V?$allocator@V?$CListenerSet@PAUIEntityPoolListener@@@@@stlpmtx_std@@@priv@stlpmtx_std@@AAEXPAV?$CListenerSet@PAUIEntityPoolListener@@@@ABV4@ABU__false_type@3@I_N@Z 320b0f30 f i EntityPoolManager.obj
 0001:000b0110       ??1CEntityPoolManager@@UAE@XZ 320b1110 f   EntityPoolManager.obj
 0001:000b0210       ?Serialize@CEntityPoolManager@@UAEXV?$CSerializeWrapper@UISerialize@@@@@Z 320b1210 f   EntityPoolManager.obj
 0001:000b0ab0       ?PrepareDynamicFromPool@CEntityPoolManager@@QAEPAVCEntity@@AAUSEntitySpawnParams@@_N@Z 320b1ab0 f   EntityPoolManager.obj
 0001:000b0c00       ?erase@?$_Impl_vector@V?$CListenerSet@PAUIEntityPoolListener@@@@V?$allocator@V?$CListenerSet@PAUIEntityPoolListener@@@@@stlpmtx_std@@@priv@stlpmtx_std@@QAEPAV?$CListenerSet@PAUIEntityPoolListener@@@@PAV4@0@Z 320b1c00 f i EntityPoolManager.obj
 0001:000b0c60       ??_GCEntityPoolManager@@UAEPAXI@Z 320b1c60 f i EntityPoolManager.obj
 0001:000b0c60       ??_ECEntityPoolManager@@UAEPAXI@Z 320b1c60 f i EntityPoolManager.obj
 0001:000b0c90       ?resize@?$_Impl_vector@V?$CListenerSet@PAUIEntityPoolListener@@@@V?$allocator@V?$CListenerSet@PAUIEntityPoolListener@@@@@stlpmtx_std@@@priv@stlpmtx_std@@QAEXIABV?$CListenerSet@PAUIEntityPoolListener@@@@@Z 320b1c90 f i EntityPoolManager.obj
 0001:000b0d10       ??0CEntityPoolManager@@QAE@PAVCEntitySystem@@@Z 320b1d10 f   EntityPoolManager.obj
 0001:000b0fd0       ??0CEntityPoolSignature@@QAE@XZ 320b1fd0 f   EntityPoolSignature.obj
 0001:000b1080       ?CalculateFromEntity@CEntityPoolSignature@@QAE_NPAVCEntity@@@Z 320b2080 f   EntityPoolSignature.obj
 0001:000b11f0       ?CompareNodeAttributes@CEntityPoolSignature@@CA_NABVXmlNodeRef@@0@Z 320b21f0 f   EntityPoolSignature.obj
 0001:000b1360       ?CompareNodes@CEntityPoolSignature@@CA_NABVXmlNodeRef@@0_N@Z 320b2360 f   EntityPoolSignature.obj
 0001:000b1540       ?CompareSignature@CEntityPoolSignature@@QBE_NABV1@@Z 320b2540 f   EntityPoolSignature.obj
 0001:000b1640       _memset                    320b2640 f   MSVCRT:MSVCR100.dll
 0001:000b1646       __purecall                 320b2646 f   MSVCRT:MSVCR100.dll
 0001:000b164c       _memcpy                    320b264c f   MSVCRT:MSVCR100.dll
 0001:000b1652       __onexit                   320b2652 f   MSVCRT:atonexit.obj
 0001:000b16f3       _atexit                    320b26f3 f   MSVCRT:atonexit.obj
 0001:000b170a       __CIacos                   320b270a f   MSVCRT:MSVCR100.dll
 0001:000b1710       __CIpow                    320b2710 f   MSVCRT:MSVCR100.dll
 0001:000b1720       __allmul                   320b2720 f   MSVCRT:llmul.obj
 0001:000b1760       __chkstk                   320b2760 f   MSVCRT:chkstk.obj
 0001:000b1760       __alloca_probe             320b2760     MSVCRT:chkstk.obj
 0001:000b178c       ?what@exception@std@@UBEPBDXZ 320b278c f   MSVCRT:MSVCR100.dll
 0001:000b17a0       __allshl                   320b27a0 f   MSVCRT:llshl.obj
 0001:000b17c0       __aullshr                  320b27c0 f   MSVCRT:ullshr.obj
 0001:000b17e0       __CIasin                   320b27e0 f   MSVCRT:MSVCR100.dll
 0001:000b17f0       __ftol2_sse                320b27f0 f   MSVCRT:ftol2.obj
 0001:000b17f9       __ftol2_pentium4           320b27f9 f   MSVCRT:ftol2.obj
 0001:000b180c       __ftol2_sse_excpt          320b280c f   MSVCRT:ftol2.obj
 0001:000b1826       __ftol2                    320b2826 f   MSVCRT:ftol2.obj
 0001:000b189c       _floor                     320b289c f   MSVCRT:MSVCR100.dll
 0001:000b18b0       __alloca_probe_16          320b28b0 f   MSVCRT:alloca16.obj
 0001:000b18c6       __alloca_probe_8           320b28c6     MSVCRT:alloca16.obj
 0001:000b192a       __CRT_INIT@12              320b292a f   MSVCRT:crtdll.obj
 0001:000b1c4a       __DllMainCRTStartup@12     320b2c4a f   MSVCRT:crtdll.obj
 0001:000b1c6e       __unlock                   320b2c6e f   MSVCRT:MSVCR100.dll
 0001:000b1c74       ___dllonexit               320b2c74 f   MSVCRT:MSVCR100.dll
 0001:000b1c7a       __lock                     320b2c7a f   MSVCRT:MSVCR100.dll
 0001:000b1c80       __SEH_prolog4              320b2c80 f   MSVCRT:sehprolg4.obj
 0001:000b1cc5       __SEH_epilog4              320b2cc5 f   MSVCRT:sehprolg4.obj
 0001:000b1cd9       __except_handler4          320b2cd9 f   MSVCRT:chandler4gs.obj
 0001:000b1cfe       ___sse2_available_init     320b2cfe f   MSVCRT:cpu_disp.obj
 0001:000b1d0e       ___clean_type_info_names   320b2d0e f   MSVCRT:tncleanup.obj
 0001:000b1d1a       __RTC_Initialize           320b2d1a f   MSVCRT:_initsect_.obj
 0001:000b1d40       __RTC_Terminate            320b2d40 f   MSVCRT:_initsect_.obj
 0001:000b1d70       __ValidateImageBase        320b2d70 f   MSVCRT:pesect.obj
 0001:000b1db0       __FindPESection            320b2db0 f   MSVCRT:pesect.obj
 0001:000b1e00       __IsNonwritableInCurrentImage 320b2e00 f   MSVCRT:pesect.obj
 0001:000b1ebc       __initterm                 320b2ebc f   MSVCRT:MSVCR100.dll
 0001:000b1ec2       __initterm_e               320b2ec2 f   MSVCRT:MSVCR100.dll
 0001:000b1ec8       __amsg_exit                320b2ec8 f   MSVCRT:MSVCR100.dll
 0001:000b1ece       ___CppXcptFilter           320b2ece f   MSVCRT:MSVCR100.dll
 0001:000b1ed4       _DllMain@12                320b2ed4 f   MSVCRT:dllmain.obj
 0001:000b1ef8       ___security_init_cookie    320b2ef8 f   MSVCRT:gs_support.obj
 0001:000b1f93       @__security_check_cookie@4 320b2f93 f   MSVCRT:secchk.obj
 0001:000b1fa2       __except_handler4_common   320b2fa2 f   MSVCRT:MSVCR100.dll
 0001:000b1fa8       ___clean_type_info_names_internal 320b2fa8 f   MSVCRT:MSVCR100.dll
 0001:000b1fae       ___report_gsfailure        320b2fae f   MSVCRT:gs_report.obj
 0001:000b20b4       __crt_debugger_hook        320b30b4 f   MSVCRT:MSVCR100.dll
 0001:000b23f0       ??__Fs_dummyMemReplay@?1??CryGetIMemReplay@@YAPAUIMemReplay@@XZ@YAXXZ 320b33f0 f i AreaSolid.obj
 0001:000b2470       ??__Fp@?1??CreateClassInstance@CFactory@CEngineModule_EntitySystem@@UBE?AV?$shared_ptr@UICryUnknown@@@boost@@XZ@YAXXZ 320b3470 f i CryEntityDLL.obj
 0001:000b24e0       ??__FserializeString@?1??SetSharedSerializeString@?$CSerializeWrapper@UISerialize@@@@QAEAAUSSerializeString@@ABV?$CryStringT@D@@@Z@YAXXZ 320b34e0 f i EntityLayer.obj
 0001:000b2620       ??__FInfo@?1??TypeInfo@?$TFixed@E$00$0PP@@@QBEABUCTypeInfo@@XZ@YAXXZ 320b3620 f i ScriptBind_Entity.obj
 0002:00000000       __imp__InterlockedCompareExchange@12 320b4000     kernel32:KERNEL32.dll
 0002:00000004       __imp__InitializeCriticalSection@4 320b4004     kernel32:KERNEL32.dll
 0002:00000008       __imp__DeleteCriticalSection@4 320b4008     kernel32:KERNEL32.dll
 0002:0000000c       __imp__EnterCriticalSection@4 320b400c     kernel32:KERNEL32.dll
 0002:00000010       __imp__LeaveCriticalSection@4 320b4010     kernel32:KERNEL32.dll
 0002:00000014       __imp__GetCurrentThreadId@0 320b4014     kernel32:KERNEL32.dll
 0002:00000018       __imp__LoadLibraryA@4      320b4018     kernel32:KERNEL32.dll
 0002:0000001c       __imp__GetProcAddress@8    320b401c     kernel32:KERNEL32.dll
 0002:00000020       __imp__GetModuleHandleA@4  320b4020     kernel32:KERNEL32.dll
 0002:00000024       __imp__IsDebuggerPresent@0 320b4024     kernel32:KERNEL32.dll
 0002:00000028       __imp__Sleep@4             320b4028     kernel32:KERNEL32.dll
 0002:0000002c       __imp__InterlockedIncrement@4 320b402c     kernel32:KERNEL32.dll
 0002:00000030       __imp__InterlockedDecrement@4 320b4030     kernel32:KERNEL32.dll
 0002:00000034       __imp__InterlockedExchangeAdd@8 320b4034     kernel32:KERNEL32.dll
 0002:00000038       __imp__GetCurrentProcess@0 320b4038     kernel32:KERNEL32.dll
 0002:0000003c       __imp__TerminateProcess@8  320b403c     kernel32:KERNEL32.dll
 0002:00000040       __imp__SetUnhandledExceptionFilter@4 320b4040     kernel32:KERNEL32.dll
 0002:00000044       __imp__GetSystemTimeAsFileTime@4 320b4044     kernel32:KERNEL32.dll
 0002:00000048       __imp__GetCurrentProcessId@0 320b4048     kernel32:KERNEL32.dll
 0002:0000004c       __imp__GetTickCount@0      320b404c     kernel32:KERNEL32.dll
 0002:00000050       __imp__QueryPerformanceCounter@4 320b4050     kernel32:KERNEL32.dll
 0002:00000054       __imp__DisableThreadLibraryCalls@4 320b4054     kernel32:KERNEL32.dll
 0002:00000058       __imp__IsProcessorFeaturePresent@4 320b4058     kernel32:KERNEL32.dll
 0002:0000005c       __imp__InterlockedExchange@8 320b405c     kernel32:KERNEL32.dll
 0002:00000060       __imp__DecodePointer@4     320b4060     kernel32:KERNEL32.dll
 0002:00000064       __imp__EncodePointer@4     320b4064     kernel32:KERNEL32.dll
 0002:00000068       __imp__UnhandledExceptionFilter@4 320b4068     kernel32:KERNEL32.dll
 0002:0000006c       \177KERNEL32_NULL_THUNK_DATA 320b406c     kernel32:KERNEL32.dll
 0002:00000070       __imp__sscanf_s            320b4070     MSVCRT:MSVCR100.dll
 0002:00000074       __imp__sprintf             320b4074     MSVCRT:MSVCR100.dll
 0002:00000078       __imp__strcspn             320b4078     MSVCRT:MSVCR100.dll
 0002:0000007c       __imp__strchr              320b407c     MSVCRT:MSVCR100.dll
 0002:00000080       __imp__atof                320b4080     MSVCRT:MSVCR100.dll
 0002:00000084       __imp__islower             320b4084     MSVCRT:MSVCR100.dll
 0002:00000088       __imp___set_invalid_parameter_handler 320b4088     MSVCRT:MSVCR100.dll
 0002:0000008c       __imp___set_purecall_handler 320b408c     MSVCRT:MSVCR100.dll
 0002:00000090       __imp_??0exception@std@@QAE@ABQBDH@Z 320b4090     MSVCRT:MSVCR100.dll
 0002:00000094       __imp_?what@exception@std@@UBEPBDXZ 320b4094     MSVCRT:MSVCR100.dll
 0002:00000098       __imp_??1exception@std@@UAE@XZ 320b4098     MSVCRT:MSVCR100.dll
 0002:0000009c       __imp___ui64toa            320b409c     MSVCRT:MSVCR100.dll
 0002:000000a0       __imp___CIasin             320b40a0     MSVCRT:MSVCR100.dll
 0002:000000a4       __imp__strncmp             320b40a4     MSVCRT:MSVCR100.dll
 0002:000000a8       __imp__stricmp             320b40a8     MSVCRT:MSVCR100.dll
 0002:000000a8       __imp___stricmp            320b40a8     MSVCRT:MSVCR100.dll
 0002:000000a8       __imp__strcmpi             320b40a8     MSVCRT:MSVCR100.dll
 0002:000000ac       __imp__strncpy             320b40ac     MSVCRT:MSVCR100.dll
 0002:000000b0       __imp__atoi                320b40b0     MSVCRT:MSVCR100.dll
 0002:000000b4       __imp__strstr              320b40b4     MSVCRT:MSVCR100.dll
 0002:000000b8       __imp___vscprintf          320b40b8     MSVCRT:MSVCR100.dll
 0002:000000bc       __imp___vsnprintf          320b40bc     MSVCRT:MSVCR100.dll
 0002:000000bc       __imp__vsnprintf           320b40bc     MSVCRT:MSVCR100.dll
 0002:000000c0       __imp__floor               320b40c0     MSVCRT:MSVCR100.dll
 0002:000000c4       __imp__strcpy_s            320b40c4     MSVCRT:MSVCR100.dll
 0002:000000c8       __imp__qsort               320b40c8     MSVCRT:MSVCR100.dll
 0002:000000cc       __imp__atol                320b40cc     MSVCRT:MSVCR100.dll
 0002:000000d0       __imp___snprintf           320b40d0     MSVCRT:MSVCR100.dll
 0002:000000d4       __imp___finite             320b40d4     MSVCRT:MSVCR100.dll
 0002:000000d8       __imp__fread               320b40d8     MSVCRT:MSVCR100.dll
 0002:000000dc       __imp__strncpy_s           320b40dc     MSVCRT:MSVCR100.dll
 0002:000000e0       __imp__fclose              320b40e0     MSVCRT:MSVCR100.dll
 0002:000000e4       __imp__fopen               320b40e4     MSVCRT:MSVCR100.dll
 0002:000000e8       __imp__isalnum             320b40e8     MSVCRT:MSVCR100.dll
 0002:000000ec       __imp___unlock             320b40ec     MSVCRT:MSVCR100.dll
 0002:000000f0       __imp____dllonexit         320b40f0     MSVCRT:MSVCR100.dll
 0002:000000f4       __imp___lock               320b40f4     MSVCRT:MSVCR100.dll
 0002:000000f8       __imp___onexit             320b40f8     MSVCRT:MSVCR100.dll
 0002:000000fc       __imp___vsnprintf_s        320b40fc     MSVCRT:MSVCR100.dll
 0002:000000fc       __imp__vsnprintf_s         320b40fc     MSVCRT:MSVCR100.dll
 0002:00000100       __imp___malloc_crt         320b4100     MSVCRT:MSVCR100.dll
 0002:00000104       __imp__free                320b4104     MSVCRT:MSVCR100.dll
 0002:00000108       __imp___encoded_null       320b4108     MSVCRT:MSVCR100.dll
 0002:0000010c       __imp___initterm           320b410c     MSVCRT:MSVCR100.dll
 0002:00000110       __imp___initterm_e         320b4110     MSVCRT:MSVCR100.dll
 0002:00000114       __imp___amsg_exit          320b4114     MSVCRT:MSVCR100.dll
 0002:00000118       __imp____CppXcptFilter     320b4118     MSVCRT:MSVCR100.dll
 0002:0000011c       __imp___except_handler4_common 320b411c     MSVCRT:MSVCR100.dll
 0002:00000120       __imp____clean_type_info_names_internal 320b4120     MSVCRT:MSVCR100.dll
 0002:00000124       __imp___crt_debugger_hook  320b4124     MSVCRT:MSVCR100.dll
 0002:00000128       __imp___CIpow              320b4128     MSVCRT:MSVCR100.dll
 0002:0000012c       __imp___CIacos             320b412c     MSVCRT:MSVCR100.dll
 0002:00000130       __imp__exit                320b4130     MSVCRT:MSVCR100.dll
 0002:00000134       __imp__puts                320b4134     MSVCRT:MSVCR100.dll
 0002:00000138       __imp__abort               320b4138     MSVCRT:MSVCR100.dll
 0002:0000013c       __imp__memcpy              320b413c     MSVCRT:MSVCR100.dll
 0002:00000140       __imp__memmove             320b4140     MSVCRT:MSVCR100.dll
 0002:00000144       __imp___purecall           320b4144     MSVCRT:MSVCR100.dll
 0002:00000148       __imp__memset              320b4148     MSVCRT:MSVCR100.dll
 0002:0000014c       __imp___strnicmp           320b414c     MSVCRT:MSVCR100.dll
 0002:0000014c       __imp__strnicmp            320b414c     MSVCRT:MSVCR100.dll
 0002:00000150       __imp__ltoa                320b4150     MSVCRT:MSVCR100.dll
 0002:00000150       __imp___ltoa               320b4150     MSVCRT:MSVCR100.dll
 0002:00000154       __imp__isupper             320b4154     MSVCRT:MSVCR100.dll
 0002:00000158       __imp___ultoa              320b4158     MSVCRT:MSVCR100.dll
 0002:00000158       __imp__ultoa               320b4158     MSVCRT:MSVCR100.dll
 0002:0000015c       \177MSVCR100_NULL_THUNK_DATA 320b415c     MSVCRT:MSVCR100.dll
 0002:00000160       __imp__MessageBoxA@16      320b4160     user32:USER32.dll
 0002:00000164       \177USER32_NULL_THUNK_DATA 320b4164     user32:USER32.dll
 0002:00000168       ___xc_a                    320b4168     MSVCRT:cinitexe.obj
 0002:000001c0       ___xc_z                    320b41c0     MSVCRT:cinitexe.obj
 0002:000001c4       ___xi_a                    320b41c4     MSVCRT:cinitexe.obj
 0002:000001d0       ___xi_z                    320b41d0     MSVCRT:cinitexe.obj
 0002:00000200       __mask@@NegFloat@          320b4200     AffineParts.obj
 0002:00000210       __real@3f800000            320b4210     AffineParts.obj
 0002:00000218       __real@3fe0000000000000    320b4218     AffineParts.obj
 0002:00000220       __real@00000000            320b4220     AffineParts.obj
 0002:00000224       __real@40000000            320b4224     AffineParts.obj
 0002:00000228       __real@bf800000            320b4228     AffineParts.obj
 0002:00000230       __real@3eb0c6f7a0b5ed8d    320b4230     AffineParts.obj
 0002:00000238       __real@3f000000            320b4238     AffineParts.obj
 0002:00000240       __real@4059000000000000    320b4240     AffineParts.obj
 0002:00000248       __real@3e80000000000000    320b4248     AffineParts.obj
 0002:00000250       __real@3f3504f3            320b4250     AffineParts.obj
 0002:00000254       ?EPSILON@AreaUtil@@3MB     320b4254     AreaSolid.obj
 0002:00000260       ??_7IMemReplay@@6B@        320b4260     AreaSolid.obj
 0002:000002f8       ??_C@_0P@PCJPAHLM@out?5of?5memory?6?$AA@ 320b42f8     AreaSolid.obj
 0002:00000308       ??_C@_06NBFPPGEG@vector?$AA@ 320b4308     AreaSolid.obj
 0002:00000310       __real@3fc00000            320b4310     AreaSolid.obj
 0002:00000314       __real@00800000            320b4314     AreaSolid.obj
 0002:00000318       ??_7CDummyMemReplay@@6B@   320b4318     AreaSolid.obj
 0002:000003b0       __real@d8635fa9            320b43b0     AreaSolid.obj
 0002:000003b4       __real@58635fa9            320b43b4     AreaSolid.obj
 0002:000003b8       __real@bba3d70a            320b43b8     AreaSolid.obj
 0002:000003bc       ??_7ISoundEventListener@@6B@ 320b43bc     SoundProxy.obj
 0002:000003bc       ??_7ISystemEventListener@@6B@ 320b43bc     CryEntityDLL.obj
 0002:000003bc       ??_7IOwnedObject@@6B@      320b43bc     BreakablePlane.obj
 0002:000003c8       ??_7ISplineInterpolator@@6B@ 320b43c8     BreakablePlane.obj
 0002:00000420       __real@437f0000            320b4420     BreakablePlane.obj
 0002:00000424       __real@42fe0000            320b4424     BreakablePlane.obj
 0002:00000428       ??_C@_07ODPOPIG@_broken?$AA@ 320b4428     BreakablePlane.obj
 0002:00000430       __real@34000000            320b4430     BreakablePlane.obj
 0002:00000434       __real@46fffe00            320b4434     BreakablePlane.obj
 0002:00000438       __real@38000100            320b4438     BreakablePlane.obj
 0002:0000043c       __real@3f7ff972            320b443c     BreakablePlane.obj
 0002:00000440       __real@40490fdb            320b4440     BreakablePlane.obj
 0002:00000444       __real@1e3ce508            320b4444     BreakablePlane.obj
 0002:00000448       __real@3fd5555560000000    320b4448     BreakablePlane.obj
 0002:00000450       __real@43340000            320b4450     BreakablePlane.obj
 0002:00000454       __real@43b40000            320b4454     BreakablePlane.obj
 0002:00000458       __real@3e800000            320b4458     BreakablePlane.obj
 0002:0000045c       ??_C@_00CNPNBAHC@?$AA@     320b445c     BreakablePlane.obj
 0002:00000460       __real@3f4f5c28            320b4460     BreakablePlane.obj
 0002:00000464       __real@44610000            320b4464     BreakablePlane.obj
 0002:00000468       __real@3e99999a            320b4468     BreakablePlane.obj
 0002:0000046c       ??_7CBreakablePlane@@6B@   320b446c     BreakablePlane.obj
 0002:00000474       __real@c9742400            320b4474     BreakablePlane.obj
 0002:00000478       __real@49742400            320b4478     BreakablePlane.obj
 0002:0000047c       __real@3d4ccccd            320b447c     BreakablePlane.obj
 0002:00000480       __real@4000000000000000    320b4480     BreakablePlane.obj
 0002:00000488       __real@bf7ff972            320b4488     BreakablePlane.obj
 0002:0000048c       __real@38d1b717            320b448c     BreakablePlane.obj
 0002:00000490       __real@2edbe6ff            320b4490     BreakablePlane.obj
 0002:00000494       __real@3f670a3d            320b4494     BreakablePlane.obj
 0002:00000498       __real@3ba3d70a            320b4498     BreakablePlane.obj
 0002:0000049c       __real@40133333            320b449c     BreakablePlane.obj
 0002:000004a0       __real@3cf5c28f            320b44a0     BreakablePlane.obj
 0002:000004a4       __real@3f333333            320b44a4     BreakablePlane.obj
 0002:000004a8       __real@3f7fbe77            320b44a8     BreakablePlane.obj
 0002:000004b0       ??_C@_0EM@EMKNFFCL@?$FLBreakable2d?$FN?5?3?5geometry?5has?5sev@ 320b44b0     BreakablePlane.obj
 0002:000004fc       __real@3f7851ec            320b44fc     BreakablePlane.obj
 0002:00000500       __real@3f733333            320b4500     BreakablePlane.obj
 0002:00000508       ??_C@_0EN@KMHFILF@?$FLBreakable2d?$FN?5?3?5breakable?5tessel@ 320b4508     BreakablePlane.obj
 0002:00000558       __real@3d99999a            320b4558     BreakablePlane.obj
 0002:0000055c       __real@3f7eb852            320b455c     BreakablePlane.obj
 0002:00000560       __real@3c23d70a            320b4560     BreakablePlane.obj
 0002:00000568       ??_C@_0EG@NJIJMPKL@?$FLBreakable2d?$FN?5?3?5geometry?5is?5not?5@ 320b4568     BreakablePlane.obj
 0002:000005b0       __real@40800000            320b45b0     BreakablePlane.obj
 0002:000005b4       __real@26901d7d            320b45b4     BreakablePlane.obj
 0002:000005b8       __real@3f8147ae            320b45b8     BreakablePlane.obj
 0002:000005bc       __real@3f7d70a4            320b45bc     BreakablePlane.obj
 0002:000005c0       __real@3f0147ae            320b45c0     BreakablePlane.obj
 0002:000005c4       __real@3f2aaaab            320b45c4     BreakablePlane.obj
 0002:000005c8       __real@3eaaaaab            320b45c8     BreakablePlane.obj
 0002:000005cc       __real@d01502f9            320b45cc     BreakablePlane.obj
 0002:000005d0       __real@501502f9            320b45d0     BreakablePlane.obj
 0002:000005d4       ??_7?$TSpline@U?$SplineKey@M@spline@@U?$TCoeffBasis@M@2@@spline@@6B@ 320b45d4     BreakablePlane.obj
 0002:000005e4       ??_7?$TSplineSlopes@MU?$SplineKey@M@spline@@$00@spline@@6B@ 320b45e4     BreakablePlane.obj
 0002:000005f4       __real@40400000            320b45f4     BreakablePlane.obj
 0002:000005f8       ??_7ISplineBackup@@6B@     320b45f8     BreakablePlane.obj
 0002:00000604       __real@3b808081            320b4604     BreakablePlane.obj
 0002:00000608       __real@3d000000            320b4608     BreakablePlane.obj
 0002:00000610       ??_7?$TCurve@U?$TFixed@E$00$0PP@@@@@6B@ 320b4610     BreakablePlane.obj
 0002:00000668       ??_7?$SSplineBackup@V?$OptSpline@U?$TFixed@E$00$0PP@@@V?$TSplineSlopes@MU?$SplineKey@M@spline@@$00@spline@@@spline@@@spline@@6B@ 320b4668     BreakablePlane.obj
 0002:00000674       __real@42c80000            320b4674     BreakablePlane.obj
 0002:00000678       __real@42480000            320b4678     BreakablePlane.obj
 0002:0000067c       __real@447a0000            320b467c     BreakablePlane.obj
 0002:00000680       __real@3e4ccccd            320b4680     BreakablePlane.obj
 0002:00000684       ??_C@_0BG@GGDKGFHA@breakable_plane_piece?$AA@ 320b4684     BreakablePlane.obj
 0002:0000069c       ??_C@_07MCAEODGB@Default?$AA@ 320b469c     BreakablePlane.obj
 0002:000006a4       __real@41100000            320b46a4     BreakablePlane.obj
 0002:000006a8       __real@47c35000            320b46a8     BreakablePlane.obj
 0002:000006ac       __real@3bb60b61            320b46ac     BreakablePlane.obj
 0002:000006b0       __real@41200000            320b46b0     BreakablePlane.obj
 0002:000006b8       ??_C@_0FA@PBBIBOLL@?$FLBreakable2d?$FN?5?3?5geometry?5is?5not?5@ 320b46b8     BreakablePlane.obj
 0002:00000708       ??_C@_0BL@BCEMJAIP@g_breakage_particles_limit?$AA@ 320b4708     BreakablePlane.obj
 0002:00000724       ??_C@_0BP@OPIGKHHA@CBreakablePlane?3?3ProcessImpact?$AA@ 320b4724     BreakablePlane.obj
 0002:00000744       ??_C@_04LOAJBDKD@true?$AA@ 320b4744     CryEntityDLL.obj
 0002:0000074c       ??_C@_05LAPONLG@false?$AA@ 320b474c     CryEntityDLL.obj
 0002:00000754       ??_C@_01GBGANLPD@0?$AA@    320b4754     CryEntityDLL.obj
 0002:00000758       ??_C@_02BEIEFPIG@?$CFg?$AA@ 320b4758     CryEntityDLL.obj
 0002:0000075c       ??_C@_04HGGMHPIM@?$CF?4?$CKf?$AA@ 320b475c     CryEntityDLL.obj
 0002:00000764       ??_C@_04GPHHEOMN@?$CF?4?$CKg?$AA@ 320b4764     CryEntityDLL.obj
 0002:0000076c       ??_C@_04GHNNFJCK@?$CF?40f?$AA@ 320b476c     CryEntityDLL.obj
 0002:00000778       __real@4024000000000000    320b4778     CryEntityDLL.obj
 0002:00000780       __real@2f800000            320b4780     CryEntityDLL.obj
 0002:00000784       __real@4f800000            320b4784     CryEntityDLL.obj
 0002:00000788       ??_7CTypeInfo@@6B@         320b4788     CryEntityDLL.obj
 0002:000007bc       ??_C@_0DJ@DLJMMMP@Could?5not?5access?5CrySystem?4dll?5?$CI@ 320b47bc     CryEntityDLL.obj
 0002:000007f8       ??_C@_0P@NHEMOHAI@Memory?5Manager?$AA@ 320b47f8     CryEntityDLL.obj
 0002:00000808       ??_C@_0O@FFDHMLKN@CrySystem?4dll?$AA@ 320b4808     CryEntityDLL.obj
 0002:00000818       ??_C@_0BO@JDKBDPNB@CryGetIMemoryManagerInterface?$AA@ 320b4818     CryEntityDLL.obj
 0002:00000838       ??_C@_0BB@PNKHDABP@CrySystemCrtFree?$AA@ 320b4838     CryEntityDLL.obj
 0002:0000084c       ??_C@_0BB@MFMFBMDO@CrySystemCrtSize?$AA@ 320b484c     CryEntityDLL.obj
 0002:00000860       ??_C@_0BD@BBIFHONI@CrySystemCrtMalloc?$AA@ 320b4860     CryEntityDLL.obj
 0002:00000874       ??_C@_0O@LCCIKADF@CryGetMemSize?$AA@ 320b4874     CryEntityDLL.obj
 0002:00000884       ??_C@_07CKAGCLEE@CryFree?$AA@ 320b4884     CryEntityDLL.obj
 0002:0000088c       ??_C@_0L@FICCDMFO@CryRealloc?$AA@ 320b488c     CryEntityDLL.obj
 0002:00000898       ??_C@_09MCKPOEAK@CryMalloc?$AA@ 320b4898     CryEntityDLL.obj
 0002:000008a4       ??_7ICryUnknown@@6B@       320b48a4     CryEntityDLL.obj
 0002:000008b8       ?iid@?1??IID@ICryUnknown@@CAABUCryGUID@@XZ@4U3@B 320b48b8     CryEntityDLL.obj
 0002:000008c8       ?iid@?1??IID@IEngineModule@@CAABUCryGUID@@XZ@4U3@B 320b48c8     CryEntityDLL.obj
 0002:000008d8       ??_7ICryFactory@@6B@       320b48d8     CryEntityDLL.obj
 0002:000008f0       ??_7?$TTypeInfo@M@@6B@     320b48f0     CryEntityDLL.obj
 0002:00000924       ??_C@_02DKCKIIND@?$CFs?$AA@ 320b4924     CryEntityDLL.obj
 0002:00000928       ??_C@_0BD@PJOKHJBB@Pure?5function?5call?$AA@ 320b4928     CryEntityDLL.obj
 0002:0000093c       ??_C@_0CL@LKHBOBAH@Invalid?5parameter?5detected?5in?5CR@ 320b493c     CryEntityDLL.obj
 0002:00000968       ??_C@_0BO@HAMEIFMK@Critical?5Section?5hanging?5lock?$AA@ 320b4968     CryEntityDLL.obj
 0002:00000988       ??_7CSystemEventListner_Entity@@6B@ 320b4988     CryEntityDLL.obj
 0002:00000990       ??_7?$TIntTypeInfo@H@@6B@  320b4990     CryEntityDLL.obj
 0002:000009c4       __real@4f000000            320b49c4     CryEntityDLL.obj
 0002:000009c8       __real@cf000000            320b49c8     CryEntityDLL.obj
 0002:000009cc       ??_7?$TIntTypeInfo@I@@6B@  320b49cc     CryEntityDLL.obj
 0002:00000a00       ??_7?$TIntTypeInfo@_K@@6B@ 320b4a00     CryEntityDLL.obj
 0002:00000a34       ??_7CEnumInfo@@6B@         320b4a34     CryEntityDLL.obj
 0002:00000a68       ??_7CEngineModule_EntitySystem@@6B@ 320b4a68     CryEntityDLL.obj
 0002:00000a84       ??_C@_0BA@BIPJEEEL@CryEntitySystem?$AA@ 320b4a84     CryEntityDLL.obj
 0002:00000a94       ??_C@_09BHIABECK@CryEngine?$AA@ 320b4a94     CryEntityDLL.obj
 0002:00000aa0       ??_C@_04DDKJGDCM@bool?$AA@ 320b4aa0     CryEntityDLL.obj
 0002:00000aa8       ??_C@_05KNFBNCOH@float?$AA@ 320b4aa8     CryEntityDLL.obj
 0002:00000ab0       ??_C@_06ICGJLFIM@string?$AA@ 320b4ab0     CryEntityDLL.obj
 0002:00000ab8       ??_7CFactory@CEngineModule_EntitySystem@@6B@ 320b4ab8     CryEntityDLL.obj
 0002:00000ad0       ??_7bad_alloc@std@@6B@     320b4ad0     CryEntityDLL.obj
 0002:00000ad8       ??_C@_0P@GHFPNOJB@bad?5allocation?$AA@ 320b4ad8     CryEntityDLL.obj
 0002:00000ae8       ??_C@_0BN@DGCNMMEP@EngineModule_CryEntitySystem?$AA@ 320b4ae8     CryEntityDLL.obj
 0002:00000b08       ?cid@?1??GetClassID@CFactory@CEngineModule_EntitySystem@@UBEABUCryGUID@@XZ@4U4@B 320b4b08     CryEntityDLL.obj
 0002:00000b18       ??_7sp_counted_base@detail@boost@@6B@ 320b4b18     CryEntityDLL.obj
 0002:00000b28       ??_7?$sp_counted_impl_p@VCEngineModule_EntitySystem@@@detail@boost@@6B@ 320b4b28     CryEntityDLL.obj
 0002:00000b38       ??_C@_0BN@FOKPCDPC@Boost?5threw?5an?5exception?3?5?$CFs?$AA@ 320b4b38     CryEntityDLL.obj
 0002:00000b58       ??_C@_03JBIPMCLC@int?$AA@  320b4b58     CryEntityDLL.obj
 0002:00000b5c       ??_C@_0N@OFHMGPAL@unsigned?5int?$AA@ 320b4b5c     CryEntityDLL.obj
 0002:00000b6c       ??_C@_06KKKLBFKN@uint64?$AA@ 320b4b6c     CryEntityDLL.obj
 0002:00000b74       ??_7CStructInfo@@6B@       320b4b74     CryEntityDLL.obj
 0002:00000ba8       ??_C@_01PKGAHCOL@?$CJ?$AA@ 320b4ba8     CryEntityDLL.obj
 0002:00000bac       ??_C@_01ODHLEDKK@?$CI?$AA@ 320b4bac     CryEntityDLL.obj
 0002:00000bb0       ??_C@_01IHBHIGKO@?0?$AA@   320b4bb0     CryEntityDLL.obj
 0002:00000bb4       ??_C@_01KHDNNMEB@?$AB?$AA@ 320b4bb4     CryEntityDLL.obj
 0002:00000bb8       ??_C@_01GMMHALAP@?A?$AA@   320b4bb8     CryEntityDLL.obj
 0002:00000bbc       ??_C@_01JMLOEEAK@?$IB?$AA@ 320b4bbc     CryEntityDLL.obj
 0002:00000bc0       ??_C@_01FHEEJDEE@A?$AA@    320b4bc0     CryEntityDLL.obj
 0002:00000bc4       ??_C@_0BJ@IBIGFDEG@ENTITY_EVENT_DEACTIVATED?$AA@ 320b4bc4     Entity.obj
 0002:00000be0       ??_C@_0BH@EJNOPPK@ENTITY_EVENT_ACTIVATED?$AA@ 320b4be0     Entity.obj
 0002:00000bf8       ??_C@_0BI@OIAIALFO@ENTITY_EVENT_CROSS_AREA?$AA@ 320b4bf8     Entity.obj
 0002:00000c10       ??_C@_0BD@CIIFOGIJ@ENTITY_EVENT_ONHIT?$AA@ 320b4c10     Entity.obj
 0002:00000c24       ??_C@_0BG@BPLAAKOA@ENTITY_EVENT_MATERIAL?$AA@ 320b4c24     Entity.obj
 0002:00000c3c       ??_C@_0BF@ONJGGNLL@ENTITY_EVENT_VISIBLE?$AA@ 320b4c3c     Entity.obj
 0002:00000c54       ??_C@_0BH@KHCFJHNL@ENTITY_EVENT_INVISIBLE?$AA@ 320b4c54     Entity.obj
 0002:00000c6c       ??_C@_0BM@ICKNMDHF@ENTITY_EVENT_POST_SERIALIZE?$AA@ 320b4c6c     Entity.obj
 0002:00000c88       ??_C@_0BL@LGMIIGJP@ENTITY_EVENT_PRE_SERIALIZE?$AA@ 320b4c88     Entity.obj
 0002:00000ca4       ??_C@_0CA@EEGOACHO@ENTITY_EVENT_LEAVE_SCRIPT_STATE?$AA@ 320b4ca4     Entity.obj
 0002:00000cc4       ??_C@_0CA@JEIJIDAF@ENTITY_EVENT_ENTER_SCRIPT_STATE?$AA@ 320b4cc4     Entity.obj
 0002:00000ce4       ??_C@_0BI@CNLMMDDN@ENTITY_EVENT_START_GAME?$AA@ 320b4ce4     Entity.obj
 0002:00000cfc       ??_C@_0BJ@BMNGHGEG@ENTITY_EVENT_START_LEVEL?$AA@ 320b4cfc     Entity.obj
 0002:00000d18       ??_C@_0BK@JOONPFAA@ENTITY_EVENT_LEVEL_LOADED?$AA@ 320b4d18     Entity.obj
 0002:00000d34       ??_C@_0BO@LBBEKNBP@ENTITY_EVENT_PREPHYSICSUPDATE?$AA@ 320b4d34     Entity.obj
 0002:00000d54       ??_C@_0BE@BAMBGIED@ENTITY_EVENT_RENDER?$AA@ 320b4d54     Entity.obj
 0002:00000d68       ??_C@_0BH@KGJBFPFI@ENTITY_EVENT_COLLISION?$AA@ 320b4d68     Entity.obj
 0002:00000d80       ??_C@_0BO@INOBKELA@ENTITY_EVENT_NOT_SEEN_TIMEOUT?$AA@ 320b4d80     Entity.obj
 0002:00000da0       ??_C@_0BI@OKCNKBEP@ENTITY_EVENT_SOUND_DONE?$AA@ 320b4da0     Entity.obj
 0002:00000db8       ??_C@_0BF@OFFEFNPA@ENTITY_EVENT_AI_DONE?$AA@ 320b4db8     Entity.obj
 0002:00000dd0       ??_C@_0BI@FPMKDKFN@ENTITY_EVENT_PHYS_BREAK?$AA@ 320b4dd0     Entity.obj
 0002:00000de8       ??_C@_0BL@NAPEGKHD@ENTITY_EVENT_PHYS_POSTSTEP?$AA@ 320b4de8     Entity.obj
 0002:00000e04       ??_C@_0BK@LMFLENAC@ENTITY_EVENT_MOVENEARAREA?$AA@ 320b4e04     Entity.obj
 0002:00000e20       ??_C@_0BM@CMJDDIFA@ENTITY_EVENT_MOVEINSIDEAREA?$AA@ 320b4e20     Entity.obj
 0002:00000e3c       ??_C@_0BL@CPBINCNC@ENTITY_EVENT_LEAVENEARAREA?$AA@ 320b4e3c     Entity.obj
 0002:00000e58       ??_C@_0BL@FKDAIG@ENTITY_EVENT_ENTERNEARAREA?$AA@ 320b4e58     Entity.obj
 0002:00000e74       ??_C@_0BH@PKOKBFAE@ENTITY_EVENT_LEAVEAREA?$AA@ 320b4e74     Entity.obj
 0002:00000e8c       ??_C@_0BH@PIBECLCM@ENTITY_EVENT_ENTERAREA?$AA@ 320b4e8c     Entity.obj
 0002:00000ea4       ??_C@_0BK@IEJKGJEC@ENTITY_EVENT_SCRIPT_EVENT?$AA@ 320b4ea4     Entity.obj
 0002:00000ec0       ??_C@_0CC@NGIDLLFG@ENTITY_EVENT_PHYSICS_CHANGE_STAT@ 320b4ec0     Entity.obj
 0002:00000ee4       ??_C@_0BM@JNHLGCIE@ENTITY_EVENT_ENABLE_PHYSICS?$AA@ 320b4ee4     Entity.obj
 0002:00000f00       ??_C@_0BE@MGMKGFNC@ENTITY_EVENT_UNHIDE?$AA@ 320b4f00     Entity.obj
 0002:00000f14       ??_C@_0BC@GBAANABE@ENTITY_EVENT_HIDE?$AA@ 320b4f14     Entity.obj
 0002:00000f28       ??_C@_0BE@LDAAMPD@ENTITY_EVENT_DELINK?$AA@ 320b4f28     Entity.obj
 0002:00000f3c       ??_C@_0BC@HJENOIM@ENTITY_EVENT_LINK?$AA@ 320b4f3c     Entity.obj
 0002:00000f50       ??_C@_0BJ@CHKHNOAF@ENTITY_EVENT_DETACH_THIS?$AA@ 320b4f50     Entity.obj
 0002:00000f6c       ??_C@_0BE@LNOBDIMP@ENTITY_EVENT_DETACH?$AA@ 320b4f6c     Entity.obj
 0002:00000f80       ??_C@_0BJ@NAHMLCBO@ENTITY_EVENT_ATTACH_THIS?$AA@ 320b4f80     Entity.obj
 0002:00000f9c       ??_C@_0BE@CHFDMGFG@ENTITY_EVENT_ATTACH?$AA@ 320b4f9c     Entity.obj
 0002:00000fb0       ??_C@_0BD@GOBPOPCH@ENTITY_EVENT_RESET?$AA@ 320b4fb0     Entity.obj
 0002:00000fc4       ??_C@_0BH@HOCIFIMJ@ENTITY_EVENT_VISIBLITY?$AA@ 320b4fc4     Entity.obj
 0002:00000fdc       ??_C@_0BC@IMAMOHBP@ENTITY_EVENT_DONE?$AA@ 320b4fdc     Entity.obj
 0002:00000ff0       ??_C@_0BC@JKLGHBFO@ENTITY_EVENT_INIT?$AA@ 320b4ff0     Entity.obj
 0002:00001004       ??_C@_0BD@JLCKGGBB@ENTITY_EVENT_TIMER?$AA@ 320b5004     Entity.obj
 0002:00001018       ??_C@_0BD@BAICECFL@ENTITY_EVENT_XFORM?$AA@ 320b5018     Entity.obj
 0002:00001080       ??_7IEntityProxy@@6B@      320b5080     Entity.obj
 0002:000010b8       ??_7IAttachmentObject@@6B@ 320b50b8     Entity.obj
 0002:000010f8       ??_7IEntity@@6B@           320b50f8     Entity.obj
 0002:000012a0       ??_C@_01EOFPKCAF@?$EA?$AA@ 320b52a0     Entity.obj
 0002:000012a4       ??_7CEntityNodeProxy@@6B@  320b52a4     Entity.obj
 0002:000012d8       ??_7CEntityAttachment@@6B@ 320b52d8     Entity.obj
 0002:00001318       ??_C@_0GA@PJEHEJL@?$CBUnremovable?5entities?5should?5nev@ 320b5318     Entity.obj
 0002:00001378       ??_C@_0DM@PNDBMDH@Couldn?8t?5create?5entity?5?$CFs?3?5proxy@ 320b5378     Entity.obj
 0002:000013b8       ??_C@_0IF@JOMDHMIM@?$CBTrying?5to?5dynamically?5load?5ligh@ 320b53b8     Entity.obj
 0002:00001440       ??_C@_0CN@DKGEIDCE@?$DMFrame?3?$CFd?$DO?$DMEntityEvent?$DO?5?$FL?$CFs?$FN?$CI?$CFX?$CJ@ 320b5440     Entity.obj
 0002:00001470       ??_C@_02DPKJAMEF@?$CFd?$AA@ 320b5470     Entity.obj
 0002:00001474       __real@3fc90fdb            320b5474     Entity.obj
 0002:00001478       ??_C@_0O@LFGNNOCC@LUA?5call?5?$CI?$CFs?$CJ?$AA@ 320b5478     Entity.obj
 0002:00001488       ??_7CSubstitutionProxy@@6B@ 320b5488     Entity.obj
 0002:000014c4       __real@399d4952            320b54c4     Entity.obj
 0002:000014c8       ??_C@_0BA@FAFOPGPI@CEntity?3?3Update?$AA@ 320b54c8     Entity.obj
 0002:000014d8       ??_C@_0BK@INBLJDKJ@CEntity?3?3PrePhysicsUpdate?$AA@ 320b54d8     Entity.obj
 0002:000014f8       ??_7CEntity@@6B@           320b54f8     Entity.obj
 0002:000016b4       __real@3a83126f            320b56b4     Entity.obj
 0002:000016b8       ??_C@_08GHMHMIKM@__usable?$AA@ 320b56b8     Entity.obj
 0002:000016c4       ??_C@_09FKAPMINN@bHasSubst?$AA@ 320b56c4     Entity.obj
 0002:000016d0       ??_C@_0O@KCMNDECC@EntityProxies?$AA@ 320b56d0     Entity.obj
 0002:000016e0       ??_C@_0L@NDJPGNLG@sshidemask?$AA@ 320b56e0     Entity.obj
 0002:000016ec       ??_C@_05NAKFKLNM@noobj?$AA@ 320b56ec     Entity.obj
 0002:000016f4       ??_C@_04IJEANHEE@mass?$AA@ 320b56f4     Entity.obj
 0002:000016fc       ??_C@_06HDLLMMEJ@update?$AA@ 320b56fc     Entity.obj
 0002:00001704       ??_C@_05GECEPKB@flags?$AA@ 320b5704     Entity.obj
 0002:0000170c       ??_C@_06OIIICDLO@XformT?$AA@ 320b570c     Entity.obj
 0002:00001714       ??_C@_06NLCPOPJP@Xform2?$AA@ 320b5714     Entity.obj
 0002:0000171c       ??_C@_06PAACLMFM@Xform1?$AA@ 320b571c     Entity.obj
 0002:00001724       ??_C@_06OJBJINBN@Xform0?$AA@ 320b5724     Entity.obj
 0002:0000172c       ??_C@_08CNEAOEII@hasXform?$AA@ 320b572c     Entity.obj
 0002:00001738       ??_C@_02EGCJHIOB@id?$AA@   320b5738     Entity.obj
 0002:0000173c       ??_C@_04DPEGMFKN@Slot?$AA@ 320b573c     Entity.obj
 0002:00001744       ??_C@_08GGFNOLHJ@numslots?$AA@ 320b5744     Entity.obj
 0002:00001750       ??_C@_08OHGOKOGA@rotation?$AA@ 320b5750     Entity.obj
 0002:0000175c       ??_C@_05MHMEBBGO@scale?$AA@ 320b575c     Entity.obj
 0002:00001764       ??_C@_08OAGMDKAF@position?$AA@ 320b5764     Entity.obj
 0002:00001770       ??_C@_09KOIOCIHC@?$DMUNKNOWN?$DO?$AA@ 320b5770     Entity.obj
 0002:0000177c       ??_C@_0BF@LGBKNEBF@Entity?5serialization?$AA@ 320b577c     Entity.obj
 0002:00001794       ??_C@_08NNGAPGNE@LightBox?$AA@ 320b5794     Entity.obj
 0002:000017a0       ??_C@_0L@KKEKGINL@LightShape?$AA@ 320b57a0     Entity.obj
 0002:000017ac       ??_C@_01JOAMLHOP@?9?$AA@   320b57ac     Entity.obj
 0002:000017b0       ??_C@_02GFKOMOKH@?5?$CI?$AA@ 320b57b0     Entity.obj
 0002:000017b4       ??_C@_05MHNANJII@sound?$AA@ 320b57b4     Entity.obj
 0002:000017bc       ??_C@_0M@KOOCGHBK@AreaTrigger?$AA@ 320b57bc     Entity.obj
 0002:000017c8       ??_C@_0BB@HHHBOMJ@ProximityTrigger?$AA@ 320b57c8     Entity.obj
 0002:000017dc       ??_C@_0BD@LANHDIFF@CEntity?3?3SendEvent?$AA@ 320b57dc     Entity.obj
 0002:000017f0       ??_C@_0BC@KCBBFLJK@CEntity?3?3ShutDown?$AA@ 320b57f0     Entity.obj
 0002:00001804       ??_C@_0O@LIJMHNDI@OnBeingReused?$AA@ 320b5804     Entity.obj
 0002:00001814       ??_C@_0CI@ONOHKGPC@Trying?5to?5attaching?5Entity?5?$CFs?5to@ 320b5814     Entity.obj
 0002:0000183c       ??_7?$_i_reference_target@H@@6B@ 320b583c     EntityArchetype.obj
 0002:00001848       ??_C@_0CI@IOKCCNHB@Deleting?5Reference?5Counted?5Objec@ 320b5848     EntityArchetype.obj
 0002:00001870       ??_C@_0IC@DFBDLODH@?$FLEntitySystem?$FN?5CEntityArchetype?3@ 320b5870     EntityArchetype.obj
 0002:000018f4       ??_C@_0BO@CFCDFDLK@AdditionalArchetypeProperties?$AA@ 320b58f4     EntityArchetype.obj
 0002:00001914       ??_C@_08DFDJKJDE@?$CFs?5Begin?$AA@ 320b5914     EntityArchetype.obj
 0002:00001920       ??_C@_06FMHDIGFH@?$CFs?5End?$AA@ 320b5920     EntityArchetype.obj
 0002:00001928       ??_7CEntityArchetype@@6B?$_i_reference_target@H@@@ 320b5928     EntityArchetype.obj
 0002:00001934       ??_7CEntityArchetype@@6BIEntityArchetype@@@ 320b5934     EntityArchetype.obj
 0002:00001948       ??_C@_01LFCBOECM@?4?$AA@   320b5948     EntityArchetype.obj
 0002:0000194c       ??_C@_01KMDKNFGN@?1?$AA@   320b594c     EntityArchetype.obj
 0002:00001950       ??_C@_0BP@FDAILCID@CEntityArchetypeManager?3?3Reset?$AA@ 320b5950     EntityArchetype.obj
 0002:00001970       ??_C@_0L@KOOGALIH@Properties?$AA@ 320b5970     EntityArchetype.obj
 0002:0000197c       ??_C@_0DG@ENHPFPFP@EntityArchetype?5?$CFs?5references?5un@ 320b597c     EntityArchetype.obj
 0002:000019b4       ??_C@_05EKAMNAII@Class?$AA@ 320b59b4     EntityArchetype.obj
 0002:000019bc       ??_C@_04FABLJDN@Name?$AA@  320b59bc     EntityArchetype.obj
 0002:000019c4       ??_C@_0BA@OJLJDANF@EntityPrototype?$AA@ 320b59c4     EntityArchetype.obj
 0002:000019d4       ??_C@_03PJHHNEEI@xml?$AA@  320b59d4     EntityArchetype.obj
 0002:000019d8       ??_C@_0BI@HKJJINHI@?1Libs?1EntityArchetypes?1?$AA@ 320b59d8     EntityArchetype.obj
 0002:000019f0       ??_C@_03NFKEKGGK@all?$AA@  320b59f0     EntityCVars.obj
 0002:000019f4       ??_C@_0BG@NODPPGBF@OnSysSpecLightChanged?$AA@ 320b59f4     EntityCVars.obj
 0002:00001a0c       ??_C@_0BB@HKHKCKIB@?$CFs?3?5?$CFd?5instances?$AA@ 320b5a0c     EntityCVars.obj
 0002:00001a20       ??_C@_0FB@DCLGMKGJ@?9?9?9?9?9?9?9?9?9?9?9?9?9?9?9?9?9?9?9?9?9?9?9?9?9?9?9?9?9?9?9?9@ 320b5a20     EntityCVars.obj
 0002:00001a74       ??_C@_0N@IFGNLJBD@es_debugAnim?$AA@ 320b5a74     EntityCVars.obj
 0002:00001a84       ??_C@_0CH@BIIFLLFJ@Debug?5entity?5animation?5?$CItoggle?5o@ 320b5a84     EntityCVars.obj
 0002:00001aac       ??_C@_0BH@NCMMLOCL@es_debugEntityLifetime?$AA@ 320b5aac     EntityCVars.obj
 0002:00001ac4       ??_C@_0CK@EGOJOAFB@Debug?5entities?5creation?5and?5dele@ 320b5ac4     EntityCVars.obj
 0002:00001af0       ??_C@_0P@HOBDKNLF@sys_spec_light?$AA@ 320b5af0     EntityCVars.obj
 0002:00001b00       ??_C@_0N@GIOHDHOI@r_MotionBlur?$AA@ 320b5b00     EntityCVars.obj
 0002:00001b10       ??_C@_0BC@IMPLDGCP@es_FarPhysTimeout?$AA@ 320b5b10     EntityCVars.obj
 0002:00001b24       ??_C@_0DC@INGILDLE@Timeout?5for?5faraway?5physics?5forc@ 320b5b24     EntityCVars.obj
 0002:00001b58       ??_C@_0BI@EPOIFJOO@es_MaxPhysDistInvisible?$AA@ 320b5b58     EntityCVars.obj
 0002:00001b70       ??_C@_0FJ@OHFJBKE@Invisible?5physical?5entities?5fart@ 320b5b70     EntityCVars.obj
 0002:00001bcc       __real@42200000            320b5bcc     EntityCVars.obj
 0002:00001bd0       ??_C@_0BE@OEEPLMIL@es_MaxPhysDistCloth?$AA@ 320b5bd0     EntityCVars.obj
 0002:00001be8       ??_C@_0EM@CBAMAEFM@Cloth?5entities?5farther?5from?5the?5@ 320b5be8     EntityCVars.obj
 0002:00001c34       ??_C@_0P@EIMKHFDE@es_MaxPhysDist?$AA@ 320b5c34     EntityCVars.obj
 0002:00001c48       ??_C@_0EP@GJGPCIDF@Physical?5entities?5farther?5from?5t@ 320b5c48     EntityCVars.obj
 0002:00001c98       __real@43960000            320b5c98     EntityCVars.obj
 0002:00001c9c       ??_C@_0BL@IBLKECML@es_UsePhysVisibilityChecks?$AA@ 320b5c9c     EntityCVars.obj
 0002:00001cb8       ??_C@_0FP@CLJBIOIG@Activates?5physics?5quality?5degrad@ 320b5cb8     EntityCVars.obj
 0002:00001d18       ??_C@_0BG@OAILAMMC@es_DrawSoundProxyZRay?$AA@ 320b5d18     EntityCVars.obj
 0002:00001d30       ??_C@_0DD@FEOBDONC@Enables?5drawing?5of?5Z?5ray?5on?5chec@ 320b5d30     EntityCVars.obj
 0002:00001d64       ??_C@_0BB@ENOCPFOB@es_DrawAreaDebug?$AA@ 320b5d64     EntityCVars.obj
 0002:00001d78       ??_C@_0DG@LGHLGGHI@Enables?5debug?5drawing?5of?5Areas?0?5@ 320b5d78     EntityCVars.obj
 0002:00001db0       ??_C@_0BA@FGKAJEJM@es_DrawAreaGrid?$AA@ 320b5db0     EntityCVars.obj
 0002:00001dc0       ??_C@_0BN@DIOOMDKJ@Enables?5drawing?5of?5Area?5Grid?$AA@ 320b5dc0     EntityCVars.obj
 0002:00001de0       ??_C@_0N@CBKGEOKK@es_DrawAreas?$AA@ 320b5de0     EntityCVars.obj
 0002:00001df0       ??_C@_0BJ@GBEPDBLC@Enables?5drawing?5of?5Areas?$AA@ 320b5df0     EntityCVars.obj
 0002:00001e0c       ??_C@_0O@NMNIKCJB@es_updateType?$AA@ 320b5e0c     EntityCVars.obj
 0002:00001e1c       ??_C@_0CM@JBCHFHFL@Defines?5how?5we?5update?5type?5for?5t@ 320b5e1c     EntityCVars.obj
 0002:00001e48       ??_C@_0CD@BCDNFHNI@es_ClearPoolBookmarksOnLayerUnlo@ 320b5e48     EntityCVars.obj
 0002:00001e70       ??_C@_0FF@HMIHPIFL@Clear?5pool?5bookmarks?5when?5a?5laye@ 320b5e70     EntityCVars.obj
 0002:00001ec8       ??_C@_0BM@JCAIPKML@es_SaveLoadUseLUANoSaveFlag?$AA@ 320b5ec8     EntityCVars.obj
 0002:00001ee8       ??_C@_0FL@GGBDGODC@Save?$CGLoad?5optimization?5?3?5use?5lua@ 320b5ee8     EntityCVars.obj
 0002:00001f44       ??_C@_0BC@MHKFOHEH@es_LayerDebugInfo?$AA@ 320b5f44     EntityCVars.obj
 0002:00001f58       ??_C@_0IF@NCMHAIHP@Render?5debug?5info?5on?5active?5laye@ 320b5f58     EntityCVars.obj
 0002:00001fe0       ??_C@_0BO@PGAOBOMA@es_LayerSaveLoadSerialization?$AA@ 320b5fe0     EntityCVars.obj
 0002:00002000       ??_C@_0JM@CJGGOEIA@Switches?5layer?5entity?5serializat@ 320b6000     EntityCVars.obj
 0002:0000209c       ??_C@_0BD@HNLIDPFA@es_DebugPoolFilter?$AA@ 320b609c     EntityCVars.obj
 0002:000020b0       ??_C@_0EM@DGNJGCAG@Filter?5entity?5pool?5debugging?5for@ 320b60b0     EntityCVars.obj
 0002:000020fc       ??_C@_0BG@EKCIIFFF@es_TestPoolSignatures?$AA@ 320b60fc     EntityCVars.obj
 0002:00002118       ??_C@_0FP@BJILCDNF@Enable?5signature?5testing?5on?5enti@ 320b6118     EntityCVars.obj
 0002:00002178       ??_C@_0N@DCJKCOGH@es_DebugPool?$AA@ 320b6178     EntityCVars.obj
 0002:00002188       ??_C@_0CF@LJLPFEFN@Enable?5debug?5drawing?5of?5entity?5p@ 320b6188     EntityCVars.obj
 0002:000021b0       ??_C@_0BB@PFNNKLAP@es_EnablePoolUse?$AA@ 320b61b0     EntityCVars.obj
 0002:000021c8       ??_C@_0JD@PBNOKCEA@Force?5toggle?5the?5use?5of?5entity?5p@ 320b61c8     EntityCVars.obj
 0002:0000225c       ??_C@_0BK@GHIGKNOI@es_DebugEntityUsageFilter?$AA@ 320b625c     EntityCVars.obj
 0002:00002278       ??_C@_0EO@PCBLAGOO@Filter?5entity?5usage?5debugging?5to@ 320b6278     EntityCVars.obj
 0002:000022c8       ??_C@_0BE@BHJMLICC@es_DebugEntityUsage?$AA@ 320b62c8     EntityCVars.obj
 0002:000022e0       ??_C@_0PP@LJLPCFJL@Draws?5information?5to?5the?5screen?5@ 320b62e0     EntityCVars.obj
 0002:000023e0       ??_C@_0BJ@JCPOFFFK@es_DrawProximityTriggers?$AA@ 320b63e0     EntityCVars.obj
 0002:00002400       ??_C@_0KK@CCDPIAPA@Shows?5Proximity?5Triggers?4?6Usage?3@ 320b6400     EntityCVars.obj
 0002:000024ac       ??_C@_0BD@EDBCGJKM@es_DisableTriggers?$AA@ 320b64ac     EntityCVars.obj
 0002:000024c0       ??_C@_0DL@FGFHHFNF@Disable?5enter?1leave?5events?5for?5p@ 320b64c0     EntityCVars.obj
 0002:000024fc       ??_C@_0P@FAAGBIJM@es_DebugEvents?$AA@ 320b64fc     EntityCVars.obj
 0002:0000250c       ??_C@_0CB@KEHNDBLA@Enables?5logging?5of?5entity?5events@ 320b650c     EntityCVars.obj
 0002:00002530       ??_C@_0BD@NCGFCHMB@es_DebugFindEntity?$AA@ 320b6530     EntityCVars.obj
 0002:00002544       ??_C@_0P@IANDIPNK@es_DebugTimers?$AA@ 320b6544     EntityCVars.obj
 0002:00002558       ??_C@_0BGJ@EHMAEKCO@This?5is?5for?5profiling?5and?5debugg@ 320b6558     EntityCVars.obj
 0002:000026c4       ??_C@_0BC@PMMIENKA@es_log_collisions?$AA@ 320b66c4     EntityCVars.obj
 0002:000026d8       ??_C@_0CB@LFNGFEKA@Enables?5collision?5events?5logging@ 320b66d8     EntityCVars.obj
 0002:000026fc       ??_C@_0BL@HPLFKGAE@es_enable_full_script_save?$AA@ 320b66fc     EntityCVars.obj
 0002:00002718       ??_C@_0DF@JOOJOENM@Enable?5?$CIexperimental?$CJ?5full?5scrip@ 320b6718     EntityCVars.obj
 0002:00002750       ??_C@_0BK@BFPGIJA@es_debug_not_seen_timeout?$AA@ 320b6750     EntityCVars.obj
 0002:0000276c       ??_C@_0DN@NJFBBHKP@if?5true?0?5log?5messages?5when?5entit@ 320b676c     EntityCVars.obj
 0002:000027ac       ??_C@_0BE@GIJBGGML@es_not_seen_timeout?$AA@ 320b67ac     EntityCVars.obj
 0002:000027c0       ??_C@_0EM@DOHDAAOC@number?5of?5seconds?5after?5which?5to@ 320b67c0     EntityCVars.obj
 0002:0000280c       ??_C@_0BE@JFCCOAAG@es_CharZOffsetSpeed?$AA@ 320b680c     EntityCVars.obj
 0002:00002820       ??_C@_0DP@KABFHEE@sets?5the?5character?5Z?9offset?5chan@ 320b6820     EntityCVars.obj
 0002:00002860       ??_C@_0BB@EFGMBLKE@es_HitDeadBodies?$AA@ 320b6860     EntityCVars.obj
 0002:00002878       ??_C@_0ED@LLDBGENK@specifies?5whether?5dead?5bodies?5ar@ 320b6878     EntityCVars.obj
 0002:000028bc       ??_C@_0BB@JJLFMDIO@es_HitCharacters?$AA@ 320b68bc     EntityCVars.obj
 0002:000028d0       ??_C@_0EI@FBLECOIB@specifies?5whether?5alive?5characte@ 320b68d0     EntityCVars.obj
 0002:00002918       ??_C@_0BB@GKGLJDLP@es_SplashTimeout?$AA@ 320b6918     EntityCVars.obj
 0002:00002930       ??_C@_0EO@IDGPCEFL@minimum?5time?5interval?5between?5co@ 320b6930     EntityCVars.obj
 0002:00002980       ??_C@_0BD@JDJLPAIM@es_SplashThreshold?$AA@ 320b6980     EntityCVars.obj
 0002:00002998       ??_C@_0GD@GEDMPCOC@minimum?5instantaneous?5water?5resi@ 320b6998     EntityCVars.obj
 0002:000029fc       ??_C@_0BH@KIBPFKIJ@es_DebrisLifetimeScale?$AA@ 320b69fc     EntityCVars.obj
 0002:00002a14       ??_C@_0CC@EBGFAGPD@Usage?3?5es_DebrisLifetimeScale?51?4@ 320b6a14     EntityCVars.obj
 0002:00002a38       ??_C@_0BF@KOFFBMGC@es_MaxImpulseAdjMass?$AA@ 320b6a38     EntityCVars.obj
 0002:00002a50       ??_C@_0CD@PJGJPNKL@Usage?3?5es_MaxImpulseAdjMass?52000@ 320b6a50     EntityCVars.obj
 0002:00002a74       __real@44fa0000            320b6a74     EntityCVars.obj
 0002:00002a78       ??_C@_0BA@JLBGAMIK@es_ImpulseScale?$AA@ 320b6a78     EntityCVars.obj
 0002:00002a88       ??_C@_0BL@CDFCDIFC@Usage?3?5es_ImpulseScale?50?40?$AA@ 320b6a88     EntityCVars.obj
 0002:00002aa4       ??_C@_0BB@EHONFFNI@es_MinImpulseVel?$AA@ 320b6aa4     EntityCVars.obj
 0002:00002ab8       ??_C@_0BM@CKFDNHFG@Usage?3?5es_MinImpulseVel?50?40?$AA@ 320b6ab8     EntityCVars.obj
 0002:00002ad4       ??_C@_0BF@CIJJPKFK@es_VisCheckForUpdate?$AA@ 320b6ad4     EntityCVars.obj
 0002:00002aec       ??_C@_0DF@OGMEBMGJ@Usage?3?5es_VisCheckForUpdate?5?$FL0?11@ 320b6aec     EntityCVars.obj
 0002:00002b24       ??_C@_0BJ@IKODCMEB@es_UpdateCollisionScript?$AA@ 320b6b24     EntityCVars.obj
 0002:00002b40       ??_C@_0DJ@PIBONJBJ@Usage?3?5es_UpdateCollisionScript?5@ 320b6b40     EntityCVars.obj
 0002:00002b7c       ??_C@_0P@EAHPKDDM@es_UpdateTimer?$AA@ 320b6b7c     EntityCVars.obj
 0002:00002b8c       ??_C@_0CP@CCMGPPCJ@Usage?3?5es_UpdateTimer?5?$FL0?11?$FN?6Defa@ 320b6b8c     EntityCVars.obj
 0002:00002bbc       ??_C@_0BD@NPHKAEIN@es_UpdateContainer?$AA@ 320b6bbc     EntityCVars.obj
 0002:00002bd0       ??_C@_0DD@FLOOMCPB@Usage?3?5es_UpdateContainer?5?$FL0?11?$FN?6@ 320b6bd0     EntityCVars.obj
 0002:00002c04       ??_C@_0BD@HJFKDMCF@es_UpdateCollision?$AA@ 320b6c04     EntityCVars.obj
 0002:00002c18       ??_C@_0IJ@FIKMENHJ@Toggles?5updating?5of?5entity?5colli@ 320b6c18     EntityCVars.obj
 0002:00002ca4       ??_C@_0BC@NPHLLHKJ@es_UpdateEntities?$AA@ 320b6ca4     EntityCVars.obj
 0002:00002cb8       ??_C@_0HL@BGEGINNC@Toggles?5entity?5updating?4?6Usage?3?5@ 320b6cb8     EntityCVars.obj
 0002:00002d34       ??_C@_0M@GDIJLIJK@es_UpdateAI?$AA@ 320b6d34     EntityCVars.obj
 0002:00002d40       ??_C@_0HM@CJPHAHD@Toggles?5updating?5of?5AI?5entities?4@ 320b6d40     EntityCVars.obj
 0002:00002dbc       ??_C@_0BB@KAGNGDOB@es_UpdatePhysics?$AA@ 320b6dbc     EntityCVars.obj
 0002:00002dd0       ??_C@_0IH@OPOOGIHK@Toggles?5updating?5of?5entity?5physi@ 320b6dd0     EntityCVars.obj
 0002:00002e58       ??_C@_0BA@KLKCMJLL@es_UpdateScript?$AA@ 320b6e58     EntityCVars.obj
 0002:00002e68       ??_C@_0DA@HIIFJEMN@Usage?3?5es_UpdateScript?5?$FL0?11?$FN?6Def@ 320b6e68     EntityCVars.obj
 0002:00002e98       ??_C@_0BD@OGKJNNPK@es_profileentities?$AA@ 320b6e98     EntityCVars.obj
 0002:00002eac       ??_C@_0DE@NIJJBDIE@Usage?3?5es_profileentities?51?02?03?6@ 320b6eac     EntityCVars.obj
 0002:00002ee0       ??_C@_0L@GJFKCMN@es_helpers?$AA@ 320b6ee0     EntityCVars.obj
 0002:00002ef0       ??_C@_0GB@IAGLOMHE@Toggles?5helpers?4?6Usage?3?5es_helpe@ 320b6ef0     EntityCVars.obj
 0002:00002f54       ??_C@_09MIGBPOEL@es_bboxes?$AA@ 320b6f54     EntityCVars.obj
 0002:00002f60       ??_C@_0GO@KHFCALII@Toggles?5entity?5bounding?5boxes?4?6U@ 320b6f60     EntityCVars.obj
 0002:00002fd0       ??_C@_0O@GNMFEIHI@p_CharacterIK?$AA@ 320b6fd0     EntityCVars.obj
 0002:00002fe0       ??_C@_0GM@FCPIHGOI@Toggles?5character?5IK?4?6Usage?3?5p_c@ 320b6fe0     EntityCVars.obj
 0002:0000304c       ??_C@_08NDFOPNLF@es_debug?$AA@ 320b704c     EntityCVars.obj
 0002:00003058       ??_C@_0EG@DKPILDCM@Enable?5entity?5debugging?5info?6Usa@ 320b7058     EntityCVars.obj
 0002:000030a0       ??_C@_0BG@HPCFKBMM@es_SortUpdatesByClass?$AA@ 320b70a0     EntityCVars.obj
 0002:000030b8       ??_C@_0DF@IEGOFJCO@Sort?5entity?5updates?5by?5class?5?$CIpo@ 320b70b8     EntityCVars.obj
 0002:000030f0       ??_C@_0BC@INDJFIJI@es_dump_bookmarks?$AA@ 320b70f0     EntityCVars.obj
 0002:00003104       ??_C@_0DA@IECMDIAB@Dumps?5information?5about?5all?5book@ 320b7104     EntityCVars.obj
 0002:00003134       ??_C@_0BF@EKJGINDM@es_compile_area_grid?$AA@ 320b7134     EntityCVars.obj
 0002:0000314c       ??_C@_0CF@IHNLAIIK@Trigger?5a?5recompile?5of?5the?5area?5@ 320b714c     EntityCVars.obj
 0002:00003174       ??_C@_0BO@CALCHBBE@es_dump_entity_classes_in_use?$AA@ 320b7174     EntityCVars.obj
 0002:00003194       ??_C@_0BO@JAEAONPP@Dumps?5all?5used?5entity?5classes?$AA@ 320b7194     EntityCVars.obj
 0002:000031b4       ??_C@_0BB@ELLFLJEB@es_dump_entities?$AA@ 320b71b4     EntityCVars.obj
 0002:000031c8       ??_C@_0CJ@HGPAGMPO@Dumps?5current?5entities?5and?5their@ 320b71c8     EntityCVars.obj
 0002:000031f4       ??_7IEntityEventDistributer@@6B@ 320b71f4     EntityEventDistributer.obj
 0002:00003218       ?_list@?1??_S_primes@?$_Stl_prime@_N@priv@stlpmtx_std@@CAPBIAAI@Z@4QBIB 320b7218     EntityEventDistributer.obj
 0002:00003290       ??_7CEntityEventDistributer@@6B@ 320b7290     EntityEventDistributer.obj
 0002:000032b0       ??_C@_0L@PIOLEGBL@Constraint?$AA@ 320b72b0     EntityLayer.obj
 0002:000032bc       ??_C@_0M@CJMKOLJE@Deactivated?$AA@ 320b72bc     EntityLayer.obj
 0002:000032c8       ??_C@_09OMCOPAKI@Activated?$AA@ 320b72c8     EntityLayer.obj
 0002:000032d4       ??_C@_0O@HEIHEFCJ@Layer?5?8?$CFs?8?5?$CFs?$AA@ 320b72d4     EntityLayer.obj
 0002:000032e4       ??_C@_0N@JKLGFKLI@Deactivating?$AA@ 320b72e4     EntityLayer.obj
 0002:000032f4       ??_C@_0L@LFBMMCCE@Activating?$AA@ 320b72f4     EntityLayer.obj
 0002:00003300       ??_7CEntityLayer@@6B@      320b7300     EntityLayer.obj
 0002:00003304       ??_C@_06MDLIGPKC@active?$AA@ 320b7304     EntityLayer.obj
 0002:0000330c       ??_C@_07HCCGGAEA@noAwake?$AA@ 320b730c     EntityLayer.obj
 0002:00003314       ??_C@_06JIKFICKK@hidden?$AA@ 320b7314     EntityLayer.obj
 0002:0000331c       ??_C@_08JJAAIGGM@entityId?$AA@ 320b731c     EntityLayer.obj
 0002:00003328       ??_C@_0O@JKHLLEJG@LayerEntities?$AA@ 320b7328     EntityLayer.obj
 0002:00003338       ??_C@_05IOMEMJEC@count?$AA@ 320b7338     EntityLayer.obj
 0002:00003340       ??_C@_0P@HHIIGJCA@m_isSerialized?$AA@ 320b7340     EntityLayer.obj
 0002:00003350       ??_C@_0N@FNCJDJMK@enabledBrush?$AA@ 320b7350     EntityLayer.obj
 0002:00003360       ??_C@_07MHHIKOPA@enabled?$AA@ 320b7360     EntityLayer.obj
 0002:00003368       ??_C@_04MEMAJGDJ@name?$AA@ 320b7368     EntityLayer.obj
 0002:00003370       ??_C@_05NHNHDHBP@Layer?$AA@ 320b7370     EntityLayer.obj
 0002:00003378       ??_C@_06HPGEIPLA@?$DMnull?$DO?$AA@ 320b7378     EntitySystem.obj
 0002:00003380       ??_C@_07KAALEJHI@?$DMlocal?$DO?$AA@ 320b7380     EntitySystem.obj
 0002:0000338c       ??_7IEntityIt@@6B@         320b738c     EntitySystem.obj
 0002:000033a8       ??_7IEntitySystem@@6B@     320b73a8     EntitySystem.obj
 0002:00003494       ??_C@_0BG@ICFDNKJC@e_ViewDistRatioDetail?$AA@ 320b7494     EntitySystem.obj
 0002:000034ac       ??_C@_0BG@IMFDNAMJ@e_ViewDistRatioCustom?$AA@ 320b74ac     EntitySystem.obj
 0002:000034c4       ??_C@_0BA@ECEJHKAC@e_ViewDistRatio?$AA@ 320b74c4     EntitySystem.obj
 0002:000034d4       ??_C@_0O@LEAIHJGG@e_ViewDistMin?$AA@ 320b74d4     EntitySystem.obj
 0002:000034e4       __real@3727c5ac            320b74e4     EntitySystem.obj
 0002:000034e8       ??_7CEntityItMap@@6B@      320b74e8     EntitySystem.obj
 0002:00003504       __real@3f99999a            320b7504     EntitySystem.obj
 0002:00003508       ??_C@_09HGKPJIGD@triggered?$AA@ 320b7508     EntitySystem.obj
 0002:00003514       ??_C@_0CG@BBLNKDMC@CEntitySystem?3?3DoPrePhysicsUpdat@ 320b7514     EntitySystem.obj
 0002:0000353c       __real@4cbebc20            320b753c     EntitySystem.obj
 0002:00003540       ??_C@_0BM@NKGDGMMD@SEntityLoadParams?5Clone?5Xml?$AA@ 320b7540     EntitySystem.obj
 0002:0000355c       ??_C@_0CE@MNKCFDHL@CEntitySystem?3?3PostPumpLoggedEve@ 320b755c     EntitySystem.obj
 0002:00003580       ??_C@_0EG@CJDEIACM@CEntitySystem?3?3LoadEntities?5?3?5No@ 320b7580     EntitySystem.obj
 0002:000035c8       ??_C@_0EH@NNFGLMKL@CEntitySystem?3?3LoadEntities?5?3?5Fa@ 320b75c8     EntitySystem.obj
 0002:00003610       ??_C@_0N@KCOGAMLF@LoadEntities?$AA@ 320b7610     EntitySystem.obj
 0002:00003620       ??_C@_0BM@CBCGNGHE@CEntitySystem?3?3LoadEntities?$AA@ 320b7620     EntitySystem.obj
 0002:0000363c       ??_C@_0BL@CIPOHCKE@Entity?3?5?5?$CF8?45f?5?$CF8?45f?5?$CF8?45f?$AA@ 320b763c     EntitySystem.obj
 0002:00003658       __real@3dcccccd            320b7658     EntitySystem.obj
 0002:0000365c       ??_C@_0BL@BNODFFGE@Physics?3?5?$CF8?45f?5?$CF8?45f?5?$CF8?45f?$AA@ 320b765c     EntitySystem.obj
 0002:00003678       __real@3f8ccccd            320b7678     EntitySystem.obj
 0002:0000367c       __real@3fcccccd            320b767c     EntitySystem.obj
 0002:00003680       __real@3fa66666            320b7680     EntitySystem.obj
 0002:00003684       ??_C@_0N@KAKPEJDJ@?$CF?43f?5ms?5?3?5?$CFs?$AA@ 320b7684     EntitySystem.obj
 0002:00003694       ??_C@_0BJ@MNHGEMHI@?$CF?43f?5ms?5?3?5?$CFs?5?$CI?$CF0?42f?5ago?$CJ?$AA@ 320b7694     EntitySystem.obj
 0002:000036b0       ??_C@_0CF@OAMBGBJA@CEntitySystem?3?3UpdateNotSeenTime@ 320b76b0     EntitySystem.obj
 0002:000036d8       ??_C@_0BG@OHHHPLBD@CharacterAttachHelper?$AA@ 320b76d8     EntitySystem.obj
 0002:000036f0       ??_C@_0CC@GGAKFHAK@CEntitySystem?3?3DoPrePhysicsUpdat@ 320b76f0     EntitySystem.obj
 0002:00003714       ??_C@_0BF@OICFAIPE@FindEntityByName?3?5?$CFs?$AA@ 320b7714     EntitySystem.obj
 0002:0000372c       ??_C@_0BI@MDNHCBAA@FindEntityByGuid?3?5?$CFI64X?$AA@ 320b772c     EntitySystem.obj
 0002:00003744       ??_C@_05NNFHCGPF@?$CFs?4?$CFs?$AA@ 320b7744     EntitySystem.obj
 0002:0000374c       ??_C@_07BGPNANBL@Library?$AA@ 320b774c     EntitySystem.obj
 0002:00003754       ??_C@_0BE@KJDJFMJA@STL?5Allocator?5Waste?$AA@ 320b7754     EntitySystem.obj
 0002:00003768       ??_C@_0L@BMGKBDKM@EntityLoad?$AA@ 320b7768     EntitySystem.obj
 0002:00003774       ??_C@_0L@HLDNMOCN@EntityPool?$AA@ 320b7774     EntitySystem.obj
 0002:00003780       ??_C@_08HPDMGIEC@Entities?$AA@ 320b7780     EntitySystem.obj
 0002:0000378c       ??_C@_0O@JEAHIPMK@DefaultLoaded?$AA@ 320b778c     EntitySystem.obj
 0002:0000379c       ??_C@_05HPIOJMLH@Specs?$AA@ 320b779c     EntitySystem.obj
 0002:000037a4       ??_C@_07ONFAPAAB@Physics?$AA@ 320b77a4     EntitySystem.obj
 0002:000037ac       ??_C@_02HOGEDOAB@Id?$AA@   320b77ac     EntitySystem.obj
 0002:000037b0       ??_C@_06EBOPLIP@Parent?$AA@ 320b77b0     EntitySystem.obj
 0002:000037b8       ??_C@_06IJMNPAPH@Layers?$AA@ 320b77b8     EntitySystem.obj
 0002:000037c0       ??_C@_0BK@KPLPDAAO@CEntitySystem?3?3LoadLayers?$AA@ 320b77c0     EntitySystem.obj
 0002:000037dc       ??_C@_0L@LAOEILMP@bSerialize?$AA@ 320b77dc     EntitySystem.obj
 0002:000037e8       ??_C@_0CG@LMKGPMLB@CEntitySystem?3?3SpawnEntity?5?$CFs?5?$CFs@ 320b77e8     EntitySystem.obj
 0002:00003810       ??_C@_04MLLLIHIP@null?$AA@ 320b7810     EntitySystem.obj
 0002:00003818       ??_C@_0EA@FHHEFFF@Entity?5with?5id?$DN?$CFd?0?5?$CFs?5already?5sp@ 320b7818     EntitySystem.obj
 0002:00003858       ??_C@_0FM@IHGOPIJB@CEntitySystem?3?3SpawnEntity?5Faile@ 320b7858     EntitySystem.obj
 0002:000038b8       ??_C@_0GJ@DLOPDNOA@Spawning?5entity?5?$CFs?5of?5class?5?$CFs?5r@ 320b78b8     EntitySystem.obj
 0002:00003924       ??_C@_0P@PIGDNLGP@SpawnEntity?5?$CFs?$AA@ 320b7924     EntitySystem.obj
 0002:00003938       ??_C@_0EP@IOENKEJM@?$CBName?5?8?$CFs?8?5contains?5?$CFu?5illegal?5c@ 320b7938     EntitySystem.obj
 0002:00003988       ??_C@_0BD@MOFFFFDL@no?5class?5specified?$AA@ 320b7988     EntitySystem.obj
 0002:0000399c       ??_C@_0BL@IOIAFOBC@CEntitySystem?3?3SpawnEntity?$AA@ 320b799c     EntitySystem.obj
 0002:000039b8       __real@45800000            320b79b8     EntitySystem.obj
 0002:000039bc       ??_C@_0CH@PJJNHKM@CEntitySystem?3?3DeleteEntity?5?$CFs?5?$CF@ 320b79bc     EntitySystem.obj
 0002:000039e4       ??_C@_0BM@CFHOLMBF@CEntitySystem?3?3DeleteEntity?$AA@ 320b79e4     EntitySystem.obj
 0002:00003a00       ??_C@_0BC@OBMFOHEL@net_assertlogging?$AA@ 320b7a00     EntitySystem.obj
 0002:00003a14       ??_C@_0DO@KDBEPABM@Trying?5to?5remove?5entity?5with?5mis@ 320b7a14     EntitySystem.obj
 0002:00003a54       ??_C@_0DD@KDPLCGGD@Removing?5entity?5during?5system?5lo@ 320b7a54     EntitySystem.obj
 0002:00003a88       ??_C@_0CH@NMBPOAIG@CEntitySystem?3?3RemoveEntity?5?$CFs?5?$CF@ 320b7a88     EntitySystem.obj
 0002:00003ab0       ??_C@_0BM@MJMGKCJN@CEntitySystem?3?3RemoveEntity?$AA@ 320b7ab0     EntitySystem.obj
 0002:00003acc       ??_C@_0BN@PKPHLOPJ@Entities?3?5Total?$DN?$CFd?5Active?$DN?$CFd?$AA@ 320b7acc     EntitySystem.obj
 0002:00003aec       ??_C@_0L@BJKHNODE@?$CI?$CFd?$CJ?5?3?5?$CFs?5?$AA@ 320b7aec     EntitySystem.obj
 0002:00003af8       ??_C@_0EB@CNIADIAB@Entities?3?5Total?$DN?$CFd?0?5Active?$DN?$CFd?0?5R@ 320b7af8     EntitySystem.obj
 0002:00003b3c       ??_C@_0BJ@OMLGPEPL@?$CFd?5Active?5Entity?5Timers?4?$AA@ 320b7b3c     EntitySystem.obj
 0002:00003b58       ??_C@_0BN@IAOJBAEI@?$CFd?5Visible?5Entities?5Updated?4?$AA@ 320b7b58     EntitySystem.obj
 0002:00003b78       ??_C@_0BF@DOKOCMEI@?$CFd?5Entities?5Updated?4?$AA@ 320b7b78     EntitySystem.obj
 0002:00003b90       __real@41400000            320b7b90     EntitySystem.obj
 0002:00003b94       ??_C@_0DN@JLMGINJO@Entity?3?5?$CFs?5is?5force?5being?5update@ 320b7b94     EntitySystem.obj
 0002:00003bd4       ??_C@_0DO@CKDJKIFG@Entity?3?5?$CFs?5is?5updated?0?5but?5is?5no@ 320b7bd4     EntitySystem.obj
 0002:00003c14       ??_C@_0CA@DBOIMFGE@?$CI?$CFd?$CJ?5?$CF?43f?5ms?5?3?5?$CFs?5?9AI?5?$DN?$CFs?5?$CI?$CFs?$CJ?5?$AA@ 320b7c14     EntitySystem.obj
 0002:00003c38       ??_C@_0ED@FANHINPL@?$CI?$CFd?$CJ?5?$CF?43f?5ms?5?3?5?$CFs?5?$CIwas?5last?5visi@ 320b7c38     EntitySystem.obj
 0002:00003c7c       ??_C@_09JGIHABLK@NOT?5an?5AI?$AA@ 320b7c7c     EntitySystem.obj
 0002:00003c88       __real@428c0000            320b7c88     EntitySystem.obj
 0002:00003c8c       ??_C@_0DI@GJOADFCN@?$DN?$DN?$DN?$DN?$DN?$DN?$DN?$DN?$DN?$DN?$DN?$DN?$DN?$DN?$DN?$DN?$DN?5Entity?5Update?5@ 320b7c8c     EntitySystem.obj
 0002:00003cc8       ??_C@_0EB@FECOKAMP@OnTimer?5Event?5?$CItimerID?$DN?$CFd?0time?$DN?$CF@ 320b7cc8     EntitySystem.obj
 0002:00003d0c       ??_C@_08INHMCBAE@inactive?$AA@ 320b7d0c     EntitySystem.obj
 0002:00003d18       ??_C@_0BM@GOJEGBCI@CEntitySystem?3?3UpdateTimers?$AA@ 320b7d18     EntitySystem.obj
 0002:00003d34       ??_C@_0DI@BCKMAIBA@?$CF5d?3?5Salt?3?$CFd?5?5?$CF?942s?5?5?$CF?914s?5?5pos?3@ 320b7d34     EntitySystem.obj
 0002:00003d6c       ??_C@_0N@BNNINCAF@?$FL$9Hidden$o?$FN?$AA@ 320b7d6c     EntitySystem.obj
 0002:00003d7c       ??_C@_0P@BJFFLHA@?$FL$9Inactive$o?$FN?$AA@ 320b7d7c     EntitySystem.obj
 0002:00003d8c       ??_C@_0N@HJLCDKBK@?$FL$3Active$o?$FN?$AA@ 320b7d8c     EntitySystem.obj
 0002:00003d9c       ??_C@_03LNHFLHIO@$o?$FN?$AA@ 320b7d9c     EntitySystem.obj
 0002:00003da0       ??_C@_03PDHHMLMG@?$FL$9?$AA@ 320b7da0     EntitySystem.obj
 0002:00003da4       ??_C@_06PJIGMIJB@Client?$AA@ 320b7da4     EntitySystem.obj
 0002:00003dac       ??_C@_06LGMEBDBC@Server?$AA@ 320b7dac     EntitySystem.obj
 0002:00003db4       ??_C@_08KAAPDIAN@NoRemove?$AA@ 320b7db4     EntitySystem.obj
 0002:00003dc0       ??_C@_0M@DBPJAGNB@ClientState?$AA@ 320b7dc0     EntitySystem.obj
 0002:00003dcc       ??_C@_07MOJJLFJK@PhysMod?$AA@ 320b7dcc     EntitySystem.obj
 0002:00003dd4       ??_C@_0BE@BEBFLMGE@es_deactivateEntity?$AA@ 320b7dd4     EntitySystem.obj
 0002:00003de8       ??_C@_0BG@GAIHDNEC@Deactivates?5an?5entity?$AA@ 320b7de8     EntitySystem.obj
 0002:00003e00       ??_C@_0BC@PAMFNEGH@es_activateEntity?$AA@ 320b7e00     EntitySystem.obj
 0002:00003e14       ??_C@_0BE@KFGCBIOP@Activates?5an?5entity?$AA@ 320b7e14     EntitySystem.obj
 0002:00003e28       ??_C@_0BA@DPBBKBFB@es_removeEntity?$AA@ 320b7e28     EntitySystem.obj
 0002:00003e38       ??_C@_0BC@CDCKGOPF@Removes?5an?5entity?$AA@ 320b7e38     EntitySystem.obj
 0002:00003e4c       __real@c7c35000            320b7e4c     EntitySystem.obj
 0002:00003e50       ??_7CEntitySystem@@6B@     320b7e50     EntitySystem.obj
 0002:00003f3c       ??_C@_06KBCHOIMA@Entity?$AA@ 320b7f3c     EntitySystem.obj
 0002:00003f44       ??_C@_0DE@PHABGONE@Initializing?5entity?5?8?$CFs?8?5of?5clas@ 320b7f44     EntitySystem.obj
 0002:00003f78       ??_C@_0BJ@JLFLJFED@?5?$CFd?5entities?5?$CI?$CFd?5active?$CJ?$AA@ 320b7f78     EntitySystem.obj
 0002:00003f94       ??_C@_04GCLKCGOG@?5?5?$CFs?$AA@ 320b7f94     EntitySystem.obj
 0002:00003f9c       ??_C@_0CI@IMGKKDNB@Brushes?3?5?$CFd?0?5Entities?3?5?$CFd?$DL?5Mem?3?5@ 320b7f9c     EntitySystem.obj
 0002:00003fc4       __real@43af0000            320b7fc4     EntitySystem.obj
 0002:00003fc8       ??_C@_0DE@CBHAHLLH@Brushes?3?5?$CFd?0?5Decals?3?5?$CFd?0?5Entitie@ 320b7fc8     EntitySystem.obj
 0002:00003ffc       __real@3a800000            320b7ffc     EntitySystem.obj
 0002:00004000       ??_C@_09MOMPMHGD@?5?5?$CFs?5?$CI?$CFs?$CJ?$AA@ 320b8000     EntitySystem.obj
 0002:0000400c       ??_C@_08BEHKFNNO@disabled?$AA@ 320b800c     EntitySystem.obj
 0002:00004018       ??_C@_0BN@BAAGJABG@?$CFs?5?$CIPakInfo?5?9?5?$CF1?41f?5MB?5?9?5?$CFs?$CJ?$AA@ 320b8018     EntitySystem.obj
 0002:00004038       ??_C@_0BB@JNKDNJNI@was?5not?5disabled?$AA@ 320b8038     EntitySystem.obj
 0002:0000404c       ??_C@_0CD@CMFCJPKC@?$CFs?5?$CIPakInfo?3?5?$CF1?41f?5MB?5?1?5?$CF1?41f?5MB@ 320b804c     EntitySystem.obj
 0002:00004070       ??_C@_0L@OABKKMFC@All?5Layers?$AA@ 320b8070     EntitySystem.obj
 0002:0000407c       ??_C@_0BE@PKOOEAFK@Active?5Brush?5Layers?$AA@ 320b807c     EntitySystem.obj
 0002:00004090       ??_C@_0M@KACMPEAN@All?5Layers?3?$AA@ 320b8090     EntitySystem.obj
 0002:0000409c       ??_C@_0BH@OPHGBBCE@?5?5?$CF20s?3?5?$CF1?41f?5MB?5?9?5?$CFs?$CJ?$AA@ 320b809c     EntitySystem.obj
 0002:000040b4       ??_C@_0CG@ILGHLDKG@Layer?5Pak?5Stats?3?5?$CF1?41f?5MB?5?1?5?$CF1?41@ 320b80b4     EntitySystem.obj
 0002:000040dc       __real@35800000            320b80dc     EntitySystem.obj
 0002:000040e0       __real@42280000            320b80e0     EntitySystem.obj
 0002:000040e4       ??_C@_0BB@FKJGLAGO@?$CF?41f?5ms?3?5?$CFs?5?$CI?$CFs?$CJ?$AA@ 320b80e4     EntitySystem.obj
 0002:000040f8       ??_C@_03GCDBBDDL@Off?$AA@  320b80f8     EntitySystem.obj
 0002:000040fc       ??_C@_02IAAGKKDJ@On?$AA@   320b80fc     EntitySystem.obj
 0002:00004100       __real@41a00000            320b8100     EntitySystem.obj
 0002:00004104       __real@41f00000            320b8104     EntitySystem.obj
 0002:00004108       ??_C@_09CPECGIIJ@?$CFu?5?$CI?$CFuKb?$CJ?$AA@ 320b8108     EntitySystem.obj
 0002:00004114       ??_C@_02GMHACPFF@?$CFu?$AA@ 320b8114     EntitySystem.obj
 0002:00004118       ??_C@_07BNNKKIEN@?$CFu?5?1?5?$CFu?$AA@ 320b8118     EntitySystem.obj
 0002:00004120       __real@41d00000            320b8120     EntitySystem.obj
 0002:00004124       __real@44228000            320b8124     EntitySystem.obj
 0002:00004128       ??_C@_0O@JFKPCLGD@?$FLOnly?5Hidden?$FN?$AA@ 320b8128     EntitySystem.obj
 0002:00004138       __real@44098000            320b8138     EntitySystem.obj
 0002:0000413c       ??_C@_0N@JHDJFOHM@Memory?5Usage?$AA@ 320b813c     EntitySystem.obj
 0002:0000414c       __real@43e10000            320b814c     EntitySystem.obj
 0002:00004150       ??_C@_06FHBILLDG@Hidden?$AA@ 320b8150     EntitySystem.obj
 0002:00004158       ??_C@_06MAFFGDO@Active?$AA@ 320b8158     EntitySystem.obj
 0002:00004160       __real@437a0000            320b8160     EntitySystem.obj
 0002:00004164       ??_C@_0BE@OGLLBAFH@Total?5?1?5Pool?5Counts?$AA@ 320b8164     EntitySystem.obj
 0002:00004178       __real@41300000            320b8178     EntitySystem.obj
 0002:0000417c       ??_C@_01LBDDMOBJ@?$FN?$AA@ 320b817c     EntitySystem.obj
 0002:00004180       ??_C@_02GBLMOEJC@?5?$FL?$AA@ 320b8180     EntitySystem.obj
 0002:00004184       ??_C@_0N@CHJPIFDC@Entity?5Class?$AA@ 320b8184     EntitySystem.obj
 0002:00004194       ??_C@_0CO@GJDEHLOC@SetTimer?5?$CItimerID?$DN?$CFd?0time?$DN?$CFdms?$CJ?5@ 320b8194     EntitySystem.obj
 0002:000041c4       ??_C@_09IIHJADCI@startTime?$AA@ 320b81c4     EntitySystem.obj
 0002:000041d0       ??_C@_07GDDJAGCK@timerID?$AA@ 320b81d0     EntitySystem.obj
 0002:000041d8       ??_C@_09KIALCCEB@eventTime?$AA@ 320b81d8     EntitySystem.obj
 0002:000041e4       ??_C@_08MIEKCMO@entityID?$AA@ 320b81e4     EntitySystem.obj
 0002:000041f0       ??_C@_05NHFJDMOA@Timer?$AA@ 320b81f0     EntitySystem.obj
 0002:000041f8       ??_C@_0L@HOPENLNO@timerCount?$AA@ 320b81f8     EntitySystem.obj
 0002:00004204       ??_C@_0L@IKHCCDCO@PauseStart?$AA@ 320b8204     EntitySystem.obj
 0002:00004210       ??_C@_06IFNLNCGM@Paused?$AA@ 320b8210     EntitySystem.obj
 0002:00004218       ??_C@_06KEMPJBHB@Timers?$AA@ 320b8218     EntitySystem.obj
 0002:00004220       ??_C@_0BG@PPKDJELM@CEntitySystem?3?3Update?$AA@ 320b8220     EntitySystem.obj
 0002:00004238       ??_C@_0CP@FDCKFCMC@EntityId?5?$CI0x?$CFX?$CJ?5added?5to?5not?5see@ 320b8238     EntityTimeoutList.obj
 0002:00004268       ??_C@_0EP@IFICNHPK@CEntityTimeoutList?3?3ResetTimeout@ 320b8268     EntityTimeoutList.obj
 0002:000042b8       ??_C@_0HD@KMHNLOON@CEntityTimeoutList?3?3CEntityTimeo@ 320b82b8     EntityTimeoutList.obj
 0002:00004338       ??_C@_0BD@OFOGHKHB@OnPreparedFromPool?$AA@ 320b8338     EntityScript.obj
 0002:0000434c       ??_C@_0L@NGMJLKPO@OnUnHidden?$AA@ 320b834c     EntityScript.obj
 0002:00004358       ??_C@_08OIDHAOLJ@OnHidden?$AA@ 320b8358     EntityScript.obj
 0002:00004364       ??_C@_0M@PNNKPOOD@OnStartGame?$AA@ 320b8364     EntityScript.obj
 0002:00004370       ??_C@_0N@OIOJMLAK@OnStartLevel?$AA@ 320b8370     EntityScript.obj
 0002:00004380       ??_C@_0O@JGODGMFJ@OnLevelLoaded?$AA@ 320b8380     EntityScript.obj
 0002:00004390       ??_C@_0M@CNCPFKAF@OnSoundDone?$AA@ 320b8390     EntityScript.obj
 0002:0000439c       ??_C@_0P@DPJOLHKI@OnPhysicsBreak?$AA@ 320b839c     EntityScript.obj
 0002:000043ac       ??_C@_0BB@NPFFOJDA@OnAnimationEvent?$AA@ 320b83ac     EntityScript.obj
 0002:000043c0       ??_C@_0P@IBOIKOBF@OnEndAnimation?$AA@ 320b83c0     EntityScript.obj
 0002:000043d0       ??_C@_0BB@HMOCOEML@OnStartAnimation?$AA@ 320b83d0     EntityScript.obj
 0002:000043e4       ??_C@_0M@JGCIHLKM@OnCollision?$AA@ 320b83e4     EntityScript.obj
 0002:000043f0       ??_C@_06GJPOLLJG@OnMove?$AA@ 320b83f0     EntityScript.obj
 0002:000043f8       ??_C@_0N@GKOLIBMI@OnUnBindThis?$AA@ 320b83f8     EntityScript.obj
 0002:00004408       ??_C@_08LJGKMGBN@OnUnBind?$AA@ 320b8408     EntityScript.obj
 0002:00004414       ??_C@_0L@BJNPBBGB@OnBindThis?$AA@ 320b8414     EntityScript.obj
 0002:00004420       ??_C@_06MFOLLABC@OnBind?$AA@ 320b8420     EntityScript.obj
 0002:00004428       ??_C@_0BK@CINIENFK@OnLocalClientMoveNearArea?$AA@ 320b8428     EntityScript.obj
 0002:00004444       ??_C@_0BN@KANGLHGF@OnLocalClientProceedFadeArea?$AA@ 320b8444     EntityScript.obj
 0002:00004464       ??_C@_0BL@NEHJAHPH@OnLocalClientLeaveNearArea?$AA@ 320b8464     EntityScript.obj
 0002:00004480       ??_C@_0BL@PLDLOFKD@OnLocalClientEnterNearArea?$AA@ 320b8480     EntityScript.obj
 0002:0000449c       ??_C@_0BH@LAGGNCGL@OnLocalClientLeaveArea?$AA@ 320b849c     EntityScript.obj
 0002:000044b4       ??_C@_0BH@LCJIOMED@OnLocalClientEnterArea?$AA@ 320b84b4     EntityScript.obj
 0002:000044cc       ??_C@_0P@DAIBMGL@OnMoveNearArea?$AA@ 320b84cc     EntityScript.obj
 0002:000044dc       ??_C@_0BC@KAAMIGCI@OnProceedFadeArea?$AA@ 320b84dc     EntityScript.obj
 0002:000044f0       ??_C@_0BA@IFIMNHJM@OnLeaveNearArea?$AA@ 320b84f0     EntityScript.obj
 0002:00004500       ??_C@_0BA@KKMODFMI@OnEnterNearArea?$AA@ 320b8500     EntityScript.obj
 0002:00004510       ??_C@_0M@LJCBOPE@OnLeaveArea?$AA@ 320b8510     EntityScript.obj
 0002:0000451c       ??_C@_0M@JGMCANM@OnEnterArea?$AA@ 320b851c     EntityScript.obj
 0002:00004528       ??_C@_08BJHKHJEG@OnDamage?$AA@ 320b8528     EntityScript.obj
 0002:00004534       ??_C@_07JNAMBEDG@OnEvent?$AA@ 320b8534     EntityScript.obj
 0002:0000453c       ??_C@_07CIINKFND@OnTimer?$AA@ 320b853c     EntityScript.obj
 0002:00004544       ??_C@_08DCJEAFK@OnUpdate?$AA@ 320b8544     EntityScript.obj
 0002:00004550       ??_C@_0L@HONLPIJA@OnEndState?$AA@ 320b8550     EntityScript.obj
 0002:0000455c       ??_C@_0N@HAHALOPE@OnBeginState?$AA@ 320b855c     EntityScript.obj
 0002:0000456c       ??_7IEntityScript@@6B@     320b856c     EntityScript.obj
 0002:00004578       ??_C@_0BL@JECODOOM@CEntityScript?3?3Call_OnInit?$AA@ 320b8578     EntityScript.obj
 0002:00004594       ??_7CEntityScript@@6B@     320b8594     EntityScript.obj
 0002:000045a8       ??_C@_06OKBMNGLE@States?$AA@ 320b85a8     EntityScript.obj
 0002:000045b0       ??_C@_0L@BMCCMADP@OnShutDown?$AA@ 320b85b0     EntityScript.obj
 0002:000045bc       ??_C@_06GAGBLNGO@OnInit?$AA@ 320b85bc     EntityScript.obj
 0002:000045c4       ??_C@_09GOJICBBC@OnDestroy?$AA@ 320b85c4     EntityScript.obj
 0002:000045d0       ??_C@_07OLHLPFGD@OnSpawn?$AA@ 320b85d0     EntityScript.obj
 0002:000045d8       ??_C@_06GOJKNBFM@entity?$AA@ 320b85d8     EntityScript.obj
 0002:000045e0       ??_C@_04PNENAKPF@vec3?$AA@ 320b85e0     EntityScript.obj
 0002:000045e8       ??_C@_06ENCLGNJJ@Event_?$AA@ 320b85e8     EntityScript.obj
 0002:000045f0       ??_C@_07LGFKBKFE@Outputs?$AA@ 320b85f0     EntityScript.obj
 0002:000045f8       ??_C@_06HDCHCENJ@Inputs?$AA@ 320b85f8     EntityScript.obj
 0002:00004600       ??_C@_0L@FCJIIJAL@FlowEvents?$AA@ 320b8600     EntityScript.obj
 0002:0000460c       ??_C@_07NNLICMOF@OnReset?$AA@ 320b860c     EntityScript.obj
 0002:00004614       ??_C@_0P@BABMPPMC@Entity?5Scripts?$AA@ 320b8614     EntityScript.obj
 0002:00004638       ??_7CScriptableBase@@6B@   320b8638     ScriptBind_Entity.obj
 0002:00004648       ??_7CLightAttachment@@6B@  320b8648     ScriptBind_Entity.obj
 0002:00004688       __real@40c90fdb            320b8688     ScriptBind_Entity.obj
 0002:0000468c       __real@3de147ae            320b868c     ScriptBind_Entity.obj
 0002:00004690       __real@40c00000            320b8690     ScriptBind_Entity.obj
 0002:00004694       __real@c0000000            320b8694     ScriptBind_Entity.obj
 0002:00004698       ??_7CSKELAttachment@@6B@   320b8698     ScriptBind_Entity.obj
 0002:000046d8       __real@51ba43b7            320b86d8     ScriptBind_Entity.obj
 0002:000046dc       __real@3c8efa35            320b86dc     ScriptBind_Entity.obj
 0002:000046e0       __real@358637bd            320b86e0     ScriptBind_Entity.obj
 0002:000046e4       ??_C@_09BIFFMKFL@EGeomType?$AA@ 320b86e4     ScriptBind_Entity.obj
 0002:000046f0       ??_C@_0O@GCNGPJPL@GeomType_None?$AA@ 320b86f0     ScriptBind_Entity.obj
 0002:00004700       ??_C@_0BF@FNHMLHJF@GeomType_BoundingBox?$AA@ 320b8700     ScriptBind_Entity.obj
 0002:00004718       ??_C@_0BB@EGBHBLBF@GeomType_Physics?$AA@ 320b8718     ScriptBind_Entity.obj
 0002:0000472c       ??_C@_0BA@NJGFLABO@GeomType_Render?$AA@ 320b872c     ScriptBind_Entity.obj
 0002:0000473c       ??_C@_09LMFKFIJM@EGeomForm?$AA@ 320b873c     ScriptBind_Entity.obj
 0002:00004748       ??_C@_0BC@EDPJPAAC@GeomForm_Vertices?$AA@ 320b8748     ScriptBind_Entity.obj
 0002:0000475c       ??_C@_0P@GPDJOGJG@GeomForm_Edges?$AA@ 320b875c     ScriptBind_Entity.obj
 0002:0000476c       ??_C@_0BB@KJLPDGEJ@GeomForm_Surface?$AA@ 320b876c     ScriptBind_Entity.obj
 0002:00004780       ??_C@_0BA@MAJAOBB@GeomForm_Volume?$AA@ 320b8780     ScriptBind_Entity.obj
 0002:00004790       ??_C@_0CG@LAFILCND@?$FL?$CFs?$FN?5?$CFd?5arguments?5passed?0?51?5expe@ 320b8790     ScriptBind_Entity.obj
 0002:000047b8       ??_C@_0BM@OEPNNAB@CScriptBind_Entity?3?3SetName?$AA@ 320b87b8     ScriptBind_Entity.obj
 0002:000047d4       ??_C@_0CG@CLPNPOLM@?$FL?$CFs?$FN?5?$CFd?5arguments?5passed?0?50?5expe@ 320b87d4     ScriptBind_Entity.obj
 0002:000047fc       ??_C@_0BO@IDANECFF@CScriptBind_Entity?3?3GetAIName?$AA@ 320b87fc     ScriptBind_Entity.obj
 0002:0000481c       ??_C@_0BM@PGLOOCNA@CScriptBind_Entity?3?3GetName?$AA@ 320b881c     ScriptBind_Entity.obj
 0002:00004838       ??_C@_0BN@PNFDAIAK@CScriptBind_Entity?3?3GetRawId?$AA@ 320b8838     ScriptBind_Entity.obj
 0002:00004858       ??_C@_0CB@GGJJPFEC@CScriptBind_Entity?3?3GetArchetype@ 320b8858     ScriptBind_Entity.obj
 0002:0000487c       ??_C@_03JAHONMHP@cpf?$AA@  320b887c     ScriptBind_Entity.obj
 0002:00004880       ??_C@_03MGFGPPEN@cga?$AA@  320b8880     ScriptBind_Entity.obj
 0002:00004884       ??_C@_03ILFBNHND@cdf?$AA@  320b8884     ScriptBind_Entity.obj
 0002:00004888       ??_C@_03KMOFPJOC@chr?$AA@  320b8888     ScriptBind_Entity.obj
 0002:00004890       ??_C@_0EB@IPMEPECP@LUA?5is?5Unable?5to?5Precache?5Effect@ 320b8890     ScriptBind_Entity.obj
 0002:000048d8       ??_7CCGFAttachment@@6B@    320b88d8     ScriptBind_Entity.obj
 0002:00004918       ??_C@_0DM@JIKAELJO@FATAL?5ERROR?3?5CScriptBind_Entity?3@ 320b8918     ScriptBind_Entity.obj
 0002:00004954       ??_C@_0BP@IPEDBMEK@CScriptBind_Entity?3?3NetPresent?$AA@ 320b8954     ScriptBind_Entity.obj
 0002:00004974       ??_C@_0CH@BMFFAJGD@CScriptBind_Entity?3?3SetStateClie@ 320b8974     ScriptBind_Entity.obj
 0002:000049a0       ??_C@_0EC@NGDANNOE@CScriptBind_Entity?3?3StartAnimati@ 320b89a0     ScriptBind_Entity.obj
 0002:000049e4       ??_C@_04HIBGFPH@NULL?$AA@  320b89e4     ScriptBind_Entity.obj
 0002:000049f0       ??_C@_0EP@DMMMGALB@CScriptBind_Entity?3?3StartAnimati@ 320b89f0     ScriptBind_Entity.obj
 0002:00004a40       __real@3e19999a            320b8a40     ScriptBind_Entity.obj
 0002:00004a44       ??_C@_0CJ@ICNPKDA@CScriptBind_Entity?3?3SetRegisterI@ 320b8a44     ScriptBind_Entity.obj
 0002:00004a70       __real@42b40000            320b8a70     ScriptBind_Entity.obj
 0002:00004a74       __real@42340000            320b8a74     ScriptBind_Entity.obj
 0002:00004a78       ??_C@_0DG@NDOEHGGA@CancelSubpipe?3?5wrong?5parameter?5t@ 320b8a78     ScriptBind_Entity.obj
 0002:00004ab0       ??_C@_0CJ@HPHNMKAA@CancelSubpipe?3?5only?51?5parameter?5@ 320b8ab0     ScriptBind_Entity.obj
 0002:00004adc       ??_C@_0CC@PDPFPCCF@IsUsingPipe?3?5wrong?5parameter?5typ@ 320b8adc     ScriptBind_Entity.obj
 0002:00004b00       ??_C@_0CA@OAHPLNNB@IsUsingPipe?3?5too?5few?5parameters?$AA@ 320b8b00     ScriptBind_Entity.obj
 0002:00004b20       ??_C@_0CE@MGFJBHEO@CScriptBind_Entity?3?3GetCurAnimat@ 320b8b20     ScriptBind_Entity.obj
 0002:00004b44       ??_C@_0CJ@PCLDGAKG@CScriptBind_Entity?3?3GetBoneNameF@ 320b8b44     ScriptBind_Entity.obj
 0002:00004b70       ??_C@_0EG@MDCLELII@CScriptBind_Entity?3?3GetAnimation@ 320b8b70     ScriptBind_Entity.obj
 0002:00004bb8       ??_C@_0CA@CDBONEIJ@CScriptBind_Entity?3?3SetMaterial?$AA@ 320b8bb8     ScriptBind_Entity.obj
 0002:00004bd8       ??_C@_0DA@JPJKJAFC@Material?5not?5found?5?8?$CFs?8?5in?5?$CFs?3Re@ 320b8bd8     ScriptBind_Entity.obj
 0002:00004c08       ??_C@_0EM@IEAGGPOD@Material?5Parameter?3?5?$CFs?5is?5not?5va@ 320b8c08     ScriptBind_Entity.obj
 0002:00004c54       ??_C@_0BN@KAMIEFAN@CScriptBind_Entity?3?3GetSpeed?$AA@ 320b8c54     ScriptBind_Entity.obj
 0002:00004c74       ??_C@_0BM@LLDOKDKN@CScriptBind_Entity?3?3GetMass?$AA@ 320b8c74     ScriptBind_Entity.obj
 0002:00004c90       ??_C@_0CF@EBHFMMO@CScriptBind_Entity?3?3SetViewDistR@ 320b8c90     ScriptBind_Entity.obj
 0002:00004cb8       ??_C@_0CA@PPEDBJEI@CScriptBind_Entity?3?3SetLodRatio?$AA@ 320b8cb8     ScriptBind_Entity.obj
 0002:00004cd8       ??_C@_0BJ@GLAHBFDP@CScriptBind_Entity?3?3Hide?$AA@ 320b8cd8     ScriptBind_Entity.obj
 0002:00004cf4       ??_C@_0CJ@CDKKPICC@CScriptBind_Entity?3?3NoExplosionC@ 320b8cf4     ScriptBind_Entity.obj
 0002:00004d20       ??_C@_07GFBFDLBM@gravity?$AA@ 320b8d20     ScriptBind_Entity.obj
 0002:00004d28       __real@c11cf5c3            320b8d28     ScriptBind_Entity.obj
 0002:00004d30       __real@3f50624dd2f1a9fc    320b8d30     ScriptBind_Entity.obj
 0002:00004d38       __real@bf50624dd2f1a9fc    320b8d38     ScriptBind_Entity.obj
 0002:00004d40       __real@3f1a36e2eb1c432d    320b8d40     ScriptBind_Entity.obj
 0002:00004d48       ??_C@_0CL@EHKJFCAF@Entity?5?$CFs?0?5slot?5?$CFd?5is?5not?5partic@ 320b8d48     ScriptBind_Entity.obj
 0002:00004d74       __real@bf000000            320b8d74     ScriptBind_Entity.obj
 0002:00004d78       ??_7CCustomInfo@?$TFixed@E$00$0PP@@@6B@ 320b8d78     ScriptBind_Entity.obj
 0002:00004dac       ??_C@_08KJMHCJDL@TFixed?$DM?$DO?$AA@ 320b8dac     ScriptBind_Entity.obj
 0002:00004db8       ??_C@_01GLPGHMHM@z?$AA@    320b8db8     ScriptBind_Entity.obj
 0002:00004dbc       ??_C@_01EANLCPLP@y?$AA@    320b8dbc     ScriptBind_Entity.obj
 0002:00004dc0       ??_C@_01FJMABOPO@x?$AA@    320b8dc0     ScriptBind_Entity.obj
 0002:00004dc4       ??_C@_0BF@DCNHDLIJ@Character?5Attachment?$AA@ 320b8dc4     ScriptBind_Entity.obj
 0002:00004de0       ??_7CEffectAttachment@@6B@ 320b8de0     ScriptBind_Entity.obj
 0002:00004e20       __real@bdcccccd            320b8e20     ScriptBind_Entity.obj
 0002:00004e24       ??_C@_0DN@KCKLCOBD@ERROR?3?5CScriptObjectWeapon?3?3GetB@ 320b8e24     ScriptBind_Entity.obj
 0002:00004e68       ??_C@_0EO@IHFILMCK@LoadParticleEffect?5?$CIfrom?5lua?$CJ?4?5e@ 320b8e68     ScriptBind_Entity.obj
 0002:00004eb8       ??_C@_06CBHGEMFM@?$DMNULL?$DO?$AA@ 320b8eb8     ScriptBind_Entity.obj
 0002:00004ec0       ??_C@_06OPINLJAN@bPrime?$AA@ 320b8ec0     ScriptBind_Entity.obj
 0002:00004ec8       ??_C@_0N@IEMAGKCC@esAttachForm?$AA@ 320b8ec8     ScriptBind_Entity.obj
 0002:00004ed8       ??_C@_0N@CAMPPIOF@esAttachType?$AA@ 320b8ed8     ScriptBind_Entity.obj
 0002:00004ee8       ??_C@_0N@KIHNDJIO@bEnableSound?$AA@ 320b8ee8     ScriptBind_Entity.obj
 0002:00004ef8       ??_C@_0O@BJHPCLJD@bCountPerUnit?$AA@ 320b8ef8     ScriptBind_Entity.obj
 0002:00004f08       ??_C@_0L@BCBJOECP@CountScale?$AA@ 320b8f08     ScriptBind_Entity.obj
 0002:00004f14       ??_C@_0L@PMDODIGI@SpeedScale?$AA@ 320b8f14     ScriptBind_Entity.obj
 0002:00004f20       ??_C@_05MAGIBEFI@Scale?$AA@ 320b8f20     ScriptBind_Entity.obj
 0002:00004f28       ??_C@_08CHNCHBNG@Strength?$AA@ 320b8f28     ScriptBind_Entity.obj
 0002:00004f34       ??_C@_0M@FBBAHGNK@PulsePeriod?$AA@ 320b8f34     ScriptBind_Entity.obj
 0002:00004f40       ??_C@_0GD@LHLOJOJL@Ignoring?5obsolete?5SpawnPeriod?$DN?$CFg@ 320b8f40     ScriptBind_Entity.obj
 0002:00004fa4       ??_C@_0M@KCKBMOIC@SpawnPeriod?$AA@ 320b8fa4     ScriptBind_Entity.obj
 0002:00004fb0       ??_C@_0BA@PMEHHPAI@detach_distance?$AA@ 320b8fb0     ScriptBind_Entity.obj
 0002:00004fc0       ??_C@_09DEHKFMCJ@threshold?$AA@ 320b8fc0     ScriptBind_Entity.obj
 0002:00004fcc       ??_C@_06NHCMNMEH@origin?$AA@ 320b8fcc     ScriptBind_Entity.obj
 0002:00004fd4       ??_C@_0M@JPLLDLN@plane_index?$AA@ 320b8fd4     ScriptBind_Entity.obj
 0002:00004fe0       ??_C@_0N@POJIAJEP@crack_weaken?$AA@ 320b8fe0     ScriptBind_Entity.obj
 0002:00004ff0       ??_C@_0BB@LOLNBMEM@max_twist_torque?$AA@ 320b8ff0     ScriptBind_Entity.obj
 0002:00005004       ??_C@_0BA@DPGLNBMG@max_shift_force?$AA@ 320b9004     ScriptBind_Entity.obj
 0002:00005014       ??_C@_0P@IOMLIAAE@max_push_force?$AA@ 320b9014     ScriptBind_Entity.obj
 0002:00005024       ??_C@_0BI@DCBJLCKM@max_simultaneous_cracks?$AA@ 320b9024     ScriptBind_Entity.obj
 0002:0000503c       ??_C@_07FEJKIDLJ@cyl_pos?$AA@ 320b903c     ScriptBind_Entity.obj
 0002:00005044       ??_C@_0L@LOGHODCF@cyl_height?$AA@ 320b9044     ScriptBind_Entity.obj
 0002:00005050       ??_C@_05DPIGJLFE@cyl_r?$AA@ 320b9050     ScriptBind_Entity.obj
 0002:00005058       ??_C@_0L@PKHBJPDN@eye_height?$AA@ 320b9058     ScriptBind_Entity.obj
 0002:00005064       ??_C@_0N@DHJCEHBJ@pivot_height?$AA@ 320b9064     ScriptBind_Entity.obj
 0002:00005074       ??_C@_0P@DCHOCNHI@max_vel_ground?$AA@ 320b9074     ScriptBind_Entity.obj
 0002:00005084       ??_C@_09NFIEOJGK@is_active?$AA@ 320b9084     ScriptBind_Entity.obj
 0002:00005090       ??_C@_09MBBAKDHD@bSwimming?$AA@ 320b9090     ScriptBind_Entity.obj
 0002:0000509c       ??_C@_0O@FCKBPALA@k_air_control?$AA@ 320b909c     ScriptBind_Entity.obj
 0002:000050ac       ??_C@_09IICCNKEF@k_inertia?$AA@ 320b90ac     ScriptBind_Entity.obj
 0002:000050b8       ??_C@_04PLMLMMEO@full?$AA@ 320b90b8     ScriptBind_Entity.obj
 0002:000050c0       ??_C@_0M@DAOCHMIM@no_rotation?$AA@ 320b90c0     ScriptBind_Entity.obj
 0002:000050cc       ??_C@_05MAIECAHP@plane?$AA@ 320b90cc     ScriptBind_Entity.obj
 0002:000050d4       ??_C@_04HJPCFDOP@line?$AA@ 320b90d4     ScriptBind_Entity.obj
 0002:000050dc       ??_C@_0BA@HDKPGPBM@max_bend_torque?$AA@ 320b90dc     ScriptBind_Entity.obj
 0002:000050ec       ??_C@_0P@HJPIADFO@max_pull_force?$AA@ 320b90ec     ScriptBind_Entity.obj
 0002:000050fc       ??_C@_05LGMNIHAM@yzmax?$AA@ 320b90fc     ScriptBind_Entity.obj
 0002:00005104       ??_C@_05KEEGGDGD@yzmin?$AA@ 320b9104     ScriptBind_Entity.obj
 0002:0000510c       ??_C@_04JHMANONL@xmax?$AA@ 320b910c     ScriptBind_Entity.obj
 0002:00005114       ??_C@_04IFELDKLE@xmin?$AA@ 320b9114     ScriptBind_Entity.obj
 0002:0000511c       ??_C@_0N@OFMDNCKE@ignore_buddy?$AA@ 320b911c     ScriptBind_Entity.obj
 0002:0000512c       ??_C@_0N@CILEGOMK@frame1_inner?$AA@ 320b912c     ScriptBind_Entity.obj
 0002:0000513c       ??_C@_06CJEAIKMO@frame1?$AA@ 320b913c     ScriptBind_Entity.obj
 0002:00005144       ??_C@_0N@OEBOGOFE@frame0_inner?$AA@ 320b9144     ScriptBind_Entity.obj
 0002:00005154       ??_C@_06DAFLLLIP@frame0?$AA@ 320b9154     ScriptBind_Entity.obj
 0002:0000515c       ??_C@_05JHLBIJAO@pivot?$AA@ 320b915c     ScriptBind_Entity.obj
 0002:00005164       ??_C@_0P@DANEDEOO@phys_entity_id?$AA@ 320b9164     ScriptBind_Entity.obj
 0002:00005174       ??_C@_0P@GMGOOFK@stiffness_tang?$AA@ 320b9174     ScriptBind_Entity.obj
 0002:00005184       ??_C@_0P@CDJKKENE@stiffness_norm?$AA@ 320b9184     ScriptBind_Entity.obj
 0002:00005194       ??_C@_0L@FDLNIEGL@mass_decay?$AA@ 320b9194     ScriptBind_Entity.obj
 0002:000051a0       ??_C@_0P@MDAMHDNK@collision_mask?$AA@ 320b91a0     ScriptBind_Entity.obj
 0002:000051b0       ??_C@_0BG@GEMPNBBA@max_collision_impulse?$AA@ 320b91b0     ScriptBind_Entity.obj
 0002:000051c8       ??_C@_0BI@DNLIDDDK@collision_impulse_scale?$AA@ 320b91c8     ScriptBind_Entity.obj
 0002:000051e0       ??_C@_0BA@ONIEOAFB@explosion_scale?$AA@ 320b91e0     ScriptBind_Entity.obj
 0002:000051f0       ??_C@_0O@CILFFAGJ@impulse_scale?$AA@ 320b91f0     ScriptBind_Entity.obj
 0002:00005200       ??_C@_08FJNPIHOL@accuracy?$AA@ 320b9200     ScriptBind_Entity.obj
 0002:0000520c       ??_C@_09KFGKBHHC@max_iters?$AA@ 320b920c     ScriptBind_Entity.obj
 0002:00005218       ??_C@_0O@DFOJLNIP@damping_ratio?$AA@ 320b9218     ScriptBind_Entity.obj
 0002:00005228       ??_C@_08HCMBNGKH@hardness?$AA@ 320b9228     ScriptBind_Entity.obj
 0002:00005234       ??_C@_0O@FALOKCLA@max_safe_step?$AA@ 320b9234     ScriptBind_Entity.obj
 0002:00005244       ??_C@_09GLPKLBIH@thickness?$AA@ 320b9244     ScriptBind_Entity.obj
 0002:00005250       ??_C@_0L@KBOEHCAC@bShootable?$AA@ 320b9250     ScriptBind_Entity.obj
 0002:0000525c       ??_C@_09GOAMIHLB@shootable?$AA@ 320b925c     ScriptBind_Entity.obj
 0002:00005268       ??_C@_0BL@LILLOEMB@bCheckAttachmentCollisions?$AA@ 320b9268     ScriptBind_Entity.obj
 0002:00005284       ??_C@_0BI@LNJJAKOB@bCheckTerrainCollisions?$AA@ 320b9284     ScriptBind_Entity.obj
 0002:0000529c       ??_C@_0BB@IJLODCEN@bCheckCollisions?$AA@ 320b929c     ScriptBind_Entity.obj
 0002:000052b0       ??_C@_07DDHNKDGP@timeout?$AA@ 320b92b0     ScriptBind_Entity.obj
 0002:000052b8       ??_C@_04DKHFBEKB@end1?$AA@ 320b92b8     ScriptBind_Entity.obj
 0002:000052c0       ??_C@_0BB@BJNLFGAA@entity_part_id_1?$AA@ 320b92c0     ScriptBind_Entity.obj
 0002:000052d4       ??_C@_0O@CFJICDBH@entity_name_1?$AA@ 320b92d4     ScriptBind_Entity.obj
 0002:000052e4       ??_C@_0BB@CNLFMCID@entity_phys_id_1?$AA@ 320b92e4     ScriptBind_Entity.obj
 0002:000052f8       ??_C@_04BBFIEHGC@end2?$AA@ 320b92f8     ScriptBind_Entity.obj
 0002:00005300       ??_C@_0BB@DCPGAFMD@entity_part_id_2?$AA@ 320b9300     ScriptBind_Entity.obj
 0002:00005314       ??_C@_0O@OLFHANE@entity_name_2?$AA@ 320b9314     ScriptBind_Entity.obj
 0002:00005324       ??_C@_0BB@GJIJBEA@entity_phys_id_2?$AA@ 320b9324     ScriptBind_Entity.obj
 0002:00005338       ??_C@_03JBJLGPFL@end?$AA@  320b9338     ScriptBind_Entity.obj
 0002:0000533c       ??_C@_0P@CGPJOBCK@entity_part_id?$AA@ 320b933c     ScriptBind_Entity.obj
 0002:0000534c       ??_C@_07DONMPJIA@?$CDworld?$CD?$AA@ 320b934c     ScriptBind_Entity.obj
 0002:00005354       ??_C@_0M@GIDEKDMA@entity_name?$AA@ 320b9354     ScriptBind_Entity.obj
 0002:00005360       ??_C@_0P@GLIGIICK@entity_phys_id?$AA@ 320b9360     ScriptBind_Entity.obj
 0002:00005370       ??_C@_04HHNJMEDN@wind?$AA@ 320b9370     ScriptBind_Entity.obj
 0002:00005378       ??_C@_0N@KDMMBMGM@unproj_limit?$AA@ 320b9378     ScriptBind_Entity.obj
 0002:00005388       ??_C@_09DJHBENNM@pose_type?$AA@ 320b9388     ScriptBind_Entity.obj
 0002:00005394       ??_C@_0N@PHFPPFHJ@pose_damping?$AA@ 320b9394     ScriptBind_Entity.obj
 0002:000053a4       ??_C@_0P@JJLBIPLA@pose_stiffness?$AA@ 320b93a4     ScriptBind_Entity.obj
 0002:000053b4       ??_C@_0L@DIEHIELD@num_subvtx?$AA@ 320b93b4     ScriptBind_Entity.obj
 0002:000053c0       ??_C@_08IFFONDCK@num_segs?$AA@ 320b93c0     ScriptBind_Entity.obj
 0002:000053cc       ??_C@_09IPLOBAIC@max_force?$AA@ 320b93cc     ScriptBind_Entity.obj
 0002:000053d8       ??_C@_0M@MGCJACPI@sensor_size?$AA@ 320b93d8     ScriptBind_Entity.obj
 0002:000053e4       ??_C@_0P@JCKMMPHJ@air_resistance?$AA@ 320b93e4     ScriptBind_Entity.obj
 0002:000053f4       ??_C@_0O@KHLFHJNO@wind_variance?$AA@ 320b93f4     ScriptBind_Entity.obj
 0002:00005404       ??_C@_0O@PBHAKGNG@friction_pull?$AA@ 320b9404     ScriptBind_Entity.obj
 0002:00005414       ??_C@_08LKDNMFOC@friction?$AA@ 320b9414     ScriptBind_Entity.obj
 0002:00005420       ??_C@_09KEINEMDH@coll_dist?$AA@ 320b9420     ScriptBind_Entity.obj
 0002:0000542c       ??_C@_06IJDLPEM@length?$AA@ 320b942c     ScriptBind_Entity.obj
 0002:00005434       ??_C@_08PJLDMOKI@kdashpot?$AA@ 320b9434     ScriptBind_Entity.obj
 0002:00005440       ??_C@_07KEKOBKBG@dashpot?$AA@ 320b9440     ScriptBind_Entity.obj
 0002:00005448       ??_C@_09CNHECHOC@stiffness?$AA@ 320b9448     ScriptBind_Entity.obj
 0002:00005454       ??_C@_03LJAEFNNE@max?$AA@  320b9454     ScriptBind_Entity.obj
 0002:00005458       ??_C@_03KLIPLJLL@min?$AA@  320b9458     ScriptBind_Entity.obj
 0002:0000545c       ??_C@_09FGJHPIID@bone_name?$AA@ 320b945c     ScriptBind_Entity.obj
 0002:00005468       ??_C@_0P@FFAGOAOI@lying_sim_type?$AA@ 320b9468     ScriptBind_Entity.obj
 0002:00005478       ??_C@_08FONLGGHN@sim_type?$AA@ 320b9478     ScriptBind_Entity.obj
 0002:00005484       ??_C@_0BB@IMIAMBLF@check_collisions?$AA@ 320b9484     ScriptBind_Entity.obj
 0002:00005498       ??_C@_0M@DDKDFCNA@is_grounded?$AA@ 320b9498     ScriptBind_Entity.obj
 0002:000054a4       ??_C@_0BC@IMLFLJDH@lying_sleep_speed?$AA@ 320b94a4     ScriptBind_Entity.obj
 0002:000054b8       ??_C@_0O@IGIHCCMB@lying_damping?$AA@ 320b94b8     ScriptBind_Entity.obj
 0002:000054c8       ??_C@_0P@PIFPDMBP@lying_gravityx?$AA@ 320b94c8     ScriptBind_Entity.obj
 0002:000054d8       ??_C@_0P@OBEEANFO@lying_gravityy?$AA@ 320b94d8     ScriptBind_Entity.obj
 0002:000054e8       ??_C@_0P@MKGJFOJN@lying_gravityz?$AA@ 320b94e8     ScriptBind_Entity.obj
 0002:000054f8       ??_C@_0O@GDEMIPND@lying_gravity?$AA@ 320b94f8     ScriptBind_Entity.obj
 0002:00005508       ??_C@_0BC@KHMCKGKN@lying_mode_ncolls?$AA@ 320b9508     ScriptBind_Entity.obj
 0002:0000551c       ??_C@_0N@BKCCPLHM@water_origin?$AA@ 320b951c     ScriptBind_Entity.obj
 0002:0000552c       ??_C@_0N@EHLFJEEA@water_normal?$AA@ 320b952c     ScriptBind_Entity.obj
 0002:0000553c       ??_C@_0BC@HNAIMIJK@water_sleep_speed?$AA@ 320b953c     ScriptBind_Entity.obj
 0002:00005550       ??_C@_0BB@CIPCDOE@water_resistance?$AA@ 320b9550     ScriptBind_Entity.obj
 0002:00005564       ??_C@_0O@DBBIHBAN@water_damping?$AA@ 320b9564     ScriptBind_Entity.obj
 0002:00005574       ??_C@_0O@MBJDEEBJ@water_density?$AA@ 320b9574     ScriptBind_Entity.obj
 0002:00005584       ??_C@_01MHEDDDHA@v?$AA@    320b9584     ScriptBind_Entity.obj
 0002:00005588       ??_C@_0BB@NIGEDLJA@bUseSimpleSolver?$AA@ 320b9588     ScriptBind_Entity.obj
 0002:0000559c       ??_C@_0O@HKLBKNLH@bFixedDamping?$AA@ 320b959c     ScriptBind_Entity.obj
 0002:000055ac       ??_C@_0BG@HJJGFHNO@max_logged_collisions?$AA@ 320b95ac     ScriptBind_Entity.obj
 0002:000055c4       ??_C@_0L@PCJMIDJC@min_energy?$AA@ 320b95c4     ScriptBind_Entity.obj
 0002:000055d0       ??_C@_07HAFFKDBK@density?$AA@ 320b95d0     ScriptBind_Entity.obj
 0002:000055d8       ??_C@_0BB@PINMJPMI@freefall_damping?$AA@ 320b95d8     ScriptBind_Entity.obj
 0002:000055ec       ??_C@_07IANOJGAO@damping?$AA@ 320b95ec     ScriptBind_Entity.obj
 0002:000055f4       ??_C@_0BC@IBPNNPAG@freefall_gravityx?$AA@ 320b95f4     ScriptBind_Entity.obj
 0002:00005608       ??_C@_0BC@JIOGOOEH@freefall_gravityy?$AA@ 320b9608     ScriptBind_Entity.obj
 0002:0000561c       ??_C@_0BC@LDMLLNIE@freefall_gravityz?$AA@ 320b961c     ScriptBind_Entity.obj
 0002:00005630       ??_C@_0BB@BNBHDCNK@freefall_gravity?$AA@ 320b9630     ScriptBind_Entity.obj
 0002:00005644       ??_C@_08PDICLKIK@gravityx?$AA@ 320b9644     ScriptBind_Entity.obj
 0002:00005650       ??_C@_08OKJJILML@gravityy?$AA@ 320b9650     ScriptBind_Entity.obj
 0002:0000565c       ??_C@_08MBLENIAI@gravityz?$AA@ 320b965c     ScriptBind_Entity.obj
 0002:00005668       ??_C@_0M@OCNGFCID@sleep_speed?$AA@ 320b9668     ScriptBind_Entity.obj
 0002:00005674       ??_C@_0O@FENAAHIH@max_time_step?$AA@ 320b9674     ScriptBind_Entity.obj
 0002:00005684       ??_C@_08KFMAPCCA@canBrake?$AA@ 320b9684     ScriptBind_Entity.obj
 0002:00005690       ??_C@_0N@KFJGGDPK@max_friction?$AA@ 320b9690     ScriptBind_Entity.obj
 0002:000056a0       ??_C@_0N@OFNJBLIM@min_friction?$AA@ 320b96a0     ScriptBind_Entity.obj
 0002:000056b0       ??_C@_08JMBLBDIB@susp_len?$AA@ 320b96b0     ScriptBind_Entity.obj
 0002:000056bc       ??_C@_0L@FHJANBOP@is_driving?$AA@ 320b96bc     ScriptBind_Entity.obj
 0002:000056c8       ??_C@_05HKPEHFPI@wheel?$AA@ 320b96c8     ScriptBind_Entity.obj
 0002:000056d0       ??_C@_07KJLEGEAK@maxGear?$AA@ 320b96d0     ScriptBind_Entity.obj
 0002:000056d8       ??_C@_07EPNEMLOL@minGear?$AA@ 320b96d8     ScriptBind_Entity.obj
 0002:000056e0       ??_C@_0BA@PJLKABGE@engine_startRPM?$AA@ 320b96e0     ScriptBind_Entity.obj
 0002:000056f0       ??_C@_0P@PHEAOBMJ@slip_threshold?$AA@ 320b96f0     ScriptBind_Entity.obj
 0002:00005700       ??_C@_0BE@OMBKKPHI@gear_dir_switch_RPM?$AA@ 320b9700     ScriptBind_Entity.obj
 0002:00005714       ??_C@_0BD@MMMIMMI@dyn_friction_ratio?$AA@ 320b9714     ScriptBind_Entity.obj
 0002:00005728       ??_C@_0N@IPFOFCEF@brake_torque?$AA@ 320b9728     ScriptBind_Entity.obj
 0002:00005738       ??_C@_05NKODJPOO@gears?$AA@ 320b9738     ScriptBind_Entity.obj
 0002:00005740       ??_C@_0N@JKFBFFPP@clutch_speed?$AA@ 320b9740     ScriptBind_Entity.obj
 0002:00005750       ??_C@_0L@HHGBOMEO@stabilizer?$AA@ 320b9750     ScriptBind_Entity.obj
 0002:0000575c       ??_C@_0BE@CEFMNMDE@engine_shiftdownRPM?$AA@ 320b975c     ScriptBind_Entity.obj
 0002:00005770       ??_C@_0BC@PCFENJJL@engine_shiftupRPM?$AA@ 320b9770     ScriptBind_Entity.obj
 0002:00005784       ??_C@_0P@JGPJJHEA@engine_idleRPM?$AA@ 320b9784     ScriptBind_Entity.obj
 0002:00005794       ??_C@_0O@FLFHOPKA@engine_minRPM?$AA@ 320b9794     ScriptBind_Entity.obj
 0002:000057a4       ??_C@_0BF@DBFPEHOH@max_braking_friction?$AA@ 320b97a4     ScriptBind_Entity.obj
 0002:000057bc       ??_C@_0BA@BOELIEEL@damping_vehicle?$AA@ 320b97bc     ScriptBind_Entity.obj
 0002:000057cc       ??_C@_0BE@OBIGAJJI@sleep_speed_vehicle?$AA@ 320b97cc     ScriptBind_Entity.obj
 0002:000057e0       ??_C@_0BG@FNPPNPNL@max_time_step_vehicle?$AA@ 320b97e0     ScriptBind_Entity.obj
 0002:000057f8       ??_C@_0BC@JIEPMFCH@intergration_type?$AA@ 320b97f8     ScriptBind_Entity.obj
 0002:0000580c       ??_C@_0O@FIKEAPOP@engine_maxRPM?$AA@ 320b980c     ScriptBind_Entity.obj
 0002:0000581c       ??_C@_0O@FFFPMCJD@engine_maxrpm?$AA@ 320b981c     ScriptBind_Entity.obj
 0002:0000582c       ??_C@_09HFFLCDL@max_steer?$AA@ 320b982c     ScriptBind_Entity.obj
 0002:00005838       ??_C@_0N@BKKDMJFH@engine_power?$AA@ 320b9838     ScriptBind_Entity.obj
 0002:00005848       ??_C@_0O@DIGOKPAL@axle_friction?$AA@ 320b9848     ScriptBind_Entity.obj
 0002:00005858       ??_C@_0BF@PAEALOMC@constant_orientation?$AA@ 320b9858     ScriptBind_Entity.obj
 0002:00005870       ??_C@_0BD@OEMIJLNL@collider_to_ignore?$AA@ 320b9870     ScriptBind_Entity.obj
 0002:00005884       ??_C@_0O@NENDNMBP@water_gravity?$AA@ 320b9884     ScriptBind_Entity.obj
 0002:00005894       ??_C@_01NOFIACDB@w?$AA@    320b9894     ScriptBind_Entity.obj
 0002:00005898       ??_C@_06IKLLLDHL@normal?$AA@ 320b9898     ScriptBind_Entity.obj
 0002:000058a0       ??_C@_0O@OPKMONPE@pierceability?$AA@ 320b98a0     ScriptBind_Entity.obj
 0002:000058b0       ??_C@_0M@CPDNCBIL@surface_idx?$AA@ 320b98b0     ScriptBind_Entity.obj
 0002:000058bc       ??_C@_0P@MIEIKOLB@min_bounce_vel?$AA@ 320b98bc     ScriptBind_Entity.obj
 0002:000058cc       ??_C@_08FGOJBMBB@acc_lift?$AA@ 320b98cc     ScriptBind_Entity.obj
 0002:000058d8       ??_C@_0L@OIINBEGG@acc_thrust?$AA@ 320b98d8     ScriptBind_Entity.obj
 0002:000058e4       ??_C@_0BD@LCECJCDG@k_water_resistance?$AA@ 320b98e4     ScriptBind_Entity.obj
 0002:000058f8       ??_C@_0BB@MEMNBGJ@k_air_resistance?$AA@ 320b98f8     ScriptBind_Entity.obj
 0002:0000590c       ??_C@_0BB@EJPANJDN@initial_velocity?$AA@ 320b990c     ScriptBind_Entity.obj
 0002:00005920       ??_C@_07MBJMFGGL@heading?$AA@ 320b9920     ScriptBind_Entity.obj
 0002:00005928       ??_C@_04IAGNFIBA@size?$AA@ 320b9928     ScriptBind_Entity.obj
 0002:00005930       ??_C@_06GMILPGDN@partid?$AA@ 320b9930     ScriptBind_Entity.obj
 0002:00005938       ??_C@_0O@LKIIAMCC@mat_breakable?$AA@ 320b9938     ScriptBind_Entity.obj
 0002:00005948       ??_C@_0P@GCMGJNHH@flags_collider?$AA@ 320b9948     ScriptBind_Entity.obj
 0002:00005958       ??_C@_0BE@JGPBLKM@flags_collider_mask?$AA@ 320b9958     ScriptBind_Entity.obj
 0002:0000596c       ??_C@_0BK@EFCCKBPG@collisionClassIgnoreUNSET?$AA@ 320b996c     ScriptBind_Entity.obj
 0002:00005988       ??_C@_0BE@IGKDPCKD@collisionClassUNSET?$AA@ 320b9988     ScriptBind_Entity.obj
 0002:0000599c       ??_C@_0BF@HNPAGFDJ@collisionClassIgnore?$AA@ 320b999c     ScriptBind_Entity.obj
 0002:000059b4       ??_C@_0P@IGDAAND@collisionClass?$AA@ 320b99b4     ScriptBind_Entity.obj
 0002:000059c4       ??_C@_0L@GECKPNLI@flags_mask?$AA@ 320b99c4     ScriptBind_Entity.obj
 0002:000059d0       ??_C@_0N@CLGPNGKP@foreignFlags?$AA@ 320b99d0     ScriptBind_Entity.obj
 0002:000059e0       ??_C@_0M@NGJNFAJM@foreignData?$AA@ 320b99e0     ScriptBind_Entity.obj
 0002:000059ec       ??_C@_08NMIAAFAA@frame2v1?$AA@ 320b99ec     ScriptBind_Entity.obj
 0002:000059f8       ??_C@_08MFJLDEEB@frame2v0?$AA@ 320b99f8     ScriptBind_Entity.obj
 0002:00005a04       ??_C@_08MODFKKOO@frame1v1?$AA@ 320b9a04     ScriptBind_Entity.obj
 0002:00005a10       ??_C@_08NHCOJLKP@frame1v0?$AA@ 320b9a10     ScriptBind_Entity.obj
 0002:00005a1c       ??_C@_06IGAKEMNE@point2?$AA@ 320b9a1c     ScriptBind_Entity.obj
 0002:00005a24       ??_C@_06KNCHBPBH@point1?$AA@ 320b9a24     ScriptBind_Entity.obj
 0002:00005a2c       ??_C@_07LFHEJDJG@partid2?$AA@ 320b9a2c     ScriptBind_Entity.obj
 0002:00005a34       ??_C@_07JOFJMAFF@partid1?$AA@ 320b9a34     ScriptBind_Entity.obj
 0002:00005a3c       __real@41000000            320b9a3c     ScriptBind_Entity.obj
 0002:00005a40       ??_C@_0DL@LAFFPNGB@ERROR?3?5CScriptObjectWeapon?3?3GetB@ 320b9a40     ScriptBind_Entity.obj
 0002:00005a7c       __real@c11ccccd            320b9a7c     ScriptBind_Entity.obj
 0002:00005a80       ??_C@_0BP@DPMIDAMI@CScriptBind_Entity?3?3GetGravity?$AA@ 320b9a80     ScriptBind_Entity.obj
 0002:00005aa0       ??_C@_08PNMNOKOB@entities?$AA@ 320b9aa0     ScriptBind_Entity.obj
 0002:00005aac       ??_C@_08OEMCHAOB@contacts?$AA@ 320b9aac     ScriptBind_Entity.obj
 0002:00005ab8       ??_C@_08DFIAGKEA@collider?$AA@ 320b9ab8     ScriptBind_Entity.obj
 0002:00005ac4       ??_C@_07IHECPBBE@partid0?$AA@ 320b9ac4     ScriptBind_Entity.obj
 0002:00005acc       ??_C@_06BBLOAEEI@center?$AA@ 320b9acc     ScriptBind_Entity.obj
 0002:00005ad4       ??_C@_0N@LOJNGBFM@FallOffScale?$AA@ 320b9ad4     ScriptBind_Entity.obj
 0002:00005ae4       ??_C@_0N@FCLHNOGE@FallOffShift?$AA@ 320b9ae4     ScriptBind_Entity.obj
 0002:00005af4       ??_C@_0P@NCJDECHD@FallOffDirLati?$AA@ 320b9af4     ScriptBind_Entity.obj
 0002:00005b04       ??_C@_0P@LNHODOGI@FallOffDirLong?$AA@ 320b9b04     ScriptBind_Entity.obj
 0002:00005b14       ??_C@_09BMPHBPKF@SoftEdges?$AA@ 320b9b14     ScriptBind_Entity.obj
 0002:00005b20       ??_C@_0M@GGCKEINF@fHDRDynamic?$AA@ 320b9b20     ScriptBind_Entity.obj
 0002:00005b2c       ??_C@_0L@LMADJJLL@NearCutoff?$AA@ 320b9b2c     ScriptBind_Entity.obj
 0002:00005b38       ??_C@_0O@PGNFPKNC@DensityOffset?$AA@ 320b9b38     ScriptBind_Entity.obj
 0002:00005b48       ??_C@_0O@FLILJIAI@GlobalDensity?$AA@ 320b9b48     ScriptBind_Entity.obj
 0002:00005b58       ??_C@_0BD@CJBKOFEA@bUseGlobalFogColor?$AA@ 320b9b58     ScriptBind_Entity.obj
 0002:00005b6c       ??_C@_0M@NGPPAHCC@color_Color?$AA@ 320b9b6c     ScriptBind_Entity.obj
 0002:00005b78       ??_C@_04EBKMHHBE@Size?$AA@ 320b9b78     ScriptBind_Entity.obj
 0002:00005b80       ??_C@_0L@FPPPCJKO@VolumeType?$AA@ 320b9b80     ScriptBind_Entity.obj
 0002:00005b8c       ??_C@_0O@PFOFOJE@fFadeDistance?$AA@ 320b9b8c     ScriptBind_Entity.obj
 0002:00005b9c       ??_C@_0BE@CHGKAGOM@vector_SpaceLoopBox?$AA@ 320b9b9c     ScriptBind_Entity.obj
 0002:00005bb0       ??_C@_0N@OEHAKPOO@vector_Speed?$AA@ 320b9bb0     ScriptBind_Entity.obj
 0002:00005bc0       ??_C@_09IOGLHCGO@bAutoMove?$AA@ 320b9bc0     ScriptBind_Entity.obj
 0002:00005bcc       ??_C@_08KNOEMJMM@material?$AA@ 320b9bcc     ScriptBind_Entity.obj
 0002:00005bd8       ??_C@_08GILMLDKH@backface?$AA@ 320b9bd8     ScriptBind_Entity.obj
 0002:00005be4       ??_C@_08LHFODBFO@distance?$AA@ 320b9be4     ScriptBind_Entity.obj
 0002:00005bf0       ??_C@_0M@KCMDKMEG@baricentric?$AA@ 320b9bf0     ScriptBind_Entity.obj
 0002:00005bfc       ??_C@_03DPFGDANO@uv2?$AA@  320b9bfc     ScriptBind_Entity.obj
 0002:00005c00       ??_C@_03BEHLGDBN@uv1?$AA@  320b9c00     ScriptBind_Entity.obj
 0002:00005c04       ??_C@_03NGAFCFM@uv0?$AA@   320b9c04     ScriptBind_Entity.obj
 0002:00005c08       ??_C@_02LNLCGGHO@v2?$AA@   320b9c08     ScriptBind_Entity.obj
 0002:00005c0c       ??_C@_02JGJPDFLN@v1?$AA@   320b9c0c     ScriptBind_Entity.obj
 0002:00005c10       ??_C@_02IPIEAEPM@v0?$AA@   320b9c10     ScriptBind_Entity.obj
 0002:00005c18       ??_C@_0FA@LOABCBNK@ActivateOutput?$CI?$CFs?0value?$CJ?5called?5@ 320b9c18     ScriptBind_Entity.obj
 0002:00005c68       ??_C@_0DM@EJDLJNBC@ActivateOutput?5called?5with?5undef@ 320b9c68     ScriptBind_Entity.obj
 0002:00005ca4       ??_C@_0BJ@IKBGFCL@RagDollized?5with?5mass?5?$CFf?$AA@ 320b9ca4     ScriptBind_Entity.obj
 0002:00005cc0       __real@40b00000            320b9cc0     ScriptBind_Entity.obj
 0002:00005cc4       __real@42920000            320b9cc4     ScriptBind_Entity.obj
 0002:00005cc8       __real@42a00000            320b9cc8     ScriptBind_Entity.obj
 0002:00005ccc       ??_C@_01MCMALHOG@a?$AA@    320b9ccc     ScriptBind_Entity.obj
 0002:00005cd0       ??_C@_01OJONOECF@b?$AA@    320b9cd0     ScriptBind_Entity.obj
 0002:00005cd4       ??_C@_01JEJKBAGA@g?$AA@    320b9cd4     ScriptBind_Entity.obj
 0002:00005cd8       ??_C@_01KDCPPGHE@r?$AA@    320b9cd8     ScriptBind_Entity.obj
 0002:00005cdc       ??_C@_0CG@MHMGGACD@?$FL?$CFs?$FN?5?$CFd?5arguments?5passed?0?52?5expe@ 320b9cdc     ScriptBind_Entity.obj
 0002:00005d04       ??_C@_0CD@BBFDLPJL@CScriptBind_Entity?3?3SetPublicPar@ 320b9d04     ScriptBind_Entity.obj
 0002:00005d28       ??_C@_06PGMJADPC@nFlags?$AA@ 320b9d28     ScriptBind_Entity.obj
 0002:00005d30       ??_C@_04GPMDFGEJ@type?$AA@ 320b9d30     ScriptBind_Entity.obj
 0002:00005d38       ??_7CScriptBind_Entity@@6B@ 320b9d38     ScriptBind_Entity.obj
 0002:00005d4c       ??_C@_01GAPBHFFA@T?$AA@    320b9d4c     ScriptBind_Entity.obj
 0002:00005d50       __real@406fe00000000000    320b9d50     ScriptBind_Entity.obj
 0002:00005d58       ??_C@_0N@IGDIPJAP@SplineElem?$DM?$DO?$AA@ 320b9d58     ScriptBind_Entity.obj
 0002:00005d68       ??_C@_05LPIJGKJ@Value?$AA@ 320b9d68     ScriptBind_Entity.obj
 0002:00005d70       ??_C@_05EDKIKEAI@fTime?$AA@ 320b9d70     ScriptBind_Entity.obj
 0002:00005d78       ??_C@_03DAKNAIGI@idx?$AA@  320b9d78     ScriptBind_Entity.obj
 0002:00005d7c       ??_C@_04MDNLLEAH@vPos?$AA@ 320b9d7c     ScriptBind_Entity.obj
 0002:00005d84       ??_C@_03PCBNCGFH@pos?$AA@  320b9d84     ScriptBind_Entity.obj
 0002:00005d88       ??_C@_0O@MMPEOLLD@deferred_geom?$AA@ 320b9d88     ScriptBind_Entity.obj
 0002:00005d98       ??_C@_0O@BICFJHM@time_scrubbed?$AA@ 320b9d98     ScriptBind_Entity.obj
 0002:00005da8       ??_C@_0BM@JCLKBMIK@time_scrubbing_in_trackview?$AA@ 320b9da8     ScriptBind_Entity.obj
 0002:00005dc4       ??_C@_0BA@HGOBEMFK@light_animation?$AA@ 320b9dc4     ScriptBind_Entity.obj
 0002:00005dd4       ??_C@_0CH@GPAHCJDH@Light?5reflection?5texture?5not?5fou@ 320b9dd4     ScriptBind_Entity.obj
 0002:00005dfc       ??_C@_0BD@IGPNAJNL@reflection_texture?$AA@ 320b9dfc     ScriptBind_Entity.obj
 0002:00005e10       __real@43070000            320b9e10     ScriptBind_Entity.obj
 0002:00005e14       ??_C@_0BK@LJJEJONI@Textures?1defaults?1red?4dds?$AA@ 320b9e14     ScriptBind_Entity.obj
 0002:00005e30       ??_C@_0CG@FNOEHKK@Light?5projector?5texture?5not?5foun@ 320b9e30     ScriptBind_Entity.obj
 0002:00005e58       ??_C@_07MBGBNJBB@cubemap?$AA@ 320b9e58     ScriptBind_Entity.obj
 0002:00005e60       ??_C@_0BC@HKEHDKFM@projector_texture?$AA@ 320b9e60     ScriptBind_Entity.obj
 0002:00005e74       ??_C@_0P@BFAEBMJA@proj_nearplane?$AA@ 320b9e74     ScriptBind_Entity.obj
 0002:00005e84       ??_C@_08ENFBAMPB@proj_fov?$AA@ 320b9e84     ScriptBind_Entity.obj
 0002:00005e90       ??_C@_0O@CJKIICOO@attach_to_sun?$AA@ 320b9e90     ScriptBind_Entity.obj
 0002:00005ea0       __real@3f355555            320b9ea0     ScriptBind_Entity.obj
 0002:00005ea4       ??_C@_09NGEPABBE@flare_FOV?$AA@ 320b9ea4     ScriptBind_Entity.obj
 0002:00005eb0       ??_C@_0N@NJLGFBA@flare_enable?$AA@ 320b9eb0     ScriptBind_Entity.obj
 0002:00005ec0       ??_C@_0M@PNMLIHJM@flare_Flare?$AA@ 320b9ec0     ScriptBind_Entity.obj
 0002:00005ecc       ??_C@_0BI@GLHFMIME@attenuation_falloff_max?$AA@ 320b9ecc     ScriptBind_Entity.obj
 0002:00005ee4       ??_C@_0O@MODPBEIG@sort_priority?$AA@ 320b9ee4     ScriptBind_Entity.obj
 0002:00005ef4       ??_C@_06NOKHKJEC@hdrdyn?$AA@ 320b9ef4     ScriptBind_Entity.obj
 0002:00005efc       ??_C@_0BH@MHLPEAKP@fade_dimensions_bottom?$AA@ 320b9efc     ScriptBind_Entity.obj
 0002:00005f14       ??_C@_0BE@FLFNDNCF@fade_dimensions_top?$AA@ 320b9f14     ScriptBind_Entity.obj
 0002:00005f28       ??_C@_0BE@JJOFONLJ@fade_dimensions_far?$AA@ 320b9f28     ScriptBind_Entity.obj
 0002:00005f3c       ??_C@_0BF@OFPDEAO@fade_dimensions_near?$AA@ 320b9f3c     ScriptBind_Entity.obj
 0002:00005f54       ??_C@_0BG@CJNLJIFK@fade_dimensions_right?$AA@ 320b9f54     ScriptBind_Entity.obj
 0002:00005f6c       ??_C@_0BF@CHIKNGGN@fade_dimensions_left?$AA@ 320b9f6c     ScriptBind_Entity.obj
 0002:00005f84       __real@43800000            320b9f84     ScriptBind_Entity.obj
 0002:00005f88       ??_C@_0BD@CDEKNNOE@shadowUpdate_ratio?$AA@ 320b9f88     ScriptBind_Entity.obj
 0002:00005f9c       ??_C@_0BH@FHDMIJON@shadowUpdate_MinRadius?$AA@ 320b9f9c     ScriptBind_Entity.obj
 0002:00005fb4       ??_C@_0BE@FMCBEEMP@shadowMinResolution?$AA@ 320b9fb4     ScriptBind_Entity.obj
 0002:00005fc8       ??_C@_0BC@GNKJBIOP@shadow_slope_bias?$AA@ 320b9fc8     ScriptBind_Entity.obj
 0002:00005fdc       ??_C@_0M@DHEEFDBJ@shadow_bias?$AA@ 320b9fdc     ScriptBind_Entity.obj
 0002:00005fe8       ??_C@_0L@BBFBCBHN@box_length?$AA@ 320b9fe8     ScriptBind_Entity.obj
 0002:00005ff4       ??_C@_0L@KEHFNODH@box_height?$AA@ 320b9ff4     ScriptBind_Entity.obj
 0002:00006000       ??_C@_09CIAIHHPI@box_width?$AA@ 320ba000     ScriptBind_Entity.obj
 0002:0000600c       ??_C@_0P@NNMNIGHF@box_projection?$AA@ 320ba00c     ScriptBind_Entity.obj
 0002:0000601c       ??_C@_0BG@LJGHMGAB@area_diffuse_softness?$AA@ 320ba01c     ScriptBind_Entity.obj
 0002:00006034       ??_C@_0O@EJPOELFP@area_spec_tex?$AA@ 320ba034     ScriptBind_Entity.obj
 0002:00006044       ??_C@_08DIFNPFEO@area_fov?$AA@ 320ba044     ScriptBind_Entity.obj
 0002:00006050       ??_C@_0M@LOGHCJPL@area_height?$AA@ 320ba050     ScriptBind_Entity.obj
 0002:0000605c       ??_C@_0L@OACLMGOM@area_width?$AA@ 320ba05c     ScriptBind_Entity.obj
 0002:00006068       ??_C@_0M@HMEPJJLM@cast_shadow?$AA@ 320ba068     ScriptBind_Entity.obj
 0002:00006074       ??_C@_0BE@KJDINKNK@specular_multiplier?$AA@ 320ba074     ScriptBind_Entity.obj
 0002:00006088       ??_C@_0O@GDPFAHNI@diffuse_color?$AA@ 320ba088     ScriptBind_Entity.obj
 0002:00006098       ??_C@_0BD@KHONJDD@irradiance_volumes?$AA@ 320ba098     ScriptBind_Entity.obj
 0002:000060ac       ??_C@_0P@HFLPFNOJ@deferred_light?$AA@ 320ba0ac     ScriptBind_Entity.obj
 0002:000060bc       ??_C@_0L@GIMEJMBD@area_light?$AA@ 320ba0bc     ScriptBind_Entity.obj
 0002:000060c8       ??_C@_07LIABELBC@ambient?$AA@ 320ba0c8     ScriptBind_Entity.obj
 0002:000060d0       ??_C@_0M@MJDDIEMJ@has_cbuffer?$AA@ 320ba0d0     ScriptBind_Entity.obj
 0002:000060dc       ??_C@_0M@JIOKGBCI@indoor_only?$AA@ 320ba0dc     ScriptBind_Entity.obj
 0002:000060e8       ??_C@_04PADNKBEK@fake?$AA@ 320ba0e8     ScriptBind_Entity.obj
 0002:000060f0       ??_C@_0N@JCGAFEEJ@hasclipbound?$AA@ 320ba0f0     ScriptBind_Entity.obj
 0002:00006100       ??_C@_0BC@OMAJPEBJ@disable_x360_opto?$AA@ 320ba100     ScriptBind_Entity.obj
 0002:00006114       ??_C@_0BA@HBLBHICG@ignore_visareas?$AA@ 320ba114     ScriptBind_Entity.obj
 0002:00006124       ??_C@_0P@PNLFDPHO@this_area_only?$AA@ 320ba124     ScriptBind_Entity.obj
 0002:00006134       ??_C@_0CP@JECPLGIJ@Deferred?5diffuse?5cubemap?5texture@ 320ba134     ScriptBind_Entity.obj
 0002:00006164       ??_C@_0CH@DKIKEFKO@Deferred?5cubemap?5texture?5not?5fou@ 320ba164     ScriptBind_Entity.obj
 0002:0000618c       ??_C@_09IDFDHOCA@?$CFs?$CFs?$CFs?4?$CFs?$AA@ 320ba18c     ScriptBind_Entity.obj
 0002:00006198       ??_C@_05OGIEPGMJ@_diff?$AA@ 320ba198     ScriptBind_Entity.obj
 0002:000061a0       ??_C@_0BB@FOGBLD@deferred_cubemap?$AA@ 320ba1a0     ScriptBind_Entity.obj
 0002:000061b4       ??_C@_06KGHINEPG@radius?$AA@ 320ba1b4     ScriptBind_Entity.obj
 0002:000061bc       ??_C@_0L@DOHNHILA@cheapLight?$AA@ 320ba1bc     ScriptBind_Entity.obj
 0002:000061c8       ??_C@_0L@MLHIMACD@anim_phase?$AA@ 320ba1c8     ScriptBind_Entity.obj
 0002:000061d4       ??_C@_0L@JDKOBHBK@anim_speed?$AA@ 320ba1d4     ScriptBind_Entity.obj
 0002:000061e0       ??_C@_05IAKJCFIM@style?$AA@ 320ba1e0     ScriptBind_Entity.obj
 0002:000061e8       ??_C@_01ICJEACDI@?$DL?$AA@ 320ba1e8     ScriptBind_Entity.obj
 0002:000061ec       ??_C@_0L@LFGNALKI@bRigidCore?$AA@ 320ba1ec     ScriptBind_Entity.obj
 0002:000061f8       ??_C@_0BB@OOPFKAK@AttachmentPartId?$AA@ 320ba1f8     ScriptBind_Entity.obj
 0002:0000620c       ??_C@_0N@KPDPFGEP@AttachmentId?$AA@ 320ba20c     ScriptBind_Entity.obj
 0002:0000621c       ??_C@_06GPGIDCJA@points?$AA@ 320ba21c     ScriptBind_Entity.obj
 0002:00006224       ??_C@_04HABAAEPG@axis?$AA@ 320ba224     ScriptBind_Entity.obj
 0002:0000622c       ??_C@_07EPGABBNN@box_max?$AA@ 320ba22c     ScriptBind_Entity.obj
 0002:00006234       ??_C@_07FNOLPFLC@box_min?$AA@ 320ba234     ScriptBind_Entity.obj
 0002:0000623c       ??_C@_0L@GDPBJPKC@resistance?$AA@ 320ba23c     ScriptBind_Entity.obj
 0002:00006248       ??_C@_08PPLCFKON@variance?$AA@ 320ba248     ScriptBind_Entity.obj
 0002:00006254       ??_C@_0N@IHPOOCAJ@falloffInner?$AA@ 320ba254     ScriptBind_Entity.obj
 0002:00006264       ??_C@_07JONEAHHA@falloff?$AA@ 320ba264     ScriptBind_Entity.obj
 0002:0000626c       ??_C@_07HIAOBKCE@uniform?$AA@ 320ba26c     ScriptBind_Entity.obj
 0002:00006274       ??_C@_04KPICECCB@Area?$AA@ 320ba274     ScriptBind_Entity.obj
 0002:0000627c       ??_C@_0L@FDDHNFJ@gearRatios?$AA@ 320ba27c     ScriptBind_Entity.obj
 0002:00006288       ??_C@_0BG@GFBHONKN@steerTrackNeutralTurn?$AA@ 320ba288     ScriptBind_Entity.obj
 0002:000062a0       ??_C@_06LHAOKEGO@wheels?$AA@ 320ba2a0     ScriptBind_Entity.obj
 0002:000062a8       ??_C@_0M@MEAFJKEC@dynFriction?$AA@ 320ba2a8     ScriptBind_Entity.obj
 0002:000062b4       ??_C@_0BB@MGBFJPLF@gearDirSwitchRPM?$AA@ 320ba2b4     ScriptBind_Entity.obj
 0002:000062c8       ??_C@_0O@IILPBJ@slipThreshold?$AA@ 320ba2c8     ScriptBind_Entity.obj
 0002:000062d8       ??_C@_09KIBCGPL@minEnergy?$AA@ 320ba2d8     ScriptBind_Entity.obj
 0002:000062e4       ??_C@_0M@OOJMDCCJ@maxTimeStep?$AA@ 320ba2e4     ScriptBind_Entity.obj
 0002:000062f0       ??_C@_08KOLJJKBD@maxSteer?$AA@ 320ba2f0     ScriptBind_Entity.obj
 0002:000062fc       ??_C@_0BD@KJNJCIHH@maxBrakingFriction?$AA@ 320ba2fc     ScriptBind_Entity.obj
 0002:00006310       ??_C@_0BA@MGLJDEEN@integrationType?$AA@ 320ba310     ScriptBind_Entity.obj
 0002:00006320       ??_C@_0P@KBBHLCNA@engineStartRPM?$AA@ 320ba320     ScriptBind_Entity.obj
 0002:00006330       ??_C@_0BB@CHDJANIK@engineShiftUpRPM?$AA@ 320ba330     ScriptBind_Entity.obj
 0002:00006344       ??_C@_0BD@PGDLDMIE@engineShiftDownRPM?$AA@ 320ba344     ScriptBind_Entity.obj
 0002:00006358       ??_C@_0M@FLHMAEHK@enginePower?$AA@ 320ba358     ScriptBind_Entity.obj
 0002:00006364       ??_C@_0N@BOMJGMBI@engineMinRPM?$AA@ 320ba364     ScriptBind_Entity.obj
 0002:00006374       ??_C@_0N@BNDKIMFH@engineMaxRPM?$AA@ 320ba374     ScriptBind_Entity.obj
 0002:00006384       ??_C@_0O@FDAGDCHN@engineIdleRPM?$AA@ 320ba384     ScriptBind_Entity.obj
 0002:00006394       ??_C@_0M@OKIHMAIH@clutchSpeed?$AA@ 320ba394     ScriptBind_Entity.obj
 0002:000063a0       ??_C@_0M@KKAMMPPJ@brakeTorque?$AA@ 320ba3a0     ScriptBind_Entity.obj
 0002:000063ac       ??_C@_0N@ENJCCKHH@axleFriction?$AA@ 320ba3ac     ScriptBind_Entity.obj
 0002:000063bc       ??_C@_07EKPBFBMM@Wheeled?$AA@ 320ba3bc     ScriptBind_Entity.obj
 0002:000063c4       ??_C@_0BD@BPODOOJF@timeImpulseRecover?$AA@ 320ba3c4     ScriptBind_Entity.obj
 0002:000063d8       ??_C@_0P@HKLLLCON@min_fall_angle?$AA@ 320ba3d8     ScriptBind_Entity.obj
 0002:000063e8       ??_C@_0P@EFDAFGKO@max_jump_angle?$AA@ 320ba3e8     ScriptBind_Entity.obj
 0002:000063f8       ??_C@_0BA@PHNFBAFB@max_climb_angle?$AA@ 320ba3f8     ScriptBind_Entity.obj
 0002:00006408       ??_C@_0BA@MFCPJLC@min_slide_angle?$AA@ 320ba408     ScriptBind_Entity.obj
 0002:00006418       ??_C@_0N@JAMKHGMD@inertiaAccel?$AA@ 320ba418     ScriptBind_Entity.obj
 0002:00006428       ??_C@_07IKGGBMHK@inertia?$AA@ 320ba428     ScriptBind_Entity.obj
 0002:00006430       ??_C@_0M@JFMIBLNG@height_head?$AA@ 320ba430     ScriptBind_Entity.obj
 0002:0000643c       ??_C@_0M@PMLALDOH@head_radius?$AA@ 320ba43c     ScriptBind_Entity.obj
 0002:00006448       ??_C@_0N@MPJIOODI@height_pivot?$AA@ 320ba448     ScriptBind_Entity.obj
 0002:00006458       ??_C@_0L@LOLELGEE@height_eye?$AA@ 320ba458     ScriptBind_Entity.obj
 0002:00006464       ??_C@_06LNLHEAAG@height?$AA@ 320ba464     ScriptBind_Entity.obj
 0002:0000646c       ??_C@_06JGIKNHLC@Living?$AA@ 320ba46c     ScriptBind_Entity.obj
 0002:00006474       ??_C@_0BC@GOHEOECB@no_path_alignment?$AA@ 320ba474     ScriptBind_Entity.obj
 0002:00006488       ??_C@_07LGKPJIDE@no_spin?$AA@ 320ba488     ScriptBind_Entity.obj
 0002:00006490       ??_C@_07LHEIFGCE@no_roll?$AA@ 320ba490     ScriptBind_Entity.obj
 0002:00006498       ??_C@_0P@OKNMMADN@single_contact?$AA@ 320ba498     ScriptBind_Entity.obj
 0002:000064a8       ??_C@_05DBCPOPCA@wspin?$AA@ 320ba4a8     ScriptBind_Entity.obj
 0002:000064b0       ??_C@_08ICEJNDOI@velocity?$AA@ 320ba4b0     ScriptBind_Entity.obj
 0002:000064bc       ??_C@_0L@GODMBODA@accel_lift?$AA@ 320ba4bc     ScriptBind_Entity.obj
 0002:000064c8       ??_C@_0N@IKBMFIHM@accel_thrust?$AA@ 320ba4c8     ScriptBind_Entity.obj
 0002:000064d8       ??_C@_08HIFHGEKA@Particle?$AA@ 320ba4d8     ScriptBind_Entity.obj
 0002:000064e4       ??_C@_08EBPMEEHK@CGFprops?$AA@ 320ba4e4     ScriptBind_Entity.obj
 0002:000064f0       ??_C@_03ONFBEKOG@lod?$AA@  320ba4f0     ScriptBind_Entity.obj
 0002:000064f4       ??_C@_0BA@KAMBHNIJ@stiffness_scale?$AA@ 320ba4f4     ScriptBind_Entity.obj
 0002:00006504       ??_C@_0BC@EMGAGLJJ@flagsColliderMask?$AA@ 320ba504     ScriptBind_Entity.obj
 0002:00006518       ??_C@_0O@LHPDLPPH@flagsCollider?$AA@ 320ba518     ScriptBind_Entity.obj
 0002:00006528       ??_C@_09FGHKFENE@flagsMask?$AA@ 320ba528     ScriptBind_Entity.obj
 0002:00006534       ??_C@_05MFEJDJP@value?$AA@ 320ba534     ScriptBind_Entity.obj
 0002:0000653c       ??_C@_06JMGHNNK@params?$AA@ 320ba53c     ScriptBind_Entity.obj
 0002:00006544       ??_C@_0CF@LAMDNHP@InsertSubpipe?3?5Wrong?5parameter?5t@ 320ba544     ScriptBind_Entity.obj
 0002:0000656c       ??_C@_0CC@FDDDEJLD@InsertSubpipe?3?5Too?5few?5parameter@ 320ba56c     ScriptBind_Entity.obj
 0002:00006590       ??_C@_0DC@CJCGPHGA@InsertSubpipe?3?5The?5entity?8s?5AI?5i@ 320ba590     ScriptBind_Entity.obj
 0002:000065c4       ??_C@_0CL@GOGALFIG@InsertSubpipe?3?5The?5entity?5does?5n@ 320ba5c4     ScriptBind_Entity.obj
 0002:000065f0       ??_C@_0CC@EINNAIIL@SelectPipe?3?5Wrong?5parameter?5type@ 320ba5f0     ScriptBind_Entity.obj
 0002:00006614       ??_C@_0DE@FAHFLKKB@?$FLAIWARNING?$FN?5Entity?5?$CFs?5failed?5to?5@ 320ba614     ScriptBind_Entity.obj
 0002:00006648       ??_C@_0BP@DKLKNGN@SelectPipe?3?5Too?5few?5parameters?$AA@ 320ba648     ScriptBind_Entity.obj
 0002:00006668       ??_C@_0CP@MENHAOKJ@SelectPipe?3?5The?5entity?8s?5AI?5is?5n@ 320ba668     ScriptBind_Entity.obj
 0002:00006698       ??_C@_0CI@GFJGDEBK@SelectPipe?3?5The?5entity?5does?5not?5@ 320ba698     ScriptBind_Entity.obj
 0002:000066c0       ??_C@_0BP@IAEJOGJH@ATTACHMENT_KEEP_TRANSFORMATION?$AA@ 320ba6c0     ScriptBind_Entity.obj
 0002:000066e0       ??_C@_07LPLELEBD@PE_AREA?$AA@ 320ba6e0     ScriptBind_Entity.obj
 0002:000066e8       ??_C@_07DCBEKHPO@PE_SOFT?$AA@ 320ba6e8     ScriptBind_Entity.obj
 0002:000066f0       ??_C@_07EEAGHCJM@PE_ROPE?$AA@ 320ba6f0     ScriptBind_Entity.obj
 0002:000066f8       ??_C@_0P@GJFCIKMJ@PE_ARTICULATED?$AA@ 320ba6f8     ScriptBind_Entity.obj
 0002:00006708       ??_C@_0M@MLKNDIIB@PE_PARTICLE?$AA@ 320ba708     ScriptBind_Entity.obj
 0002:00006714       ??_C@_0BC@OFIJOFAN@PE_WHEELEDVEHICLE?$AA@ 320ba714     ScriptBind_Entity.obj
 0002:00006728       ??_C@_08CGHMDAPO@PE_RIGID?$AA@ 320ba728     ScriptBind_Entity.obj
 0002:00006734       ??_C@_09ICONKGJO@PE_LIVING?$AA@ 320ba734     ScriptBind_Entity.obj
 0002:00006740       ??_C@_09LNKDEMKN@PE_STATIC?$AA@ 320ba740     ScriptBind_Entity.obj
 0002:0000674c       ??_C@_07PHKOIGGF@PE_NONE?$AA@ 320ba74c     ScriptBind_Entity.obj
 0002:00006754       ??_C@_0BF@PECEJAP@ENTITY_UPDATE_ALWAYS?$AA@ 320ba754     ScriptBind_Entity.obj
 0002:0000676c       ??_C@_0BO@BDMMADOM@ENTITY_UPDATE_PHYSICS_VISIBLE?$AA@ 320ba76c     ScriptBind_Entity.obj
 0002:0000678c       ??_C@_0BG@CJGNBFJE@ENTITY_UPDATE_PHYSICS?$AA@ 320ba78c     ScriptBind_Entity.obj
 0002:000067a4       ??_C@_0BG@CHLMOAJ@ENTITY_UPDATE_VISIBLE?$AA@ 320ba7a4     ScriptBind_Entity.obj
 0002:000067bc       ??_C@_0BK@BBEEOOGK@ENTITY_UPDATE_POT_VISIBLE?$AA@ 320ba7bc     ScriptBind_Entity.obj
 0002:000067d8       ??_C@_0BH@MNPAACIK@ENTITY_UPDATE_IN_RANGE?$AA@ 320ba7d8     ScriptBind_Entity.obj
 0002:000067f0       ??_C@_0BE@BANFPNNB@ENTITY_UPDATE_NEVER?$AA@ 320ba7f0     ScriptBind_Entity.obj
 0002:00006804       ??_C@_0BK@FOKHDBHM@ENTITY_FLAG_GOOD_OCCLUDER?$AA@ 320ba804     ScriptBind_Entity.obj
 0002:00006820       ??_C@_0BH@CPKMLPGB@ENTITY_FLAG_CASTSHADOW?$AA@ 320ba820     ScriptBind_Entity.obj
 0002:00006838       ??_C@_0BI@CKBHHGLN@ENTITY_FLAG_AI_HIDEABLE?$AA@ 320ba838     ScriptBind_Entity.obj
 0002:00006850       ??_C@_0BJ@CHMAPNHB@ENTITY_FLAG_VOLUME_SOUND?$AA@ 320ba850     ScriptBind_Entity.obj
 0002:0000686c       ??_C@_0BF@ELIIGHPH@ENTITY_FLAG_ON_RADAR?$AA@ 320ba86c     ScriptBind_Entity.obj
 0002:00006884       ??_C@_0BJ@BDHIJOKO@ENTITY_FLAG_NO_PROXIMITY?$AA@ 320ba884     ScriptBind_Entity.obj
 0002:000068a0       ??_C@_0BE@CFKFBAHN@ENTITY_FLAG_NO_SAVE?$AA@ 320ba8a0     ScriptBind_Entity.obj
 0002:000068b4       ??_C@_0BK@NIKIJADF@ENTITY_FLAG_TRIGGER_AREAS?$AA@ 320ba8b4     ScriptBind_Entity.obj
 0002:000068d0       ??_C@_0CC@GJKGEDMK@ENTITY_FLAG_IGNORE_PHYSICS_UPDAT@ 320ba8d0     ScriptBind_Entity.obj
 0002:000068f4       ??_C@_0BM@MIJAKBG@ENTITY_FLAG_CALCBBOX_USEALL?$AA@ 320ba8f4     ScriptBind_Entity.obj
 0002:00006910       ??_C@_0BI@LDKPEEII@ENTITY_FLAG_SERVER_ONLY?$AA@ 320ba910     ScriptBind_Entity.obj
 0002:00006928       ??_C@_0BI@LAEDLKDG@ENTITY_FLAG_CLIENT_ONLY?$AA@ 320ba928     ScriptBind_Entity.obj
 0002:00006940       ??_C@_0BJ@EKGCJLPG@ENTITY_FLAG_CALC_PHYSICS?$AA@ 320ba940     ScriptBind_Entity.obj
 0002:0000695c       ??_C@_0CE@LEBCIGAH@ENTITY_FLAG_NOT_REGISTER_IN_SECT@ 320ba95c     ScriptBind_Entity.obj
 0002:00006980       ??_C@_0BH@JCGBKMCJ@ENTITY_FLAG_WRITE_ONLY?$AA@ 320ba980     ScriptBind_Entity.obj
 0002:00006998       ??_C@_0BN@DJKPEBKE@FOREIGNFLAGS_MOVING_PLATFORM?$AA@ 320ba998     ScriptBind_Entity.obj
 0002:000069b8       ??_C@_0M@KAOENOII@AREA_SPLINE?$AA@ 320ba9b8     ScriptBind_Entity.obj
 0002:000069c4       ??_C@_0O@GHNOADLG@AREA_CYLINDER?$AA@ 320ba9c4     ScriptBind_Entity.obj
 0002:000069d4       ??_C@_0L@LKHDAAFF@AREA_SHAPE?$AA@ 320ba9d4     ScriptBind_Entity.obj
 0002:000069e0       ??_C@_0O@GGALCEOF@AREA_GEOMETRY?$AA@ 320ba9e0     ScriptBind_Entity.obj
 0002:000069f0       ??_C@_0M@KIOJNOE@AREA_SPHERE?$AA@ 320ba9f0     ScriptBind_Entity.obj
 0002:000069fc       ??_C@_08JHNBFOLE@AREA_BOX?$AA@ 320ba9fc     ScriptBind_Entity.obj
 0002:00006a08       ??_C@_0BB@FKKDPKLG@ent_sort_by_mass?$AA@ 320baa08     ScriptBind_Entity.obj
 0002:00006a1c       ??_C@_07PILACILF@ent_all?$AA@ 320baa1c     ScriptBind_Entity.obj
 0002:00006a24       ??_C@_0M@GPLOPBFO@ent_terrain?$AA@ 320baa24     ScriptBind_Entity.obj
 0002:00006a30       ??_C@_0BA@HFPJPMGN@ent_independent?$AA@ 320baa30     ScriptBind_Entity.obj
 0002:00006a40       ??_C@_0L@GADIPNLG@ent_living?$AA@ 320baa40     ScriptBind_Entity.obj
 0002:00006a4c       ??_C@_09HADDCMPP@ent_rigid?$AA@ 320baa4c     ScriptBind_Entity.obj
 0002:00006a58       ??_C@_0BD@LHFAFOGK@ent_sleeping_rigid?$AA@ 320baa58     ScriptBind_Entity.obj
 0002:00006a6c       ??_C@_0L@FPHGBHIF@ent_static?$AA@ 320baa6c     ScriptBind_Entity.obj
 0002:00006a78       ??_C@_0BM@HBNPGBMB@geom_colltype_foliage_proxy?$AA@ 320baa78     ScriptBind_Entity.obj
 0002:00006a94       ??_C@_0BI@HIGMIMHI@geom_colltype_explosion?$AA@ 320baa94     ScriptBind_Entity.obj
 0002:00006aac       ??_C@_0BF@IILFDIAC@geom_colltype_player?$AA@ 320baaac     ScriptBind_Entity.obj
 0002:00006ac4       ??_C@_0P@GBBJCMGE@geom_colltype0?$AA@ 320baac4     ScriptBind_Entity.obj
 0002:00006ad4       ??_C@_0M@KAOHHCLE@geom_floats?$AA@ 320baad4     ScriptBind_Entity.obj
 0002:00006ae0       ??_C@_0O@GIHMIPEP@geom_collides?$AA@ 320baae0     ScriptBind_Entity.obj
 0002:00006af0       ??_C@_0BG@NBMHBAEO@geom_colltype_vehicle?$AA@ 320baaf0     ScriptBind_Entity.obj
 0002:00006b08       ??_C@_0BC@HPDIELNA@geom_colltype_ray?$AA@ 320bab08     ScriptBind_Entity.obj
 0002:00006b1c       ??_C@_0BE@ECEKOHDN@rope_subdivide_segs?$AA@ 320bab1c     ScriptBind_Entity.obj
 0002:00006b30       ??_C@_0P@OBHIIFC@rope_traceable?$AA@ 320bab30     ScriptBind_Entity.obj
 0002:00006b40       ??_C@_0O@HEHNCIKA@rope_collides?$AA@ 320bab40     ScriptBind_Entity.obj
 0002:00006b50       ??_C@_0BO@ONOKLALC@pef_always_notify_on_deletion?$AA@ 320bab50     ScriptBind_Entity.obj
 0002:00006b70       ??_C@_0BL@HGBOCADG@pef_override_impulse_scale?$AA@ 320bab70     ScriptBind_Entity.obj
 0002:00006b8c       ??_C@_0N@HHMOJNA@pef_disabled?$AA@ 320bab8c     ScriptBind_Entity.obj
 0002:00006b9c       ??_C@_0BE@IHAEMKOB@lef_snap_velocities?$AA@ 320bab9c     ScriptBind_Entity.obj
 0002:00006bb0       ??_C@_0BD@FGJKILMK@particle_traceable?$AA@ 320babb0     ScriptBind_Entity.obj
 0002:00006bc4       ??_C@_0BG@CKNCBAFM@ref_use_simple_solver?$AA@ 320babc4     ScriptBind_Entity.obj
 0002:00006bdc       ??_C@_0BA@NEBPGIFP@pef_never_break?$AA@ 320babdc     ScriptBind_Entity.obj
 0002:00006bec       ??_C@_0O@EIDFNGOM@pef_traceable?$AA@ 320babec     ScriptBind_Entity.obj
 0002:00006bfc       ??_C@_0BB@KCKHBIME@particle_no_spin?$AA@ 320babfc     ScriptBind_Entity.obj
 0002:00006c10       ??_C@_0BL@FIBJMLJP@particle_no_path_alignment?$AA@ 320bac10     ScriptBind_Entity.obj
 0002:00006c2c       ??_C@_0BB@KDEANGNE@particle_no_roll?$AA@ 320bac2c     ScriptBind_Entity.obj
 0002:00006c40       ??_C@_0BO@BOJPEIGG@particle_constant_orientation?$AA@ 320bac40     ScriptBind_Entity.obj
 0002:00006c60       ??_C@_0BI@HPBJGFDF@particle_single_contact?$AA@ 320bac60     ScriptBind_Entity.obj
 0002:00006c78       ??_C@_0BB@EBLIDDN@lef_push_players?$AA@ 320bac78     ScriptBind_Entity.obj
 0002:00006c8c       ??_C@_0BB@BPIOHCMJ@lef_push_objects?$AA@ 320bac8c     ScriptBind_Entity.obj
 0002:00006ca0       ??_C@_0BB@GFIDPGLJ@pef_ignore_areas?$AA@ 320baca0     ScriptBind_Entity.obj
 0002:00006cb4       ??_C@_0BC@PHFOJJNI@pef_fixed_damping?$AA@ 320bacb4     ScriptBind_Entity.obj
 0002:00006cc8       ??_C@_0BK@DCDNHJPG@pef_never_affect_triggers?$AA@ 320bacc8     ScriptBind_Entity.obj
 0002:00006ce4       ??_C@_0BK@HDJCOBMA@pef_monitor_state_changes?$AA@ 320bace4     ScriptBind_Entity.obj
 0002:00006d00       ??_C@_0BK@ENNLBNI@pef_cannot_squash_players?$AA@ 320bad00     ScriptBind_Entity.obj
 0002:00006d1c       ??_C@_0BI@DKMECAFN@pef_pushable_by_players?$AA@ 320bad1c     ScriptBind_Entity.obj
 0002:00006d34       ??_C@_0BM@BALBPMMC@PHYSICPARAM_AUTO_DETACHMENT?$AA@ 320bad34     ScriptBind_Entity.obj
 0002:00006d50       ??_C@_0BI@LNINLOPJ@PHYSICPARAM_FOREIGNDATA?$AA@ 320bad50     ScriptBind_Entity.obj
 0002:00006d68       ??_C@_0BJ@GDDENIAJ@PHYSICPARAM_GROUND_PLANE?$AA@ 320bad68     ScriptBind_Entity.obj
 0002:00006d84       ??_C@_0BM@PPCGLAKE@PHYSICPARAM_SUPPORT_LATTICE?$AA@ 320bad84     ScriptBind_Entity.obj
 0002:00006da0       ??_C@_0BH@BAIMKIAO@PHYSICPARAM_PART_FLAGS?$AA@ 320bada0     ScriptBind_Entity.obj
 0002:00006db8       ??_C@_0BF@ENNFAPKK@PHYSICPARAM_VELOCITY?$AA@ 320badb8     ScriptBind_Entity.obj
 0002:00006dd0       ??_C@_0BG@MAHJGFOJ@PHYSICPARAM_PLAYERDIM?$AA@ 320badd0     ScriptBind_Entity.obj
 0002:00006de8       ??_C@_0BG@PHHCJFFK@PHYSICPARAM_PLAYERDYN?$AA@ 320bade8     ScriptBind_Entity.obj
 0002:00006e00       ??_C@_0BO@BBPPPALD@PHYSICPARAM_REMOVE_CONSTRAINT?$AA@ 320bae00     ScriptBind_Entity.obj
 0002:00006e20       ??_C@_0BH@JOJENHGK@PHYSICPARAM_CONSTRAINT?$AA@ 320bae20     ScriptBind_Entity.obj
 0002:00006e38       ??_C@_0BF@NKFLAIML@PHYSICPARAM_BUOYANCY?$AA@ 320bae38     ScriptBind_Entity.obj
 0002:00006e50       ??_C@_0BF@FPMOCOCH@PHYSICPARAM_SOFTBODY?$AA@ 320bae50     ScriptBind_Entity.obj
 0002:00006e68       ??_C@_0BB@PHEJINLE@PHYSICPARAM_ROPE?$AA@ 320bae68     ScriptBind_Entity.obj
 0002:00006e7c       ??_C@_0BC@NMONNBEK@PHYSICPARAM_JOINT?$AA@ 320bae7c     ScriptBind_Entity.obj
 0002:00006e90       ??_C@_0BI@KEKAHIBC@PHYSICPARAM_ARTICULATED?$AA@ 320bae90     ScriptBind_Entity.obj
 0002:00006ea8       ??_C@_0BH@KACHMCG@PHYSICPARAM_SIMULATION?$AA@ 320baea8     ScriptBind_Entity.obj
 0002:00006ec0       ??_C@_0BC@BFBNNEBP@PHYSICPARAM_WHEEL?$AA@ 320baec0     ScriptBind_Entity.obj
 0002:00006ed4       ??_C@_0BE@DEBKENHN@PHYSICPARAM_VEHICLE?$AA@ 320baed4     ScriptBind_Entity.obj
 0002:00006ee8       ??_C@_0BF@DFDKDKEB@PHYSICPARAM_PARTICLE?$AA@ 320baee8     ScriptBind_Entity.obj
 0002:00006f00       ??_C@_0BM@PGDINMMM@PHYSICPARAM_COLLISION_CLASS?$AA@ 320baf00     ScriptBind_Entity.obj
 0002:00006f1c       ??_C@_0BC@GJKLOOEG@PHYSICPARAM_FLAGS?$AA@ 320baf1c     ScriptBind_Entity.obj
 0002:00006f30       ??_C@_0BA@PBHLELGJ@MTL_LAYER_CLOAK?$AA@ 320baf30     ScriptBind_Entity.obj
 0002:00006f40       ??_C@_0O@NLHHNMDJ@MTL_LAYER_WET?$AA@ 320baf40     ScriptBind_Entity.obj
 0002:00006f50       ??_C@_0BB@LMAHHBOE@MTL_LAYER_FROZEN?$AA@ 320baf50     ScriptBind_Entity.obj
 0002:00006f64       ??_C@_0M@GMJFPFEA@NULL_ENTITY?$AA@ 320baf64     ScriptBind_Entity.obj
 0002:00006f70       ??_C@_0N@GGGLDOCO@UnSeenFrames?$AA@ 320baf70     ScriptBind_Entity.obj
 0002:00006f80       ??_C@_0BC@EPJNEJLI@CreateCameraProxy?$AA@ 320baf80     ScriptBind_Entity.obj
 0002:00006f94       ??_C@_0P@OOHIBEDE@ActivateOutput?$AA@ 320baf94     ScriptBind_Entity.obj
 0002:00006fa4       ??_C@_0BG@NFEGBHBH@ProcessBroadcastEvent?$AA@ 320bafa4     ScriptBind_Entity.obj
 0002:00006fbc       ??_C@_0BE@GBJNIBL@AttachSurfaceEffect?$AA@ 320bafbc     ScriptBind_Entity.obj
 0002:00006fd0       ??_C@_0DP@OIDAEGAG@nSlot?0?5effect?0?5countPerUnit?0?5for@ 320bafd0     ScriptBind_Entity.obj
 0002:00007010       ??_C@_0O@EEIDEHKK@BreakToPieces?$AA@ 320bb010     ScriptBind_Entity.obj
 0002:00007020       ??_C@_0EE@BHJLPEPI@nSlot?0?5nPiecesSlot?0?5fExplodeImp?0@ 320bb020     ScriptBind_Entity.obj
 0002:00007064       ??_C@_0BD@JNECHFDP@IsEntityInsideArea?$AA@ 320bb064     ScriptBind_Entity.obj
 0002:00007078       ??_C@_0BB@KIJPCOIL@areaId?0?5entityId?$AA@ 320bb078     ScriptBind_Entity.obj
 0002:0000708c       ??_C@_0BC@BHEHHECL@IsPointInsideArea?$AA@ 320bb08c     ScriptBind_Entity.obj
 0002:000070a0       ??_C@_0O@JJKFMOAD@areaId?0?5point?$AA@ 320bb0a0     ScriptBind_Entity.obj
 0002:000070b0       ??_C@_0O@HOCGLLDE@NoBulletForce?$AA@ 320bb0b0     ScriptBind_Entity.obj
 0002:000070c0       ??_C@_05HDBKIDE@state?$AA@ 320bb0c0     ScriptBind_Entity.obj
 0002:000070c8       ??_C@_0BB@GDFHOHHM@GetPhysicalStats?$AA@ 320bb0c8     ScriptBind_Entity.obj
 0002:000070dc       ??_C@_0BF@JOMPGJHB@NoExplosionCollision?$AA@ 320bb0dc     ScriptBind_Entity.obj
 0002:000070f4       ??_C@_0BD@HCDBCDML@SetStateClientside?$AA@ 320bb0f4     ScriptBind_Entity.obj
 0002:00007108       ??_C@_0BB@IBFDDNDL@AwakeEnvironment?$AA@ 320bb108     ScriptBind_Entity.obj
 0002:0000711c       ??_C@_0BA@LDDEPGM@CheckCollisions?$AA@ 320bb11c     ScriptBind_Entity.obj
 0002:0000712c       ??_C@_04EACEFPPN@Hide?$AA@ 320bb12c     ScriptBind_Entity.obj
 0002:00007134       ??_C@_0BI@JJPNBDDB@CharacterUpdateOnRender?$AA@ 320bb134     ScriptBind_Entity.obj
 0002:0000714c       ??_C@_0BP@NBOCNDOI@characterSlot?0?5bUpdateOnRender?$AA@ 320bb14c     ScriptBind_Entity.obj
 0002:0000716c       ??_C@_0BG@CMLIBLKF@CharacterUpdateAlways?$AA@ 320bb16c     ScriptBind_Entity.obj
 0002:00007184       ??_C@_0BF@ILMMOFBK@ForceCharacterUpdate?$AA@ 320bb184     ScriptBind_Entity.obj
 0002:0000719c       ??_C@_0BM@OOFMKKIE@characterSlot?0?5alwaysUpdate?$AA@ 320bb19c     ScriptBind_Entity.obj
 0002:000071b8       ??_C@_0N@HPECPAA@EnableDecals?$AA@ 320bb1b8     ScriptBind_Entity.obj
 0002:000071c8       ??_C@_0N@PMJKBNPI@slot?0?5enable?$AA@ 320bb1c8     ScriptBind_Entity.obj
 0002:000071d8       ??_C@_0N@HJBIPKBE@RemoveDecals?$AA@ 320bb1d8     ScriptBind_Entity.obj
 0002:000071e8       ??_C@_0M@PLFAMDAL@SetLodRatio?$AA@ 320bb1e8     ScriptBind_Entity.obj
 0002:000071f4       ??_C@_0M@PEEOBFII@GetLodRatio?$AA@ 320bb1f4     ScriptBind_Entity.obj
 0002:00007200       ??_C@_0BF@KMLOEFJP@SetViewDistUnlimited?$AA@ 320bb200     ScriptBind_Entity.obj
 0002:00007218       ??_C@_0BB@CIKBPPIH@SetViewDistRatio?$AA@ 320bb218     ScriptBind_Entity.obj
 0002:0000722c       ??_C@_0BB@EMPIEBDF@GetViewDistRatio?$AA@ 320bb22c     ScriptBind_Entity.obj
 0002:00007240       ??_C@_0BF@DINIPHGE@GetTimeSinceLastSeen?$AA@ 320bb240     ScriptBind_Entity.obj
 0002:00007258       ??_C@_0L@OLJNPPME@CountLinks?$AA@ 320bb258     ScriptBind_Entity.obj
 0002:00007264       ??_C@_0M@GMJEEKAK@GetLinkName?$AA@ 320bb264     ScriptBind_Entity.obj
 0002:00007270       ??_C@_08NKLPAFH@targetId?$AA@ 320bb270     ScriptBind_Entity.obj
 0002:0000727c       ??_C@_07OPNFJOHA@GetLink?$AA@ 320bb27c     ScriptBind_Entity.obj
 0002:00007284       ??_C@_0P@EBGHIDOM@RemoveAllLinks?$AA@ 320bb284     ScriptBind_Entity.obj
 0002:00007294       ??_C@_0L@OPGPBDFJ@RemoveLink?$AA@ 320bb294     ScriptBind_Entity.obj
 0002:000072a0       ??_C@_0O@OCLOJCPB@GetLinkTarget?$AA@ 320bb2a0     ScriptBind_Entity.obj
 0002:000072b0       ??_C@_0O@JNKACBIG@SetLinkTarget?$AA@ 320bb2b0     ScriptBind_Entity.obj
 0002:000072c0       ??_C@_0P@LIBLGLCP@name?0?5targetId?$AA@ 320bb2c0     ScriptBind_Entity.obj
 0002:000072d0       ??_C@_0L@HMKIDDMA@CreateLink?$AA@ 320bb2d0     ScriptBind_Entity.obj
 0002:000072dc       ??_C@_0BD@EALKBBBF@GetSubmergedVolume?$AA@ 320bb2dc     ScriptBind_Entity.obj
 0002:000072f0       ??_C@_0BP@OJFEEHNC@slot?0?5planeNormal?0?5planeOrigin?$AA@ 320bb2f0     ScriptBind_Entity.obj
 0002:00007310       ??_C@_0L@PHDEGGEO@GetGravity?$AA@ 320bb310     ScriptBind_Entity.obj
 0002:0000731c       ??_C@_09LPPMLMKA@GetVolume?$AA@ 320bb31c     ScriptBind_Entity.obj
 0002:00007328       ??_C@_07IBOEDHFF@GetMass?$AA@ 320bb328     ScriptBind_Entity.obj
 0002:00007330       ??_C@_0O@ELJALOGK@SetVelocityEx?$AA@ 320bb330     ScriptBind_Entity.obj
 0002:00007340       ??_C@_0BK@CMCNKLH@velocity?0?5angularVelocity?$AA@ 320bb340     ScriptBind_Entity.obj
 0002:0000735c       ??_C@_0M@IKABEOO@SetVelocity?$AA@ 320bb35c     ScriptBind_Entity.obj
 0002:00007368       ??_C@_0O@DEIOANBN@GetVelocityEx?$AA@ 320bb368     ScriptBind_Entity.obj
 0002:00007378       ??_C@_0M@HLOMCGN@GetVelocity?$AA@ 320bb378     ScriptBind_Entity.obj
 0002:00007384       ??_C@_0BJ@DLJDHJGJ@SetDefaultIdleAnimations?$AA@ 320bb384     ScriptBind_Entity.obj
 0002:000073a0       ??_C@_0P@PLCLGKMP@VectorToGlobal?$AA@ 320bb3a0     ScriptBind_Entity.obj
 0002:000073b0       ??_C@_0O@GLHLHCJD@VectorToLocal?$AA@ 320bb3b0     ScriptBind_Entity.obj
 0002:000073c0       ??_C@_09PFFEPMEL@slot?0?5dir?$AA@ 320bb3c0     ScriptBind_Entity.obj
 0002:000073cc       ??_C@_08MLAJJHEC@ToGlobal?$AA@ 320bb3cc     ScriptBind_Entity.obj
 0002:000073d8       ??_C@_07PMHJBGHM@ToLocal?$AA@ 320bb3d8     ScriptBind_Entity.obj
 0002:000073e0       ??_C@_0BE@LJBLANKD@EnableMaterialLayer?$AA@ 320bb3e0     ScriptBind_Entity.obj
 0002:000073f4       ??_C@_0O@ELGNLMOJ@enable?0?5layer?$AA@ 320bb3f4     ScriptBind_Entity.obj
 0002:00007404       ??_C@_0BE@LIFAMDEL@MaterialFlashInvoke?$AA@ 320bb404     ScriptBind_Entity.obj
 0002:00007418       ??_C@_0BA@DEINLHEE@GetMaterialVec3?$AA@ 320bb418     ScriptBind_Entity.obj
 0002:00007428       ??_C@_0BA@GJLMFFN@SetMaterialVec3?$AA@ 320bb428     ScriptBind_Entity.obj
 0002:00007438       ??_C@_0CD@JFHHHCHH@nSlot?0nSubMtlId?0sParamName?0vVect@ 320bb438     ScriptBind_Entity.obj
 0002:0000745c       ??_C@_0BB@BBPOJBEA@GetMaterialFloat?$AA@ 320bb45c     ScriptBind_Entity.obj
 0002:00007470       ??_C@_0BL@FKADBBDM@nSlot?0nSubMtlId?0sParamName?$AA@ 320bb470     ScriptBind_Entity.obj
 0002:0000748c       ??_C@_0BB@HFKHCPPC@SetMaterialFloat?$AA@ 320bb48c     ScriptBind_Entity.obj
 0002:000074a0       ??_C@_0CC@EHCDENDN@nSlot?0nSubMtlId?0sParamName?0fValu@ 320bb4a0     ScriptBind_Entity.obj
 0002:000074c4       ??_C@_0O@NOJMBGPK@CloneMaterial?$AA@ 320bb4c4     ScriptBind_Entity.obj
 0002:000074d4       ??_C@_0O@EAOLAMOH@ResetMaterial?$AA@ 320bb4d4     ScriptBind_Entity.obj
 0002:000074e4       ??_C@_0BA@CIMOMNHB@ReplaceMaterial?$AA@ 320bb4e4     ScriptBind_Entity.obj
 0002:000074f4       ??_C@_0BI@MPMIFIGM@slot?0?5name?0?5replacement?$AA@ 320bb4f4     ScriptBind_Entity.obj
 0002:0000750c       ??_C@_0BC@EMJDHOGD@GetEntityMaterial?$AA@ 320bb50c     ScriptBind_Entity.obj
 0002:00007520       ??_C@_0M@CIBDNIEJ@GetMaterial?$AA@ 320bb520     ScriptBind_Entity.obj
 0002:0000752c       ??_C@_0M@CHANAOMK@SetMaterial?$AA@ 320bb52c     ScriptBind_Entity.obj
 0002:00007538       ??_C@_0BE@CKFEDBGN@GetExplosionImpulse?$AA@ 320bb538     ScriptBind_Entity.obj
 0002:0000754c       ??_C@_0BI@EHDBMOBF@GetExplosionObstruction?$AA@ 320bb54c     ScriptBind_Entity.obj
 0002:00007564       ??_C@_08BDJEOFLH@GetSpeed?$AA@ 320bb564     ScriptBind_Entity.obj
 0002:00007570       ??_C@_06KGFFMMMJ@Damage?$AA@ 320bb570     ScriptBind_Entity.obj
 0002:00007578       ??_C@_08HMJDFDMJ@IsHidden?$AA@ 320bb578     ScriptBind_Entity.obj
 0002:00007584       ??_C@_08GNIJCMCG@GetState?$AA@ 320bb584     ScriptBind_Entity.obj
 0002:00007590       ??_C@_09BEAPFJND@IsInState?$AA@ 320bb590     ScriptBind_Entity.obj
 0002:0000759c       ??_C@_09PIINJFBN@GotoState?$AA@ 320bb59c     ScriptBind_Entity.obj
 0002:000075a8       ??_C@_06PBLDBJGJ@sState?$AA@ 320bb5a8     ScriptBind_Entity.obj
 0002:000075b0       ??_C@_0BG@EAAFGOAL@PhysicalizeAttachment?$AA@ 320bb5b0     ScriptBind_Entity.obj
 0002:000075c8       ??_C@_0CL@MEOEEOJP@characterSlot?0?5attachmentName?0?5p@ 320bb5c8     ScriptBind_Entity.obj
 0002:000075f4       ??_C@_0BF@BHNMNHNG@HideAttachmentMaster?$AA@ 320bb5f4     ScriptBind_Entity.obj
 0002:0000760c       ??_C@_0BE@HAHBKHOM@characterSlot?0?5hide?$AA@ 320bb60c     ScriptBind_Entity.obj
 0002:00007620       ??_C@_0BD@KCBDKLOF@HideAllAttachments?$AA@ 320bb620     ScriptBind_Entity.obj
 0002:00007634       ??_C@_0CA@NGBMOAAP@characterSlot?0?5hide?0?5hideShadow?$AA@ 320bb634     ScriptBind_Entity.obj
 0002:00007654       ??_C@_0P@BCLNHEDA@HideAttachment?$AA@ 320bb654     ScriptBind_Entity.obj
 0002:00007664       ??_C@_0DA@GCMNBOGB@characterSlot?0?5attachmentName?0?5h@ 320bb664     ScriptBind_Entity.obj
 0002:00007694       ??_C@_0BB@MPJGPDIE@SetAttachmentDir?$AA@ 320bb694     ScriptBind_Entity.obj
 0002:000076a8       ??_C@_0CP@JPEMBFCM@characterSlot?0?5attachmentName?0?5d@ 320bb6a8     ScriptBind_Entity.obj
 0002:000076d8       ??_C@_0BE@BMACFLDE@SetAttachmentAngles?$AA@ 320bb6d8     ScriptBind_Entity.obj
 0002:000076ec       ??_C@_0CG@NPLHANBJ@characterSlot?0?5attachmentName?0?5a@ 320bb6ec     ScriptBind_Entity.obj
 0002:00007714       ??_C@_0BB@NHLHOLP@SetAttachmentPos?$AA@ 320bb714     ScriptBind_Entity.obj
 0002:00007728       ??_C@_0CD@FOJPBIMN@characterSlot?0?5attachmentName?0?5p@ 320bb728     ScriptBind_Entity.obj
 0002:0000774c       ??_C@_0BD@PNFIDCNF@SetAttachmentLight?$AA@ 320bb74c     ScriptBind_Entity.obj
 0002:00007760       ??_C@_0DB@PAPDIOJN@characterSlot?0?5attachmentName?0?5l@ 320bb760     ScriptBind_Entity.obj
 0002:00007794       ??_C@_0BB@NLLIFDCA@SetAttachmentCGF?$AA@ 320bb794     ScriptBind_Entity.obj
 0002:000077a8       ??_C@_0CI@MDBAOCDB@characterSlot?0?5attachmentName?0?5f@ 320bb7a8     ScriptBind_Entity.obj
 0002:000077d0       ??_C@_0BE@PFKLIBFM@SetAttachmentObject?$AA@ 320bb7d0     ScriptBind_Entity.obj
 0002:000077e4       ??_C@_0DF@GNDBOOHA@characterSlot?0?5attachmentName?0?5e@ 320bb7e4     ScriptBind_Entity.obj
 0002:0000781c       ??_C@_0BE@PLKHBAF@SetAttachmentEffect?$AA@ 320bb81c     ScriptBind_Entity.obj
 0002:00007830       ??_C@_0EF@PNHDIDEJ@characterSlot?0?5attachmentName?0?5e@ 320bb830     ScriptBind_Entity.obj
 0002:00007878       ??_C@_0BA@OMEJADPG@ResetAttachment?$AA@ 320bb878     ScriptBind_Entity.obj
 0002:00007888       ??_C@_0BB@LPOBONJC@GetAttachmentCGF?$AA@ 320bb888     ScriptBind_Entity.obj
 0002:0000789c       ??_C@_0BC@GIIMDFFO@GetAttachmentBone?$AA@ 320bb89c     ScriptBind_Entity.obj
 0002:000078b0       ??_C@_0BC@CMLGLDPP@DestroyAttachment?$AA@ 320bb8b0     ScriptBind_Entity.obj
 0002:000078c4       ??_C@_0BF@EKOELJIM@CreateSkinAttachment?$AA@ 320bb8c4     ScriptBind_Entity.obj
 0002:000078dc       ??_C@_0BO@HIHFDACD@characterSlot?0?5attachmentName?$AA@ 320bb8dc     ScriptBind_Entity.obj
 0002:000078fc       ??_C@_0BF@KCDANAGG@CreateBoneAttachment?$AA@ 320bb8fc     ScriptBind_Entity.obj
 0002:00007918       ??_C@_0EH@IJEGBAMC@characterSlot?0?5boneName?0?5attachm@ 320bb918     ScriptBind_Entity.obj
 0002:00007960       ??_C@_0BA@DMHIHNOA@GetTouchedPoint?$AA@ 320bb960     ScriptBind_Entity.obj
 0002:00007970       ??_C@_0BE@OIBHIAHO@GetTouchedSurfaceID?$AA@ 320bb970     ScriptBind_Entity.obj
 0002:00007984       ??_C@_0BF@EPNGPBPF@GetBoneNameFromTable?$AA@ 320bb984     ScriptBind_Entity.obj
 0002:0000799c       ??_C@_0BH@FFKIIOOB@GetBoneAngularVelocity?$AA@ 320bb99c     ScriptBind_Entity.obj
 0002:000079b4       ??_C@_0BA@OJIMGCJK@GetBoneVelocity?$AA@ 320bb9b4     ScriptBind_Entity.obj
 0002:000079c4       ??_C@_0BI@ONFCOBGG@characterSlot?0?5boneName?$AA@ 320bb9c4     ScriptBind_Entity.obj
 0002:000079dc       ??_C@_0L@MKJJFEKI@GetBoneDir?$AA@ 320bb9dc     ScriptBind_Entity.obj
 0002:000079e8       ??_C@_0L@IHENJJD@GetBonePos?$AA@ 320bb9e8     ScriptBind_Entity.obj
 0002:000079f4       ??_C@_0BF@BFMEFKMJ@SetSoundEffectRadius?$AA@ 320bb9f4     ScriptBind_Entity.obj
 0002:00007a0c       ??_C@_0O@PEJLNFFI@fEffectRadius?$AA@ 320bba0c     ScriptBind_Entity.obj
 0002:00007a1c       ??_C@_0L@BNMHANDA@PauseSound?$AA@ 320bba1c     ScriptBind_Entity.obj
 0002:00007a28       ??_C@_0BA@KCEPHGHB@nSoundId?0bPause?$AA@ 320bba28     ScriptBind_Entity.obj
 0002:00007a38       ??_C@_0O@KNHEJMNP@StopAllSounds?$AA@ 320bba38     ScriptBind_Entity.obj
 0002:00007a48       ??_C@_09IIPLNIMF@StopSound?$AA@ 320bba48     ScriptBind_Entity.obj
 0002:00007a54       ??_C@_0P@KIDELOBF@SetStaticSound?$AA@ 320bba54     ScriptBind_Entity.obj
 0002:00007a64       ??_C@_0P@KKOCENGO@soundId?0static?$AA@ 320bba64     ScriptBind_Entity.obj
 0002:00007a74       ??_C@_0BD@NFOHEJFE@SetSoundSphereSpec?$AA@ 320bba74     ScriptBind_Entity.obj
 0002:00007a88       ??_C@_0BA@GOIAANHI@soundId?0?5radius?$AA@ 320bba88     ScriptBind_Entity.obj
 0002:00007a98       ??_C@_0BB@BHNODJNF@PlaySoundEventEx?$AA@ 320bba98     ScriptBind_Entity.obj
 0002:00007ab0       ??_C@_0EP@FKIGOKGK@sSoundOrEventName?0nSoundFlags?0nV@ 320bbab0     ScriptBind_Entity.obj
 0002:00007b00       ??_C@_0P@IHOCNFPE@PlaySoundEvent?$AA@ 320bbb00     ScriptBind_Entity.obj
 0002:00007b10       ??_C@_0DK@FPLDCDKN@sSoundOrEventName?0?5vOffset?0?5vDir@ 320bbb10     ScriptBind_Entity.obj
 0002:00007b4c       ??_C@_09PEMGNEEO@PlaySound?$AA@ 320bbb4c     ScriptBind_Entity.obj
 0002:00007b58       ??_C@_0BB@DLAJHDPE@SetAnimationFlip?$AA@ 320bbb58     ScriptBind_Entity.obj
 0002:00007b6c       ??_C@_0BE@MHPCJMPI@characterSlot?0?5flip?$AA@ 320bbb6c     ScriptBind_Entity.obj
 0002:00007b80       ??_C@_0BD@EBLLJFEN@GetAnimationLength?$AA@ 320bbb80     ScriptBind_Entity.obj
 0002:00007b94       ??_C@_0BJ@EGCLIFAL@characterSlot?0?5animation?$AA@ 320bbb94     ScriptBind_Entity.obj
 0002:00007bb0       ??_C@_0BE@CNNNIIGB@SetScriptUpdateRate?$AA@ 320bbbb0     ScriptBind_Entity.obj
 0002:00007bc4       ??_C@_0O@LJOLINID@nMilliseconds?$AA@ 320bbbc4     ScriptBind_Entity.obj
 0002:00007bd4       ??_C@_09NINJKNPI@KillTimer?$AA@ 320bbbd4     ScriptBind_Entity.obj
 0002:00007be0       ??_C@_08ELGBKOLJ@SetTimer?$AA@ 320bbbe0     ScriptBind_Entity.obj
 0002:00007bec       ??_C@_0BA@KJGENFPA@GetCurAnimation?$AA@ 320bbbec     ScriptBind_Entity.obj
 0002:00007bfc       ??_C@_0M@OLKJABCF@IsUsingPipe?$AA@ 320bbbfc     ScriptBind_Entity.obj
 0002:00007c08       ??_C@_0BB@NLJKFLKH@PassParamsToPipe?$AA@ 320bbc08     ScriptBind_Entity.obj
 0002:00007c1c       ??_C@_0O@JGHHKPGO@CancelSubpipe?$AA@ 320bbc1c     ScriptBind_Entity.obj
 0002:00007c2c       ??_C@_0O@MLFIPMGJ@InsertSubpipe?$AA@ 320bbc2c     ScriptBind_Entity.obj
 0002:00007c3c       ??_C@_0L@HIBNHPDC@SelectPipe?$AA@ 320bbc3c     ScriptBind_Entity.obj
 0002:00007c48       ??_C@_0BC@BNEKKGFN@SetAnimationSpeed?$AA@ 320bbc48     ScriptBind_Entity.obj
 0002:00007c5c       ??_C@_0BM@EECIOMOO@characterSlot?0?5layer?0?5speed?$AA@ 320bbc5c     ScriptBind_Entity.obj
 0002:00007c78       ??_C@_0BG@OIIFBGON@DisableAnimationEvent?$AA@ 320bbc78     ScriptBind_Entity.obj
 0002:00007c90       ??_C@_0BF@JBGDLLLO@SetAnimationKeyEvent?$AA@ 320bbc90     ScriptBind_Entity.obj
 0002:00007ca8       ??_C@_0BB@ECBCLHFO@GetAnimationTime?$AA@ 320bbca8     ScriptBind_Entity.obj
 0002:00007cbc       ??_C@_0N@HEKMAHFG@nSlot?0nLayer?$AA@ 320bbcbc     ScriptBind_Entity.obj
 0002:00007ccc       ??_C@_0BB@CGELAJOM@SetAnimationTime?$AA@ 320bbccc     ScriptBind_Entity.obj
 0002:00007ce0       ??_C@_0BD@DJDKPIHH@nSlot?0nLayer?0fTime?$AA@ 320bbce0     ScriptBind_Entity.obj
 0002:00007cf4       ??_C@_0BC@BBCEPML@SetAnimationEvent?$AA@ 320bbcf4     ScriptBind_Entity.obj
 0002:00007d08       ??_C@_0BB@MJEJPGFN@nSlot?0sAnimation?$AA@ 320bbd08     ScriptBind_Entity.obj
 0002:00007d1c       ??_C@_0P@JMOGOAEN@SetPublicParam?$AA@ 320bbd1c     ScriptBind_Entity.obj
 0002:00007d2c       ??_C@_0BA@NPNLHNFF@SetUpdatePolicy?$AA@ 320bbd2c     ScriptBind_Entity.obj
 0002:00007d3c       ??_C@_0O@MGHGCOMO@nUpdatePolicy?$AA@ 320bbd3c     ScriptBind_Entity.obj
 0002:00007d4c       ??_C@_0L@HPPPBLCC@IsFromPool?$AA@ 320bbd4c     ScriptBind_Entity.obj
 0002:00007d58       ??_C@_08CHIOLOMB@IsActive?$AA@ 320bbd58     ScriptBind_Entity.obj
 0002:00007d64       ??_C@_08HNNCLIA@Activate?$AA@ 320bbd64     ScriptBind_Entity.obj
 0002:00007d70       ??_C@_07GGIFPBOP@bActive?$AA@ 320bbd70     ScriptBind_Entity.obj
 0002:00007d78       ??_C@_0BA@JCGMADJM@GetUpdateRadius?$AA@ 320bbd78     ScriptBind_Entity.obj
 0002:00007d88       ??_C@_0BA@KAHKHBIF@SetUpdateRadius?$AA@ 320bbd88     ScriptBind_Entity.obj
 0002:00007d98       ??_C@_0BH@OMKKMIGP@ForwardTriggerEventsTo?$AA@ 320bbd98     ScriptBind_Entity.obj
 0002:00007db0       ??_C@_0BC@LIBJJGJB@InvalidateTrigger?$AA@ 320bbdb0     ScriptBind_Entity.obj
 0002:00007dc4       ??_C@_0P@HFCPLEOJ@GetTriggerBBox?$AA@ 320bbdc4     ScriptBind_Entity.obj
 0002:00007dd4       ??_C@_0P@LLDBEOMF@SetTriggerBBox?$AA@ 320bbdd4     ScriptBind_Entity.obj
 0002:00007de4       ??_C@_0BG@IIOEAEEO@GetProjectedWorldBBox?$AA@ 320bbde4     ScriptBind_Entity.obj
 0002:00007dfc       ??_C@_0N@JACINOOP@GetWorldBBox?$AA@ 320bbdfc     ScriptBind_Entity.obj
 0002:00007e0c       ??_C@_0N@HCPDHGOI@GetLocalBBox?$AA@ 320bbe0c     ScriptBind_Entity.obj
 0002:00007e1c       ??_C@_0N@GENLKKE@SetLocalBBox?$AA@ 320bbe1c     ScriptBind_Entity.obj
 0002:00007e2c       ??_C@_07JOGNENNC@min?0max?$AA@ 320bbe2c     ScriptBind_Entity.obj
 0002:00007e34       ??_C@_0N@BOHABMKM@TriggerEvent?$AA@ 320bbe34     ScriptBind_Entity.obj
 0002:00007e44       ??_C@_0O@HLHPHPAI@AddConstraint?$AA@ 320bbe44     ScriptBind_Entity.obj
 0002:00007e54       ??_C@_0L@IDFDGLFD@AddImpulse?$AA@ 320bbe54     ScriptBind_Entity.obj
 0002:00007e60       ??_C@_0BD@KBJDGNPO@IsAnimationRunning?$AA@ 320bbe60     ScriptBind_Entity.obj
 0002:00007e74       ??_C@_0BD@BMLHHCNA@SetDirectionVector?$AA@ 320bbe74     ScriptBind_Entity.obj
 0002:00007e88       ??_C@_0BA@OPKMMGKP@direction?0?5?$FLup?$FN?$AA@ 320bbe88     ScriptBind_Entity.obj
 0002:00007e98       ??_C@_0BD@OGJNEEDI@GetDirectionVector?$AA@ 320bbe98     ScriptBind_Entity.obj
 0002:00007eac       ??_C@_0M@BOLHMNGM@IsColliding?$AA@ 320bbeac     ScriptBind_Entity.obj
 0002:00007eb8       ??_C@_0BF@LFEIGLGD@SetRegisterInSectors?$AA@ 320bbeb8     ScriptBind_Entity.obj
 0002:00007ed0       ??_C@_0N@MOPKEIPF@RenderShadow?$AA@ 320bbed0     ScriptBind_Entity.obj
 0002:00007ee0       ??_C@_0BB@PIOIMFOE@GetSlotHelperPos?$AA@ 320bbee0     ScriptBind_Entity.obj
 0002:00007ef4       ??_C@_0BO@GNOFJMFI@slot?0?5helperName?0?5objectSpace?$AA@ 320bbef4     ScriptBind_Entity.obj
 0002:00007f14       ??_C@_0BA@IBKOCHFD@GetHelperAngles?$AA@ 320bbf14     ScriptBind_Entity.obj
 0002:00007f24       ??_C@_0N@KLJIPLHA@GetHelperDir?$AA@ 320bbf24     ScriptBind_Entity.obj
 0002:00007f34       ??_C@_0N@GJHFHGEL@GetHelperPos?$AA@ 320bbf34     ScriptBind_Entity.obj
 0002:00007f44       ??_C@_0BE@EEDOMGJM@PlayFacialAnimation?$AA@ 320bbf44     ScriptBind_Entity.obj
 0002:00007f58       ??_C@_0O@COJIBOFA@name?0?5looping?$AA@ 320bbf58     ScriptBind_Entity.obj
 0002:00007f68       ??_C@_0CA@NGCGANPC@EnableProceduralFacialAnimation?$AA@ 320bbf68     ScriptBind_Entity.obj
 0002:00007f88       ??_C@_0BH@DFCPCHDE@EnableBoneAnimationAll?$AA@ 320bbf88     ScriptBind_Entity.obj
 0002:00007fa0       ??_C@_0BN@EOKHNKP@characterSlot?0?5layer?0?5enable?$AA@ 320bbfa0     ScriptBind_Entity.obj
 0002:00007fc0       ??_C@_0BE@MJLKHFIF@EnableBoneAnimation?$AA@ 320bbfc0     ScriptBind_Entity.obj
 0002:00007fd4       ??_C@_0CH@GGAMOPHD@characterSlot?0?5layer?0?5boneName?0?5@ 320bbfd4     ScriptBind_Entity.obj
 0002:00007ffc       ??_C@_0BF@CKEGNCKI@SetAnimationBlendOut?$AA@ 320bbffc     ScriptBind_Entity.obj
 0002:00008014       ??_C@_0BK@JAHHBILC@RedirectAnimationToLayer0?$AA@ 320bc014     ScriptBind_Entity.obj
 0002:00008030       ??_C@_0BI@LBBEOMCA@characterSlot?0?5redirect?$AA@ 320bc030     ScriptBind_Entity.obj
 0002:00008048       ??_C@_0P@OEECKIM@ResetAnimation?$AA@ 320bc048     ScriptBind_Entity.obj
 0002:00008058       ??_C@_0O@FKLKJHLG@StopAnimation?$AA@ 320bc058     ScriptBind_Entity.obj
 0002:00008068       ??_C@_0BF@LNFHECBF@characterSlot?0?5layer?$AA@ 320bc068     ScriptBind_Entity.obj
 0002:00008080       ??_C@_0P@OANJDLJM@StartAnimation?$AA@ 320bc080     ScriptBind_Entity.obj
 0002:00008090       ??_C@_0L@EHLPEKMM@NetPresent?$AA@ 320bc090     ScriptBind_Entity.obj
 0002:0000809c       ??_C@_0BD@BBPNOFCE@EnableInheritXForm?$AA@ 320bc09c     ScriptBind_Entity.obj
 0002:000080b0       ??_C@_08FNFLPFI@GetChild?$AA@ 320bc0b0     ScriptBind_Entity.obj
 0002:000080bc       ??_C@_06KKPBBPNA@nIndex?$AA@ 320bc0bc     ScriptBind_Entity.obj
 0002:000080c4       ??_C@_0O@HMBCELHA@GetChildCount?$AA@ 320bc0c4     ScriptBind_Entity.obj
 0002:000080d4       ??_C@_09DIHAALNP@GetParent?$AA@ 320bc0d4     ScriptBind_Entity.obj
 0002:000080e0       ??_C@_09BEAEEEEM@DetachAll?$AA@ 320bc0e0     ScriptBind_Entity.obj
 0002:000080ec       ??_C@_0L@FKMFGOIE@DetachThis?$AA@ 320bc0ec     ScriptBind_Entity.obj
 0002:000080f8       ??_C@_0M@BFGMJGIB@AttachChild?$AA@ 320bc0f8     ScriptBind_Entity.obj
 0002:00008104       ??_C@_0BF@DDNENPLO@childEntityId?0?5flags?$AA@ 320bc104     ScriptBind_Entity.obj
 0002:0000811c       ??_C@_0N@DBPPCHF@IntersectRay?$AA@ 320bc11c     ScriptBind_Entity.obj
 0002:0000812c       ??_C@_0CF@PGBEFLIM@slot?0?5rayOrigin?0?5rayDir?0?5maxDist@ 320bc12c     ScriptBind_Entity.obj
 0002:00008154       ??_C@_08PCKODEBG@HasFlags?$AA@ 320bc154     ScriptBind_Entity.obj
 0002:00008160       ??_C@_08GMPKMLLD@GetFlags?$AA@ 320bc160     ScriptBind_Entity.obj
 0002:0000816c       ??_C@_08JNNGNIMO@SetFlags?$AA@ 320bc16c     ScriptBind_Entity.obj
 0002:00008178       ??_C@_0M@GHHBBPLO@flags?0?5mode?$AA@ 320bc178     ScriptBind_Entity.obj
 0002:00008184       ??_C@_09KIAKEEGH@GetAIName?$AA@ 320bc184     ScriptBind_Entity.obj
 0002:00008190       ??_C@_09IGEPGFPF@SetAIName?$AA@ 320bc190     ScriptBind_Entity.obj
 0002:0000819c       ??_C@_0N@IJEIPGLC@GetArchetype?$AA@ 320bc19c     ScriptBind_Entity.obj
 0002:000081ac       ??_C@_08EOAPKILA@GetRawId?$AA@ 320bc1ac     ScriptBind_Entity.obj
 0002:000081b8       ??_C@_07MMGEHGCI@GetName?$AA@ 320bc1b8     ScriptBind_Entity.obj
 0002:000081c0       ??_C@_07DEJFEJPJ@SetName?$AA@ 320bc1c0     ScriptBind_Entity.obj
 0002:000081c8       ??_C@_0BA@BEEMDAJC@SetColliderMode?$AA@ 320bc1c8     ScriptBind_Entity.obj
 0002:000081d8       ??_C@_0BG@JLDPKONH@ReattachSoftEntityVtx?$AA@ 320bc1d8     ScriptBind_Entity.obj
 0002:000081f0       ??_C@_0BA@KHLNHLMJ@EntityId?0?5nPart?$AA@ 320bc1f0     ScriptBind_Entity.obj
 0002:00008200       ??_C@_0BC@JBCLCIPG@UpdateSlotPhysics?$AA@ 320bc200     ScriptBind_Entity.obj
 0002:00008214       ??_C@_0BA@DEAMHFOI@PhysicalizeSlot?$AA@ 320bc214     ScriptBind_Entity.obj
 0002:00008224       ??_C@_0BE@ILEDLOPK@slot?0?5physicsParams?$AA@ 320bc224     ScriptBind_Entity.obj
 0002:00008238       ??_C@_0L@EGJCMGEO@RagDollize?$AA@ 320bc238     ScriptBind_Entity.obj
 0002:00008244       ??_C@_0BJ@OJLLDPBP@SetCharacterPhysicParams?$AA@ 320bc244     ScriptBind_Entity.obj
 0002:00008260       ??_C@_0BA@MFCGIEAA@SetPhysicParams?$AA@ 320bc260     ScriptBind_Entity.obj
 0002:00008270       ??_C@_0BG@PEBCPEPN@ActivatePlayerPhysics?$AA@ 320bc270     ScriptBind_Entity.obj
 0002:00008288       ??_C@_0O@OKGDGFG@EnablePhysics?$AA@ 320bc288     ScriptBind_Entity.obj
 0002:00008298       ??_C@_07EAOEHPHH@bEnable?$AA@ 320bc298     ScriptBind_Entity.obj
 0002:000082a0       ??_C@_0N@BJGGDLCL@AwakePhysics?$AA@ 320bc2a0     ScriptBind_Entity.obj
 0002:000082b0       ??_C@_06OJHONJGK@nAwake?$AA@ 320bc2b0     ScriptBind_Entity.obj
 0002:000082b8       ??_C@_0BG@KLLNDLIA@AwakeCharacterPhysics?$AA@ 320bc2b8     ScriptBind_Entity.obj
 0002:000082d0       ??_C@_0BL@EDAGBOOF@nSlot?0sRootBoneName?0nAwake?$AA@ 320bc2d0     ScriptBind_Entity.obj
 0002:000082ec       ??_C@_0N@KDGAJJNH@ResetPhysics?$AA@ 320bc2ec     ScriptBind_Entity.obj
 0002:000082fc       ??_C@_0P@ONIILIFF@DestroyPhysics?$AA@ 320bc2fc     ScriptBind_Entity.obj
 0002:0000830c       ??_C@_0M@HMGGCEBF@Physicalize?$AA@ 320bc30c     ScriptBind_Entity.obj
 0002:00008318       ??_C@_0CC@MFNCGAKL@nSlot?0nPhysicsType?0tPhysicsParam@ 320bc318     ScriptBind_Entity.obj
 0002:0000833c       ??_C@_0N@NDBDHEPG@FreeAllSlots?$AA@ 320bc33c     ScriptBind_Entity.obj
 0002:0000834c       ??_C@_08NNCHDHNF@FreeSlot?$AA@ 320bc34c     ScriptBind_Entity.obj
 0002:00008358       ??_C@_0BL@JOAEAEKJ@IgnorePhysicsUpdatesOnSlot?$AA@ 320bc358     ScriptBind_Entity.obj
 0002:00008374       ??_C@_08EJIAJINA@DrawSlot?$AA@ 320bc374     ScriptBind_Entity.obj
 0002:00008380       ??_C@_0O@CFMHFKKC@nSlot?0nEnable?$AA@ 320bc380     ScriptBind_Entity.obj
 0002:00008390       ??_C@_0P@FCFGANJL@IsEntityInside?$AA@ 320bc390     ScriptBind_Entity.obj
 0002:000083a0       ??_C@_08BLPBAEMP@EntityId?$AA@ 320bc3a0     ScriptBind_Entity.obj
 0002:000083ac       ??_C@_0N@BDDKLBO@GetBoneLocal?$AA@ 320bc3ac     ScriptBind_Entity.obj
 0002:000083bc       ??_C@_0O@OHHEODMA@GetWorldScale?$AA@ 320bc3bc     ScriptBind_Entity.obj
 0002:000083cc       ??_C@_0P@FMAOPHPP@GetWorldAngles?$AA@ 320bc3cc     ScriptBind_Entity.obj
 0002:000083dc       ??_C@_0M@OFOPJAPL@GetWorldPos?$AA@ 320bc3dc     ScriptBind_Entity.obj
 0002:000083e8       ??_C@_0P@JCBAANND@SetWorldAngles?$AA@ 320bc3e8     ScriptBind_Entity.obj
 0002:000083f8       ??_C@_0M@OKPBEGHI@SetWorldPos?$AA@ 320bc3f8     ScriptBind_Entity.obj
 0002:00008404       ??_C@_0O@HJPCKNML@GetLocalScale?$AA@ 320bc404     ScriptBind_Entity.obj
 0002:00008414       ??_C@_0P@MLECKIDJ@GetLocalAngles?$AA@ 320bc414     ScriptBind_Entity.obj
 0002:00008424       ??_C@_0M@IGDNIDDC@GetLocalPos?$AA@ 320bc424     ScriptBind_Entity.obj
 0002:00008430       ??_C@_0P@FFMFCBF@SetLocalAngles?$AA@ 320bc430     ScriptBind_Entity.obj
 0002:00008440       ??_C@_0M@IJCDFFLB@SetLocalPos?$AA@ 320bc440     ScriptBind_Entity.obj
 0002:0000844c       ??_C@_0M@LKLJGNMP@UpdateAreas?$AA@ 320bc44c     ScriptBind_Entity.obj
 0002:00008458       ??_C@_0M@DCKJCANL@GetDistance?$AA@ 320bc458     ScriptBind_Entity.obj
 0002:00008464       ??_C@_0BF@OEECADOG@GetWorldBoundsCenter?$AA@ 320bc464     ScriptBind_Entity.obj
 0002:0000847c       ??_C@_0BD@LDGOMJN@GetCenterOfMassPos?$AA@ 320bc47c     ScriptBind_Entity.obj
 0002:00008490       ??_C@_08KNHMJFHM@GetScale?$AA@ 320bc490     ScriptBind_Entity.obj
 0002:0000849c       ??_C@_09JOJDAACO@GetAngles?$AA@ 320bc49c     ScriptBind_Entity.obj
 0002:000084a8       ??_C@_06DLMABKBK@GetPos?$AA@ 320bc4a8     ScriptBind_Entity.obj
 0002:000084b0       ??_C@_04BDGDJDM@vDir?$AA@  320bc4b0     ScriptBind_Entity.obj
 0002:000084b8       ??_C@_0BP@NJHIMFHF@CalcWorldAnglesFromRelativeDir?$AA@ 320bc4b8     ScriptBind_Entity.obj
 0002:000084d8       ??_C@_06EKABDFK@fScale?$AA@ 320bc4d8     ScriptBind_Entity.obj
 0002:000084e0       ??_C@_08FMFAIGAB@SetScale?$AA@ 320bc4e0     ScriptBind_Entity.obj
 0002:000084ec       ??_C@_07DAIMGIHO@vAngles?$AA@ 320bc4ec     ScriptBind_Entity.obj
 0002:000084f4       ??_C@_09LANGCBLM@SetAngles?$AA@ 320bc4f4     ScriptBind_Entity.obj
 0002:00008500       ??_C@_06KIFBKCMH@SetPos?$AA@ 320bc500     ScriptBind_Entity.obj
 0002:00008508       ??_C@_0N@JBINBOMJ@GetCharacter?$AA@ 320bc508     ScriptBind_Entity.obj
 0002:00008518       ??_C@_0BA@NONNCFIO@GetSlotWorldDir?$AA@ 320bc518     ScriptBind_Entity.obj
 0002:00008528       ??_C@_0BA@BMDAKILF@GetSlotWorldPos?$AA@ 320bc528     ScriptBind_Entity.obj
 0002:00008538       ??_C@_0P@CPDNCDFL@slot?0?5pos?0?5dir?$AA@ 320bc538     ScriptBind_Entity.obj
 0002:00008548       ??_C@_0P@PLGAODAH@SetSlotWorldTM?$AA@ 320bc548     ScriptBind_Entity.obj
 0002:00008558       ??_C@_09DHLJHBHA@slot?0?5pos?$AA@ 320bc558     ScriptBind_Entity.obj
 0002:00008564       ??_C@_0BD@CAFNEFC@MultiplyWithSlotTM?$AA@ 320bc564     ScriptBind_Entity.obj
 0002:00008578       ??_C@_0CE@MCIPICAF@srcSlot?0destSlot?0includeTranslat@ 320bc578     ScriptBind_Entity.obj
 0002:0000859c       ??_C@_0L@ENEHLBG@CopySlotTM?$AA@ 320bc59c     ScriptBind_Entity.obj
 0002:000085a8       ??_C@_0M@POFKCKHH@IsSlotValid?$AA@ 320bc5a8     ScriptBind_Entity.obj
 0002:000085b4       ??_C@_0N@LJLCFHDH@GetSlotScale?$AA@ 320bc5b4     ScriptBind_Entity.obj
 0002:000085c4       ??_C@_0O@HPIJFGPE@GetSlotAngles?$AA@ 320bc5c4     ScriptBind_Entity.obj
 0002:000085d4       ??_C@_0O@CAAFIOE@nSlot?0vAngles?$AA@ 320bc5d4     ScriptBind_Entity.obj
 0002:000085e4       ??_C@_0O@JHOFID@SetSlotAngles?$AA@ 320bc5e4     ScriptBind_Entity.obj
 0002:000085f4       ??_C@_0L@BPFBJPCM@GetSlotPos?$AA@ 320bc5f4     ScriptBind_Entity.obj
 0002:00008600       ??_C@_0BA@KEMJMPKC@nSlot?0vPos?0vDir?$AA@ 320bc600     ScriptBind_Entity.obj
 0002:00008610       ??_C@_0BB@NBODKCGP@SetSlotPosAndDir?$AA@ 320bc610     ScriptBind_Entity.obj
 0002:00008624       ??_C@_0L@OFCKIDFB@nSlot?0vPos?$AA@ 320bc624     ScriptBind_Entity.obj
 0002:00008630       ??_C@_0L@BHOCIGF@SetSlotPos?$AA@ 320bc630     ScriptBind_Entity.obj
 0002:0000863c       ??_C@_0N@PALCIPBL@GetSlotCount?$AA@ 320bc63c     ScriptBind_Entity.obj
 0002:0000864c       ??_C@_05GPGNDLEK@child?$AA@ 320bc64c     ScriptBind_Entity.obj
 0002:00008654       ??_C@_0O@HDMEEKAJ@GetParentSlot?$AA@ 320bc654     ScriptBind_Entity.obj
 0002:00008664       ??_C@_0O@IJLCCCOG@child?0?5parent?$AA@ 320bc664     ScriptBind_Entity.obj
 0002:00008674       ??_C@_0O@MNKPJHO@SetParentSlot?$AA@ 320bc674     ScriptBind_Entity.obj
 0002:00008684       ??_C@_0N@BJDAPNC@RenderAlways?$AA@ 320bc684     ScriptBind_Entity.obj
 0002:00008694       ??_C@_06OFNJOBDK@enable?$AA@ 320bc694     ScriptBind_Entity.obj
 0002:0000869c       ??_C@_0BG@PHOFLGPF@RegisterForAreaEvents?$AA@ 320bc69c     ScriptBind_Entity.obj
 0002:000086b4       ??_C@_0BG@DPEDFOAN@DeleteParticleEmitter?$AA@ 320bc6b4     ScriptBind_Entity.obj
 0002:000086cc       ??_C@_0BA@HDIMKJJO@IsSlotCharacter?$AA@ 320bc6cc     ScriptBind_Entity.obj
 0002:000086dc       ??_C@_0P@FAFGGKFA@IsSlotGeometry?$AA@ 320bc6dc     ScriptBind_Entity.obj
 0002:000086ec       ??_C@_0M@PAGGLPCM@IsSlotLight?$AA@ 320bc6ec     ScriptBind_Entity.obj
 0002:000086f8       ??_C@_04POIHOKKJ@slot?$AA@ 320bc6f8     ScriptBind_Entity.obj
 0002:00008700       ??_C@_0BG@GLDFPDHN@IsSlotParticleEmitter?$AA@ 320bc700     ScriptBind_Entity.obj
 0002:00008718       ??_C@_0M@NFLFFIP@sEffectName?$AA@ 320bc718     ScriptBind_Entity.obj
 0002:00008724       ??_C@_0BG@NLMCHJFP@PreLoadParticleEffect?$AA@ 320bc724     ScriptBind_Entity.obj
 0002:00008740       ??_C@_0FB@PIEPKLBP@nSlot?0sEffectName?0bPrime?0fPulseP@ 320bc740     ScriptBind_Entity.obj
 0002:00008794       ??_C@_0BD@CNNDDOM@LoadParticleEffect?$AA@ 320bc794     ScriptBind_Entity.obj
 0002:000087a8       ??_C@_0CG@DACBCPO@nSlot?0tVolumeObjectMovementPrope@ 320bc7a8     ScriptBind_Entity.obj
 0002:000087d0       ??_C@_0CC@HJBEEFOI@SetVolumeObjectMovementPropertie@ 320bc7d0     ScriptBind_Entity.obj
 0002:000087f4       ??_C@_0BB@ICLGOECO@LoadVolumeObject?$AA@ 320bc7f4     ScriptBind_Entity.obj
 0002:00008808       ??_C@_0BA@EPPGBHBI@LoadPrismObject?$AA@ 320bc808     ScriptBind_Entity.obj
 0002:00008818       ??_C@_0CC@FKAODIGE@nSlot?0fFadeTime?0fNewGlobalDensit@ 320bc818     ScriptBind_Entity.obj
 0002:0000883c       ??_C@_0BC@DBFAEEEC@FadeGlobalDensity?$AA@ 320bc83c     ScriptBind_Entity.obj
 0002:00008850       ??_C@_0BP@DHOEADLH@nSlot?0sLightShapeFile?0nLSFlags?$AA@ 320bc850     ScriptBind_Entity.obj
 0002:00008870       ??_C@_0P@LLGIGHDK@LoadLightShape?$AA@ 320bc870     ScriptBind_Entity.obj
 0002:00008880       ??_C@_0BM@HKBAAAHG@nSlot?0tFogVolumeDescription?$AA@ 320bc880     ScriptBind_Entity.obj
 0002:0000889c       ??_C@_0O@BECANGBD@LoadFogVolume?$AA@ 320bc89c     ScriptBind_Entity.obj
 0002:000088ac       ??_C@_0BP@GHIHFFG@nSlot?0tCloudMovementProperties?$AA@ 320bc8ac     ScriptBind_Entity.obj
 0002:000088cc       ??_C@_0BL@BDCLPCFL@SetCloudMovementProperties?$AA@ 320bc8cc     ScriptBind_Entity.obj
 0002:000088e8       ??_C@_0BF@HBMLPAFI@nSlot?0sCloudFilename?$AA@ 320bc8e8     ScriptBind_Entity.obj
 0002:00008900       ??_C@_09JNHBPHMC@LoadCloud?$AA@ 320bc900     ScriptBind_Entity.obj
 0002:0000890c       ??_C@_0L@BGMDAKEE@nLightSlot?$AA@ 320bc90c     ScriptBind_Entity.obj
 0002:00008918       ??_C@_0BO@KJEHHMNM@SetSelfAsLightCasterException?$AA@ 320bc918     ScriptBind_Entity.obj
 0002:00008938       ??_C@_0BG@LLELPAHJ@UpdateLightClipBounds?$AA@ 320bc938     ScriptBind_Entity.obj
 0002:00008950       ??_C@_0BI@MKOAFPEP@nSlot?0tLightDescription?$AA@ 320bc950     ScriptBind_Entity.obj
 0002:00008968       ??_C@_09DPEPMAPK@LoadLight?$AA@ 320bc968     ScriptBind_Entity.obj
 0002:00008974       ??_C@_0O@GAIDCAHM@LoadCharacter?$AA@ 320bc974     ScriptBind_Entity.obj
 0002:00008984       ??_C@_0BK@KJDNOKEO@nSlot?0sFilename?0sGeomName?$AA@ 320bc984     ScriptBind_Entity.obj
 0002:000089a0       ??_C@_0O@GMGPDMNC@LoadSubObject?$AA@ 320bc9a0     ScriptBind_Entity.obj
 0002:000089b0       ??_C@_05HKFIPNDJ@nSlot?$AA@ 320bc9b0     ScriptBind_Entity.obj
 0002:000089b8       ??_C@_0BC@CEABFAH@LoadObjectLattice?$AA@ 320bc9b8     ScriptBind_Entity.obj
 0002:000089cc       ??_C@_0BI@ILKCALHC@nSlot?0sFilename?0?5nFlags?$AA@ 320bc9cc     ScriptBind_Entity.obj
 0002:000089e4       ??_C@_0BE@FEDGBOCE@LoadObjectWithFlags?$AA@ 320bc9e4     ScriptBind_Entity.obj
 0002:000089f8       ??_C@_0BA@CHGCCOBM@nSlot?0sFilename?$AA@ 320bc9f8     ScriptBind_Entity.obj
 0002:00008a08       ??_C@_0L@FOLIKLPH@LoadObject?$AA@ 320bca08     ScriptBind_Entity.obj
 0002:00008a14       ??_C@_0BK@CLCFBDBH@CheckShaderParamCallbacks?$AA@ 320bca14     ScriptBind_Entity.obj
 0002:00008a30       ??_C@_0BC@LEPNIKII@CreateRenderProxy?$AA@ 320bca30     ScriptBind_Entity.obj
 0002:00008a44       ??_C@_0L@NHHADBIJ@DeleteThis?$AA@ 320bca44     ScriptBind_Entity.obj
 0002:00008a50       ??_C@_04EFDEBPGB@Keys?$AA@ 320bca50     ScriptBind_Entity.obj
 0002:00008a58       ??_C@_0BD@IDCALHLD@PropertiesInstance?$AA@ 320bca58     ScriptProperties.obj
 0002:00008a6c       ??_C@_0M@JOACKEPJ@Properties2?$AA@ 320bca6c     ScriptProperties.obj
 0002:00008a78       ??_7CScriptProxy@@6B@      320bca78     ScriptProxy.obj
 0002:00008b00       ??_C@_05ENKANFLO@class?$AA@ 320bcb00     ScriptProxy.obj
 0002:00008b08       ??_C@_06PLACEAIE@__this?$AA@ 320bcb08     ScriptProxy.obj
 0002:00008b10       ??_C@_06FEOMBGJC@OnLoad?$AA@ 320bcb10     ScriptProxy.obj
 0002:00008b18       ??_C@_06FGPBOFEG@OnSave?$AA@ 320bcb18     ScriptProxy.obj
 0002:00008b20       ??_C@_0BD@NGONBH@CScriptProxy?3?3Init?$AA@ 320bcb20     ScriptProxy.obj
 0002:00008b34       ??_C@_0BF@NDFKHCCI@CScriptProxy?3?3Reload?$AA@ 320bcb34     ScriptProxy.obj
 0002:00008b4c       ??_C@_0DF@CKIKDDGE@GotoState?5called?5with?5unknown?5st@ 320bcb4c     ScriptProxy.obj
 0002:00008b84       ??_C@_0L@CDCJHBPP@ScriptData?$AA@ 320bcb84     ScriptProxy.obj
 0002:00008b90       ??_C@_0BD@BGEKCOBC@OnGetPoolSignature?$AA@ 320bcb90     ScriptProxy.obj
 0002:00008ba4       ??_C@_0M@PIDEOBPN@ScriptProxy?$AA@ 320bcba4     ScriptProxy.obj
 0002:00008bb0       ??_C@_0P@KAKBPDHP@FullScriptData?$AA@ 320bcbb0     ScriptProxy.obj
 0002:00008bc0       ??_C@_0M@GCMECBP@currStateId?$AA@ 320bcbc0     ScriptProxy.obj
 0002:00008bcc       ??_C@_0BB@CIBFMCJK@scriptUpdateRate?$AA@ 320bcbcc     ScriptProxy.obj
 0002:00008be0       ??_C@_0BL@PDHJPGKM@Script?5proxy?5serialization?$AA@ 320bcbe0     ScriptProxy.obj
 0002:00008bfc       ??_C@_05LCLENNFI@table?$AA@ 320bcbfc     ScriptProxy.obj
 0002:00008c04       ??_C@_06JJLAMBGK@target?$AA@ 320bcc04     ScriptProxy.obj
 0002:00008c0c       ??_C@_09IJDJFKBE@target_id?$AA@ 320bcc0c     ScriptProxy.obj
 0002:00008c18       ??_C@_0M@NDGIMNEF@target_type?$AA@ 320bcc18     ScriptProxy.obj
 0002:00008c24       ??_C@_0L@PLCNFHFO@materialId?$AA@ 320bcc24     ScriptProxy.obj
 0002:00008c30       ??_C@_0M@DFOLEMEI@target_mass?$AA@ 320bcc30     ScriptProxy.obj
 0002:00008c3c       ??_C@_0BA@LGPNKBME@target_velocity?$AA@ 320bcc3c     ScriptProxy.obj
 0002:00008c4c       ??_C@_03DAPAKLGM@dir?$AA@  320bcc4c     ScriptProxy.obj
 0002:00008c50       ??_C@_0BK@DDMBOPOF@CScriptProxy?3?3OnCollision?$AA@ 320bcc50     ScriptProxy.obj
 0002:00008c6c       ??_C@_0BF@JGLPLDKG@CScriptProxy?3?3Update?$AA@ 320bcc6c     ScriptProxy.obj
 0002:00008c84       ??_C@_0L@JOIOLMFA@OnPostLoad?$AA@ 320bcc84     ScriptProxy.obj
 0002:00008c90       ??_C@_06HEBKAGDH@Events?$AA@ 320bcc90     ScriptProxy.obj
 0002:00008c98       ??_C@_0M@GJNJGBFO@SourceEvent?$AA@ 320bcc98     ScriptProxy.obj
 0002:00008ca4       ??_C@_06FGANPIPG@Target?$AA@ 320bcca4     ScriptProxy.obj
 0002:00008cac       ??_C@_05GCNIINAF@Event?$AA@ 320bccac     ScriptProxy.obj
 0002:00008cb4       ??_C@_0N@BCPLHDMD@EventTargets?$AA@ 320bccb4     ScriptProxy.obj
 0002:00008cc4       ??_7IThreadTask@@6B@       320bccc4     PhysicsEventListener.obj
 0002:00008cd4       ??_7CMultiThreadRefCount@@6B@ 320bccd4     PhysicsEventListener.obj
 0002:00008cd4       ??_7SThreadTaskInfo@@6B@   320bccd4     PhysicsEventListener.obj
 0002:00008cd8       ??_7CDeferredMeshUpdatePrep@@6B@ 320bccd8     PhysicsEventListener.obj
 0002:00008d00       ??_C@_07JOKPLCMC@pieces?$DN?$AA@ 320bcd00     PhysicsEventListener.obj
 0002:00008d08       ??_C@_07DALNOEPL@breaker?$AA@ 320bcd08     PhysicsEventListener.obj
 0002:00008d10       ??_C@_06HOPIODND@effect?$AA@ 320bcd10     PhysicsEventListener.obj
 0002:00008d18       ??_C@_06KEFIBDPP@$joint?$AA@ 320bcd18     PhysicsEventListener.obj
 0002:00008d20       ??_C@_0O@FOAJLHHG@joint_shatter?$AA@ 320bcd20     PhysicsEventListener.obj
 0002:00008d30       ??_C@_0M@MEHNKFAL@joint_break?$AA@ 320bcd30     PhysicsEventListener.obj
 0002:00008d3c       ??_C@_0BH@HEFMDDPG@physics_on_joint_break?$AA@ 320bcd3c     PhysicsEventListener.obj
 0002:00008d54       ??_C@_07OMIAIDGL@outdoor?$AA@ 320bcd54     PhysicsEventListener.obj
 0002:00008d5c       ??_C@_06BPDGOGCM@indoor?$AA@ 320bcd5c     PhysicsEventListener.obj
 0002:00008d64       ??_C@_0O@NDBBHIDE@PhysicalProxy?$AA@ 320bcd64     PhysicsProxy.obj
 0002:00008d74       ??_C@_08PLCBAIEK@CharRope?$AA@ 320bcd74     PhysicsProxy.obj
 0002:00008d80       ??_C@_0BC@EIAPDFBA@SerializableRopes?$AA@ 320bcd80     PhysicsProxy.obj
 0002:00008d94       ??_C@_0N@HEKMDLFM@PhysicsProxy?$AA@ 320bcd94     PhysicsProxy.obj
 0002:00008da4       ??_C@_0N@HCMKGPFI@PhysicsState?$AA@ 320bcda4     PhysicsProxy.obj
 0002:00008db8       ??_C@_0EF@HOGPHFNC@articulated?5entity?5simulated?5as?5@ 320bcdb8     PhysicsProxy.obj
 0002:00008e00       __real@56b5e621            320bce00     PhysicsProxy.obj
 0002:00008e08       ??_7CPhysicalProxy@@6B@    320bce08     PhysicsProxy.obj
 0002:00008e80       __real@c2c80000            320bce80     PhysicsProxy.obj
 0002:00008e88       ??_C@_0FF@EMMDBNIH@?$DMCPhysicalProxy?3?3PhysicalizeSoft@ 320bce88     PhysicsProxy.obj
 0002:00008ee0       ??_C@_0EP@DMLJKFGH@?$DMCPhysicalProxy?3?3PhysicalizeArea@ 320bcee0     PhysicsProxy.obj
 0002:00008f30       ??_C@_0BL@MGJKDDJM@CPhysicalProxy?3?3AddImpulse?$AA@ 320bcf30     PhysicsProxy.obj
 0002:00008f4c       ??_C@_0BA@LPPFBGIH@splinters_cloud?$AA@ 320bcf4c     PhysicsProxy.obj
 0002:00008f5c       ??_C@_0BM@JLMFLNIM@physics_on_tree_joint_break?$AA@ 320bcf5c     PhysicsProxy.obj
 0002:00008f78       __real@3ca3d70a            320bcf78     PhysicsProxy.obj
 0002:00008f7c       ??_C@_0BM@LIIBBGM@OnCollision?5?$CFs?5?$CITarget?3?5?$CFs?$CJ?$AA@ 320bcf7c     PhysicsProxy.obj
 0002:00008f98       ??_C@_09MGFHLAFE@?$DMUnknown?$DO?$AA@ 320bcf98     PhysicsProxy.obj
 0002:00008fa4       ??_C@_0BM@HHPIDCGM@CPhysicalProxy?3?3Physicalize?$AA@ 320bcfa4     PhysicsProxy.obj
 0002:00008fc0       ??_C@_0DA@CEOLDOJJ@Too?5big?5physical?5bounding?5box?5se@ 320bcfc0     PhysicsProxy.obj
 0002:00008ff0       ??_C@_0CB@BNPMOKCA@CPhysicalProxy?3?3SetTriggerBounds@ 320bcff0     PhysicsProxy.obj
 0002:00009014       ??_C@_0BP@CBHJNBM@CPhysicalProxy?3?3CheckColliders?$AA@ 320bd014     PhysicsProxy.obj
 0002:00009034       ??_C@_09BPFGNKAB@RopeProxy?$AA@ 320bd034     RopeProxy.obj
 0002:00009040       ??_C@_09IBBCHLFO@joint_lim?$AA@ 320bd040     RopeProxy.obj
 0002:0000904c       ??_C@_0N@GJOLBADM@water_resist?$AA@ 320bd04c     RopeProxy.obj
 0002:0000905c       ??_C@_0L@LMPFDFOO@air_resist?$AA@ 320bd05c     RopeProxy.obj
 0002:00009068       ??_C@_08KKHHJJBA@wind_var?$AA@ 320bd068     RopeProxy.obj
 0002:00009074       ??_C@_07BJBOFKDG@tension?$AA@ 320bd074     RopeProxy.obj
 0002:0000907c       ??_C@_0M@CDIKEKP@ph_sub_vtxs?$AA@ 320bd07c     RopeProxy.obj
 0002:00009088       ??_C@_0L@GNLDCEIB@ph_num_seg?$AA@ 320bd088     RopeProxy.obj
 0002:00009094       ??_C@_04BKPAKOEE@texv?$AA@ 320bd094     RopeProxy.obj
 0002:0000909c       ??_C@_04DBNNPNIH@texu?$AA@ 320bd09c     RopeProxy.obj
 0002:000090a4       ??_C@_09BAMCCABN@num_sides?$AA@ 320bd0a4     RopeProxy.obj
 0002:000090b0       ??_C@_07PCOPNCNE@num_seg?$AA@ 320bd0b0     RopeProxy.obj
 0002:000090b8       ??_C@_0O@MIAMFGLP@anchor_radius?$AA@ 320bd0b8     RopeProxy.obj
 0002:000090c8       ??_7CRopeProxy@@6B@        320bd0c8     RopeProxy.obj
 0002:00009100       ??_C@_06GEMKPBPA@Offset?$AA@ 320bd100     RopeProxy.obj
 0002:00009108       ??_C@_0BC@LLIPMHNB@SegmentToAttachTo?$AA@ 320bd108     RopeProxy.obj
 0002:0000911c       ??_C@_05MAHMNMLO@Sound?$AA@ 320bd11c     RopeProxy.obj
 0002:00009124       ??_C@_03FCCPIJGJ@Pos?$AA@  320bd124     RopeProxy.obj
 0002:00009128       ??_C@_06KANFALAM@Points?$AA@ 320bd128     RopeProxy.obj
 0002:00009130       ??_C@_04FEDAIEKO@Rope?$AA@ 320bd130     RopeProxy.obj
 0002:00009138       ??_C@_0O@PFEFBGD@MatLayersMask?$AA@ 320bd138     RopeProxy.obj
 0002:00009148       __real@42ca0000            320bd148     EntityObject.obj
 0002:0000914c       ??_C@_0BM@BCELPMHC@e_FoliageWindActivationDist?$AA@ 320bd14c     EntityObject.obj
 0002:00009168       ??_C@_0DA@KECJKAED@CEntityObject?3?3Render?3?5Invalid?5w@ 320bd168     EntityObject.obj
 0002:00009198       ??_C@_0DB@MKCEPICM@CEntityObject?3?3OnXForm?3?5Invalid?5@ 320bd198     EntityObject.obj
 0002:000091cc       __real@3c888889            320bd1cc     EntityObject.obj
 0002:000091d0       __real@42652ee1            320bd1d0     EntityObject.obj
 0002:000091d8       ?iid@?1??IID@IShaderParamCallback@@CAABUCryGUID@@XZ@4U3@B 320bd1d8     RenderProxy.obj
 0002:000091e8       ??_7IShadowCaster@@6B@     320bd1e8     RenderProxy.obj
 0002:00009208       __real@42800000            320bd208     RenderProxy.obj
 0002:0000920c       ??_C@_0DE@PJJBFCOF@BBox?5contain?5invalid?5floating?5va@ 320bd20c     RenderProxy.obj
 0002:00009240       ??_7IEntityRenderProxy@@6B@ 320bd240     RenderProxy.obj
 0002:00009348       __real@3f808102            320bd348     RenderProxy.obj
 0002:0000934c       ??_C@_0O@OGEADPKO@ViewDistRatio?$AA@ 320bd34c     RenderProxy.obj
 0002:0000935c       ??_C@_08PDEIIGKO@LodRatio?$AA@ 320bd35c     RenderProxy.obj
 0002:00009368       ??_C@_0M@BAHCOLJF@RenderProxy?$AA@ 320bd368     RenderProxy.obj
 0002:00009374       __real@7f7fffff            320bd374     RenderProxy.obj
 0002:00009378       ??_C@_0BF@DNBDKGN@CRenderProxy?3?3Render?$AA@ 320bd378     RenderProxy.obj
 0002:00009390       ??_C@_0GK@PJLMPMCO@CRenderProxy?3?3RegisterForRenderi@ 320bd390     RenderProxy.obj
 0002:000093fc       ??_C@_0BJ@MIJILBCL@e_FoliageBranchesTimeout?$AA@ 320bd3fc     RenderProxy.obj
 0002:00009418       ??_C@_0BG@DBKOMNBC@RenderProxy?5Allocator?$AA@ 320bd418     RenderProxy.obj
 0002:00009430       ??_C@_0BF@PAGEDCIJ@CRenderProxy?3?3Update?$AA@ 320bd430     RenderProxy.obj
 0002:00009448       ??_C@_09PIAIFBON@Rendering?$AA@ 320bd448     RenderProxy.obj
 0002:00009454       ??_C@_0DN@FBGMPNNM@RenderProxy?5not?5seen?3?5id?5?$DN?5?$CC0x?$CFX@ 320bd454     RenderProxy.obj
 0002:00009498       ??_7CRenderProxy@@6BIEntityRenderProxy@@@ 320bd498     RenderProxy.obj
 0002:000095a0       ??_7CRenderProxy@@6BIRenderNode@@@ 320bd5a0     RenderProxy.obj
 0002:000096bc       __real@3c800000            320bd6bc     RenderProxy.obj
 0002:000096c0       ??_C@_0HE@BNBCNGPJ@CRenderProxy?3?3SetSlotCharacter?$CI?$CJ@ 320bd6c0     RenderProxy.obj
 0002:00009738       ??_C@_0ED@FFEPCELA@?$FLRenderProxy?3?3LoadGeometry?$FN?5Call@ 320bd738     RenderProxy.obj
 0002:00009780       ??_C@_0EE@MCLIDNKC@?$FLRenderProxy?3?3LoadCharacter?$FN?5Cal@ 320bd780     RenderProxy.obj
 0002:000097c4       ??_C@_0L@LIOBPHGH@CheapLight?$AA@ 320bd7c4     RenderProxy.obj
 0002:000097d0       ??_C@_09NCLMNOLJ@Particles?$AA@ 320bd7d0     RenderProxy.obj
 0002:000097dc       ??_C@_09PPGNMBGC@MatLayers?$AA@ 320bd7dc     RenderProxy.obj
 0002:000097e8       __real@3f4ccccd            320bd7e8     AreaProxy.obj
 0002:000097ec       ??_C@_09EOFEFOJA@AreaProxy?$AA@ 320bd7ec     AreaProxy.obj
 0002:000097f8       ??_7CAreaProxy@@6B@        320bd7f8     AreaProxy.obj
 0002:000098a0       ??_C@_0BC@FCFDBAEL@ed_lowercasepaths?$AA@ 320bd8a0     AreaProxy.obj
 0002:000098b4       ??_C@_08JFELGNCJ@OnEnable?$AA@ 320bd8b4     AreaProxy.obj
 0002:000098c0       ??_C@_07MIKIFGAL@Disable?$AA@ 320bd8c0     AreaProxy.obj
 0002:000098c8       ??_C@_06CKGENIKG@Enable?$AA@ 320bd8c8     AreaProxy.obj
 0002:000098d0       ??_C@_06IHBCN@Side?$CFd?$AA@ 320bd8d0     AreaProxy.obj
 0002:000098d8       ??_C@_05BGOFFEGG@Point?$AA@ 320bd8d8     AreaProxy.obj
 0002:000098e0       ??_C@_09GACHPFDC@SoundData?$AA@ 320bd8e0     AreaProxy.obj
 0002:000098ec       ??_C@_06EGIKIAFJ@BoxMax?$AA@ 320bd8ec     AreaProxy.obj
 0002:000098f4       ??_C@_06FEABGEDG@BoxMin?$AA@ 320bd8f4     AreaProxy.obj
 0002:000098fc       ??_C@_02JDPG@rb?$AA@       320bd8fc     AreaProxy.obj
 0002:00009900       ??_C@_07OMDAAECB@?$CFlevel?$CF?$AA@ 320bd900     AreaProxy.obj
 0002:00009908       ??_C@_0BC@CDJFGCLE@AreaSolidFileName?$AA@ 320bd908     AreaProxy.obj
 0002:0000991c       ??_C@_0N@JGBDNKMD@BezierPoints?$AA@ 320bd91c     AreaProxy.obj
 0002:0000992c       ??_C@_0BF@MLFJEIOI@DontDisableInvisible?$AA@ 320bd92c     AreaProxy.obj
 0002:00009944       ??_C@_07JMGDFJEK@Gravity?$AA@ 320bd944     AreaProxy.obj
 0002:0000994c       ??_C@_0N@HHPNONEM@VolumeRadius?$AA@ 320bd94c     AreaProxy.obj
 0002:0000995c       ??_C@_0N@EHJGIDKG@SphereCenter?$AA@ 320bd95c     AreaProxy.obj
 0002:0000996c       ??_C@_0N@PAFAFDBI@SphereRadius?$AA@ 320bd96c     AreaProxy.obj
 0002:0000997c       ??_C@_06HCAKHJJK@Height?$AA@ 320bd97c     AreaProxy.obj
 0002:00009984       ??_C@_0O@MKGDNKOC@ObstructSound?$AA@ 320bd984     AreaProxy.obj
 0002:00009994       ??_C@_08KGEIBGG@Priority?$AA@ 320bd994     AreaProxy.obj
 0002:000099a0       ??_C@_09IAKIBBN@Proximity?$AA@ 320bd9a0     AreaProxy.obj
 0002:000099ac       ??_C@_05MBDCODDP@Group?$AA@ 320bd9ac     AreaProxy.obj
 0002:000099b4       ??_C@_08HIPCGCNC@def_head?$AA@ 320bd9b4     SoundProxy.obj
 0002:000099c0       ??_C@_0L@GHIHOBPC@Bip01?5Head?$AA@ 320bd9c0     SoundProxy.obj
 0002:000099cc       ??_C@_05JMBBACAO@voice?$AA@ 320bd9cc     SoundProxy.obj
 0002:000099d4       ??_C@_06HDFPFMNM@spread?$AA@ 320bd9d4     SoundProxy.obj
 0002:000099dc       ??_C@_0BF@DKDLAOGL@environment_listener?$AA@ 320bd9dc     SoundProxy.obj
 0002:000099f4       ??_C@_0BC@LOALLGKE@environment_sound?$AA@ 320bd9f4     SoundProxy.obj
 0002:00009a08       ??_C@_0CA@EFOPHGBH@RayWorldIntersection?$CIEntitySys?$CJ?$AA@ 320bda08     SoundProxy.obj
 0002:00009a28       ??_7CSoundProxy@@6BISoundEventListener@@@ 320bda28     SoundProxy.obj
 0002:00009a30       ??_7CSoundProxy@@6BIEntitySoundProxy@@@ 320bda30     SoundProxy.obj
 0002:00009ac0       ??_C@_0DD@KCEAFOLO@?$DMSound?$DO?5Trying?5to?5play?5?$DM?$CFs?$DO?5on?5?$CF@ 320bdac0     SoundProxy.obj
 0002:00009af8       ??_C@_0GP@FCHBPGHE@?$DMSound?$DO?5Trying?5to?5play?5a?5sound?5a@ 320bdaf8     SoundProxy.obj
 0002:00009b68       ??_C@_0N@KJCPPENH@ClientServer?$AA@ 320bdb68     FlowGraphProxy.obj
 0002:00009b78       ??_C@_0L@INJCILBP@ClientOnly?$AA@ 320bdb78     FlowGraphProxy.obj
 0002:00009b84       ??_C@_0M@LBDADJEK@MultiPlayer?$AA@ 320bdb84     FlowGraphProxy.obj
 0002:00009b90       ??_C@_0FG@IECOEBGN@?$FLFlowGraphProxy?$FN?5Skipped?5loading@ 320bdb90     FlowGraphProxy.obj
 0002:00009be8       ??_C@_09POICFOIO@FlowGraph?$AA@ 320bdbe8     FlowGraphProxy.obj
 0002:00009bf4       ??_C@_0P@FEMNCOF@FlowGraphProxy?$AA@ 320bdbf4     FlowGraphProxy.obj
 0002:00009c04       ??_C@_0CA@MNPMLPOC@Unable?5to?5reload?5flowgraph?5here?$AA@ 320bdc04     FlowGraphProxy.obj
 0002:00009c28       ??_7CFlowGraphProxy@@6B@   320bdc28     FlowGraphProxy.obj
 0002:00009c6c       ??_C@_0BC@LKAPCLOK@e_OnDemandMaxSize?$AA@ 320bdc6c     SubstitutionProxy.obj
 0002:00009c80       ??_C@_0BC@MNNLJLEK@e_OnDemandPhysics?$AA@ 320bdc80     SubstitutionProxy.obj
 0002:00009c94       ??_C@_0BC@JIOMGDFM@SubstitutionProxy?$AA@ 320bdc94     SubstitutionProxy.obj
 0002:00009ca8       __real@3a6bedfa            320bdca8     SubstitutionProxy.obj
 0002:00009cac       ??_C@_08KHMAMEDA@SubstPos?$AA@ 320bdcac     SubstitutionProxy.obj
 0002:00009cb8       ??_C@_0M@MIAMOGLP@SubstCenter?$AA@ 320bdcb8     SubstitutionProxy.obj
 0002:00009cc8       ??_7CTriggerProxy@@6B@     320bdcc8     TriggerProxy.obj
 0002:00009d0c       ??_C@_0N@HKFDGIKP@TriggerProxy?$AA@ 320bdd0c     TriggerProxy.obj
 0002:00009d1c       ??_C@_0M@OLBCCIKF@CameraProxy?$AA@ 320bdd1c     CameraProxy.obj
 0002:00009d28       __real@44800000            320bdd28     CameraProxy.obj
 0002:00009d2c       __real@42700000            320bdd2c     CameraProxy.obj
 0002:00009d30       __real@c2a00000            320bdd30     CameraProxy.obj
 0002:00009d34       __real@3faaaaab            320bdd34     CameraProxy.obj
 0002:00009d38       __real@3fa78d36            320bdd38     CameraProxy.obj
 0002:00009d3c       __real@43700000            320bdd3c     CameraProxy.obj
 0002:00009d40       __real@c3a00000            320bdd40     CameraProxy.obj
 0002:00009d48       __real@3fe4f1a6c0000000    320bdd48     CameraProxy.obj
 0002:00009d50       ??_7CCameraProxy@@6B@      320bdd50     CameraProxy.obj
 0002:00009d8c       __real@40e90fdb            320bdd8c     EntityNodeProxy.obj
 0002:00009d90       ??_C@_0CM@MDCDMMAJ@Failed?5to?5find?5material?5for?5foot@ 320bdd90     EntityNodeProxy.obj
 0002:00009dbc       ??_C@_07DLHCIBDH@default?$AA@ 320bddbc     EntityNodeProxy.obj
 0002:00009dc4       ??_C@_08OJAFAPFK@footstep?$AA@ 320bddc4     EntityNodeProxy.obj
 0002:00009dd0       ??_7IEntityClass@@6B@      320bddd0     EntityClass.obj
 0002:00009e18       ??_7CEntityClass@@6B@      320bde18     EntityClass.obj
 0002:00009e5c       ??_7IEntityClassRegistry@@6B@ 320bde5c     EntityClassRegistry.obj
 0002:00009e5c       ??_7IAreaManager@@6B@      320bde5c     AreaManager.obj
 0002:00009e84       ??_C@_0CF@JCBHDEEP@EntityScript?5?$CFs?5failed?5to?5initia@ 320bde84     EntityClassRegistry.obj
 0002:00009eac       ??_C@_0CI@LNFCLBGD@Scripts?1Entities?1Default?1RopeEnt@ 320bdeac     EntityClassRegistry.obj
 0002:00009ed4       ??_C@_0L@DPFKNAEA@RopeEntity?$AA@ 320bded4     EntityClassRegistry.obj
 0002:00009ee0       ??_C@_0CI@INPLEPCN@Scripts?1Entities?1Default?1GeomEnt@ 320bdee0     EntityClassRegistry.obj
 0002:00009f08       ??_C@_0L@FHEFLOBF@GeomEntity?$AA@ 320bdf08     EntityClassRegistry.obj
 0002:00009f18       ??_C@_0FM@KAPNIFL@?$FLCEntityClassRegistry?$FN?5LoadClass@ 320bdf18     EntityClassRegistry.obj
 0002:00009f74       ??_C@_09EPJGIIIJ@Invisible?$AA@ 320bdf74     EntityClassRegistry.obj
 0002:00009f80       ??_C@_06CEFAHBNL@Script?$AA@ 320bdf80     EntityClassRegistry.obj
 0002:00009f88       ??_C@_06IGECIDCI@?1?$CK?4ent?$AA@ 320bdf88     EntityClassRegistry.obj
 0002:00009f90       ??_C@_02CFKBDFGI@?1?2?$AA@ 320bdf90     EntityClassRegistry.obj
 0002:00009f94       ??_7CEntityClassRegistry@@6B@ 320bdf94     EntityClassRegistry.obj
 0002:00009fc0       ??_C@_0FC@EPNMACPC@CEntityClassRegistry?3?3RegisterCl@ 320bdfc0     EntityClassRegistry.obj
 0002:0000a014       ??_C@_0N@KHMKNHMO@e_ObjQuality?$AA@ 320be014     EntityLoadManager.obj
 0002:0000a024       ??_C@_07BANFLEJO@MinSpec?$AA@ 320be024     EntityLoadManager.obj
 0002:0000a030       ??_C@_0EM@OOHNAJGM@Entity?5class?5?$CFs?5used?5by?5entity?5?$CF@ 320be030     EntityLoadManager.obj
 0002:0000a07c       ??_C@_0BD@GGPMAHFD@CreatedThroughPool?$AA@ 320be07c     EntityLoadManager.obj
 0002:0000a090       ??_C@_0EJ@MDHJKKHC@Archetype?5?$CFs?5used?5by?5entity?5?$CFs?5c@ 320be090     EntityLoadManager.obj
 0002:0000a0dc       ??_C@_09FLECHFNM@Archetype?$AA@ 320be0dc     EntityLoadManager.obj
 0002:0000a0e8       ??_C@_08PGMHMLNK@NoDecals?$AA@ 320be0e8     EntityLoadManager.obj
 0002:0000a0f4       ??_C@_0M@DLDAIHGI@OutdoorOnly?$AA@ 320be0f4     EntityLoadManager.obj
 0002:0000a100       ??_C@_0N@DNNHPEIA@GoodOccluder?$AA@ 320be100     EntityLoadManager.obj
 0002:0000a110       ??_C@_0L@MBLKBNFB@CastShadow?$AA@ 320be110     EntityLoadManager.obj
 0002:0000a11c       ??_C@_0L@FKANMEPO@EntityGuid?$AA@ 320be11c     EntityLoadManager.obj
 0002:0000a128       ??_C@_06OLMBOMJH@Rotate?$AA@ 320be128     EntityLoadManager.obj
 0002:0000a130       ??_C@_0M@HEPBNCBF@EntityClass?$AA@ 320be130     EntityLoadManager.obj
 0002:0000a13c       ??_C@_0N@JLMLBHNO@HiddenInGame?$AA@ 320be13c     EntityLoadManager.obj
 0002:0000a14c       ??_C@_06FOLGHFDA@RelPos?$AA@ 320be14c     EntityLoadManager.obj
 0002:0000a154       ??_C@_06LLPOCLHM@RelRot?$AA@ 320be154     EntityLoadManager.obj
 0002:0000a15c       ??_C@_08IPFKHCPE@TargetId?$AA@ 320be15c     EntityLoadManager.obj
 0002:0000a168       ??_C@_0M@HBBANCO@EntityLinks?$AA@ 320be168     EntityLoadManager.obj
 0002:0000a174       ??_C@_08OIKOLDOC@ParentId?$AA@ 320be174     EntityLoadManager.obj
 0002:0000a180       ??_C@_08OOJNLKLP@Geometry?$AA@ 320be180     EntityLoadManager.obj
 0002:0000a18c       ??_C@_08CPBFELGP@Material?$AA@ 320be18c     EntityLoadManager.obj
 0002:0000a198       ??_C@_0BC@GBCBLMFN@PrototypeMaterial?$AA@ 320be198     EntityLoadManager.obj
 0002:0000a1ac       ??_C@_09DIKEFLGO@Entity?5?$CFs?$AA@ 320be1ac     EntityLoadManager.obj
 0002:0000a1b8       ??_C@_0EE@NMPKDIGJ@CEntityLoadManager?3?3ParseEntitie@ 320be1b8     EntityLoadManager.obj
 0002:0000a1fc       ??_C@_07NBCGADJA@Unknown?$AA@ 320be1fc     EntityLoadManager.obj
 0002:0000a204       ??_C@_0BB@PEAOPEHN@ReloadProperties?$AA@ 320be204     EntityLoadManager.obj
 0002:0000a218       ??_C@_0BE@PAPJNMCB@Parsing?5entity?5?8?$CFs?8?$AA@ 320be218     EntityLoadManager.obj
 0002:0000a22c       ??_C@_0CC@FOFAEPOP@CEntityLoadManager?3?3ParseEntitie@ 320be22c     EntityLoadManager.obj
 0002:0000a250       ??_C@_0BH@NJKPLNL@Parsing?5?$CFu?5entities?4?4?4?$AA@ 320be250     EntityLoadManager.obj
 0002:0000a268       ??_7IArea@@6B@             320be268     Area.obj
 0002:0000a268       ??_7IEntityArchetype@@6B@  320be268     EntityArchetype.obj
 0002:0000a280       __real@3e7ad7f29abcaf48    320be280     Area.obj
 0002:0000a288       ??_C@_0CH@DFGHGAKE@?$DMAreaManager?$DO?5Area?5?$CFd?5Direct?5Eve@ 320be288     Area.obj
 0002:0000a2b0       ??_C@_0L@BNDNFOF@MOVEINSIDE?$AA@ 320be2b0     Area.obj
 0002:0000a2bc       ??_C@_08GLNKAOBE@MOVENEAR?$AA@ 320be2bc     Area.obj
 0002:0000a2c8       ??_C@_0CH@ICLBGGBL@?$DMAreaManager?$DO?5Area?5?$CFd?5Queued?5Eve@ 320be2c8     Area.obj
 0002:0000a2f0       ??_C@_09EEINCFMI@LEAVENEAR?$AA@ 320be2f0     Area.obj
 0002:0000a2fc       ??_C@_05GACDJFGI@LEAVE?$AA@ 320be2fc     Area.obj
 0002:0000a304       ??_C@_05EMNIMLKD@ENTER?$AA@ 320be304     Area.obj
 0002:0000a30c       ??_C@_09EGHDBLOA@ENTERNEAR?$AA@ 320be30c     Area.obj
 0002:0000a318       ??_7CArea@@6B@             320be318     Area.obj
 0002:0000a32c       __real@40a00000            320be32c     Area.obj
 0002:0000a330       ??_C@_0M@DJIGNEPH@DETACH_THIS?$AA@ 320be330     Area.obj
 0002:0000a33c       __real@4b189680            320be33c     Area.obj
 0002:0000a340       ?GRID_CELL_SIZE@CAreaGrid@@1IB 320be340     AreaGrid.obj
 0002:0000a344       ?GRID_CELL_SIZE_R@CAreaGrid@@1MB 320be344     AreaGrid.obj
 0002:0000a348       ??_C@_0DE@DOFFPAFA@Area?5Grid?5Mem?5Use?3?5num?5cells?3?5?$CFd@ 320be348     AreaGrid.obj
 0002:0000a37c       __real@3faccccd            320be37c     AreaGrid.obj
 0002:0000a384       ??_C@_0BD@HBPKGFLI@CAreaGrid?3?3Compile?$AA@ 320be384     AreaGrid.obj
 0002:0000a398       ??_C@_0BK@FFIHABHN@CAreaManager?3?3ProcessArea?$AA@ 320be398     AreaManager.obj
 0002:0000a3b4       ??_C@_0DD@GIDECOM@AreaIndex?5?3?$CFd?5Priority?5?3?$CFd?5Dista@ 320be3b4     AreaManager.obj
 0002:0000a3e8       ??_C@_03DENIJNGB@Far?$AA@  320be3e8     AreaManager.obj
 0002:0000a3ec       ??_C@_04IGPKFDJI@Near?$AA@ 320be3ec     AreaManager.obj
 0002:0000a3f4       ??_C@_06COPGKAIJ@Inside?$AA@ 320be3f4     AreaManager.obj
 0002:0000a3fc       ??_C@_0CJ@EBDFGMHI@Num?5entries?5in?5cache?3?5?$CFd?5total?5a@ 320be3fc     AreaManager.obj
 0002:0000a428       ??_C@_04LIFAFMCE@?$FL?$CFs?$FN?$AA@ 320be428     AreaManager.obj
 0002:0000a430       __real@43480000            320be430     AreaManager.obj
 0002:0000a434       ??_7CAreaManager@@6B@      320be434     AreaManager.obj
 0002:0000a45c       ??_C@_0BL@JLKGBNNP@CAreaManager?3?3UpdatePlayer?$AA@ 320be45c     AreaManager.obj
 0002:0000a478       __real@44160000            320be478     AreaManager.obj
 0002:0000a47c       ??_C@_0CO@FJHFDGD@playerToUpdate?$DN?$CFd?5?$CI?$CFs?$CJ?5pos?$DN?$CI?$CF?42f@ 320be47c     AreaManager.obj
 0002:0000a4b0       ??_7IBreakableManager@@6B@ 320be4b0     BreakableManager.obj
 0002:0000a514       ??_C@_0BA@EEGMFOFG@Surface?5Effect?5?$AA@ 320be514     BreakableManager.obj
 0002:0000a524       ??_C@_0P@IEFIAICF@freeze_shatter?$AA@ 320be524     BreakableManager.obj
 0002:0000a534       ??_C@_07OKFGPCEA@destroy?$AA@ 320be534     BreakableManager.obj
 0002:0000a540       ??_7CBreakableManager@@6B@ 320be540     BreakableManager.obj
 0002:0000a5a8       ??_C@_08CFKLHNPN@Breakage?$AA@ 320be5a8     BreakableManager.obj
 0002:0000a5b4       ??_C@_0P@PCAIFDGI@breakage_carve?$AA@ 320be5b4     BreakableManager.obj
 0002:0000a5c4       ??_C@_08KHFKPPFO@breakage?$AA@ 320be5c4     BreakableManager.obj
 0002:0000a5d0       ??_C@_06OOBPHOGO@kwater?$AA@ 320be5d0     BreakableManager.obj
 0002:0000a5d8       ??_C@_07NJDCDANA@rotaxes?$AA@ 320be5d8     BreakableManager.obj
 0002:0000a5e0       ??_C@_07EHAPCMGK@sizevar?$AA@ 320be5e0     BreakableManager.obj
 0002:0000a5e8       ??_C@_07DCLBNMLN@generic?$AA@ 320be5e8     BreakableManager.obj
 0002:0000a5f0       ??_C@_04ODKJLCFC@bone?$AA@ 320be5f0     BreakableManager.obj
 0002:0000a5f8       ??_C@_06NAKANDOK@Remain?$AA@ 320be5f8     BreakableManager.obj
 0002:0000a600       ??_C@_04KGFMLCPK@Main?$AA@ 320be600     BreakableManager.obj
 0002:0000a608       ??_C@_0CD@JNFAMNIB@CBreakableManager?3?3BreakIntoPiec@ 320be608     BreakableManager.obj
 0002:0000a62c       __real@41700000            320be62c     BreakableManager.obj
 0002:0000a630       ??_C@_09JPBGPBK@splinters?$AA@ 320be630     BreakableManager.obj
 0002:0000a63c       ??_C@_09BBABGHMP@entity_mp?$AA@ 320be63c     BreakableManager.obj
 0002:0000a648       ??_C@_06DKNBAMDM@floats?$AA@ 320be648     BreakableManager.obj
 0002:0000a650       ??_C@_0P@NGOEINEK@Partition?5Grid?$AA@ 320be650     PartitionGrid.obj
 0002:0000a660       ??_7Test@CryUnitTest@@6B@  320be660     PartitionGrid.obj
 0002:0000a670       ??_7CUT_PartitionGrid@@6B@ 320be670     PartitionGrid.obj
 0002:0000a680       ??_C@_0BK@GEILLOMP@CPartitionGrid?3?3Rellocate?$AA@ 320be680     PartitionGrid.obj
 0002:0000a69c       ??_C@_0DA@GGMFGFKO@query?4pEntities?5?$CG?$CG?5query?4pEntiti@ 320be69c     PartitionGrid.obj
 0002:0000a6cc       __real@461c4000            320be6cc     PartitionGrid.obj
 0002:0000a6d0       ??_C@_0DA@HPNOFEOP@query?4pEntities?5?$CG?$CG?5query?4pEntiti@ 320be6d0     PartitionGrid.obj
 0002:0000a700       ??_C@_0DA@DAJPMCCI@query?4pEntities?5?$CG?$CG?5query?4pEntiti@ 320be700     PartitionGrid.obj
 0002:0000a730       __real@43c80000            320be730     PartitionGrid.obj
 0002:0000a734       __real@441b0000            320be734     PartitionGrid.obj
 0002:0000a738       __real@442f0000            320be738     PartitionGrid.obj
 0002:0000a73c       __real@43fb8000            320be73c     PartitionGrid.obj
 0002:0000a740       __real@43fa8000            320be740     PartitionGrid.obj
 0002:0000a744       __real@43fa0000            320be744     PartitionGrid.obj
 0002:0000a748       ??_C@_0EM@BKODBDDG@pGrid?9?$DOm_nHeight?5?$DN?$DN?5?$CIint?$CJ?$CIfMeter@ 320be748     PartitionGrid.obj
 0002:0000a798       ??_C@_0EL@EJICFBJG@pGrid?9?$DOm_nWidth?5?$DN?$DN?5?$CIint?$CJ?$CIfMeters@ 320be798     PartitionGrid.obj
 0002:0000a7e8       ??_C@_0FJ@BMPKBING@D?3?2BuildScript?4NET?2dev_c3?2pc?2Bui@ 320be7e8     PartitionGrid.obj
 0002:0000a844       ??_C@_0BC@KPKADODC@CUT_PartitionGrid?$AA@ 320be844     PartitionGrid.obj
 0002:0000a858       __real@80000000            320be858     ProximityTriggerSystem.obj
 0002:0000a85c       ??_C@_0CE@EOPEPAJO@CProximityTriggerSystem?3?3SendEve@ 320be85c     ProximityTriggerSystem.obj
 0002:0000a880       __real@42fa0000            320be880     ProximityTriggerSystem.obj
 0002:0000a884       ??_C@_0CG@OFABDEJH@CProximityTriggerSystem?3?3SortTri@ 320be884     ProximityTriggerSystem.obj
 0002:0000a8ac       ??_C@_0CA@BIFPHHFP@CProximityTriggerSystem?3?3Update?$AA@ 320be8ac     ProximityTriggerSystem.obj
 0002:0000a8d0       ??_C@_0FD@EJBALABA@?$FLEntity?5Pool?$FN?5WARNING?3?5DEBUG?3?5Si@ 320be8d0     EntityPool.obj
 0002:0000a928       ??_C@_0EG@JNHLGNFE@?$FLEntity?5Pool?$FN?5DEBUG?3?5Signature?5p@ 320be928     EntityPool.obj
 0002:0000a970       ??_C@_0CB@EEKKFDCE@CEntityPool?3?3ContainsEntityClass@ 320be970     EntityPool.obj
 0002:0000a994       ??_C@_0CJ@IALFLCG@Found?5invalid?5pool?5entity?5?$CIentit@ 320be994     EntityPool.obj
 0002:0000a9c0       ??_C@_0CF@IMLHGAGE@CEntityPool?3?3GetPoolEntityWithPo@ 320be9c0     EntityPool.obj
 0002:0000a9e8       ??_C@_0CK@FIMBOIEH@CEntityPool?3?3GetPoolEntityFromIn@ 320be9e8     EntityPool.obj
 0002:0000aa14       ??_C@_0L@LAAPPAK@PoolEntity?$AA@ 320bea14     EntityPool.obj
 0002:0000aa20       ??_C@_0BP@GKKNLKID@CEntityPool?3?3DestroyPoolEntity?$AA@ 320bea20     EntityPool.obj
 0002:0000aa40       ??_C@_0BD@HPHJKOJI@Create?5Pool?5Entity?$AA@ 320bea40     EntityPool.obj
 0002:0000aa54       ??_C@_0BO@DFMPIEJI@CEntityPool?3?3CreatePoolEntity?$AA@ 320bea54     EntityPool.obj
 0002:0000aa74       ??_C@_0BP@IENJEAOO@CEntityPool?3?3OnPoolEntityInUse?$AA@ 320bea74     EntityPool.obj
 0002:0000aa94       ??_C@_0CC@CGNCKFFO@CEntityPool?3?3OnPoolEntityReturne@ 320bea94     EntityPool.obj
 0002:0000aab8       ??_C@_0FF@PHCOBBDN@CEntityPool?3?3CreatePool?$CI?$CJ?5Failed@ 320beab8     EntityPool.obj
 0002:0000ab10       ??_C@_0P@LEFKFGDB@Create?5Pool?5?$CFs?$AA@ 320beb10     EntityPool.obj
 0002:0000ab20       ??_C@_0BI@NAAJMFAJ@CEntityPool?3?3CreatePool?$AA@ 320beb20     EntityPool.obj
 0002:0000ab38       ??_C@_03NPBFACHO@?5?$CL?5?$AA@ 320beb38     EntityPool.obj
 0002:0000ab3c       ??_C@_0BJ@CFDFMEOP@CEntityPool?3?3ConsumePool?$AA@ 320beb3c     EntityPool.obj
 0002:0000ab58       ??_C@_0JC@HOENOLJM@?$FLEntity?5Pool?$FN?5Pool?5?8?$CFs?8?5has?5reac@ 320beb58     EntityPool.obj
 0002:0000abec       ??_C@_0CI@JCICJNIO@CEntityPool?3?3GetPoolEntityFromAc@ 320bebec     EntityPool.obj
 0002:0000ac14       ??_C@_0BC@EDKDLGEH@Pool?5Definitions?3?$AA@ 320bec14     EntityPool.obj
 0002:0000ac28       ??_C@_0BH@EBGDIKM@?5?9?5Return?5Weight?3?5?$CF?43f?$AA@ 320bec28     EntityPool.obj
 0002:0000ac40       ??_C@_07IBEGINLN@?$CFs?5?$CI?$CFu?$CJ?$AA@ 320bec40     EntityPool.obj
 0002:0000ac48       ??_C@_0BD@GGKOGHN@In?5Use?5?9?5Count?3?5?$CFu?$AA@ 320bec48     EntityPool.obj
 0002:0000ac5c       ??_C@_02KEGNLNML@?0?5?$AA@ 320bec5c     EntityPool.obj
 0002:0000ac60       ??_C@_0BH@PIPIKEAL@Not?5In?5Use?5?9?5Count?3?5?$CFu?$AA@ 320bec60     EntityPool.obj
 0002:0000ac78       ??_C@_0BJ@ECFKGBPP@Force?5Reused?5Counter?3?5?$CFd?$AA@ 320bec78     EntityPool.obj
 0002:0000ac94       ??_C@_0CC@JFEGKBCD@Pool?5?8?$CFs?8?5?$CIDefault?5Class?5?$DN?5?8?$CFs?8?$CJ@ 320bec94     EntityPool.obj
 0002:0000acb8       ??_C@_0HB@GKHJAPGB@?$FLEntity?5Pool?$FN?5Pool?5?8?$CFs?8?5has?5reac@ 320becb8     EntityPool.obj
 0002:0000ad30       ??_C@_0HG@HDJCFBMJ@?$FLEntity?5Pool?$FN?5Pool?5?8?$CFs?8?5was?5too?5@ 320bed30     EntityPool.obj
 0002:0000ada8       ??_C@_0BP@JLDMMOJD@CEntityPool?3?3GetEntityFromPool?$AA@ 320beda8     EntityPool.obj
 0002:0000adc8       __real@418c0000            320bedc8     EntityPoolDefinition.obj
 0002:0000adcc       ??_C@_0P@JKOMJFJC@?$CFs?5?$CIMax?3?5?$CFu?$CJ?$CFs?$AA@ 320bedcc     EntityPoolDefinition.obj
 0002:0000addc       ??_C@_09HEMHKAGH@?5?$FLFORCED?$FN?$AA@ 320beddc     EntityPoolDefinition.obj
 0002:0000ade8       ??_C@_0GN@ILOHJFJE@?$FLEntity?5Pool?$FN?5LoadFromXml?3?5?8Cont@ 320bede8     EntityPoolDefinition.obj
 0002:0000ae58       ??_C@_0ED@JEHGENBD@?$FLEntity?5Pool?$FN?5LoadFromXml?3?5Class@ 320bee58     EntityPoolDefinition.obj
 0002:0000aea0       ??_C@_0GC@MPGCJGO@?$FLEntity?5Pool?$FN?5LoadFromXml?3?5?8Cont@ 320beea0     EntityPoolDefinition.obj
 0002:0000af04       ??_C@_08BIDPDEIA@Contains?$AA@ 320bef04     EntityPoolDefinition.obj
 0002:0000af10       ??_C@_0BB@JKGGGDFI@forcedBookmarked?$AA@ 320bef10     EntityPoolDefinition.obj
 0002:0000af24       ??_C@_0BC@BGPCHCFM@defaultBookmarked?$AA@ 320bef24     EntityPoolDefinition.obj
 0002:0000af38       ??_C@_07GDPCCCPH@maxSize?$AA@ 320bef38     EntityPoolDefinition.obj
 0002:0000af40       ??_C@_05CHKBJBFP@hasAI?$AA@ 320bef40     EntityPoolDefinition.obj
 0002:0000af48       ??_C@_0DN@BJOGDOOH@?$FLEntity?5Pool?$FN?5LoadFromXml?3?5?8empt@ 320bef48     EntityPoolDefinition.obj
 0002:0000af88       ??_C@_0L@DEJKLMDK@emptyClass?$AA@ 320bef88     EntityPoolDefinition.obj
 0002:0000af94       ??_C@_0CD@OIDLEJD@CEntityPoolDefinition?3?3LoadFromX@ 320bef94     EntityPoolDefinition.obj
 0002:0000afb8       ??_C@_0DA@IFFGAEIA@CEntityPoolDefinition?3?3TestEntit@ 320befb8     EntityPoolDefinition.obj
 0002:0000afe8       ??_C@_0BI@LNMANPBF@OnEntityBookmarkCreated?$AA@ 320befe8     EntityPoolManager.obj
 0002:0000b000       ??_C@_0BG@KLICCAEM@GetReturnToPoolWeight?$AA@ 320bf000     EntityPoolManager.obj
 0002:0000b018       ??_C@_0BC@FBLLFHEI@BookmarkLastState?$AA@ 320bf018     EntityPoolManager.obj
 0002:0000b02c       ??_C@_0BA@JLDALONP@EntityPools?4xml?$AA@ 320bf02c     EntityPoolManager.obj
 0002:0000b03c       ??_C@_0CL@ILDEGBBB@Scripts?1Entities?1EntityPoolDefin@ 320bf03c     EntityPoolManager.obj
 0002:0000b06c       ??_7IEntityPoolManager@@6B@ 320bf06c     EntityPoolManager.obj
 0002:0000b0a0       ??_C@_0L@LFFADMLN@bIsDynamic?$AA@ 320bf0a0     EntityPoolManager.obj
 0002:0000b0ac       ??_C@_09IDFGMDMG@bCallInit?$AA@ 320bf0ac     EntityPoolManager.obj
 0002:0000b0b8       ??_C@_0M@EBAPDAGO@forcePoolId?$AA@ 320bf0b8     EntityPoolManager.obj
 0002:0000b0c4       ??_C@_07LEAAGLHO@Request?$AA@ 320bf0c4     EntityPoolManager.obj
 0002:0000b0cc       ??_C@_0CK@EJFBMCN@CEntityPoolManager?3?3GetReturnToP@ 320bf0cc     EntityPoolManager.obj
 0002:0000b0f8       ??_C@_0CC@LDHNAKMM@CEntityPoolManager?3?3GetPoolEntit@ 320bf0f8     EntityPoolManager.obj
 0002:0000b11c       ??_C@_0M@EADFAGLD@Definitions?$AA@ 320bf11c     EntityPoolManager.obj
 0002:0000b128       ??_C@_05HPELEJBD@Pools?$AA@ 320bf128     EntityPoolManager.obj
 0002:0000b130       ??_C@_0CG@OGBMNCLG@CEntityPoolManager?3?3OnPoolEntity@ 320bf130     EntityPoolManager.obj
 0002:0000b158       ??_C@_0BI@LNIHPNP@Bookmarked?5Entities?3?5?$CFu?$AA@ 320bf158     EntityPoolManager.obj
 0002:0000b170       __real@41900000            320bf170     EntityPoolManager.obj
 0002:0000b174       ??_C@_0BF@IAEGBKJN@Total?5Pool?5Count?3?5?$CFu?$AA@ 320bf174     EntityPoolManager.obj
 0002:0000b18c       ??_C@_0BH@JBEECMAB@Logged?5?8?$CFu?8?5bookmarks?4?$AA@ 320bf18c     EntityPoolManager.obj
 0002:0000b1a4       ??_C@_0BH@HLKPLFOC@?$CFs?1Bookmarks?1?$CFs?1?$CFs?4xml?$AA@ 320bf1a4     EntityPoolManager.obj
 0002:0000b1bc       ??_C@_06PHOHJIND@?$CFUSER?$CF?$AA@ 320bf1bc     EntityPoolManager.obj
 0002:0000b1c4       ??_C@_07DLHMCMEP@NoLevel?$AA@ 320bf1c4     EntityPoolManager.obj
 0002:0000b1cc       ??_C@_0BO@BDNDHAEF@Has?5Static?5Instanced?5Data?3?5?$CFs?$AA@ 320bf1cc     EntityPoolManager.obj
 0002:0000b1ec       ??_C@_0BF@JOCMKILD@Memory?5Footprint?3?5?$CFu?$AA@ 320bf1ec     EntityPoolManager.obj
 0002:0000b204       ??_C@_0BJ@PJBNKGLG@Has?5Serialized?5State?3?5?$CFs?$AA@ 320bf204     EntityPoolManager.obj
 0002:0000b220       ??_C@_0BC@CMJNDHPN@Static?5Entity?3?5?$CFs?$AA@ 320bf220     EntityPoolManager.obj
 0002:0000b234       ??_C@_0BH@JDHDAIDD@Has?5?$CCNo?5Save?$CC?5flag?3?5?$CFs?$AA@ 320bf234     EntityPoolManager.obj
 0002:0000b24c       ??_C@_02JINPPBEP@No?$AA@   320bf24c     EntityPoolManager.obj
 0002:0000b250       ??_C@_03CCLAEDDF@Yes?$AA@  320bf250     EntityPoolManager.obj
 0002:0000b254       ??_C@_0BA@NMJMNMEA@Reserved?5Id?3?5?$CFu?$AA@ 320bf254     EntityPoolManager.obj
 0002:0000b264       ??_C@_09OOOPONEB@Class?3?5?$CFs?$AA@ 320bf264     EntityPoolManager.obj
 0002:0000b270       ??_C@_09IOKHABFE@Layer?3?5?$CFs?$AA@ 320bf270     EntityPoolManager.obj
 0002:0000b27c       ??_C@_0L@FHIOMHBJ@_No?5Layer_?$AA@ 320bf27c     EntityPoolManager.obj
 0002:0000b288       ??_C@_08NAIIIBAK@Name?3?5?$CFs?$AA@ 320bf288     EntityPoolManager.obj
 0002:0000b294       ??_C@_09KPDPELDN@_No?5Name_?$AA@ 320bf294     EntityPoolManager.obj
 0002:0000b2a0       ??_C@_0CA@ENHLMEJN@Dumping?5all?5entity?5bookmarks?4?4?4?$AA@ 320bf2a0     EntityPoolManager.obj
 0002:0000b2c0       ??_C@_0CO@MCJNEBNF@Dumping?5entity?5bookmarks?5that?5co@ 320bf2c0     EntityPoolManager.obj
 0002:0000b2f0       ??_C@_04ILJKNBN@guid?$AA@  320bf2f0     EntityPoolManager.obj
 0002:0000b2f8       ??_C@_0L@LEIPJILE@sArchetype?$AA@ 320bf2f8     EntityPoolManager.obj
 0002:0000b304       ??_C@_06LLCCGEOD@sClass?$AA@ 320bf304     EntityPoolManager.obj
 0002:0000b30c       ??_C@_0L@CMIBPMME@sLayerName?$AA@ 320bf30c     EntityPoolManager.obj
 0002:0000b318       ??_C@_05PPFHJAOM@sName?$AA@ 320bf318     EntityPoolManager.obj
 0002:0000b320       ??_C@_0M@ENJDMDBH@DynamicInfo?$AA@ 320bf320     EntityPoolManager.obj
 0002:0000b32c       ??_C@_0DC@DLDEEFCO@?$FLEntity?5Pool?$FN?5Failed?5when?5creati@ 320bf32c     EntityPoolManager.obj
 0002:0000b360       ??_C@_0EO@CNHJEHNK@Creating?5entity?5pool?5for?5?8?$CFs?8?5?$CId@ 320bf360     EntityPoolManager.obj
 0002:0000b3b0       ??_C@_0BK@BFAHJMNL@Preparing?5entity?5pools?4?4?4?$AA@ 320bf3b0     EntityPoolManager.obj
 0002:0000b3cc       ??_C@_0CB@LJHFBDNL@CEntityPoolManager?3?3PreparePools@ 320bf3cc     EntityPoolManager.obj
 0002:0000b3f0       ??_C@_07IICMJPKE@Proxies?$AA@ 320bf3f0     EntityPoolManager.obj
 0002:0000b3f8       ??_C@_07ECEMPDJM@General?$AA@ 320bf3f8     EntityPoolManager.obj
 0002:0000b400       ??_C@_0L@CDABPFGM@Definition?$AA@ 320bf400     EntityPoolManager.obj
 0002:0000b40c       ??_C@_0BG@MBCFGJKC@EntityPoolDefinitions?$AA@ 320bf40c     EntityPoolManager.obj
 0002:0000b424       ??_C@_0CE@HFGMPMBK@CEntityPoolManager?3?3LoadDefiniti@ 320bf424     EntityPoolManager.obj
 0002:0000b448       ??_C@_0FM@FEMPGOAK@SerializeBookmarkEntity?3?5Failed?5@ 320bf448     EntityPoolManager.obj
 0002:0000b4a8       ??_C@_0FM@IKLNIHCH@SerializeBookmarkEntity?3?5Failed?5@ 320bf4a8     EntityPoolManager.obj
 0002:0000b504       ??_C@_0BG@DGPMJCIE@Serialize?5Bookmark?5?$CFs?$AA@ 320bf504     EntityPoolManager.obj
 0002:0000b51c       ??_C@_0DG@HFCEFPMP@?$FLEntity?5Pool?$FN?5Failed?5to?5load?5Poo@ 320bf51c     EntityPoolManager.obj
 0002:0000b554       ??_C@_0BL@LAKELMDA@Prepare?5Static?5Bookmark?5?$CFs?$AA@ 320bf554     EntityPoolManager.obj
 0002:0000b570       ??_C@_0CL@MBDHPBLC@CEntityPoolManager?3?3LoadBookmark@ 320bf570     EntityPoolManager.obj
 0002:0000b59c       ??_C@_0BM@EIPIHGFK@Prepare?5Dynamic?5Bookmark?5?$CFs?$AA@ 320bf59c     EntityPoolManager.obj
 0002:0000b5b8       ??_C@_0CI@EELEKODJ@CEntityPoolManager?3?3LoadDynamicF@ 320bf5b8     EntityPoolManager.obj
 0002:0000b5e0       ??_C@_0CL@ECNAECMN@CEntityPoolManager?3?3PrepareDynam@ 320bf5e0     EntityPoolManager.obj
 0002:0000b60c       ??_C@_0BD@FBHGCBJO@Return?5Bookmark?5?$CFs?$AA@ 320bf60c     EntityPoolManager.obj
 0002:0000b620       ??_C@_0CE@FMIDMINK@CEntityPoolManager?3?3PrepareFromP@ 320bf620     EntityPoolManager.obj
 0002:0000b644       ??_C@_07DHDGIPKD@RootSID?$AA@ 320bf644     EntityPoolManager.obj
 0002:0000b64c       ??_C@_0BA@MIDAKKDO@Add?5Bookmark?5?$CFs?$AA@ 320bf64c     EntityPoolManager.obj
 0002:0000b65c       ??_C@_0CE@KCLJMMPI@CEntityPoolManager?3?3AddPoolBookm@ 320bf65c     EntityPoolManager.obj
 0002:0000b680       ??_7CEntityPoolManager@@6B@ 320bf680     EntityPoolManager.obj
 0002:0000b6b4       ??_C@_05GNKDLNNI@uSize?$AA@ 320bf6b4     EntityPoolManager.obj
 0002:0000b6bc       ??_C@_0BG@PBNONJFP@m_PrepareRequestQueue?$AA@ 320bf6bc     EntityPoolManager.obj
 0002:0000b6d4       ??_C@_0L@IINPOMLJ@aiObjectId?$AA@ 320bf6d4     EntityPoolManager.obj
 0002:0000b6e0       ??_C@_0M@DBJJFIOK@savedPoolId?$AA@ 320bf6e0     EntityPoolManager.obj
 0002:0000b6ec       ??_C@_0L@IKFBOGBE@bookmarkId?$AA@ 320bf6ec     EntityPoolManager.obj
 0002:0000b6f8       ??_C@_08MMNAJMJK@Bookmark?$AA@ 320bf6f8     EntityPoolManager.obj
 0002:0000b704       ??_C@_0BE@EBCOCGME@numBookmarksDynamic?$AA@ 320bf704     EntityPoolManager.obj
 0002:0000b718       ??_C@_0BD@PIHBFFPN@numBookmarksStatic?$AA@ 320bf718     EntityPoolManager.obj
 0002:0000b72c       ??_C@_0BM@HFALIMIO@EntityPoolManager_Bookmarks?$AA@ 320bf72c     EntityPoolManager.obj
 0002:0000b748       ??_C@_0BE@MLGDHEEN@EntityPoolSignature?$AA@ 320bf748     EntityPoolSignature.obj
 0002:0000b75c       ??_C@_0CK@OKLMBKBM@CEntityPoolSignature?3?3CalculateF@ 320bf75c     EntityPoolSignature.obj
 0002:0000b788       ??_C@_0CM@JMBOLPHF@CEntityPoolSignature?3?3CompareNod@ 320bf788     EntityPoolSignature.obj
 0002:0000b7b4       ??_C@_0CD@DPNACMCM@CEntityPoolSignature?3?3CompareNod@ 320bf7b4     EntityPoolSignature.obj
 0002:0000b7d8       ??_C@_0CH@JAHNPBAG@CEntityPoolSignature?3?3CompareSig@ 320bf7d8     EntityPoolSignature.obj
 0002:0000b800       __pDefaultRawDllMain       320bf800     MSVCRT:crtdll.obj
 0002:0000b800       __pRawDllMain              320bf800     MSVCRT:crtdll.obj
 0002:0000b810       __load_config_used         320bf810     MSVCRT:loadcfg.obj
 0002:0000b8c0       ___safe_se_handler_table   320bf8c0     <linker-defined>
 0002:0000b8c4       ___rtc_iaa                 320bf8c4     MSVCRT:_initsect_.obj
 0002:0000b8c8       ___rtc_izz                 320bf8c8     MSVCRT:_initsect_.obj
 0002:0000b8cc       ___rtc_taa                 320bf8cc     MSVCRT:_initsect_.obj
 0002:0000b8d0       ___rtc_tzz                 320bf8d0     MSVCRT:_initsect_.obj
 0002:0000b93c       __IMPORT_DESCRIPTOR_KERNEL32 320bf93c     kernel32:KERNEL32.dll
 0002:0000b950       __IMPORT_DESCRIPTOR_USER32 320bf950     user32:USER32.dll
 0002:0000b964       __IMPORT_DESCRIPTOR_MSVCR100 320bf964     MSVCRT:MSVCR100.dll
 0002:0000b978       __NULL_IMPORT_DESCRIPTOR   320bf978     kernel32:KERNEL32.dll
 0003:0000005c       ?fVec3_Zero@?$Vec3Constants@M@@2U?$Vec3_tpl@M@@B 320c105c     BreakablePlane.obj
 0003:00000068       ?fVec3_One@?$Vec3Constants@M@@2U?$Vec3_tpl@M@@B 320c1068     BreakablePlane.obj
 0003:00000078       ?m_seed@CLCGRndGen@@0_KA   320c1078     CryEntityDLL.obj
 0003:00000084       ?sEmptyStringBuffer@?1??_emptyHeader@?$CryStringT@D@@KAPAUStrHeader@2@XZ@4PAU32@A 320c1084     CryEntityDLL.obj
 0003:000000a0       ?s_eventsName@@3PAUSEventName@@A 320c10a0     Entity.obj
 0003:00000208       ?m_szDescription@CEntity@@0V?$CryStringT@D@@A 320c1208     Entity.obj
 0003:0000020c       ?es_UsePhysVisibilityChecks@CVar@@2HA 320c120c     EntityCVars.obj
 0003:00000210       ?es_DebugEntityUsageFilter@CVar@@2PBDB 320c1210     EntityCVars.obj
 0003:00000214       ?es_DebugPoolFilter@CVar@@2PBDB 320c1214     EntityCVars.obj
 0003:00000218       ?es_SaveLoadUseLUANoSaveFlag@CVar@@2HA 320c1218     EntityCVars.obj
 0003:0000021c       ?es_ClearPoolBookmarksOnLayerUnload@CVar@@2HA 320c121c     EntityCVars.obj
 0003:00000268       ?fVec2_Zero@?$Vec2Constants@M@@2U?$Vec2_tpl@M@@A 320c1268     stdafx.obj
 0003:00000270       ?fVec2_OneX@?$Vec2Constants@M@@2U?$Vec2_tpl@M@@A 320c1270     stdafx.obj
 0003:00000278       ?fVec2_OneY@?$Vec2Constants@M@@2U?$Vec2_tpl@M@@A 320c1278     stdafx.obj
 0003:00000280       ?fVec2_One@?$Vec2Constants@M@@2U?$Vec2_tpl@M@@A 320c1280     stdafx.obj
 0003:00000390       ?fVec3_OneX@?$Vec3Constants@M@@2U?$Vec3_tpl@M@@B 320c1390     ScriptBind_Entity.obj
 0003:0000039c       ?g_lastReceivedEventId@@3HA 320c139c     PhysicsEventListener.obj
 0003:000003a0       ?g_lastExecutedEventId@@3HA 320c13a0     PhysicsEventListener.obj
 0003:000003ac       ?s_fViewDistRatio@CRenderProxy@@0MA 320c13ac     RenderProxy.obj
 0003:000003b0       ?s_fViewDistRatioCustom@CRenderProxy@@0MA 320c13b0     RenderProxy.obj
 0003:000003b4       ?s_fViewDistRatioDetail@CRenderProxy@@0MA 320c13b4     RenderProxy.obj
 0003:000003c0       ?s_bitFieldSizeU32@CAreaBitField@@1IA 320c13c0     AreaGrid.obj
 0003:000003c4       ?s_maxNumAreas@CAreaBitField@@1IA 320c13c4     AreaGrid.obj
 0003:000003d0       ?auto_unittest_instance_CUT_PartitionGrid@@3VCUT_PartitionGrid@@A 320c13d0     PartitionGrid.obj
 0003:00000420       ___native_dllmain_reason   320c1420     MSVCRT:natstart.obj
 0003:00000424       ___native_vcclrit_reason   320c1424     MSVCRT:natstart.obj
 0003:00000428       ___security_cookie         320c1428     MSVCRT:gs_cookie.obj
 0003:0000042c       ___security_cookie_complement 320c142c     MSVCRT:gs_cookie.obj
 0003:00000430       ?s_pMemReplay@?1??CryGetIMemReplay@@YAPAUIMemReplay@@XZ@4PAU2@A 320c1430     AreaSolid.obj
 0003:00000434       ?s_dummyMemReplay@?1??CryGetIMemReplay@@YAPAUIMemReplay@@XZ@4UCDummyMemReplay@@A 320c1434     AreaSolid.obj
 0003:00000438       ??_B?1??CryGetIMemReplay@@YAPAUIMemReplay@@XZ@51 320c1438     AreaSolid.obj
 0003:0000043c       ?g_nPieces@CBreakablePlane@@2HA 320c143c     BreakablePlane.obj
 0003:00000440       ?g_maxPieceLifetime@CBreakablePlane@@2MA 320c1440     BreakablePlane.obj
 0003:00000444       ?s_EmptyElems@?1??set_null@?$SmallDynStorage@U?$SplineKey@M@spline@@HUStandardAlloc@NAlloc@@@NArray@@IAEXXZ@4PAU?$SplineKey@M@spline@@A 320c1444     BreakablePlane.obj
 0003:00000448       ?s_EmptyHeader@?1??set_null@?$SmallDynStorage@U?$SplineKey@M@spline@@HUStandardAlloc@NAlloc@@@NArray@@IAEXXZ@4UEmptyHeader@23@A 320c1448     BreakablePlane.obj
 0003:00000450       ??_B?1??set_null@?$SmallDynStorage@U?$SplineKey@M@spline@@HUStandardAlloc@NAlloc@@@NArray@@IAEXXZ@51 320c1450     BreakablePlane.obj
 0003:000007d4       ?numAllocations@_CryMemoryManagerPoolHelper@@2HC 320c17d4     CryEntityDLL.obj
 0003:000007d8       ?requestedMemory@_CryMemoryManagerPoolHelper@@2JC 320c17d8     CryEntityDLL.obj
 0003:000007dc       ?freedMemory@_CryMemoryManagerPoolHelper@@2JC 320c17dc     CryEntityDLL.obj
 0003:000007e0       ?allocatedMemory@_CryMemoryManagerPoolHelper@@2JC 320c17e0     CryEntityDLL.obj
 0003:000007e4       ?gEnv@@3PAUSSystemGlobalEnvironment@@A 320c17e4     CryEntityDLL.obj
 0003:000007e8       ?m_pFirst@Test@CryUnitTest@@2PAU12@A 320c17e8     CryEntityDLL.obj
 0003:000007ec       ?m_pLast@Test@CryUnitTest@@2PAU12@A 320c17ec     CryEntityDLL.obj
 0003:000007f0       ?g_pHeadToRegFactories@@3PAUSRegFactoryNode@@A 320c17f0     CryEntityDLL.obj
 0003:000007f4       ?g_bProfilerEnabled@@3_NA  320c17f4     CryEntityDLL.obj
 0003:000007f8       ?g_iTraceAllocations@@3HA  320c17f8     CryEntityDLL.obj
 0003:000007fc       ?_CryMalloc@_CryMemoryManagerPoolHelper@@2P6APAXIAAII@ZA 320c17fc     CryEntityDLL.obj
 0003:00000800       ?_CryGetMemSize@_CryMemoryManagerPoolHelper@@2P6AIPAXI@ZA 320c1800     CryEntityDLL.obj
 0003:00000804       ?_CryRealloc@_CryMemoryManagerPoolHelper@@2P6APAXPAXIAAI1I@ZA 320c1804     CryEntityDLL.obj
 0003:00000808       ?_CryFree@_CryMemoryManagerPoolHelper@@2P6AIPAXI@ZA 320c1808     CryEntityDLL.obj
 0003:0000080c       ?_CryCrtMalloc@_CryMemoryManagerPoolHelper@@2P6APAXI@ZA 320c180c     CryEntityDLL.obj
 0003:00000810       ?_CryCrtRealloc@_CryMemoryManagerPoolHelper@@2P6APAXPAXI@ZA 320c1810     CryEntityDLL.obj
 0003:00000814       ?_CryCrtFree@_CryMemoryManagerPoolHelper@@2P6AIPAX@ZA 320c1814     CryEntityDLL.obj
 0003:00000818       ?_CryCrtSize@_CryMemoryManagerPoolHelper@@2P6AIPAX@ZA 320c1818     CryEntityDLL.obj
 0003:0000081c       ?_CryGetIMemoryManagerInterface@_CryMemoryManagerPoolHelper@@2P6AXPAPAX@ZA 320c181c     CryEntityDLL.obj
 0003:00000820       ?m_bInitialized@_CryMemoryManagerPoolHelper@@2HA 320c1820     CryEntityDLL.obj
 0003:00000824       ?g_pIEntitySystem@@3PAVCEntitySystem@@A 320c1824     CryEntityDLL.obj
 0003:00000828       ?g_random_generator@@3VCLCGRndGen@@A 320c1828     CryEntityDLL.obj
 0003:0000082c       ?s_factory@CFactory@CEngineModule_EntitySystem@@0V12@A 320c182c     CryEntityDLL.obj
 0003:0000085c       ?s_used_memory@?1??_usedMemory@?$CryStringT@_W@@SAIH@Z@4IA 320c185c     CryEntityDLL.obj
 0003:00000860       ?s_used_memory@?1??_usedMemory@?$CryStackStringT@D$0BA@@@SAII@Z@4IA 320c1860     CryEntityDLL.obj
 0003:00000864       ?s_used_memory@?1??_usedMemory@?$CryStackStringT@D$0BAA@@@SAII@Z@4IA 320c1864     CryEntityDLL.obj
 0003:00000868       ?s_used_memory@?1??_usedMemory@?$CryStringT@D@@SAIH@Z@4IA 320c1868     CryEntityDLL.obj
 0003:00000880       ?supportedIIDs@?1???0CFactory@CEngineModule_EntitySystem@@AAE@XZ@4PAUCryGUID@@A 320c1880     CryEntityDLL.obj
 0003:000008d0       ?p@?1??CreateClassInstance@CFactory@CEngineModule_EntitySystem@@UBE?AV?$shared_ptr@UICryUnknown@@@boost@@XZ@4V?$shared_ptr@VCEngineModule_EntitySystem@@@5@A 320c18d0     CryEntityDLL.obj
 0003:000008d8       ??_B?1??CreateClassInstance@CFactory@CEngineModule_EntitySystem@@UBE?AV?$shared_ptr@UICryUnknown@@@boost@@XZ@51 320c18d8     CryEntityDLL.obj
 0003:000016c4       ?sIdentityMatrix@?A0x9962e041@@3U?$Matrix34_tpl@M@@A 320c26c4     Entity.obj
 0003:000016f4       ?s_EmptyElems@?1??set_null@?$SmallDynStorage@V?$CryStringT@D@@HUStandardAlloc@NAlloc@@@NArray@@IAEXXZ@4PAV?$CryStringT@D@@A 320c26f4     EntityArchetype.obj
 0003:000016f8       ?s_EmptyHeader@?1??set_null@?$SmallDynStorage@V?$CryStringT@D@@HUStandardAlloc@NAlloc@@@NArray@@IAEXXZ@4UEmptyHeader@23@A 320c26f8     EntityArchetype.obj
 0003:00001700       ??_B?1??set_null@?$SmallDynStorage@V?$CryStringT@D@@HUStandardAlloc@NAlloc@@@NArray@@IAEXXZ@51 320c2700     EntityArchetype.obj
 0003:00001704       ?es_FarPhysTimeout@CVar@@2MA 320c2704     EntityCVars.obj
 0003:00001708       ?es_MaxPhysDistCloth@CVar@@2MA 320c2708     EntityCVars.obj
 0003:0000170c       ?es_MaxPhysDistInvisible@CVar@@2MA 320c270c     EntityCVars.obj
 0003:00001710       ?es_MaxPhysDist@CVar@@2MA  320c2710     EntityCVars.obj
 0003:00001714       ?pDebug@CVar@@2PAUICVar@@A 320c2714     EntityCVars.obj
 0003:00001718       ?pCharacterIK@CVar@@2PAUICVar@@A 320c2718     EntityCVars.obj
 0003:0000171c       ?pProfileEntities@CVar@@2PAUICVar@@A 320c271c     EntityCVars.obj
 0003:00001720       ?pUpdateScript@CVar@@2PAUICVar@@A 320c2720     EntityCVars.obj
 0003:00001724       ?pUpdateTimer@CVar@@2PAUICVar@@A 320c2724     EntityCVars.obj
 0003:00001728       ?pUpdateCamera@CVar@@2PAUICVar@@A 320c2728     EntityCVars.obj
 0003:0000172c       ?pUpdatePhysics@CVar@@2PAUICVar@@A 320c272c     EntityCVars.obj
 0003:00001730       ?pUpdateAI@CVar@@2PAUICVar@@A 320c2730     EntityCVars.obj
 0003:00001734       ?pUpdateEntities@CVar@@2PAUICVar@@A 320c2734     EntityCVars.obj
 0003:00001738       ?pUpdateCollision@CVar@@2PAUICVar@@A 320c2738     EntityCVars.obj
 0003:0000173c       ?pUpdateCollisionScript@CVar@@2PAUICVar@@A 320c273c     EntityCVars.obj
 0003:00001740       ?pUpdateContainer@CVar@@2PAUICVar@@A 320c2740     EntityCVars.obj
 0003:00001744       ?pUpdateCoocooEgg@CVar@@2PAUICVar@@A 320c2744     EntityCVars.obj
 0003:00001748       ?pPiercingCamera@CVar@@2PAUICVar@@A 320c2748     EntityCVars.obj
 0003:0000174c       ?pVisCheckForUpdate@CVar@@2PAUICVar@@A 320c274c     EntityCVars.obj
 0003:00001750       ?pEntityBBoxes@CVar@@2PAUICVar@@A 320c2750     EntityCVars.obj
 0003:00001754       ?pEntityHelpers@CVar@@2PAUICVar@@A 320c2754     EntityCVars.obj
 0003:00001758       ?pMinImpulseVel@CVar@@2PAUICVar@@A 320c2758     EntityCVars.obj
 0003:0000175c       ?pImpulseScale@CVar@@2PAUICVar@@A 320c275c     EntityCVars.obj
 0003:00001760       ?pMaxImpulseAdjMass@CVar@@2PAUICVar@@A 320c2760     EntityCVars.obj
 0003:00001764       ?pDebrisLifetimeScale@CVar@@2PAUICVar@@A 320c2764     EntityCVars.obj
 0003:00001768       ?pSplashThreshold@CVar@@2PAUICVar@@A 320c2768     EntityCVars.obj
 0003:0000176c       ?pSplashTimeout@CVar@@2PAUICVar@@A 320c276c     EntityCVars.obj
 0003:00001770       ?pHitCharacters@CVar@@2PAUICVar@@A 320c2770     EntityCVars.obj
 0003:00001774       ?pHitDeadBodies@CVar@@2PAUICVar@@A 320c2774     EntityCVars.obj
 0003:00001778       ?pCharZOffsetSpeed@CVar@@2PAUICVar@@A 320c2778     EntityCVars.obj
 0003:0000177c       ?pEnableFullScriptSave@CVar@@2PAUICVar@@A 320c277c     EntityCVars.obj
 0003:00001780       ?pLogCollisions@CVar@@2PAUICVar@@A 320c2780     EntityCVars.obj
 0003:00001784       ?pNotSeenTimeout@CVar@@2PAUICVar@@A 320c2784     EntityCVars.obj
 0003:00001788       ?pDebugNotSeenTimeout@CVar@@2PAUICVar@@A 320c2788     EntityCVars.obj
 0003:0000178c       ?pDrawAreas@CVar@@2PAUICVar@@A 320c278c     EntityCVars.obj
 0003:00001790       ?pDrawAreaGrid@CVar@@2PAUICVar@@A 320c2790     EntityCVars.obj
 0003:00001794       ?pDrawAreaDebug@CVar@@2PAUICVar@@A 320c2794     EntityCVars.obj
 0003:00001798       ?pDrawSoundProxyZRay@CVar@@2PAUICVar@@A 320c2798     EntityCVars.obj
 0003:0000179c       ?pMotionBlur@CVar@@2PAUICVar@@A 320c279c     EntityCVars.obj
 0003:000017a0       ?pSysSpecLight@CVar@@2PAUICVar@@A 320c27a0     EntityCVars.obj
 0003:000017a4       ?es_DebugTimers@CVar@@2HA  320c27a4     EntityCVars.obj
 0003:000017a8       ?es_DebugFindEntity@CVar@@2HA 320c27a8     EntityCVars.obj
 0003:000017ac       ?es_DebugEvents@CVar@@2HA  320c27ac     EntityCVars.obj
 0003:000017b0       ?es_SortUpdatesByClass@CVar@@2HA 320c27b0     EntityCVars.obj
 0003:000017b4       ?es_debugEntityLifetime@CVar@@2HA 320c27b4     EntityCVars.obj
 0003:000017b8       ?es_DisableTriggers@CVar@@2HA 320c27b8     EntityCVars.obj
 0003:000017bc       ?es_DrawProximityTriggers@CVar@@2HA 320c27bc     EntityCVars.obj
 0003:000017c0       ?es_DebugEntityUsage@CVar@@2HA 320c27c0     EntityCVars.obj
 0003:000017c4       ?es_EnablePoolUse@CVar@@2HA 320c27c4     EntityCVars.obj
 0003:000017c8       ?es_DebugPool@CVar@@2HA    320c27c8     EntityCVars.obj
 0003:000017cc       ?es_TestPoolSignatures@CVar@@2HA 320c27cc     EntityCVars.obj
 0003:000017d0       ?es_LayerSaveLoadSerialization@CVar@@2HA 320c27d0     EntityCVars.obj
 0003:000017d4       ?es_LayerDebugInfo@CVar@@2HA 320c27d4     EntityCVars.obj
 0003:000017d8       ?pUpdateType@CVar@@2PAUICVar@@A 320c27d8     EntityCVars.obj
 0003:000017dc       ?serializeString@?1??SetSharedSerializeString@?$CSerializeWrapper@UISerialize@@@@QAEAAUSSerializeString@@ABV?$CryStringT@D@@@Z@4U3@A 320c27dc     EntityLayer.obj
 0003:000017e0       ??_B?1??SetSharedSerializeString@?$CSerializeWrapper@UISerialize@@@@QAEAAUSSerializeString@@ABV?$CryStringT@D@@@Z@51 320c27e0     EntityLayer.obj
 0003:000017f0       ?g_Alloc_RenderProxy@@3PAV?$PoolAllocatorNoMT@$0LA@$0A@@stl@@A 320c27f0     EntitySystem.obj
 0003:000017f4       ?g_Alloc_EntitySlot@@3PAV?$PoolAllocatorNoMT@$0JI@$0A@@stl@@A 320c27f4     EntitySystem.obj
 0003:00002604       ?allocator@?$STLPoolAllocatorStatic@$0CI@UPSyncNone@stl@@$0A@$0A@U?$_Rb_tree_node@U?$pair@$$CBVCTimeValue@@USEntityTimerEvent@@@stlpmtx_std@@@priv@stlpmtx_std@@@stl@@2PAV?$SizePoolAllocator@V?$HeapAllocator@UPSyncNone@stl@@$00VGlobalHeapSysAllocator@2@@stl@@@2@A 320c3604     EntitySystem.obj
 0003:0000377c       ?s_EmptyElems@?1??set_null@?$SmallDynStorage@VCEntry@CEntityTimeoutList@@HUStandardAlloc@NAlloc@@@NArray@@IAEXXZ@4PAVCEntry@CEntityTimeoutList@@A 320c477c     EntityTimeoutList.obj
 0003:00003780       ?s_EmptyHeader@?1??set_null@?$SmallDynStorage@VCEntry@CEntityTimeoutList@@HUStandardAlloc@NAlloc@@@NArray@@IAEXXZ@4UEmptyHeader@23@A 320c4780     EntityTimeoutList.obj
 0003:00003788       ??_B?1??set_null@?$SmallDynStorage@VCEntry@CEntityTimeoutList@@HUStandardAlloc@NAlloc@@@NArray@@IAEXXZ@51 320c4788     EntityTimeoutList.obj
 0003:00003790       ?g_globalSections@?$Node_Alloc_Lock@$00$00@@2PAUInternalCriticalSectionDummy@@A 320c4790     stdafx.obj
 0003:00005810       ?m_bInitialized@?$Node_Alloc_Lock@$00$00@@2_NA 320c6810     stdafx.obj
 0003:00005814       ?s_EmptyElems@?1??set_null@?$SmallDynStorage@UGoalParams@@HUStandardAlloc@NAlloc@@@NArray@@IAEXXZ@4PAUGoalParams@@A 320c6814     ScriptBind_Entity.obj
 0003:00005818       ?s_EmptyHeader@?1??set_null@?$SmallDynStorage@UGoalParams@@HUStandardAlloc@NAlloc@@@NArray@@IAEXXZ@4UEmptyHeader@23@A 320c6818     ScriptBind_Entity.obj
 0003:00005820       ??_B?1??set_null@?$SmallDynStorage@UGoalParams@@HUStandardAlloc@NAlloc@@@NArray@@IAEXXZ@51 320c6820     ScriptBind_Entity.obj
 0003:000083f4       ?Info@?1??TypeInfo@?$TFixed@E$00$0PP@@@QBEABUCTypeInfo@@XZ@4UCCustomInfo@2@A 320c93f4     ScriptBind_Entity.obj
 0003:00008400       ??_B?1??TypeInfo@?$TFixed@E$00$0PP@@@QBEABUCTypeInfo@@XZ@51 320c9400     ScriptBind_Entity.obj
 0003:00008404       ?digits@?3??ToString@CCustomInfo@?$TFixed@E$00$0PP@@@UBE?AV?$CryStringT@D@@PBXUFToString@@0@Z@4HA 320c9404     ScriptBind_Entity.obj
 0003:00008408       ??_B?3??ToString@CCustomInfo@?$TFixed@E$00$0PP@@@UBE?AV?$CryStringT@D@@PBXUFToString@@0@Z@53 320c9408     ScriptBind_Entity.obj
 0003:0000840c       ?Info@?1??TypeInfo@?$SplineElem@U?$TFixed@E$00$0PP@@@@@QBEABUCTypeInfo@@XZ@4UCStructInfo@@A 320c940c     ScriptBind_Entity.obj
 0003:00008444       ?Vars@?1??TypeInfo@?$SplineElem@U?$TFixed@E$00$0PP@@@@@QBEABUCTypeInfo@@XZ@4PAUCVarInfo@3@A 320c9444     ScriptBind_Entity.obj
 0003:00008480       ??_B?1??TypeInfo@?$SplineElem@U?$TFixed@E$00$0PP@@@@@QBEABUCTypeInfo@@XZ@51 320c9480     ScriptBind_Entity.obj
 0003:00008484       ?Info@?1??TypeInfo@?$SplineElem@M@@QBEABUCTypeInfo@@XZ@4UCStructInfo@@A 320c9484     ScriptBind_Entity.obj
 0003:000084bc       ?Vars@?1??TypeInfo@?$SplineElem@M@@QBEABUCTypeInfo@@XZ@4PAUCVarInfo@3@A 320c94bc     ScriptBind_Entity.obj
 0003:000084f8       ??_B?1??TypeInfo@?$SplineElem@M@@QBEABUCTypeInfo@@XZ@51 320c94f8     ScriptBind_Entity.obj
 0003:00009308       ?g_meshPreps@@3PAVCDeferredMeshUpdatePrep@@A 320ca308     PhysicsEventListener.obj
 0003:00009990       ?s_EmptyElems@?1??set_null@?$SmallDynStorage@PAUIPhysicalEntity@@HUStandardAlloc@NAlloc@@@NArray@@IAEXXZ@4PAPAUIPhysicalEntity@@A 320ca990     PhysicsProxy.obj
 0003:00009994       ?s_EmptyHeader@?1??set_null@?$SmallDynStorage@PAUIPhysicalEntity@@HUStandardAlloc@NAlloc@@@NArray@@IAEXXZ@4UEmptyHeader@23@A 320ca994     PhysicsProxy.obj
 0003:0000999c       ??_B?1??set_null@?$SmallDynStorage@PAUIPhysicalEntity@@HUStandardAlloc@NAlloc@@@NArray@@IAEXXZ@51 320ca99c     PhysicsProxy.obj
 0003:0000a7a0       ?s_EmptyElems@?1??set_null@?$SmallDynStorage@U?$Vec3_tpl@M@@HUStandardAlloc@NAlloc@@@NArray@@IAEXXZ@4PAU?$Vec3_tpl@M@@A 320cb7a0     RopeProxy.obj
 0003:0000a7a4       ?s_EmptyHeader@?1??set_null@?$SmallDynStorage@U?$Vec3_tpl@M@@HUStandardAlloc@NAlloc@@@NArray@@IAEXXZ@4UEmptyHeader@23@A 320cb7a4     RopeProxy.obj
 0003:0000a7ac       ??_B?1??set_null@?$SmallDynStorage@U?$Vec3_tpl@M@@HUStandardAlloc@NAlloc@@@NArray@@IAEXXZ@51 320cb7ac     RopeProxy.obj
 0003:0000a7b8       ?sIdentMatrix@?A0xadbd02f3@@3U?$Matrix34_tpl@M@@A 320cb7b8     EntityObject.obj
 0003:0000a7e8       ?gsWaterLevel@CRenderProxy@@0MA 320cb7e8     RenderProxy.obj
 0003:0000a7ec       ?s_fViewDistMin@CRenderProxy@@0MA 320cb7ec     RenderProxy.obj
 0003:0000a7f0       ?s_pTimeoutList@CRenderProxy@@0PAVCEntityTimeoutList@@A 320cb7f0     RenderProxy.obj
 0003:0000af64       ?s_used_memory@?1??_usedMemory@?$CryStackStringT@D$0CAA@@@SAII@Z@4IA 320cbf64     AreaProxy.obj
 0003:0000af68       ?s_tmpWorldPoints@CAreaProxy@@0V?$vector@U?$Vec3_tpl@M@@V?$allocator@U?$Vec3_tpl@M@@@stlpmtx_std@@@stlpmtx_std@@A 320cbf68     AreaProxy.obj
 0003:0000afa0       ?s_pBitArrayMem@CAreaBitField@@1PAIA 320cbfa0     AreaGrid.obj
 0003:0000afa4       ?s_pBitArrayMemCurrent@CAreaBitField@@1PAIA 320cbfa4     AreaGrid.obj
 0003:0000afa8       ?s_nGridCells@CAreaBitField@@1IA 320cbfa8     AreaGrid.obj
 0003:0000afac       ?s_pAreaList@CAreaBitField@@1PAIA 320cbfac     AreaGrid.obj
 0003:0000afb0       ?s_pTempBitMem@CAreaBitField@@1PAIA 320cbfb0     AreaGrid.obj
 0003:0000ba1c       ?s_EmptyElems@?1??set_null@?$SmallDynStorage@MHUStandardAlloc@NAlloc@@@NArray@@IAEXXZ@4PAMA 320cca1c     BreakableManager.obj
 0003:0000ba20       ?s_EmptyHeader@?1??set_null@?$SmallDynStorage@MHUStandardAlloc@NAlloc@@@NArray@@IAEXXZ@4UEmptyHeader@23@A 320cca20     BreakableManager.obj
 0003:0000ba28       ??_B?1??set_null@?$SmallDynStorage@MHUStandardAlloc@NAlloc@@@NArray@@IAEXXZ@51 320cca28     BreakableManager.obj
 0003:0000ba2c       ?s_EmptyElems@?1??set_null@?$SmallDynStorage@UGeomQuery@@HUStandardAlloc@NAlloc@@@NArray@@IAEXXZ@4PAUGeomQuery@@A 320cca2c     BreakableManager.obj
 0003:0000ba30       ?s_EmptyHeader@?1??set_null@?$SmallDynStorage@UGeomQuery@@HUStandardAlloc@NAlloc@@@NArray@@IAEXXZ@4UEmptyHeader@23@A 320cca30     BreakableManager.obj
 0003:0000ba38       ??_B?1??set_null@?$SmallDynStorage@UGeomQuery@@HUStandardAlloc@NAlloc@@@NArray@@IAEXXZ@51 320cca38     BreakableManager.obj
 0003:0000bdd0       ?g_SectorGroupPoolAlloc@CPartitionGrid@@2PAV?$PoolAllocatorNoMT@$0EAE@$0A@@stl@@A 320ccdd0     PartitionGrid.obj
 0003:0000bdd4       ?g_GridLocationPoolAlloc@CPartitionGrid@@2PAV?$PoolAllocatorNoMT@$0BI@$0A@@stl@@A 320ccdd4     PartitionGrid.obj
 0003:0000bdd8       ?autoreg_unittest_CUT_PartitionGrid@@3VCAutoRegisterUnitTest@CryUnitTest@@A 320ccdd8     PartitionGrid.obj
 0003:0000c154       ?g_pProximityElement_PoolAlloc@CProximityTriggerSystem@@2PAV?$PoolAllocatorNoMT@$0CM@$0A@@stl@@A 320cd154     ProximityTriggerSystem.obj
 0003:00013070       ?__type_info_root_node@@3U__type_info_node@@A 320d4070     MSVCRT:tncleanup.obj
 0003:0001339c       ___native_startup_state    320d439c     <common>
 0003:000133a0       ___native_startup_lock     320d43a0     <common>
 0003:000133a4       ___sse2_available          320d43a4     <common>
 0003:000133a8       ___dyn_tls_init_callback   320d43a8     <common>
 0003:000133ac       ___onexitend               320d43ac     <common>
 0003:000133b0       ___onexitbegin             320d43b0     <common>
 0004:00000000       ?m_Self@CrySimpleThreadSelf@@1PAV1@A 320d5000     CryEntityDLL.obj

 entry point at        0001:000b1c4a

 Static symbols

 0001:00000000       ?find_max_col@@YAHQAY03M@Z 32001000 f   AffineParts.obj
 0001:00000100       ?Qt_FromMatrix@@YA?AUQuatern@@QAY03M@Z 32001100 f   AffineParts.obj
 0001:000002f0       ?make_reflector@@YAXPAM0@Z 320012f0 f   AffineParts.obj
 0001:000003a0       ?do_rank1@@YAXQAY03M0@Z    320013a0 f   AffineParts.obj
 0001:00000b30       ?do_rank2@@YAXQAY03M00@Z   32001b30 f   AffineParts.obj
 0001:00001170       ?polar_decomp@@YAMQAY03M00@Z 32002170 f   AffineParts.obj
 0001:00001c20       ?spect_decomp@@YA?AUQuatern@@QAY03M0@Z 32002c20 f   AffineParts.obj
 0001:00001f00       ?spectral_decomp_affine@@YAXQAY03MPAUSAffineParts@@@Z 32002f00 f   AffineParts.obj
 0001:00019690       ?VarFromString@@YAHABUCVarInfo@CTypeInfo@@PAXAAPBDUFFromString@@AAV?$CryStackStringT@D$0BAA@@@@Z 3201a690 f   CryEntityDLL.obj
 0001:000243e0       ?OnUpdateTypeChange@@YAXPAUICVar@@@Z 320253e0 f   EntityCVars.obj
 0001:000245d0       ?OnSysSpecLightChange@@YAXPAUICVar@@@Z 320255d0 f   EntityCVars.obj
 0001:00065ef0       ?ValidateSetParams@?A0x987469b6@@YAHPBUEventPhys@@@Z 32066ef0 f   PhysicsProxy.obj
 0001:00072b90       ??RRecurser@?1??CheckCharacterForMorphs@CRenderProxy@@AAE_NPAUICharacterInstance@@@Z@QAEX0@Z 32073b90 f   RenderProxy.obj
 0001:00097c10       ??1MFXExec@?1??BreakIntoPieces@CBreakableManager@@QAEXAAUGeomRef@@ABU?$Matrix34_tpl@M@@PAUIStatObj@@1ABUBreakageParams@IBreakableManager@@H@Z@QAE@XZ 32098c10 f   BreakableManager.obj
 0001:000a4370       ?AABBDifference@@YAXABUAABB@@0PAU1@PAH@Z 320a5370 f   ProximityTriggerSystem.obj
 0001:000b18dc       _pre_c_init                320b28dc f   MSVCRT:crtdll.obj
 0001:000b1b34       ___DllMainCRTStartup       320b2b34 f   MSVCRT:crtdll.obj
 0001:000b20c0       ??__Eg_random_generator@@YAXXZ 320b30c0 f   CryEntityDLL.obj
 0001:000b20e0       ??__Eg_system_event_listener_entity@@YAXXZ 320b30e0 f   CryEntityDLL.obj
 0001:000b20f0       ??__E?s_factory@CFactory@CEngineModule_EntitySystem@@0V12@A@@YAXXZ 320b30f0 f   CryEntityDLL.obj
 0001:000b2110       ??__EsIdentityMatrix@?A0x9962e041@@YAXXZ 320b3110 f   Entity.obj
 0001:000b2180       ??__E?m_szDescription@CEntity@@0V?$CryStringT@D@@A@@YAXXZ 320b3180 f   Entity.obj
 0001:000b2190       ??__ECryUserInvalidID@@YAXXZ 320b3190 f   EntitySystem.obj
 0001:000b21a0       ??__ECrySessionInvalidID@@YAXXZ 320b31a0 f   EntitySystem.obj
 0001:000b21b0       ??__EautoInitializer@@YAXXZ 320b31b0 f   stdafx.obj
 0001:000b21f0       ??__Eg_meshPreps@@YAXXZ    320b31f0 f   PhysicsEventListener.obj
 0001:000b2260       ??__ECryUserInvalidID@@YAXXZ 320b3260 f   PhysicsProxy.obj
 0001:000b2270       ??__ECrySessionInvalidID@@YAXXZ 320b3270 f   PhysicsProxy.obj
 0001:000b2280       ??__EsIdentMatrix@?A0xadbd02f3@@YAXXZ 320b3280 f   EntityObject.obj
 0001:000b22f0       ??__E?s_tmpWorldPoints@CAreaProxy@@0V?$vector@U?$Vec3_tpl@M@@V?$allocator@U?$Vec3_tpl@M@@@stlpmtx_std@@@stlpmtx_std@@A@@YAXXZ 320b32f0 f   AreaProxy.obj
 0001:000b2320       ??__ECryUserInvalidID@@YAXXZ 320b3320 f   EntityLoadManager.obj
 0001:000b2330       ??__ECrySessionInvalidID@@YAXXZ 320b3330 f   EntityLoadManager.obj
 0001:000b2340       ??__ECryUserInvalidID@@YAXXZ 320b3340 f   BreakableManager.obj
 0001:000b2350       ??__ECrySessionInvalidID@@YAXXZ 320b3350 f   BreakableManager.obj
 0001:000b2360       ??__Eauto_unittest_instance_CUT_PartitionGrid@@YAXXZ 320b3360 f   PartitionGrid.obj
 0001:000b2370       ??__Eautoreg_unittest_CUT_PartitionGrid@@YAXXZ 320b3370 f   PartitionGrid.obj
 0001:000b23d0       ??__ECryUserInvalidID@@YAXXZ 320b33d0 f   EntityPoolManager.obj
 0001:000b23e0       ??__ECrySessionInvalidID@@YAXXZ 320b33e0 f   EntityPoolManager.obj
 0001:000b2400       ??__F?s_factory@CFactory@CEngineModule_EntitySystem@@0V12@A@@YAXXZ 320b3400 f   CryEntityDLL.obj
 0001:000b2420       ??__FInfo@?1???$TypeInfo@M@@YAABUCTypeInfo@@PBM@Z@YAXXZ 320b3420 f   CryEntityDLL.obj
 0001:000b2430       ??__Fg_system_event_listener_entity@@YAXXZ 320b3430 f   CryEntityDLL.obj
 0001:000b2440       ??__FInfo@?1???$TypeInfo@H@@YAABUCTypeInfo@@PBH@Z@YAXXZ 320b3440 f   CryEntityDLL.obj
 0001:000b2450       ??__FInfo@?1???$TypeInfo@I@@YAABUCTypeInfo@@PBI@Z@YAXXZ 320b3450 f   CryEntityDLL.obj
 0001:000b2460       ??__FInfo@?1???$TypeInfo@_K@@YAABUCTypeInfo@@PB_K@Z@YAXXZ 320b3460 f   CryEntityDLL.obj
 0001:000b24b0       ??__F?m_szDescription@CEntity@@0V?$CryStringT@D@@A@@YAXXZ 320b34b0 f   Entity.obj
 0001:000b2510       ??__FCrySessionInvalidID@@YAXXZ 320b3510 f   EntitySystem.obj
 0001:000b2550       ??__FCryUserInvalidID@@YAXXZ 320b3550 f   EntitySystem.obj
 0001:000b2590       ??__FclassEntitiesMap@?1??DebugDrawEntityUsage@CEntitySystem@@AAEXXZ@YAXXZ 320b3590 f   EntitySystem.obj
 0001:000b25f0       ??__FautoInitializer@@YAXXZ 320b35f0 f   stdafx.obj
 0001:000b2600       ??__FInfo@?1???$TypeInfo@W4EGeomType@@@@YAABUCTypeInfo@@PBW4EGeomType@@@Z@YAXXZ 320b3600 f   ScriptBind_Entity.obj
 0001:000b2610       ??__FInfo@?1???$TypeInfo@W4EGeomForm@@@@YAABUCTypeInfo@@PBW4EGeomForm@@@Z@YAXXZ 320b3610 f   ScriptBind_Entity.obj
 0001:000b2630       ??__FInfo@?1??TypeInfo@?$SplineElem@M@@QBEABUCTypeInfo@@XZ@YAXXZ 320b3630 f   ScriptBind_Entity.obj
 0001:000b2660       ??__FInfo@?1??TypeInfo@?$SplineElem@U?$TFixed@E$00$0PP@@@@@QBEABUCTypeInfo@@XZ@YAXXZ 320b3660 f   ScriptBind_Entity.obj
 0001:000b2690       ??__Fareas@?5??IsEntityInsideArea@CScriptBind_Entity@@IAEHPAUIFunctionHandler@@HTScriptHandle@@@Z@YAXXZ 320b3690 f   ScriptBind_Entity.obj
 0001:000b26c0       ??__Fareas@?3??IsPointInsideArea@CScriptBind_Entity@@IAEHPAUIFunctionHandler@@HU?$Vec3_tpl@M@@@Z@YAXXZ 320b36c0 f   ScriptBind_Entity.obj
 0001:000b26f0       ??__Fg_meshPreps@@YAXXZ    320b36f0 f   PhysicsEventListener.obj
 0001:000b2710       ??__FCrySessionInvalidID@@YAXXZ 320b3710 f   PhysicsProxy.obj
 0001:000b2750       ??__FCryUserInvalidID@@YAXXZ 320b3750 f   PhysicsProxy.obj
 0001:000b2790       ??__Fs_colliders@?L@??CheckColliders@CPhysicalProxy@@IAEXXZ@YAXXZ 320b3790 f   PhysicsProxy.obj
 0001:000b27c0       ??__F?s_tmpWorldPoints@CAreaProxy@@0V?$vector@U?$Vec3_tpl@M@@V?$allocator@U?$Vec3_tpl@M@@@stlpmtx_std@@@stlpmtx_std@@A@@YAXXZ 320b37c0 f   AreaProxy.obj
 0001:000b27f0       ??__FCrySessionInvalidID@@YAXXZ 320b37f0 f   EntityLoadManager.obj
 0001:000b2830       ??__FCryUserInvalidID@@YAXXZ 320b3830 f   EntityLoadManager.obj
 0001:000b2870       ??__FCrySessionInvalidID@@YAXXZ 320b3870 f   BreakableManager.obj
 0001:000b28b0       ??__FCryUserInvalidID@@YAXXZ 320b38b0 f   BreakableManager.obj
 0001:000b28f0       ??__Fauto_unittest_instance_CUT_PartitionGrid@@YAXXZ 320b38f0 f   PartitionGrid.obj
 0001:000b2930       ??__FCrySessionInvalidID@@YAXXZ 320b3930 f   EntityPoolManager.obj
 0001:000b2970       ??__FCryUserInvalidID@@YAXXZ 320b3970 f   EntityPoolManager.obj
